 mysqlmanager

 Timestamp is 4bbdf154 (Thu Apr 08 17:08:04 2010)

 Preferred load address is 00400000

 Start         Length     Name                   Class
 0001:00000000 000bcec4H .text                   CODE
 0001:000bced0 00001021H .text$yc                CODE
 0001:000bdef1 00001019H .text$yd                CODE
 0002:00000000 00000104H .CRT$XCA                DATA
 0002:00000104 00000109H .CRT$XCU                DATA
 0002:00000210 00000104H .CRT$XCZ                DATA
 0002:00000314 00000104H .CRT$XIA                DATA
 0002:00000418 00000118H .CRT$XIC                DATA
 0002:00000530 00000104H .CRT$XIY                DATA
 0002:00000634 00000104H .CRT$XIZ                DATA
 0002:00000738 00000004H .CRT$XLA                DATA
 0002:0000073c 00000004H .CRT$XLZ                DATA
 0002:00000740 00000104H .CRT$XPA                DATA
 0002:00000844 00000104H .CRT$XPX                DATA
 0002:00000948 00000104H .CRT$XPXA               DATA
 0002:00000a4c 00000104H .CRT$XPZ                DATA
 0002:00000b50 00000104H .CRT$XTA                DATA
 0002:00000c54 00000104H .CRT$XTZ                DATA
 0002:00000d60 0001bc17H .rdata                  DATA
 0002:0001c978 0000011cH .rdata$T                DATA
 0002:0001ca94 000001abH .rdata$debug            DATA
 0002:0001cc40 00002de3H .rdata$r                DATA
 0002:0001fa30 0000010eH .rdata$sxdata           DATA
 0002:0001fb40 00000104H .rtc$IAA                DATA
 0002:0001fc44 00000104H .rtc$IZZ                DATA
 0002:0001fd48 00000104H .rtc$TAA                DATA
 0002:0001fe4c 00000104H .rtc$TZZ                DATA
 0002:0001ff50 00001078H .xdata$x                DATA
 0002:00020fc8 00000000H .edata                  DATA
 0003:00000000 0014f6c9H .data                   DATA
 0003:0014f6e0 000047a4H .bss                    DATA
 0004:00000000 00000050H .idata$2                DATA
 0004:00000050 00000014H .idata$3                DATA
 0004:00000064 00000404H .idata$4                DATA
 0004:00000468 00000404H .idata$5                DATA
 0004:0000086c 00000dbeH .idata$6                DATA
 0005:00000000 00000101H .tls                    DATA
 0005:00000108 00000186H .tls$                   DATA
 0005:0000028e 00000101H .tls$ZZZ                DATA

  Address         Publics by Value              Rva+Base       Lib:Object

 0000:00000000       __except_list              00000000     <absolute>
 0000:00000003       ___safe_se_handler_count   00000003     <absolute>
 0000:0000002c       __tls_array                0000002c     <absolute>
 0000:00000000       ___ImageBase               00400000     <linker-defined>
 0001:000012a0       ?reserve@Buffer@@QAEHII@Z  004022a0 f   buffer.obj
 0001:000013c0       ?get_size@Buffer@@QAEHXZ   004023c0 f   buffer.obj
 0001:000013d0       ?is_error@Buffer@@QAEHXZ   004023d0 f   buffer.obj
 0001:000013e0       ?append@Buffer@@QAEHIPBDI@Z 004023e0 f   buffer.obj
 0001:00001430       ?get_instance_map@Manager@@SAPAVInstance_map@@XZ 00402430 f i command.obj
 0001:00001440       ?get_guardian@Manager@@SAPAVGuardian@@XZ 00402440 f i command.obj
 0001:00001450       ??0Command@@QAE@XZ         00402450 f   command.obj
 0001:00001480       ??1Command@@UAE@XZ         00402480 f   command.obj
 0001:00001490       ??_ECommand@@UAEPAXI@Z     00402490 f i command.obj
 0001:00001490       ??_GCommand@@UAEPAXI@Z     00402490 f i command.obj
 0001:000014c0       ?alloc_str@Named_value@@SAPADPBUst_mysql_lex_string@@@Z 004024c0 f i commands.obj
 0001:000014e0       ?free_str@Named_value@@SAXPAPAD@Z 004024e0 f i commands.obj
 0001:00001500       ??0Named_value@@QAE@XZ     00402500 f i commands.obj
 0001:00001520       ??0Named_value@@QAE@PAD0@Z 00402520 f i commands.obj
 0001:00001540       ?get_name@Named_value@@QAEPADXZ 00402540 f i commands.obj
 0001:00001550       ?get_value@Named_value@@QAEPADXZ 00402550 f i commands.obj
 0001:00001560       ?free@Named_value@@QAEXXZ  00402560 f i commands.obj
 0001:00001590       ?get_size@Named_value_arr@@QBEHXZ 00402590 f i commands.obj
 0001:000015a0       ?get_element@Named_value_arr@@QBE?AVNamed_value@@H@Z 004025a0 f i commands.obj
 0001:000015e0       ?add_element@Named_value_arr@@QAE_NPAVNamed_value@@@Z 004025e0 f i commands.obj
 0001:00001600       ?get_word@@YAXPAPBDPAIW4enum_seek_method@@@Z 00402600 f i commands.obj
 0001:00001700       ?get_num_options@Instance_options@@QBEHXZ 00402700 f i commands.obj
 0001:00001710       ?get_option@Instance_options@@QBE?AVNamed_value@@H@Z 00402710 f i commands.obj
 0001:00001750       ?get_str@Instance_name@@QBEPBUst_mysql_lex_string@@XZ 00402750 f i commands.obj
 0001:00001760       ?is_mysqld_compatible@Instance@@QBE_NXZ 00402760 f i commands.obj
 0001:00001770       ?is_configured@Instance@@QBE_NXZ 00402770 f i commands.obj
 0001:00001780       ?get_name@Instance@@QBEPBUst_mysql_lex_string@@XZ 00402780 f i commands.obj
 0001:00001790       ?set_state@Instance@@QAEXW4enum_instance_state@1@@Z 00402790 f i commands.obj
 0001:000017a0       ?get_instance_name@Instance_cmd@@IBEPBUst_mysql_lex_string@@XZ 004027a0 f i commands.obj
 0001:000017c0       ??0Buffer@@QAE@I@Z         004027c0 f i commands.obj
 0001:00001800       ??1Buffer@@QAE@XZ          00402800 f i commands.obj
 0001:00001810       ??0Iterator@Instance_map@@QAE@PAV1@@Z 00402810 f i commands.obj
 0001:000018c0       ??0Instance_name@@QAE@PBUst_mysql_lex_string@@@Z 004028c0 f   commands.obj
 0001:00001910       ?write_header@Show_instances@@AAEHPAUst_net@@@Z 00402910 f   commands.obj
 0001:00001990       ?write_data@Show_instances@@AAEHPAUst_net@@@Z 00402990 f   commands.obj
 0001:00001af0       ?execute@Flush_instances@@UAEHPAUst_net@@K@Z 00402af0 f   commands.obj
 0001:00001b30       ??0Instance_cmd@@QAE@PBUst_mysql_lex_string@@@Z 00402b30 f   commands.obj
 0001:00001b60       ??1Instance_cmd@@UAE@XZ    00402b60 f i commands.obj
 0001:00001b70       ??0Abstract_instance_cmd@@QAE@PBUst_mysql_lex_string@@@Z 00402b70 f   commands.obj
 0001:00001b90       ??1Abstract_instance_cmd@@UAE@XZ 00402b90 f i commands.obj
 0001:00001ba0       ?execute@Abstract_instance_cmd@@UAEHPAUst_net@@K@Z 00402ba0 f   commands.obj
 0001:00001c40       ??0Show_instance_status@@QAE@PBUst_mysql_lex_string@@@Z 00402c40 f   commands.obj
 0001:00001c60       ??1Show_instance_status@@UAE@XZ 00402c60 f i commands.obj
 0001:00001c70       ?send_ok_response@Show_instance_status@@MAEHPAUst_net@@K@Z 00402c70 f   commands.obj
 0001:00001cb0       ?write_header@Show_instance_status@@AAEHPAUst_net@@@Z 00402cb0 f   commands.obj
 0001:00001db0       ?write_data@Show_instance_status@@AAEHPAUst_net@@PAVInstance@@@Z 00402db0 f   commands.obj
 0001:00001fb0       ??0Show_instance_options@@QAE@PBUst_mysql_lex_string@@@Z 00402fb0 f   commands.obj
 0001:00001fd0       ??1Show_instance_options@@UAE@XZ 00402fd0 f i commands.obj
 0001:00001fe0       ?send_ok_response@Show_instance_options@@MAEHPAUst_net@@K@Z 00402fe0 f   commands.obj
 0001:00002020       ?write_header@Show_instance_options@@AAEHPAUst_net@@@Z 00403020 f   commands.obj
 0001:000020a0       ?write_data@Show_instance_options@@AAEHPAUst_net@@PAVInstance@@@Z 004030a0 f   commands.obj
 0001:00002280       ??0Start_instance@@QAE@PBUst_mysql_lex_string@@@Z 00403280 f   commands.obj
 0001:000022a0       ??1Start_instance@@UAE@XZ  004032a0 f i commands.obj
 0001:000022b0       ?execute_impl@Start_instance@@MAEHPAUst_net@@PAVInstance@@@Z 004032b0 f   commands.obj
 0001:00002320       ?send_ok_response@Start_instance@@MAEHPAUst_net@@K@Z 00403320 f   commands.obj
 0001:00002350       ??0Stop_instance@@QAE@PBUst_mysql_lex_string@@@Z 00403350 f   commands.obj
 0001:00002370       ??1Stop_instance@@UAE@XZ   00403370 f i commands.obj
 0001:00002380       ?execute_impl@Stop_instance@@MAEHPAUst_net@@PAVInstance@@@Z 00403380 f   commands.obj
 0001:000023d0       ?send_ok_response@Stop_instance@@MAEHPAUst_net@@K@Z 004033d0 f   commands.obj
 0001:00002400       ??0Create_instance@@QAE@PBUst_mysql_lex_string@@@Z 00403400 f   commands.obj
 0001:00002430       ??1Create_instance@@UAE@XZ 00403430 f i commands.obj
 0001:00002450       ?parse_args@Create_instance@@AAE_NPAPBD@Z 00403450 f   commands.obj
 0001:00002680       ?execute@Create_instance@@MAEHPAUst_net@@K@Z 00403680 f   commands.obj
 0001:00002790       ??0Drop_instance@@QAE@PBUst_mysql_lex_string@@@Z 00403790 f   commands.obj
 0001:000027b0       ??1Drop_instance@@UAE@XZ   004037b0 f i commands.obj
 0001:000027c0       ?execute@Drop_instance@@MAEHPAUst_net@@K@Z 004037c0 f   commands.obj
 0001:000028f0       ??0Show_instance_log@@QAE@PBUst_mysql_lex_string@@W4Log_type@@II@Z 004038f0 f   commands.obj
 0001:00002940       ??1Show_instance_log@@UAE@XZ 00403940 f i commands.obj
 0001:00002950       ?send_ok_response@Show_instance_log@@MAEHPAUst_net@@K@Z 00403950 f   commands.obj
 0001:00002990       ?check_params@Show_instance_log@@AAEHPAVInstance@@@Z 00403990 f   commands.obj
 0001:000029f0       ?write_header@Show_instance_log@@AAEHPAUst_net@@@Z 004039f0 f   commands.obj
 0001:00002a50       ?write_data@Show_instance_log@@AAEHPAUst_net@@PAVInstance@@@Z 00403a50 f   commands.obj
 0001:00002c90       ??0Show_instance_log_files@@QAE@PBUst_mysql_lex_string@@@Z 00403c90 f   commands.obj
 0001:00002cb0       ??1Show_instance_log_files@@UAE@XZ 00403cb0 f i commands.obj
 0001:00002cc0       ?send_ok_response@Show_instance_log_files@@MAEHPAUst_net@@K@Z 00403cc0 f   commands.obj
 0001:00002d00       ?write_header@Show_instance_log_files@@AAEHPAUst_net@@@Z 00403d00 f   commands.obj
 0001:00002da0       ?write_data@Show_instance_log_files@@AAEHPAUst_net@@PAVInstance@@@Z 00403da0 f   commands.obj
 0001:00002fb0       ?get_instance_name@Instance_options_list@@QBEPBUst_mysql_lex_string@@XZ 00403fb0 f i commands.obj
 0001:00002fc0       ??0Instance_options_list@@QAE@PBUst_mysql_lex_string@@@Z 00403fc0 f   commands.obj
 0001:00002ff0       ?init@Instance_options_list@@QAE_NXZ 00403ff0 f   commands.obj
 0001:00003020       ??1Instance_options_list@@QAE@XZ 00404020 f i commands.obj
 0001:00003030       ??0Abstract_option_cmd@@IAE@XZ 00404030 f   commands.obj
 0001:00003050       ??1Abstract_option_cmd@@UAE@XZ 00404050 f   commands.obj
 0001:00003080       ?correct_file@Abstract_option_cmd@@IAEHPAVInstance@@PAVNamed_value@@_N@Z 00404080 f   commands.obj
 0001:000030f0       ?execute_impl@Abstract_option_cmd@@AAEHPAUst_net@@K@Z 004040f0 f   commands.obj
 0001:00003280       ?process_option@Set_option@@MAEHPAVInstance@@PAVNamed_value@@@Z 00404280 f   commands.obj
 0001:00003310       ?process_option@Unset_option@@MAEHPAVInstance@@PAVNamed_value@@@Z 00404310 f   commands.obj
 0001:00003350       ?execute@Syntax_error@@UAEHPAUst_net@@K@Z 00404350 f   commands.obj
 0001:00003360       ?execute@Show_instances@@UAEHPAUst_net@@K@Z 00404360 f   commands.obj
 0001:000033c0       ??_EInstance_cmd@@UAEPAXI@Z 004043c0 f i commands.obj
 0001:000033c0       ??_GInstance_cmd@@UAEPAXI@Z 004043c0 f i commands.obj
 0001:000033f0       ??_GAbstract_instance_cmd@@UAEPAXI@Z 004043f0 f i commands.obj
 0001:000033f0       ??_EAbstract_instance_cmd@@UAEPAXI@Z 004043f0 f i commands.obj
 0001:00003420       ??_EShow_instance_status@@UAEPAXI@Z 00404420 f i commands.obj
 0001:00003420       ??_GShow_instance_status@@UAEPAXI@Z 00404420 f i commands.obj
 0001:00003450       ?execute_impl@Show_instance_status@@MAEHPAUst_net@@PAVInstance@@@Z 00404450 f   commands.obj
 0001:00003490       ??_EShow_instance_options@@UAEPAXI@Z 00404490 f i commands.obj
 0001:00003490       ??_GShow_instance_options@@UAEPAXI@Z 00404490 f i commands.obj
 0001:000034c0       ?execute_impl@Show_instance_options@@MAEHPAUst_net@@PAVInstance@@@Z 004044c0 f   commands.obj
 0001:00003500       ??_EStart_instance@@UAEPAXI@Z 00404500 f i commands.obj
 0001:00003500       ??_GStart_instance@@UAEPAXI@Z 00404500 f i commands.obj
 0001:00003530       ??_GStop_instance@@UAEPAXI@Z 00404530 f i commands.obj
 0001:00003530       ??_EStop_instance@@UAEPAXI@Z 00404530 f i commands.obj
 0001:00003560       ??_ECreate_instance@@UAEPAXI@Z 00404560 f i commands.obj
 0001:00003560       ??_GCreate_instance@@UAEPAXI@Z 00404560 f i commands.obj
 0001:000035a0       ?init@Create_instance@@QAE_NPAPBD@Z 004045a0 f   commands.obj
 0001:000035e0       ??_EDrop_instance@@UAEPAXI@Z 004045e0 f i commands.obj
 0001:000035e0       ??_GDrop_instance@@UAEPAXI@Z 004045e0 f i commands.obj
 0001:00003610       ??_GShow_instance_log@@UAEPAXI@Z 00404610 f i commands.obj
 0001:00003610       ??_EShow_instance_log@@UAEPAXI@Z 00404610 f i commands.obj
 0001:00003640       ?execute_impl@Show_instance_log@@MAEHPAUst_net@@PAVInstance@@@Z 00404640 f   commands.obj
 0001:00003690       ??_EShow_instance_log_files@@UAEPAXI@Z 00404690 f i commands.obj
 0001:00003690       ??_GShow_instance_log_files@@UAEPAXI@Z 00404690 f i commands.obj
 0001:000036c0       ?execute_impl@Show_instance_log_files@@MAEHPAUst_net@@PAVInstance@@@Z 004046c0 f   commands.obj
 0001:00003700       ??_GInstance_options_list@@QAEPAXI@Z 00404700 f i commands.obj
 0001:00003730       ??_EAbstract_option_cmd@@UAEPAXI@Z 00404730 f i commands.obj
 0001:00003730       ??_GAbstract_option_cmd@@UAEPAXI@Z 00404730 f i commands.obj
 0001:00003760       ?execute@Abstract_option_cmd@@UAEHPAUst_net@@K@Z 00404760 f   commands.obj
 0001:000037a0       ?get_instance_options_list@Abstract_option_cmd@@AAEPAVInstance_options_list@@PBUst_mysql_lex_string@@@Z 004047a0 f   commands.obj
 0001:00003870       ?add_option@Abstract_option_cmd@@QAE_NPBUst_mysql_lex_string@@PAVNamed_value@@@Z 00404870 f   commands.obj
 0001:000038b0       ?init@Abstract_option_cmd@@QAE_NPAPBD@Z 004048b0 f   commands.obj
 0001:00003910       ?parse_args@Set_option@@MAE_NPAPBD@Z 00404910 f   commands.obj
 0001:00003c00       ?parse_args@Unset_option@@MAE_NPAPBD@Z 00404c00 f   commands.obj
 0001:00003e20       ??0Thread_info@@QAE@XZ     00404e20 f i guardian.obj
 0001:00003e30       ??0Thread@@QAE@XZ          00404e30 f i guardian.obj
 0001:00003e40       ??_EThread@@MAEPAXI@Z      00404e40 f i guardian.obj
 0001:00003e40       ??_GThread@@MAEPAXI@Z      00404e40 f i guardian.obj
 0001:00003e70       ?is_guarded@Instance@@QBE_NXZ 00404e70 f i guardian.obj
 0001:00003e80       ?get_state@Instance@@QBE?AW4enum_instance_state@1@XZ 00404e80 f i guardian.obj
 0001:00003e90       ?is_crashed@Instance@@QAE_NXZ 00404e90 f i guardian.obj
 0001:00003ea0       ??0Guardian@@QAE@PAVThread_registry@@PAVInstance_map@@@Z 00404ea0 f   guardian.obj
 0001:00003ef0       ?process_instance@Guardian@@AAEXPAVInstance@@@Z 00404ef0 f   guardian.obj
 0001:00004230       ?ping@Guardian@@QAEXXZ     00405230 f   guardian.obj
 0001:00004240       ?init@Guardian@@QAEXXZ     00405240 f   guardian.obj
 0001:000042b0       ?stop_instances@Guardian@@AAEXXZ 004052b0 f   guardian.obj
 0001:000043d0       ?lock@Guardian@@QAEXXZ     004053d0 f   guardian.obj
 0001:000043e0       ?unlock@Guardian@@QAEXXZ   004053e0 f   guardian.obj
 0001:000043f0       ??1Guardian@@UAE@XZ        004053f0 f   guardian.obj
 0001:00004430       ?request_shutdown@Guardian@@QAEXXZ 00405430 f   guardian.obj
 0001:00004460       ?run@Guardian@@MAEXXZ      00405460 f   guardian.obj
 0001:00004600       ?is_stopped@Guardian@@QAE_NXZ 00405600 f   guardian.obj
 0001:00004630       ??_GGuardian@@UAEPAXI@Z    00405630 f i guardian.obj
 0001:00004630       ??_EGuardian@@UAEPAXI@Z    00405630 f i guardian.obj
 0001:00004670       ?get_thread_registry@Manager@@SAPAVThread_registry@@XZ 00405670 f i instance.obj
 0001:000048b0       ?SafeTerminateProcess@@YAHPAXI@Z 004058b0 f   instance.obj
 0001:000049f0       ?kill@@YAHHH@Z             004059f0 f   instance.obj
 0001:00004a30       ??0Instance_monitor@@QAE@PAVInstance@@@Z 00405a30 f i instance.obj
 0001:00004a50       ??1Instance_monitor@@UAE@XZ 00405a50 f i instance.obj
 0001:00004a60       ?is_name_valid@Instance@@SA_NPBUst_mysql_lex_string@@@Z 00405a60 f   instance.obj
 0001:00004ac0       ?is_mysqld_compatible_name@Instance@@SA_NPBUst_mysql_lex_string@@@Z 00405ac0 f   instance.obj
 0001:00004af0       ?get_instance_state_name@Instance@@CAPBDW4enum_instance_state@1@@Z 00405af0 f   instance.obj
 0001:00004b70       ??0Instance@@QAE@XZ        00405b70 f   instance.obj
 0001:00004be0       ??1Instance@@QAE@XZ        00405be0 f   instance.obj
 0001:00004c20       ?init@Instance@@QAE_NPBUst_mysql_lex_string@@@Z 00405c20 f   instance.obj
 0001:00004c50       ?complete_initialization@Instance@@QAE_NXZ 00405c50 f   instance.obj
 0001:00004c80       ?is_mysqld_running@Instance@@QAE_NXZ 00405c80 f   instance.obj
 0001:00004d80       ?kill_mysqld@Instance@@QAE_NH@Z 00405d80 f   instance.obj
 0001:00004e40       ?lock@Instance@@QAEXXZ     00405e40 f   instance.obj
 0001:00004e60       ?unlock@Instance@@QAEXXZ   00405e60 f   instance.obj
 0001:00004e80       ?reset_stat@Instance@@QAEXXZ 00405e80 f   instance.obj
 0001:00004eb0       ?remove_pid@Instance@@AAEXXZ 00405eb0 f   instance.obj
 0001:00004ef0       ?wait_for_stop@Instance@@AAE_NXZ 00405ef0 f   instance.obj
 0001:00004fa0       ??_EInstance_monitor@@UAEPAXI@Z 00405fa0 f i instance.obj
 0001:00004fa0       ??_GInstance_monitor@@UAEPAXI@Z 00405fa0 f i instance.obj
 0001:00004fd0       ?start_and_monitor_instance@Instance_monitor@@IAEXXZ 00405fd0 f   instance.obj
 0001:00005140       ?is_active@Instance@@QAE_NXZ 00406140 f   instance.obj
 0001:00005170       ?start_mysqld@Instance@@QAE_NXZ 00406170 f   instance.obj
 0001:00005210       ?stop_mysqld@Instance@@QAE_NXZ 00406210 f   instance.obj
 0001:00005300       ?get_state_name@Instance@@QAEPBDXZ 00406300 f   instance.obj
 0001:00005350       ?run@Instance_monitor@@MAEXXZ 00406350 f   instance.obj
 0001:00005390       ??_GInstance@@QAEPAXI@Z    00406390 f i instance_map.obj
 0001:00005420       ??0Instance_map@@QAE@XZ    00406420 f   instance_map.obj
 0001:00005440       ?lock@Instance_map@@QAEXXZ 00406440 f   instance_map.obj
 0001:00005450       ?unlock@Instance_map@@QAEXXZ 00406450 f   instance_map.obj
 0001:00005460       ?add_instance@Instance_map@@QAEHPAVInstance@@@Z 00406460 f   instance_map.obj
 0001:00005480       ?remove_instance@Instance_map@@QAEHPAVInstance@@@Z 00406480 f   instance_map.obj
 0001:000054a0       ?create_instance@Instance_map@@QAEHPBUst_mysql_lex_string@@PBVNamed_value_arr@@@Z 004064a0 f   instance_map.obj
 0001:00005680       ?find@Instance_map@@QAEPAVInstance@@PBUst_mysql_lex_string@@@Z 00406680 f   instance_map.obj
 0001:000056a0       ?go_to_first@Iterator@Instance_map@@QAEXXZ 004066a0 f   instance_map.obj
 0001:000056b0       ?next@Iterator@Instance_map@@QAEPAVInstance@@XZ 004066b0 f   instance_map.obj
 0001:000056e0       ?create_instance_in_file@@YAHPBUst_mysql_lex_string@@PBVNamed_value_arr@@@Z 004066e0 f   instance_map.obj
 0001:000059e0       ?process_one_option@Instance_map@@QAEHPBUst_mysql_lex_string@@PBD@Z 004069e0 f   instance_map.obj
 0001:00005ba0       ?init@Instance_map@@QAE_NXZ 00406ba0 f   instance_map.obj
 0001:00005be0       ?reset@Instance_map@@QAE_NXZ 00406be0 f   instance_map.obj
 0001:00005c00       ??1Instance_map@@QAE@XZ    00406c00 f   instance_map.obj
 0001:00005ca0       ?is_there_active_instance@Instance_map@@QAE_NXZ 00406ca0 f   instance_map.obj
 0001:00005d10       ?complete_initialization@Instance_map@@AAE_NXZ 00406d10 f   instance_map.obj
 0001:00005e50       ?load@Instance_map@@QAEHXZ 00406e50 f   instance_map.obj
 0001:00005f70       ?strstr@@YAPADPADPBD@Z     00406f70 f i instance_options.obj
 0001:00005f80       ?alloc_str@Named_value@@SAPADPBD@Z 00406f80 f i instance_options.obj
 0001:00005fa0       ?remove_element@Named_value_arr@@QAEXH@Z 00406fa0 f i instance_options.obj
 0001:00006010       ?replace_element@Named_value_arr@@QAE_NHPAVNamed_value@@@Z 00407010 f i instance_options.obj
 0001:00006170       ?is_option_im_specific@Instance_options@@SA_NPBD@Z 00407170 f   instance_options.obj
 0001:000061e0       ??0Instance_options@@QAE@XZ 004071e0 f   instance_options.obj
 0001:00006280       ?get_default_option@Instance_options@@AAEHPADIPBD@Z 00407280 f   instance_options.obj
 0001:00006360       ?fill_instance_version@Instance_options@@AAE_NXZ 00407360 f   instance_options.obj
 0001:00006500       ?fill_mysqld_real_path@Instance_options@@AAE_NXZ 00407500 f   instance_options.obj
 0001:000066b0       ?fill_log_options@Instance_options@@AAE_NXZ 004076b0 f   instance_options.obj
 0001:00006aa0       ?get_pid_filename@Instance_options@@QAEHPAD@Z 00407aa0 f   instance_options.obj
 0001:00006b60       ?unlink_pidfile@Instance_options@@QAEHXZ 00407b60 f   instance_options.obj
 0001:00006b70       ?load_pid@Instance_options@@QAEHXZ 00407b70 f   instance_options.obj
 0001:00006be0       ?update_var@Instance_options@@AAEXPBD0@Z 00407be0 f   instance_options.obj
 0001:00006d40       ?find_option@Instance_options@@AAEHPBD@Z 00407d40 f   instance_options.obj
 0001:00006e00       ?add_to_argv@Instance_options@@AAEHPBD@Z 00407e00 f   instance_options.obj
 0001:00006e30       ?print_argv@Instance_options@@QAEXXZ 00407e30 f   instance_options.obj
 0001:00006e90       ?init@Instance_options@@QAE_NPBUst_mysql_lex_string@@@Z 00407e90 f   instance_options.obj
 0001:00006f10       ??1Instance_options@@QAE@XZ 00407f10 f   instance_options.obj
 0001:00006f40       ?get_shutdown_delay@Instance_options@@QBEIXZ 00407f40 f   instance_options.obj
 0001:00006f60       ?get_mysqld_port@Instance_options@@QBEHXZ 00407f60 f   instance_options.obj
 0001:00006f80       ?set_option@Instance_options@@QAE_NPAVNamed_value@@@Z 00407f80 f   instance_options.obj
 0001:00007090       ?unset_option@Instance_options@@QAEXPBD@Z 00408090 f   instance_options.obj
 0001:000070d0       ?complete_initialization@Instance_options@@QAE_NXZ 004080d0 f   instance_options.obj
 0001:000074a0       ?is_shutdown@Thread_registry@@QAE_NXZ 004084a0 f i listener.obj
 0001:00007510       ??0Listener@@QAE@PAVThread_registry@@PAVUser_map@@@Z 00408510 f   listener.obj
 0001:00007540       ??1Listener@@UAE@XZ        00408540 f i listener.obj
 0001:00007550       ?create_tcp_socket@Listener@@AAEHXZ 00408550 f   listener.obj
 0001:00007740       ?handle_new_mysql_connection@Listener@@AAEXPAUst_vio@@@Z 00408740 f   listener.obj
 0001:000077d0       ??_EListener@@UAEPAXI@Z    004087d0 f i listener.obj
 0001:000077d0       ??_GListener@@UAEPAXI@Z    004087d0 f i listener.obj
 0001:00007800       ?run@Listener@@MAEXXZ      00408800 f   listener.obj
 0001:00007cb0       ?log_init@@YAXXZ           00408cb0 f   log.obj
 0001:00007cd0       ?log_error@@YAXPBDZZ       00408cd0 f   log.obj
 0001:00007d40       ?log_info@@YAXPBDZZ        00408d40 f   log.obj
 0001:00007d70       ?die@@YAXPBDZZ             00408d70 f   log.obj
 0001:00007de0       ?onsignal@@YAXH@Z          00408de0 f   manager.obj
 0001:00007df0       ?set_signals@@YAXPAH@Z     00408df0 f   manager.obj
 0001:00007e20       ?my_sigwait@@YAHPBHPAH@Z   00408e20 f   manager.obj
 0001:00007e50       ??0ThreadModelChecker@?A0x2a2a756e@@QAE@XZ 00408e50 f i manager.obj
 0001:00007e70       ?is_linux_threads@ThreadModelChecker@?A0x2a2a756e@@QBE_NXZ 00408e70 f i manager.obj
 0001:00007e80       ?run@ThreadModelChecker@?A0x2a2a756e@@MAEXXZ 00408e80 f i manager.obj
 0001:00007ea0       ??1ThreadModelChecker@?A0x2a2a756e@@UAE@XZ 00408ea0 f i manager.obj
 0001:00007eb0       ?check_if_linux_threads@?A0x2a2a756e@@YA_NPA_N@Z 00408eb0 f   manager.obj
 0001:00007f20       ?stop_all_threads@Manager@@CAXXZ 00408f20 f   manager.obj
 0001:00007f50       ?init_user_map@Manager@@CA_NPAVUser_map@@@Z 00408f50 f   manager.obj
 0001:00007fe0       ?flush_instances@Manager@@SAHXZ 00408fe0 f   manager.obj
 0001:00008080       ??_GThreadModelChecker@?A0x2a2a756e@@UAEPAXI@Z 00409080 f i manager.obj
 0001:00008080       ??_EThreadModelChecker@?A0x2a2a756e@@UAEPAXI@Z 00409080 f i manager.obj
 0001:000080b0       ?main@Manager@@SAHXZ       004090b0 f   manager.obj
 0001:00008580       ?message@@YAPBDI@Z         00409580 f   messages.obj
 0001:00008590       ?errno_to_sqlstate@@YAPBDI@Z 00409590 f   messages.obj
 0001:000085b0       ??0Mysql_connection@@QAE@PAVThread_registry@@PAVUser_map@@PAUst_vio@@K@Z 004095b0 f   mysql_connection.obj
 0001:000085e0       _my_net_local_init         004095e0 f   mysql_connection.obj
 0001:00008630       _slave_io_thread_detach_vio 00409630 f   mysql_connection.obj
 0001:00008640       ?init@Mysql_connection@@AAE_NXZ 00409640 f   mysql_connection.obj
 0001:000086f0       ?cleanup@Mysql_connection@@AAEXXZ 004096f0 f   mysql_connection.obj
 0001:00008720       ??1Mysql_connection@@UAE@XZ 00409720 f   mysql_connection.obj
 0001:00008750       ?check_connection@Mysql_connection@@AAEHXZ 00409750 f   mysql_connection.obj
 0001:000089e0       ?dispatch_command@Mysql_connection@@AAEHW4enum_server_command@@PBD@Z 004099e0 f   mysql_connection.obj
 0001:00008b70       ??_GMysql_connection@@UAEPAXI@Z 00409b70 f i mysql_connection.obj
 0001:00008b70       ??_EMysql_connection@@UAEPAXI@Z 00409b70 f i mysql_connection.obj
 0001:00008ba0       ?do_command@Mysql_connection@@AAEHXZ 00409ba0 f   mysql_connection.obj
 0001:00008c90       ?main@Mysql_connection@@AAEXXZ 00409c90 f   mysql_connection.obj
 0001:00008d50       ?run@Mysql_connection@@MAEXXZ 00409d50 f   mysql_connection.obj
 0001:00008df0       _main                      00409df0 f   mysqlmanager.obj
 0001:00008e80       ?strchr@@YAPADPADH@Z       00409e80 f i options.obj
 0001:00008e90       ?strrchr@@YAPADPADH@Z      00409e90 f i options.obj
 0001:00008ea0       ??0User_management_cmd@@QAE@XZ 00409ea0 f i options.obj
 0001:00008eb0       ??1User_management_cmd@@UAE@XZ 00409eb0 f i options.obj
 0001:00008ec0       ??_EUser_management_cmd@@UAEPAXI@Z 00409ec0 f i options.obj
 0001:00008ec0       ??_GUser_management_cmd@@UAEPAXI@Z 00409ec0 f i options.obj
 0001:00008ef0       ??0Print_password_line_cmd@@QAE@XZ 00409ef0 f i options.obj
 0001:00008f00       ??1Print_password_line_cmd@@UAE@XZ 00409f00 f i options.obj
 0001:00008f10       ??0Add_user_cmd@@QAE@XZ    00409f10 f i options.obj
 0001:00008f20       ??1Add_user_cmd@@UAE@XZ    00409f20 f i options.obj
 0001:00008f30       ??0Drop_user_cmd@@QAE@XZ   00409f30 f i options.obj
 0001:00008f40       ??1Drop_user_cmd@@UAE@XZ   00409f40 f i options.obj
 0001:00008f50       ??0Edit_user_cmd@@QAE@XZ   00409f50 f i options.obj
 0001:00008f60       ??1Edit_user_cmd@@UAE@XZ   00409f60 f i options.obj
 0001:00008f70       ??0Clean_db_cmd@@QAE@XZ    00409f70 f i options.obj
 0001:00008f80       ??1Clean_db_cmd@@UAE@XZ    00409f80 f i options.obj
 0001:00008f90       ??0Check_db_cmd@@QAE@XZ    00409f90 f i options.obj
 0001:00008fa0       ??1Check_db_cmd@@UAE@XZ    00409fa0 f i options.obj
 0001:00008fb0       ??0List_users_cmd@@QAE@XZ  00409fb0 f i options.obj
 0001:00008fc0       ??1List_users_cmd@@UAE@XZ  00409fc0 f i options.obj
 0001:00009350       ?cleanup@Options@@SAXXZ    0040a350 f   options.obj
 0001:00009520       ??_EPrint_password_line_cmd@@UAEPAXI@Z 0040a520 f i options.obj
 0001:00009520       ??_GPrint_password_line_cmd@@UAEPAXI@Z 0040a520 f i options.obj
 0001:00009550       ??_GAdd_user_cmd@@UAEPAXI@Z 0040a550 f i options.obj
 0001:00009550       ??_EAdd_user_cmd@@UAEPAXI@Z 0040a550 f i options.obj
 0001:00009580       ??_GDrop_user_cmd@@UAEPAXI@Z 0040a580 f i options.obj
 0001:00009580       ??_EDrop_user_cmd@@UAEPAXI@Z 0040a580 f i options.obj
 0001:000095b0       ??_EEdit_user_cmd@@UAEPAXI@Z 0040a5b0 f i options.obj
 0001:000095b0       ??_GEdit_user_cmd@@UAEPAXI@Z 0040a5b0 f i options.obj
 0001:000095e0       ??_EClean_db_cmd@@UAEPAXI@Z 0040a5e0 f i options.obj
 0001:000095e0       ??_GClean_db_cmd@@UAEPAXI@Z 0040a5e0 f i options.obj
 0001:00009610       ??_GCheck_db_cmd@@UAEPAXI@Z 0040a610 f i options.obj
 0001:00009610       ??_ECheck_db_cmd@@UAEPAXI@Z 0040a610 f i options.obj
 0001:00009640       ??_EList_users_cmd@@UAEPAXI@Z 0040a640 f i options.obj
 0001:00009640       ??_GList_users_cmd@@UAEPAXI@Z 0040a640 f i options.obj
 0001:00009670       ?load@Options@@SAHHPAPAD@Z 0040a670 f   options.obj
 0001:000097f0       ??0Show_instances@@QAE@XZ  0040a7f0 f i parse.obj
 0001:00009810       ??1Show_instances@@UAE@XZ  0040a810 f i parse.obj
 0001:00009820       ??0Flush_instances@@QAE@XZ 0040a820 f i parse.obj
 0001:00009840       ??1Flush_instances@@UAE@XZ 0040a840 f i parse.obj
 0001:00009850       ??0Set_option@@QAE@XZ      0040a850 f i parse.obj
 0001:00009870       ??1Set_option@@UAE@XZ      0040a870 f i parse.obj
 0001:00009880       ??0Unset_option@@QAE@XZ    0040a880 f i parse.obj
 0001:000098a0       ??1Unset_option@@UAE@XZ    0040a8a0 f i parse.obj
 0001:000098b0       ??0Syntax_error@@QAE@XZ    0040a8b0 f i parse.obj
 0001:000098d0       ??1Syntax_error@@UAE@XZ    0040a8d0 f i parse.obj
 0001:000098e0       ??0Named_value_arr@@QAE@XZ 0040a8e0 f   parse.obj
 0001:000098f0       ?init@Named_value_arr@@QAE_NXZ 0040a8f0 f   parse.obj
 0001:00009920       ??1Named_value_arr@@QAE@XZ 0040a920 f   parse.obj
 0001:000099b0       ?find_token@@YA?AW4Token@@PBDI@Z 0040a9b0 f i parse.obj
 0001:00009a10       ?get_token@@YA?AW4Token@@PAPBDPAI@Z 0040aa10 f   parse.obj
 0001:00009a50       ?shift_token@@YA?AW4Token@@PAPBDPAI@Z 0040aa50 f   parse.obj
 0001:00009a80       ?get_text_id@@YAHPAPBDPAUst_mysql_lex_string@@@Z 0040aa80 f   parse.obj
 0001:00009b00       ?parse_option_value@@YA_NPBDPAIPAPAD@Z 0040ab00 f   parse.obj
 0001:00009ca0       ?skip_spaces@@YAXPAPBD@Z   0040aca0 f   parse.obj
 0001:00009ce0       ?parse_command@@YAPAVCommand@@PBD@Z 0040ace0 f   parse.obj
 0001:0000a430       ??_EShow_instances@@UAEPAXI@Z 0040b430 f i parse.obj
 0001:0000a430       ??_GShow_instances@@UAEPAXI@Z 0040b430 f i parse.obj
 0001:0000a460       ??_EFlush_instances@@UAEPAXI@Z 0040b460 f i parse.obj
 0001:0000a460       ??_GFlush_instances@@UAEPAXI@Z 0040b460 f i parse.obj
 0001:0000a490       ??_GSet_option@@UAEPAXI@Z  0040b490 f i parse.obj
 0001:0000a490       ??_ESet_option@@UAEPAXI@Z  0040b490 f i parse.obj
 0001:0000a4c0       ??_GUnset_option@@UAEPAXI@Z 0040b4c0 f i parse.obj
 0001:0000a4c0       ??_EUnset_option@@UAEPAXI@Z 0040b4c0 f i parse.obj
 0001:0000a4f0       ??_ESyntax_error@@UAEPAXI@Z 0040b4f0 f i parse.obj
 0001:0000a4f0       ??_GSyntax_error@@UAEPAXI@Z 0040b4f0 f i parse.obj
 0001:0000a520       ?trim_space@?A0x60d3fd73@@YAXPAPBDPAI@Z 0040b520 f   parse_output.obj
 0001:0000a5a0       ??0Mysqld_output_parser@?A0x60d3fd73@@QAE@XZ 0040b5a0 f i parse_output.obj
 0001:0000a5b0       ??1Mysqld_output_parser@?A0x60d3fd73@@UAE@XZ 0040b5b0 f i parse_output.obj
 0001:0000a5c0       ??_EMysqld_output_parser@?A0x60d3fd73@@UAEPAXI@Z 0040b5c0 f i parse_output.obj
 0001:0000a5c0       ??_GMysqld_output_parser@?A0x60d3fd73@@UAEPAXI@Z 0040b5c0 f i parse_output.obj
 0001:0000a5f0       ?parse@Mysqld_output_parser@?A0x60d3fd73@@QAE_NPBD0IPADIW4enum_option_type@@@Z 0040b5f0 f   parse_output.obj
 0001:0000a750       ??0Mysqld_output_parser_win@?A0x60d3fd73@@QAE@XZ 0040b750 f i parse_output.obj
 0001:0000a770       ??1Mysqld_output_parser_win@?A0x60d3fd73@@UAE@XZ 0040b770 f i parse_output.obj
 0001:0000a780       ?run_command@Mysqld_output_parser_win@?A0x60d3fd73@@MAE_NPBD@Z 0040b780 f   parse_output.obj
 0001:0000a880       ?read_line@Mysqld_output_parser_win@?A0x60d3fd73@@MAE_NPADI@Z 0040b880 f   parse_output.obj
 0001:0000a930       ?cleanup@Mysqld_output_parser_win@?A0x60d3fd73@@MAE_NXZ 0040b930 f   parse_output.obj
 0001:0000a960       ?parse_output_and_get_value@@YA_NPBD0IPADIW4enum_option_type@@@Z 0040b960 f   parse_output.obj
 0001:0000a9c0       ??_GMysqld_output_parser_win@?A0x60d3fd73@@UAEPAXI@Z 0040b9c0 f i parse_output.obj
 0001:0000a9c0       ??_EMysqld_output_parser_win@?A0x60d3fd73@@UAEPAXI@Z 0040b9c0 f i parse_output.obj
 0001:0000a9f0       ?create_pid_file@@YA_NPBDH@Z 0040b9f0 f   priv.obj
 0001:0000aac0       ?net_send_error@@YAHPAUst_net@@I@Z 0040bac0 f   protocol.obj
 0001:0000abb0       ?net_send_error_323@@YAHPAUst_net@@I@Z 0040bbb0 f   protocol.obj
 0001:0000ac80       ?net_store_length@@YAPADPADI@Z 0040bc80 f   protocol.obj
 0001:0000acb0       ?store_to_protocol_packet@@YAHPAVBuffer@@PBDPAII@Z 0040bcb0 f   protocol.obj
 0001:0000ad30       ?store_to_protocol_packet@@YAHPAVBuffer@@PBDPAI@Z 0040bd30 f   protocol.obj
 0001:0000ad70       ?send_eof@@YAHPAUst_net@@@Z 0040bd70 f   protocol.obj
 0001:0000add0       ?send_fields@@YAHPAUst_net@@PAUst_list@@@Z 0040bdd0 f   protocol.obj
 0001:0000b000       ?net_send_ok@@YAHPAUst_net@@KPBD@Z 0040c000 f   protocol.obj
 0001:0000b140       ?init@Thread_info@@AAEX_N@Z 0040c140 f   thread_registry.obj
 0001:0000b160       ??0Thread_registry@@QAE@XZ 0040c160 f   thread_registry.obj
 0001:0000b1b0       ??1Thread_registry@@QAE@XZ 0040c1b0 f   thread_registry.obj
 0001:0000b210       ?register_thread@Thread_registry@@QAEXPAVThread_info@@_N@Z 0040c210 f   thread_registry.obj
 0001:0000b270       ?unregister_thread@Thread_registry@@QAEXPAVThread_info@@@Z 0040c270 f   thread_registry.obj
 0001:0000b2d0       ?cond_wait@Thread_registry@@QAEHPAVThread_info@@PAUpthread_cond_t@@PAU_RTL_CRITICAL_SECTION@@@Z 0040c2d0 f   thread_registry.obj
 0001:0000b350       ?cond_timedwait@Thread_registry@@QAEHPAVThread_info@@PAUpthread_cond_t@@PAU_RTL_CRITICAL_SECTION@@PAUtimespec@@@Z 0040c350 f   thread_registry.obj
 0001:0000b3e0       ?request_shutdown@Thread_registry@@QAEXXZ 0040c3e0 f   thread_registry.obj
 0001:0000b400       ?interrupt_threads@Thread_registry@@AAEXXZ 0040c400 f   thread_registry.obj
 0001:0000b460       ?wait_for_threads_to_unregister@Thread_registry@@AAEXXZ 0040c460 f   thread_registry.obj
 0001:0000b4f0       ??1Thread@@MAE@XZ          0040c4f0 f   thread_registry.obj
 0001:0000b500       ?thread_func@Thread@@CAPAXPAX@Z 0040c500 f   thread_registry.obj
 0001:0000b520       ?start@Thread@@QAE_NW4enum_thread_type@1@@Z 0040c520 f   thread_registry.obj
 0001:0000b5a0       ?join@Thread@@QAE_NXZ      0040c5a0 f   thread_registry.obj
 0001:0000b5c0       ?get_error_status@Thread_registry@@QAEHXZ 0040c5c0 f   thread_registry.obj
 0001:0000b5f0       ?set_error_status@Thread_registry@@QAEXXZ 0040c5f0 f   thread_registry.obj
 0001:0000b620       ?deliver_shutdown@Thread_registry@@QAEXXZ 0040c620 f   thread_registry.obj
 0001:0000b670       ??0User@@QAE@XZ            0040c670 f i user_map.obj
 0001:0000b680       ?set_password@User@@QAEXPBD@Z 0040c680 f i user_map.obj
 0001:0000b6a0       ??0Iterator@User_map@@QAE@PAV1@@Z 0040c6a0 f i user_map.obj
 0001:0000b6c0       ??0User@@QAE@PBUst_mysql_lex_string@@PBD@Z 0040c6c0 f   user_map.obj
 0001:0000b700       ?init@User@@QAEHPBD@Z      0040c700 f   user_map.obj
 0001:0000b8b0       ?reset@Iterator@User_map@@QAEXXZ 0040c8b0 f   user_map.obj
 0001:0000b8c0       ?next@Iterator@User_map@@QAEPAUUser@@XZ 0040c8c0 f   user_map.obj
 0001:0000b8f0       ?init@User_map@@QAEHXZ     0040c8f0 f   user_map.obj
 0001:0000b940       ??0User_map@@QAE@XZ        0040c940 f   user_map.obj
 0001:0000b950       ??1User_map@@QAE@XZ        0040c950 f   user_map.obj
 0001:0000b970       ?load@User_map@@QAEHPBDPAPBD@Z 0040c970 f   user_map.obj
 0001:0000bcc0       ?save@User_map@@QAEHPBDPAPBD@Z 0040ccc0 f   user_map.obj
 0001:0000be10       ?find_user@User_map@@QAEPAUUser@@PBUst_mysql_lex_string@@@Z 0040ce10 f   user_map.obj
 0001:0000be30       ?find_user@User_map@@QBEPBUUser@@PBUst_mysql_lex_string@@@Z 0040ce30 f   user_map.obj
 0001:0000be40       ?add_user@User_map@@QAE_NPAUUser@@@Z 0040ce40 f   user_map.obj
 0001:0000be60       ?remove_user@User_map@@QAE_NPAUUser@@@Z 0040ce60 f   user_map.obj
 0001:0000be80       ?authenticate@User_map@@QBEHPBUst_mysql_lex_string@@PBD1@Z 0040ce80 f   user_map.obj
 0001:0000bec0       ??0IMService@@AAE@XZ       0040cec0 f   IMService.obj
 0001:0000bef0       ?Shutdown@WindowsService@@MAEXXZ 0040cef0 f i IMService.obj
 0001:0000bf00       ?Pause@WindowsService@@MAEXXZ 0040cf00 f i IMService.obj
 0001:0000bf10       ?Continue@WindowsService@@MAEXXZ 0040cf10 f i IMService.obj
 0001:0000bf20       ??1IMService@@AAE@XZ       0040cf20 f   IMService.obj
 0001:0000bf30       ?Stop@IMService@@MAEXXZ    0040cf30 f   IMService.obj
 0001:0000bf50       ?Run@IMService@@MAEXKPAPAD@Z 0040cf50 f   IMService.obj
 0001:0000bfb0       ?Log@IMService@@MAEXPBD@Z  0040cfb0 f   IMService.obj
 0001:0000bfd0       ?main@IMService@@SAHXZ     0040cfd0 f   IMService.obj
 0001:0000c140       ??0WindowsService@@QAE@PBD0@Z 0040d140 f   WindowsService.obj
 0001:0000c190       ?Stop@WindowsService@@MAEXXZ 0040d190 f i WindowsService.obj
 0001:0000c1a0       ?Log@WindowsService@@MAEXPBD@Z 0040d1a0 f i WindowsService.obj
 0001:0000c1b0       ??1WindowsService@@QAE@XZ  0040d1b0 f   WindowsService.obj
 0001:0000c1c0       ?IsInstalled@WindowsService@@QAEHXZ 0040d1c0 f   WindowsService.obj
 0001:0000c210       ?SetAcceptedControls@WindowsService@@QAEXK@Z 0040d210 f   WindowsService.obj
 0001:0000c220       ?ReportStatus@WindowsService@@IAEHKKK@Z 0040d220 f   WindowsService.obj
 0001:0000c2e0       ?HandleControlCode@WindowsService@@IAEXK@Z 0040d2e0 f   WindowsService.obj
 0001:0000c380       ?ControlHandler@WindowsService@@SGXK@Z 0040d380 f   WindowsService.obj
 0001:0000c390       ?Install@WindowsService@@QAEHPBD0@Z 0040d390 f   WindowsService.obj
 0001:0000c480       ?Remove@WindowsService@@QAEHXZ 0040d480 f   WindowsService.obj
 0001:0000c510       ?RegisterAndRun@WindowsService@@IAEXKPAPAD@Z 0040d510 f   WindowsService.obj
 0001:0000c580       ?ServiceMain@WindowsService@@SGXKPAPAD@Z 0040d580 f   WindowsService.obj
 0001:0000c590       ?Init@WindowsService@@QAEHXZ 0040d590 f   WindowsService.obj
 0001:0000c860       ?execute@Print_password_line_cmd@@UAEHXZ 0040d860 f   user_management_commands.obj
 0001:0000c920       ?execute@Add_user_cmd@@UAEHXZ 0040d920 f   user_management_commands.obj
 0001:0000ca70       ?execute@Drop_user_cmd@@UAEHXZ 0040da70 f   user_management_commands.obj
 0001:0000cb40       ?execute@Edit_user_cmd@@UAEHXZ 0040db40 f   user_management_commands.obj
 0001:0000cc40       ?execute@Clean_db_cmd@@UAEHXZ 0040dc40 f   user_management_commands.obj
 0001:0000ccc0       ?execute@Check_db_cmd@@UAEHXZ 0040dcc0 f   user_management_commands.obj
 0001:0000cd00       ?execute@List_users_cmd@@UAEHXZ 0040dd00 f   user_management_commands.obj
 0001:0000cdb0       _my_net_init               0040ddb0 f   net_serv.obj
 0001:0000ce50       _net_end                   0040de50 f   net_serv.obj
 0001:0000ce70       _net_realloc               0040de70 f   net_serv.obj
 0001:0000cfa0       _net_clear                 0040dfa0 f   net_serv.obj
 0001:0000d020       _net_real_write            0040e020 f   net_serv.obj
 0001:0000d4c0       _my_net_read               0040e4c0 f   net_serv.obj
 0001:0000d710       _my_net_set_read_timeout   0040e710 f   net_serv.obj
 0001:0000d740       _my_net_set_write_timeout  0040e740 f   net_serv.obj
 0001:0000d770       _net_flush                 0040e770 f   net_serv.obj
 0001:0000d8d0       _my_net_write              0040e8d0 f   net_serv.obj
 0001:0000d9d0       _net_write_command         0040e9d0 f   net_serv.obj
 0001:0000dba0       _net_field_length@4        0040eba0 f   pack.obj
 0001:0000dc10       _net_field_length_ll       0040ec10 f   pack.obj
 0001:0000dc80       _net_store_length          0040ec80 f   pack.obj
 0001:0000dd20       _randominit                0040ed20 f   password.obj
 0001:0000dd60       _my_rnd                    0040ed60 f   password.obj
 0001:0000ddb0       _hash_password             0040edb0 f   password.obj
 0001:0000de50       _my_make_scrambled_password_323 0040ee50 f   password.obj
 0001:0000dea0       _make_scrambled_password_323 0040eea0 f   password.obj
 0001:0000dee0       _scramble_323              0040eee0 f   password.obj
 0001:0000e030       _check_scramble_323        0040f030 f   password.obj
 0001:0000e1b0       _get_salt_from_password_323 0040f1b0 f   password.obj
 0001:0000e320       _make_password_from_salt_323 0040f320 f   password.obj
 0001:0000e350       _create_random_string      0040f350 f   password.obj
 0001:0000e3b0       _octet2hex                 0040f3b0 f   password.obj
 0001:0000e4e0       _my_make_scrambled_password 0040f4e0 f   password.obj
 0001:0000e5b0       _make_scrambled_password   0040f5b0 f   password.obj
 0001:0000e5f0       _scramble                  0040f5f0 f   password.obj
 0001:0000e730       _check_scramble            0040f730 f   password.obj
 0001:0000e8f0       _get_salt_from_password    0040f8f0 f   password.obj
 0001:0000e910       _make_password_from_salt   0040f910 f   password.obj
 0001:0000e940       _mysql_errno_to_sqlstate   0040f940 f   sql_state.obj
 0001:0000e9a0       _my_connect                0040f9a0 f   client.obj
 0001:0000e9c0       _set_mysql_error           0040f9c0 f   client.obj
 0001:0000ea30       _net_clear_error           0040fa30 f   client.obj
 0001:0000eab0       _create_named_pipe         0040fab0 f   client.obj
 0001:0000ed00       _free_rows                 0040fd00 f   client.obj
 0001:0000ed30       _free_old_query            0040fd30 f   client.obj
 0001:0000ede0       _mysql_free_result@4       0040fde0 f   client.obj
 0001:0000ef20       _mysql_read_default_options 0040ff20 f   client.obj
 0001:0000f4d0       _unpack_fields             004104d0 f   client.obj
 0001:0000f8b0       _mysql_init@4              004108b0 f   client.obj
 0001:0000f9a0       _mysql_ssl_set@24          004109a0 f   client.obj
 0001:0000fb20       _mysql_get_ssl_cipher@4    00410b20 f   client.obj
 0001:0000fca0       _mysql_init_character_set  00410ca0 f   client.obj
 0001:0000ff40       _mysql_select_db@8         00410f40 f   client.obj
 0001:000101f0       _mysql_detach_stmt_list    004111f0 f   client.obj
 0001:00010200       _mysql_send_query@12       00411200 f   client.obj
 0001:00010240       _mysql_real_query@12       00411240 f   client.obj
 0001:00010290       _mysql_store_result@4      00411290 f   client.obj
 0001:00010560       _mysql_fetch_lengths@4     00411560 f   client.obj
 0001:000105a0       _mysql_options@12          004115a0 f   client.obj
 0001:000108f0       _mysql_num_rows@4          004118f0 f   client.obj
 0001:00010900       _mysql_num_fields@4        00411900 f   client.obj
 0001:00010910       _mysql_errno@4             00411910 f   client.obj
 0001:00010930       _mysql_error@4             00411930 f   client.obj
 0001:00010950       _mysql_get_server_version@4 00411950 f   client.obj
 0001:000109c0       _mysql_set_character_set@8 004119c0 f   client.obj
 0001:00010b10       _end_server                00411b10 f   client.obj
 0001:00010b70       _mysql_close@4             00411b70 f   client.obj
 0001:00010c50       _cli_safe_read             00411c50 f   client.obj
 0001:00010e30       _cli_read_rows             00411e30 f   client.obj
 0001:00011230       _mysql_real_connect@32     00412230 f   client.obj
 0001:00012240       _mysql_reconnect           00413240 f   client.obj
 0001:000126b0       _mysql_fetch_row@4         004136b0 f   client.obj
 0001:000127a0       _cli_advanced_command      004137a0 f   client.obj
 0001:00012980       _get_tty_password          00413980 f   get_password.obj
 0001:00012ab0       _init_client_errs          00413ab0 f   errmsg.obj
 0001:00012ad0       _finish_client_errs        00413ad0 f   errmsg.obj
 0001:00012ae8       _InitializeCriticalSection@4 00413ae8 f   kernel32:KERNEL32.dll
 0001:00012aee       _EnterCriticalSection@4    00413aee f   kernel32:KERNEL32.dll
 0001:00012af4       _LeaveCriticalSection@4    00413af4 f   kernel32:KERNEL32.dll
 0001:00012afa       _DeleteCriticalSection@4   00413afa f   kernel32:KERNEL32.dll
 0001:00012b00       _GetSystemTimeAsFileTime@4 00413b00 f   kernel32:KERNEL32.dll
 0001:00012b06       _CloseHandle@4             00413b06 f   kernel32:KERNEL32.dll
 0001:00012b0c       _GetExitCodeProcess@8      00413b0c f   kernel32:KERNEL32.dll
 0001:00012b12       _WaitForSingleObject@8     00413b12 f   kernel32:KERNEL32.dll
 0001:00012b18       _CreateProcessA@40         00413b18 f   kernel32:KERNEL32.dll
 0001:00012b1e       _SetLastError@4            00413b1e f   kernel32:KERNEL32.dll
 0001:00012b24       _GetLastError@0            00413b24 f   kernel32:KERNEL32.dll
 0001:00012b2a       _CreateRemoteThread@28     00413b2a f   kernel32:KERNEL32.dll
 0001:00012b30       _GetProcAddress@8          00413b30 f   kernel32:KERNEL32.dll
 0001:00012b36       _DuplicateHandle@28        00413b36 f   kernel32:KERNEL32.dll
 0001:00012b3c       _GetCurrentProcess@0       00413b3c f   kernel32:KERNEL32.dll
 0001:00012b42       _GetModuleHandleA@4        00413b42 f   kernel32:KERNEL32.dll
 0001:00012b48       _TerminateProcess@8        00413b48 f   kernel32:KERNEL32.dll
 0001:00012b4e       _OpenProcess@12            00413b4e f   kernel32:KERNEL32.dll
 0001:00012b54       _GetCurrentThreadId@0      00413b54 f   kernel32:KERNEL32.dll
 0001:00012b5a       _Sleep@4                   00413b5a f   kernel32:KERNEL32.dll
 0001:00012b60       _GetFullPathNameA@16       00413b60 f   kernel32:KERNEL32.dll
 0001:00012b66       _GetModuleFileNameA@12     00413b66 f   kernel32:KERNEL32.dll
 0001:00012b6c       _SetHandleInformation@12   00413b6c f   kernel32:KERNEL32.dll
 0001:00012b72       _CreatePipe@16             00413b72 f   kernel32:KERNEL32.dll
 0001:00012b78       _ReadFile@20               00413b78 f   kernel32:KERNEL32.dll
 0001:00012b7e       _SetNamedPipeHandleState@16 00413b7e f   kernel32:KERNEL32.dll
 0001:00012b84       _WaitNamedPipeA@8          00413b84 f   kernel32:KERNEL32.dll
 0001:00012b8a       _CreateFileA@28            00413b8a f   kernel32:KERNEL32.dll
 0001:00012b90       _CloseServiceHandle@4      00413b90 f   advapi32:ADVAPI32.dll
 0001:00012b96       _OpenServiceA@12           00413b96 f   advapi32:ADVAPI32.dll
 0001:00012b9c       _OpenSCManagerA@12         00413b9c f   advapi32:ADVAPI32.dll
 0001:00012ba2       _SetServiceStatus@8        00413ba2 f   advapi32:ADVAPI32.dll
 0001:00012ba8       _CreateServiceA@52         00413ba8 f   advapi32:ADVAPI32.dll
 0001:00012bae       _DeleteService@4           00413bae f   advapi32:ADVAPI32.dll
 0001:00012bb4       _RegisterServiceCtrlHandlerA@8 00413bb4 f   advapi32:ADVAPI32.dll
 0001:00012bba       _StartServiceCtrlDispatcherA@4 00413bba f   advapi32:ADVAPI32.dll
 0001:00012bc0       _my_realloc                00413bc0 f   mysys:my_realloc.obj
 0001:00012c40       _my_malloc                 00413c40 f   mysys:my_malloc.obj
 0001:00012cc0       _my_no_flags_free          00413cc0 f   mysys:my_malloc.obj
 0001:00012ce0       _my_memdup                 00413ce0 f   mysys:my_malloc.obj
 0001:00012d10       _my_strdup                 00413d10 f   mysys:my_malloc.obj
 0001:00012d60       _my_strndup                00413d60 f   mysys:my_malloc.obj
 0001:00012da0       _init_dynamic_array2       00413da0 f   mysys:array.obj
 0001:00012e20       _init_dynamic_array        00413e20 f   mysys:array.obj
 0001:00012e40       _alloc_dynamic             00413e40 f   mysys:array.obj
 0001:00012ed0       _pop_dynamic               00413ed0 f   mysys:array.obj
 0001:00012ef0       _allocate_dynamic          00413ef0 f   mysys:array.obj
 0001:00012f70       _get_dynamic               00413f70 f   mysys:array.obj
 0001:00012fb0       _delete_dynamic            00413fb0 f   mysys:array.obj
 0001:00012ff0       _delete_dynamic_element    00413ff0 f   mysys:array.obj
 0001:00013020       _freeze_size               00414020 f   mysys:array.obj
 0001:00013060       _get_index_dynamic         00414060 f   mysys:array.obj
 0001:00013080       _insert_dynamic            00414080 f   mysys:array.obj
 0001:000130d0       _set_dynamic               004140d0 f   mysys:array.obj
 0001:00013140       _my_charset_same           00414140 f   mysys:charset.obj
 0001:000137a0       _get_charsets_dir          004147a0 f   mysys:charset.obj
 0001:00013860       _add_compiled_collation    00414860 f   mysys:charset.obj
 0001:00013930       _free_charsets             00414930 f   mysys:charset.obj
 0001:00013940       _get_collation_number      00414940 f   mysys:charset.obj
 0001:00013960       _get_charset_number        00414960 f   mysys:charset.obj
 0001:000139d0       _get_charset_name          004149d0 f   mysys:charset.obj
 0001:00013b00       _get_charset               00414b00 f   mysys:charset.obj
 0001:00013be0       _get_charset_by_name       00414be0 f   mysys:charset.obj
 0001:00013c80       _get_charset_by_csname     00414c80 f   mysys:charset.obj
 0001:00013d30       _resolve_charset           00414d30 f   mysys:charset.obj
 0001:00013d60       _resolve_collation         00414d60 f   mysys:charset.obj
 0001:00013d90       _escape_string_for_mysql   00414d90 f   mysys:charset.obj
 0001:00013f40       _fs_character_set          00414f40 f   mysys:charset.obj
 0001:00013fd0       _escape_quotes_for_mysql   00414fd0 f   mysys:charset.obj
 0001:000140b0       _list_add                  004150b0 f   mysys:list.obj
 0001:000140e0       _list_delete               004150e0 f   mysys:list.obj
 0001:00014110       _list_free                 00415110 f   mysys:list.obj
 0001:00014150       _list_cons                 00415150 f   mysys:list.obj
 0001:00014180       _list_reverse              00415180 f   mysys:list.obj
 0001:000141b0       _list_length               004151b0 f   mysys:list.obj
 0001:000141d0       _list_walk                 004151d0 f   mysys:list.obj
 0001:00014240       _modify_defaults_file      00415240 f   mysys:default_modify.obj
 0001:000146b0       _my_read                   004156b0 f   mysys:my_read.obj
 0001:000147e0       _my_seek                   004157e0 f   mysys:my_seek.obj
 0001:00014880       _my_tell                   00415880 f   mysys:my_seek.obj
 0001:000148e0       _my_dirend                 004158e0 f   mysys:my_lib.obj
 0001:00014950       _my_dir                    00415950 f   mysys:my_lib.obj
 0001:00014be0       _my_fstat                  00415be0 f   mysys:my_lib.obj
 0001:00014c00       _my_stat                   00415c00 f   mysys:my_lib.obj
 0001:00014c90       _my_close                  00415c90 f   mysys:my_open.obj
 0001:00014d50       _my_register_filename      00415d50 f   mysys:my_open.obj
 0001:00014e60       _my_sopen                  00415e60 f   mysys:my_open.obj
 0001:00015100       _my_open                   00416100 f   mysys:my_open.obj
 0001:000151b0       __my_hash_init             004161b0 f   mysys:hash.obj
 0001:00015250       _my_hash_free              00416250 f   mysys:hash.obj
 0001:00015280       _my_hash_reset             00416280 f   mysys:hash.obj
 0001:000153f0       _my_hash_delete            004163f0 f   mysys:hash.obj
 0001:00015630       _my_hash_element           00416630 f   mysys:hash.obj
 0001:00015650       _my_hash_replace           00416650 f   mysys:hash.obj
 0001:00015670       _my_hash_first             00416670 f   mysys:hash.obj
 0001:00015720       _my_hash_next              00416720 f   mysys:hash.obj
 0001:00015790       _my_hash_update            00416790 f   mysys:hash.obj
 0001:00015990       _my_hash_search            00416990 f   mysys:hash.obj
 0001:000159b0       _my_hash_insert            004169b0 f   mysys:hash.obj
 0001:00015ca0       _pthread_cond_init         00416ca0 f   mysys:my_wincond.obj
 0001:00015d00       _pthread_cond_destroy      00416d00 f   mysys:my_wincond.obj
 0001:00015d50       _pthread_cond_timedwait    00416d50 f   mysys:my_wincond.obj
 0001:00015e30       _pthread_cond_signal       00416e30 f   mysys:my_wincond.obj
 0001:00015e60       _pthread_cond_broadcast    00416e60 f   mysys:my_wincond.obj
 0001:00015ea0       _pthread_attr_init         00416ea0 f   mysys:my_wincond.obj
 0001:00015ec0       _pthread_attr_setstacksize 00416ec0 f   mysys:my_wincond.obj
 0001:00015ed0       _pthread_attr_setprio      00416ed0 f   mysys:my_wincond.obj
 0001:00015ee0       _pthread_attr_destroy      00416ee0 f   mysys:my_wincond.obj
 0001:00015ef0       _localtime_r               00416ef0 f   mysys:my_wincond.obj
 0001:00015f60       _pthread_cond_wait         00416f60 f   mysys:my_wincond.obj
 0001:00015f80       _my_sleep                  00416f80 f   mysys:my_sleep.obj
 0001:00015fa0       _my_write                  00416fa0 f   mysys:my_write.obj
 0001:000160f0       _my_access                 004170f0 f   mysys:my_access.obj
 0001:00016180       _check_if_legal_tablename  00417180 f   mysys:my_access.obj
 0001:000161d0       _check_if_legal_filename   004171d0 f   mysys:my_access.obj
 0001:00016300       _get_defaults_options      00417300 f   mysys:default.obj
 0001:000163d0       _free_defaults             004173d0 f   mysys:default.obj
 0001:00016e70       _my_print_default_files    00417e70 f   mysys:default.obj
 0001:00016ff0       _print_defaults            00417ff0 f   mysys:default.obj
 0001:00017110       _my_search_option_files    00418110 f   mysys:default.obj
 0001:00017380       _my_load_defaults          00418380 f   mysys:default.obj
 0001:00017660       _load_defaults             00418660 f   mysys:default.obj
 0001:00017690       _init_alloc_root           00418690 f   mysys:my_alloc.obj
 0001:000176f0       _reset_root_defaults       004186f0 f   mysys:my_alloc.obj
 0001:00017790       _alloc_root                00418790 f   mysys:my_alloc.obj
 0001:00017870       _multi_alloc_root          00418870 f   mysys:my_alloc.obj
 0001:00017930       _free_root                 00418930 f   mysys:my_alloc.obj
 0001:000179d0       _set_prealloc_root         004189d0 f   mysys:my_alloc.obj
 0001:00017a20       _strmake_root              00418a20 f   mysys:my_alloc.obj
 0001:00017a60       _memdup_root               00418a60 f   mysys:my_alloc.obj
 0001:00017a90       _strdup_root               00418a90 f   mysys:my_alloc.obj
 0001:00017ac0       _strlength                 00418ac0 f   mysys:mf_format.obj
 0001:00017b10       _fn_format                 00418b10 f   mysys:mf_format.obj
 0001:00017d50       _my_load_path              00418d50 f   mysys:mf_loadpath.obj
 0001:00017e90       _my_fclose                 00418e90 f   mysys:my_fopen.obj
 0001:00017fb0       _my_fopen                  00418fb0 f   mysys:my_fopen.obj
 0001:00018120       _my_fdopen                 00419120 f   mysys:my_fopen.obj
 0001:00018220       _dirname_length            00419220 f   mysys:mf_dirname.obj
 0001:00018270       _convert_dirname           00419270 f   mysys:mf_dirname.obj
 0001:00018320       _dirname_part              00419320 f   mysys:mf_dirname.obj
 0001:00018350       _my_thread_global_end      00419350 f   mysys:my_thr_init.obj
 0001:00018460       _my_thread_end             00419460 f   mysys:my_thr_init.obj
 0001:000184d0       __my_thread_var            004194d0 f   mysys:my_thr_init.obj
 0001:000184f0       _my_thread_dbug_id         004194f0 f   mysys:my_thr_init.obj
 0001:00018500       _my_thread_name            00419500 f   mysys:my_thr_init.obj
 0001:00018520       _my_thread_init            00419520 f   mysys:my_thr_init.obj
 0001:000185a0       _my_thread_global_init     004195a0 f   mysys:my_thr_init.obj
 0001:00018660       _my_delete                 00419660 f   mysys:my_delete.obj
 0001:000186e0       _nt_share_delete           004196e0 f   mysys:my_delete.obj
 0001:00018810       _my_end                    00419810 f   mysys:my_init.obj
 0001:000188e0       _my_parameter_handler      004198e0 f   mysys:my_init.obj
 0001:00018c00       _my_init                   00419c00 f   mysys:my_init.obj
 0001:00018d40       _my_getopt_register_get_addr 00419d40 f   mysys:my_getopt.obj
 0001:00018da0       _getopt_compare_strings    00419da0 f   mysys:my_getopt.obj
 0001:00018ef0       _getopt_ll_limit_value     00419ef0 f   mysys:my_getopt.obj
 0001:00019060       _getopt_ull_limit_value    0041a060 f   mysys:my_getopt.obj
 0001:00019430       _my_print_help             0041a430 f   mysys:my_getopt.obj
 0001:00019660       _my_print_variables        0041a660 f   mysys:my_getopt.obj
 0001:00019a30       _my_cleanup_options        0041aa30 f   mysys:my_getopt.obj
 0001:00019c00       _handle_options            0041ac00 f   mysys:my_getopt.obj
 0001:0001a610       _gmtime_r                  0041b610 f   mysys:my_pthread.obj
 0001:0001a650       _pthread_no_free           0041b650 f   mysys:my_pthread.obj
 0001:0001a660       _pthread_dummy             0041b660 f   mysys:my_pthread.obj
 0001:0001a670       _win_pthread_init          0041b670 f   mysys:my_winthread.obj
 0001:0001a680       _win_pthread_mutex_trylock 0041b680 f   mysys:my_winthread.obj
 0001:0001a6b0       _pthread_exit              0041b6b0 f   mysys:my_winthread.obj
 0001:0001a6c0       _win_pthread_setspecific   0041b6c0 f   mysys:my_winthread.obj
 0001:0001a6e0       _my_pthread_once           0041b6e0 f   mysys:my_winthread.obj
 0001:0001a730       _pthread_start             0041b730 f   mysys:my_winthread.obj
 0001:0001a780       _pthread_create            0041b780 f   mysys:my_winthread.obj
 0001:0001a810       _my_error                  0041b810 f   mysys:my_error.obj
 0001:0001a8c0       _my_printf_error           0041b8c0 f   mysys:my_error.obj
 0001:0001a930       _my_message                0041b930 f   mysys:my_error.obj
 0001:0001a940       _my_error_register         0041b940 f   mysys:my_error.obj
 0001:0001a9c0       _my_error_unregister       0041b9c0 f   mysys:my_error.obj
 0001:0001aa10       _my_error_unregister_all   0041ba10 f   mysys:my_error.obj
 0001:0001aa50       _my_compress_alloc         0041ba50 f   mysys:my_compress.obj
 0001:0001aae0       _my_uncompress             0041bae0 f   mysys:my_compress.obj
 0001:0001ab60       _unpackfrm                 0041bb60 f   mysys:my_compress.obj
 0001:0001abf0       _my_compress               0041bbf0 f   mysys:my_compress.obj
 0001:0001ac50       _packfrm                   0041bc50 f   mysys:my_compress.obj
 0001:0001ace0       _mysql_sha1_reset          0041bce0 f   mysys:sha1.obj
 0001:0001b380       _mysql_sha1_result         0041c380 f   mysys:sha1.obj
 0001:0001b3f0       _mysql_sha1_input          0041c3f0 f   mysys:sha1.obj
 0001:0001b440       _find_type                 0041c440 f   mysys:typelib.obj
 0001:0001b5d0       _get_type                  0041c5d0 f   mysys:typelib.obj
 0001:0001b5f0       _find_typeset              0041c5f0 f   mysys:typelib.obj
 0001:0001b690       _copy_typelib              0041c690 f   mysys:typelib.obj
 0001:0001b760       _find_type_or_exit         0041c760 f   mysys:typelib.obj
 0001:0001b830       _make_type                 0041c830 f   mysys:typelib.obj
 0001:0001b860       _my_multi_malloc           0041c860 f   mysys:mulalloc.obj
 0001:0001b8d0       _my_gethostbyname_r        0041c8d0 f   mysys:my_gethostbyname.obj
 0001:0001b900       _my_gethostbyname_r_free   0041c900 f   mysys:my_gethostbyname.obj
 0001:0001b910       _thr_alarm_kill            0041c910 f   mysys:thr_alarm.obj
 0001:0001b920       _process_alarm             0041c920 f   mysys:thr_alarm.obj
 0001:0001b930       _thr_alarm                 0041c930 f   mysys:thr_alarm.obj
 0001:0001b980       _thr_got_alarm             0041c980 f   mysys:thr_alarm.obj
 0001:0001b9f0       _thr_end_alarm             0041c9f0 f   mysys:thr_alarm.obj
 0001:0001ba20       _end_thr_alarm             0041ca20 f   mysys:thr_alarm.obj
 0001:0001ba30       _init_thr_alarm            0041ca30 f   mysys:thr_alarm.obj
 0001:0001ba40       _thr_alarm_info            0041ca40 f   mysys:thr_alarm.obj
 0001:0001ba50       _resize_thr_alarm          0041ca50 f   mysys:thr_alarm.obj
 0001:0001ba60       _my_once_alloc             0041ca60 f   mysys:my_once.obj
 0001:0001bb20       _my_once_strdup            0041cb20 f   mysys:my_once.obj
 0001:0001bb70       _my_once_memdup            0041cb70 f   mysys:my_once.obj
 0001:0001bba0       _my_once_free              0041cba0 f   mysys:my_once.obj
 0001:0001bbd0       _my_getwd                  0041cbd0 f   mysys:my_getwd.obj
 0001:0001bc70       _test_if_hard_path         0041cc70 f   mysys:my_getwd.obj
 0001:0001bcc0       _has_path                  0041ccc0 f   mysys:my_getwd.obj
 0001:0001bd00       _my_setwd                  0041cd00 f   mysys:my_getwd.obj
 0001:0001bdb0       _init_compiled_charsets    0041cdb0 f   mysys:charset-def.obj
 0001:0001c090       _my_fread                  0041d090 f   mysys:my_fstream.obj
 0001:0001c160       _my_fseek                  0041d160 f   mysys:my_fstream.obj
 0001:0001c190       _my_ftell                  0041d190 f   mysys:my_fstream.obj
 0001:0001c1a0       _my_fwrite                 0041d1a0 f   mysys:my_fstream.obj
 0001:0001c2b0       _my_chsize                 0041d2b0 f   mysys:my_chsize.obj
 0001:0001c440       _my_filename               0041d440 f   mysys:my_div.obj
 0001:0001c470       _my_qsort                  0041d470 f   mysys:mf_qsort.obj
 0001:0001cb00       _init_glob_errs            0041db00 f   mysys:errors.obj
 0001:0001cb10       _wait_for_free_space       0041db10 f   mysys:errors.obj
 0001:0001cb80       _array_append_string_unique 0041db80 f   mysys:mf_arr_appstr.obj
 0001:0001cc00       _cleanup_dirname           0041dc00 f   mysys:mf_pack.obj
 0001:0001d060       _symdirget                 0041e060 f   mysys:mf_pack.obj
 0001:0001d1a0       _system_filename           0041e1a0 f   mysys:mf_pack.obj
 0001:0001d1c0       _intern_filename           0041e1c0 f   mysys:mf_pack.obj
 0001:0001d240       _pack_dirname              0041e240 f   mysys:mf_pack.obj
 0001:0001d5d0       _normalize_dirname         0041e5d0 f   mysys:mf_pack.obj
 0001:0001d670       _unpack_dirname            0041e670 f   mysys:mf_pack.obj
 0001:0001d770       _unpack_filename           0041e770 f   mysys:mf_pack.obj
 0001:0001d830       _fn_ext                    0041e830 f   mysys:mf_fn_ext.obj
 0001:0001d890       _my_readlink               0041e890 f   mysys:my_symlink.obj
 0001:0001d8b0       _my_symlink                0041e8b0 f   mysys:my_symlink.obj
 0001:0001d8c0       _my_is_symlink             0041e8c0 f   mysys:my_symlink.obj
 0001:0001d8e0       _my_realpath               0041e8e0 f   mysys:my_symlink.obj
 0001:0001d900       _my_message_no_curses      0041e900 f   mysys:my_messnc.obj
 0001:0001d9a0       _my_sync                   0041e9a0 f   mysys:my_sync.obj
 0001:0001da30       _my_sync_dir               0041ea30 f   mysys:my_sync.obj
 0001:0001da40       _my_sync_dir_by_file       0041ea40 f   mysys:my_sync.obj
 0001:0001da50       _strnmov                   0041ea50 f   strings:strnmov.obj
 0001:0001da80       _strmake                   0041ea80 f   strings:strmake.obj
 0001:0001dab0       _int2str                   0041eab0 f   strings:int2str.obj
 0001:0001db90       _int10_to_str              0041eb90 f   strings:int2str.obj
 0001:0001dc40       _strxnmov                  0041ec40 f   strings:strxnmov.obj
 0001:0001dc90       _strmov                    0041ec90 f   strings:strmov.obj
 0001:0001dcb0       _strend                    0041ecb0 f   strings:strend.obj
 0001:0001dcd0       _strxmov                   0041ecd0 f   strings:strxmov.obj
 0001:0001dd10       _is_prefix                 0041ed10 f   strings:is_prefix.obj
 0001:0001dd40       _my_strtoll10              0041ed40 f   strings:my_strtoll10.obj
 0001:0001e2a0       _my_hash_sort_latin1_de    0041f2a0 f   strings:ctype-latin1.obj
 0001:0001e340       _my_vsnprintf              0041f340 f   strings:my_vsnprintf.obj
 0001:0001e650       _my_snprintf               0041f650 f   strings:my_vsnprintf.obj
 0001:0001e670       _strcend                   0041f670 f   strings:strcend.obj
 0001:0001e6a0       _my_strnxfrmlen_simple     0041f6a0 f   strings:ctype-simple.obj
 0001:0001e6c0       _my_strnxfrm_simple        0041f6c0 f   strings:ctype-simple.obj
 0001:0001e740       _my_strnncoll_simple       0041f740 f   strings:ctype-simple.obj
 0001:0001e7c0       _my_strnncollsp_simple     0041f7c0 f   strings:ctype-simple.obj
 0001:0001e880       _my_caseup_str_8bit        0041f880 f   strings:ctype-simple.obj
 0001:0001e8c0       _my_casedn_str_8bit        0041f8c0 f   strings:ctype-simple.obj
 0001:0001e900       _my_caseup_8bit            0041f900 f   strings:ctype-simple.obj
 0001:0001e930       _my_casedn_8bit            0041f930 f   strings:ctype-simple.obj
 0001:0001e960       _my_strcasecmp_8bit        0041f960 f   strings:ctype-simple.obj
 0001:0001e9c0       _my_mb_wc_8bit             0041f9c0 f   strings:ctype-simple.obj
 0001:0001ea00       _my_wc_mb_8bit             0041fa00 f   strings:ctype-simple.obj
 0001:0001ea60       _my_snprintf_8bit          0041fa60 f   strings:ctype-simple.obj
 0001:0001ea80       _my_hash_sort_simple       0041fa80 f   strings:ctype-simple.obj
 0001:0001eb00       _my_strntol_8bit           0041fb00 f   strings:ctype-simple.obj
 0001:0001ec60       _my_strntoul_8bit          0041fc60 f   strings:ctype-simple.obj
 0001:0001eda0       _my_strntoll_8bit          0041fda0 f   strings:ctype-simple.obj
 0001:0001ef60       _my_strntoull_8bit         0041ff60 f   strings:ctype-simple.obj
 0001:0001f0f0       _my_strntod_8bit           004200f0 f   strings:ctype-simple.obj
 0001:0001f120       _my_long10_to_str_8bit     00420120 f   strings:ctype-simple.obj
 0001:0001f1f0       _my_longlong10_to_str_8bit 004201f0 f   strings:ctype-simple.obj
 0001:0001f320       _my_wildcmp_8bit           00420320 f   strings:ctype-simple.obj
 0001:0001f4c0       _my_like_range_simple      004204c0 f   strings:ctype-simple.obj
 0001:0001f5e0       _my_scan_8bit              004205e0 f   strings:ctype-simple.obj
 0001:0001f650       _my_fill_8bit              00420650 f   strings:ctype-simple.obj
 0001:0001f670       _my_numchars_8bit          00420670 f   strings:ctype-simple.obj
 0001:0001f680       _my_numcells_8bit          00420680 f   strings:ctype-simple.obj
 0001:0001f690       _my_charpos_8bit           00420690 f   strings:ctype-simple.obj
 0001:0001f6a0       _my_well_formed_len_8bit   004206a0 f   strings:ctype-simple.obj
 0001:0001f6c0       _my_lengthsp_8bit          004206c0 f   strings:ctype-simple.obj
 0001:0001f6e0       _my_instr_simple           004206e0 f   strings:ctype-simple.obj
 0001:0001fba0       _my_strtoll10_8bit         00420ba0 f   strings:ctype-simple.obj
 0001:0001fbc0       _my_mb_ctype_8bit          00420bc0 f   strings:ctype-simple.obj
 0001:0001fc00       _my_strntoull10rnd_8bit    00420c00 f   strings:ctype-simple.obj
 0001:000200a0       _my_propagate_simple       004210a0 f   strings:ctype-simple.obj
 0001:000200b0       _my_propagate_complex      004210b0 f   strings:ctype-simple.obj
 0001:00020180       _my_lengthsp_binary        00421180 f   strings:ctype-bin.obj
 0001:00020330       _my_mbcharlen_8bit         00421330 f   strings:ctype-bin.obj
 0001:00020390       _my_hash_sort_8bit_bin     00421390 f   strings:ctype-bin.obj
 0001:000203f0       _my_hash_sort_bin          004213f0 f   strings:ctype-bin.obj
 0001:00020440       _my_wildcmp_bin            00421440 f   strings:ctype-bin.obj
 0001:00020d40       _my_parse_charset_xml      00421d40 f   strings:ctype.obj
 0001:00020e00       _my_string_repertoire      00421e00 f   strings:ctype.obj
 0001:00020e80       _my_charset_repertoire     00421e80 f   strings:ctype.obj
 0001:00020ea0       _my_charset_is_ascii_based 00421ea0 f   strings:ctype.obj
 0001:00020ee0       _my_charset_is_8bit_pure_ascii 00421ee0 f   strings:ctype.obj
 0001:00022b00       _str2int                   00423b00 f   strings:str2int.obj
 0001:00022cb0       _strtoll                   00423cb0 f   strings:strtoll.obj
 0001:00022ed0       _llstr                     00423ed0 f   strings:llstr.obj
 0001:00022ef0       _ullstr                    00423ef0 f   strings:llstr.obj
 0001:00022f10       _my_strtod                 00423f10 f   strings:strtod.obj
 0001:00023280       _my_atof                   00424280 f   strings:strtod.obj
 0001:000232b0       _longlong2str              004242b0 f   strings:longlong2str.obj
 0001:000233e0       _longlong10_to_str         004243e0 f   strings:longlong2str.obj
 0001:000234f0       _my_wildcmp_unicode        004244f0 f   strings:ctype-utf8.obj
 0001:000267c0       _my_strntol_ucs2           004277c0 f   strings:ctype-ucs2.obj
 0001:000269d0       _my_strntoul_ucs2          004279d0 f   strings:ctype-ucs2.obj
 0001:00026bc0       _my_strntoll_ucs2          00427bc0 f   strings:ctype-ucs2.obj
 0001:00026e50       _my_strntoull_ucs2         00427e50 f   strings:ctype-ucs2.obj
 0001:000270a0       _my_strntod_ucs2           004280a0 f   strings:ctype-ucs2.obj
 0001:00027190       _my_strntoull10rnd_ucs2    00428190 f   strings:ctype-ucs2.obj
 0001:00027280       _my_l10tostr_ucs2          00428280 f   strings:ctype-ucs2.obj
 0001:00027380       _my_ll10tostr_ucs2         00428380 f   strings:ctype-ucs2.obj
 0001:000274c0       _my_strtoll10_ucs2         004284c0 f   strings:ctype-ucs2.obj
 0001:00027b80       _my_like_range_ucs2        00428b80 f   strings:ctype-ucs2.obj
 0001:00027e50       _my_scan_ucs2              00428e50 f   strings:ctype-ucs2.obj
 0001:00028960       _my_strnncoll_gbk_internal 00429960 f   strings:ctype-gbk.obj
 0001:00028a60       _my_strnncoll_gbk          00429a60 f   strings:ctype-gbk.obj
 0001:0002c560       _bchange                   0042d560 f   strings:bchange.obj
 0001:0002c5c0       _bmove_upp                 0042d5c0 f   strings:bmove_upp.obj
 0001:0002cd10       _my_xml_parse              0042dd10 f   strings:xml.obj
 0001:0002d0e0       _my_xml_parser_create      0042e0e0 f   strings:xml.obj
 0001:0002d100       _my_xml_parser_free        0042e100 f   strings:xml.obj
 0001:0002d110       _my_xml_set_value_handler  0042e110 f   strings:xml.obj
 0001:0002d120       _my_xml_set_enter_handler  0042e120 f   strings:xml.obj
 0001:0002d130       _my_xml_set_leave_handler  0042e130 f   strings:xml.obj
 0001:0002d140       _my_xml_set_user_data      0042e140 f   strings:xml.obj
 0001:0002d150       _my_xml_error_string       0042e150 f   strings:xml.obj
 0001:0002d160       _my_xml_error_pos          0042e160 f   strings:xml.obj
 0001:0002d190       _my_xml_error_lineno       0042e190 f   strings:xml.obj
 0001:0002d1c0       _my_caseup_str_mb          0042e1c0 f   strings:ctype-mb.obj
 0001:0002d210       _my_casedn_str_mb          0042e210 f   strings:ctype-mb.obj
 0001:0002d260       _my_caseup_mb              0042e260 f   strings:ctype-mb.obj
 0001:0002d2b0       _my_casedn_mb              0042e2b0 f   strings:ctype-mb.obj
 0001:0002d300       _my_strcasecmp_mb          0042e300 f   strings:ctype-mb.obj
 0001:0002d3a0       _my_wildcmp_mb             0042e3a0 f   strings:ctype-mb.obj
 0001:0002d7f0       _my_numchars_mb            0042e7f0 f   strings:ctype-mb.obj
 0001:0002d830       _my_charpos_mb             0042e830 f   strings:ctype-mb.obj
 0001:0002d890       _my_well_formed_len_mb     0042e890 f   strings:ctype-mb.obj
 0001:0002d900       _my_instr_mb               0042e900 f   strings:ctype-mb.obj
 0001:0002dca0       _my_like_range_mb          0042eca0 f   strings:ctype-mb.obj
 0001:0002e310       _my_numcells_mb            0042f310 f   strings:ctype-mb.obj
 0001:0002e380       _my_mb_ctype_mb            0042f380 f   strings:ctype-mb.obj
 0001:0002e420       _vio_delete                0042f420 f   vio:vio.obj
 0001:0002e450       _vio_end                   0042f450 f   vio:vio.obj
 0001:0002e640       _vio_reset                 0042f640 f   vio:vio.obj
 0001:0002e670       _vio_new                   0042f670 f   vio:vio.obj
 0001:0002e6f0       _vio_new_win32pipe         0042f6f0 f   vio:vio.obj
 0001:0002e740       _vio_new_win32shared_memory 0042f740 f   vio:vio.obj
 0001:0002e7e0       _vio_errno                 0042f7e0 f   vio:viosocket.obj
 0001:0002e7f0       _vio_read                  0042f7f0 f   vio:viosocket.obj
 0001:0002e810       _vio_read_buff             0042f810 f   vio:viosocket.obj
 0001:0002e8b0       _vio_write                 0042f8b0 f   vio:viosocket.obj
 0001:0002e8d0       _vio_blocking              0042f8d0 f   vio:viosocket.obj
 0001:0002e940       _vio_is_blocking           0042f940 f   vio:viosocket.obj
 0001:0002e950       _vio_fastsend              0042f950 f   vio:viosocket.obj
 0001:0002e980       _vio_keepalive             0042f980 f   vio:viosocket.obj
 0001:0002e9c0       _vio_should_retry          0042f9c0 f   vio:viosocket.obj
 0001:0002e9f0       _vio_was_interrupted       0042f9f0 f   vio:viosocket.obj
 0001:0002ea20       _vio_close                 0042fa20 f   vio:viosocket.obj
 0001:0002ea70       _vio_description           0042fa70 f   vio:viosocket.obj
 0001:0002ea80       _vio_type                  0042fa80 f   vio:viosocket.obj
 0001:0002ea90       _vio_fd                    0042fa90 f   vio:viosocket.obj
 0001:0002eaa0       _vio_peer_addr             0042faa0 f   vio:viosocket.obj
 0001:0002eb20       _vio_in_addr               0042fb20 f   vio:viosocket.obj
 0001:0002eb40       _vio_poll_read             0042fb40 f   vio:viosocket.obj
 0001:0002eb50       _vio_timeout               0042fb50 f   vio:viosocket.obj
 0001:0002ebd0       _vio_read_pipe             0042fbd0 f   vio:viosocket.obj
 0001:0002ec20       _vio_write_pipe            0042fc20 f   vio:viosocket.obj
 0001:0002ec70       _vio_close_pipe            0042fc70 f   vio:viosocket.obj
 0001:0002ecb0       _vio_win32_timeout         0042fcb0 f   vio:viosocket.obj
 0001:0002ecf0       _vio_read_shared_memory    0042fcf0 f   vio:viosocket.obj
 0001:0002edd0       _vio_write_shared_memory   0042fdd0 f   vio:viosocket.obj
 0001:0002ee80       _vio_close_shared_memory   0042fe80 f   vio:viosocket.obj
 0001:0002ef60       _vio_ssl_read              0042ff60 f   vio:viossl.obj
 0001:0002ef80       _vio_ssl_write             0042ff80 f   vio:viossl.obj
 0001:0002efa0       _vio_ssl_close             0042ffa0 f   vio:viossl.obj
 0001:0002efe0       _vio_ssl_delete            0042ffe0 f   vio:viossl.obj
 0001:0002f0f0       _sslaccept                 004300f0 f   vio:viossl.obj
 0001:0002f110       _sslconnect                00430110 f   vio:viossl.obj
 0001:0002f130       _vio_ssl_blocking          00430130 f   vio:viossl.obj
 0001:0002f1d0       _sslGetErrString           004301d0 f   vio:viosslfactories.obj
 0001:0002f400       _new_VioSSLConnectorFd     00430400 f   vio:viosslfactories.obj
 0001:0002f460       _new_VioSSLAcceptorFd      00430460 f   vio:viosslfactories.obj
 0001:0002f4c0       _free_vio_ssl_acceptor_fd  004304c0 f   vio:viosslfactories.obj
 0001:0002f4e0       ??2@YAPAXIPAUDummy@@@Z     004304e0 f i yassl:ssl.obj
 0001:0002f4f0       ??1Message@yaSSL@@UAE@XZ   004304f0 f i yassl:ssl.obj
 0001:0002f500       ??_EMessage@yaSSL@@UAEPAXI@Z 00430500 f i yassl:ssl.obj
 0001:0002f500       ??_GMessage@yaSSL@@UAEPAXI@Z 00430500 f i yassl:ssl.obj
 0001:0002f520       ??1Alert@yaSSL@@UAE@XZ     00430520 f i yassl:ssl.obj
 0001:0002f530       ??1HandShakeBase@yaSSL@@UAE@XZ 00430530 f i yassl:ssl.obj
 0001:0002f540       ??_EHandShakeBase@yaSSL@@UAEPAXI@Z 00430540 f i yassl:ssl.obj
 0001:0002f540       ??_GHandShakeBase@yaSSL@@UAEPAXI@Z 00430540 f i yassl:ssl.obj
 0001:0002f560       ??0EncryptedInfo@yaSSL@@QAE@XZ 00430560 f i yassl:ssl.obj
 0001:0002f570       ?min@TaoCrypt@@YAIII@Z     00430570 f i yassl:ssl.obj
 0001:0002f580       ??0Error@TaoCrypt@@QAE@W4ErrorNumber@1@@Z 00430580 f i yassl:ssl.obj
 0001:0002f590       ?assign@BIGNUM@yaSSL@@QAEXPBEI@Z 00430590 f i yassl:ssl.obj
 0001:0002f5a0       ??1Finished@yaSSL@@UAE@XZ  004305a0 f i yassl:ssl.obj
 0001:0002f5b0       ??1HASH@TaoCrypt@@UAE@XZ   004305b0 f i yassl:ssl.obj
 0001:0002f5c0       ??_GHASH@TaoCrypt@@UAEPAXI@Z 004305c0 f i yassl:ssl.obj
 0001:0002f5c0       ??_EHASH@TaoCrypt@@UAEPAXI@Z 004305c0 f i yassl:ssl.obj
 0001:0002f5e0       ??1HASHwithTransform@TaoCrypt@@UAE@XZ 004305e0 f i yassl:ssl.obj
 0001:0002f5f0       ??0MD5@TaoCrypt@@QAE@XZ    004305f0 f i yassl:ssl.obj
 0001:0002f610       ?getByteOrder@MD5@TaoCrypt@@UBE?AW4ByteOrder@2@XZ 00430610 f i yassl:ssl.obj
 0001:0002f620       ?getBlockSize@MD5@TaoCrypt@@UBEIXZ 00430620 f i yassl:ssl.obj
 0001:0002f630       ?getDigestSize@MD5@TaoCrypt@@UBEIXZ 00430630 f i yassl:ssl.obj
 0001:0002f640       ?getPadSize@MD5@TaoCrypt@@UBEIXZ 00430640 f i yassl:ssl.obj
 0001:0002f650       ??1MD5@TaoCrypt@@UAE@XZ    00430650 f i yassl:ssl.obj
 0001:0002f660       ??0MD4@TaoCrypt@@QAE@XZ    00430660 f i yassl:ssl.obj
 0001:0002f680       ?getByteOrder@MD4@TaoCrypt@@UBE?AW4ByteOrder@2@XZ 00430680 f i yassl:ssl.obj
 0001:0002f690       ?getBlockSize@MD4@TaoCrypt@@UBEIXZ 00430690 f i yassl:ssl.obj
 0001:0002f6a0       ?getDigestSize@MD4@TaoCrypt@@UBEIXZ 004306a0 f i yassl:ssl.obj
 0001:0002f6b0       ?getPadSize@MD4@TaoCrypt@@UBEIXZ 004306b0 f i yassl:ssl.obj
 0001:0002f6c0       ??1MD4@TaoCrypt@@UAE@XZ    004306c0 f i yassl:ssl.obj
 0001:0002f6d0       _yaSSLv3_server_method     004306d0 f   yassl:ssl.obj
 0001:0002f710       _yaSSLv3_client_method     00430710 f   yassl:ssl.obj
 0001:0002f750       _yaTLSv1_server_method     00430750 f   yassl:ssl.obj
 0001:0002f790       _yaTLSv1_client_method     00430790 f   yassl:ssl.obj
 0001:0002f7d0       _yaTLSv1_1_server_method   004307d0 f   yassl:ssl.obj
 0001:0002f810       _yaTLSv1_1_client_method   00430810 f   yassl:ssl.obj
 0001:0002f850       _yaSSLv23_server_method    00430850 f   yassl:ssl.obj
 0001:0002f890       _yaSSLv23_client_method    00430890 f   yassl:ssl.obj
 0001:0002f8d0       _yaSSL_CTX_new             004308d0 f   yassl:ssl.obj
 0001:0002f900       _yaSSL_new                 00430900 f   yassl:ssl.obj
 0001:0002f930       _yaSSL_set_fd              00430930 f   yassl:ssl.obj
 0001:0002f950       _yaSSL_get_fd              00430950 f   yassl:ssl.obj
 0001:0002f960       _yaSSL_connect             00430960 f   yassl:ssl.obj
 0001:0002fbb0       _yaSSL_write               00430bb0 f   yassl:ssl.obj
 0001:0002fbc0       ??1Data@yaSSL@@UAE@XZ      00430bc0 f i yassl:ssl.obj
 0001:0002fbd0       _yaSSL_accept              00430bd0 f   yassl:ssl.obj
 0001:0002fe50       _yaSSL_do_handshake        00430e50 f   yassl:ssl.obj
 0001:0002fe80       _yaSSL_clear               00430e80 f   yassl:ssl.obj
 0001:0002fea0       _yaSSL_shutdown            00430ea0 f   yassl:ssl.obj
 0001:0002ff10       _yaSSL_set_quiet_shutdown  00430f10 f   yassl:ssl.obj
 0001:0002ff30       _yaSSL_get_quiet_shutdown  00430f30 f   yassl:ssl.obj
 0001:0002ff40       _yaSSL_CTX_set_session_cache_mode 00430f40 f   yassl:ssl.obj
 0001:0002ff70       _yaSSL_get_session         00430f70 f   yassl:ssl.obj
 0001:0002ffc0       _yaSSL_set_session         00430fc0 f   yassl:ssl.obj
 0001:00030000       _yaSSL_session_reused      00431000 f   yassl:ssl.obj
 0001:00030020       _yaSSL_SESSION_set_timeout 00431020 f   yassl:ssl.obj
 0001:00030040       _yaSSL_get_default_timeout 00431040 f   yassl:ssl.obj
 0001:00030050       _yaSSL_flush_sessions      00431050 f   yassl:ssl.obj
 0001:00030070       _yaSSL_get_cipher          00431070 f   yassl:ssl.obj
 0001:00030090       _yaSSL_get_shared_ciphers  00431090 f   yassl:ssl.obj
 0001:000300b0       _yaSSL_get_cipher_list     004310b0 f   yassl:ssl.obj
 0001:00030100       _yaSSL_CTX_set_cipher_list 00431100 f   yassl:ssl.obj
 0001:00030120       _yaSSL_get_version         00431120 f   yassl:ssl.obj
 0001:00030140       _yaSSLeay_version          00431140 f   yassl:ssl.obj
 0001:00030150       _yaSSL_get_error           00431150 f   yassl:ssl.obj
 0001:00030160       _yaSSL_set_compression     00431160 f   yassl:ssl.obj
 0001:00030170       _yaSSL_get_peer_certificate 00431170 f   yassl:ssl.obj
 0001:00030190       _yaX509_free               00431190 f   yassl:ssl.obj
 0001:000301a0       _yaX509_STORE_CTX_get_current_cert 004311a0 f   yassl:ssl.obj
 0001:000301b0       _yaX509_STORE_CTX_get_error 004311b0 f   yassl:ssl.obj
 0001:000301c0       _yaX509_STORE_CTX_get_error_depth 004311c0 f   yassl:ssl.obj
 0001:000301d0       _yaX509_NAME_oneline       004311d0 f   yassl:ssl.obj
 0001:00030250       _yaX509_get_issuer_name    00431250 f   yassl:ssl.obj
 0001:00030260       _yaX509_get_subject_name   00431260 f   yassl:ssl.obj
 0001:00030270       _yaSSL_load_error_strings  00431270 f   yassl:ssl.obj
 0001:00030280       _yaSSL_set_connect_state   00431280 f   yassl:ssl.obj
 0001:00030290       _yaSSL_set_accept_state    00431290 f   yassl:ssl.obj
 0001:000302b0       _yaSSL_get_verify_result   004312b0 f   yassl:ssl.obj
 0001:000302c0       _yaSSL_CTX_sess_set_cache_size 004312c0 f   yassl:ssl.obj
 0001:000302d0       _yaSSL_CTX_get_session_cache_mode 004312d0 f   yassl:ssl.obj
 0001:000302e0       _yaSSL_CTX_set_tmp_dh      004312e0 f   yassl:ssl.obj
 0001:00030300       _yaSSL_CTX_set_verify      00431300 f   yassl:ssl.obj
 0001:00030340       _yaSSL_CTX_set_default_verify_paths 00431340 f   yassl:ssl.obj
 0001:00030350       _yaSSL_CTX_set_session_id_context 00431350 f   yassl:ssl.obj
 0001:00030360       _yaSSL_CTX_check_private_key 00431360 f   yassl:ssl.obj
 0001:00030370       _yaSSL_CTX_sess_accept     00431370 f   yassl:ssl.obj
 0001:00030380       _yaSSL_CTX_sess_connect    00431380 f   yassl:ssl.obj
 0001:00030390       _yaSSL_CTX_sess_accept_good 00431390 f   yassl:ssl.obj
 0001:000303a0       _yaSSL_CTX_sess_connect_good 004313a0 f   yassl:ssl.obj
 0001:000303b0       _yaSSL_CTX_sess_accept_renegotiate 004313b0 f   yassl:ssl.obj
 0001:000303c0       _yaSSL_CTX_sess_connect_renegotiate 004313c0 f   yassl:ssl.obj
 0001:000303d0       _yaSSL_CTX_sess_hits       004313d0 f   yassl:ssl.obj
 0001:000303e0       _yaSSL_CTX_sess_cb_hits    004313e0 f   yassl:ssl.obj
 0001:000303f0       _yaSSL_CTX_sess_cache_full 004313f0 f   yassl:ssl.obj
 0001:00030400       _yaSSL_CTX_sess_misses     00431400 f   yassl:ssl.obj
 0001:00030410       _yaSSL_CTX_sess_timeouts   00431410 f   yassl:ssl.obj
 0001:00030420       _yaSSL_CTX_sess_number     00431420 f   yassl:ssl.obj
 0001:00030430       _yaSSL_CTX_sess_get_cache_size 00431430 f   yassl:ssl.obj
 0001:00030440       _yaSSL_CTX_get_verify_mode 00431440 f   yassl:ssl.obj
 0001:00030450       _yaSSL_get_verify_mode     00431450 f   yassl:ssl.obj
 0001:00030470       _yaSSL_CTX_get_verify_depth 00431470 f   yassl:ssl.obj
 0001:00030480       _yaSSL_get_verify_depth    00431480 f   yassl:ssl.obj
 0001:000304a0       _yaSSL_CTX_set_options     004314a0 f   yassl:ssl.obj
 0001:000304b0       _yaSSL_CTX_set_info_callback 004314b0 f   yassl:ssl.obj
 0001:000304c0       _yaOpenSSL_add_all_algorithms 004314c0 f   yassl:ssl.obj
 0001:000304d0       _yaSSL_library_init        004314d0 f   yassl:ssl.obj
 0001:000304e0       _yaDH_new                  004314e0 f   yassl:ssl.obj
 0001:00030500       ??0BIGNUM@yaSSL@@QAE@XZ    00431500 f i yassl:ssl.obj
 0001:00030510       _yaERR_get_error_line_data 00431510 f   yassl:ssl.obj
 0001:00030520       _yaERR_print_errors_fp     00431520 f   yassl:ssl.obj
 0001:00030530       _yaERR_error_string        00431530 f   yassl:ssl.obj
 0001:00030560       _yaX509_verify_cert_error_string 00431560 f   yassl:ssl.obj
 0001:00030570       _yaEVP_md5                 00431570 f   yassl:ssl.obj
 0001:00030580       _yaEVP_des_ede3_cbc        00431580 f   yassl:ssl.obj
 0001:00030590       _yaEVP_BytesToKey          00431590 f   yassl:ssl.obj
 0001:00030800       _yaDES_set_key_unchecked   00431800 f   yassl:ssl.obj
 0001:00030820       _yaDES_ede3_cbc_encrypt    00431820 f   yassl:ssl.obj
 0001:00030900       _yaRAND_status             00431900 f   yassl:ssl.obj
 0001:00030910       _yaDES_set_key             00431910 f   yassl:ssl.obj
 0001:00030930       _yaDES_set_odd_parity      00431930 f   yassl:ssl.obj
 0001:00030940       _yaDES_ecb_encrypt         00431940 f   yassl:ssl.obj
 0001:000309b0       _yaSSL_CTX_set_default_passwd_cb_userdata 004319b0 f   yassl:ssl.obj
 0001:000309c0       _yaSSL_get_certificate     004319c0 f   yassl:ssl.obj
 0001:000309d0       _yaSSL_get_privatekey      004319d0 f   yassl:ssl.obj
 0001:000309e0       _yaSSL_SESSION_free        004319e0 f   yassl:ssl.obj
 0001:000309f0       _yaX509_get_pubkey         004319f0 f   yassl:ssl.obj
 0001:00030a00       _yaEVP_PKEY_copy_parameters 00431a00 f   yassl:ssl.obj
 0001:00030a10       _yaEVP_PKEY_free           00431a10 f   yassl:ssl.obj
 0001:00030a20       _yaERR_error_string_n      00431a20 f   yassl:ssl.obj
 0001:00030a40       _yaERR_free_strings        00431a40 f   yassl:ssl.obj
 0001:00030a50       _yaEVP_cleanup             00431a50 f   yassl:ssl.obj
 0001:00030a60       _yaX509_get_notBefore      00431a60 f   yassl:ssl.obj
 0001:00030a70       _yaX509_get_notAfter       00431a70 f   yassl:ssl.obj
 0001:00030a80       _yaSSLv2_client_method     00431a80 f   yassl:ssl.obj
 0001:00030a90       _yaSSL_get1_session        00431a90 f   yassl:ssl.obj
 0001:00030aa0       _yaGENERAL_NAMES_free      00431aa0 f   yassl:ssl.obj
 0001:00030ab0       _yask_GENERAL_NAME_num     00431ab0 f   yassl:ssl.obj
 0001:00030ac0       _yask_GENERAL_NAME_value   00431ac0 f   yassl:ssl.obj
 0001:00030ad0       _yaASN1_STRING_data        00431ad0 f   yassl:ssl.obj
 0001:00030ae0       _yaASN1_STRING_length      00431ae0 f   yassl:ssl.obj
 0001:00030af0       _yaASN1_STRING_type        00431af0 f   yassl:ssl.obj
 0001:00030b00       _yaX509_NAME_get_index_by_NID 00431b00 f   yassl:ssl.obj
 0001:00030b40       _yaX509_NAME_ENTRY_get_data 00431b40 f   yassl:ssl.obj
 0001:00030b50       _yaX509_NAME_get_entry     00431b50 f   yassl:ssl.obj
 0001:00030b60       _yaASN1_STRING_to_UTF8     00431b60 f   yassl:ssl.obj
 0001:00030bb0       _yaX509_get_ext_d2i        00431bb0 f   yassl:ssl.obj
 0001:00030bc0       _yaMD4_Init                00431bc0 f   yassl:ssl.obj
 0001:00030bf0       _yaMD4_Update              00431bf0 f   yassl:ssl.obj
 0001:00030c10       _yaMD4_Final               00431c10 f   yassl:ssl.obj
 0001:00030c30       _yaMD5_Init                00431c30 f   yassl:ssl.obj
 0001:00030c60       _yaMD5_Update              00431c60 f   yassl:ssl.obj
 0001:00030c80       _yaMD5_Final               00431c80 f   yassl:ssl.obj
 0001:00030ca0       _yaRAND_bytes              00431ca0 f   yassl:ssl.obj
 0001:00030cf0       _yaSSL_peek                00431cf0 f   yassl:ssl.obj
 0001:00030d30       _yaSSL_pending             00431d30 f   yassl:ssl.obj
 0001:00030d50       _yaSSL_CTX_set_default_passwd_cb 00431d50 f   yassl:ssl.obj
 0001:00030d60       _yaSSLeay_add_ssl_algorithms 00431d60 f   yassl:ssl.obj
 0001:00030d70       _yaERR_remove_state        00431d70 f   yassl:ssl.obj
 0001:00030d80       _yaERR_GET_REASON          00431d80 f   yassl:ssl.obj
 0001:00030d90       _err_helper                00431d90 f   yassl:ssl.obj
 0001:00030dc0       _yaERR_peek_error          00431dc0 f   yassl:ssl.obj
 0001:00030dd0       _yaERR_get_error           00431dd0 f   yassl:ssl.obj
 0001:00030de0       _yaRAND_screen             00431de0 f   yassl:ssl.obj
 0001:00030df0       _yaRAND_file_name          00431df0 f   yassl:ssl.obj
 0001:00030e00       _yaRAND_write_file         00431e00 f   yassl:ssl.obj
 0001:00030e10       _yaRAND_load_file          00431e10 f   yassl:ssl.obj
 0001:00030e20       _yaRSA_free                00431e20 f   yassl:ssl.obj
 0001:00030e30       _yaRSA_generate_key        00431e30 f   yassl:ssl.obj
 0001:00030e40       _yaX509_LOOKUP_add_dir     00431e40 f   yassl:ssl.obj
 0001:00030e50       _yaX509_LOOKUP_load_file   00431e50 f   yassl:ssl.obj
 0001:00030e60       _yaX509_LOOKUP_hash_dir    00431e60 f   yassl:ssl.obj
 0001:00030e70       _yaX509_LOOKUP_file        00431e70 f   yassl:ssl.obj
 0001:00030e80       _yaX509_STORE_add_lookup   00431e80 f   yassl:ssl.obj
 0001:00030e90       _yaX509_STORE_get_by_subject 00431e90 f   yassl:ssl.obj
 0001:00030ea0       _yaX509_STORE_new          00431ea0 f   yassl:ssl.obj
 0001:00030eb0       _yaSSL_alert_type_string_long 00431eb0 f   yassl:ssl.obj
 0001:00030ec0       _yaSSL_alert_desc_string_long 00431ec0 f   yassl:ssl.obj
 0001:00030ed0       _yaSSL_state_string_long   00431ed0 f   yassl:ssl.obj
 0001:00030ee0       _yaSSL_CTX_set_tmp_rsa_callback 00431ee0 f   yassl:ssl.obj
 0001:00030ef0       _yaSSL_CTX_set_timeout     00431ef0 f   yassl:ssl.obj
 0001:00030f00       _yaSSL_CTX_use_certificate_chain_file 00431f00 f   yassl:ssl.obj
 0001:00030f10       _yaSSL_CTX_use_RSAPrivateKey_file 00431f10 f   yassl:ssl.obj
 0001:00030f20       _yaSSL_set_rfd             00431f20 f   yassl:ssl.obj
 0001:00030f30       _yaSSL_set_wfd             00431f30 f   yassl:ssl.obj
 0001:00030f40       _yaSSL_want_read           00431f40 f   yassl:ssl.obj
 0001:00030f50       _yaSSL_want_write          00431f50 f   yassl:ssl.obj
 0001:00030f60       _yaSSL_set_shutdown        00431f60 f   yassl:ssl.obj
 0001:00030f70       _yaSSL_get_current_cipher  00431f70 f   yassl:ssl.obj
 0001:00030f80       _yaSSL_CIPHER_description  00431f80 f   yassl:ssl.obj
 0001:00030f90       ?size@?$Block@EV?$AllocatorWithCleanup@E@TaoCrypt@@@TaoCrypt@@QBEIXZ 00431f90 f i yassl:ssl.obj
 0001:00030fa0       ?get_buffer@?$Block@EV?$AllocatorWithCleanup@E@TaoCrypt@@@TaoCrypt@@QBEPAEXZ 00431fa0 f i yassl:ssl.obj
 0001:00030fb0       ??0?$auto_ptr@UBulkCipher@yaSSL@@@mySTL@@QAE@PAUBulkCipher@yaSSL@@@Z 00431fb0 f i yassl:ssl.obj
 0001:00030fc0       ??C?$auto_ptr@UBulkCipher@yaSSL@@@mySTL@@QBEPAUBulkCipher@yaSSL@@XZ 00431fc0 f i yassl:ssl.obj
 0001:00030fd0       ??0?$auto_ptr@Vx509@yaSSL@@@mySTL@@QAE@PAVx509@yaSSL@@@Z 00431fd0 f i yassl:ssl.obj
 0001:00030fe0       ??C?$auto_ptr@Vx509@yaSSL@@@mySTL@@QBEPAVx509@yaSSL@@XZ 00431fe0 f i yassl:ssl.obj
 0001:00030ff0       ?release@?$auto_ptr@Vx509@yaSSL@@@mySTL@@QAEPAVx509@yaSSL@@XZ 00431ff0 f i yassl:ssl.obj
 0001:00031000       ??0?$auto_ptr@UBIGNUM@yaSSL@@@mySTL@@QAE@PAUBIGNUM@yaSSL@@@Z 00432000 f i yassl:ssl.obj
 0001:00031010       ?get@?$auto_ptr@UBIGNUM@yaSSL@@@mySTL@@QBEPAUBIGNUM@yaSSL@@XZ 00432010 f i yassl:ssl.obj
 0001:00031020       ?release@?$auto_ptr@UBIGNUM@yaSSL@@@mySTL@@QAEPAUBIGNUM@yaSSL@@XZ 00432020 f i yassl:ssl.obj
 0001:00031030       ?CheckSize@?$AllocatorBase@E@TaoCrypt@@KAXI@Z 00432030 f i yassl:ssl.obj
 0001:00031040       ??$tcArrayDelete@E@TaoCrypt@@YAXPAE@Z 00432040 f i yassl:ssl.obj
 0001:00031050       ??$ysDelete@UDH@yaSSL@@@yaSSL@@YAXPAUDH@0@@Z 00432050 f i yassl:ssl.obj
 0001:00031060       ??$swap@V?$AllocatorWithCleanup@E@TaoCrypt@@@mySTL@@YAXAAV?$AllocatorWithCleanup@E@TaoCrypt@@0@Z 00432060 f i yassl:ssl.obj
 0001:00031070       ??$ysDelete@UBulkCipher@yaSSL@@@yaSSL@@YAXPAUBulkCipher@0@@Z 00432070 f i yassl:ssl.obj
 0001:00031090       ??_Gx509@yaSSL@@QAEPAXI@Z  00432090 f i yassl:ssl.obj
 0001:000310b0       ??_GSSL_CTX@yaSSL@@QAEPAXI@Z 004320b0 f i yassl:ssl.obj
 0001:000310d0       ??1BIGNUM@yaSSL@@QAE@XZ    004320d0 f i yassl:ssl.obj
 0001:000310e0       ??1Security@yaSSL@@QAE@XZ  004320e0 f i yassl:ssl.obj
 0001:00031100       ??1sslHashes@yaSSL@@QAE@XZ 00432100 f i yassl:ssl.obj
 0001:00031120       ??_GMD5@TaoCrypt@@UAEPAXI@Z 00432120 f i yassl:ssl.obj
 0001:00031120       ??_EMD5@TaoCrypt@@UAEPAXI@Z 00432120 f i yassl:ssl.obj
 0001:00031140       ??_GMD4@TaoCrypt@@UAEPAXI@Z 00432140 f i yassl:ssl.obj
 0001:00031140       ??_EMD4@TaoCrypt@@UAEPAXI@Z 00432140 f i yassl:ssl.obj
 0001:00031160       ?size@Source@TaoCrypt@@QBEIXZ 00432160 f i yassl:ssl.obj
 0001:00031170       ?get_buffer@Source@TaoCrypt@@QBEPBEXZ 00432170 f i yassl:ssl.obj
 0001:00031180       _yaSSLv3_method            00432180 f   yassl:ssl.obj
 0001:00031190       _yaSSL_read                00432190 f   yassl:ssl.obj
 0001:000311d0       _yaSSL_get_cipher_name     004321d0 f   yassl:ssl.obj
 0001:000311e0       ?allocate@?$AllocatorWithCleanup@E@TaoCrypt@@QAEPAEIPBX@Z 004321e0 f i yassl:ssl.obj
 0001:00031200       ?deallocate@?$AllocatorWithCleanup@E@TaoCrypt@@QAEXPAXI@Z 00432200 f i yassl:ssl.obj
 0001:00031220       ?Destroy@?$auto_ptr@UBulkCipher@yaSSL@@@mySTL@@AAEXXZ 00432220 f i yassl:ssl.obj
 0001:00031230       ??$ysDelete@Vx509@yaSSL@@@yaSSL@@YAXPAVx509@0@@Z 00432230 f i yassl:ssl.obj
 0001:00031250       ??$ysDelete@VSSL_CTX@yaSSL@@@yaSSL@@YAXPAVSSL_CTX@0@@Z 00432250 f i yassl:ssl.obj
 0001:00031270       ??$StdReallocate@EV?$AllocatorWithCleanup@E@TaoCrypt@@@TaoCrypt@@YAPAEAAV?$AllocatorWithCleanup@E@0@PAEII_N@Z 00432270 f i yassl:ssl.obj
 0001:00031300       ??_GBIGNUM@yaSSL@@QAEPAXI@Z 00432300 f i yassl:ssl.obj
 0001:00031320       ??1SSL@yaSSL@@QAE@XZ       00432320 f i yassl:ssl.obj
 0001:00031380       _yaSSL_CTX_free            00432380 f   yassl:ssl.obj
 0001:00031390       ??0?$Block@EV?$AllocatorWithCleanup@E@TaoCrypt@@@TaoCrypt@@QAE@PBEI@Z 00432390 f i yassl:ssl.obj
 0001:000313c0       ??1?$Block@EV?$AllocatorWithCleanup@E@TaoCrypt@@@TaoCrypt@@QAE@XZ 004323c0 f i yassl:ssl.obj
 0001:000313e0       ??1?$auto_ptr@UBulkCipher@yaSSL@@@mySTL@@QAE@XZ 004323e0 f i yassl:ssl.obj
 0001:000313f0       ?reset@?$auto_ptr@UBulkCipher@yaSSL@@@mySTL@@QAEXPAUBulkCipher@yaSSL@@@Z 004323f0 f i yassl:ssl.obj
 0001:00031410       ?reallocate@?$AllocatorWithCleanup@E@TaoCrypt@@QAEPAEPAEII_N@Z 00432410 f i yassl:ssl.obj
 0001:00031430       ?Destroy@?$auto_ptr@Vx509@yaSSL@@@mySTL@@AAEXXZ 00432430 f i yassl:ssl.obj
 0001:00031440       ?New@?$Block@EV?$AllocatorWithCleanup@E@TaoCrypt@@@TaoCrypt@@QAEXI@Z 00432440 f i yassl:ssl.obj
 0001:00031470       ??$ysDelete@UBIGNUM@yaSSL@@@yaSSL@@YAXPAUBIGNUM@0@@Z 00432470 f i yassl:ssl.obj
 0001:00031490       ??_GSSL@yaSSL@@QAEPAXI@Z   00432490 f i yassl:ssl.obj
 0001:000314b0       ??0Source@TaoCrypt@@QAE@PBEI@Z 004324b0 f i yassl:ssl.obj
 0001:000314f0       ??1Source@TaoCrypt@@QAE@XZ 004324f0 f i yassl:ssl.obj
 0001:00031510       ??1HexDecoder@TaoCrypt@@QAE@XZ 00432510 f i yassl:ssl.obj
 0001:00031530       _yaDH_free                 00432530 f   yassl:ssl.obj
 0001:00031560       ??1?$auto_ptr@Vx509@yaSSL@@@mySTL@@QAE@XZ 00432560 f i yassl:ssl.obj
 0001:00031570       ?CleanNew@?$Block@EV?$AllocatorWithCleanup@E@TaoCrypt@@@TaoCrypt@@QAEXI@Z 00432570 f i yassl:ssl.obj
 0001:000315b0       ?Destroy@?$auto_ptr@UBIGNUM@yaSSL@@@mySTL@@AAEXXZ 004325b0 f i yassl:ssl.obj
 0001:000315c0       ??$ysDelete@VSSL@yaSSL@@@yaSSL@@YAXPAVSSL@0@@Z 004325c0 f i yassl:ssl.obj
 0001:000315e0       _yaSSL_free                004325e0 f   yassl:ssl.obj
 0001:000315f0       ??0?$Block@EV?$AllocatorWithCleanup@E@TaoCrypt@@@TaoCrypt@@QAE@I@Z 004325f0 f i yassl:ssl.obj
 0001:00031640       ??1?$auto_ptr@UBIGNUM@yaSSL@@@mySTL@@QAE@XZ 00432640 f i yassl:ssl.obj
 0001:00031650       ?reset@?$auto_ptr@UBIGNUM@yaSSL@@@mySTL@@QAEXPAUBIGNUM@yaSSL@@@Z 00432650 f i yassl:ssl.obj
 0001:00031670       ??0HexDecoder@TaoCrypt@@QAE@AAVSource@1@@Z 00432670 f i yassl:ssl.obj
 0001:000316c0       ?read_file@yaSSL@@YAHPAVSSL_CTX@1@PBDHW4CertType@1@@Z 004326c0 f   yassl:ssl.obj
 0001:00031b10       _yaSSL_CTX_use_certificate_file 00432b10 f   yassl:ssl.obj
 0001:00031b30       _yaSSL_CTX_use_PrivateKey_file 00432b30 f   yassl:ssl.obj
 0001:00031b50       _yaSSL_CTX_load_verify_locations 00432b50 f   yassl:ssl.obj
 0001:00031c90       _yaBN_bin2bn               00432c90 f   yassl:ssl.obj
 0001:00031d00       ??0Lock@Mutex@yaSSL@@QAE@AAV12@@Z 00432d00 f i yassl:yassl_int.obj
 0001:00031d10       ??0Ciphers@yaSSL@@QAE@XZ   00432d10 f i yassl:yassl_int.obj
 0001:00031d20       ??0DH_Parms@yaSSL@@QAE@XZ  00432d20 f i yassl:yassl_int.obj
 0001:00031d40       ??0Stats@yaSSL@@QAE@XZ     00432d40 f i yassl:yassl_int.obj
 0001:00031d80       ?c32to24@yaSSL@@YAXIAAY02E@Z 00432d80 f   yassl:yassl_int.obj
 0001:00031da0       ?c24to32@yaSSL@@YAXQBEAAI@Z 00432da0 f   yassl:yassl_int.obj
 0001:00031dd0       ?c24to32@yaSSL@@YAIQBE@Z   00432dd0 f   yassl:yassl_int.obj
 0001:00031df0       ?ato16@yaSSL@@YAXPBEAAG@Z  00432df0 f   yassl:yassl_int.obj
 0001:00031e10       ?ato24@yaSSL@@YAXPBEAAY02E@Z 00432e10 f   yassl:yassl_int.obj
 0001:00031e30       ?c16toa@yaSSL@@YAXGPAE@Z   00432e30 f   yassl:yassl_int.obj
 0001:00031e40       ?c24toa@yaSSL@@YAXQBEPAE@Z 00432e40 f   yassl:yassl_int.obj
 0001:00031e60       ?c32toa@yaSSL@@YAXIPAE@Z   00432e60 f   yassl:yassl_int.obj
 0001:00031e90       ??0States@yaSSL@@QAE@XZ    00432e90 f   yassl:yassl_int.obj
 0001:00031ec0       ?getRecord@States@yaSSL@@QBEABW4RecordLayerState@2@XZ 00432ec0 f   yassl:yassl_int.obj
 0001:00031ed0       ?getHandShake@States@yaSSL@@QBEABW4HandShakeState@2@XZ 00432ed0 f   yassl:yassl_int.obj
 0001:00031ee0       ?getClient@States@yaSSL@@QBEABW4ClientState@2@XZ 00432ee0 f   yassl:yassl_int.obj
 0001:00031ef0       ?getServer@States@yaSSL@@QBEABW4ServerState@2@XZ 00432ef0 f   yassl:yassl_int.obj
 0001:00031f00       ?GetConnect@States@yaSSL@@QBEABW4ConnectState@2@XZ 00432f00 f   yassl:yassl_int.obj
 0001:00031f10       ?GetAccept@States@yaSSL@@QBEABW4AcceptState@2@XZ 00432f10 f   yassl:yassl_int.obj
 0001:00031f20       ?getString@States@yaSSL@@QBEPBDXZ 00432f20 f   yassl:yassl_int.obj
 0001:00031f30       ?What@States@yaSSL@@QBE?AW4YasslError@2@XZ 00432f30 f   yassl:yassl_int.obj
 0001:00031f40       ?useRecord@States@yaSSL@@QAEAAW4RecordLayerState@2@XZ 00432f40 f   yassl:yassl_int.obj
 0001:00031f50       ?useHandShake@States@yaSSL@@QAEAAW4HandShakeState@2@XZ 00432f50 f   yassl:yassl_int.obj
 0001:00031f60       ?useClient@States@yaSSL@@QAEAAW4ClientState@2@XZ 00432f60 f   yassl:yassl_int.obj
 0001:00031f70       ?useServer@States@yaSSL@@QAEAAW4ServerState@2@XZ 00432f70 f   yassl:yassl_int.obj
 0001:00031f80       ?UseConnect@States@yaSSL@@QAEAAW4ConnectState@2@XZ 00432f80 f   yassl:yassl_int.obj
 0001:00031f90       ?UseAccept@States@yaSSL@@QAEAAW4AcceptState@2@XZ 00432f90 f   yassl:yassl_int.obj
 0001:00031fa0       ?useString@States@yaSSL@@QAEPADXZ 00432fa0 f   yassl:yassl_int.obj
 0001:00031fb0       ?SetError@States@yaSSL@@QAEXW4YasslError@2@@Z 00432fb0 f   yassl:yassl_int.obj
 0001:00031fc0       ?getMessage@sslFactory@yaSSL@@QBEABV?$Factory@UMessage@yaSSL@@HP6APAU12@XZ@2@XZ 00432fc0 f   yassl:yassl_int.obj
 0001:00031fd0       ?getHandShake@sslFactory@yaSSL@@QBEABV?$Factory@VHandShakeBase@yaSSL@@HP6APAV12@XZ@2@XZ 00432fd0 f   yassl:yassl_int.obj
 0001:00031fe0       ?getServerKey@sslFactory@yaSSL@@QBEABV?$Factory@UServerKeyBase@yaSSL@@HP6APAU12@XZ@2@XZ 00432fe0 f   yassl:yassl_int.obj
 0001:00031ff0       ?getClientKey@sslFactory@yaSSL@@QBEABV?$Factory@UClientKeyBase@yaSSL@@HP6APAU12@XZ@2@XZ 00432ff0 f   yassl:yassl_int.obj
 0001:00032000       ?SetCompression@SSL@yaSSL@@QAEHXZ 00433000 f   yassl:yassl_int.obj
 0001:00032010       ?SetError@SSL@yaSSL@@QAEXW4YasslError@2@@Z 00433010 f   yassl:yassl_int.obj
 0001:00032020       ?SetQuietShutdown@SSL@yaSSL@@QAEX_N@Z 00433020 f   yassl:yassl_int.obj
 0001:00032030       ?useBuffers@SSL@yaSSL@@QAEAAVBuffers@2@XZ 00433030 f   yassl:yassl_int.obj
 0001:000320f0       ?order_error@SSL@yaSSL@@QAEXXZ 004330f0 f   yassl:yassl_int.obj
 0001:00032100       ??0SumData@yassl_int_cpp_local1@yaSSL@@QAE@XZ 00433100 f i yassl:yassl_int.obj
 0001:00032110       ??RSumData@yassl_int_cpp_local1@yaSSL@@QAEXPAVinput_buffer@2@@Z 00433110 f i yassl:yassl_int.obj
 0001:00032130       ??0SumBuffer@yassl_int_cpp_local1@yaSSL@@QAE@XZ 00433130 f i yassl:yassl_int.obj
 0001:00032140       ??RSumBuffer@yassl_int_cpp_local1@yaSSL@@QAEXPAVoutput_buffer@2@@Z 00433140 f i yassl:yassl_int.obj
 0001:00032160       ?Send@SSL@yaSSL@@QAEXPBEI@Z 00433160 f   yassl:yassl_int.obj
 0001:00032190       ?getCrypto@SSL@yaSSL@@QBEABVCrypto@2@XZ 00433190 f   yassl:yassl_int.obj
 0001:000321a0       ?getSecurity@SSL@yaSSL@@QBEABVSecurity@2@XZ 004331a0 f   yassl:yassl_int.obj
 0001:000321b0       ?getStates@SSL@yaSSL@@QBEABVStates@2@XZ 004331b0 f   yassl:yassl_int.obj
 0001:000321c0       ?getHashes@SSL@yaSSL@@QBEABVsslHashes@2@XZ 004331c0 f   yassl:yassl_int.obj
 0001:000321d0       ?getSocket@SSL@yaSSL@@QBEABVSocket@2@XZ 004331d0 f   yassl:yassl_int.obj
 0001:000321e0       ?GetError@SSL@yaSSL@@QBE?AW4YasslError@2@XZ 004331e0 f   yassl:yassl_int.obj
 0001:000321f0       ?GetQuietShutdown@SSL@yaSSL@@QBE_NXZ 004331f0 f   yassl:yassl_int.obj
 0001:00032200       ?useCrypto@SSL@yaSSL@@QAEAAVCrypto@2@XZ 00433200 f   yassl:yassl_int.obj
 0001:00032210       ?useSecurity@SSL@yaSSL@@QAEAAVSecurity@2@XZ 00433210 f   yassl:yassl_int.obj
 0001:00032220       ?useStates@SSL@yaSSL@@QAEAAVStates@2@XZ 00433220 f   yassl:yassl_int.obj
 0001:00032230       ?useHashes@SSL@yaSSL@@QAEAAVsslHashes@2@XZ 00433230 f   yassl:yassl_int.obj
 0001:00032240       ?useSocket@SSL@yaSSL@@QAEAAVSocket@2@XZ 00433240 f   yassl:yassl_int.obj
 0001:00032250       ?useLog@SSL@yaSSL@@QAEAAVLog@2@XZ 00433250 f   yassl:yassl_int.obj
 0001:00032260       ?HasData@SSL@yaSSL@@QBE_NXZ 00433260 f   yassl:yassl_int.obj
 0001:00032270       ??0SSL_SESSION@yaSSL@@QAE@AAVRandomPool@1@@Z 00433270 f   yassl:yassl_int.obj
 0001:000322c0       ?GetID@SSL_SESSION@yaSSL@@QBEPBEXZ 004332c0 f   yassl:yassl_int.obj
 0001:000322d0       ?GetSecret@SSL_SESSION@yaSSL@@QBEPBEXZ 004332d0 f   yassl:yassl_int.obj
 0001:000322e0       ?GetSuite@SSL_SESSION@yaSSL@@QBEPBEXZ 004332e0 f   yassl:yassl_int.obj
 0001:000322f0       ?GetPeerX509@SSL_SESSION@yaSSL@@QBEPAVX509@2@XZ 004332f0 f   yassl:yassl_int.obj
 0001:00032300       ?GetBornOn@SSL_SESSION@yaSSL@@QBEIXZ 00433300 f   yassl:yassl_int.obj
 0001:00032310       ?GetTimeOut@SSL_SESSION@yaSSL@@QBEIXZ 00433310 f   yassl:yassl_int.obj
 0001:00032320       ?SetTimeOut@SSL_SESSION@yaSSL@@QAEXI@Z 00433320 f   yassl:yassl_int.obj
 0001:00032330       ??0sess_match@yassl_int_cpp_local2@yaSSL@@QAE@PBE@Z 00433330 f i yassl:yassl_int.obj
 0001:00032340       ??Rsess_match@yassl_int_cpp_local2@yaSSL@@QAE_NPAVSSL_SESSION@2@@Z 00433340 f i yassl:yassl_int.obj
 0001:000323e0       ?GetSelf@yassl_int_cpp_local2@yaSSL@@YAKXZ 004333e0 f   yassl:yassl_int.obj
 0001:000323f0       ??0thr_match@yassl_int_cpp_local2@yaSSL@@QAE@XZ 004333f0 f i yassl:yassl_int.obj
 0001:00032400       ??Rthr_match@yassl_int_cpp_local2@yaSSL@@QAE_NUThreadError@2@@Z 00433400 f i yassl:yassl_int.obj
 0001:00032410       ??0SSL_METHOD@yaSSL@@QAE@W4ConnectionEnd@1@UProtocolVersion@1@_N@Z 00433410 f   yassl:yassl_int.obj
 0001:00032440       ?getVersion@SSL_METHOD@yaSSL@@QBE?AUProtocolVersion@2@XZ 00433440 f   yassl:yassl_int.obj
 0001:00032450       ?getSide@SSL_METHOD@yaSSL@@QBE?AW4ConnectionEnd@2@XZ 00433450 f   yassl:yassl_int.obj
 0001:00032460       ?setVerifyPeer@SSL_METHOD@yaSSL@@QAEXXZ 00433460 f   yassl:yassl_int.obj
 0001:00032470       ?setVerifyNone@SSL_METHOD@yaSSL@@QAEXXZ 00433470 f   yassl:yassl_int.obj
 0001:00032480       ?setFailNoCert@SSL_METHOD@yaSSL@@QAEXXZ 00433480 f   yassl:yassl_int.obj
 0001:00032490       ?verifyPeer@SSL_METHOD@yaSSL@@QBE_NXZ 00433490 f   yassl:yassl_int.obj
 0001:000324a0       ?verifyNone@SSL_METHOD@yaSSL@@QBE_NXZ 004334a0 f   yassl:yassl_int.obj
 0001:000324b0       ?failNoCert@SSL_METHOD@yaSSL@@QBE_NXZ 004334b0 f   yassl:yassl_int.obj
 0001:000324c0       ?multipleProtocol@SSL_METHOD@yaSSL@@QBE_NXZ 004334c0 f   yassl:yassl_int.obj
 0001:000324d0       ??1DH_Parms@yaSSL@@QAE@XZ  004334d0 f i yassl:yassl_int.obj
 0001:000324f0       ?GetCA_List@SSL_CTX@yaSSL@@QBEABV?$list@PAVx509@yaSSL@@@mySTL@@XZ 004334f0 f   yassl:yassl_int.obj
 0001:00032500       ?getVerifyCallback@SSL_CTX@yaSSL@@QBEP6AHHPAUX509_STORE_CTX@2@@ZXZ 00433500 f   yassl:yassl_int.obj
 0001:00032510       ?getCert@SSL_CTX@yaSSL@@QBEPBVx509@2@XZ 00433510 f   yassl:yassl_int.obj
 0001:00032520       ?getKey@SSL_CTX@yaSSL@@QBEPBVx509@2@XZ 00433520 f   yassl:yassl_int.obj
 0001:00032530       ?getMethod@SSL_CTX@yaSSL@@QBEPBVSSL_METHOD@2@XZ 00433530 f   yassl:yassl_int.obj
 0001:00032540       ?GetCiphers@SSL_CTX@yaSSL@@QBEABUCiphers@2@XZ 00433540 f   yassl:yassl_int.obj
 0001:00032550       ?GetDH_Parms@SSL_CTX@yaSSL@@QBEABUDH_Parms@2@XZ 00433550 f   yassl:yassl_int.obj
 0001:00032560       ?GetStats@SSL_CTX@yaSSL@@QBEABUStats@2@XZ 00433560 f   yassl:yassl_int.obj
 0001:00032570       ?GetPasswordCb@SSL_CTX@yaSSL@@QBEP6AHPADHHPAX@ZXZ 00433570 f   yassl:yassl_int.obj
 0001:00032580       ?SetPasswordCb@SSL_CTX@yaSSL@@QAEXP6AHPADHHPAX@Z@Z 00433580 f   yassl:yassl_int.obj
 0001:00032590       ?GetUserData@SSL_CTX@yaSSL@@QBEPAXXZ 00433590 f   yassl:yassl_int.obj
 0001:000325a0       ?GetSessionCacheOff@SSL_CTX@yaSSL@@QBE_NXZ 004335a0 f   yassl:yassl_int.obj
 0001:000325b0       ?GetSessionCacheFlushOff@SSL_CTX@yaSSL@@QBE_NXZ 004335b0 f   yassl:yassl_int.obj
 0001:000325c0       ?SetUserData@SSL_CTX@yaSSL@@QAEXPAX@Z 004335c0 f   yassl:yassl_int.obj
 0001:000325d0       ?SetSessionCacheOff@SSL_CTX@yaSSL@@QAEXXZ 004335d0 f   yassl:yassl_int.obj
 0001:000325e0       ?SetSessionCacheFlushOff@SSL_CTX@yaSSL@@QAEXXZ 004335e0 f   yassl:yassl_int.obj
 0001:000325f0       ?setVerifyPeer@SSL_CTX@yaSSL@@QAEXXZ 004335f0 f   yassl:yassl_int.obj
 0001:00032600       ?setVerifyNone@SSL_CTX@yaSSL@@QAEXXZ 00433600 f   yassl:yassl_int.obj
 0001:00032610       ?setFailNoCert@SSL_CTX@yaSSL@@QAEXXZ 00433610 f   yassl:yassl_int.obj
 0001:00032620       ?setVerifyCallback@SSL_CTX@yaSSL@@QAEXP6AHHPAUX509_STORE_CTX@2@@Z@Z 00433620 f   yassl:yassl_int.obj
 0001:00032630       ?SetDH@SSL_CTX@yaSSL@@QAE_NABUDH@2@@Z 00433630 f   yassl:yassl_int.obj
 0001:00032670       ?SetCipherList@SSL_CTX@yaSSL@@QAE_NPBD@Z 00433670 f   yassl:yassl_int.obj
 0001:000327b0       ?IncrementStats@SSL_CTX@yaSSL@@QAEXW4StatsField@2@@Z 004337b0 f   yassl:yassl_int.obj
 0001:000328a0       ??0Crypto@yaSSL@@QAE@XZ    004338a0 f   yassl:yassl_int.obj
 0001:000328d0       ?get_digest@Crypto@yaSSL@@QBEABUDigest@2@XZ 004338d0 f   yassl:yassl_int.obj
 0001:000328e0       ?get_cipher@Crypto@yaSSL@@QBEABUBulkCipher@2@XZ 004338e0 f   yassl:yassl_int.obj
 0001:000328f0       ?get_dh@Crypto@yaSSL@@QBEABVDiffieHellman@2@XZ 004338f0 f   yassl:yassl_int.obj
 0001:00032900       ?get_random@Crypto@yaSSL@@QBEABVRandomPool@2@XZ 00433900 f   yassl:yassl_int.obj
 0001:00032910       ?get_certManager@Crypto@yaSSL@@QBEABVCertManager@2@XZ 00433910 f   yassl:yassl_int.obj
 0001:00032920       ?use_digest@Crypto@yaSSL@@QAEAAUDigest@2@XZ 00433920 f   yassl:yassl_int.obj
 0001:00032930       ?use_cipher@Crypto@yaSSL@@QAEAAUBulkCipher@2@XZ 00433930 f   yassl:yassl_int.obj
 0001:00032940       ?use_dh@Crypto@yaSSL@@QAEAAVDiffieHellman@2@XZ 00433940 f   yassl:yassl_int.obj
 0001:00032950       ?use_random@Crypto@yaSSL@@QAEAAVRandomPool@2@XZ 00433950 f   yassl:yassl_int.obj
 0001:00032960       ?use_certManager@Crypto@yaSSL@@QAEAAVCertManager@2@XZ 00433960 f   yassl:yassl_int.obj
 0001:00032970       ?SetDH@Crypto@yaSSL@@QAEXPAVDiffieHellman@2@@Z 00433970 f   yassl:yassl_int.obj
 0001:00032980       ?SetDH@Crypto@yaSSL@@QAEXABUDH_Parms@2@@Z 00433980 f   yassl:yassl_int.obj
 0001:000329c0       ?DhSet@Crypto@yaSSL@@QAE_NXZ 004339c0 f   yassl:yassl_int.obj
 0001:000329d0       ?setDigest@Crypto@yaSSL@@QAEXPAUDigest@2@@Z 004339d0 f   yassl:yassl_int.obj
 0001:000329e0       ?setCipher@Crypto@yaSSL@@QAEXPAUBulkCipher@2@@Z 004339e0 f   yassl:yassl_int.obj
 0001:000329f0       ?get_MD5@sslHashes@yaSSL@@QBEABVMD5@2@XZ 004339f0 f   yassl:yassl_int.obj
 0001:00032a00       ?get_SHA@sslHashes@yaSSL@@QBEABVSHA@2@XZ 00433a00 f   yassl:yassl_int.obj
 0001:00032a10       ?get_verify@sslHashes@yaSSL@@QBEABVFinished@2@XZ 00433a10 f   yassl:yassl_int.obj
 0001:00032a20       ?get_certVerify@sslHashes@yaSSL@@QBEABUHashes@2@XZ 00433a20 f   yassl:yassl_int.obj
 0001:00032a30       ?use_MD5@sslHashes@yaSSL@@QAEAAVMD5@2@XZ 00433a30 f   yassl:yassl_int.obj
 0001:00032a40       ?use_SHA@sslHashes@yaSSL@@QAEAAVSHA@2@XZ 00433a40 f   yassl:yassl_int.obj
 0001:00032a50       ?use_verify@sslHashes@yaSSL@@QAEAAVFinished@2@XZ 00433a50 f   yassl:yassl_int.obj
 0001:00032a60       ?use_certVerify@sslHashes@yaSSL@@QAEAAUHashes@2@XZ 00433a60 f   yassl:yassl_int.obj
 0001:00032a70       ?SetRawInput@Buffers@yaSSL@@QAEXPAVinput_buffer@2@@Z 00433a70 f   yassl:yassl_int.obj
 0001:00032a80       ?TakeRawInput@Buffers@yaSSL@@QAEPAVinput_buffer@2@XZ 00433a80 f   yassl:yassl_int.obj
 0001:00032a90       ?getData@Buffers@yaSSL@@QBEABV?$list@PAVinput_buffer@yaSSL@@@mySTL@@XZ 00433a90 f   yassl:yassl_int.obj
 0001:00032aa0       ?getHandShake@Buffers@yaSSL@@QBEABV?$list@PAVoutput_buffer@yaSSL@@@mySTL@@XZ 00433aa0 f   yassl:yassl_int.obj
 0001:00032ab0       ?useData@Buffers@yaSSL@@QAEAAV?$list@PAVinput_buffer@yaSSL@@@mySTL@@XZ 00433ab0 f   yassl:yassl_int.obj
 0001:00032ac0       ?useHandShake@Buffers@yaSSL@@QAEAAV?$list@PAVoutput_buffer@yaSSL@@@mySTL@@XZ 00433ac0 f   yassl:yassl_int.obj
 0001:00032ad0       ?get_connection@Security@yaSSL@@QBEABUConnection@2@XZ 00433ad0 f   yassl:yassl_int.obj
 0001:00032ae0       ?GetContext@Security@yaSSL@@QBEPBVSSL_CTX@2@XZ 00433ae0 f   yassl:yassl_int.obj
 0001:00032af0       ?get_parms@Security@yaSSL@@QBEABUParameters@2@XZ 00433af0 f   yassl:yassl_int.obj
 0001:00032b00       ?get_resume@Security@yaSSL@@QBEABVSSL_SESSION@2@XZ 00433b00 f   yassl:yassl_int.obj
 0001:00032b10       ?get_resuming@Security@yaSSL@@QBE_NXZ 00433b10 f   yassl:yassl_int.obj
 0001:00032b20       ?use_connection@Security@yaSSL@@QAEAAUConnection@2@XZ 00433b20 f   yassl:yassl_int.obj
 0001:00032b30       ?use_parms@Security@yaSSL@@QAEAAUParameters@2@XZ 00433b30 f   yassl:yassl_int.obj
 0001:00032b40       ?use_resume@Security@yaSSL@@QAEAAVSSL_SESSION@2@XZ 00433b40 f   yassl:yassl_int.obj
 0001:00032b50       ?set_resuming@Security@yaSSL@@QAEX_N@Z 00433b50 f   yassl:yassl_int.obj
 0001:00032b60       ??0X509_NAME@yaSSL@@QAE@PBDI@Z 00433b60 f   yassl:yassl_int.obj
 0001:00032ba0       ?GetName@X509_NAME@yaSSL@@QBEPBDXZ 00433ba0 f   yassl:yassl_int.obj
 0001:00032bb0       ?GetLength@X509_NAME@yaSSL@@QBEIXZ 00433bb0 f   yassl:yassl_int.obj
 0001:00032bc0       ?GetIssuer@X509@yaSSL@@QAEPAVX509_NAME@2@XZ 00433bc0 f   yassl:yassl_int.obj
 0001:00032bd0       ?GetSubject@X509@yaSSL@@QAEPAVX509_NAME@2@XZ 00433bd0 f   yassl:yassl_int.obj
 0001:00032be0       ??0StringHolder@yaSSL@@QAE@PBDH@Z 00433be0 f   yassl:yassl_int.obj
 0001:00032c20       ?GetString@StringHolder@yaSSL@@QAEPAUASN1_STRING@2@XZ 00433c20 f   yassl:yassl_int.obj
 0001:00032c30       ?Compress@yaSSL@@YAHPBEHAAVinput_buffer@1@@Z 00433c30 f   yassl:yassl_int.obj
 0001:00032c40       ?DeCompress@yaSSL@@YAHAAVinput_buffer@1@H0@Z 00433c40 f   yassl:yassl_int.obj
 0001:00032c50       ??0?$list@PAVx509@yaSSL@@@mySTL@@QAE@XZ 00433c50 f i yassl:yassl_int.obj
 0001:00032c60       ??0?$list@PAVSSL_SESSION@yaSSL@@@mySTL@@QAE@XZ 00433c60 f i yassl:yassl_int.obj
 0001:00032c70       ??0?$list@UThreadError@yaSSL@@@mySTL@@QAE@XZ 00433c70 f i yassl:yassl_int.obj
 0001:00032c80       ??0?$list@PAVinput_buffer@yaSSL@@@mySTL@@QAE@XZ 00433c80 f i yassl:yassl_int.obj
 0001:00032c90       ?size@?$list@PAVinput_buffer@yaSSL@@@mySTL@@QBEIXZ 00433c90 f i yassl:yassl_int.obj
 0001:00032ca0       ??0?$list@PAVoutput_buffer@yaSSL@@@mySTL@@QAE@XZ 00433ca0 f i yassl:yassl_int.obj
 0001:00032cb0       ?size@?$list@PAVoutput_buffer@yaSSL@@@mySTL@@QBEIXZ 00433cb0 f i yassl:yassl_int.obj
 0001:00032cc0       ??Diterator@?$list@PAVx509@yaSSL@@@mySTL@@QBEAAPAVx509@yaSSL@@XZ 00433cc0 f i yassl:yassl_int.obj
 0001:00032cd0       ??Eiterator@?$list@PAVx509@yaSSL@@@mySTL@@QAEAAV012@XZ 00433cd0 f i yassl:yassl_int.obj
 0001:00032ce0       ??9iterator@?$list@PAVx509@yaSSL@@@mySTL@@QBE_NABV012@@Z 00433ce0 f i yassl:yassl_int.obj
 0001:00032d00       ??Diterator@?$list@PAVinput_buffer@yaSSL@@@mySTL@@QBEAAPAVinput_buffer@yaSSL@@XZ 00433d00 f i yassl:yassl_int.obj
 0001:00032d10       ??Eiterator@?$list@PAVinput_buffer@yaSSL@@@mySTL@@QAE?AV012@H@Z 00433d10 f i yassl:yassl_int.obj
 0001:00032d20       ??Diterator@?$list@PAVSSL_SESSION@yaSSL@@@mySTL@@QBEAAPAVSSL_SESSION@yaSSL@@XZ 00433d20 f i yassl:yassl_int.obj
 0001:00032d30       ??Eiterator@?$list@PAVSSL_SESSION@yaSSL@@@mySTL@@QAEAAV012@XZ 00433d30 f i yassl:yassl_int.obj
 0001:00032d40       ??9iterator@?$list@PAVSSL_SESSION@yaSSL@@@mySTL@@QBE_NABV012@@Z 00433d40 f i yassl:yassl_int.obj
 0001:00032d60       ??9iterator@?$list@UThreadError@yaSSL@@@mySTL@@QBE_NABV012@@Z 00433d60 f i yassl:yassl_int.obj
 0001:00032d80       ??0iterator@?$list@PAVx509@yaSSL@@@mySTL@@QAE@PAUnode@12@@Z 00433d80 f i yassl:yassl_int.obj
 0001:00032d90       ??0iterator@?$list@PAVinput_buffer@yaSSL@@@mySTL@@QAE@PAUnode@12@@Z 00433d90 f i yassl:yassl_int.obj
 0001:00032da0       ??0iterator@?$list@PAVoutput_buffer@yaSSL@@@mySTL@@QAE@PAUnode@12@@Z 00433da0 f i yassl:yassl_int.obj
 0001:00032db0       ??0iterator@?$list@PAVSSL_SESSION@yaSSL@@@mySTL@@QAE@PAUnode@12@@Z 00433db0 f i yassl:yassl_int.obj
 0001:00032dc0       ??0iterator@?$list@UThreadError@yaSSL@@@mySTL@@QAE@PAUnode@12@@Z 00433dc0 f i yassl:yassl_int.obj
 0001:00032dd0       ??Diterator@?$list@UThreadError@yaSSL@@@mySTL@@QBEAAUThreadError@yaSSL@@XZ 00433dd0 f i yassl:yassl_int.obj
 0001:00032de0       ??0?$vector_base@U?$pair@HP6APAUMessage@yaSSL@@XZ@mySTL@@@mySTL@@QAE@XZ 00433de0 f i yassl:yassl_int.obj
 0001:00032df0       ??0?$vector_base@U?$pair@HP6APAVHandShakeBase@yaSSL@@XZ@mySTL@@@mySTL@@QAE@XZ 00433df0 f i yassl:yassl_int.obj
 0001:00032e00       ??0?$vector_base@U?$pair@HP6APAUServerKeyBase@yaSSL@@XZ@mySTL@@@mySTL@@QAE@XZ 00433e00 f i yassl:yassl_int.obj
 0001:00032e10       ??0?$vector_base@U?$pair@HP6APAUClientKeyBase@yaSSL@@XZ@mySTL@@@mySTL@@QAE@XZ 00433e10 f i yassl:yassl_int.obj
 0001:00032e20       ??$GetArrayMemory@E@mySTL@@YAPAEI@Z 00433e20 f i yassl:yassl_int.obj
 0001:00032e30       ?front@?$list@PAVinput_buffer@yaSSL@@@mySTL@@QBEPAVinput_buffer@yaSSL@@XZ 00433e30 f i yassl:yassl_int.obj
 0001:00032e40       ?front@?$list@PAVoutput_buffer@yaSSL@@@mySTL@@QBEPAVoutput_buffer@yaSSL@@XZ 00433e40 f i yassl:yassl_int.obj
 0001:00032e50       ??$find_if@Viterator@?$list@PAVSSL_SESSION@yaSSL@@@mySTL@@Usess_match@yassl_int_cpp_local2@yaSSL@@@mySTL@@YA?AViterator@?$list@PAVSSL_SESSION@yaSSL@@@0@V120@0Usess_match@yassl_int_cpp_local2@yaSSL@@@Z 00433e50 f i yassl:yassl_int.obj
 0001:00032e90       ??$ysDelete@VSSL_METHOD@yaSSL@@@yaSSL@@YAXPAVSSL_METHOD@0@@Z 00433e90 f i yassl:yassl_int.obj
 0001:00032ea0       ??$ysDelete@UDigest@yaSSL@@@yaSSL@@YAXPAUDigest@0@@Z 00433ea0 f i yassl:yassl_int.obj
 0001:00032ec0       ??$ysArrayDelete@D@yaSSL@@YAXPAD@Z 00433ec0 f i yassl:yassl_int.obj
 0001:00032ed0       ??$ysArrayDelete@E@yaSSL@@YAXPAE@Z 00433ed0 f i yassl:yassl_int.obj
 0001:00032ee0       ??$FreeArrayMemory@U?$pair@HP6APAUMessage@yaSSL@@XZ@mySTL@@@mySTL@@YAXPAU?$pair@HP6APAUMessage@yaSSL@@XZ@0@@Z 00433ee0 f i yassl:yassl_int.obj
 0001:00032ef0       ??$FreeArrayMemory@U?$pair@HP6APAVHandShakeBase@yaSSL@@XZ@mySTL@@@mySTL@@YAXPAU?$pair@HP6APAVHandShakeBase@yaSSL@@XZ@0@@Z 00433ef0 f i yassl:yassl_int.obj
 0001:00032f00       ??$FreeArrayMemory@U?$pair@HP6APAUServerKeyBase@yaSSL@@XZ@mySTL@@@mySTL@@YAXPAU?$pair@HP6APAUServerKeyBase@yaSSL@@XZ@0@@Z 00433f00 f i yassl:yassl_int.obj
 0001:00032f10       ??$FreeArrayMemory@U?$pair@HP6APAUClientKeyBase@yaSSL@@XZ@mySTL@@@mySTL@@YAXPAU?$pair@HP6APAUClientKeyBase@yaSSL@@XZ@0@@Z 00433f10 f i yassl:yassl_int.obj
 0001:00032f20       ??_Ginput_buffer@yaSSL@@QAEPAXI@Z 00433f20 f i yassl:yassl_int.obj
 0001:00032f40       ??_Goutput_buffer@yaSSL@@QAEPAXI@Z 00433f40 f i yassl:yassl_int.obj
 0001:00032f60       ??_GDiffieHellman@yaSSL@@QAEPAXI@Z 00433f60 f i yassl:yassl_int.obj
 0001:00032f80       ??Eiterator@?$list@PAVinput_buffer@yaSSL@@@mySTL@@QAEAAV012@XZ 00433f80 f i yassl:yassl_int.obj
 0001:00032f90       ??9iterator@?$list@PAVinput_buffer@yaSSL@@@mySTL@@QBE_NABV012@@Z 00433f90 f i yassl:yassl_int.obj
 0001:00032fb0       ??Diterator@?$list@PAVoutput_buffer@yaSSL@@@mySTL@@QBEAAPAVoutput_buffer@yaSSL@@XZ 00433fb0 f i yassl:yassl_int.obj
 0001:00032fc0       ??Eiterator@?$list@PAVoutput_buffer@yaSSL@@@mySTL@@QAEAAV012@XZ 00433fc0 f i yassl:yassl_int.obj
 0001:00032fd0       ??9iterator@?$list@PAVoutput_buffer@yaSSL@@@mySTL@@QBE_NABV012@@Z 00433fd0 f i yassl:yassl_int.obj
 0001:00032ff0       ??Eiterator@?$list@UThreadError@yaSSL@@@mySTL@@QAEAAV012@XZ 00433ff0 f i yassl:yassl_int.obj
 0001:00033000       ??0node@?$list@PAVx509@yaSSL@@@mySTL@@QAE@PAVx509@yaSSL@@@Z 00434000 f i yassl:yassl_int.obj
 0001:00033020       ??0node@?$list@PAVinput_buffer@yaSSL@@@mySTL@@QAE@PAVinput_buffer@yaSSL@@@Z 00434020 f i yassl:yassl_int.obj
 0001:00033040       ??0node@?$list@PAVSSL_SESSION@yaSSL@@@mySTL@@QAE@PAVSSL_SESSION@yaSSL@@@Z 00434040 f i yassl:yassl_int.obj
 0001:00033060       ??0node@?$list@UThreadError@yaSSL@@@mySTL@@QAE@UThreadError@yaSSL@@@Z 00434060 f i yassl:yassl_int.obj
 0001:00033080       ??0node@?$list@PAVoutput_buffer@yaSSL@@@mySTL@@QAE@PAVoutput_buffer@yaSSL@@@Z 00434080 f i yassl:yassl_int.obj
 0001:000330a0       ??$destroy@Unode@?$list@PAVx509@yaSSL@@@mySTL@@@mySTL@@YAXPAUnode@?$list@PAVx509@yaSSL@@@0@@Z 004340a0 f i yassl:yassl_int.obj
 0001:000330b0       ??$destroy@Unode@?$list@PAVSSL_SESSION@yaSSL@@@mySTL@@@mySTL@@YAXPAUnode@?$list@PAVSSL_SESSION@yaSSL@@@0@@Z 004340b0 f i yassl:yassl_int.obj
 0001:000330c0       ??$destroy@Unode@?$list@UThreadError@yaSSL@@@mySTL@@@mySTL@@YAXPAUnode@?$list@UThreadError@yaSSL@@@0@@Z 004340c0 f i yassl:yassl_int.obj
 0001:000330d0       ??$destroy@Unode@?$list@PAVinput_buffer@yaSSL@@@mySTL@@@mySTL@@YAXPAUnode@?$list@PAVinput_buffer@yaSSL@@@0@@Z 004340d0 f i yassl:yassl_int.obj
 0001:000330e0       ??$destroy@Unode@?$list@PAVoutput_buffer@yaSSL@@@mySTL@@@mySTL@@YAXPAUnode@?$list@PAVoutput_buffer@yaSSL@@@0@@Z 004340e0 f i yassl:yassl_int.obj
 0001:000330f0       ??$swap@PAVSSL_SESSION@yaSSL@@@mySTL@@YAXAAPAVSSL_SESSION@yaSSL@@0@Z 004340f0 f i yassl:yassl_int.obj
 0001:00033110       ??$destroy@U?$pair@HP6APAUMessage@yaSSL@@XZ@mySTL@@@mySTL@@YAXPAU?$pair@HP6APAUMessage@yaSSL@@XZ@0@@Z 00434110 f i yassl:yassl_int.obj
 0001:00033120       ??$destroy@U?$pair@HP6APAVHandShakeBase@yaSSL@@XZ@mySTL@@@mySTL@@YAXPAU?$pair@HP6APAVHandShakeBase@yaSSL@@XZ@0@@Z 00434120 f i yassl:yassl_int.obj
 0001:00033130       ??$destroy@U?$pair@HP6APAUServerKeyBase@yaSSL@@XZ@mySTL@@@mySTL@@YAXPAU?$pair@HP6APAUServerKeyBase@yaSSL@@XZ@0@@Z 00434130 f i yassl:yassl_int.obj
 0001:00033140       ??$destroy@U?$pair@HP6APAUClientKeyBase@yaSSL@@XZ@mySTL@@@mySTL@@YAXPAU?$pair@HP6APAUClientKeyBase@yaSSL@@XZ@0@@Z 00434140 f i yassl:yassl_int.obj
 0001:00033150       ??$swap@PAVx509@yaSSL@@@mySTL@@YAXAAPAVx509@yaSSL@@0@Z 00434150 f i yassl:yassl_int.obj
 0001:00033170       ??$swap@PAVoutput_buffer@yaSSL@@@mySTL@@YAXAAPAVoutput_buffer@yaSSL@@0@Z 00434170 f i yassl:yassl_int.obj
 0001:00033190       ??$swap@PAVinput_buffer@yaSSL@@@mySTL@@YAXAAPAVinput_buffer@yaSSL@@0@Z 00434190 f i yassl:yassl_int.obj
 0001:000331b0       ?GetMemory@mySTL@@YAPAXI@Z 004341b0 f i yassl:yassl_int.obj
 0001:000331c0       ??0sslHashes@yaSSL@@QAE@XZ 004341c0 f i yassl:yassl_int.obj
 0001:000331e0       ?set_pending@SSL@yaSSL@@QAEXE@Z 004341e0 f   yassl:yassl_int.obj
 0001:00033f20       ?set_random@SSL@yaSSL@@QAEXPBEW4ConnectionEnd@2@@Z 00434f20 f   yassl:yassl_int.obj
 0001:00033f50       ?set_preMaster@SSL@yaSSL@@QAEXPBEI@Z 00434f50 f   yassl:yassl_int.obj
 0001:00033f80       ?UnSetCompression@SSL@yaSSL@@QAEXXZ 00434f80 f   yassl:yassl_int.obj
 0001:00033f90       ?CompressionOn@SSL@yaSSL@@QBE_NXZ 00434f90 f   yassl:yassl_int.obj
 0001:00033fa0       ?set_masterSecret@SSL@yaSSL@@QAEXPBE@Z 00434fa0 f   yassl:yassl_int.obj
 0001:00033fc0       ?set_sessionID@SSL@yaSSL@@QAEXPBE@Z 00434fc0 f   yassl:yassl_int.obj
 0001:00033ff0       ?setKeys@SSL@yaSSL@@AAEXXZ 00434ff0 f   yassl:yassl_int.obj
 0001:00034090       ?get_SEQIncrement@SSL@yaSSL@@QAEI_N@Z 00435090 f   yassl:yassl_int.obj
 0001:000340c0       ?get_macSecret@SSL@yaSSL@@QAEPBE_N@Z 004350c0 f   yassl:yassl_int.obj
 0001:00034100       ?verifyState@SSL@yaSSL@@QAEXABURecordLayerHeader@2@@Z 00435100 f   yassl:yassl_int.obj
 0001:00034160       ?verifyState@SSL@yaSSL@@QAEXW4ClientState@2@@Z 00435160 f   yassl:yassl_int.obj
 0001:00034190       ?verifyState@SSL@yaSSL@@QAEXW4ServerState@2@@Z 00435190 f   yassl:yassl_int.obj
 0001:000341c0       ?verfiyHandShakeComplete@SSL@yaSSL@@QAEXXZ 004351c0 f   yassl:yassl_int.obj
 0001:000341f0       ?verifyClientState@SSL@yaSSL@@AAEXW4HandShakeType@2@@Z 004351f0 f   yassl:yassl_int.obj
 0001:000342c0       ?verifyServerState@SSL@yaSSL@@AAEXW4HandShakeType@2@@Z 004352c0 f   yassl:yassl_int.obj
 0001:00034370       ?matchSuite@SSL@yaSSL@@QAEXPBEI@Z 00435370 f   yassl:yassl_int.obj
 0001:00034400       ?GetMultiProtocol@SSL@yaSSL@@QBE_NXZ 00435400 f   yassl:yassl_int.obj
 0001:00034420       ?isTLS@SSL@yaSSL@@QBE_NXZ  00435420 f   yassl:yassl_int.obj
 0001:00034430       ?isTLSv1_1@SSL@yaSSL@@QBE_NXZ 00435430 f   yassl:yassl_int.obj
 0001:00034440       ??1X509_NAME@yaSSL@@QAE@XZ 00435440 f   yassl:yassl_int.obj
 0001:00034460       ?GetBefore@X509@yaSSL@@QAEPAUASN1_STRING@2@XZ 00435460 f   yassl:yassl_int.obj
 0001:00034470       ?GetAfter@X509@yaSSL@@QAEPAUASN1_STRING@2@XZ 00435470 f   yassl:yassl_int.obj
 0001:00034480       ?GetEntry@X509_NAME@yaSSL@@QAEPAUASN1_STRING@2@H@Z 00435480 f   yassl:yassl_int.obj
 0001:00034510       ??1StringHolder@yaSSL@@QAE@XZ 00435510 f   yassl:yassl_int.obj
 0001:00034520       ?begin@?$list@PAVx509@yaSSL@@@mySTL@@QBE?AViterator@12@XZ 00435520 f i yassl:yassl_int.obj
 0001:00034530       ?end@?$list@PAVx509@yaSSL@@@mySTL@@QBE?AViterator@12@XZ 00435530 f i yassl:yassl_int.obj
 0001:00034540       ?begin@?$list@PAVSSL_SESSION@yaSSL@@@mySTL@@QBE?AViterator@12@XZ 00435540 f i yassl:yassl_int.obj
 0001:00034550       ?end@?$list@PAVSSL_SESSION@yaSSL@@@mySTL@@QBE?AViterator@12@XZ 00435550 f i yassl:yassl_int.obj
 0001:00034560       ?begin@?$list@UThreadError@yaSSL@@@mySTL@@QBE?AViterator@12@XZ 00435560 f i yassl:yassl_int.obj
 0001:00034570       ?end@?$list@UThreadError@yaSSL@@@mySTL@@QBE?AViterator@12@XZ 00435570 f i yassl:yassl_int.obj
 0001:00034580       ?begin@?$list@PAVinput_buffer@yaSSL@@@mySTL@@QBE?AViterator@12@XZ 00435580 f i yassl:yassl_int.obj
 0001:00034590       ?end@?$list@PAVinput_buffer@yaSSL@@@mySTL@@QBE?AViterator@12@XZ 00435590 f i yassl:yassl_int.obj
 0001:000345a0       ?begin@?$list@PAVoutput_buffer@yaSSL@@@mySTL@@QBE?AViterator@12@XZ 004355a0 f i yassl:yassl_int.obj
 0001:000345b0       ?end@?$list@PAVoutput_buffer@yaSSL@@@mySTL@@QBE?AViterator@12@XZ 004355b0 f i yassl:yassl_int.obj
 0001:000345c0       ??Citerator@?$list@UThreadError@yaSSL@@@mySTL@@QBEPAUThreadError@yaSSL@@XZ 004355c0 f i yassl:yassl_int.obj
 0001:000345d0       ??1?$vector_base@U?$pair@HP6APAUMessage@yaSSL@@XZ@mySTL@@@mySTL@@QAE@XZ 004355d0 f i yassl:yassl_int.obj
 0001:000345e0       ??1?$vector_base@U?$pair@HP6APAVHandShakeBase@yaSSL@@XZ@mySTL@@@mySTL@@QAE@XZ 004355e0 f i yassl:yassl_int.obj
 0001:000345f0       ??1?$vector_base@U?$pair@HP6APAUServerKeyBase@yaSSL@@XZ@mySTL@@@mySTL@@QAE@XZ 004355f0 f i yassl:yassl_int.obj
 0001:00034600       ??1?$vector_base@U?$pair@HP6APAUClientKeyBase@yaSSL@@XZ@mySTL@@@mySTL@@QAE@XZ 00435600 f i yassl:yassl_int.obj
 0001:00034610       ??$FreeArrayMemory@X@mySTL@@YAXPAX@Z 00435610 f i yassl:yassl_int.obj
 0001:00034620       ?push_back@?$list@PAVx509@yaSSL@@@mySTL@@QAEXPAVx509@yaSSL@@@Z 00435620 f i yassl:yassl_int.obj
 0001:00034670       ?push_back@?$list@PAVSSL_SESSION@yaSSL@@@mySTL@@QAEXPAVSSL_SESSION@yaSSL@@@Z 00435670 f i yassl:yassl_int.obj
 0001:000346c0       ?push_back@?$list@UThreadError@yaSSL@@@mySTL@@QAEXUThreadError@yaSSL@@@Z 004356c0 f i yassl:yassl_int.obj
 0001:00034720       ?push_back@?$list@PAVinput_buffer@yaSSL@@@mySTL@@QAEXPAVinput_buffer@yaSSL@@@Z 00435720 f i yassl:yassl_int.obj
 0001:00034770       ?push_back@?$list@PAVoutput_buffer@yaSSL@@@mySTL@@QAEXPAVoutput_buffer@yaSSL@@@Z 00435770 f i yassl:yassl_int.obj
 0001:000347c0       ??$for_each@Viterator@?$list@PAVinput_buffer@yaSSL@@@mySTL@@USumData@yassl_int_cpp_local1@yaSSL@@@mySTL@@YA?AUSumData@yassl_int_cpp_local1@yaSSL@@Viterator@?$list@PAVinput_buffer@yaSSL@@@0@0U123@@Z 004357c0 f i yassl:yassl_int.obj
 0001:00034800       ??$ysDelete@Vinput_buffer@yaSSL@@@yaSSL@@YAXPAVinput_buffer@0@@Z 00435800 f i yassl:yassl_int.obj
 0001:00034820       ??$for_each@Viterator@?$list@PAVoutput_buffer@yaSSL@@@mySTL@@USumBuffer@yassl_int_cpp_local1@yaSSL@@@mySTL@@YA?AUSumBuffer@yassl_int_cpp_local1@yaSSL@@Viterator@?$list@PAVoutput_buffer@yaSSL@@@0@0U123@@Z 00435820 f i yassl:yassl_int.obj
 0001:00034860       ??$ysDelete@Voutput_buffer@yaSSL@@@yaSSL@@YAXPAVoutput_buffer@0@@Z 00435860 f i yassl:yassl_int.obj
 0001:00034880       ??$find_if@Viterator@?$list@UThreadError@yaSSL@@@mySTL@@Uthr_match@yassl_int_cpp_local2@yaSSL@@@mySTL@@YA?AViterator@?$list@UThreadError@yaSSL@@@0@V120@0Uthr_match@yassl_int_cpp_local2@yaSSL@@@Z 00435880 f i yassl:yassl_int.obj
 0001:000348b0       ??$ysDelete@VDiffieHellman@yaSSL@@@yaSSL@@YAXPAVDiffieHellman@0@@Z 004358b0 f i yassl:yassl_int.obj
 0001:000348d0       ??$destroy@PAU?$pair@HP6APAUMessage@yaSSL@@XZ@mySTL@@@mySTL@@YAXPAU?$pair@HP6APAUMessage@yaSSL@@XZ@0@0@Z 004358d0 f i yassl:yassl_int.obj
 0001:000348e0       ??$destroy@PAU?$pair@HP6APAVHandShakeBase@yaSSL@@XZ@mySTL@@@mySTL@@YAXPAU?$pair@HP6APAVHandShakeBase@yaSSL@@XZ@0@0@Z 004358e0 f i yassl:yassl_int.obj
 0001:000348f0       ??$destroy@PAU?$pair@HP6APAUServerKeyBase@yaSSL@@XZ@mySTL@@@mySTL@@YAXPAU?$pair@HP6APAUServerKeyBase@yaSSL@@XZ@0@0@Z 004358f0 f i yassl:yassl_int.obj
 0001:00034900       ??$destroy@PAU?$pair@HP6APAUClientKeyBase@yaSSL@@XZ@mySTL@@@mySTL@@YAXPAU?$pair@HP6APAUClientKeyBase@yaSSL@@XZ@0@0@Z 00435900 f i yassl:yassl_int.obj
 0001:00034910       ??$checked_delete@Vx509@yaSSL@@@yaSSL@@YAXPAVx509@0@@Z 00435910 f i yassl:yassl_int.obj
 0001:00034920       ??$checked_delete@Voutput_buffer@yaSSL@@@yaSSL@@YAXPAVoutput_buffer@0@@Z 00435920 f i yassl:yassl_int.obj
 0001:00034930       ??$checked_delete@Vinput_buffer@yaSSL@@@yaSSL@@YAXPAVinput_buffer@0@@Z 00435930 f i yassl:yassl_int.obj
 0001:00034940       ?FreeMemory@mySTL@@YAXPAX@Z 00435940 f i yassl:yassl_int.obj
 0001:00034950       ??1X509@yaSSL@@QAE@XZ      00435950 f i yassl:yassl_int.obj
 0001:00034980       ?storeKeys@SSL@yaSSL@@AAEXPBE@Z 00435980 f   yassl:yassl_int.obj
 0001:00034a40       ?bufferedData@SSL@yaSSL@@QAEIXZ 00435a40 f   yassl:yassl_int.obj
 0001:00034a70       ?PeekData@SSL@yaSSL@@QAEXAAVData@2@@Z 00435a70 f   yassl:yassl_int.obj
 0001:00034b90       ?verifyState@SSL@yaSSL@@QAEXABVHandShakeHeader@2@@Z 00435b90 f   yassl:yassl_int.obj
 0001:00034bf0       ?addData@SSL@yaSSL@@QAEXPAVinput_buffer@2@@Z 00435bf0 f   yassl:yassl_int.obj
 0001:00034c20       ?addBuffer@SSL@yaSSL@@QAEXPAVoutput_buffer@2@@Z 00435c20 f   yassl:yassl_int.obj
 0001:00034c40       ?AddCA@SSL_CTX@yaSSL@@QAEXPAVx509@2@@Z 00435c40 f   yassl:yassl_int.obj
 0001:00034c50       ??1Crypto@yaSSL@@QAE@XZ    00435c50 f   yassl:yassl_int.obj
 0001:00034c90       ??0X509@yaSSL@@QAE@PBDI0I0H0H@Z 00435c90 f   yassl:yassl_int.obj
 0001:00034ce0       ??1?$vector@U?$pair@HP6APAUMessage@yaSSL@@XZ@mySTL@@@mySTL@@QAE@XZ 00435ce0 f i yassl:yassl_int.obj
 0001:00034cf0       ??1?$vector@U?$pair@HP6APAVHandShakeBase@yaSSL@@XZ@mySTL@@@mySTL@@QAE@XZ 00435cf0 f i yassl:yassl_int.obj
 0001:00034d00       ??1?$vector@U?$pair@HP6APAUServerKeyBase@yaSSL@@XZ@mySTL@@@mySTL@@QAE@XZ 00435d00 f i yassl:yassl_int.obj
 0001:00034d10       ??1?$vector@U?$pair@HP6APAUClientKeyBase@yaSSL@@XZ@mySTL@@@mySTL@@QAE@XZ 00435d10 f i yassl:yassl_int.obj
 0001:00034d20       ??0?$vector@U?$pair@HP6APAUMessage@yaSSL@@XZ@mySTL@@@mySTL@@QAE@XZ 00435d20 f i yassl:yassl_int.obj
 0001:00034d30       ??0?$vector@U?$pair@HP6APAVHandShakeBase@yaSSL@@XZ@mySTL@@@mySTL@@QAE@XZ 00435d30 f i yassl:yassl_int.obj
 0001:00034d40       ??0?$vector@U?$pair@HP6APAUServerKeyBase@yaSSL@@XZ@mySTL@@@mySTL@@QAE@XZ 00435d40 f i yassl:yassl_int.obj
 0001:00034d50       ??0?$vector@U?$pair@HP6APAUClientKeyBase@yaSSL@@XZ@mySTL@@@mySTL@@QAE@XZ 00435d50 f i yassl:yassl_int.obj
 0001:00034d60       ??1?$list@PAVx509@yaSSL@@@mySTL@@QAE@XZ 00435d60 f i yassl:yassl_int.obj
 0001:00034d80       ??1?$list@PAVSSL_SESSION@yaSSL@@@mySTL@@QAE@XZ 00435d80 f i yassl:yassl_int.obj
 0001:00034da0       ??1?$list@UThreadError@yaSSL@@@mySTL@@QAE@XZ 00435da0 f i yassl:yassl_int.obj
 0001:00034dc0       ??1?$list@PAVinput_buffer@yaSSL@@@mySTL@@QAE@XZ 00435dc0 f i yassl:yassl_int.obj
 0001:00034de0       ?pop_front@?$list@PAVinput_buffer@yaSSL@@@mySTL@@QAEXXZ 00435de0 f i yassl:yassl_int.obj
 0001:00034e30       ??1?$list@PAVoutput_buffer@yaSSL@@@mySTL@@QAE@XZ 00435e30 f i yassl:yassl_int.obj
 0001:00034e50       ?pop_front@?$list@PAVoutput_buffer@yaSSL@@@mySTL@@QAEXXZ 00435e50 f i yassl:yassl_int.obj
 0001:00034ea0       ??_GX509@yaSSL@@QAEPAXI@Z  00435ea0 f i yassl:yassl_int.obj
 0001:00034ee0       ?pop_front@?$list@PAVSSL_SESSION@yaSSL@@@mySTL@@QAEXXZ 00435ee0 f i yassl:yassl_int.obj
 0001:00034f30       ?pop_back@?$list@PAVSSL_SESSION@yaSSL@@@mySTL@@QAEXXZ 00435f30 f i yassl:yassl_int.obj
 0001:00034f70       ?pop_front@?$list@UThreadError@yaSSL@@@mySTL@@QAEXXZ 00435f70 f i yassl:yassl_int.obj
 0001:00034fc0       ?pop_back@?$list@UThreadError@yaSSL@@@mySTL@@QAEXXZ 00435fc0 f i yassl:yassl_int.obj
 0001:00035000       ??$?RVx509@yaSSL@@@del_ptr_zero@yaSSL@@QBEXAAPAVx509@1@@Z 00436000 f i yassl:yassl_int.obj
 0001:00035020       ??$?RVoutput_buffer@yaSSL@@@del_ptr_zero@yaSSL@@QBEXAAPAVoutput_buffer@1@@Z 00436020 f i yassl:yassl_int.obj
 0001:00035040       ??$?RVinput_buffer@yaSSL@@@del_ptr_zero@yaSSL@@QBEXAAPAVinput_buffer@1@@Z 00436040 f i yassl:yassl_int.obj
 0001:00035060       ??0Sessions@yaSSL@@AAE@XZ  00436060 f i yassl:yassl_int.obj
 0001:00035090       ??0Errors@yaSSL@@AAE@XZ    00436090 f i yassl:yassl_int.obj
 0001:000350a0       ??1Errors@yaSSL@@QAE@XZ    004360a0 f i yassl:yassl_int.obj
 0001:000350b0       ??1?$Factory@UMessage@yaSSL@@HP6APAU12@XZ@yaSSL@@QAE@XZ 004360b0 f i yassl:yassl_int.obj
 0001:000350c0       ??1?$Factory@VHandShakeBase@yaSSL@@HP6APAV12@XZ@yaSSL@@QAE@XZ 004360c0 f i yassl:yassl_int.obj
 0001:000350d0       ??1?$Factory@UServerKeyBase@yaSSL@@HP6APAU12@XZ@yaSSL@@QAE@XZ 004360d0 f i yassl:yassl_int.obj
 0001:000350e0       ??1?$Factory@UClientKeyBase@yaSSL@@HP6APAU12@XZ@yaSSL@@QAE@XZ 004360e0 f i yassl:yassl_int.obj
 0001:000350f0       ?deriveKeys@SSL@yaSSL@@QAEXXZ 004360f0 f   yassl:yassl_int.obj
 0001:000352d0       ?deriveTLSKeys@SSL@yaSSL@@QAEXXZ 004362d0 f   yassl:yassl_int.obj
 0001:00035390       ?fillData@SSL@yaSSL@@QAEXAAVData@2@@Z 00436390 f   yassl:yassl_int.obj
 0001:00035500       ?flushBuffer@SSL@yaSSL@@QAEXXZ 00436500 f   yassl:yassl_int.obj
 0001:000355d0       ?CopyX509@SSL_SESSION@yaSSL@@AAEXPAVX509@2@@Z 004365d0 f   yassl:yassl_int.obj
 0001:00035670       ??0SSL_SESSION@yaSSL@@QAE@ABVSSL@1@AAVRandomPool@1@@Z 00436670 f   yassl:yassl_int.obj
 0001:00035700       ?GetSessions@yaSSL@@YAAAVSessions@1@XZ 00436700 f   yassl:yassl_int.obj
 0001:00035750       ?GetErrors@yaSSL@@YAAAVErrors@1@XZ 00436750 f   yassl:yassl_int.obj
 0001:00035790       ??0SSL_CTX@yaSSL@@QAE@PAVSSL_METHOD@1@@Z 00436790 f   yassl:yassl_int.obj
 0001:00035850       ??0Buffers@yaSSL@@QAE@XZ   00436850 f   yassl:yassl_int.obj
 0001:00035870       ??0?$Factory@UMessage@yaSSL@@HP6APAU12@XZ@yaSSL@@QAE@P6AXAAV01@@Z@Z 00436870 f i yassl:yassl_int.obj
 0001:00035890       ??0?$Factory@VHandShakeBase@yaSSL@@HP6APAV12@XZ@yaSSL@@QAE@P6AXAAV01@@Z@Z 00436890 f i yassl:yassl_int.obj
 0001:000358b0       ??0?$Factory@UServerKeyBase@yaSSL@@HP6APAU12@XZ@yaSSL@@QAE@P6AXAAV01@@Z@Z 004368b0 f i yassl:yassl_int.obj
 0001:000358d0       ??0?$Factory@UClientKeyBase@yaSSL@@HP6APAU12@XZ@yaSSL@@QAE@P6AXAAV01@@Z@Z 004368d0 f i yassl:yassl_int.obj
 0001:000358f0       ?erase@?$list@PAVSSL_SESSION@yaSSL@@@mySTL@@QAE_NViterator@12@@Z 004368f0 f i yassl:yassl_int.obj
 0001:00035950       ?erase@?$list@UThreadError@yaSSL@@@mySTL@@QAE_NViterator@12@@Z 00436950 f i yassl:yassl_int.obj
 0001:000359b0       ??$ysDelete@VX509@yaSSL@@@yaSSL@@YAXPAVX509@0@@Z 004369b0 f i yassl:yassl_int.obj
 0001:000359f0       ??$for_each@Viterator@?$list@PAVx509@yaSSL@@@mySTL@@Udel_ptr_zero@yaSSL@@@mySTL@@YA?AUdel_ptr_zero@yaSSL@@Viterator@?$list@PAVx509@yaSSL@@@0@0U12@@Z 004369f0 f i yassl:yassl_int.obj
 0001:00035a30       ??$for_each@Viterator@?$list@PAVoutput_buffer@yaSSL@@@mySTL@@Udel_ptr_zero@yaSSL@@@mySTL@@YA?AUdel_ptr_zero@yaSSL@@Viterator@?$list@PAVoutput_buffer@yaSSL@@@0@0U12@@Z 00436a30 f i yassl:yassl_int.obj
 0001:00035a70       ??$for_each@Viterator@?$list@PAVinput_buffer@yaSSL@@@mySTL@@Udel_ptr_zero@yaSSL@@@mySTL@@YA?AUdel_ptr_zero@yaSSL@@Viterator@?$list@PAVinput_buffer@yaSSL@@@0@0U12@@Z 00436a70 f i yassl:yassl_int.obj
 0001:00035ab0       ??_GErrors@yaSSL@@QAEPAXI@Z 00436ab0 f i yassl:yassl_int.obj
 0001:00035ad0       ??1sslFactory@yaSSL@@QAE@XZ 00436ad0 f i yassl:yassl_int.obj
 0001:00035b00       ??0sslFactory@yaSSL@@AAE@XZ 00436b00 f   yassl:yassl_int.obj
 0001:00035b50       ?makeTLSMasterSecret@SSL@yaSSL@@QAEXXZ 00436b50 f   yassl:yassl_int.obj
 0001:00035bd0       ??4SSL_SESSION@yaSSL@@QAEAAV01@ABV01@@Z 00436bd0 f   yassl:yassl_int.obj
 0001:00035c40       ??1SSL_SESSION@yaSSL@@QAE@XZ 00436c40 f   yassl:yassl_int.obj
 0001:00035c60       ?GetSSL_Factory@yaSSL@@YAAAVsslFactory@1@XZ 00436c60 f   yassl:yassl_int.obj
 0001:00035c90       ?Remove@Errors@yaSSL@@QAEXXZ 00436c90 f   yassl:yassl_int.obj
 0001:00035cc0       ?Lookup@Errors@yaSSL@@QAEH_N@Z 00436cc0 f   yassl:yassl_int.obj
 0001:00035d10       ?Add@Errors@yaSSL@@QAEXH@Z 00436d10 f   yassl:yassl_int.obj
 0001:00035d40       ??1SSL_CTX@yaSSL@@QAE@XZ   00436d40 f   yassl:yassl_int.obj
 0001:00035da0       ??1Buffers@yaSSL@@QAE@XZ   00436da0 f   yassl:yassl_int.obj
 0001:00035e00       ??0Security@yaSSL@@QAE@UProtocolVersion@1@AAVRandomPool@1@W4ConnectionEnd@1@ABUCiphers@1@PAVSSL_CTX@1@_N@Z 00436e00 f   yassl:yassl_int.obj
 0001:00035e60       ??$ysDelete@VErrors@yaSSL@@@yaSSL@@YAXPAVErrors@0@@Z 00436e60 f i yassl:yassl_int.obj
 0001:00035e80       ??_GsslFactory@yaSSL@@QAEPAXI@Z 00436e80 f i yassl:yassl_int.obj
 0001:00035ec0       ??_GSSL_SESSION@yaSSL@@QAEPAXI@Z 00436ec0 f i yassl:yassl_int.obj
 0001:00035ee0       ?makeMasterSecret@SSL@yaSSL@@QAEXXZ 00436ee0 f   yassl:yassl_int.obj
 0001:000360e0       ?getFactory@SSL@yaSSL@@QBEABVsslFactory@2@XZ 004370e0 f   yassl:yassl_int.obj
 0001:000360f0       ??$ysDelete@VsslFactory@yaSSL@@@yaSSL@@YAXPAVsslFactory@0@@Z 004370f0 f i yassl:yassl_int.obj
 0001:00036130       ??$ysDelete@VSSL_SESSION@yaSSL@@@yaSSL@@YAXPAVSSL_SESSION@0@@Z 00437130 f i yassl:yassl_int.obj
 0001:00036150       ??0SSL@yaSSL@@QAE@PAVSSL_CTX@1@@Z 00437150 f   yassl:yassl_int.obj
 0001:000363b0       ??$checked_delete@VSSL_SESSION@yaSSL@@@yaSSL@@YAXPAVSSL_SESSION@0@@Z 004373b0 f i yassl:yassl_int.obj
 0001:000363c0       ??$?RVSSL_SESSION@yaSSL@@@del_ptr_zero@yaSSL@@QBEXAAPAVSSL_SESSION@1@@Z 004373c0 f i yassl:yassl_int.obj
 0001:000363e0       ?lookup@Sessions@yaSSL@@QAEPAVSSL_SESSION@2@PBEPAV32@@Z 004373e0 f   yassl:yassl_int.obj
 0001:00036460       ?remove@Sessions@yaSSL@@QAEXPBE@Z 00437460 f   yassl:yassl_int.obj
 0001:000364b0       ?Flush@Sessions@yaSSL@@QAEXXZ 004374b0 f   yassl:yassl_int.obj
 0001:00036510       ??$for_each@Viterator@?$list@PAVSSL_SESSION@yaSSL@@@mySTL@@Udel_ptr_zero@yaSSL@@@mySTL@@YA?AUdel_ptr_zero@yaSSL@@Viterator@?$list@PAVSSL_SESSION@yaSSL@@@0@0U12@@Z 00437510 f i yassl:yassl_int.obj
 0001:00036550       ?set_session@SSL@yaSSL@@QAEXPAVSSL_SESSION@2@@Z 00437550 f   yassl:yassl_int.obj
 0001:000365c0       ?add@Sessions@yaSSL@@QAEXABVSSL@2@@Z 004375c0 f   yassl:yassl_int.obj
 0001:00036640       ??1Sessions@yaSSL@@QAE@XZ  00437640 f   yassl:yassl_int.obj
 0001:00036670       ??_GSessions@yaSSL@@QAEPAXI@Z 00437670 f i yassl:yassl_int.obj
 0001:00036690       ??$ysDelete@VSessions@yaSSL@@@yaSSL@@YAXPAVSessions@0@@Z 00437690 f i yassl:yassl_int.obj
 0001:000366b0       _yayaSSL_CleanUp           004376b0 f   yassl:yassl_int.obj
 0001:000366f0       ??1Digest@yaSSL@@UAE@XZ    004376f0 f i yassl:crypto_wrapper.obj
 0001:00036700       ??_GDigest@yaSSL@@UAEPAXI@Z 00437700 f i yassl:crypto_wrapper.obj
 0001:00036700       ??_EDigest@yaSSL@@UAEPAXI@Z 00437700 f i yassl:crypto_wrapper.obj
 0001:00036720       ??1BulkCipher@yaSSL@@UAE@XZ 00437720 f i yassl:crypto_wrapper.obj
 0001:00036730       ??_GBulkCipher@yaSSL@@UAEPAXI@Z 00437730 f i yassl:crypto_wrapper.obj
 0001:00036730       ??_EBulkCipher@yaSSL@@UAEPAXI@Z 00437730 f i yassl:crypto_wrapper.obj
 0001:00036750       ??1Auth@yaSSL@@UAE@XZ      00437750 f i yassl:crypto_wrapper.obj
 0001:00036760       ??_GAuth@yaSSL@@UAEPAXI@Z  00437760 f i yassl:crypto_wrapper.obj
 0001:00036760       ??_EAuth@yaSSL@@UAEPAXI@Z  00437760 f i yassl:crypto_wrapper.obj
 0001:00036780       ?BitsToBytes@TaoCrypt@@YAII@Z 00437780 f i yassl:crypto_wrapper.obj
 0001:00036790       ?What@Error@TaoCrypt@@QBE?AW4ErrorNumber@2@XZ 00437790 f i yassl:crypto_wrapper.obj
 0001:000367a0       ??0SHA@TaoCrypt@@QAE@XZ    004377a0 f i yassl:crypto_wrapper.obj
 0001:000367c0       ?getByteOrder@SHA@TaoCrypt@@UBE?AW4ByteOrder@2@XZ 004377c0 f i yassl:crypto_wrapper.obj
 0001:000367d0       ?getBlockSize@SHA@TaoCrypt@@UBEIXZ 004377d0 f i yassl:crypto_wrapper.obj
 0001:000367e0       ?getDigestSize@SHA@TaoCrypt@@UBEIXZ 004377e0 f i yassl:crypto_wrapper.obj
 0001:000367f0       ?getPadSize@SHA@TaoCrypt@@UBEIXZ 004377f0 f i yassl:crypto_wrapper.obj
 0001:00036800       ??1SHA@TaoCrypt@@UAE@XZ    00437800 f i yassl:crypto_wrapper.obj
 0001:00036810       ??0RIPEMD160@TaoCrypt@@QAE@XZ 00437810 f i yassl:crypto_wrapper.obj
 0001:00036830       ?getByteOrder@RIPEMD160@TaoCrypt@@UBE?AW4ByteOrder@2@XZ 00437830 f i yassl:crypto_wrapper.obj
 0001:00036840       ?getBlockSize@RIPEMD160@TaoCrypt@@UBEIXZ 00437840 f i yassl:crypto_wrapper.obj
 0001:00036850       ?getDigestSize@RIPEMD160@TaoCrypt@@UBEIXZ 00437850 f i yassl:crypto_wrapper.obj
 0001:00036860       ?getPadSize@RIPEMD160@TaoCrypt@@UBEIXZ 00437860 f i yassl:crypto_wrapper.obj
 0001:00036870       ??1RIPEMD160@TaoCrypt@@UAE@XZ 00437870 f i yassl:crypto_wrapper.obj
 0001:00036880       ??0Mode_BASE@TaoCrypt@@QAE@HW4CipherDir@1@W4Mode@1@@Z 00437880 f i yassl:crypto_wrapper.obj
 0001:000368b0       ??1Mode_BASE@TaoCrypt@@UAE@XZ 004378b0 f i yassl:crypto_wrapper.obj
 0001:000368c0       ?SetIV@Mode_BASE@TaoCrypt@@QAEXPBE@Z 004378c0 f i yassl:crypto_wrapper.obj
 0001:000368e0       ??_GMode_BASE@TaoCrypt@@UAEPAXI@Z 004378e0 f i yassl:crypto_wrapper.obj
 0001:000368e0       ??_EMode_BASE@TaoCrypt@@UAEPAXI@Z 004378e0 f i yassl:crypto_wrapper.obj
 0001:00036900       ?ECB_Process@Mode_BASE@TaoCrypt@@IAEXPAEPBEI@Z 00437900 f i yassl:crypto_wrapper.obj
 0001:00036950       ?CBC_Encrypt@Mode_BASE@TaoCrypt@@IAEXPAEPBEI@Z 00437950 f i yassl:crypto_wrapper.obj
 0001:000369c0       ?CBC_Decrypt@Mode_BASE@TaoCrypt@@IAEXPAEPBEI@Z 004379c0 f i yassl:crypto_wrapper.obj
 0001:00036a80       ??0DES@TaoCrypt@@QAE@W4CipherDir@1@W4Mode@1@@Z 00437a80 f i yassl:crypto_wrapper.obj
 0001:00036ab0       ??1DES@TaoCrypt@@UAE@XZ    00437ab0 f i yassl:crypto_wrapper.obj
 0001:00036ac0       ??0DES_EDE3@TaoCrypt@@QAE@W4CipherDir@1@W4Mode@1@@Z 00437ac0 f i yassl:crypto_wrapper.obj
 0001:00036af0       ?SetIV@DES_EDE3@TaoCrypt@@QAEXPBE@Z 00437af0 f i yassl:crypto_wrapper.obj
 0001:00036b10       ??1DES_EDE3@TaoCrypt@@UAE@XZ 00437b10 f i yassl:crypto_wrapper.obj
 0001:00036b20       ??0ARC4@TaoCrypt@@QAE@XZ   00437b20 f i yassl:crypto_wrapper.obj
 0001:00036b30       ??0AES@TaoCrypt@@QAE@W4CipherDir@1@W4Mode@1@@Z 00437b30 f i yassl:crypto_wrapper.obj
 0001:00036b60       ?SetIV@AES@TaoCrypt@@QAEXPBE@Z 00437b60 f i yassl:crypto_wrapper.obj
 0001:00036b80       ??1AES@TaoCrypt@@UAE@XZ    00437b80 f i yassl:crypto_wrapper.obj
 0001:00036b90       ?GetError@OS_Seed@TaoCrypt@@QBE?AUError@2@XZ 00437b90 f i yassl:crypto_wrapper.obj
 0001:00036ba0       ??1RandomNumberGenerator@TaoCrypt@@QAE@XZ 00437ba0 f i yassl:crypto_wrapper.obj
 0001:00036bb0       ?GetError@RandomNumberGenerator@TaoCrypt@@QBE?AW4ErrorNumber@2@XZ 00437bb0 f i yassl:crypto_wrapper.obj
 0001:00036bc0       ?Ref@Integer@TaoCrypt@@QAEAAV12@XZ 00437bc0 f i yassl:crypto_wrapper.obj
 0001:00036bd0       ??0PK_Lengths@TaoCrypt@@QAE@ABVInteger@1@@Z 00437bd0 f i yassl:crypto_wrapper.obj
 0001:00036be0       ?PaddedBlockBitLength@PK_Lengths@TaoCrypt@@QBEIXZ 00437be0 f i yassl:crypto_wrapper.obj
 0001:00036bf0       ?PaddedBlockByteLength@PK_Lengths@TaoCrypt@@QBEIXZ 00437bf0 f i yassl:crypto_wrapper.obj
 0001:00036c00       ?FixedCiphertextLength@PK_Lengths@TaoCrypt@@QBEIXZ 00437c00 f i yassl:crypto_wrapper.obj
 0001:00036c10       ?Initialize@RSA_PublicKey@TaoCrypt@@QAEXABVInteger@2@0@Z 00437c10 f i yassl:crypto_wrapper.obj
 0001:00036c30       ?GetModulus@RSA_PublicKey@TaoCrypt@@QBEABVInteger@2@XZ 00437c30 f i yassl:crypto_wrapper.obj
 0001:00036c40       ?FixedCiphertextLength@RSA_PublicKey@TaoCrypt@@QAEIXZ 00437c40 f i yassl:crypto_wrapper.obj
 0001:00036c50       ?Swap@RSA_PublicKey@TaoCrypt@@QAEXAAV12@@Z 00437c50 f i yassl:crypto_wrapper.obj
 0001:00036c70       ?GetPrivateExponent@RSA_PrivateKey@TaoCrypt@@QBEABVInteger@2@XZ 00437c70 f i yassl:crypto_wrapper.obj
 0001:00036c80       ?Swap@DH@TaoCrypt@@QAEXAAV12@@Z 00437c80 f i yassl:crypto_wrapper.obj
 0001:00036ca0       ?SetP@DH@TaoCrypt@@QAEXABVInteger@2@@Z 00437ca0 f i yassl:crypto_wrapper.obj
 0001:00036cb0       ?SetG@DH@TaoCrypt@@QAEXABVInteger@2@@Z 00437cb0 f i yassl:crypto_wrapper.obj
 0001:00036cc0       ?GetP@DH@TaoCrypt@@QAEAAVInteger@2@XZ 00437cc0 f i yassl:crypto_wrapper.obj
 0001:00036cd0       ?GetG@DH@TaoCrypt@@QAEAAVInteger@2@XZ 00437cd0 f i yassl:crypto_wrapper.obj
 0001:00036ce0       ?GetByteLength@DH@TaoCrypt@@QBEIXZ 00437ce0 f i yassl:crypto_wrapper.obj
 0001:00036cf0       ??0MD5Impl@MD5@yaSSL@@QAE@XZ 00437cf0 f i yassl:crypto_wrapper.obj
 0001:00036d10       ??0MD5Impl@MD5@yaSSL@@QAE@ABV1TaoCrypt@@@Z 00437d10 f i yassl:crypto_wrapper.obj
 0001:00036d30       ??0Digest@yaSSL@@QAE@XZ    00437d30 f i yassl:crypto_wrapper.obj
 0001:00036d40       ??0MD5@yaSSL@@QAE@ABV01@@Z 00437d40 f   yassl:crypto_wrapper.obj
 0001:00036d80       ??4MD5@yaSSL@@QAEAAV01@ABV01@@Z 00437d80 f   yassl:crypto_wrapper.obj
 0001:00036da0       ?get_digestSize@MD5@yaSSL@@UBEIXZ 00437da0 f   yassl:crypto_wrapper.obj
 0001:00036db0       ?get_padSize@MD5@yaSSL@@UBEIXZ 00437db0 f   yassl:crypto_wrapper.obj
 0001:00036dc0       ?get_digest@MD5@yaSSL@@UAEXPAEPBEI@Z 00437dc0 f   yassl:crypto_wrapper.obj
 0001:00036df0       ?get_digest@MD5@yaSSL@@UAEXPAE@Z 00437df0 f   yassl:crypto_wrapper.obj
 0001:00036e00       ?update@MD5@yaSSL@@UAEXPBEI@Z 00437e00 f   yassl:crypto_wrapper.obj
 0001:00036e10       ??0SHAImpl@SHA@yaSSL@@QAE@XZ 00437e10 f i yassl:crypto_wrapper.obj
 0001:00036e30       ??0SHAImpl@SHA@yaSSL@@QAE@ABV1TaoCrypt@@@Z 00437e30 f i yassl:crypto_wrapper.obj
 0001:00036e50       ??0SHA@yaSSL@@QAE@XZ       00437e50 f   yassl:crypto_wrapper.obj
 0001:00036ea0       ??0SHA@yaSSL@@QAE@ABV01@@Z 00437ea0 f   yassl:crypto_wrapper.obj
 0001:00036ee0       ??4SHA@yaSSL@@QAEAAV01@ABV01@@Z 00437ee0 f   yassl:crypto_wrapper.obj
 0001:00036f00       ?get_digestSize@SHA@yaSSL@@UBEIXZ 00437f00 f   yassl:crypto_wrapper.obj
 0001:00036f10       ?get_padSize@SHA@yaSSL@@UBEIXZ 00437f10 f   yassl:crypto_wrapper.obj
 0001:00036f20       ?get_digest@SHA@yaSSL@@UAEXPAEPBEI@Z 00437f20 f   yassl:crypto_wrapper.obj
 0001:00036f50       ?get_digest@SHA@yaSSL@@UAEXPAE@Z 00437f50 f   yassl:crypto_wrapper.obj
 0001:00036f60       ?update@SHA@yaSSL@@UAEXPBEI@Z 00437f60 f   yassl:crypto_wrapper.obj
 0001:00036f70       ??0RMDImpl@RMD@yaSSL@@QAE@XZ 00437f70 f i yassl:crypto_wrapper.obj
 0001:00036f90       ??0RMDImpl@RMD@yaSSL@@QAE@ABVRIPEMD160@TaoCrypt@@@Z 00437f90 f i yassl:crypto_wrapper.obj
 0001:00036fb0       ??0RMD@yaSSL@@QAE@XZ       00437fb0 f   yassl:crypto_wrapper.obj
 0001:00037000       ??0RMD@yaSSL@@QAE@ABV01@@Z 00438000 f   yassl:crypto_wrapper.obj
 0001:00037040       ??4RMD@yaSSL@@QAEAAV01@ABV01@@Z 00438040 f   yassl:crypto_wrapper.obj
 0001:00037060       ?get_digestSize@RMD@yaSSL@@UBEIXZ 00438060 f   yassl:crypto_wrapper.obj
 0001:00037070       ?get_padSize@RMD@yaSSL@@UBEIXZ 00438070 f   yassl:crypto_wrapper.obj
 0001:00037080       ?get_digest@RMD@yaSSL@@UAEXPAEPBEI@Z 00438080 f   yassl:crypto_wrapper.obj
 0001:000370b0       ?get_digest@RMD@yaSSL@@UAEXPAE@Z 004380b0 f   yassl:crypto_wrapper.obj
 0001:000370c0       ?update@RMD@yaSSL@@UAEXPBEI@Z 004380c0 f   yassl:crypto_wrapper.obj
 0001:000370d0       ??1?$HMAC@VMD5@TaoCrypt@@@TaoCrypt@@QAE@XZ 004380d0 f i yassl:crypto_wrapper.obj
 0001:000370e0       ?get_digestSize@HMAC_MD5@yaSSL@@UBEIXZ 004380e0 f   yassl:crypto_wrapper.obj
 0001:000370f0       ?get_padSize@HMAC_MD5@yaSSL@@UBEIXZ 004380f0 f   yassl:crypto_wrapper.obj
 0001:00037100       ??1?$HMAC@VSHA@TaoCrypt@@@TaoCrypt@@QAE@XZ 00438100 f i yassl:crypto_wrapper.obj
 0001:00037110       ?get_digestSize@HMAC_SHA@yaSSL@@UBEIXZ 00438110 f   yassl:crypto_wrapper.obj
 0001:00037120       ?get_padSize@HMAC_SHA@yaSSL@@UBEIXZ 00438120 f   yassl:crypto_wrapper.obj
 0001:00037130       ??1?$HMAC@VRIPEMD160@TaoCrypt@@@TaoCrypt@@QAE@XZ 00438130 f i yassl:crypto_wrapper.obj
 0001:00037140       ?get_digestSize@HMAC_RMD@yaSSL@@UBEIXZ 00438140 f   yassl:crypto_wrapper.obj
 0001:00037150       ?get_padSize@HMAC_RMD@yaSSL@@UBEIXZ 00438150 f   yassl:crypto_wrapper.obj
 0001:00037160       ??0BulkCipher@yaSSL@@QAE@XZ 00438160 f i yassl:crypto_wrapper.obj
 0001:00037170       ??1?$BlockCipher@$0A@VDES@TaoCrypt@@$00@TaoCrypt@@QAE@XZ 00438170 f i yassl:crypto_wrapper.obj
 0001:00037180       ??1?$BlockCipher@$00VDES@TaoCrypt@@$00@TaoCrypt@@QAE@XZ 00438180 f i yassl:crypto_wrapper.obj
 0001:00037190       ??1?$BlockCipher@$0A@VDES_EDE3@TaoCrypt@@$00@TaoCrypt@@QAE@XZ 00438190 f i yassl:crypto_wrapper.obj
 0001:000371a0       ??1?$BlockCipher@$00VDES_EDE3@TaoCrypt@@$00@TaoCrypt@@QAE@XZ 004381a0 f i yassl:crypto_wrapper.obj
 0001:000371b0       ??0RC4Impl@RC4@yaSSL@@QAE@XZ 004381b0 f i yassl:crypto_wrapper.obj
 0001:000371c0       ?set_encryptKey@RC4@yaSSL@@UAEXPBE0@Z 004381c0 f   yassl:crypto_wrapper.obj
 0001:000371d0       ?set_decryptKey@RC4@yaSSL@@UAEXPBE0@Z 004381d0 f   yassl:crypto_wrapper.obj
 0001:000371f0       ?encrypt@RC4@yaSSL@@UAEXPAEPBEI@Z 004381f0 f   yassl:crypto_wrapper.obj
 0001:00037200       ?decrypt@RC4@yaSSL@@UAEXPAEPBEI@Z 00438200 f   yassl:crypto_wrapper.obj
 0001:00037210       ??1?$BlockCipher@$0A@VAES@TaoCrypt@@$00@TaoCrypt@@QAE@XZ 00438210 f i yassl:crypto_wrapper.obj
 0001:00037220       ??1?$BlockCipher@$00VAES@TaoCrypt@@$00@TaoCrypt@@QAE@XZ 00438220 f i yassl:crypto_wrapper.obj
 0001:00037230       ?get_keySize@AES@yaSSL@@UBEHXZ 00438230 f   yassl:crypto_wrapper.obj
 0001:00037240       ??0RandomImpl@RandomPool@yaSSL@@QAE@XZ 00438240 f i yassl:crypto_wrapper.obj
 0001:00037250       ?GetError@RandomPool@yaSSL@@QBEHXZ 00438250 f   yassl:crypto_wrapper.obj
 0001:00037260       ?Fill@RandomPool@yaSSL@@QBEXPAEI@Z 00438260 f   yassl:crypto_wrapper.obj
 0001:00037270       ??0Auth@yaSSL@@QAE@XZ      00438270 f i yassl:crypto_wrapper.obj
 0001:00037280       ?get_signatureLength@DSS@yaSSL@@UBEIXZ 00438280 f   yassl:crypto_wrapper.obj
 0001:00037290       ?get_cipherLength@RSA@yaSSL@@QBEIXZ 00438290 f   yassl:crypto_wrapper.obj
 0001:000372a0       ?get_signatureLength@RSA@yaSSL@@UBEIXZ 004382a0 f   yassl:crypto_wrapper.obj
 0001:000372b0       ??4Integer@yaSSL@@QAEAAV01@ABV01@@Z 004382b0 f   yassl:crypto_wrapper.obj
 0001:000372d0       ?AllocKeys@DHImpl@DiffieHellman@yaSSL@@QAEXIII@Z 004382d0 f i yassl:crypto_wrapper.obj
 0001:00037310       ?makeAgreement@DiffieHellman@yaSSL@@QAEXPBEI@Z 00438310 f   yassl:crypto_wrapper.obj
 0001:00037330       ?get_agreedKeyLength@DiffieHellman@yaSSL@@QBEIXZ 00438330 f   yassl:crypto_wrapper.obj
 0001:00037340       ?get_agreedKey@DiffieHellman@yaSSL@@QBEPBEXZ 00438340 f   yassl:crypto_wrapper.obj
 0001:00037350       ?get_publicKey@DiffieHellman@yaSSL@@QBEPBEXZ 00438350 f   yassl:crypto_wrapper.obj
 0001:00037360       ??1?$Block@IV?$AlignedAllocator@I@TaoCrypt@@@TaoCrypt@@QAE@XZ 00438360 f i yassl:crypto_wrapper.obj
 0001:00037370       ??0?$BlockCipher@$0A@VDES@TaoCrypt@@$00@TaoCrypt@@QAE@XZ 00438370 f i yassl:crypto_wrapper.obj
 0001:000373a0       ?Process@?$BlockCipher@$0A@VDES@TaoCrypt@@$00@TaoCrypt@@QAEXPAEPBEI@Z 004383a0 f i yassl:crypto_wrapper.obj
 0001:000373b0       ?SetKey@?$BlockCipher@$0A@VDES@TaoCrypt@@$00@TaoCrypt@@QAEXPBEI0@Z 004383b0 f i yassl:crypto_wrapper.obj
 0001:000373e0       ??0?$BlockCipher@$00VDES@TaoCrypt@@$00@TaoCrypt@@QAE@XZ 004383e0 f i yassl:crypto_wrapper.obj
 0001:00037410       ?Process@?$BlockCipher@$00VDES@TaoCrypt@@$00@TaoCrypt@@QAEXPAEPBEI@Z 00438410 f i yassl:crypto_wrapper.obj
 0001:00037420       ?SetKey@?$BlockCipher@$00VDES@TaoCrypt@@$00@TaoCrypt@@QAEXPBEI0@Z 00438420 f i yassl:crypto_wrapper.obj
 0001:00037450       ??0?$BlockCipher@$0A@VDES_EDE3@TaoCrypt@@$00@TaoCrypt@@QAE@XZ 00438450 f i yassl:crypto_wrapper.obj
 0001:00037480       ?Process@?$BlockCipher@$0A@VDES_EDE3@TaoCrypt@@$00@TaoCrypt@@QAEXPAEPBEI@Z 00438480 f i yassl:crypto_wrapper.obj
 0001:00037490       ?SetKey@?$BlockCipher@$0A@VDES_EDE3@TaoCrypt@@$00@TaoCrypt@@QAEXPBEI0@Z 00438490 f i yassl:crypto_wrapper.obj
 0001:000374c0       ??0?$BlockCipher@$00VDES_EDE3@TaoCrypt@@$00@TaoCrypt@@QAE@XZ 004384c0 f i yassl:crypto_wrapper.obj
 0001:000374f0       ?Process@?$BlockCipher@$00VDES_EDE3@TaoCrypt@@$00@TaoCrypt@@QAEXPAEPBEI@Z 004384f0 f i yassl:crypto_wrapper.obj
 0001:00037500       ?SetKey@?$BlockCipher@$00VDES_EDE3@TaoCrypt@@$00@TaoCrypt@@QAEXPBEI0@Z 00438500 f i yassl:crypto_wrapper.obj
 0001:00037530       ??0?$BlockCipher@$0A@VAES@TaoCrypt@@$00@TaoCrypt@@QAE@XZ 00438530 f i yassl:crypto_wrapper.obj
 0001:00037560       ?Process@?$BlockCipher@$0A@VAES@TaoCrypt@@$00@TaoCrypt@@QAEXPAEPBEI@Z 00438560 f i yassl:crypto_wrapper.obj
 0001:00037570       ?SetKey@?$BlockCipher@$0A@VAES@TaoCrypt@@$00@TaoCrypt@@QAEXPBEI0@Z 00438570 f i yassl:crypto_wrapper.obj
 0001:000375b0       ??0?$BlockCipher@$00VAES@TaoCrypt@@$00@TaoCrypt@@QAE@XZ 004385b0 f i yassl:crypto_wrapper.obj
 0001:000375e0       ?Process@?$BlockCipher@$00VAES@TaoCrypt@@$00@TaoCrypt@@QAEXPAEPBEI@Z 004385e0 f i yassl:crypto_wrapper.obj
 0001:000375f0       ?SetKey@?$BlockCipher@$00VAES@TaoCrypt@@$00@TaoCrypt@@QAEXPBEI0@Z 004385f0 f i yassl:crypto_wrapper.obj
 0001:00037630       ??0?$RSA_Decryptor@VRSA_BlockType2@TaoCrypt@@@TaoCrypt@@QAE@ABVRSA_PrivateKey@1@@Z 00438630 f i yassl:crypto_wrapper.obj
 0001:00037640       ??0?$RSA_Encryptor@VRSA_BlockType2@TaoCrypt@@@TaoCrypt@@QAE@ABVRSA_PublicKey@1@@Z 00438640 f i yassl:crypto_wrapper.obj
 0001:00037650       ??$SaturatingSubtract@II@TaoCrypt@@YAIII@Z 00438650 f i yassl:crypto_wrapper.obj
 0001:00037670       ?Init@?$HMAC@VMD5@TaoCrypt@@@TaoCrypt@@QAEXXZ 00438670 f i yassl:crypto_wrapper.obj
 0001:00037690       ?SetKey@?$HMAC@VMD5@TaoCrypt@@@TaoCrypt@@QAEXPBEI@Z 00438690 f i yassl:crypto_wrapper.obj
 0001:00037770       ?Init@?$HMAC@VSHA@TaoCrypt@@@TaoCrypt@@QAEXXZ 00438770 f i yassl:crypto_wrapper.obj
 0001:00037790       ?SetKey@?$HMAC@VSHA@TaoCrypt@@@TaoCrypt@@QAEXPBEI@Z 00438790 f i yassl:crypto_wrapper.obj
 0001:00037870       ?Init@?$HMAC@VRIPEMD160@TaoCrypt@@@TaoCrypt@@QAEXXZ 00438870 f i yassl:crypto_wrapper.obj
 0001:00037890       ?SetKey@?$HMAC@VRIPEMD160@TaoCrypt@@@TaoCrypt@@QAEXPBEI@Z 00438890 f i yassl:crypto_wrapper.obj
 0001:00037970       ??$ysDelete@URC4Impl@RC4@yaSSL@@@yaSSL@@YAXPAURC4Impl@RC4@0@@Z 00438970 f i yassl:crypto_wrapper.obj
 0001:00037980       ??1MD5Impl@MD5@yaSSL@@QAE@XZ 00438980 f i yassl:crypto_wrapper.obj
 0001:00037990       ??1SHAImpl@SHA@yaSSL@@QAE@XZ 00438990 f i yassl:crypto_wrapper.obj
 0001:000379a0       ??1RMDImpl@RMD@yaSSL@@QAE@XZ 004389a0 f i yassl:crypto_wrapper.obj
 0001:000379b0       ??1HMAC_MD5Impl@HMAC_MD5@yaSSL@@QAE@XZ 004389b0 f i yassl:crypto_wrapper.obj
 0001:000379c0       ??1HMAC_SHAImpl@HMAC_SHA@yaSSL@@QAE@XZ 004389c0 f i yassl:crypto_wrapper.obj
 0001:000379d0       ??1HMAC_RMDImpl@HMAC_RMD@yaSSL@@QAE@XZ 004389d0 f i yassl:crypto_wrapper.obj
 0001:000379e0       ??1DESImpl@DES@yaSSL@@QAE@XZ 004389e0 f i yassl:crypto_wrapper.obj
 0001:00037a00       ??1DES_EDEImpl@DES_EDE@yaSSL@@QAE@XZ 00438a00 f i yassl:crypto_wrapper.obj
 0001:00037a20       ??1AESImpl@AES@yaSSL@@QAE@XZ 00438a20 f i yassl:crypto_wrapper.obj
 0001:00037a40       ??1RandomImpl@RandomPool@yaSSL@@QAE@XZ 00438a40 f i yassl:crypto_wrapper.obj
 0001:00037a50       ??0?$RSA_Encryptor@VRSA_BlockType1@TaoCrypt@@@TaoCrypt@@QAE@ABVRSA_PublicKey@1@@Z 00438a50 f i yassl:crypto_wrapper.obj
 0001:00037a60       ?KeyInnerHash@?$HMAC@VMD5@TaoCrypt@@@TaoCrypt@@AAEXXZ 00438a60 f i yassl:crypto_wrapper.obj
 0001:00037a80       ?KeyInnerHash@?$HMAC@VSHA@TaoCrypt@@@TaoCrypt@@AAEXXZ 00438a80 f i yassl:crypto_wrapper.obj
 0001:00037aa0       ?KeyInnerHash@?$HMAC@VRIPEMD160@TaoCrypt@@@TaoCrypt@@AAEXXZ 00438aa0 f i yassl:crypto_wrapper.obj
 0001:00037ac0       ??_GSHA@TaoCrypt@@UAEPAXI@Z 00438ac0 f i yassl:crypto_wrapper.obj
 0001:00037ac0       ??_ESHA@TaoCrypt@@UAEPAXI@Z 00438ac0 f i yassl:crypto_wrapper.obj
 0001:00037ae0       ??_ERIPEMD160@TaoCrypt@@UAEPAXI@Z 00438ae0 f i yassl:crypto_wrapper.obj
 0001:00037ae0       ??_GRIPEMD160@TaoCrypt@@UAEPAXI@Z 00438ae0 f i yassl:crypto_wrapper.obj
 0001:00037b00       ?Process@Mode_BASE@TaoCrypt@@UAEXPAEPBEI@Z 00438b00 f i yassl:crypto_wrapper.obj
 0001:00037b30       ??_EDES@TaoCrypt@@UAEPAXI@Z 00438b30 f i yassl:crypto_wrapper.obj
 0001:00037b30       ??_GDES@TaoCrypt@@UAEPAXI@Z 00438b30 f i yassl:crypto_wrapper.obj
 0001:00037b50       ??_EDES_EDE3@TaoCrypt@@UAEPAXI@Z 00438b50 f i yassl:crypto_wrapper.obj
 0001:00037b50       ??_GDES_EDE3@TaoCrypt@@UAEPAXI@Z 00438b50 f i yassl:crypto_wrapper.obj
 0001:00037b70       ??_GAES@TaoCrypt@@UAEPAXI@Z 00438b70 f i yassl:crypto_wrapper.obj
 0001:00037b70       ??_EAES@TaoCrypt@@UAEPAXI@Z 00438b70 f i yassl:crypto_wrapper.obj
 0001:00037b90       ??1Integer@TaoCrypt@@QAE@XZ 00438b90 f i yassl:crypto_wrapper.obj
 0001:00037ba0       ?FixedMaxPlaintextLength@PK_Lengths@TaoCrypt@@QBEIXZ 00438ba0 f i yassl:crypto_wrapper.obj
 0001:00037bc0       ??0RSA_PublicKey@TaoCrypt@@QAE@XZ 00438bc0 f i yassl:crypto_wrapper.obj
 0001:00037be0       ??0RSA_PublicKey@TaoCrypt@@QAE@ABV01@@Z 00438be0 f i yassl:crypto_wrapper.obj
 0001:00037c10       ??1RSA_PublicKey@TaoCrypt@@QAE@XZ 00438c10 f i yassl:crypto_wrapper.obj
 0001:00037c40       ??0RSA_PrivateKey@TaoCrypt@@QAE@XZ 00438c40 f i yassl:crypto_wrapper.obj
 0001:00037c90       ??0DSA_PublicKey@TaoCrypt@@QAE@XZ 00438c90 f i yassl:crypto_wrapper.obj
 0001:00037cc0       ??1DSA_PublicKey@TaoCrypt@@QAE@XZ 00438cc0 f i yassl:crypto_wrapper.obj
 0001:00037d10       ??0DH@TaoCrypt@@QAE@XZ     00438d10 f i yassl:crypto_wrapper.obj
 0001:00037d30       ??0DH@TaoCrypt@@QAE@ABV01@@Z 00438d30 f i yassl:crypto_wrapper.obj
 0001:00037d60       ?Initialize@DH@TaoCrypt@@QAEXAAVInteger@2@0@Z 00438d60 f i yassl:crypto_wrapper.obj
 0001:00037d80       ??1DH@TaoCrypt@@QAE@XZ     00438d80 f i yassl:crypto_wrapper.obj
 0001:00037db0       ??0MD5@yaSSL@@QAE@XZ       00438db0 f   yassl:crypto_wrapper.obj
 0001:00037e00       ??0DESImpl@DES@yaSSL@@QAE@XZ 00438e00 f i yassl:crypto_wrapper.obj
 0001:00037e60       ?set_encryptKey@DES@yaSSL@@UAEXPBE0@Z 00438e60 f   yassl:crypto_wrapper.obj
 0001:00037e90       ?set_decryptKey@DES@yaSSL@@UAEXPBE0@Z 00438e90 f   yassl:crypto_wrapper.obj
 0001:00037ed0       ?encrypt@DES@yaSSL@@UAEXPAEPBEI@Z 00438ed0 f   yassl:crypto_wrapper.obj
 0001:00037ee0       ?decrypt@DES@yaSSL@@UAEXPAEPBEI@Z 00438ee0 f   yassl:crypto_wrapper.obj
 0001:00037f00       ??0DES_EDEImpl@DES_EDE@yaSSL@@QAE@XZ 00438f00 f i yassl:crypto_wrapper.obj
 0001:00037f60       ?set_encryptKey@DES_EDE@yaSSL@@UAEXPBE0@Z 00438f60 f   yassl:crypto_wrapper.obj
 0001:00037f90       ?set_decryptKey@DES_EDE@yaSSL@@UAEXPBE0@Z 00438f90 f   yassl:crypto_wrapper.obj
 0001:00037fc0       ?encrypt@DES_EDE@yaSSL@@UAEXPAEPBEI@Z 00438fc0 f   yassl:crypto_wrapper.obj
 0001:00037fd0       ?decrypt@DES_EDE@yaSSL@@UAEXPAEPBEI@Z 00438fd0 f   yassl:crypto_wrapper.obj
 0001:00037ff0       ??0RC4@yaSSL@@QAE@XZ       00438ff0 f   yassl:crypto_wrapper.obj
 0001:00038010       ?get_blockSize@RC4@yaSSL@@UBEIXZ 00439010 f i yassl:crypto_wrapper.obj
 0001:00038020       ?get_keySize@RC4@yaSSL@@UBEHXZ 00439020 f i yassl:crypto_wrapper.obj
 0001:00038030       ?get_ivSize@RC4@yaSSL@@UBEHXZ 00439030 f i yassl:crypto_wrapper.obj
 0001:00038040       ??1RC4@yaSSL@@UAE@XZ       00439040 f   yassl:crypto_wrapper.obj
 0001:00038060       ??0AESImpl@AES@yaSSL@@QAE@I@Z 00439060 f i yassl:crypto_wrapper.obj
 0001:000380d0       ??0AES@yaSSL@@QAE@I@Z      004390d0 f   yassl:crypto_wrapper.obj
 0001:00038110       ?get_blockSize@AES@yaSSL@@UBEIXZ 00439110 f i yassl:crypto_wrapper.obj
 0001:00038120       ?get_ivSize@AES@yaSSL@@UBEHXZ 00439120 f i yassl:crypto_wrapper.obj
 0001:00038130       ?set_encryptKey@AES@yaSSL@@UAEXPBE0@Z 00439130 f   yassl:crypto_wrapper.obj
 0001:00038170       ?set_decryptKey@AES@yaSSL@@UAEXPBE0@Z 00439170 f   yassl:crypto_wrapper.obj
 0001:000381b0       ?encrypt@AES@yaSSL@@UAEXPAEPBEI@Z 004391b0 f   yassl:crypto_wrapper.obj
 0001:000381c0       ?decrypt@AES@yaSSL@@UAEXPAEPBEI@Z 004391c0 f   yassl:crypto_wrapper.obj
 0001:000381e0       ??0RandomPool@yaSSL@@QAE@XZ 004391e0 f   yassl:crypto_wrapper.obj
 0001:00038210       ??1DSA_PrivateKey@TaoCrypt@@QAE@XZ 00439210 f i yassl:crypto_wrapper.obj
 0001:00038270       ??1DSA_Signer@TaoCrypt@@QAE@XZ 00439270 f i yassl:crypto_wrapper.obj
 0001:000382a0       ??1DSA_Verifier@TaoCrypt@@QAE@XZ 004392a0 f i yassl:crypto_wrapper.obj
 0001:000382d0       ??1RSA_PrivateKey@TaoCrypt@@QAE@XZ 004392d0 f i yassl:crypto_wrapper.obj
 0001:00038360       ??0IntegerImpl@Integer@yaSSL@@QAE@XZ 00439360 f i yassl:crypto_wrapper.obj
 0001:00038370       ??0IntegerImpl@Integer@yaSSL@@QAE@ABV1TaoCrypt@@@Z 00439370 f i yassl:crypto_wrapper.obj
 0001:00038390       ??0Integer@yaSSL@@QAE@XZ   00439390 f   yassl:crypto_wrapper.obj
 0001:000383c0       ??0Integer@yaSSL@@QAE@ABV01@@Z 004393c0 f   yassl:crypto_wrapper.obj
 0001:00038400       ?assign@Integer@yaSSL@@QAEXPBEI@Z 00439400 f   yassl:crypto_wrapper.obj
 0001:00038440       ??0DHImpl@DiffieHellman@yaSSL@@QAE@AAVRandomNumberGenerator@TaoCrypt@@@Z 00439440 f i yassl:crypto_wrapper.obj
 0001:00038470       ??1DHImpl@DiffieHellman@yaSSL@@QAE@XZ 00439470 f i yassl:crypto_wrapper.obj
 0001:000384c0       ??0DHImpl@DiffieHellman@yaSSL@@QAE@ABU012@@Z 004394c0 f i yassl:crypto_wrapper.obj
 0001:00038520       ??0DiffieHellman@yaSSL@@QAE@PBEI0I0IABVRandomPool@1@@Z 00439520 f   yassl:crypto_wrapper.obj
 0001:00038600       ??0DiffieHellman@yaSSL@@QAE@ABVInteger@1@0ABVRandomPool@1@@Z 00439600 f   yassl:crypto_wrapper.obj
 0001:000386b0       ??0DiffieHellman@yaSSL@@QAE@ABV01@@Z 004396b0 f   yassl:crypto_wrapper.obj
 0001:000386f0       ?set_sizes@DiffieHellman@yaSSL@@QBEXAAH00@Z 004396f0 f   yassl:crypto_wrapper.obj
 0001:00038770       ?get_parms@DiffieHellman@yaSSL@@QBEXPAE00@Z 00439770 f   yassl:crypto_wrapper.obj
 0001:00038810       ??0?$HMAC@VMD5@TaoCrypt@@@TaoCrypt@@QAE@XZ 00439810 f i yassl:crypto_wrapper.obj
 0001:00038860       ??0?$HMAC@VSHA@TaoCrypt@@@TaoCrypt@@QAE@XZ 00439860 f i yassl:crypto_wrapper.obj
 0001:000388b0       ??0?$HMAC@VRIPEMD160@TaoCrypt@@@TaoCrypt@@QAE@XZ 004398b0 f i yassl:crypto_wrapper.obj
 0001:00038900       ?Update@?$HMAC@VMD5@TaoCrypt@@@TaoCrypt@@QAEXPBEI@Z 00439900 f i yassl:crypto_wrapper.obj
 0001:00038920       ?Final@?$HMAC@VMD5@TaoCrypt@@@TaoCrypt@@QAEXPAE@Z 00439920 f i yassl:crypto_wrapper.obj
 0001:00038980       ?Update@?$HMAC@VSHA@TaoCrypt@@@TaoCrypt@@QAEXPBEI@Z 00439980 f i yassl:crypto_wrapper.obj
 0001:000389a0       ?Final@?$HMAC@VSHA@TaoCrypt@@@TaoCrypt@@QAEXPAE@Z 004399a0 f i yassl:crypto_wrapper.obj
 0001:00038a00       ?Update@?$HMAC@VRIPEMD160@TaoCrypt@@@TaoCrypt@@QAEXPBEI@Z 00439a00 f i yassl:crypto_wrapper.obj
 0001:00038a20       ?Final@?$HMAC@VRIPEMD160@TaoCrypt@@@TaoCrypt@@QAEXPAE@Z 00439a20 f i yassl:crypto_wrapper.obj
 0001:00038a80       ??_GMD5Impl@MD5@yaSSL@@QAEPAXI@Z 00439a80 f i yassl:crypto_wrapper.obj
 0001:00038aa0       ??_GSHAImpl@SHA@yaSSL@@QAEPAXI@Z 00439aa0 f i yassl:crypto_wrapper.obj
 0001:00038ac0       ??_GRMDImpl@RMD@yaSSL@@QAEPAXI@Z 00439ac0 f i yassl:crypto_wrapper.obj
 0001:00038ae0       ??_GHMAC_MD5Impl@HMAC_MD5@yaSSL@@QAEPAXI@Z 00439ae0 f i yassl:crypto_wrapper.obj
 0001:00038b00       ??_GHMAC_SHAImpl@HMAC_SHA@yaSSL@@QAEPAXI@Z 00439b00 f i yassl:crypto_wrapper.obj
 0001:00038b20       ??_GHMAC_RMDImpl@HMAC_RMD@yaSSL@@QAEPAXI@Z 00439b20 f i yassl:crypto_wrapper.obj
 0001:00038b40       ??_GDESImpl@DES@yaSSL@@QAEPAXI@Z 00439b40 f i yassl:crypto_wrapper.obj
 0001:00038b70       ??_GDES_EDEImpl@DES_EDE@yaSSL@@QAEPAXI@Z 00439b70 f i yassl:crypto_wrapper.obj
 0001:00038ba0       ??_GAESImpl@AES@yaSSL@@QAEPAXI@Z 00439ba0 f i yassl:crypto_wrapper.obj
 0001:00038bd0       ??_GRandomImpl@RandomPool@yaSSL@@QAEPAXI@Z 00439bd0 f i yassl:crypto_wrapper.obj
 0001:00038bf0       ??_GDHImpl@DiffieHellman@yaSSL@@QAEPAXI@Z 00439bf0 f i yassl:crypto_wrapper.obj
 0001:00038c50       ??1DSSImpl@DSS@yaSSL@@QAE@XZ 00439c50 f i yassl:crypto_wrapper.obj
 0001:00038ca0       ??1RSAImpl@RSA@yaSSL@@QAE@XZ 00439ca0 f i yassl:crypto_wrapper.obj
 0001:00038cd0       ??1IntegerImpl@Integer@yaSSL@@QAE@XZ 00439cd0 f i yassl:crypto_wrapper.obj
 0001:00038ce0       ??4RSA_PublicKey@TaoCrypt@@QAEAAV01@ABV01@@Z 00439ce0 f i yassl:crypto_wrapper.obj
 0001:00038d50       ??0DSA_PrivateKey@TaoCrypt@@QAE@XZ 00439d50 f i yassl:crypto_wrapper.obj
 0001:00038d80       ??4DH@TaoCrypt@@QAEAAV01@ABV01@@Z 00439d80 f i yassl:crypto_wrapper.obj
 0001:00038df0       ??0HMAC_MD5Impl@HMAC_MD5@yaSSL@@QAE@XZ 00439df0 f i yassl:crypto_wrapper.obj
 0001:00038e40       ??0HMAC_MD5@yaSSL@@QAE@PBEI@Z 00439e40 f   yassl:crypto_wrapper.obj
 0001:00038e80       ?get_digest@HMAC_MD5@yaSSL@@UAEXPAEPBEI@Z 00439e80 f   yassl:crypto_wrapper.obj
 0001:00038eb0       ?get_digest@HMAC_MD5@yaSSL@@UAEXPAE@Z 00439eb0 f   yassl:crypto_wrapper.obj
 0001:00038ec0       ?update@HMAC_MD5@yaSSL@@UAEXPBEI@Z 00439ec0 f   yassl:crypto_wrapper.obj
 0001:00038ed0       ??0HMAC_SHAImpl@HMAC_SHA@yaSSL@@QAE@XZ 00439ed0 f i yassl:crypto_wrapper.obj
 0001:00038f20       ??0HMAC_SHA@yaSSL@@QAE@PBEI@Z 00439f20 f   yassl:crypto_wrapper.obj
 0001:00038f60       ?get_digest@HMAC_SHA@yaSSL@@UAEXPAEPBEI@Z 00439f60 f   yassl:crypto_wrapper.obj
 0001:00038f90       ?get_digest@HMAC_SHA@yaSSL@@UAEXPAE@Z 00439f90 f   yassl:crypto_wrapper.obj
 0001:00038fa0       ?update@HMAC_SHA@yaSSL@@UAEXPBEI@Z 00439fa0 f   yassl:crypto_wrapper.obj
 0001:00038fb0       ??0HMAC_RMDImpl@HMAC_RMD@yaSSL@@QAE@XZ 00439fb0 f i yassl:crypto_wrapper.obj
 0001:00039000       ??0HMAC_RMD@yaSSL@@QAE@PBEI@Z 0043a000 f   yassl:crypto_wrapper.obj
 0001:00039040       ?get_digest@HMAC_RMD@yaSSL@@UAEXPAEPBEI@Z 0043a040 f   yassl:crypto_wrapper.obj
 0001:00039070       ?get_digest@HMAC_RMD@yaSSL@@UAEXPAE@Z 0043a070 f   yassl:crypto_wrapper.obj
 0001:00039080       ?update@HMAC_RMD@yaSSL@@UAEXPBEI@Z 0043a080 f   yassl:crypto_wrapper.obj
 0001:00039090       ??0DES@yaSSL@@QAE@XZ       0043a090 f   yassl:crypto_wrapper.obj
 0001:000390d0       ?get_blockSize@DES@yaSSL@@UBEIXZ 0043a0d0 f i yassl:crypto_wrapper.obj
 0001:000390e0       ?get_keySize@DES@yaSSL@@UBEHXZ 0043a0e0 f i yassl:crypto_wrapper.obj
 0001:000390f0       ?get_ivSize@DES@yaSSL@@UBEHXZ 0043a0f0 f i yassl:crypto_wrapper.obj
 0001:00039100       ??0DES_EDE@yaSSL@@QAE@XZ   0043a100 f   yassl:crypto_wrapper.obj
 0001:00039140       ?get_blockSize@DES_EDE@yaSSL@@UBEIXZ 0043a140 f i yassl:crypto_wrapper.obj
 0001:00039150       ?get_keySize@DES_EDE@yaSSL@@UBEHXZ 0043a150 f i yassl:crypto_wrapper.obj
 0001:00039160       ?get_ivSize@DES_EDE@yaSSL@@UBEHXZ 0043a160 f i yassl:crypto_wrapper.obj
 0001:00039170       ??_ERC4@yaSSL@@UAEPAXI@Z   0043a170 f i yassl:crypto_wrapper.obj
 0001:00039170       ??_GRC4@yaSSL@@UAEPAXI@Z   0043a170 f i yassl:crypto_wrapper.obj
 0001:00039190       ??0DSSImpl@DSS@yaSSL@@QAE@XZ 0043a190 f i yassl:crypto_wrapper.obj
 0001:000391e0       ?sign@DSS@yaSSL@@UAEXPAEPBEIABVRandomPool@2@@Z 0043a1e0 f   yassl:crypto_wrapper.obj
 0001:00039240       ?verify@DSS@yaSSL@@UAE_NPBEI0I@Z 0043a240 f   yassl:crypto_wrapper.obj
 0001:000392a0       ??0RSAImpl@RSA@yaSSL@@QAE@XZ 0043a2a0 f i yassl:crypto_wrapper.obj
 0001:00039300       ??4DiffieHellman@yaSSL@@QAEAAV01@ABV01@@Z 0043a300 f   yassl:crypto_wrapper.obj
 0001:00039330       ??$ysDelete@UMD5Impl@MD5@yaSSL@@@yaSSL@@YAXPAUMD5Impl@MD5@0@@Z 0043a330 f i yassl:crypto_wrapper.obj
 0001:00039350       ??$ysDelete@USHAImpl@SHA@yaSSL@@@yaSSL@@YAXPAUSHAImpl@SHA@0@@Z 0043a350 f i yassl:crypto_wrapper.obj
 0001:00039370       ??$ysDelete@URMDImpl@RMD@yaSSL@@@yaSSL@@YAXPAURMDImpl@RMD@0@@Z 0043a370 f i yassl:crypto_wrapper.obj
 0001:00039390       ??$ysDelete@UHMAC_MD5Impl@HMAC_MD5@yaSSL@@@yaSSL@@YAXPAUHMAC_MD5Impl@HMAC_MD5@0@@Z 0043a390 f i yassl:crypto_wrapper.obj
 0001:000393b0       ??$ysDelete@UHMAC_SHAImpl@HMAC_SHA@yaSSL@@@yaSSL@@YAXPAUHMAC_SHAImpl@HMAC_SHA@0@@Z 0043a3b0 f i yassl:crypto_wrapper.obj
 0001:000393d0       ??$ysDelete@UHMAC_RMDImpl@HMAC_RMD@yaSSL@@@yaSSL@@YAXPAUHMAC_RMDImpl@HMAC_RMD@0@@Z 0043a3d0 f i yassl:crypto_wrapper.obj
 0001:000393f0       ??$ysDelete@UDESImpl@DES@yaSSL@@@yaSSL@@YAXPAUDESImpl@DES@0@@Z 0043a3f0 f i yassl:crypto_wrapper.obj
 0001:00039420       ??$ysDelete@UDES_EDEImpl@DES_EDE@yaSSL@@@yaSSL@@YAXPAUDES_EDEImpl@DES_EDE@0@@Z 0043a420 f i yassl:crypto_wrapper.obj
 0001:00039450       ??$ysDelete@UAESImpl@AES@yaSSL@@@yaSSL@@YAXPAUAESImpl@AES@0@@Z 0043a450 f i yassl:crypto_wrapper.obj
 0001:00039480       ??$ysDelete@URandomImpl@RandomPool@yaSSL@@@yaSSL@@YAXPAURandomImpl@RandomPool@0@@Z 0043a480 f i yassl:crypto_wrapper.obj
 0001:000394a0       ??$ysDelete@UDHImpl@DiffieHellman@yaSSL@@@yaSSL@@YAXPAUDHImpl@DiffieHellman@0@@Z 0043a4a0 f i yassl:crypto_wrapper.obj
 0001:00039500       ??_GDSSImpl@DSS@yaSSL@@QAEPAXI@Z 0043a500 f i yassl:crypto_wrapper.obj
 0001:00039560       ??_GRSAImpl@RSA@yaSSL@@QAEPAXI@Z 0043a560 f i yassl:crypto_wrapper.obj
 0001:000395a0       ??_GIntegerImpl@Integer@yaSSL@@QAEPAXI@Z 0043a5a0 f i yassl:crypto_wrapper.obj
 0001:000395d0       ??1MD5@yaSSL@@UAE@XZ       0043a5d0 f   yassl:crypto_wrapper.obj
 0001:000395f0       ??1SHA@yaSSL@@UAE@XZ       0043a5f0 f   yassl:crypto_wrapper.obj
 0001:00039610       ??1RMD@yaSSL@@UAE@XZ       0043a610 f   yassl:crypto_wrapper.obj
 0001:00039630       ??1HMAC_MD5@yaSSL@@UAE@XZ  0043a630 f   yassl:crypto_wrapper.obj
 0001:00039650       ??1HMAC_SHA@yaSSL@@UAE@XZ  0043a650 f   yassl:crypto_wrapper.obj
 0001:00039670       ??1HMAC_RMD@yaSSL@@UAE@XZ  0043a670 f   yassl:crypto_wrapper.obj
 0001:00039690       ??1DES@yaSSL@@UAE@XZ       0043a690 f   yassl:crypto_wrapper.obj
 0001:000396b0       ??1DES_EDE@yaSSL@@UAE@XZ   0043a6b0 f   yassl:crypto_wrapper.obj
 0001:000396d0       ??1AES@yaSSL@@UAE@XZ       0043a6d0 f   yassl:crypto_wrapper.obj
 0001:000396f0       ??1RandomPool@yaSSL@@QAE@XZ 0043a6f0 f   yassl:crypto_wrapper.obj
 0001:00039700       ?SetPublic@DSSImpl@DSS@yaSSL@@QAEXPBEI@Z 0043a700 f   yassl:crypto_wrapper.obj
 0001:00039780       ?SetPrivate@DSSImpl@DSS@yaSSL@@QAEXPBEI@Z 0043a780 f   yassl:crypto_wrapper.obj
 0001:00039860       ??0DSS@yaSSL@@QAE@PBEI_N@Z 0043a860 f   yassl:crypto_wrapper.obj
 0001:000398c0       ?SetPublic@RSAImpl@RSA@yaSSL@@QAEXPBEI@Z 0043a8c0 f   yassl:crypto_wrapper.obj
 0001:00039940       ?SetPrivate@RSAImpl@RSA@yaSSL@@QAEXPBEI@Z 0043a940 f   yassl:crypto_wrapper.obj
 0001:00039a00       ??0RSA@yaSSL@@QAE@PBEI_N@Z 0043aa00 f   yassl:crypto_wrapper.obj
 0001:00039a60       ??1DiffieHellman@yaSSL@@QAE@XZ 0043aa60 f   yassl:crypto_wrapper.obj
 0001:00039a70       ??1Base64Decoder@TaoCrypt@@QAE@XZ 0043aa70 f i yassl:crypto_wrapper.obj
 0001:00039a90       ??$ysDelete@UDSSImpl@DSS@yaSSL@@@yaSSL@@YAXPAUDSSImpl@DSS@0@@Z 0043aa90 f i yassl:crypto_wrapper.obj
 0001:00039af0       ??$ysDelete@URSAImpl@RSA@yaSSL@@@yaSSL@@YAXPAURSAImpl@RSA@0@@Z 0043aaf0 f i yassl:crypto_wrapper.obj
 0001:00039b30       ??$ysDelete@UIntegerImpl@Integer@yaSSL@@@yaSSL@@YAXPAUIntegerImpl@Integer@0@@Z 0043ab30 f i yassl:crypto_wrapper.obj
 0001:00039b60       ??_GMD5@yaSSL@@UAEPAXI@Z   0043ab60 f i yassl:crypto_wrapper.obj
 0001:00039b60       ??_EMD5@yaSSL@@UAEPAXI@Z   0043ab60 f i yassl:crypto_wrapper.obj
 0001:00039b80       ??_ESHA@yaSSL@@UAEPAXI@Z   0043ab80 f i yassl:crypto_wrapper.obj
 0001:00039b80       ??_GSHA@yaSSL@@UAEPAXI@Z   0043ab80 f i yassl:crypto_wrapper.obj
 0001:00039ba0       ??_ERMD@yaSSL@@UAEPAXI@Z   0043aba0 f i yassl:crypto_wrapper.obj
 0001:00039ba0       ??_GRMD@yaSSL@@UAEPAXI@Z   0043aba0 f i yassl:crypto_wrapper.obj
 0001:00039bc0       ??_GHMAC_MD5@yaSSL@@UAEPAXI@Z 0043abc0 f i yassl:crypto_wrapper.obj
 0001:00039bc0       ??_EHMAC_MD5@yaSSL@@UAEPAXI@Z 0043abc0 f i yassl:crypto_wrapper.obj
 0001:00039be0       ??_GHMAC_SHA@yaSSL@@UAEPAXI@Z 0043abe0 f i yassl:crypto_wrapper.obj
 0001:00039be0       ??_EHMAC_SHA@yaSSL@@UAEPAXI@Z 0043abe0 f i yassl:crypto_wrapper.obj
 0001:00039c00       ??_GHMAC_RMD@yaSSL@@UAEPAXI@Z 0043ac00 f i yassl:crypto_wrapper.obj
 0001:00039c00       ??_EHMAC_RMD@yaSSL@@UAEPAXI@Z 0043ac00 f i yassl:crypto_wrapper.obj
 0001:00039c20       ??_EDES@yaSSL@@UAEPAXI@Z   0043ac20 f i yassl:crypto_wrapper.obj
 0001:00039c20       ??_GDES@yaSSL@@UAEPAXI@Z   0043ac20 f i yassl:crypto_wrapper.obj
 0001:00039c40       ??_GDES_EDE@yaSSL@@UAEPAXI@Z 0043ac40 f i yassl:crypto_wrapper.obj
 0001:00039c40       ??_EDES_EDE@yaSSL@@UAEPAXI@Z 0043ac40 f i yassl:crypto_wrapper.obj
 0001:00039c60       ??_GAES@yaSSL@@UAEPAXI@Z   0043ac60 f i yassl:crypto_wrapper.obj
 0001:00039c60       ??_EAES@yaSSL@@UAEPAXI@Z   0043ac60 f i yassl:crypto_wrapper.obj
 0001:00039c80       ??1DSS@yaSSL@@UAE@XZ       0043ac80 f   yassl:crypto_wrapper.obj
 0001:00039ca0       ??1RSA@yaSSL@@UAE@XZ       0043aca0 f   yassl:crypto_wrapper.obj
 0001:00039cc0       ??1Integer@yaSSL@@QAE@XZ   0043acc0 f   yassl:crypto_wrapper.obj
 0001:00039cd0       ?Decrypt@?$RSA_Decryptor@VRSA_BlockType2@TaoCrypt@@@TaoCrypt@@QAEIPBEIPAEAAVRandomNumberGenerator@2@@Z 0043acd0 f i yassl:crypto_wrapper.obj
 0001:00039df0       ?Encrypt@?$RSA_Encryptor@VRSA_BlockType2@TaoCrypt@@@TaoCrypt@@QAEXPBEIPAEAAVRandomNumberGenerator@2@@Z 0043adf0 f i yassl:crypto_wrapper.obj
 0001:00039ed0       ?SSL_Verify@?$RSA_Encryptor@VRSA_BlockType2@TaoCrypt@@@TaoCrypt@@QAE_NPBEI0@Z 0043aed0 f i yassl:crypto_wrapper.obj
 0001:0003a010       ?Encrypt@?$RSA_Encryptor@VRSA_BlockType1@TaoCrypt@@@TaoCrypt@@QAEXPBEIPAEAAVRandomNumberGenerator@2@@Z 0043b010 f i yassl:crypto_wrapper.obj
 0001:0003a0f0       ??0Base64Decoder@TaoCrypt@@QAE@AAVSource@1@@Z 0043b0f0 f i yassl:crypto_wrapper.obj
 0001:0003a140       ??_EDSS@yaSSL@@UAEPAXI@Z   0043b140 f i yassl:crypto_wrapper.obj
 0001:0003a140       ??_GDSS@yaSSL@@UAEPAXI@Z   0043b140 f i yassl:crypto_wrapper.obj
 0001:0003a160       ??_ERSA@yaSSL@@UAEPAXI@Z   0043b160 f i yassl:crypto_wrapper.obj
 0001:0003a160       ??_GRSA@yaSSL@@UAEPAXI@Z   0043b160 f i yassl:crypto_wrapper.obj
 0001:0003a180       ?verify@RSA@yaSSL@@UAE_NPBEI0I@Z 0043b180 f   yassl:crypto_wrapper.obj
 0001:0003a1b0       ?encrypt@RSA@yaSSL@@QAEXPAEPBEIABVRandomPool@2@@Z 0043b1b0 f   yassl:crypto_wrapper.obj
 0001:0003a1e0       ?decrypt@RSA@yaSSL@@QAEXPAEPBEIABVRandomPool@2@@Z 0043b1e0 f   yassl:crypto_wrapper.obj
 0001:0003a220       ?PemToDer@yaSSL@@YAPAVx509@1@PAU_iobuf@@W4CertType@1@PAUEncryptedInfo@1@@Z 0043b220 f   yassl:crypto_wrapper.obj
 0001:0003a5e0       ?SSL_Sign@?$RSA_Decryptor@VRSA_BlockType2@TaoCrypt@@@TaoCrypt@@QAEXPBEIPAEAAVRandomNumberGenerator@2@@Z 0043b5e0 f i yassl:crypto_wrapper.obj
 0001:0003a670       ?sign@RSA@yaSSL@@UAEXPAEPBEIABVRandomPool@2@@Z 0043b670 f   yassl:crypto_wrapper.obj
 0001:0003a6b0       ??0Message@yaSSL@@QAE@XZ   0043b6b0 f i yassl:yassl_imp.obj
 0001:0003a6c0       ??0HandShakeHeader@yaSSL@@QAE@XZ 0043b6c0 f i yassl:yassl_imp.obj
 0001:0003a6d0       ??1HandShakeHeader@yaSSL@@UAE@XZ 0043b6d0 f i yassl:yassl_imp.obj
 0001:0003a6e0       ??1ServerKeyBase@yaSSL@@UAE@XZ 0043b6e0 f i yassl:yassl_imp.obj
 0001:0003a6f0       ?build@ServerKeyBase@yaSSL@@UAEXAAVSSL@2@@Z 0043b6f0 f i yassl:yassl_imp.obj
 0001:0003a700       ?read@ServerKeyBase@yaSSL@@UAEXAAVSSL@2@AAVinput_buffer@2@@Z 0043b700 f i yassl:yassl_imp.obj
 0001:0003a710       ??_GServerKeyBase@yaSSL@@UAEPAXI@Z 0043b710 f i yassl:yassl_imp.obj
 0001:0003a710       ??_EServerKeyBase@yaSSL@@UAEPAXI@Z 0043b710 f i yassl:yassl_imp.obj
 0001:0003a730       ??1ClientKeyBase@yaSSL@@UAE@XZ 0043b730 f i yassl:yassl_imp.obj
 0001:0003a740       ?build@ClientKeyBase@yaSSL@@UAEXAAVSSL@2@@Z 0043b740 f i yassl:yassl_imp.obj
 0001:0003a750       ?read@ClientKeyBase@yaSSL@@UAEXAAVSSL@2@AAVinput_buffer@2@@Z 0043b750 f i yassl:yassl_imp.obj
 0001:0003a760       ??_GClientKeyBase@yaSSL@@UAEPAXI@Z 0043b760 f i yassl:yassl_imp.obj
 0001:0003a760       ??_EClientKeyBase@yaSSL@@UAEPAXI@Z 0043b760 f i yassl:yassl_imp.obj
 0001:0003a780       ?isTLS@?A0xea27e27a@yaSSL@@YA_NUProtocolVersion@2@@Z 0043b780 f   yassl:yassl_imp.obj
 0001:0003a7a0       ??0ProtocolVersion@yaSSL@@QAE@EE@Z 0043b7a0 f   yassl:yassl_imp.obj
 0001:0003a7c0       ??0ClientKeyBase@yaSSL@@QAE@XZ 0043b7c0 f i yassl:yassl_imp.obj
 0001:0003a7d0       ?get_length@EncryptedPreMasterSecret@yaSSL@@UBEHXZ 0043b7d0 f   yassl:yassl_imp.obj
 0001:0003a7e0       ?get_clientKey@EncryptedPreMasterSecret@yaSSL@@UBEPAEXZ 0043b7e0 f   yassl:yassl_imp.obj
 0001:0003a7f0       ?alloc@EncryptedPreMasterSecret@yaSSL@@QAEXH@Z 0043b7f0 f   yassl:yassl_imp.obj
 0001:0003a810       ??0ClientDiffieHellmanPublic@yaSSL@@QAE@XZ 0043b810 f   yassl:yassl_imp.obj
 0001:0003a830       ?get_length@ClientDiffieHellmanPublic@yaSSL@@UBEHXZ 0043b830 f   yassl:yassl_imp.obj
 0001:0003a840       ?get_clientKey@ClientDiffieHellmanPublic@yaSSL@@UBEPAEXZ 0043b840 f   yassl:yassl_imp.obj
 0001:0003a850       ?alloc@ClientDiffieHellmanPublic@yaSSL@@QAEXH_N@Z 0043b850 f   yassl:yassl_imp.obj
 0001:0003a880       ??0ServerKeyBase@yaSSL@@QAE@XZ 0043b880 f i yassl:yassl_imp.obj
 0001:0003a890       ?get_length@DH_Server@yaSSL@@UBEHXZ 0043b890 f   yassl:yassl_imp.obj
 0001:0003a8a0       ?get_serverKey@DH_Server@yaSSL@@UBEPAEXZ 0043b8a0 f   yassl:yassl_imp.obj
 0001:0003a8b0       ?SetCipherNames@Parameters@yaSSL@@QAEXXZ 0043b8b0 f   yassl:yassl_imp.obj
 0001:0003a940       ??5yaSSL@@YAAAVinput_buffer@0@AAV10@AAURecordLayerHeader@0@@Z 0043b940 f   yassl:yassl_imp.obj
 0001:0003a9c0       ??6yaSSL@@YAAAVoutput_buffer@0@AAV10@ABURecordLayerHeader@0@@Z 0043b9c0 f   yassl:yassl_imp.obj
 0001:0003aa40       ??5yaSSL@@YAAAVinput_buffer@0@AAV10@AAUMessage@0@@Z 0043ba40 f   yassl:yassl_imp.obj
 0001:0003aa50       ??6yaSSL@@YAAAVoutput_buffer@0@AAV10@ABUMessage@0@@Z 0043ba50 f   yassl:yassl_imp.obj
 0001:0003aa70       ??5yaSSL@@YAAAVinput_buffer@0@AAV10@AAVHandShakeHeader@0@@Z 0043ba70 f   yassl:yassl_imp.obj
 0001:0003aad0       ??6yaSSL@@YAAAVoutput_buffer@0@AAV10@ABVHandShakeHeader@0@@Z 0043bad0 f   yassl:yassl_imp.obj
 0001:0003ab00       ?get_type@HandShakeHeader@yaSSL@@UBE?AW4ContentType@2@XZ 0043bb00 f   yassl:yassl_imp.obj
 0001:0003ab10       ?get_length@HandShakeHeader@yaSSL@@UBEGXZ 0043bb10 f   yassl:yassl_imp.obj
 0001:0003ab20       ?get_handshakeType@HandShakeHeader@yaSSL@@QBE?AW4HandShakeType@2@XZ 0043bb20 f   yassl:yassl_imp.obj
 0001:0003ab30       ?set_type@HandShakeHeader@yaSSL@@QAEXW4HandShakeType@2@@Z 0043bb30 f   yassl:yassl_imp.obj
 0001:0003ab40       ?set_length@HandShakeHeader@yaSSL@@QAEXI@Z 0043bb40 f   yassl:yassl_imp.obj
 0001:0003ab60       ?set@HandShakeHeader@yaSSL@@UAEAAVinput_buffer@2@AAV32@@Z 0043bb60 f   yassl:yassl_imp.obj
 0001:0003ab80       ?get@HandShakeHeader@yaSSL@@UBEAAVoutput_buffer@2@AAV32@@Z 0043bb80 f   yassl:yassl_imp.obj
 0001:0003aba0       ?get_length@HandShakeBase@yaSSL@@QBEHXZ 0043bba0 f   yassl:yassl_imp.obj
 0001:0003abb0       ?set_length@HandShakeBase@yaSSL@@QAEXH@Z 0043bbb0 f   yassl:yassl_imp.obj
 0001:0003abc0       ?get_type@HandShakeBase@yaSSL@@UBE?AW4HandShakeType@2@XZ 0043bbc0 f   yassl:yassl_imp.obj
 0001:0003abd0       ?set@HandShakeBase@yaSSL@@UAEAAVinput_buffer@2@AAV32@@Z 0043bbd0 f   yassl:yassl_imp.obj
 0001:0003abe0       ?get@HandShakeBase@yaSSL@@UBEAAVoutput_buffer@2@AAV32@@Z 0043bbe0 f   yassl:yassl_imp.obj
 0001:0003abf0       ?Process@HandShakeBase@yaSSL@@UAEXAAVinput_buffer@2@AAVSSL@2@@Z 0043bbf0 f   yassl:yassl_imp.obj
 0001:0003ac00       ?set@HelloRequest@yaSSL@@UAEAAVinput_buffer@2@AAV32@@Z 0043bc00 f   yassl:yassl_imp.obj
 0001:0003ac10       ?get@HelloRequest@yaSSL@@UBEAAVoutput_buffer@2@AAV32@@Z 0043bc10 f   yassl:yassl_imp.obj
 0001:0003ac20       ?Process@HelloRequest@yaSSL@@UAEXAAVinput_buffer@2@AAVSSL@2@@Z 0043bc20 f   yassl:yassl_imp.obj
 0001:0003ac30       ?get_type@HelloRequest@yaSSL@@UBE?AW4HandShakeType@2@XZ 0043bc30 f   yassl:yassl_imp.obj
 0001:0003ac40       ??5yaSSL@@YAAAVinput_buffer@0@AAV10@AAVChangeCipherSpec@0@@Z 0043bc40 f   yassl:yassl_imp.obj
 0001:0003ac60       ??6yaSSL@@YAAAVoutput_buffer@0@AAV10@ABVChangeCipherSpec@0@@Z 0043bc60 f   yassl:yassl_imp.obj
 0001:0003ac80       ??0ChangeCipherSpec@yaSSL@@QAE@XZ 0043bc80 f   yassl:yassl_imp.obj
 0001:0003ac90       ??1ChangeCipherSpec@yaSSL@@UAE@XZ 0043bc90 f i yassl:yassl_imp.obj
 0001:0003aca0       ?set@ChangeCipherSpec@yaSSL@@UAEAAVinput_buffer@2@AAV32@@Z 0043bca0 f   yassl:yassl_imp.obj
 0001:0003acc0       ?get@ChangeCipherSpec@yaSSL@@UBEAAVoutput_buffer@2@AAV32@@Z 0043bcc0 f   yassl:yassl_imp.obj
 0001:0003ace0       ?get_type@ChangeCipherSpec@yaSSL@@UBE?AW4ContentType@2@XZ 0043bce0 f   yassl:yassl_imp.obj
 0001:0003acf0       ?get_length@ChangeCipherSpec@yaSSL@@UBEGXZ 0043bcf0 f   yassl:yassl_imp.obj
 0001:0003ad00       ?Process@ChangeCipherSpec@yaSSL@@UAEXAAVinput_buffer@2@AAVSSL@2@@Z 0043bd00 f   yassl:yassl_imp.obj
 0001:0003ad80       ??0Alert@yaSSL@@QAE@W4AlertLevel@1@W4AlertDescription@1@@Z 0043bd80 f   yassl:yassl_imp.obj
 0001:0003ada0       ?get_type@Alert@yaSSL@@UBE?AW4ContentType@2@XZ 0043bda0 f   yassl:yassl_imp.obj
 0001:0003adb0       ?get_length@Alert@yaSSL@@UBEGXZ 0043bdb0 f   yassl:yassl_imp.obj
 0001:0003adc0       ??5yaSSL@@YAAAVinput_buffer@0@AAV10@AAVAlert@0@@Z 0043bdc0 f   yassl:yassl_imp.obj
 0001:0003ae00       ??6yaSSL@@YAAAVoutput_buffer@0@AAV10@ABVAlert@0@@Z 0043be00 f   yassl:yassl_imp.obj
 0001:0003ae40       ?Process@Alert@yaSSL@@UAEXAAVinput_buffer@2@AAVSSL@2@@Z 0043be40 f   yassl:yassl_imp.obj
 0001:0003b050       ??0Data@yaSSL@@QAE@XZ      0043c050 f   yassl:yassl_imp.obj
 0001:0003b070       ??0Data@yaSSL@@QAE@GPAE@Z  0043c070 f   yassl:yassl_imp.obj
 0001:0003b0a0       ?SetData@Data@yaSSL@@QAEXGPBE@Z 0043c0a0 f   yassl:yassl_imp.obj
 0001:0003b0c0       ?set@Data@yaSSL@@UAEAAVinput_buffer@2@AAV32@@Z 0043c0c0 f   yassl:yassl_imp.obj
 0001:0003b0d0       ?get_type@Data@yaSSL@@UBE?AW4ContentType@2@XZ 0043c0d0 f   yassl:yassl_imp.obj
 0001:0003b0e0       ?get_length@Data@yaSSL@@UBEGXZ 0043c0e0 f   yassl:yassl_imp.obj
 0001:0003b0f0       ?set_length@Data@yaSSL@@QAEXG@Z 0043c0f0 f   yassl:yassl_imp.obj
 0001:0003b100       ?set_buffer@Data@yaSSL@@QAEPAEXZ 0043c100 f   yassl:yassl_imp.obj
 0001:0003b110       ??6yaSSL@@YAAAVoutput_buffer@0@AAV10@ABVData@0@@Z 0043c110 f   yassl:yassl_imp.obj
 0001:0003b130       ?Process@Data@yaSSL@@UAEXAAVinput_buffer@2@AAVSSL@2@@Z 0043c130 f   yassl:yassl_imp.obj
 0001:0003b450       ??5yaSSL@@YAAAVinput_buffer@0@AAV10@AAVHandShakeBase@0@@Z 0043c450 f   yassl:yassl_imp.obj
 0001:0003b470       ??6yaSSL@@YAAAVoutput_buffer@0@AAV10@ABVHandShakeBase@0@@Z 0043c470 f   yassl:yassl_imp.obj
 0001:0003b490       ??0HandShakeBase@yaSSL@@QAE@XZ 0043c490 f i yassl:yassl_imp.obj
 0001:0003b4a0       ?get_buffer@Certificate@yaSSL@@QBEPBEXZ 0043c4a0 f   yassl:yassl_imp.obj
 0001:0003b4b0       ??6yaSSL@@YAAAVoutput_buffer@0@AAV10@ABVCertificate@0@@Z 0043c4b0 f   yassl:yassl_imp.obj
 0001:0003b520       ?Process@Certificate@yaSSL@@UAEXAAVinput_buffer@2@AAVSSL@2@@Z 0043c520 f   yassl:yassl_imp.obj
 0001:0003b670       ??0Certificate@yaSSL@@QAE@XZ 0043c670 f   yassl:yassl_imp.obj
 0001:0003b680       ??1Certificate@yaSSL@@UAE@XZ 0043c680 f i yassl:yassl_imp.obj
 0001:0003b690       ?set@Certificate@yaSSL@@UAEAAVinput_buffer@2@AAV32@@Z 0043c690 f   yassl:yassl_imp.obj
 0001:0003b6a0       ?get@Certificate@yaSSL@@UBEAAVoutput_buffer@2@AAV32@@Z 0043c6a0 f   yassl:yassl_imp.obj
 0001:0003b6c0       ?get_type@Certificate@yaSSL@@UBE?AW4HandShakeType@2@XZ 0043c6c0 f   yassl:yassl_imp.obj
 0001:0003b6d0       ??0ServerDHParams@yaSSL@@QAE@XZ 0043c6d0 f   yassl:yassl_imp.obj
 0001:0003b6f0       ?get_pSize@ServerDHParams@yaSSL@@QBEHXZ 0043c6f0 f   yassl:yassl_imp.obj
 0001:0003b700       ?get_gSize@ServerDHParams@yaSSL@@QBEHXZ 0043c700 f   yassl:yassl_imp.obj
 0001:0003b710       ?get_pubSize@ServerDHParams@yaSSL@@QBEHXZ 0043c710 f   yassl:yassl_imp.obj
 0001:0003b720       ?get_p@ServerDHParams@yaSSL@@QBEPBEXZ 0043c720 f   yassl:yassl_imp.obj
 0001:0003b730       ?get_g@ServerDHParams@yaSSL@@QBEPBEXZ 0043c730 f   yassl:yassl_imp.obj
 0001:0003b740       ?get_pub@ServerDHParams@yaSSL@@QBEPBEXZ 0043c740 f   yassl:yassl_imp.obj
 0001:0003b750       ?alloc_p@ServerDHParams@yaSSL@@QAEPAEH@Z 0043c750 f   yassl:yassl_imp.obj
 0001:0003b770       ?alloc_g@ServerDHParams@yaSSL@@QAEPAEH@Z 0043c770 f   yassl:yassl_imp.obj
 0001:0003b790       ?alloc_pub@ServerDHParams@yaSSL@@QAEPAEH@Z 0043c790 f   yassl:yassl_imp.obj
 0001:0003b7b0       ?get_length@ServerKeyBase@yaSSL@@UBEHXZ 0043c7b0 f   yassl:yassl_imp.obj
 0001:0003b7c0       ?get_serverKey@ServerKeyBase@yaSSL@@UBEPAEXZ 0043c7c0 f   yassl:yassl_imp.obj
 0001:0003b7d0       ??5yaSSL@@YAAAVinput_buffer@0@AAV10@AAVServerHello@0@@Z 0043c7d0 f   yassl:yassl_imp.obj
 0001:0003b870       ??6yaSSL@@YAAAVoutput_buffer@0@AAV10@ABVServerHello@0@@Z 0043c870 f   yassl:yassl_imp.obj
 0001:0003b910       ??0ServerHello@yaSSL@@QAE@XZ 0043c910 f   yassl:yassl_imp.obj
 0001:0003b960       ??1ServerHello@yaSSL@@UAE@XZ 0043c960 f i yassl:yassl_imp.obj
 0001:0003b970       ??0ServerHello@yaSSL@@QAE@UProtocolVersion@1@_N@Z 0043c970 f   yassl:yassl_imp.obj
 0001:0003b9d0       ?set@ServerHello@yaSSL@@UAEAAVinput_buffer@2@AAV32@@Z 0043c9d0 f   yassl:yassl_imp.obj
 0001:0003b9f0       ?get@ServerHello@yaSSL@@UBEAAVoutput_buffer@2@AAV32@@Z 0043c9f0 f   yassl:yassl_imp.obj
 0001:0003ba10       ?get_type@ServerHello@yaSSL@@UBE?AW4HandShakeType@2@XZ 0043ca10 f   yassl:yassl_imp.obj
 0001:0003ba20       ?get_random@ServerHello@yaSSL@@QBEPBEXZ 0043ca20 f   yassl:yassl_imp.obj
 0001:0003ba30       ?Process@ServerHelloDone@yaSSL@@UAEXAAVinput_buffer@2@AAVSSL@2@@Z 0043ca30 f   yassl:yassl_imp.obj
 0001:0003ba50       ??0ServerHelloDone@yaSSL@@QAE@XZ 0043ca50 f   yassl:yassl_imp.obj
 0001:0003ba60       ??1ServerHelloDone@yaSSL@@UAE@XZ 0043ca60 f i yassl:yassl_imp.obj
 0001:0003ba70       ?set@ServerHelloDone@yaSSL@@UAEAAVinput_buffer@2@AAV32@@Z 0043ca70 f   yassl:yassl_imp.obj
 0001:0003ba80       ?get@ServerHelloDone@yaSSL@@UBEAAVoutput_buffer@2@AAV32@@Z 0043ca80 f   yassl:yassl_imp.obj
 0001:0003ba90       ?get_type@ServerHelloDone@yaSSL@@UBE?AW4HandShakeType@2@XZ 0043ca90 f   yassl:yassl_imp.obj
 0001:0003baa0       ?get_length@ClientKeyBase@yaSSL@@UBEHXZ 0043caa0 f   yassl:yassl_imp.obj
 0001:0003bab0       ?get_clientKey@ClientKeyBase@yaSSL@@UBEPAEXZ 0043cab0 f   yassl:yassl_imp.obj
 0001:0003bac0       ??5yaSSL@@YAAAVinput_buffer@0@AAV10@AAVClientHello@0@@Z 0043cac0 f   yassl:yassl_imp.obj
 0001:0003bc40       ??6yaSSL@@YAAAVoutput_buffer@0@AAV10@ABVClientHello@0@@Z 0043cc40 f   yassl:yassl_imp.obj
 0001:0003bd20       ?set@ClientHello@yaSSL@@UAEAAVinput_buffer@2@AAV32@@Z 0043cd20 f   yassl:yassl_imp.obj
 0001:0003bd40       ?get@ClientHello@yaSSL@@UBEAAVoutput_buffer@2@AAV32@@Z 0043cd40 f   yassl:yassl_imp.obj
 0001:0003bd60       ?get_type@ClientHello@yaSSL@@UBE?AW4HandShakeType@2@XZ 0043cd60 f   yassl:yassl_imp.obj
 0001:0003bd70       ?get_random@ClientHello@yaSSL@@QBEPBEXZ 0043cd70 f   yassl:yassl_imp.obj
 0001:0003bd80       ??0ClientHello@yaSSL@@QAE@XZ 0043cd80 f   yassl:yassl_imp.obj
 0001:0003bdc0       ??1ClientHello@yaSSL@@UAE@XZ 0043cdc0 f i yassl:yassl_imp.obj
 0001:0003bdd0       ??0ClientHello@yaSSL@@QAE@UProtocolVersion@1@_N@Z 0043cdd0 f   yassl:yassl_imp.obj
 0001:0003be20       ??0ServerKeyExchange@yaSSL@@QAE@XZ 0043ce20 f   yassl:yassl_imp.obj
 0001:0003be30       ?build@ServerKeyExchange@yaSSL@@QAEXAAVSSL@2@@Z 0043ce30 f   yassl:yassl_imp.obj
 0001:0003be60       ?getKey@ServerKeyExchange@yaSSL@@QBEPBEXZ 0043ce60 f   yassl:yassl_imp.obj
 0001:0003be70       ?getKeyLength@ServerKeyExchange@yaSSL@@QBEHXZ 0043ce70 f   yassl:yassl_imp.obj
 0001:0003be80       ?set@ServerKeyExchange@yaSSL@@UAEAAVinput_buffer@2@AAV32@@Z 0043ce80 f   yassl:yassl_imp.obj
 0001:0003be90       ?get_type@ServerKeyExchange@yaSSL@@UBE?AW4HandShakeType@2@XZ 0043ce90 f   yassl:yassl_imp.obj
 0001:0003bea0       ?Process@CertificateRequest@yaSSL@@UAEXAAVinput_buffer@2@AAVSSL@2@@Z 0043cea0 f   yassl:yassl_imp.obj
 0001:0003bee0       ?get_type@CertificateRequest@yaSSL@@UBE?AW4HandShakeType@2@XZ 0043cee0 f   yassl:yassl_imp.obj
 0001:0003bef0       ??0CertificateVerify@yaSSL@@QAE@XZ 0043cef0 f   yassl:yassl_imp.obj
 0001:0003bf00       ??5yaSSL@@YAAAVinput_buffer@0@AAV10@AAVCertificateVerify@0@@Z 0043cf00 f   yassl:yassl_imp.obj
 0001:0003bf60       ??6yaSSL@@YAAAVoutput_buffer@0@AAV10@ABVCertificateVerify@0@@Z 0043cf60 f   yassl:yassl_imp.obj
 0001:0003bf80       ?Process@CertificateVerify@yaSSL@@UAEXAAVinput_buffer@2@AAVSSL@2@@Z 0043cf80 f   yassl:yassl_imp.obj
 0001:0003c0a0       ?get_type@CertificateVerify@yaSSL@@UBE?AW4HandShakeType@2@XZ 0043d0a0 f   yassl:yassl_imp.obj
 0001:0003c0b0       ??0ClientKeyExchange@yaSSL@@QAE@XZ 0043d0b0 f   yassl:yassl_imp.obj
 0001:0003c0c0       ?build@ClientKeyExchange@yaSSL@@QAEXAAVSSL@2@@Z 0043d0c0 f   yassl:yassl_imp.obj
 0001:0003c0f0       ?getKey@ClientKeyExchange@yaSSL@@QBEPBEXZ 0043d0f0 f   yassl:yassl_imp.obj
 0001:0003c100       ?getKeyLength@ClientKeyExchange@yaSSL@@QBEHXZ 0043d100 f   yassl:yassl_imp.obj
 0001:0003c110       ?set@ClientKeyExchange@yaSSL@@UAEAAVinput_buffer@2@AAV32@@Z 0043d110 f   yassl:yassl_imp.obj
 0001:0003c120       ?get_type@ClientKeyExchange@yaSSL@@UBE?AW4HandShakeType@2@XZ 0043d120 f   yassl:yassl_imp.obj
 0001:0003c130       ??5yaSSL@@YAAAVinput_buffer@0@AAV10@AAVFinished@0@@Z 0043d130 f   yassl:yassl_imp.obj
 0001:0003c140       ??6yaSSL@@YAAAVoutput_buffer@0@AAV10@ABVFinished@0@@Z 0043d140 f   yassl:yassl_imp.obj
 0001:0003c190       ?Process@Finished@yaSSL@@UAEXAAVinput_buffer@2@AAVSSL@2@@Z 0043d190 f   yassl:yassl_imp.obj
 0001:0003c4a0       ??0Finished@yaSSL@@QAE@XZ  0043d4a0 f   yassl:yassl_imp.obj
 0001:0003c4b0       ??_EFinished@yaSSL@@UAEPAXI@Z 0043d4b0 f i yassl:yassl_imp.obj
 0001:0003c4b0       ??_GFinished@yaSSL@@UAEPAXI@Z 0043d4b0 f i yassl:yassl_imp.obj
 0001:0003c4d0       ?set_md5@Finished@yaSSL@@QAEPAEXZ 0043d4d0 f   yassl:yassl_imp.obj
 0001:0003c4e0       ?set_sha@Finished@yaSSL@@QAEPAEXZ 0043d4e0 f   yassl:yassl_imp.obj
 0001:0003c4f0       ?set@Finished@yaSSL@@UAEAAVinput_buffer@2@AAV32@@Z 0043d4f0 f   yassl:yassl_imp.obj
 0001:0003c510       ?get@Finished@yaSSL@@UBEAAVoutput_buffer@2@AAV32@@Z 0043d510 f   yassl:yassl_imp.obj
 0001:0003c530       ?get_type@Finished@yaSSL@@UBE?AW4HandShakeType@2@XZ 0043d530 f   yassl:yassl_imp.obj
 0001:0003c540       ?clean@yaSSL@@YAXPCEIAAVRandomPool@1@@Z 0043d540 f   yassl:yassl_imp.obj
 0001:0003c580       ??0Connection@yaSSL@@QAE@UProtocolVersion@1@AAVRandomPool@1@@Z 0043d580 f   yassl:yassl_imp.obj
 0001:0003c630       ?AllocPreSecret@Connection@yaSSL@@QAEXI@Z 0043d630 f   yassl:yassl_imp.obj
 0001:0003c650       ?TurnOffTLS@Connection@yaSSL@@QAEXXZ 0043d650 f   yassl:yassl_imp.obj
 0001:0003c660       ?TurnOffTLS1_1@Connection@yaSSL@@QAEXXZ 0043d660 f   yassl:yassl_imp.obj
 0001:0003c670       ?CleanMaster@Connection@yaSSL@@QAEXXZ 0043d670 f   yassl:yassl_imp.obj
 0001:0003c6a0       ?CreateCipherSpec@yaSSL@@YAPAUMessage@1@XZ 0043d6a0 f   yassl:yassl_imp.obj
 0001:0003c6c0       ?CreateHandShake@yaSSL@@YAPAUMessage@1@XZ 0043d6c0 f   yassl:yassl_imp.obj
 0001:0003c6e0       ?CreateData@yaSSL@@YAPAUMessage@1@XZ 0043d6e0 f   yassl:yassl_imp.obj
 0001:0003c700       ??0HelloRequest@yaSSL@@QAE@XZ 0043d700 f i yassl:yassl_imp.obj
 0001:0003c710       ??1HelloRequest@yaSSL@@UAE@XZ 0043d710 f i yassl:yassl_imp.obj
 0001:0003c720       ?CreateClientHello@yaSSL@@YAPAVHandShakeBase@1@XZ 0043d720 f   yassl:yassl_imp.obj
 0001:0003c740       ?CreateServerHello@yaSSL@@YAPAVHandShakeBase@1@XZ 0043d740 f   yassl:yassl_imp.obj
 0001:0003c760       ?CreateCertificate@yaSSL@@YAPAVHandShakeBase@1@XZ 0043d760 f   yassl:yassl_imp.obj
 0001:0003c780       ?CreateServerKeyExchange@yaSSL@@YAPAVHandShakeBase@1@XZ 0043d780 f   yassl:yassl_imp.obj
 0001:0003c7a0       ?CreateServerHelloDone@yaSSL@@YAPAVHandShakeBase@1@XZ 0043d7a0 f   yassl:yassl_imp.obj
 0001:0003c7c0       ?CreateCertificateVerify@yaSSL@@YAPAVHandShakeBase@1@XZ 0043d7c0 f   yassl:yassl_imp.obj
 0001:0003c7e0       ?CreateClientKeyExchange@yaSSL@@YAPAVHandShakeBase@1@XZ 0043d7e0 f   yassl:yassl_imp.obj
 0001:0003c800       ?CreateFinished@yaSSL@@YAPAVHandShakeBase@1@XZ 0043d800 f   yassl:yassl_imp.obj
 0001:0003c820       ??0RSA_Server@yaSSL@@QAE@XZ 0043d820 f i yassl:yassl_imp.obj
 0001:0003c830       ??1RSA_Server@yaSSL@@UAE@XZ 0043d830 f i yassl:yassl_imp.obj
 0001:0003c840       ??0Fortezza_Server@yaSSL@@QAE@XZ 0043d840 f i yassl:yassl_imp.obj
 0001:0003c850       ??1Fortezza_Server@yaSSL@@UAE@XZ 0043d850 f i yassl:yassl_imp.obj
 0001:0003c860       ?CreateDHClient@yaSSL@@YAPAUClientKeyBase@1@XZ 0043d860 f   yassl:yassl_imp.obj
 0001:0003c880       ??0FortezzaKeys@yaSSL@@QAE@XZ 0043d880 f i yassl:yassl_imp.obj
 0001:0003c890       ??1FortezzaKeys@yaSSL@@UAE@XZ 0043d890 f i yassl:yassl_imp.obj
 0001:0003c8a0       ??0?$list@PAE@mySTL@@QAE@XZ 0043d8a0 f i yassl:yassl_imp.obj
 0001:0003c8b0       ??0?$auto_ptr@UAuth@yaSSL@@@mySTL@@QAE@PAUAuth@yaSSL@@@Z 0043d8b0 f i yassl:yassl_imp.obj
 0001:0003c8c0       ??C?$auto_ptr@UAuth@yaSSL@@@mySTL@@QBEPAUAuth@yaSSL@@XZ 0043d8c0 f i yassl:yassl_imp.obj
 0001:0003c8d0       ??0?$auto_ptr@VHandShakeBase@yaSSL@@@mySTL@@QAE@PAVHandShakeBase@yaSSL@@@Z 0043d8d0 f i yassl:yassl_imp.obj
 0001:0003c8e0       ??C?$auto_ptr@VHandShakeBase@yaSSL@@@mySTL@@QBEPAVHandShakeBase@yaSSL@@XZ 0043d8e0 f i yassl:yassl_imp.obj
 0001:0003c8f0       ??D?$auto_ptr@VHandShakeBase@yaSSL@@@mySTL@@QBEAAVHandShakeBase@yaSSL@@XZ 0043d8f0 f i yassl:yassl_imp.obj
 0001:0003c900       ?get@?$auto_ptr@VHandShakeBase@yaSSL@@@mySTL@@QBEPAVHandShakeBase@yaSSL@@XZ 0043d900 f i yassl:yassl_imp.obj
 0001:0003c910       ??Diterator@?$list@PAE@mySTL@@QBEAAPAEXZ 0043d910 f i yassl:yassl_imp.obj
 0001:0003c920       ??Eiterator@?$list@PAE@mySTL@@QAEAAV012@XZ 0043d920 f i yassl:yassl_imp.obj
 0001:0003c930       ??9iterator@?$list@PAE@mySTL@@QBE_NABV012@@Z 0043d930 f i yassl:yassl_imp.obj
 0001:0003c950       ??0?$auto_array@E@mySTL@@QAE@PAE@Z 0043d950 f i yassl:yassl_imp.obj
 0001:0003c960       ?get@?$auto_array@E@mySTL@@QBEPAEXZ 0043d960 f i yassl:yassl_imp.obj
 0001:0003c970       ?release@?$auto_array@E@mySTL@@QAEPAEXZ 0043d970 f i yassl:yassl_imp.obj
 0001:0003c980       ?begin@?$vector@U?$pair@HP6APAVHandShakeBase@yaSSL@@XZ@mySTL@@@mySTL@@QBEPBU?$pair@HP6APAVHandShakeBase@yaSSL@@XZ@2@XZ 0043d980 f i yassl:yassl_imp.obj
 0001:0003c990       ?end@?$vector@U?$pair@HP6APAVHandShakeBase@yaSSL@@XZ@mySTL@@@mySTL@@QBEPBU?$pair@HP6APAVHandShakeBase@yaSSL@@XZ@2@XZ 0043d990 f i yassl:yassl_imp.obj
 0001:0003c9a0       ?begin@?$vector@U?$pair@HP6APAUServerKeyBase@yaSSL@@XZ@mySTL@@@mySTL@@QBEPBU?$pair@HP6APAUServerKeyBase@yaSSL@@XZ@2@XZ 0043d9a0 f i yassl:yassl_imp.obj
 0001:0003c9b0       ?end@?$vector@U?$pair@HP6APAUServerKeyBase@yaSSL@@XZ@mySTL@@@mySTL@@QBEPBU?$pair@HP6APAUServerKeyBase@yaSSL@@XZ@2@XZ 0043d9b0 f i yassl:yassl_imp.obj
 0001:0003c9c0       ?begin@?$vector@U?$pair@HP6APAUClientKeyBase@yaSSL@@XZ@mySTL@@@mySTL@@QBEPBU?$pair@HP6APAUClientKeyBase@yaSSL@@XZ@2@XZ 0043d9c0 f i yassl:yassl_imp.obj
 0001:0003c9d0       ?end@?$vector@U?$pair@HP6APAUClientKeyBase@yaSSL@@XZ@mySTL@@@mySTL@@QBEPBU?$pair@HP6APAUClientKeyBase@yaSSL@@XZ@2@XZ 0043d9d0 f i yassl:yassl_imp.obj
 0001:0003c9e0       ??0iterator@?$list@PAE@mySTL@@QAE@PAUnode@12@@Z 0043d9e0 f i yassl:yassl_imp.obj
 0001:0003c9f0       ?capacity@?$vector@U?$pair@HP6APAUMessage@yaSSL@@XZ@mySTL@@@mySTL@@QBEIXZ 0043d9f0 f i yassl:yassl_imp.obj
 0001:0003ca00       ?size@?$vector@U?$pair@HP6APAUMessage@yaSSL@@XZ@mySTL@@@mySTL@@QBEIXZ 0043da00 f i yassl:yassl_imp.obj
 0001:0003ca10       ?capacity@?$vector@U?$pair@HP6APAVHandShakeBase@yaSSL@@XZ@mySTL@@@mySTL@@QBEIXZ 0043da10 f i yassl:yassl_imp.obj
 0001:0003ca20       ?size@?$vector@U?$pair@HP6APAVHandShakeBase@yaSSL@@XZ@mySTL@@@mySTL@@QBEIXZ 0043da20 f i yassl:yassl_imp.obj
 0001:0003ca30       ?capacity@?$vector@U?$pair@HP6APAUServerKeyBase@yaSSL@@XZ@mySTL@@@mySTL@@QBEIXZ 0043da30 f i yassl:yassl_imp.obj
 0001:0003ca40       ?size@?$vector@U?$pair@HP6APAUServerKeyBase@yaSSL@@XZ@mySTL@@@mySTL@@QBEIXZ 0043da40 f i yassl:yassl_imp.obj
 0001:0003ca50       ?capacity@?$vector@U?$pair@HP6APAUClientKeyBase@yaSSL@@XZ@mySTL@@@mySTL@@QBEIXZ 0043da50 f i yassl:yassl_imp.obj
 0001:0003ca60       ?size@?$vector@U?$pair@HP6APAUClientKeyBase@yaSSL@@XZ@mySTL@@@mySTL@@QBEIXZ 0043da60 f i yassl:yassl_imp.obj
 0001:0003ca70       ??$ysDelete@UServerKeyBase@yaSSL@@@yaSSL@@YAXPAUServerKeyBase@0@@Z 0043da70 f i yassl:yassl_imp.obj
 0001:0003ca90       ??$ysDelete@UClientKeyBase@yaSSL@@@yaSSL@@YAXPAUClientKeyBase@0@@Z 0043da90 f i yassl:yassl_imp.obj
 0001:0003cab0       ??$construct@U?$pair@HP6APAUMessage@yaSSL@@XZ@mySTL@@U12@@mySTL@@YAXPAU?$pair@HP6APAUMessage@yaSSL@@XZ@0@ABU10@@Z 0043dab0 f i yassl:yassl_imp.obj
 0001:0003cad0       ??$construct@U?$pair@HP6APAVHandShakeBase@yaSSL@@XZ@mySTL@@U12@@mySTL@@YAXPAU?$pair@HP6APAVHandShakeBase@yaSSL@@XZ@0@ABU10@@Z 0043dad0 f i yassl:yassl_imp.obj
 0001:0003caf0       ??$construct@U?$pair@HP6APAUServerKeyBase@yaSSL@@XZ@mySTL@@U12@@mySTL@@YAXPAU?$pair@HP6APAUServerKeyBase@yaSSL@@XZ@0@ABU10@@Z 0043daf0 f i yassl:yassl_imp.obj
 0001:0003cb10       ??$construct@U?$pair@HP6APAUClientKeyBase@yaSSL@@XZ@mySTL@@U12@@mySTL@@YAXPAU?$pair@HP6APAUClientKeyBase@yaSSL@@XZ@0@ABU10@@Z 0043db10 f i yassl:yassl_imp.obj
 0001:0003cb30       ??$ysDelete@UAuth@yaSSL@@@yaSSL@@YAXPAUAuth@0@@Z 0043db30 f i yassl:yassl_imp.obj
 0001:0003cb50       ??$ysDelete@VHandShakeBase@yaSSL@@@yaSSL@@YAXPAVHandShakeBase@0@@Z 0043db50 f i yassl:yassl_imp.obj
 0001:0003cb70       ??$uninit_copy@PAU?$pair@HP6APAUMessage@yaSSL@@XZ@mySTL@@PAU12@@mySTL@@YAPAU?$pair@HP6APAUMessage@yaSSL@@XZ@0@PAU10@00@Z 0043db70 f i yassl:yassl_imp.obj
 0001:0003cba0       ??$uninit_copy@PAU?$pair@HP6APAVHandShakeBase@yaSSL@@XZ@mySTL@@PAU12@@mySTL@@YAPAU?$pair@HP6APAVHandShakeBase@yaSSL@@XZ@0@PAU10@00@Z 0043dba0 f i yassl:yassl_imp.obj
 0001:0003cbd0       ??$uninit_copy@PAU?$pair@HP6APAUServerKeyBase@yaSSL@@XZ@mySTL@@PAU12@@mySTL@@YAPAU?$pair@HP6APAUServerKeyBase@yaSSL@@XZ@0@PAU10@00@Z 0043dbd0 f i yassl:yassl_imp.obj
 0001:0003cc00       ??$uninit_copy@PAU?$pair@HP6APAUClientKeyBase@yaSSL@@XZ@mySTL@@PAU12@@mySTL@@YAPAU?$pair@HP6APAUClientKeyBase@yaSSL@@XZ@0@PAU10@00@Z 0043dc00 f i yassl:yassl_imp.obj
 0001:0003cc30       ??$GetArrayMemory@U?$pair@HP6APAUMessage@yaSSL@@XZ@mySTL@@@mySTL@@YAPAU?$pair@HP6APAUMessage@yaSSL@@XZ@0@I@Z 0043dc30 f i yassl:yassl_imp.obj
 0001:0003cc50       ??$swap@PAU?$pair@HP6APAUMessage@yaSSL@@XZ@mySTL@@@mySTL@@YAXAAPAU?$pair@HP6APAUMessage@yaSSL@@XZ@0@0@Z 0043dc50 f i yassl:yassl_imp.obj
 0001:0003cc70       ??$GetArrayMemory@U?$pair@HP6APAVHandShakeBase@yaSSL@@XZ@mySTL@@@mySTL@@YAPAU?$pair@HP6APAVHandShakeBase@yaSSL@@XZ@0@I@Z 0043dc70 f i yassl:yassl_imp.obj
 0001:0003cc90       ??$swap@PAU?$pair@HP6APAVHandShakeBase@yaSSL@@XZ@mySTL@@@mySTL@@YAXAAPAU?$pair@HP6APAVHandShakeBase@yaSSL@@XZ@0@0@Z 0043dc90 f i yassl:yassl_imp.obj
 0001:0003ccb0       ??$GetArrayMemory@U?$pair@HP6APAUServerKeyBase@yaSSL@@XZ@mySTL@@@mySTL@@YAPAU?$pair@HP6APAUServerKeyBase@yaSSL@@XZ@0@I@Z 0043dcb0 f i yassl:yassl_imp.obj
 0001:0003ccd0       ??$swap@PAU?$pair@HP6APAUServerKeyBase@yaSSL@@XZ@mySTL@@@mySTL@@YAXAAPAU?$pair@HP6APAUServerKeyBase@yaSSL@@XZ@0@0@Z 0043dcd0 f i yassl:yassl_imp.obj
 0001:0003ccf0       ??$GetArrayMemory@U?$pair@HP6APAUClientKeyBase@yaSSL@@XZ@mySTL@@@mySTL@@YAPAU?$pair@HP6APAUClientKeyBase@yaSSL@@XZ@0@I@Z 0043dcf0 f i yassl:yassl_imp.obj
 0001:0003cd10       ??$swap@PAU?$pair@HP6APAUClientKeyBase@yaSSL@@XZ@mySTL@@@mySTL@@YAXAAPAU?$pair@HP6APAUClientKeyBase@yaSSL@@XZ@0@0@Z 0043dd10 f i yassl:yassl_imp.obj
 0001:0003cd30       ??0?$pair@HP6APAUMessage@yaSSL@@XZ@mySTL@@QAE@ABHABQ6APAUMessage@yaSSL@@XZ@Z 0043dd30 f i yassl:yassl_imp.obj
 0001:0003cd50       ??0?$pair@HP6APAVHandShakeBase@yaSSL@@XZ@mySTL@@QAE@ABHABQ6APAVHandShakeBase@yaSSL@@XZ@Z 0043dd50 f i yassl:yassl_imp.obj
 0001:0003cd70       ??0?$pair@HP6APAUServerKeyBase@yaSSL@@XZ@mySTL@@QAE@ABHABQ6APAUServerKeyBase@yaSSL@@XZ@Z 0043dd70 f i yassl:yassl_imp.obj
 0001:0003cd90       ??0?$pair@HP6APAUClientKeyBase@yaSSL@@XZ@mySTL@@QAE@ABHABQ6APAUClientKeyBase@yaSSL@@XZ@Z 0043dd90 f i yassl:yassl_imp.obj
 0001:0003cdb0       ??0node@?$list@PAE@mySTL@@QAE@PAE@Z 0043ddb0 f i yassl:yassl_imp.obj
 0001:0003cdd0       ??$destroy@Unode@?$list@PAE@mySTL@@@mySTL@@YAXPAUnode@?$list@PAE@0@@Z 0043ddd0 f i yassl:yassl_imp.obj
 0001:0003cde0       ??$swap@PAE@mySTL@@YAXAAPAE0@Z 0043dde0 f i yassl:yassl_imp.obj
 0001:0003ce00       ??$ysDelete@E@yaSSL@@YAXPAE@Z 0043de00 f i yassl:yassl_imp.obj
 0001:0003ce10       ??0Alert@yaSSL@@QAE@XZ     0043de10 f i yassl:yassl_imp.obj
 0001:0003ce20       ??_GAlert@yaSSL@@UAEPAXI@Z 0043de20 f i yassl:yassl_imp.obj
 0001:0003ce20       ??_EAlert@yaSSL@@UAEPAXI@Z 0043de20 f i yassl:yassl_imp.obj
 0001:0003ce40       ??_GHandShakeHeader@yaSSL@@UAEPAXI@Z 0043de40 f i yassl:yassl_imp.obj
 0001:0003ce40       ??_EHandShakeHeader@yaSSL@@UAEPAXI@Z 0043de40 f i yassl:yassl_imp.obj
 0001:0003ce60       ?build@EncryptedPreMasterSecret@yaSSL@@UAEXAAVSSL@2@@Z 0043de60 f   yassl:yassl_imp.obj
 0001:0003cf90       ?build@ClientDiffieHellmanPublic@yaSSL@@UAEXAAVSSL@2@@Z 0043df90 f   yassl:yassl_imp.obj
 0001:0003d040       ?read@EncryptedPreMasterSecret@yaSSL@@UAEXAAVSSL@2@AAVinput_buffer@2@@Z 0043e040 f   yassl:yassl_imp.obj
 0001:0003d160       ??0EncryptedPreMasterSecret@yaSSL@@QAE@XZ 0043e160 f   yassl:yassl_imp.obj
 0001:0003d180       ??1EncryptedPreMasterSecret@yaSSL@@UAE@XZ 0043e180 f   yassl:yassl_imp.obj
 0001:0003d1a0       ?read@ClientDiffieHellmanPublic@yaSSL@@UAEXAAVSSL@2@AAVinput_buffer@2@@Z 0043e1a0 f   yassl:yassl_imp.obj
 0001:0003d270       ??1ClientDiffieHellmanPublic@yaSSL@@UAE@XZ 0043e270 f   yassl:yassl_imp.obj
 0001:0003d290       ?read@DH_Server@yaSSL@@UAEXAAVSSL@2@AAVinput_buffer@2@@Z 0043e290 f   yassl:yassl_imp.obj
 0001:0003d680       ?SetSuites@Parameters@yaSSL@@QAEXUProtocolVersion@2@_N11@Z 0043e680 f   yassl:yassl_imp.obj
 0001:0003d860       ??_EChangeCipherSpec@yaSSL@@UAEPAXI@Z 0043e860 f i yassl:yassl_imp.obj
 0001:0003d860       ??_GChangeCipherSpec@yaSSL@@UAEPAXI@Z 0043e860 f i yassl:yassl_imp.obj
 0001:0003d880       ?set@Alert@yaSSL@@UAEAAVinput_buffer@2@AAV32@@Z 0043e880 f   yassl:yassl_imp.obj
 0001:0003d8a0       ?get@Alert@yaSSL@@UBEAAVoutput_buffer@2@AAV32@@Z 0043e8a0 f   yassl:yassl_imp.obj
 0001:0003d8c0       ??_EData@yaSSL@@UAEPAXI@Z  0043e8c0 f i yassl:yassl_imp.obj
 0001:0003d8c0       ??_GData@yaSSL@@UAEPAXI@Z  0043e8c0 f i yassl:yassl_imp.obj
 0001:0003d8e0       ?get@Data@yaSSL@@UBEAAVoutput_buffer@2@AAV32@@Z 0043e8e0 f   yassl:yassl_imp.obj
 0001:0003d900       ??0Certificate@yaSSL@@QAE@PBVx509@1@@Z 0043e900 f   yassl:yassl_imp.obj
 0001:0003d930       ??_ECertificate@yaSSL@@UAEPAXI@Z 0043e930 f i yassl:yassl_imp.obj
 0001:0003d930       ??_GCertificate@yaSSL@@UAEPAXI@Z 0043e930 f i yassl:yassl_imp.obj
 0001:0003d950       ??1ServerDHParams@yaSSL@@QAE@XZ 0043e950 f   yassl:yassl_imp.obj
 0001:0003d980       ?Process@ServerHello@yaSSL@@UAEXAAVinput_buffer@2@AAVSSL@2@@Z 0043e980 f   yassl:yassl_imp.obj
 0001:0003dbc0       ??_GServerHello@yaSSL@@UAEPAXI@Z 0043ebc0 f i yassl:yassl_imp.obj
 0001:0003dbc0       ??_EServerHello@yaSSL@@UAEPAXI@Z 0043ebc0 f i yassl:yassl_imp.obj
 0001:0003dbe0       ??_EServerHelloDone@yaSSL@@UAEPAXI@Z 0043ebe0 f i yassl:yassl_imp.obj
 0001:0003dbe0       ??_GServerHelloDone@yaSSL@@UAEPAXI@Z 0043ebe0 f i yassl:yassl_imp.obj
 0001:0003dc00       ?Process@ClientHello@yaSSL@@UAEXAAVinput_buffer@2@AAVSSL@2@@Z 0043ec00 f   yassl:yassl_imp.obj
 0001:0003df20       ??_GClientHello@yaSSL@@UAEPAXI@Z 0043ef20 f i yassl:yassl_imp.obj
 0001:0003df20       ??_EClientHello@yaSSL@@UAEPAXI@Z 0043ef20 f i yassl:yassl_imp.obj
 0001:0003df40       ??6yaSSL@@YAAAVoutput_buffer@0@AAV10@ABVServerKeyExchange@0@@Z 0043ef40 f   yassl:yassl_imp.obj
 0001:0003df70       ??1ServerKeyExchange@yaSSL@@UAE@XZ 0043ef70 f   yassl:yassl_imp.obj
 0001:0003df90       ?get@ServerKeyExchange@yaSSL@@UBEAAVoutput_buffer@2@AAV32@@Z 0043ef90 f   yassl:yassl_imp.obj
 0001:0003dfb0       ??1CertificateVerify@yaSSL@@UAE@XZ 0043efb0 f   yassl:yassl_imp.obj
 0001:0003dfd0       ?set@CertificateVerify@yaSSL@@UAEAAVinput_buffer@2@AAV32@@Z 0043efd0 f   yassl:yassl_imp.obj
 0001:0003dff0       ?get@CertificateVerify@yaSSL@@UBEAAVoutput_buffer@2@AAV32@@Z 0043eff0 f   yassl:yassl_imp.obj
 0001:0003e010       ??6yaSSL@@YAAAVoutput_buffer@0@AAV10@ABVClientKeyExchange@0@@Z 0043f010 f   yassl:yassl_imp.obj
 0001:0003e040       ??1ClientKeyExchange@yaSSL@@UAE@XZ 0043f040 f   yassl:yassl_imp.obj
 0001:0003e060       ?get@ClientKeyExchange@yaSSL@@UBEAAVoutput_buffer@2@AAV32@@Z 0043f060 f   yassl:yassl_imp.obj
 0001:0003e080       ?CleanPreMaster@Connection@yaSSL@@QAEXXZ 0043f080 f   yassl:yassl_imp.obj
 0001:0003e0b0       ?CreateAlert@yaSSL@@YAPAUMessage@1@XZ 0043f0b0 f   yassl:yassl_imp.obj
 0001:0003e0d0       ?CreateHelloRequest@yaSSL@@YAPAVHandShakeBase@1@XZ 0043f0d0 f   yassl:yassl_imp.obj
 0001:0003e0f0       ??_EHelloRequest@yaSSL@@UAEPAXI@Z 0043f0f0 f i yassl:yassl_imp.obj
 0001:0003e0f0       ??_GHelloRequest@yaSSL@@UAEPAXI@Z 0043f0f0 f i yassl:yassl_imp.obj
 0001:0003e110       ?CreateRSAServerKEA@yaSSL@@YAPAUServerKeyBase@1@XZ 0043f110 f   yassl:yassl_imp.obj
 0001:0003e130       ??_ERSA_Server@yaSSL@@UAEPAXI@Z 0043f130 f i yassl:yassl_imp.obj
 0001:0003e130       ??_GRSA_Server@yaSSL@@UAEPAXI@Z 0043f130 f i yassl:yassl_imp.obj
 0001:0003e150       ?CreateFortezzaServerKEA@yaSSL@@YAPAUServerKeyBase@1@XZ 0043f150 f   yassl:yassl_imp.obj
 0001:0003e170       ??_EFortezza_Server@yaSSL@@UAEPAXI@Z 0043f170 f i yassl:yassl_imp.obj
 0001:0003e170       ??_GFortezza_Server@yaSSL@@UAEPAXI@Z 0043f170 f i yassl:yassl_imp.obj
 0001:0003e190       ?CreateRSAClient@yaSSL@@YAPAUClientKeyBase@1@XZ 0043f190 f   yassl:yassl_imp.obj
 0001:0003e1b0       ?CreateFortezzaClient@yaSSL@@YAPAUClientKeyBase@1@XZ 0043f1b0 f   yassl:yassl_imp.obj
 0001:0003e1d0       ??_EFortezzaKeys@yaSSL@@UAEPAXI@Z 0043f1d0 f i yassl:yassl_imp.obj
 0001:0003e1d0       ??_GFortezzaKeys@yaSSL@@UAEPAXI@Z 0043f1d0 f i yassl:yassl_imp.obj
 0001:0003e1f0       ?begin@?$list@PAE@mySTL@@QBE?AViterator@12@XZ 0043f1f0 f i yassl:yassl_imp.obj
 0001:0003e200       ?end@?$list@PAE@mySTL@@QBE?AViterator@12@XZ 0043f200 f i yassl:yassl_imp.obj
 0001:0003e210       ?CreateObject@?$Factory@VHandShakeBase@yaSSL@@HP6APAV12@XZ@yaSSL@@QBEPAVHandShakeBase@2@ABH@Z 0043f210 f i yassl:yassl_imp.obj
 0001:0003e240       ?CreateObject@?$Factory@UServerKeyBase@yaSSL@@HP6APAU12@XZ@yaSSL@@QBEPAUServerKeyBase@2@ABH@Z 0043f240 f i yassl:yassl_imp.obj
 0001:0003e270       ?CreateObject@?$Factory@UClientKeyBase@yaSSL@@HP6APAU12@XZ@yaSSL@@QBEPAUClientKeyBase@2@ABH@Z 0043f270 f i yassl:yassl_imp.obj
 0001:0003e2a0       ?Destroy@?$auto_ptr@UAuth@yaSSL@@@mySTL@@AAEXXZ 0043f2a0 f i yassl:yassl_imp.obj
 0001:0003e2b0       ?Destroy@?$auto_ptr@VHandShakeBase@yaSSL@@@mySTL@@AAEXXZ 0043f2b0 f i yassl:yassl_imp.obj
 0001:0003e2c0       ?Destroy@?$auto_array@E@mySTL@@AAEXXZ 0043f2c0 f i yassl:yassl_imp.obj
 0001:0003e2d0       ??0?$vector_base@U?$pair@HP6APAUMessage@yaSSL@@XZ@mySTL@@@mySTL@@QAE@I@Z 0043f2d0 f i yassl:yassl_imp.obj
 0001:0003e300       ?Swap@?$vector_base@U?$pair@HP6APAUMessage@yaSSL@@XZ@mySTL@@@mySTL@@QAEXAAU12@@Z 0043f300 f i yassl:yassl_imp.obj
 0001:0003e330       ??0?$vector_base@U?$pair@HP6APAVHandShakeBase@yaSSL@@XZ@mySTL@@@mySTL@@QAE@I@Z 0043f330 f i yassl:yassl_imp.obj
 0001:0003e360       ?Swap@?$vector_base@U?$pair@HP6APAVHandShakeBase@yaSSL@@XZ@mySTL@@@mySTL@@QAEXAAU12@@Z 0043f360 f i yassl:yassl_imp.obj
 0001:0003e390       ??0?$vector_base@U?$pair@HP6APAUServerKeyBase@yaSSL@@XZ@mySTL@@@mySTL@@QAE@I@Z 0043f390 f i yassl:yassl_imp.obj
 0001:0003e3c0       ?Swap@?$vector_base@U?$pair@HP6APAUServerKeyBase@yaSSL@@XZ@mySTL@@@mySTL@@QAEXAAU12@@Z 0043f3c0 f i yassl:yassl_imp.obj
 0001:0003e3f0       ??0?$vector_base@U?$pair@HP6APAUClientKeyBase@yaSSL@@XZ@mySTL@@@mySTL@@QAE@I@Z 0043f3f0 f i yassl:yassl_imp.obj
 0001:0003e420       ?Swap@?$vector_base@U?$pair@HP6APAUClientKeyBase@yaSSL@@XZ@mySTL@@@mySTL@@QAEXAAU12@@Z 0043f420 f i yassl:yassl_imp.obj
 0001:0003e450       ?push_back@?$list@PAE@mySTL@@QAEXPAE@Z 0043f450 f i yassl:yassl_imp.obj
 0001:0003e4a0       ??$make_pair@HP6APAUMessage@yaSSL@@XZ@mySTL@@YA?AU?$pair@HP6APAUMessage@yaSSL@@XZ@0@ABHABQ6APAUMessage@yaSSL@@XZ@Z 0043f4a0 f i yassl:yassl_imp.obj
 0001:0003e4c0       ??$make_pair@HP6APAVHandShakeBase@yaSSL@@XZ@mySTL@@YA?AU?$pair@HP6APAVHandShakeBase@yaSSL@@XZ@0@ABHABQ6APAVHandShakeBase@yaSSL@@XZ@Z 0043f4c0 f i yassl:yassl_imp.obj
 0001:0003e4e0       ??$make_pair@HP6APAUServerKeyBase@yaSSL@@XZ@mySTL@@YA?AU?$pair@HP6APAUServerKeyBase@yaSSL@@XZ@0@ABHABQ6APAUServerKeyBase@yaSSL@@XZ@Z 0043f4e0 f i yassl:yassl_imp.obj
 0001:0003e500       ??$make_pair@HP6APAUClientKeyBase@yaSSL@@XZ@mySTL@@YA?AU?$pair@HP6APAUClientKeyBase@yaSSL@@XZ@0@ABHABQ6APAUClientKeyBase@yaSSL@@XZ@Z 0043f500 f i yassl:yassl_imp.obj
 0001:0003e520       ??$checked_delete@E@yaSSL@@YAXPAE@Z 0043f520 f i yassl:yassl_imp.obj
 0001:0003e530       ?createKey@ClientKeyExchange@yaSSL@@QAEXAAVSSL@2@@Z 0043f530 f   yassl:yassl_imp.obj
 0001:0003e5a0       ?createKey@ServerKeyExchange@yaSSL@@QAEXAAVSSL@2@@Z 0043f5a0 f   yassl:yassl_imp.obj
 0001:0003e610       ??_GEncryptedPreMasterSecret@yaSSL@@UAEPAXI@Z 0043f610 f i yassl:yassl_imp.obj
 0001:0003e610       ??_EEncryptedPreMasterSecret@yaSSL@@UAEPAXI@Z 0043f610 f i yassl:yassl_imp.obj
 0001:0003e630       ??_GClientDiffieHellmanPublic@yaSSL@@UAEPAXI@Z 0043f630 f i yassl:yassl_imp.obj
 0001:0003e630       ??_EClientDiffieHellmanPublic@yaSSL@@UAEPAXI@Z 0043f630 f i yassl:yassl_imp.obj
 0001:0003e650       ??0DH_Server@yaSSL@@QAE@XZ 0043f650 f   yassl:yassl_imp.obj
 0001:0003e670       ??1DH_Server@yaSSL@@UAE@XZ 0043f670 f   yassl:yassl_imp.obj
 0001:0003e6a0       ??0Parameters@yaSSL@@QAE@W4ConnectionEnd@1@ABUCiphers@1@UProtocolVersion@1@_N@Z 0043f6a0 f   yassl:yassl_imp.obj
 0001:0003e730       ?Process@ServerKeyExchange@yaSSL@@UAEXAAVinput_buffer@2@AAVSSL@2@@Z 0043f730 f   yassl:yassl_imp.obj
 0001:0003e780       ??0ServerKeyExchange@yaSSL@@QAE@AAVSSL@1@@Z 0043f780 f   yassl:yassl_imp.obj
 0001:0003e7a0       ??_EServerKeyExchange@yaSSL@@UAEPAXI@Z 0043f7a0 f i yassl:yassl_imp.obj
 0001:0003e7a0       ??_GServerKeyExchange@yaSSL@@UAEPAXI@Z 0043f7a0 f i yassl:yassl_imp.obj
 0001:0003e7c0       ?Build@CertificateRequest@yaSSL@@QAEXXZ 0043f7c0 f   yassl:yassl_imp.obj
 0001:0003e7e0       ??5yaSSL@@YAAAVinput_buffer@0@AAV10@AAVCertificateRequest@0@@Z 0043f7e0 f   yassl:yassl_imp.obj
 0001:0003e8d0       ??6yaSSL@@YAAAVoutput_buffer@0@AAV10@ABVCertificateRequest@0@@Z 0043f8d0 f   yassl:yassl_imp.obj
 0001:0003e990       ??_GCertificateVerify@yaSSL@@UAEPAXI@Z 0043f990 f i yassl:yassl_imp.obj
 0001:0003e990       ??_ECertificateVerify@yaSSL@@UAEPAXI@Z 0043f990 f i yassl:yassl_imp.obj
 0001:0003e9b0       ?Process@ClientKeyExchange@yaSSL@@UAEXAAVinput_buffer@2@AAVSSL@2@@Z 0043f9b0 f   yassl:yassl_imp.obj
 0001:0003ea30       ??0ClientKeyExchange@yaSSL@@QAE@AAVSSL@1@@Z 0043fa30 f   yassl:yassl_imp.obj
 0001:0003ea50       ??_EClientKeyExchange@yaSSL@@UAEPAXI@Z 0043fa50 f i yassl:yassl_imp.obj
 0001:0003ea50       ??_GClientKeyExchange@yaSSL@@UAEPAXI@Z 0043fa50 f i yassl:yassl_imp.obj
 0001:0003ea70       ??1Connection@yaSSL@@QAE@XZ 0043fa70 f   yassl:yassl_imp.obj
 0001:0003ea90       ?CreateDHServerKEA@yaSSL@@YAPAUServerKeyBase@1@XZ 0043fa90 f   yassl:yassl_imp.obj
 0001:0003eab0       ??1?$auto_ptr@UAuth@yaSSL@@@mySTL@@QAE@XZ 0043fab0 f i yassl:yassl_imp.obj
 0001:0003eac0       ?reset@?$auto_ptr@UAuth@yaSSL@@@mySTL@@QAEXPAUAuth@yaSSL@@@Z 0043fac0 f i yassl:yassl_imp.obj
 0001:0003eae0       ??1?$auto_ptr@VHandShakeBase@yaSSL@@@mySTL@@QAE@XZ 0043fae0 f i yassl:yassl_imp.obj
 0001:0003eaf0       ??1?$auto_array@E@mySTL@@QAE@XZ 0043faf0 f i yassl:yassl_imp.obj
 0001:0003eb00       ?reset@?$auto_array@E@mySTL@@QAEXPAE@Z 0043fb00 f i yassl:yassl_imp.obj
 0001:0003eb20       ?Swap@?$vector@U?$pair@HP6APAUMessage@yaSSL@@XZ@mySTL@@@mySTL@@QAEXAAV12@@Z 0043fb20 f i yassl:yassl_imp.obj
 0001:0003eb50       ??0?$vector@U?$pair@HP6APAUMessage@yaSSL@@XZ@mySTL@@@mySTL@@AAE@IABV01@@Z 0043fb50 f i yassl:yassl_imp.obj
 0001:0003eb90       ?Swap@?$vector@U?$pair@HP6APAVHandShakeBase@yaSSL@@XZ@mySTL@@@mySTL@@QAEXAAV12@@Z 0043fb90 f i yassl:yassl_imp.obj
 0001:0003ebc0       ??0?$vector@U?$pair@HP6APAVHandShakeBase@yaSSL@@XZ@mySTL@@@mySTL@@AAE@IABV01@@Z 0043fbc0 f i yassl:yassl_imp.obj
 0001:0003ec00       ?Swap@?$vector@U?$pair@HP6APAUServerKeyBase@yaSSL@@XZ@mySTL@@@mySTL@@QAEXAAV12@@Z 0043fc00 f i yassl:yassl_imp.obj
 0001:0003ec30       ??0?$vector@U?$pair@HP6APAUServerKeyBase@yaSSL@@XZ@mySTL@@@mySTL@@AAE@IABV01@@Z 0043fc30 f i yassl:yassl_imp.obj
 0001:0003ec70       ?Swap@?$vector@U?$pair@HP6APAUClientKeyBase@yaSSL@@XZ@mySTL@@@mySTL@@QAEXAAV12@@Z 0043fc70 f i yassl:yassl_imp.obj
 0001:0003eca0       ??0?$vector@U?$pair@HP6APAUClientKeyBase@yaSSL@@XZ@mySTL@@@mySTL@@AAE@IABV01@@Z 0043fca0 f i yassl:yassl_imp.obj
 0001:0003ece0       ??1?$list@PAE@mySTL@@QAE@XZ 0043fce0 f i yassl:yassl_imp.obj
 0001:0003ed00       ??$?RE@del_ptr_zero@yaSSL@@QBEXAAPAE@Z 0043fd00 f i yassl:yassl_imp.obj
 0001:0003ed20       ?build@DH_Server@yaSSL@@UAEXAAVSSL@2@@Z 0043fd20 f   yassl:yassl_imp.obj
 0001:0003f170       ??_EDH_Server@yaSSL@@UAEPAXI@Z 00440170 f i yassl:yassl_imp.obj
 0001:0003f170       ??_GDH_Server@yaSSL@@UAEPAXI@Z 00440170 f i yassl:yassl_imp.obj
 0001:0003f190       ?Process@HandShakeHeader@yaSSL@@UAEXAAVinput_buffer@2@AAVSSL@2@@Z 00440190 f   yassl:yassl_imp.obj
 0001:0003f280       ??0CertificateRequest@yaSSL@@QAE@XZ 00440280 f   yassl:yassl_imp.obj
 0001:0003f2b0       ?set@CertificateRequest@yaSSL@@UAEAAVinput_buffer@2@AAV32@@Z 004402b0 f   yassl:yassl_imp.obj
 0001:0003f2d0       ?get@CertificateRequest@yaSSL@@UBEAAVoutput_buffer@2@AAV32@@Z 004402d0 f   yassl:yassl_imp.obj
 0001:0003f2f0       ?Build@CertificateVerify@yaSSL@@QAEXAAVSSL@2@@Z 004402f0 f   yassl:yassl_imp.obj
 0001:0003f4a0       ?CreateCertificateRequest@yaSSL@@YAPAVHandShakeBase@1@XZ 004404a0 f   yassl:yassl_imp.obj
 0001:0003f4c0       ?push_back@?$vector@U?$pair@HP6APAUMessage@yaSSL@@XZ@mySTL@@@mySTL@@QAEXABU?$pair@HP6APAUMessage@yaSSL@@XZ@2@@Z 004404c0 f i yassl:yassl_imp.obj
 0001:0003f540       ?reserve@?$vector@U?$pair@HP6APAUMessage@yaSSL@@XZ@mySTL@@@mySTL@@QAEXI@Z 00440540 f i yassl:yassl_imp.obj
 0001:0003f590       ?push_back@?$vector@U?$pair@HP6APAVHandShakeBase@yaSSL@@XZ@mySTL@@@mySTL@@QAEXABU?$pair@HP6APAVHandShakeBase@yaSSL@@XZ@2@@Z 00440590 f i yassl:yassl_imp.obj
 0001:0003f610       ?reserve@?$vector@U?$pair@HP6APAVHandShakeBase@yaSSL@@XZ@mySTL@@@mySTL@@QAEXI@Z 00440610 f i yassl:yassl_imp.obj
 0001:0003f660       ?push_back@?$vector@U?$pair@HP6APAUServerKeyBase@yaSSL@@XZ@mySTL@@@mySTL@@QAEXABU?$pair@HP6APAUServerKeyBase@yaSSL@@XZ@2@@Z 00440660 f i yassl:yassl_imp.obj
 0001:0003f6e0       ?reserve@?$vector@U?$pair@HP6APAUServerKeyBase@yaSSL@@XZ@mySTL@@@mySTL@@QAEXI@Z 004406e0 f i yassl:yassl_imp.obj
 0001:0003f730       ?push_back@?$vector@U?$pair@HP6APAUClientKeyBase@yaSSL@@XZ@mySTL@@@mySTL@@QAEXABU?$pair@HP6APAUClientKeyBase@yaSSL@@XZ@2@@Z 00440730 f i yassl:yassl_imp.obj
 0001:0003f7b0       ?reserve@?$vector@U?$pair@HP6APAUClientKeyBase@yaSSL@@XZ@mySTL@@@mySTL@@QAEXI@Z 004407b0 f i yassl:yassl_imp.obj
 0001:0003f800       ??$for_each@Viterator@?$list@PAE@mySTL@@Udel_ptr_zero@yaSSL@@@mySTL@@YA?AUdel_ptr_zero@yaSSL@@Viterator@?$list@PAE@0@0U12@@Z 00440800 f i yassl:yassl_imp.obj
 0001:0003f840       ??1CertificateRequest@yaSSL@@UAE@XZ 00440840 f   yassl:yassl_imp.obj
 0001:0003f880       ?Reserve@?$Factory@UMessage@yaSSL@@HP6APAU12@XZ@yaSSL@@QAEXI@Z 00440880 f i yassl:yassl_imp.obj
 0001:0003f8d0       ?Register@?$Factory@UMessage@yaSSL@@HP6APAU12@XZ@yaSSL@@QAEXABHP6APAUMessage@2@XZ@Z 004408d0 f i yassl:yassl_imp.obj
 0001:0003f900       ?Reserve@?$Factory@VHandShakeBase@yaSSL@@HP6APAV12@XZ@yaSSL@@QAEXI@Z 00440900 f i yassl:yassl_imp.obj
 0001:0003f950       ?Register@?$Factory@VHandShakeBase@yaSSL@@HP6APAV12@XZ@yaSSL@@QAEXABHP6APAVHandShakeBase@2@XZ@Z 00440950 f i yassl:yassl_imp.obj
 0001:0003f980       ?Reserve@?$Factory@UServerKeyBase@yaSSL@@HP6APAU12@XZ@yaSSL@@QAEXI@Z 00440980 f i yassl:yassl_imp.obj
 0001:0003f9d0       ?Register@?$Factory@UServerKeyBase@yaSSL@@HP6APAU12@XZ@yaSSL@@QAEXABHP6APAUServerKeyBase@2@XZ@Z 004409d0 f i yassl:yassl_imp.obj
 0001:0003fa00       ?Reserve@?$Factory@UClientKeyBase@yaSSL@@HP6APAU12@XZ@yaSSL@@QAEXI@Z 00440a00 f i yassl:yassl_imp.obj
 0001:0003fa50       ?Register@?$Factory@UClientKeyBase@yaSSL@@HP6APAU12@XZ@yaSSL@@QAEXABHP6APAUClientKeyBase@2@XZ@Z 00440a50 f i yassl:yassl_imp.obj
 0001:0003fa80       ??_ECertificateRequest@yaSSL@@UAEPAXI@Z 00440a80 f i yassl:yassl_imp.obj
 0001:0003fa80       ??_GCertificateRequest@yaSSL@@UAEPAXI@Z 00440a80 f i yassl:yassl_imp.obj
 0001:0003faa0       ?InitMessageFactory@yaSSL@@YAXAAV?$Factory@UMessage@yaSSL@@HP6APAU12@XZ@1@@Z 00440aa0 f   yassl:yassl_imp.obj
 0001:0003fb60       ?InitHandShakeFactory@yaSSL@@YAXAAV?$Factory@VHandShakeBase@yaSSL@@HP6APAV12@XZ@1@@Z 00440b60 f   yassl:yassl_imp.obj
 0001:0003fcd0       ?InitServerKeyFactory@yaSSL@@YAXAAV?$Factory@UServerKeyBase@yaSSL@@HP6APAU12@XZ@1@@Z 00440cd0 f   yassl:yassl_imp.obj
 0001:0003fd70       ?InitClientKeyFactory@yaSSL@@YAXAAV?$Factory@UClientKeyBase@yaSSL@@HP6APAU12@XZ@1@@Z 00440d70 f   yassl:yassl_imp.obj
 0001:0003fe10       ??0Socket@yaSSL@@QAE@I@Z   00440e10 f   yassl:socket_wrapper.obj
 0001:0003fe30       ?set_fd@Socket@yaSSL@@QAEXI@Z 00440e30 f   yassl:socket_wrapper.obj
 0001:0003fe40       ?get_fd@Socket@yaSSL@@QBEIXZ 00440e40 f   yassl:socket_wrapper.obj
 0001:0003fe50       ??1Socket@yaSSL@@QAE@XZ    00440e50 f   yassl:socket_wrapper.obj
 0001:0003fe60       ?closeSocket@Socket@yaSSL@@QAEXXZ 00440e60 f   yassl:socket_wrapper.obj
 0001:0003fe80       ?get_ready@Socket@yaSSL@@QBEIXZ 00440e80 f   yassl:socket_wrapper.obj
 0001:0003fea0       ?send@Socket@yaSSL@@QBEIPBEIH@Z 00440ea0 f   yassl:socket_wrapper.obj
 0001:0003fef0       ?shutDown@Socket@yaSSL@@QAEXH@Z 00440ef0 f   yassl:socket_wrapper.obj
 0001:0003ff10       ?get_lastError@Socket@yaSSL@@SAHXZ 00440f10 f   yassl:socket_wrapper.obj
 0001:0003ff20       ?WouldBlock@Socket@yaSSL@@QBE_NXZ 00440f20 f   yassl:socket_wrapper.obj
 0001:0003ff30       ?IsNonBlocking@Socket@yaSSL@@QBE_NXZ 00440f30 f   yassl:socket_wrapper.obj
 0001:0003ff40       ?set_lastError@Socket@yaSSL@@SAXH@Z 00440f40 f   yassl:socket_wrapper.obj
 0001:0003ff50       ?receive@Socket@yaSSL@@QAEIPAEIH@Z 00440f50 f   yassl:socket_wrapper.obj
 0001:0003ffc0       ?wait@Socket@yaSSL@@QAE_NXZ 00440fc0 f   yassl:socket_wrapper.obj
 0001:0003ffe0       ??0Log@yaSSL@@QAE@PBD@Z    00440fe0 f   yassl:log.obj
 0001:0003fff0       ??1Log@yaSSL@@QAE@XZ       00440ff0 f   yassl:log.obj
 0001:00040000       ?Trace@Log@yaSSL@@QAEXPBD@Z 00441000 f   yassl:log.obj
 0001:00040010       ?ShowTCP@Log@yaSSL@@QAEXI_N@Z 00441010 f   yassl:log.obj
 0001:00040020       ?ShowData@Log@yaSSL@@QAEXI_N@Z 00441020 f   yassl:log.obj
 0001:00040030       ?buildClientHello@yaSSL@@YAXAAVSSL@1@AAVClientHello@1@@Z 00441030 f   yassl:handshake.obj
 0001:00040110       ?buildServerHello@yaSSL@@YAXAAVSSL@1@AAVServerHello@1@@Z 00441110 f   yassl:handshake.obj
 0001:000401f0       ?hashHandShake@yaSSL@@YAXAAVSSL@1@ABVinput_buffer@1@I@Z 004411f0 f   yassl:handshake.obj
 0001:00040250       ?buildOutput@?A0x7b3bc8e3@yaSSL@@YAXAAVoutput_buffer@2@ABURecordLayerHeader@2@ABUMessage@2@@Z 00441250 f   yassl:handshake.obj
 0001:00040290       ?buildOutput@?A0x7b3bc8e3@yaSSL@@YAXAAVoutput_buffer@2@ABURecordLayerHeader@2@ABVHandShakeHeader@2@ABVHandShakeBase@2@@Z 00441290 f   yassl:handshake.obj
 0001:000402e0       ?buildHeader@?A0x7b3bc8e3@yaSSL@@YAXAAVSSL@2@AAURecordLayerHeader@2@ABUMessage@2@@Z 004412e0 f   yassl:handshake.obj
 0001:00040330       ?buildHeaders@?A0x7b3bc8e3@yaSSL@@YAXAAVSSL@2@AAVHandShakeHeader@2@AAURecordLayerHeader@2@ABVHandShakeBase@2@@Z 00441330 f   yassl:handshake.obj
 0001:00040390       ?hashHandShake@?A0x7b3bc8e3@yaSSL@@YAXAAVSSL@2@ABVoutput_buffer@2@_N@Z 00441390 f   yassl:handshake.obj
 0001:00040410       ?buildMD5@?A0x7b3bc8e3@yaSSL@@YAXAAVSSL@2@AAVFinished@2@PBE@Z 00441410 f   yassl:handshake.obj
 0001:00040530       ?buildSHA@?A0x7b3bc8e3@yaSSL@@YAXAAVSSL@2@AAVFinished@2@PBE@Z 00441530 f   yassl:handshake.obj
 0001:00040660       ?decrypt_message@?A0x7b3bc8e3@yaSSL@@YAXAAVSSL@2@AAVinput_buffer@2@I@Z 00441660 f   yassl:handshake.obj
 0001:00040730       ??6?A0x7b3bc8e3@yaSSL@@YAAAVoutput_buffer@1@AAV21@ABVinput_buffer@1@@Z 00441730 f   yassl:handshake.obj
 0001:00040760       ??0RecordLayerHeader@yaSSL@@QAE@XZ 00441760 f i yassl:handshake.obj
 0001:00040780       ?get_xor@?A0x7b3bc8e3@yaSSL@@YAXPAEIAAVoutput_buffer@2@1@Z 00441780 f   yassl:handshake.obj
 0001:000407d0       ?buildMD5_CertVerify@?A0x7b3bc8e3@yaSSL@@YAXAAVSSL@2@PAE@Z 004417d0 f   yassl:handshake.obj
 0001:000408e0       ?buildSHA_CertVerify@?A0x7b3bc8e3@yaSSL@@YAXAAVSSL@2@PAE@Z 004418e0 f   yassl:handshake.obj
 0001:00040a00       ?hmac@yaSSL@@YAXAAVSSL@1@PAEPBEIW4ContentType@1@_N@Z 00441a00 f   yassl:handshake.obj
 0001:00040ba0       ?build_certHashes@yaSSL@@YAXAAVSSL@1@AAUHashes@1@@Z 00441ba0 f   yassl:handshake.obj
 0001:00040c90       ?sendClientHello@yaSSL@@YAXAAVSSL@1@@Z 00441c90 f   yassl:handshake.obj
 0001:00040db0       ??0?$auto_ptr@UDigest@yaSSL@@@mySTL@@QAE@PAUDigest@yaSSL@@@Z 00441db0 f i yassl:handshake.obj
 0001:00040dc0       ??C?$auto_ptr@UDigest@yaSSL@@@mySTL@@QBEPAUDigest@yaSSL@@XZ 00441dc0 f i yassl:handshake.obj
 0001:00040dd0       ??0?$auto_ptr@UMessage@yaSSL@@@mySTL@@QAE@PAUMessage@yaSSL@@@Z 00441dd0 f i yassl:handshake.obj
 0001:00040de0       ??C?$auto_ptr@UMessage@yaSSL@@@mySTL@@QBEPAUMessage@yaSSL@@XZ 00441de0 f i yassl:handshake.obj
 0001:00040df0       ??D?$auto_ptr@UMessage@yaSSL@@@mySTL@@QBEAAUMessage@yaSSL@@XZ 00441df0 f i yassl:handshake.obj
 0001:00040e00       ?get@?$auto_ptr@UMessage@yaSSL@@@mySTL@@QBEPAUMessage@yaSSL@@XZ 00441e00 f i yassl:handshake.obj
 0001:00040e10       ??0?$auto_ptr@Voutput_buffer@yaSSL@@@mySTL@@QAE@PAVoutput_buffer@yaSSL@@@Z 00441e10 f i yassl:handshake.obj
 0001:00040e20       ??C?$auto_ptr@Voutput_buffer@yaSSL@@@mySTL@@QBEPAVoutput_buffer@yaSSL@@XZ 00441e20 f i yassl:handshake.obj
 0001:00040e30       ?get@?$auto_ptr@Voutput_buffer@yaSSL@@@mySTL@@QBEPAVoutput_buffer@yaSSL@@XZ 00441e30 f i yassl:handshake.obj
 0001:00040e40       ?release@?$auto_ptr@Voutput_buffer@yaSSL@@@mySTL@@QAEPAVoutput_buffer@yaSSL@@XZ 00441e40 f i yassl:handshake.obj
 0001:00040e50       ?begin@?$vector@U?$pair@HP6APAUMessage@yaSSL@@XZ@mySTL@@@mySTL@@QBEPBU?$pair@HP6APAUMessage@yaSSL@@XZ@2@XZ 00441e50 f i yassl:handshake.obj
 0001:00040e60       ?end@?$vector@U?$pair@HP6APAUMessage@yaSSL@@XZ@mySTL@@@mySTL@@QBEPBU?$pair@HP6APAUMessage@yaSSL@@XZ@2@XZ 00441e60 f i yassl:handshake.obj
 0001:00040e70       ??$ysDelete@UMessage@yaSSL@@@yaSSL@@YAXPAUMessage@0@@Z 00441e70 f i yassl:handshake.obj
 0001:00040e90       ?ProcessOldClientHello@yaSSL@@YAXAAVinput_buffer@1@AAVSSL@1@@Z 00441e90 f   yassl:handshake.obj
 0001:00041120       ?CreateObject@?$Factory@UMessage@yaSSL@@HP6APAU12@XZ@yaSSL@@QBEPAUMessage@2@ABH@Z 00442120 f i yassl:handshake.obj
 0001:00041150       ?Destroy@?$auto_ptr@UDigest@yaSSL@@@mySTL@@AAEXXZ 00442150 f i yassl:handshake.obj
 0001:00041160       ?Destroy@?$auto_ptr@UMessage@yaSSL@@@mySTL@@AAEXXZ 00442160 f i yassl:handshake.obj
 0001:00041170       ??1?$auto_ptr@UDigest@yaSSL@@@mySTL@@QAE@XZ 00442170 f i yassl:handshake.obj
 0001:00041180       ?reset@?$auto_ptr@UDigest@yaSSL@@@mySTL@@QAEXPAUDigest@yaSSL@@@Z 00442180 f i yassl:handshake.obj
 0001:000411a0       ??1?$auto_ptr@UMessage@yaSSL@@@mySTL@@QAE@XZ 004421a0 f i yassl:handshake.obj
 0001:000411b0       ?Destroy@?$auto_ptr@Voutput_buffer@yaSSL@@@mySTL@@AAEXXZ 004421b0 f i yassl:handshake.obj
 0001:000411c0       ?p_hash@?A0x7b3bc8e3@yaSSL@@YAXAAVoutput_buffer@2@ABV32@1W4MACAlgorithm@2@@Z 004421c0 f   yassl:handshake.obj
 0001:00041360       ?TLS_hmac@yaSSL@@YAXAAVSSL@1@PAEPBEIW4ContentType@1@_N@Z 00442360 f   yassl:handshake.obj
 0001:00041500       ?PRF@yaSSL@@YAXPAEIPBEI1I1I@Z 00442500 f   yassl:handshake.obj
 0001:00041630       ?DoProcessReply@yaSSL@@YAHAAVSSL@1@@Z 00442630 f   yassl:handshake.obj
 0001:00041980       ?processReply@yaSSL@@YAXAAVSSL@1@@Z 00442980 f   yassl:handshake.obj
 0001:000419f0       ?receiveData@yaSSL@@YAHAAVSSL@1@AAVData@1@_N@Z 004429f0 f   yassl:handshake.obj
 0001:00041ac0       ??1?$auto_ptr@Voutput_buffer@yaSSL@@@mySTL@@QAE@XZ 00442ac0 f i yassl:handshake.obj
 0001:00041ad0       ?cipherFinished@?A0x7b3bc8e3@yaSSL@@YAXAAVSSL@2@AAVFinished@2@AAVoutput_buffer@2@@Z 00442ad0 f   yassl:handshake.obj
 0001:00041db0       ?buildMessage@?A0x7b3bc8e3@yaSSL@@YAXAAVSSL@2@AAVoutput_buffer@2@ABUMessage@2@@Z 00442db0 f   yassl:handshake.obj
 0001:00042070       ?buildAlert@?A0x7b3bc8e3@yaSSL@@YAXAAVSSL@2@AAVoutput_buffer@2@ABVAlert@2@@Z 00443070 f   yassl:handshake.obj
 0001:000420e0       ?buildFinishedTLS@?A0x7b3bc8e3@yaSSL@@YAXAAVSSL@2@AAVFinished@2@PBE@Z 004430e0 f   yassl:handshake.obj
 0001:000421a0       ?buildFinished@yaSSL@@YAXAAVSSL@1@AAVFinished@1@PBE@Z 004431a0 f   yassl:handshake.obj
 0001:00042270       ?sendClientKeyExchange@yaSSL@@YAXAAVSSL@1@W4BufferOutput@1@@Z 00443270 f   yassl:handshake.obj
 0001:00042380       ?sendServerKeyExchange@yaSSL@@YAXAAVSSL@1@W4BufferOutput@1@@Z 00443380 f   yassl:handshake.obj
 0001:00042480       ?sendChangeCipher@yaSSL@@YAXAAVSSL@1@W4BufferOutput@1@@Z 00443480 f   yassl:handshake.obj
 0001:00042570       ?sendFinished@yaSSL@@YAXAAVSSL@1@W4ConnectionEnd@1@W4BufferOutput@1@@Z 00443570 f   yassl:handshake.obj
 0001:000426b0       ?sendData@yaSSL@@YAHAAVSSL@1@PBXH@Z 004436b0 f   yassl:handshake.obj
 0001:00042820       ?sendAlert@yaSSL@@YAHAAVSSL@1@ABVAlert@1@@Z 00443820 f   yassl:handshake.obj
 0001:00042880       ?sendServerHello@yaSSL@@YAXAAVSSL@1@W4BufferOutput@1@@Z 00443880 f   yassl:handshake.obj
 0001:000429d0       ?sendServerHelloDone@yaSSL@@YAXAAVSSL@1@W4BufferOutput@1@@Z 004439d0 f   yassl:handshake.obj
 0001:00042ab0       ?sendCertificate@yaSSL@@YAXAAVSSL@1@W4BufferOutput@1@@Z 00443ab0 f   yassl:handshake.obj
 0001:00042ba0       ?sendCertificateRequest@yaSSL@@YAXAAVSSL@1@W4BufferOutput@1@@Z 00443ba0 f   yassl:handshake.obj
 0001:00042ca0       ?sendCertificateVerify@yaSSL@@YAXAAVSSL@1@W4BufferOutput@1@@Z 00443ca0 f   yassl:handshake.obj
 0001:00042da0       ?GetKey@PublicKey@TaoCrypt@@QBEPBEXZ 00443da0 f i yassl:cert_wrapper.obj
 0001:00042db0       ?size@PublicKey@TaoCrypt@@QBEIXZ 00443db0 f i yassl:cert_wrapper.obj
 0001:00042dc0       ?GetPublicKey@CertDecoder@TaoCrypt@@QBEABVPublicKey@2@XZ 00443dc0 f i yassl:cert_wrapper.obj
 0001:00042dd0       ?GetKeyType@CertDecoder@TaoCrypt@@QBE?AW4KeyType@2@XZ 00443dd0 f i yassl:cert_wrapper.obj
 0001:00042de0       ?GetIssuer@CertDecoder@TaoCrypt@@QBEPBDXZ 00443de0 f i yassl:cert_wrapper.obj
 0001:00042df0       ?GetCommonName@CertDecoder@TaoCrypt@@QBEPBDXZ 00443df0 f i yassl:cert_wrapper.obj
 0001:00042e00       ?GetHash@CertDecoder@TaoCrypt@@QBEPBEXZ 00443e00 f i yassl:cert_wrapper.obj
 0001:00042e10       ?GetBeforeDate@CertDecoder@TaoCrypt@@QBEPBDXZ 00443e10 f i yassl:cert_wrapper.obj
 0001:00042e20       ?GetAfterDate@CertDecoder@TaoCrypt@@QBEPBDXZ 00443e20 f i yassl:cert_wrapper.obj
 0001:00042e30       ??0x509@yaSSL@@QAE@I@Z     00443e30 f   yassl:cert_wrapper.obj
 0001:00042e50       ??0x509@yaSSL@@QAE@ABV01@@Z 00443e50 f   yassl:cert_wrapper.obj
 0001:00042e80       ?get_length@x509@yaSSL@@QBEIXZ 00443e80 f   yassl:cert_wrapper.obj
 0001:00042e90       ?get_buffer@x509@yaSSL@@QBEPBEXZ 00443e90 f   yassl:cert_wrapper.obj
 0001:00042ea0       ?use_buffer@x509@yaSSL@@QAEPAEXZ 00443ea0 f   yassl:cert_wrapper.obj
 0001:00042eb0       ?verifyPeer@CertManager@yaSSL@@QBE_NXZ 00443eb0 f   yassl:cert_wrapper.obj
 0001:00042ec0       ?verifyNone@CertManager@yaSSL@@QBE_NXZ 00443ec0 f   yassl:cert_wrapper.obj
 0001:00042ed0       ?failNoCert@CertManager@yaSSL@@QBE_NXZ 00443ed0 f   yassl:cert_wrapper.obj
 0001:00042ee0       ?sendVerify@CertManager@yaSSL@@QBE_NXZ 00443ee0 f   yassl:cert_wrapper.obj
 0001:00042ef0       ?setVerifyPeer@CertManager@yaSSL@@QAEXXZ 00443ef0 f   yassl:cert_wrapper.obj
 0001:00042f00       ?setVerifyNone@CertManager@yaSSL@@QAEXXZ 00443f00 f   yassl:cert_wrapper.obj
 0001:00042f10       ?setFailNoCert@CertManager@yaSSL@@QAEXXZ 00443f10 f   yassl:cert_wrapper.obj
 0001:00042f20       ?setSendVerify@CertManager@yaSSL@@QAEXXZ 00443f20 f   yassl:cert_wrapper.obj
 0001:00042f30       ?setVerifyCallback@CertManager@yaSSL@@QAEXP6AHHPAUX509_STORE_CTX@2@@Z@Z 00443f30 f   yassl:cert_wrapper.obj
 0001:00042f40       ?get_peerKey@CertManager@yaSSL@@QBEPBEXZ 00443f40 f   yassl:cert_wrapper.obj
 0001:00042f50       ?get_peerX509@CertManager@yaSSL@@QBEPAVX509@2@XZ 00443f50 f   yassl:cert_wrapper.obj
 0001:00042f60       ?get_peerKeyType@CertManager@yaSSL@@QBE?AW4SignatureAlgorithm@2@XZ 00443f60 f   yassl:cert_wrapper.obj
 0001:00042f70       ?get_keyType@CertManager@yaSSL@@QBE?AW4SignatureAlgorithm@2@XZ 00443f70 f   yassl:cert_wrapper.obj
 0001:00042f80       ?get_peerKeyLength@CertManager@yaSSL@@QBEIXZ 00443f80 f   yassl:cert_wrapper.obj
 0001:00042f90       ?get_privateKey@CertManager@yaSSL@@QBEPBEXZ 00443f90 f   yassl:cert_wrapper.obj
 0001:00042fa0       ?get_privateKeyLength@CertManager@yaSSL@@QBEIXZ 00443fa0 f   yassl:cert_wrapper.obj
 0001:00042fb0       ?setPeerX509@CertManager@yaSSL@@QAEXPAVX509@2@@Z 00443fb0 f   yassl:cert_wrapper.obj
 0001:00043060       ?size@?$list@PAVx509@yaSSL@@@mySTL@@QBEIXZ 00444060 f i yassl:cert_wrapper.obj
 0001:00043070       ??0?$list@PAVSigner@TaoCrypt@@@mySTL@@QAE@XZ 00444070 f i yassl:cert_wrapper.obj
 0001:00043080       ??Dreverse_iterator@?$list@PAVx509@yaSSL@@@mySTL@@QBEAAPAVx509@yaSSL@@XZ 00444080 f i yassl:cert_wrapper.obj
 0001:00043090       ??Ereverse_iterator@?$list@PAVx509@yaSSL@@@mySTL@@QAEAAV012@XZ 00444090 f i yassl:cert_wrapper.obj
 0001:000430a0       ??0iterator@?$list@PAVSigner@TaoCrypt@@@mySTL@@QAE@PAUnode@12@@Z 004440a0 f i yassl:cert_wrapper.obj
 0001:000430b0       ??0reverse_iterator@?$list@PAVx509@yaSSL@@@mySTL@@QAE@PAUnode@12@@Z 004440b0 f i yassl:cert_wrapper.obj
 0001:000430c0       ?front@?$list@PAVx509@yaSSL@@@mySTL@@QBEPAVx509@yaSSL@@XZ 004440c0 f i yassl:cert_wrapper.obj
 0001:000430d0       ??$swap@I@mySTL@@YAXAAI0@Z 004440d0 f i yassl:cert_wrapper.obj
 0001:000430f0       ??Diterator@?$list@PAVSigner@TaoCrypt@@@mySTL@@QBEAAPAVSigner@TaoCrypt@@XZ 004440f0 f i yassl:cert_wrapper.obj
 0001:00043100       ??Eiterator@?$list@PAVSigner@TaoCrypt@@@mySTL@@QAEAAV012@XZ 00444100 f i yassl:cert_wrapper.obj
 0001:00043110       ??9iterator@?$list@PAVSigner@TaoCrypt@@@mySTL@@QBE_NABV012@@Z 00444110 f i yassl:cert_wrapper.obj
 0001:00043130       ??0node@?$list@PAVSigner@TaoCrypt@@@mySTL@@QAE@PAVSigner@TaoCrypt@@@Z 00444130 f i yassl:cert_wrapper.obj
 0001:00043150       ??$destroy@Unode@?$list@PAVSigner@TaoCrypt@@@mySTL@@@mySTL@@YAXPAUnode@?$list@PAVSigner@TaoCrypt@@@0@@Z 00444150 f i yassl:cert_wrapper.obj
 0001:00043160       ??$swap@PAVSigner@TaoCrypt@@@mySTL@@YAXAAPAVSigner@TaoCrypt@@0@Z 00444160 f i yassl:cert_wrapper.obj
 0001:00043180       ??_GSigner@TaoCrypt@@QAEPAXI@Z 00444180 f i yassl:cert_wrapper.obj
 0001:000431a0       ??1x509@yaSSL@@QAE@XZ      004441a0 f   yassl:cert_wrapper.obj
 0001:000431b0       ?Swap@x509@yaSSL@@AAEXAAV12@@Z 004441b0 f   yassl:cert_wrapper.obj
 0001:000431d0       ??4x509@yaSSL@@QAEAAV01@ABV01@@Z 004441d0 f   yassl:cert_wrapper.obj
 0001:00043210       ?get_cert@CertManager@yaSSL@@QBEPBVx509@2@XZ 00444210 f   yassl:cert_wrapper.obj
 0001:00043220       ?rbegin@?$list@PAVx509@yaSSL@@@mySTL@@QBE?AVreverse_iterator@12@XZ 00444220 f i yassl:cert_wrapper.obj
 0001:00043230       ?begin@?$list@PAVSigner@TaoCrypt@@@mySTL@@QBE?AViterator@12@XZ 00444230 f i yassl:cert_wrapper.obj
 0001:00043240       ?end@?$list@PAVSigner@TaoCrypt@@@mySTL@@QBE?AViterator@12@XZ 00444240 f i yassl:cert_wrapper.obj
 0001:00043250       ?push_back@?$list@PAVSigner@TaoCrypt@@@mySTL@@QAEXPAVSigner@TaoCrypt@@@Z 00444250 f i yassl:cert_wrapper.obj
 0001:000432a0       ??$ysDelete@VSigner@TaoCrypt@@@yaSSL@@YAXPAVSigner@TaoCrypt@@@Z 004442a0 f i yassl:cert_wrapper.obj
 0001:000432c0       ?AddPeerCert@CertManager@yaSSL@@QAEXPAVx509@2@@Z 004442c0 f   yassl:cert_wrapper.obj
 0001:000432d0       ?CopySelfCert@CertManager@yaSSL@@QAEXPBVx509@2@@Z 004442d0 f   yassl:cert_wrapper.obj
 0001:00043310       ??1?$list@PAVSigner@TaoCrypt@@@mySTL@@QAE@XZ 00444310 f i yassl:cert_wrapper.obj
 0001:00043330       ??$checked_delete@VSigner@TaoCrypt@@@yaSSL@@YAXPAVSigner@TaoCrypt@@@Z 00444330 f i yassl:cert_wrapper.obj
 0001:00043340       ??0CertManager@yaSSL@@QAE@XZ 00444340 f   yassl:cert_wrapper.obj
 0001:00043390       ?CopyCaCert@CertManager@yaSSL@@QAEHPBVx509@2@@Z 00444390 f   yassl:cert_wrapper.obj
 0001:000434a0       ?Validate@CertManager@yaSSL@@QAEHXZ 004444a0 f   yassl:cert_wrapper.obj
 0001:00043760       ?SetPrivateKey@CertManager@yaSSL@@QAEHABVx509@2@@Z 00444760 f   yassl:cert_wrapper.obj
 0001:000438b0       ??$?RVSigner@TaoCrypt@@@del_ptr_zero@yaSSL@@QBEXAAPAVSigner@TaoCrypt@@@Z 004448b0 f i yassl:cert_wrapper.obj
 0001:000438d0       ??$for_each@Viterator@?$list@PAVSigner@TaoCrypt@@@mySTL@@Udel_ptr_zero@yaSSL@@@mySTL@@YA?AUdel_ptr_zero@yaSSL@@Viterator@?$list@PAVSigner@TaoCrypt@@@0@0U12@@Z 004448d0 f i yassl:cert_wrapper.obj
 0001:00043910       ??1CertManager@yaSSL@@QAE@XZ 00444910 f   yassl:cert_wrapper.obj
 0001:000439a0       ?SetErrorString@yaSSL@@YAXKPAD@Z 004449a0 f   yassl:yassl_error.obj
 0001:00043fa0       ?check@Check@yaSSL@@QAEXII@Z 00444fa0 f   yassl:buffer.obj
 0001:00043fb0       ?check@NoCheck@yaSSL@@QAEXII@Z 00444fb0 f   yassl:buffer.obj
 0001:00043fc0       ??0input_buffer@yaSSL@@QAE@XZ 00444fc0 f   yassl:buffer.obj
 0001:00043fd0       ??0input_buffer@yaSSL@@QAE@I@Z 00444fd0 f   yassl:buffer.obj
 0001:00044000       ?allocate@input_buffer@yaSSL@@QAEXI@Z 00445000 f   yassl:buffer.obj
 0001:00044020       ?get_buffer@input_buffer@yaSSL@@QBEPAEXZ 00445020 f   yassl:buffer.obj
 0001:00044030       ?get_capacity@input_buffer@yaSSL@@QBEIXZ 00445030 f   yassl:buffer.obj
 0001:00044040       ?get_current@input_buffer@yaSSL@@QBEIXZ 00445040 f   yassl:buffer.obj
 0001:00044050       ?get_size@input_buffer@yaSSL@@QBEIXZ 00445050 f   yassl:buffer.obj
 0001:00044060       ?get_remaining@input_buffer@yaSSL@@QBEIXZ 00445060 f   yassl:buffer.obj
 0001:00044070       ?set_current@input_buffer@yaSSL@@QAEXI@Z 00445070 f   yassl:buffer.obj
 0001:00044080       ??Ainput_buffer@yaSSL@@QAEABEI@Z 00445080 f   yassl:buffer.obj
 0001:000440a0       ?eof@input_buffer@yaSSL@@QAE_NXZ 004450a0 f   yassl:buffer.obj
 0001:000440b0       ?peek@input_buffer@yaSSL@@QBEEXZ 004450b0 f   yassl:buffer.obj
 0001:000440c0       ?read@input_buffer@yaSSL@@QAEXPAEI@Z 004450c0 f   yassl:buffer.obj
 0001:000440f0       ??0output_buffer@yaSSL@@QAE@XZ 004450f0 f   yassl:buffer.obj
 0001:00044100       ??0output_buffer@yaSSL@@QAE@I@Z 00445100 f   yassl:buffer.obj
 0001:00044130       ?get_size@output_buffer@yaSSL@@QBEIXZ 00445130 f   yassl:buffer.obj
 0001:00044140       ?get_capacity@output_buffer@yaSSL@@QBEIXZ 00445140 f   yassl:buffer.obj
 0001:00044150       ?set_current@output_buffer@yaSSL@@QAEXI@Z 00445150 f   yassl:buffer.obj
 0001:00044160       ?allocate@output_buffer@yaSSL@@QAEXI@Z 00445160 f   yassl:buffer.obj
 0001:00044180       ?get_buffer@output_buffer@yaSSL@@QBEPBEXZ 00445180 f   yassl:buffer.obj
 0001:00044190       ??Aoutput_buffer@yaSSL@@QAEAAEI@Z 00445190 f   yassl:buffer.obj
 0001:000441a0       ?eof@output_buffer@yaSSL@@QAE_NXZ 004451a0 f   yassl:buffer.obj
 0001:000441b0       ?write@output_buffer@yaSSL@@QAEXPBEI@Z 004451b0 f   yassl:buffer.obj
 0001:000441e0       ??1input_buffer@yaSSL@@QAE@XZ 004451e0 f   yassl:buffer.obj
 0001:000441f0       ?add_size@input_buffer@yaSSL@@QAEXI@Z 004451f0 f   yassl:buffer.obj
 0001:00044200       ?assign@input_buffer@yaSSL@@QAEXPBEI@Z 00445200 f   yassl:buffer.obj
 0001:00044230       ??0output_buffer@yaSSL@@QAE@IPBEI@Z 00445230 f   yassl:buffer.obj
 0001:00044270       ??1output_buffer@yaSSL@@QAE@XZ 00445270 f   yassl:buffer.obj
 0001:00044280       ??0input_buffer@yaSSL@@QAE@IPBEI@Z 00445280 f   yassl:buffer.obj
 0001:000442c0       ?timer@yaSSL@@YANXZ        004452c0 f   yassl:timer.obj
 0001:00044300       ?lowResTimer@yaSSL@@YAIXZ  00445300 f   yassl:timer.obj
 0001:00044330       _compress2                 00445330 f   zlib:compress.obj
 0001:000443e0       _compress                  004453e0 f   zlib:compress.obj
 0001:00044400       _compressBound             00445400 f   zlib:compress.obj
 0001:00044420       _uncompress                00445420 f   zlib:uncompr.obj
 0001:000444d0       _deflateSetDictionary      004454d0 f   zlib:deflate.obj
 0001:000445d0       _deflateSetHeader          004455d0 f   zlib:deflate.obj
 0001:00044600       _deflatePrime              00445600 f   zlib:deflate.obj
 0001:00044640       _deflateTune               00445640 f   zlib:deflate.obj
 0001:00044680       _deflateBound              00445680 f   zlib:deflate.obj
 0001:00044740       _deflate                   00445740 f   zlib:deflate.obj
 0001:00044f20       _deflateEnd                00445f20 f   zlib:deflate.obj
 0001:00045000       _deflateCopy               00446000 f   zlib:deflate.obj
 0001:00045e20       _deflateReset              00446e20 f   zlib:deflate.obj
 0001:00045eb0       _deflateParams             00446eb0 f   zlib:deflate.obj
 0001:00045f80       _deflateInit2_             00446f80 f   zlib:deflate.obj
 0001:000461a0       _deflateInit_              004471a0 f   zlib:deflate.obj
 0001:000461d0       _inflateReset              004471d0 f   zlib:inflate.obj
 0001:00046230       _inflatePrime              00447230 f   zlib:inflate.obj
 0001:00046280       _inflateInit2_             00447280 f   zlib:inflate.obj
 0001:00046350       _inflateInit_              00447350 f   zlib:inflate.obj
 0001:00046480       _inflate                   00447480 f   zlib:inflate.obj
 0001:00047a70       _inflateEnd                00448a70 f   zlib:inflate.obj
 0001:00047ac0       _inflateSetDictionary      00448ac0 f   zlib:inflate.obj
 0001:00047ba0       _inflateGetHeader          00448ba0 f   zlib:inflate.obj
 0001:00047c30       _inflateSync               00448c30 f   zlib:inflate.obj
 0001:00047d10       _inflateSyncPoint          00448d10 f   zlib:inflate.obj
 0001:00047d40       _inflateCopy               00448d40 f   zlib:inflate.obj
 0001:00047e90       _adler32                   00448e90 f   zlib:adler32.obj
 0001:00048110       _adler32_combine           00449110 f   zlib:adler32.obj
 0001:00048d80       __tr_tally                 00449d80 f   zlib:trees.obj
 0001:000494b0       __tr_init                  0044a4b0 f   zlib:trees.obj
 0001:00049870       __tr_stored_block          0044a870 f   zlib:trees.obj
 0001:00049910       __tr_align                 0044a910 f   zlib:trees.obj
 0001:00049b00       __tr_flush_block           0044ab00 f   zlib:trees.obj
 0001:00049d10       _get_crc_table             0044ad10 f   zlib:crc32.obj
 0001:0004a300       _crc32_combine             0044b300 f   zlib:crc32.obj
 0001:0004a3e0       _crc32                     0044b3e0 f   zlib:crc32.obj
 0001:0004a400       _zlibVersion               0044b400 f   zlib:zutil.obj
 0001:0004a410       _zlibCompileFlags          0044b410 f   zlib:zutil.obj
 0001:0004a420       _zError                    0044b420 f   zlib:zutil.obj
 0001:0004a440       _zcalloc                   0044b440 f   zlib:zutil.obj
 0001:0004a460       _zcfree                    0044b460 f   zlib:zutil.obj
 0001:0004a470       _inflate_fast              0044b470 f   zlib:inffast.obj
 0001:0004a930       _inflate_table             0044b930 f   zlib:inftrees.obj
 0001:0004ae1e       _gethostname@8             0044be1e f   wsock32:WSOCK32.dll
 0001:0004ae24       _ioctlsocket@12            0044be24 f   wsock32:WSOCK32.dll
 0001:0004ae2a       _closesocket@4             0044be2a f   wsock32:WSOCK32.dll
 0001:0004ae30       _listen@8                  0044be30 f   wsock32:WSOCK32.dll
 0001:0004ae36       _bind@12                   0044be36 f   wsock32:WSOCK32.dll
 0001:0004ae3c       _setsockopt@20             0044be3c f   wsock32:WSOCK32.dll
 0001:0004ae42       _htons@4                   0044be42 f   wsock32:WSOCK32.dll
 0001:0004ae48       _htonl@4                   0044be48 f   wsock32:WSOCK32.dll
 0001:0004ae4e       _inet_addr@4               0044be4e f   wsock32:WSOCK32.dll
 0001:0004ae54       _socket@12                 0044be54 f   wsock32:WSOCK32.dll
 0001:0004ae5a       _shutdown@8                0044be5a f   wsock32:WSOCK32.dll
 0001:0004ae60       _accept@12                 0044be60 f   wsock32:WSOCK32.dll
 0001:0004ae66       ___WSAFDIsSet@8            0044be66 f   wsock32:WSOCK32.dll
 0001:0004ae6c       _select@20                 0044be6c f   wsock32:WSOCK32.dll
 0001:0004ae72       _connect@12                0044be72 f   wsock32:WSOCK32.dll
 0001:0004ae78       _WSAGetLastError@0         0044be78 f   wsock32:WSOCK32.dll
 0001:0004ae7e       _WSACleanup@0              0044be7e f   wsock32:WSOCK32.dll
 0001:0004ae84       _WSAStartup@8              0044be84 f   wsock32:WSOCK32.dll
 0001:0004ae8a       _gethostbyname@4           0044be8a f   wsock32:WSOCK32.dll
 0001:0004ae90       _recv@16                   0044be90 f   wsock32:WSOCK32.dll
 0001:0004ae96       _send@16                   0044be96 f   wsock32:WSOCK32.dll
 0001:0004ae9c       _ntohs@4                   0044be9c f   wsock32:WSOCK32.dll
 0001:0004aea2       _getpeername@12            0044bea2 f   wsock32:WSOCK32.dll
 0001:0004aea8       _WSASetLastError@4         0044bea8 f   wsock32:WSOCK32.dll
 0001:0004aeae       ??_U@YAPAXI@Z              0044beae f   libcpmt:newaop.obj
 0001:0004aeb3       __fpclear                  0044beb3 f   LIBCMT:fpinit.obj
 0001:0004aeb4       __cfltcvt_init             0044beb4 f   LIBCMT:fpinit.obj
 0001:0004af14       ___setfflag                0044bf14 f   LIBCMT:fpinit.obj
 0001:0004af24       __fpmath                   0044bf24 f   LIBCMT:fpinit.obj
 0001:0004af42       ?name@type_info@@QBEPBDPAU__type_info_node@@@Z 0044bf42 f   LIBCMT:typinfo.obj
 0001:0004af51       ??1type_info@@UAE@XZ       0044bf51 f   LIBCMT:typinfo.obj
 0001:0004af5f       ??_Gtype_info@@UAEPAXI@Z   0044bf5f f i LIBCMT:typinfo.obj
 0001:0004af5f       ??_Etype_info@@UAEPAXI@Z   0044bf5f f i LIBCMT:typinfo.obj
 0001:0004af7b       ?_name_internal_method@type_info@@QBEPBDPAU__type_info_node@@@Z 0044bf7b f   LIBCMT:typinfo.obj
 0001:0004af8a       ?_type_info_dtor_internal_method@type_info@@QAEXXZ 0044bf8a f   LIBCMT:typinfo.obj
 0001:0004af92       ??8type_info@@QBE_NABV0@@Z 0044bf92 f   LIBCMT:typinfo.obj
 0001:0004afad       ??9type_info@@QBE_NABV0@@Z 0044bfad f   LIBCMT:typinfo.obj
 0001:0004afc9       ?before@type_info@@QBEHABV1@@Z 0044bfc9 f   LIBCMT:typinfo.obj
 0001:0004afe8       ?raw_name@type_info@@QBEPBDXZ 0044bfe8 f   LIBCMT:typinfo.obj
 0001:0004afec       ??0type_info@@AAE@ABV0@@Z  0044bfec f   LIBCMT:typinfo.obj
 0001:0004aff7       ??4type_info@@AAEAAV0@ABV0@@Z 0044bff7 f   LIBCMT:typinfo.obj
 0001:0004affc       __purecall                 0044bffc f   LIBCMT:purevirt.obj
 0001:0004b026       __set_purecall_handler     0044c026 f   LIBCMT:purevirt.obj
 0001:0004b048       __get_purecall_handler     0044c048 f   LIBCMT:purevirt.obj
 0001:0004b055       ??3@YAXPAX@Z               0044c055 f   LIBCMT:delete.obj
 0001:0004b130       __stat64i32                0044c130 f   LIBCMT:stati32.obj
 0001:0004b470       _strncpy                   0044c470 f   LIBCMT:strncpy.obj
 0001:0004b594       @__security_check_cookie@4 0044c594 f   LIBCMT:secchk.obj
 0001:0004b5a3       ??0bad_alloc@std@@QAE@XZ   0044c5a3 f i LIBCMT:new.obj
 0001:0004b5bc       ??1bad_alloc@std@@UAE@XZ   0044c5bc f i LIBCMT:new.obj
 0001:0004b5c7       ??_Gbad_alloc@std@@UAEPAXI@Z 0044c5c7 f i LIBCMT:new.obj
 0001:0004b5c7       ??_Ebad_alloc@std@@UAEPAXI@Z 0044c5c7 f i LIBCMT:new.obj
 0001:0004b5e9       ??0bad_alloc@std@@QAE@ABV01@@Z 0044c5e9 f i LIBCMT:new.obj
 0001:0004b601       ??2@YAPAXI@Z               0044c601 f   LIBCMT:new.obj
 0001:0004b66b       __time64                   0044c66b f   LIBCMT:time64.obj
 0001:0004b6b0       _memset                    0044c6b0 f   LIBCMT:memset.obj
 0001:0004b72a       _strncmp                   0044c72a f   LIBCMT:strncmp.obj
 0001:0004b800       _strchr                    0044c800 f   LIBCMT:strchr.obj
 0001:0004b806       ___from_strstr_to_strchr   0044c806     LIBCMT:strchr.obj
 0001:0004b8be       __invoke_watson_if_error   0044c8be f i LIBCMT:strerror.obj
 0001:0004b8e0       __get_sys_err_msg          0044c8e0 f i LIBCMT:strerror.obj
 0001:0004b903       _strerror                  0044c903 f   LIBCMT:strerror.obj
 0001:0004b96a       _strerror_s                0044c96a f   LIBCMT:strerror.obj
 0001:0004b9c9       __get_errno_from_oserr     0044c9c9 f   LIBCMT:dosmap.obj
 0001:0004ba04       __errno                    0044ca04 f   LIBCMT:dosmap.obj
 0001:0004ba17       ___doserrno                0044ca17 f   LIBCMT:dosmap.obj
 0001:0004ba2a       __dosmaperr                0044ca2a f   LIBCMT:dosmap.obj
 0001:0004ba48       __set_errno                0044ca48 f   LIBCMT:dosmap.obj
 0001:0004ba63       __get_errno                0044ca63 f   LIBCMT:dosmap.obj
 0001:0004ba8d       __set_doserrno             0044ca8d f   LIBCMT:dosmap.obj
 0001:0004baa8       __get_doserrno             0044caa8 f   LIBCMT:dosmap.obj
 0001:0004bad2       __snprintf                 0044cad2 f   LIBCMT:snprintf.obj
 0001:0004bb7f       __snprintf_l               0044cb7f f   LIBCMT:snprintf.obj
 0001:0004bba0       _strstr                    0044cba0 f   LIBCMT:strstr.obj
 0001:0004bc26       _vfscanf                   0044cc26 f   LIBCMT:fscanf.obj
 0001:0004bd63       _fscanf                    0044cd63 f   LIBCMT:fscanf.obj
 0001:0004bd80       __fscanf_l                 0044cd80 f   LIBCMT:fscanf.obj
 0001:0004bd9f       _fscanf_s                  0044cd9f f   LIBCMT:fscanf.obj
 0001:0004bdbc       __fscanf_s_l               0044cdbc f   LIBCMT:fscanf.obj
 0001:0004bddb       _printf                    0044cddb f   LIBCMT:printf.obj
 0001:0004be8a       __printf_l                 0044ce8a f   LIBCMT:printf.obj
 0001:0004bea0       __printf_s_l               0044cea0 f   LIBCMT:printf.obj
 0001:0004beb6       _printf_s                  0044ceb6 f   LIBCMT:printf.obj
 0001:0004beca       __printf_p_l               0044ceca f   LIBCMT:printf.obj
 0001:0004bee0       __printf_p                 0044cee0 f   LIBCMT:printf.obj
 0001:0004bef4       __set_printf_count_output  0044cef4 f   LIBCMT:printf.obj
 0001:0004bf19       __get_printf_count_output  0044cf19 f   LIBCMT:printf.obj
 0001:0004bf2f       _atol                      0044cf2f f   LIBCMT:atox.obj
 0001:0004bf40       __atol_l                   0044cf40 f   LIBCMT:atox.obj
 0001:0004bf55       _atoi                      0044cf55 f   LIBCMT:atox.obj
 0001:0004bf5a       __atoi_l                   0044cf5a f   LIBCMT:atox.obj
 0001:0004bf5f       __atoi64                   0044cf5f f   LIBCMT:atox.obj
 0001:0004bf70       __atoi64_l                 0044cf70 f   LIBCMT:atox.obj
 0001:0004bf85       _fprintf                   0044cf85 f   LIBCMT:fprintf.obj
 0001:0004c0d4       __fprintf_l                0044d0d4 f   LIBCMT:fprintf.obj
 0001:0004c0ee       __fprintf_s_l              0044d0ee f   LIBCMT:fprintf.obj
 0001:0004c108       _fprintf_s                 0044d108 f   LIBCMT:fprintf.obj
 0001:0004c120       __fprintf_p_l              0044d120 f   LIBCMT:fprintf.obj
 0001:0004c13a       __fprintf_p                0044d13a f   LIBCMT:fprintf.obj
 0001:0004c152       __vsnprintf_l              0044d152 f   LIBCMT:vsnprint.obj
 0001:0004c203       __vsnprintf                0044d203 f   LIBCMT:vsnprint.obj
 0001:0004c21e       _sprintf                   0044d21e f   LIBCMT:sprintf.obj
 0001:0004c299       __sprintf_l                0044d299 f   LIBCMT:sprintf.obj
 0001:0004c2b3       _sprintf_s                 0044d2b3 f   LIBCMT:sprintf.obj
 0001:0004c2cf       __sprintf_s_l              0044d2cf f   LIBCMT:sprintf.obj
 0001:0004c2ec       __snprintf_s               0044d2ec f   LIBCMT:sprintf.obj
 0001:0004c30b       __snprintf_s_l             0044d30b f   LIBCMT:sprintf.obj
 0001:0004c32b       __sprintf_p                0044d32b f   LIBCMT:sprintf.obj
 0001:0004c347       __sprintf_p_l              0044d347 f   LIBCMT:sprintf.obj
 0001:0004c364       __scprintf                 0044d364 f   LIBCMT:sprintf.obj
 0001:0004c375       __scprintf_p               0044d375 f   LIBCMT:sprintf.obj
 0001:0004c386       __scprintf_l               0044d386 f   LIBCMT:sprintf.obj
 0001:0004c39c       __scprintf_p_l             0044d39c f   LIBCMT:sprintf.obj
 0001:0004c3b2       _setbuf                    0044d3b2 f   LIBCMT:setbuf.obj
 0001:0004c3d7       ___iob_func                0044d3d7 f   LIBCMT:_file.obj
 0001:0004c3dd       ___initstdio               0044d3dd f   LIBCMT:_file.obj
 0001:0004c48e       ___endstdio                0044d48e f   LIBCMT:_file.obj
 0001:0004c4ae       __lock_file                0044d4ae f   LIBCMT:_file.obj
 0001:0004c4ea       __lock_file2               0044d4ea f   LIBCMT:_file.obj
 0001:0004c518       __unlock_file              0044d518 f   LIBCMT:_file.obj
 0001:0004c54e       __unlock_file2             0044d54e f   LIBCMT:_file.obj
 0001:0004c578       __flush                    0044d578 f   LIBCMT:fflush.obj
 0001:0004c5da       __fflush_nolock            0044d5da f   LIBCMT:fflush.obj
 0001:0004c6f6       _fflush                    0044d6f6 f   LIBCMT:fflush.obj
 0001:0004c749       __flushall                 0044d749 f   LIBCMT:fflush.obj
 0001:0004c752       __amsg_exit                0044d752 f   LIBCMT:crt0dat.obj
 0001:0004c776       ___crtCorExitProcess       0044d776 f   LIBCMT:crt0dat.obj
 0001:0004c79c       ___crtExitProcess          0044d79c f   LIBCMT:crt0dat.obj
 0001:0004c7b1       __lockexit                 0044d7b1 f   LIBCMT:crt0dat.obj
 0001:0004c7ba       __unlockexit               0044d7ba f   LIBCMT:crt0dat.obj
 0001:0004c7db       __initterm_e               0044d7db f   LIBCMT:crt0dat.obj
 0001:0004c7fb       __get_osplatform           0044d7fb f   LIBCMT:crt0dat.obj
 0001:0004c832       __get_osver                0044d832 f   LIBCMT:crt0dat.obj
 0001:0004c86e       __get_winver               0044d86e f   LIBCMT:crt0dat.obj
 0001:0004c8aa       __get_winmajor             0044d8aa f   LIBCMT:crt0dat.obj
 0001:0004c8e6       __get_winminor             0044d8e6 f   LIBCMT:crt0dat.obj
 0001:0004c922       __get_wpgmptr              0044d922 f   LIBCMT:crt0dat.obj
 0001:0004c959       __get_pgmptr               0044d959 f   LIBCMT:crt0dat.obj
 0001:0004c990       __cinit                    0044d990 f   LIBCMT:crt0dat.obj
 0001:0004cb04       _exit                      0044db04 f   LIBCMT:crt0dat.obj
 0001:0004cb15       __exit                     0044db15 f   LIBCMT:crt0dat.obj
 0001:0004cb26       __cexit                    0044db26 f   LIBCMT:crt0dat.obj
 0001:0004cb35       __c_exit                   0044db35 f   LIBCMT:crt0dat.obj
 0001:0004cb44       __init_pointers            0044db44 f   LIBCMT:crt0dat.obj
 0001:0004cb90       _vfprintf_helper           0044db90 f   LIBCMT:vfprintf.obj
 0001:0004ccde       __vfprintf_l               0044dcde f   LIBCMT:vfprintf.obj
 0001:0004ccfc       __vfprintf_s_l             0044dcfc f   LIBCMT:vfprintf.obj
 0001:0004cd1a       __vfprintf_p_l             0044dd1a f   LIBCMT:vfprintf.obj
 0001:0004cd38       _vfprintf                  0044dd38 f   LIBCMT:vfprintf.obj
 0001:0004cd54       _vfprintf_s                0044dd54 f   LIBCMT:vfprintf.obj
 0001:0004cd70       __vfprintf_p               0044dd70 f   LIBCMT:vfprintf.obj
 0001:0004cd8c       __initp_misc_winsig        0044dd8c f   LIBCMT:winsig.obj
 0001:0004ce74       ___get_sigabrt             0044de74 f   LIBCMT:winsig.obj
 0001:0004ce81       ___fpecode                 0044de81 f   LIBCMT:winsig.obj
 0001:0004ce8a       ___pxcptinfoptrs           0044de8a f   LIBCMT:winsig.obj
 0001:0004ce93       _signal                    0044de93 f   LIBCMT:winsig.obj
 0001:0004d0d0       _raise                     0044e0d0 f   LIBCMT:winsig.obj
 0001:0004d280       _srand                     0044e280 f   LIBCMT:rand.obj
 0001:0004d28d       _rand                      0044e28d f   LIBCMT:rand.obj
 0001:0004d2b0       _memcpy                    0044e2b0 f   LIBCMT:memcpy.obj
 0001:0004d615       _puts                      0044e615 f   LIBCMT:puts.obj
 0001:0004d7b0       _strrchr                   0044e7b0 f   LIBCMT:strrchr.obj
 0001:0004d7dd       _fgets                     0044e7dd f   LIBCMT:fgets.obj
 0001:0004d970       _memmove                   0044e970 f   LIBCMT:memmove.obj
 0001:0004dce0       __ftol2_sse                0044ece0 f   LIBCMT:ftol2.obj
 0001:0004dce9       __ftol2_pentium4           0044ece9 f   LIBCMT:ftol2.obj
 0001:0004dcfc       __ftol2_sse_excpt          0044ecfc f   LIBCMT:ftol2.obj
 0001:0004dd16       __ftol2                    0044ed16 f   LIBCMT:ftol2.obj
 0001:0004dd90       _floor                     0044ed90 f   LIBCMT:floor_pentium4.obj
 0001:0004ddd0       __floor_pentium4           0044edd0 f   LIBCMT:floor_pentium4.obj
 0001:0004deb1       __getenv_helper_nolock     0044eeb1 f   LIBCMT:getenv.obj
 0001:0004e067       _getenv                    0044f067 f   LIBCMT:getenv.obj
 0001:0004e0ea       _getenv_s                  0044f0ea f   LIBCMT:getenv.obj
 0001:0004e1c2       __dupenv_s                 0044f1c2 f   LIBCMT:getenv.obj
 0001:0004e2a8       ??0_LocaleUpdate@@QAE@PAUlocaleinfo_struct@@@Z 0044f2a8 f i LIBCMT:strtol.obj
 0001:0004e32a       ??1_LocaleUpdate@@QAE@XZ   0044f32a f i LIBCMT:strtol.obj
 0001:0004e338       ?GetLocaleT@_LocaleUpdate@@QAEPAUlocaleinfo_struct@@XZ 0044f338 f i LIBCMT:strtol.obj
 0001:0004e566       _strtol                    0044f566 f   LIBCMT:strtol.obj
 0001:0004e58f       __strtol_l                 0044f58f f   LIBCMT:strtol.obj
 0001:0004e5aa       _strtoul                   0044f5aa f   LIBCMT:strtol.obj
 0001:0004e5d4       __strtoul_l                0044f5d4 f   LIBCMT:strtol.obj
 0001:0004e5ef       __isalpha_l                0044f5ef f i LIBCMT:_ctype.obj
 0001:0004e643       _isalpha                   0044f643 f i LIBCMT:_ctype.obj
 0001:0004e66e       __isupper_l                0044f66e f i LIBCMT:_ctype.obj
 0001:0004e6bd       _isupper                   0044f6bd f i LIBCMT:_ctype.obj
 0001:0004e6e6       __islower_l                0044f6e6 f i LIBCMT:_ctype.obj
 0001:0004e735       _islower                   0044f735 f i LIBCMT:_ctype.obj
 0001:0004e75e       __isdigit_l                0044f75e f i LIBCMT:_ctype.obj
 0001:0004e7ad       _isdigit                   0044f7ad f i LIBCMT:_ctype.obj
 0001:0004e7d6       __isxdigit_l               0044f7d6 f i LIBCMT:_ctype.obj
 0001:0004e82a       _isxdigit                  0044f82a f i LIBCMT:_ctype.obj
 0001:0004e855       __isspace_l                0044f855 f i LIBCMT:_ctype.obj
 0001:0004e8a4       _isspace                   0044f8a4 f i LIBCMT:_ctype.obj
 0001:0004e8cd       __ispunct_l                0044f8cd f i LIBCMT:_ctype.obj
 0001:0004e91c       _ispunct                   0044f91c f i LIBCMT:_ctype.obj
 0001:0004e945       __isalnum_l                0044f945 f i LIBCMT:_ctype.obj
 0001:0004e999       _isalnum                   0044f999 f i LIBCMT:_ctype.obj
 0001:0004e9c4       __isprint_l                0044f9c4 f i LIBCMT:_ctype.obj
 0001:0004ea18       _isprint                   0044fa18 f i LIBCMT:_ctype.obj
 0001:0004ea43       __isgraph_l                0044fa43 f i LIBCMT:_ctype.obj
 0001:0004ea97       _isgraph                   0044fa97 f i LIBCMT:_ctype.obj
 0001:0004eac2       __iscntrl_l                0044fac2 f i LIBCMT:_ctype.obj
 0001:0004eb11       _iscntrl                   0044fb11 f i LIBCMT:_ctype.obj
 0001:0004eb3a       ___isascii                 0044fb3a f i LIBCMT:_ctype.obj
 0001:0004eb47       ___toascii                 0044fb47 f i LIBCMT:_ctype.obj
 0001:0004eb4f       __iscsymf_l                0044fb4f f i LIBCMT:_ctype.obj
 0001:0004eb6e       ___iscsymf                 0044fb6e f i LIBCMT:_ctype.obj
 0001:0004eb88       __iscsym_l                 0044fb88 f i LIBCMT:_ctype.obj
 0001:0004eba7       ___iscsym                  0044fba7 f i LIBCMT:_ctype.obj
 0001:0004ebc3       __MarkAllocaS              0044fbc3 f i LIBCMT:getch.obj
 0001:0004ebd5       __freea                    0044fbd5 f i LIBCMT:getch.obj
 0001:0004ebf0       __ungetch_nolock           0044fbf0 f   LIBCMT:getch.obj
 0001:0004ec11       __getextendedkeycode       0044fc11 f   LIBCMT:getch.obj
 0001:0004ecbe       __getch_nolock             0044fcbe f   LIBCMT:getch.obj
 0001:0004ed81       __getche_nolock            0044fd81 f   LIBCMT:getch.obj
 0001:0004edb8       __kbhit_nolock             0044fdb8 f   LIBCMT:getch.obj
 0001:0004eee0       __ungetch                  0044fee0 f   LIBCMT:getch.obj
 0001:0004ef24       __getch                    0044ff24 f   LIBCMT:getch.obj
 0001:0004ef62       __getche                   0044ff62 f   LIBCMT:getch.obj
 0001:0004efa0       __kbhit                    0044ffa0 f   LIBCMT:getch.obj
 0001:0004efde       __cputs                    0044ffde f   LIBCMT:cputs.obj
 0001:0004f072       __set_osplatform           00450072 f i LIBCMT:crt0.obj
 0001:0004f07c       __set_osver                0045007c f i LIBCMT:crt0.obj
 0001:0004f086       __set_winver               00450086 f i LIBCMT:crt0.obj
 0001:0004f090       __set_winmajor             00450090 f i LIBCMT:crt0.obj
 0001:0004f09a       __set_winminor             0045009a f i LIBCMT:crt0.obj
 0001:0004f2bf       _mainCRTStartup            004502bf f   LIBCMT:crt0.obj
 0001:0004f2c9       _realloc                   004502c9 f   LIBCMT:realloc.obj
 0001:0004f4e4       __recalloc                 004504e4 f   LIBCMT:realloc.obj
 0001:0004f55d       _V6_HeapAlloc              0045055d f   LIBCMT:malloc.obj
 0001:0004f5ac       __heap_alloc               004505ac f i LIBCMT:malloc.obj
 0001:0004f621       _malloc                    00450621 f   LIBCMT:malloc.obj
 0001:0004f6e4       _free                      004506e4 f   LIBCMT:free.obj
 0001:0004f772       __lseeki64_nolock          00450772 f   LIBCMT:lseeki64.obj
 0001:0004f7f5       __lseeki64                 004507f5 f   LIBCMT:lseeki64.obj
 0001:0004f90e       __telli64                  0045090e f   LIBCMT:telli64.obj
 0001:0004f921       __fstat64i32               00450921 f   LIBCMT:fstati32.obj
 0001:0004fc72       ___time64_t_from_ft        00450c72 f   LIBCMT:findfi32.obj
 0001:0004fcd8       __findfirst64i32           00450cd8 f   LIBCMT:findfi32.obj
 0001:0004fe08       __findnext64i32            00450e08 f   LIBCMT:findfi32.obj
 0001:0004ff37       __findclose                00450f37 f   LIBCMT:findfile.obj
 0001:0004ff57       ___timet_from_ft           00450f57 f   LIBCMT:findfile.obj
 0001:0004ffbb       __findfirst32              00450fbb f   LIBCMT:findfile.obj
 0001:000500e2       __findnext32               004510e2 f   LIBCMT:findfile.obj
 0001:00050208       __set_osfhnd               00451208 f   LIBCMT:osfinfo.obj
 0001:00050285       __free_osfhnd              00451285 f   LIBCMT:osfinfo.obj
 0001:00050306       __get_osfhandle            00451306 f   LIBCMT:osfinfo.obj
 0001:00050377       ___lock_fhandle            00451377 f   LIBCMT:osfinfo.obj
 0001:00050417       __unlock_fhandle           00451417 f   LIBCMT:osfinfo.obj
 0001:00050439       __alloc_osfhnd             00451439 f   LIBCMT:osfinfo.obj
 0001:000505d3       __open_osfhandle           004515d3 f   LIBCMT:osfinfo.obj
 0001:000506e8       __umask_s                  004516e8 f   LIBCMT:umask.obj
 0001:00050731       __umask                    00451731 f   LIBCMT:umask.obj
 0001:00050731       _umask                     00451731 f   LIBCMT:umask.obj
 0001:00050752       __localtime64_s            00451752 f   LIBCMT:loctim64.obj
 0001:00050a17       __localtime64              00451a17 f   LIBCMT:loctim64.obj
 0001:00050a40       __alldiv                   00451a40 f   LIBCMT:lldiv.obj
 0001:00050af0       __chkstk                   00451af0 f   LIBCMT:chkstk.obj
 0001:00050af0       __alloca_probe             00451af0     LIBCMT:chkstk.obj
 0001:00050b1b       _fputs                     00451b1b f   LIBCMT:fputs.obj
 0001:00050c5d       _fputc                     00451c5d f   LIBCMT:fputc.obj
 0001:00050d9c       _putc                      00451d9c f   LIBCMT:fputc.obj
 0001:00050edb       __fclose_nolock            00451edb f   LIBCMT:fclose.obj
 0001:00050f4d       _fclose                    00451f4d f   LIBCMT:fclose.obj
 0001:00050fc9       __fsopen                   00451fc9 f   LIBCMT:fopen.obj
 0001:0005108d       _fopen                     0045208d f   LIBCMT:fopen.obj
 0001:000510a0       _fopen_s                   004520a0 f   LIBCMT:fopen.obj
 0001:000510f0       __set_daylight             004520f0 f i LIBCMT:tzset.obj
 0001:000510fc       __set_dstbias              004520fc f i LIBCMT:tzset.obj
 0001:00051108       __set_timezone             00452108 f i LIBCMT:tzset.obj
 0001:00051828       ___tzset                   00452828 f   LIBCMT:tzset.obj
 0001:00051877       __tzset                    00452877 f   LIBCMT:tzset.obj
 0001:000518af       __isindst                  004528af f   LIBCMT:tzset.obj
 0001:000518f0       __initp_misc_invarg        004528f0 f   LIBCMT:invarg.obj
 0001:000518fa       __invoke_watson            004528fa f   LIBCMT:invarg.obj
 0001:000519f6       __set_invalid_parameter_handler 004529f6 f   LIBCMT:invarg.obj
 0001:00051a18       __get_invalid_parameter_handler 00452a18 f   LIBCMT:invarg.obj
 0001:00051a25       ?_invoke_watson@@YAXPBG00II@Z 00452a25 f   LIBCMT:invarg.obj
 0001:00051a2e       __invalid_parameter        00452a2e f   LIBCMT:invarg.obj
 0001:00051a52       __invalid_parameter_noinfo 00452a52 f   LIBCMT:invarg.obj
 0001:00051a62       ?_invalid_parameter@@YAXPBG00II@Z 00452a62 f   LIBCMT:invarg.obj
 0001:00051a70       __aulldiv                  00452a70 f   LIBCMT:ulldiv.obj
 0001:00051ae0       __allmul                   00452ae0 f   LIBCMT:llmul.obj
 0001:00051b20       __aulldvrm                 00452b20 f   LIBCMT:ulldvrm.obj
 0001:00051bb5       __fputchar                 00452bb5 f   LIBCMT:fputchar.obj
 0001:00051bca       _putchar                   00452bca f   LIBCMT:fputchar.obj
 0001:00051bcf       __gmtime64_s               00452bcf f   LIBCMT:gmtime64.obj
 0001:00051e0b       __gmtime64                 00452e0b f   LIBCMT:gmtime64.obj
 0001:00051e2f       __endthread                00452e2f f   LIBCMT:thread.obj
 0001:00051f2d       __beginthread              00452f2d f   LIBCMT:thread.obj
 0001:00051ff0       __allshl                   00452ff0 f   LIBCMT:llshl.obj
 0001:0005200f       _feof                      0045300f f   LIBCMT:feoferr.obj
 0001:0005203e       _ferror                    0045303e f   LIBCMT:feoferr.obj
 0001:0005206d       __fread_nolock_s           0045306d f   LIBCMT:fread.obj
 0001:00052273       __fread_nolock             00453273 f   LIBCMT:fread.obj
 0001:0005228e       _fread_s                   0045328e f   LIBCMT:fread.obj
 0001:00052324       _fread                     00453324 f   LIBCMT:fread.obj
 0001:0005233f       __ftell_nolock             0045333f f   LIBCMT:ftell.obj
 0001:000524d7       _ftell                     004534d7 f   LIBCMT:ftell.obj
 0001:00052545       __fseek_nolock             00453545 f   LIBCMT:fseek.obj
 0001:000525cc       _fseek                     004535cc f   LIBCMT:fseek.obj
 0001:00052651       __fwrite_nolock            00453651 f   LIBCMT:fwrite.obj
 0001:000527b0       _fwrite                    004537b0 f   LIBCMT:fwrite.obj
 0001:00052840       __alloca_probe_16          00453840 f   LIBCMT:alloca16.obj
 0001:00052856       __alloca_probe_8           00453856     LIBCMT:alloca16.obj
 0001:0005286c       __commit                   0045386c f   LIBCMT:commit.obj
 0001:0005294d       _ldiv                      0045394d f   LIBCMT:ldiv.obj
 0001:00052967       _strnlen                   00453967 f   LIBCMT:strlen_s.obj
 0001:00052a50       _qsort                     00453a50 f   LIBCMT:qsort.obj
 0001:00052cf7       __copysign                 00453cf7 f   LIBCMT:ieeemisc.obj
 0001:00052d1d       __chgsign                  00453d1d f   LIBCMT:ieeemisc.obj
 0001:00052d48       __scalb                    00453d48 f   LIBCMT:ieeemisc.obj
 0001:00052d5e       __logb                     00453d5e f   LIBCMT:ieeemisc.obj
 0001:00052e41       __nextafter                00453e41 f   LIBCMT:ieeemisc.obj
 0001:000530d6       __finite                   004540d6 f   LIBCMT:ieeemisc.obj
 0001:000530eb       __isnan                    004540eb f   LIBCMT:ieeemisc.obj
 0001:00053119       __fpclass                  00454119 f   LIBCMT:ieeemisc.obj
 0001:000531ad       ??_V@YAXPAX@Z              004541ad f   LIBCMT:delete2.obj
 0001:000531b2       _rewind                    004541b2 f   LIBCMT:rewind.obj
 0001:00053280       _strncat                   00454280 f   LIBCMT:strncat.obj
 0001:000533b5       __forcdecpt_l              004543b5 f   LIBCMT:cvt.obj
 0001:00053426       __cropzeros_l              00454426 f   LIBCMT:cvt.obj
 0001:000534a6       __positive                 004544a6 f   LIBCMT:cvt.obj
 0001:000534bc       __fassign_l                004544bc f   LIBCMT:cvt.obj
 0001:000534fc       __fassign                  004544fc f   LIBCMT:cvt.obj
 0001:00053530       __forcdecpt                00454530 f   LIBCMT:cvt.obj
 0001:0005353e       __cropzeros                0045453e f   LIBCMT:cvt.obj
 0001:000536b9       __cftoe_l                  004546b9 f   LIBCMT:cvt.obj
 0001:00053787       __cftoe                    00454787 f   LIBCMT:cvt.obj
 0001:000537a5       __cftoa_l                  004547a5 f   LIBCMT:cvt.obj
 0001:00053b16       __cftoa                    00454b16 f   LIBCMT:cvt.obj
 0001:00053c29       __cftof_l                  00454c29 f   LIBCMT:cvt.obj
 0001:00053ce2       __cftof                    00454ce2 f   LIBCMT:cvt.obj
 0001:00053cfd       __cftog_l                  00454cfd f   LIBCMT:cvt.obj
 0001:00053df5       __cftog                    00454df5 f   LIBCMT:cvt.obj
 0001:00053e13       __cfltcvt_l                00454e13 f   LIBCMT:cvt.obj
 0001:00053e99       __cfltcvt                  00454e99 f   LIBCMT:cvt.obj
 0001:00053eba       __initp_misc_cfltcvt_tab   00454eba f   LIBCMT:cmiscdat.obj
 0001:00053ed9       __setdefaultprecision      00454ed9 f   LIBCMT:fp8.obj
 0001:00053f02       __ms_p5_test_fdiv          00454f02 f   LIBCMT:testfdiv.obj
 0001:00053f3e       __ms_p5_mp_test_fdiv       00454f3e f   LIBCMT:testfdiv.obj
 0001:00053f67       ?_Type_info_dtor@type_info@@CAXPAV1@@Z 00454f67 f   LIBCMT:typname.obj
 0001:00053fd7       ?_Name_base@type_info@@CAPBDPBV1@PAU__type_info_node@@@Z 00454fd7 f   LIBCMT:typname.obj
 0001:000540cc       ?_Type_info_dtor_internal@type_info@@CAXPAV1@@Z 004550cc f   LIBCMT:typname.obj
 0001:0005413c       ___unDNameHelper           0045513c f   LIBCMT:typname.obj
 0001:0005416d       ?_Name_base_internal@type_info@@CAPBDPBV1@PAU__type_info_node@@@Z 0045516d f   LIBCMT:typname.obj
 0001:00054258       ___clean_type_info_names_internal 00455258 f   LIBCMT:typname.obj
 0001:000542b0       _strcmp                    004552b0 f   LIBCMT:strcmp.obj
 0001:00054338       _abort                     00455338 f   LIBCMT:abort.obj
 0001:0005442b       __set_abort_behavior       0045542b f   LIBCMT:abort.obj
 0001:00054449       __NMSG_WRITE               00455449 f   LIBCMT:crt0msg.obj
 0001:000545e9       __GET_RTERRMSG             004555e9 f   LIBCMT:crt0msg.obj
 0001:00054609       __FF_MSGBANNER             00455609 f   LIBCMT:crt0msg.obj
 0001:000546ae       __encode_pointer           004556ae f   LIBCMT:tidtable.obj
 0001:0005471c       __encoded_null             0045571c f   LIBCMT:tidtable.obj
 0001:00054725       __decode_pointer           00455725 f   LIBCMT:tidtable.obj
 0001:00054793       ___crtTlsAlloc@4           00455793 f   LIBCMT:tidtable.obj
 0001:0005479c       ___fls_getvalue@4          0045579c f   LIBCMT:tidtable.obj
 0001:000547b1       ___get_flsindex            004557b1 f   LIBCMT:tidtable.obj
 0001:000547b7       ___set_flsgetvalue         004557b7 f   LIBCMT:tidtable.obj
 0001:000547e9       ___fls_setvalue@8          004557e9 f   LIBCMT:tidtable.obj
 0001:00054802       __mtterm                   00455802 f   LIBCMT:tidtable.obj
 0001:0005483f       __initptd                  0045583f f   LIBCMT:tidtable.obj
 0001:000548fe       __getptd_noexit            004558fe f   LIBCMT:tidtable.obj
 0001:00054975       __getptd                   00455975 f   LIBCMT:tidtable.obj
 0001:0005498d       __freefls@4                0045598d f   LIBCMT:tidtable.obj
 0001:00054aae       __freeptd                  00455aae f   LIBCMT:tidtable.obj
 0001:00054b17       ___threadid                00455b17 f   LIBCMT:tidtable.obj
 0001:00054b1d       ___threadhandle            00455b1d f   LIBCMT:tidtable.obj
 0001:00054b23       __mtinit                   00455b23 f   LIBCMT:tidtable.obj
 0001:00054ca7       ___getlocaleinfo           00455ca7 f   LIBCMT:inithelp.obj
 0001:00054e01       __initp_misc_purevirt      00455e01 f   LIBCMT:inithelp.obj
 0001:00054e10       _strlen                    00455e10 f   LIBCMT:strlen.obj
 0001:00054e9b       __fullpath                 00455e9b f   LIBCMT:fullpath.obj
 0001:00054fa3       ___dtoxmode                00455fa3 f   LIBCMT:stat.obj
 0001:00055132       __stat32                   00456132 f   LIBCMT:stat.obj
 0001:0005543b       ___loctotime64_t           0045643b f   LIBCMT:dtoxtm64.obj
 0001:000556a4       __getdrive                 004566a4 f   LIBCMT:drive.obj
 0001:0005576a       __chdrive                  0045676a f   LIBCMT:drive.obj
 0001:0005580b       __mbctolower_l             0045680b f   LIBCMT:mbtolwr.obj
 0001:000558af       __mbctolower               004568af f   LIBCMT:mbtolwr.obj
 0001:000558bd       __mbspbrk_l                004568bd f   LIBCMT:mbspbrk.obj
 0001:00055987       __mbspbrk                  00456987 f   LIBCMT:mbspbrk.obj
 0001:0005599a       ___report_gsfailure        0045699a f   LIBCMT:gs_report.obj
 0001:00055a9e       ??0exception@std@@QAE@XZ   00456a9e f   LIBCMT:stdexcpt.obj
 0001:00055aaf       ??0exception@std@@QAE@ABQBD@Z 00456aaf f   LIBCMT:stdexcpt.obj
 0001:00055afd       ??0exception@std@@QAE@ABQBDH@Z 00456afd f   LIBCMT:stdexcpt.obj
 0001:00055b15       ??0exception@std@@QAE@ABV01@@Z 00456b15 f   LIBCMT:stdexcpt.obj
 0001:00055b6d       ??4exception@std@@QAEAAV01@ABV01@@Z 00456b6d f   LIBCMT:stdexcpt.obj
 0001:00055bc3       ??1exception@std@@UAE@XZ   00456bc3 f   LIBCMT:stdexcpt.obj
 0001:00055bd9       ?what@exception@std@@UBEPBDXZ 00456bd9 f   LIBCMT:stdexcpt.obj
 0001:00055be6       ??0bad_cast@std@@QAE@PBD@Z 00456be6 f   LIBCMT:stdexcpt.obj
 0001:00055bff       ??0bad_cast@std@@QAE@ABV01@@Z 00456bff f   LIBCMT:stdexcpt.obj
 0001:00055c17       ??1bad_cast@std@@UAE@XZ    00456c17 f   LIBCMT:stdexcpt.obj
 0001:00055c22       ??0bad_typeid@std@@QAE@PBD@Z 00456c22 f   LIBCMT:stdexcpt.obj
 0001:00055c3b       ??0bad_typeid@std@@QAE@ABV01@@Z 00456c3b f   LIBCMT:stdexcpt.obj
 0001:00055c53       ??1bad_typeid@std@@UAE@XZ  00456c53 f   LIBCMT:stdexcpt.obj
 0001:00055c5e       ??0__non_rtti_object@std@@QAE@PBD@Z 00456c5e f   LIBCMT:stdexcpt.obj
 0001:00055c76       ??0__non_rtti_object@std@@QAE@ABV01@@Z 00456c76 f   LIBCMT:stdexcpt.obj
 0001:00055c8e       ??1__non_rtti_object@std@@UAE@XZ 00456c8e f   LIBCMT:stdexcpt.obj
 0001:00055c99       ??_Eexception@std@@UAEPAXI@Z 00456c99 f i LIBCMT:stdexcpt.obj
 0001:00055c99       ??_Gexception@std@@UAEPAXI@Z 00456c99 f i LIBCMT:stdexcpt.obj
 0001:00055cb5       ??_Gbad_cast@std@@UAEPAXI@Z 00456cb5 f i LIBCMT:stdexcpt.obj
 0001:00055cb5       ??_Ebad_cast@std@@UAEPAXI@Z 00456cb5 f i LIBCMT:stdexcpt.obj
 0001:00055cd7       ??_Ebad_typeid@std@@UAEPAXI@Z 00456cd7 f i LIBCMT:stdexcpt.obj
 0001:00055cd7       ??_Gbad_typeid@std@@UAEPAXI@Z 00456cd7 f i LIBCMT:stdexcpt.obj
 0001:00055cf9       ??_E__non_rtti_object@std@@UAEPAXI@Z 00456cf9 f i LIBCMT:stdexcpt.obj
 0001:00055cf9       ??_G__non_rtti_object@std@@UAEPAXI@Z 00456cf9 f i LIBCMT:stdexcpt.obj
 0001:00055dd4       ___onexitinit              00456dd4 f   LIBCMT:onexit.obj
 0001:00055e03       __onexit                   00456e03 f   LIBCMT:onexit.obj
 0001:00055e3f       _atexit                    00456e3f f   LIBCMT:onexit.obj
 0001:00055e51       __initp_heap_handler       00456e51 f   LIBCMT:handler.obj
 0001:00055e5b       ?_set_new_handler@@YAP6AHI@ZP6AHI@Z@Z 00456e5b f   LIBCMT:handler.obj
 0001:00055e8c       ?_set_new_handler@@YAP6AHI@ZH@Z 00456e8c f   LIBCMT:handler.obj
 0001:00055e95       ?_query_new_handler@@YAP6AHI@ZXZ 00456e95 f   LIBCMT:handler.obj
 0001:00055ea2       __callnewh                 00456ea2 f   LIBCMT:handler.obj
 0001:00055ec4       __CxxThrowException@8      00456ec4 f   LIBCMT:throw.obj
 0001:00055f65       __VEC_memzero              00456f65 f   LIBCMT:p4_memset.obj
 0001:00055ff4       __sse2_mathfcns_init       00456ff4 f   LIBCMT:mathfcns.obj
 0001:00056008       __set_SSE2_enable          00457008 f   LIBCMT:mathfcns.obj
 0001:0005601c       ___sys_nerr                0045701c f   LIBCMT:syserr.obj
 0001:00056022       ___sys_errlist             00457022 f   LIBCMT:syserr.obj
 0001:00056028       _strcpy_s                  00457028 f   LIBCMT:strcpy_s.obj
 0001:0005608d       _wait_a_bit                0045708d f i LIBCMT:crtheap.obj
 0001:000560ae       __set_malloc_crt_max_wait  004570ae f   LIBCMT:crtheap.obj
 0001:000560be       __malloc_crt               004570be f   LIBCMT:crtheap.obj
 0001:000560fe       __calloc_crt               004570fe f   LIBCMT:crtheap.obj
 0001:00056146       __realloc_crt              00457146 f   LIBCMT:crtheap.obj
 0001:00056191       __recalloc_crt             00457191 f   LIBCMT:crtheap.obj
 0001:000561e1       @_malloc_crt_fastcall@4    004571e1 f   LIBCMT:crtheap.obj
 0001:000561e9       @_calloc_crt_fastcall@8    004571e9 f   LIBCMT:crtheap.obj
 0001:000561f3       @_realloc_crt_fastcall@8   004571f3 f   LIBCMT:crtheap.obj
 0001:000561fd       _strncpy_s                 004571fd f   LIBCMT:strncpy_s.obj
 0001:000562b0       __flsbuf                   004572b0 f   LIBCMT:_flsbuf.obj
 0001:000564b1       _get_int_arg               004574b1 f i LIBCMT:output.obj
 0001:000564be       _get_int64_arg             004574be f i LIBCMT:output.obj
 0001:000564ce       _get_short_arg             004574ce f i LIBCMT:output.obj
 0001:000564dc       __output_l                 004574dc f   LIBCMT:output.obj
 0001:00056e70       __ioinit                   00457e70 f   LIBCMT:ioinit.obj
 0001:000570c4       __ioterm                   004580c4 f   LIBCMT:ioinit.obj
 0001:00057110       __fileno                   00458110 f   LIBCMT:fileno.obj
 0001:00057110       _fileno                    00458110 f   LIBCMT:fileno.obj
 0001:00057140       __SEH_prolog4              00458140 f   LIBCMT:sehprolg4.obj
 0001:00057185       __SEH_epilog4              00458185 f   LIBCMT:sehprolg4.obj
 0001:000571d0       __except_handler4          004581d0 f   LIBCMT:chandler4.obj
 0001:000573ba       __INTRN_LOCALE_CONV        004583ba f i LIBCMT:input.obj
 0001:00057427       __input_l                  00458427 f   LIBCMT:input.obj
 0001:00058128       __input_s_l                00459128 f   LIBCMT:inputs.obj
 0001:00058e53       __stbuf                    00459e53 f   LIBCMT:_sftbuf.obj
 0001:00058ee9       __ftbuf                    00459ee9 f   LIBCMT:_sftbuf.obj
 0001:00058f18       _vprintf_helper            00459f18 f   LIBCMT:vprintf.obj
 0001:00058fa8       __vprintf_l                00459fa8 f   LIBCMT:vprintf.obj
 0001:00058fc2       __vprintf_s_l              00459fc2 f   LIBCMT:vprintf.obj
 0001:00058fdc       __vprintf_p_l              00459fdc f   LIBCMT:vprintf.obj
 0001:00058ff6       _vprintf                   00459ff6 f   LIBCMT:vprintf.obj
 0001:0005900e       _vprintf_s                 0045a00e f   LIBCMT:vprintf.obj
 0001:00059026       __vprintf_p                0045a026 f   LIBCMT:vprintf.obj
 0001:000592d2       __strtoi64                 0045a2d2 f   LIBCMT:strtoq.obj
 0001:000592fb       __strtoi64_l               0045a2fb f   LIBCMT:strtoq.obj
 0001:00059316       __strtoui64                0045a316 f   LIBCMT:strtoq.obj
 0001:00059340       __strtoui64_l              0045a340 f   LIBCMT:strtoq.obj
 0001:0005935b       __vsprintf_l               0045a35b f   LIBCMT:vsprintf.obj
 0001:000593d7       _vsprintf                  0045a3d7 f   LIBCMT:vsprintf.obj
 0001:000593ee       __vscprintf_helper         0045a3ee f   LIBCMT:vsprintf.obj
 0001:00059443       __vscprintf                0045a443 f   LIBCMT:vsprintf.obj
 0001:0005945b       __vscprintf_l              0045a45b f   LIBCMT:vsprintf.obj
 0001:00059475       __vscprintf_p              0045a475 f   LIBCMT:vsprintf.obj
 0001:0005948d       __vscprintf_p_l            0045a48d f   LIBCMT:vsprintf.obj
 0001:000594a7       __vsnprintf_helper         0045a4a7 f   LIBCMT:vsnprnc.obj
 0001:00059571       __vsnprintf_c              0045a571 f   LIBCMT:vsnprnc.obj
 0001:00059598       __vsnprintf_c_l            0045a598 f   LIBCMT:vsnprnc.obj
 0001:000595c0       __vsprintf_s_l             0045a5c0 f   LIBCMT:vsnprnc.obj
 0001:00059646       _vsprintf_s                0045a646 f   LIBCMT:vsnprnc.obj
 0001:00059661       __vsnprintf_s_l            0045a661 f   LIBCMT:vsnprnc.obj
 0001:00059766       __vsnprintf_s              0045a766 f   LIBCMT:vsnprnc.obj
 0001:00059784       __vsprintf_p               0045a784 f   LIBCMT:vsnprnc.obj
 0001:000597ab       __vsprintf_p_l             0045a7ab f   LIBCMT:vsnprnc.obj
 0001:000597d3       _setvbuf                   0045a7d3 f   LIBCMT:setvbuf.obj
 0001:000598d1       __fcloseall                0045a8d1 f   LIBCMT:closeall.obj
 0001:00059970       __mtinitlocks              0045a970 f   LIBCMT:mlock.obj
 0001:000599b9       __mtdeletelocks            0045a9b9 f   LIBCMT:mlock.obj
 0001:00059a0e       __unlock                   0045aa0e f   LIBCMT:mlock.obj
 0001:00059a23       __lockerr_exit             0045aa23 f   LIBCMT:mlock.obj
 0001:00059a3b       __mtinitlocknum            0045aa3b f   LIBCMT:mlock.obj
 0001:00059afe       __lock                     0045aafe f   LIBCMT:mlock.obj
 0001:00059b2f       __write_nolock             0045ab2f f   LIBCMT:write.obj
 0001:0005a151       __write                    0045b151 f   LIBCMT:write.obj
 0001:0005a151       _write                     0045b151 f   LIBCMT:write.obj
 0001:0005a22d       __RTC_Initialize           0045b22d f   LIBCMT:initsect.obj
 0001:0005a251       __RTC_Terminate            0045b251 f   LIBCMT:initsect.obj
 0001:0005a280       __ValidateImageBase        0045b280 f   LIBCMT:pesect.obj
 0001:0005a2b0       __FindPESection            0045b2b0 f   LIBCMT:pesect.obj
 0001:0005a300       __IsNonwritableInCurrentImage 0045b300 f   LIBCMT:pesect.obj
 0001:0005a3bb       ?terminate@@YAXXZ          0045b3bb f   LIBCMT:hooks.obj
 0001:0005a3f4       ?unexpected@@YAXXZ         0045b3f4 f   LIBCMT:hooks.obj
 0001:0005a407       ?_inconsistency@@YAXXZ     0045b407 f   LIBCMT:hooks.obj
 0001:0005a43e       __initp_eh_hooks           0045b43e f   LIBCMT:hooks.obj
 0001:0005a44f       __initp_misc_winxfltr      0045b44f f   LIBCMT:winxfltr.obj
 0001:0005a482       __XcptFilter               0045b482 f   LIBCMT:winxfltr.obj
 0001:0005a5e0       ___CppXcptFilter           0045b5e0 f   LIBCMT:winxfltr.obj
 0001:0005a5fb       __initp_misc_rand_s        0045b5fb f   LIBCMT:rand_s.obj
 0001:0005a605       _rand_s                    0045b605 f   LIBCMT:rand_s.obj
 0001:0005a709       __initp_misc_initcrit      0045b709 f   LIBCMT:initcrit.obj
 0001:0005a723       ___crtInitCritSecAndSpinCount 0045b723 f   LIBCMT:initcrit.obj
 0001:0005a889       __output_s_l               0045b889 f   LIBCMT:outputs.obj
 0001:0005b239       __validate_param_reuseA    0045c239 f   LIBCMT:outputp.obj
 0001:0005b403       _get_crtdouble_arg         0045c403 f i LIBCMT:outputp.obj
 0001:0005b413       __output_p_l               0045c413 f   LIBCMT:outputp.obj
 0001:0005c422       __VEC_memcpy               0045d422 f   LIBCMT:p4_memcpy.obj
 0001:0005c505       __filbuf                   0045d505 f   LIBCMT:_filbuf.obj
 0001:0005c625       ___libm_setusermatherr     0045d625 f   LIBCMT:libm_error.obj
 0001:0005c64e       ___libm_error_support      0045d64e f   LIBCMT:libm_error.obj
 0001:0005c8fe       __floor_default            0045d8fe f   LIBCMT:floor.obj
 0001:0005c9cf       __mbsnbicoll_l             0045d9cf f   LIBCMT:mbsnbico.obj
 0001:0005cabb       __mbsnbicoll               0045dabb f   LIBCMT:mbsnbico.obj
 0001:0005cad2       ___wtomb_environ           0045dad2 f   LIBCMT:wtombenv.obj
 0001:0005cb67       __calloc_impl              0045db67 f   LIBCMT:calloc.obj
 0001:0005cc85       _calloc                    0045dc85 f   LIBCMT:calloc.obj
 0001:0005ced2       ___updatetmbcinfo          0045ded2 f   LIBCMT:mbctype.obj
 0001:0005cff0       __setmbcp_nolock           0045dff0 f   LIBCMT:mbctype.obj
 0001:0005d1c9       __getmbcp                  0045e1c9 f   LIBCMT:mbctype.obj
 0001:0005d205       __setmbcp                  0045e205 f   LIBCMT:mbctype.obj
 0001:0005d39f       ___initmbctable            0045e39f f   LIBCMT:mbctype.obj
 0001:0005d3bd       ____setlc_active_func      0045e3bd f   LIBCMT:setlocal.obj
 0001:0005d3c3       ____unguarded_readlc_active_add_func 0045e3c3 f   LIBCMT:setlocal.obj
 0001:0005d3c9       ___freetlocinfo            0045e3c9 f   LIBCMT:setlocal.obj
 0001:0005d509       ___addlocaleref            0045e509 f   LIBCMT:setlocal.obj
 0001:0005d58f       ___removelocaleref         0045e58f f   LIBCMT:setlocal.obj
 0001:0005d67d       ___updatetlocinfo          0045e67d f   LIBCMT:setlocal.obj
 0001:0005d6f3       __configthreadlocale       0045e6f3 f   LIBCMT:setlocal.obj
 0001:0005d7ac       __free_locale              0045e7ac f   LIBCMT:setlocal.obj
 0001:0005d842       ___free_locale             0045e842 f   LIBCMT:setlocal.obj
 0001:0005d847       __get_current_locale       0045e847 f   LIBCMT:setlocal.obj
 0001:0005d8cf       ___get_current_locale      0045e8cf f   LIBCMT:setlocal.obj
 0001:0005d8d4       ___init_dummy              0045e8d4 f   LIBCMT:setlocal.obj
 0001:0005d8d7       __strcats                  0045e8d7 f   LIBCMT:setlocal.obj
 0001:0005d915       ___lc_strtolc              0045e915 f   LIBCMT:setlocal.obj
 0001:0005da3e       ___lc_lctostr              0045ea3e f   LIBCMT:setlocal.obj
 0001:0005dc1a       __expandlocale             0045ec1a f   LIBCMT:setlocal.obj
 0001:0005e2b2       __create_locale            0045f2b2 f   LIBCMT:setlocal.obj
 0001:0005e3a5       ___create_locale           0045f3a5 f   LIBCMT:setlocal.obj
 0001:0005e3aa       _setlocale                 0045f3aa f   LIBCMT:setlocal.obj
 0001:0005e51a       __isctype_l                0045f51a f   LIBCMT:isctype.obj
 0001:0005e5d0       __isctype                  0045f5d0 f   LIBCMT:isctype.obj
 0001:0005e5ff       ___initconin               0045f5ff f   LIBCMT:initcon.obj
 0001:0005e61e       ___initconout              0045f61e f   LIBCMT:initcon.obj
 0001:0005e63d       ___termcon                 0045f63d f   LIBCMT:initcon.obj
 0001:0005e66a       __putch_nolock             0045f66a f   LIBCMT:putch.obj
 0001:0005e6e2       __putch                    0045f6e2 f   LIBCMT:putch.obj
 0001:0005e724       ?__CxxUnhandledExceptionFilter@@YGJPAU_EXCEPTION_POINTERS@@@Z 0045f724 f   LIBCMT:unhandld.obj
 0001:0005e761       ___CxxSetUnhandledExceptionFilter 0045f761 f   LIBCMT:unhandld.obj
 0001:0005e76f       __setenvp                  0045f76f f   LIBCMT:stdenvp.obj
 0001:0005e84a       __set_pgmptr               0045f84a f i LIBCMT:stdargv.obj
 0001:0005e9ec       __setargv                  0045f9ec f   LIBCMT:stdargv.obj
 0001:0005eaa5       ___crtGetEnvironmentStringsA 0045faa5 f   LIBCMT:a_env.obj
 0001:0005ebda       ___heap_select             0045fbda f   LIBCMT:heapinit.obj
 0001:0005ec35       __heap_init                0045fc35 f   LIBCMT:heapinit.obj
 0001:0005ec8f       __heap_term                0045fc8f f   LIBCMT:heapinit.obj
 0001:0005ed03       __get_heap_handle          0045fd03 f   LIBCMT:heapinit.obj
 0001:0005ed09       ___security_init_cookie    0045fd09 f   LIBCMT:gs_support.obj
 0001:0005ed9d       __get_sbh_threshold        0045fd9d f   LIBCMT:sbheap.obj
 0001:0005edbe       __set_amblksiz             0045fdbe f   LIBCMT:sbheap.obj
 0001:0005ee04       __get_amblksiz             0045fe04 f   LIBCMT:sbheap.obj
 0001:0005ee40       ___sbh_heap_init           0045fe40 f   LIBCMT:sbheap.obj
 0001:0005ee88       ___sbh_find_block          0045fe88 f   LIBCMT:sbheap.obj
 0001:0005eeb3       ___sbh_free_block          0045feb3 f   LIBCMT:sbheap.obj
 0001:0005f1c7       ___sbh_alloc_new_region    004601c7 f   LIBCMT:sbheap.obj
 0001:0005f277       ___sbh_alloc_new_group     00460277 f   LIBCMT:sbheap.obj
 0001:0005f37d       ___sbh_resize_block        0046037d f   LIBCMT:sbheap.obj
 0001:0005f65c       ___sbh_heapmin             0046065c f   LIBCMT:sbheap.obj
 0001:0005f729       ___sbh_heap_check          00460729 f   LIBCMT:sbheap.obj
 0001:0005fa0b       __set_sbh_threshold        00460a0b f   LIBCMT:sbheap.obj
 0001:0005fab3       ___sbh_alloc_block         00460ab3 f   LIBCMT:sbheap.obj
 0001:0005fd96       __msize                    00460d96 f   LIBCMT:msize.obj
 0001:0005fe39       ___loctotime32_t           00460e39 f   LIBCMT:dtoxtime.obj
 0001:0006003d       __get_daylight             0046103d f   LIBCMT:timeset.obj
 0001:00060071       __get_dstbias              00461071 f   LIBCMT:timeset.obj
 0001:000600a5       __get_timezone             004610a5 f   LIBCMT:timeset.obj
 0001:000600d9       __get_tzname               004610d9 f   LIBCMT:timeset.obj
 0001:0006017b       ___daylight                0046117b f   LIBCMT:timeset.obj
 0001:00060181       ___dstbias                 00461181 f   LIBCMT:timeset.obj
 0001:00060187       ___timezone                00461187 f   LIBCMT:timeset.obj
 0001:0006018d       ___tzname                  0046118d f   LIBCMT:timeset.obj
 0001:000601a0       __allrem                   004611a0 f   LIBCMT:llrem.obj
 0001:00060252       __gmtime32_s               00461252 f   LIBCMT:gmtime.obj
 0001:0006037f       ___getgmtimebuf            0046137f f   LIBCMT:gmtime.obj
 0001:000603c7       __gmtime32                 004613c7 f   LIBCMT:gmtime.obj
 0001:000603eb       __close_nolock             004613eb f   LIBCMT:close.obj
 0001:00060482       _close                     00461482 f   LIBCMT:close.obj
 0001:00060482       __close                    00461482 f   LIBCMT:close.obj
 0001:0006054f       __freebuf                  0046154f f   LIBCMT:_freebuf.obj
 0001:0006057b       __openfile                 0046157b f   LIBCMT:_open.obj
 0001:0006081b       __getstream                0046181b f   LIBCMT:stream.obj
 0001:00060954       __local_unwind4            00461954 f   LIBCMT:exsup4.obj
 0001:00060a2a       __seh_longjmp_unwind4@4    00461a2a f   LIBCMT:exsup4.obj
 0001:00060a46       @_EH4_CallFilterFunc@8     00461a46 f   LIBCMT:exsup4.obj
 0001:00060a5d       @_EH4_TransferToHandler@8  00461a5d f   LIBCMT:exsup4.obj
 0001:00060a76       @_EH4_GlobalUnwind@4       00461a76 f   LIBCMT:exsup4.obj
 0001:00060a90       @_EH4_LocalUnwind@16       00461a90 f   LIBCMT:exsup4.obj
 0001:00060aa7       ___init_ctype              00461aa7 f   LIBCMT:initctyp.obj
 0001:00060e3c       ____mb_cur_max_func        00461e3c f   LIBCMT:initctyp.obj
 0001:00060e65       ____mb_cur_max_l_func      00461e65 f   LIBCMT:initctyp.obj
 0001:00060e7b       ____lc_codepage_func       00461e7b f   LIBCMT:initctyp.obj
 0001:00060ea1       ____lc_collate_cp_func     00461ea1 f   LIBCMT:initctyp.obj
 0001:00060ec7       ____lc_handle_func         00461ec7 f   LIBCMT:initctyp.obj
 0001:00060eed       __crt_debugger_hook        00461eed f   LIBCMT:dbghook.obj
 0001:00060ef5       __read_nolock              00461ef5 f   LIBCMT:read.obj
 0001:000614b6       _read                      004624b6 f   LIBCMT:read.obj
 0001:000614b6       __read                     004624b6 f   LIBCMT:read.obj
 0001:000615b3       _memcpy_s                  004625b3 f   LIBCMT:memcpy_s.obj
 0001:0006162e       __lseek_nolock             0046262e f   LIBCMT:lseek.obj
 0001:000616a0       __lseek                    004626a0 f   LIBCMT:lseek.obj
 0001:0006177c       _ldexp                     0046277c f   LIBCMT:ldexp.obj
 0001:0006192a       __set_exp                  0046292a f   LIBCMT:util.obj
 0001:00061954       __get_exp                  00462954 f   LIBCMT:util.obj
 0001:00061969       __add_exp                  00462969 f   LIBCMT:util.obj
 0001:00061993       __set_bexp                 00462993 f   LIBCMT:util.obj
 0001:000619b8       __sptype                   004629b8 f   LIBCMT:util.obj
 0001:00061a13       __decomp                   00462a13 f   LIBCMT:util.obj
 0001:00061ac2       __raise_exc_ex             00462ac2 f   LIBCMT:fpexcept.obj
 0001:00061d9c       __raise_exc                00462d9c f   LIBCMT:fpexcept.obj
 0001:00061dbd       __raise_excf               00462dbd f   LIBCMT:fpexcept.obj
 0001:00061dde       __handle_exc               00462dde f   LIBCMT:fpexcept.obj
 0001:00061fbf       __set_errno_from_matherr   00462fbf f   LIBCMT:fpexcept.obj
 0001:00062007       __errcode                  00463007 f   LIBCMT:fpexcept.obj
 0001:00062034       __umatherr                 00463034 f   LIBCMT:fpexcept.obj
 0001:000620d2       __handle_qnan1             004630d2 f   LIBCMT:fpexcept.obj
 0001:00062125       __handle_qnan2             00463125 f   LIBCMT:fpexcept.obj
 0001:00062184       __except1                  00463184 f   LIBCMT:fpexcept.obj
 0001:0006223e       __except2                  0046323e f   LIBCMT:fpexcept.obj
 0001:0006230a       __statfp                   0046330a f   LIBCMT:fpctrl.obj
 0001:00062315       __clrfp                    00463315 f   LIBCMT:fpctrl.obj
 0001:00062321       __ctrlfp                   00463321 f   LIBCMT:fpctrl.obj
 0001:00062348       __set_statfp               00463348 f   LIBCMT:fpctrl.obj
 0001:0006239e       ___get_fpsr_sse2           0046339e f   LIBCMT:fpctrl.obj
 0001:000623ba       ___set_fpsr_sse2           004633ba f   LIBCMT:fpctrl.obj
 0001:0006242c       ___fclrf_sse2              0046342c f   LIBCMT:fpctrl.obj
 0001:00062444       ___statfp_sse2             00463444 f   LIBCMT:fpctrl.obj
 0001:00062457       ___clrfp_sse2              00463457 f   LIBCMT:fpctrl.obj
 0001:0006246f       ___ctrlfp_sse2             0046346f f   LIBCMT:fpctrl.obj
 0001:000624a3       ___set_statfp_sse2         004634a3 f   LIBCMT:fpctrl.obj
 0001:000624b9       __tolower                  004634b9 f   LIBCMT:tolower.obj
 0001:000624c1       __tolower_l                004634c1 f   LIBCMT:tolower.obj
 0001:000625d8       _tolower                   004635d8 f   LIBCMT:tolower.obj
 0001:000625ff       __atodbl_l                 004635ff f   LIBCMT:atodbl.obj
 0001:000626a5       __atodbl                   004636a5 f   LIBCMT:atodbl.obj
 0001:000626b8       __atoldbl_l                004636b8 f   LIBCMT:atodbl.obj
 0001:0006275f       __atoldbl                  0046375f f   LIBCMT:atodbl.obj
 0001:00062772       __atoflt_l                 00463772 f   LIBCMT:atodbl.obj
 0001:00062818       __atoflt                   00463818 f   LIBCMT:atodbl.obj
 0001:0006282b       __set_output_format        0046382b f   LIBCMT:outputformat.obj
 0001:00062862       __get_output_format        00463862 f   LIBCMT:outputformat.obj
 0001:00062868       __fptostr                  00463868 f   LIBCMT:_fptostr.obj
 0001:00062925       ___dtold                   00463925 f   LIBCMT:cfout.obj
 0001:000629e0       __fltout2                  004639e0 f   LIBCMT:cfout.obj
 0001:00062a70       __alldvrm                  00463a70 f   LIBCMT:lldvrm.obj
 0001:00062b50       __aullshr                  00463b50 f   LIBCMT:ullshr.obj
 0001:00062b6f       __fptrap                   00463b6f f   LIBCMT:crt0fp.obj
 0001:00062b78       __controlfp_s              00463b78 f   LIBCMT:contrlfp.obj
 0001:00062be2       ??0Block@HeapManager@@QAE@XZ 00463be2 f i LIBCMT:undname.obj
 0001:00062be8       ?Constructor@HeapManager@@QAEXP6APAXI@ZP6AXPAX@Z@Z 00463be8 f i LIBCMT:undname.obj
 0001:00062c03       ?Destructor@HeapManager@@QAEXXZ 00463c03 f i LIBCMT:undname.obj
 0001:00062c29       ?getNumberOfDimensions@UnDecorator@@CAHXZ 00463c29 f   LIBCMT:undname.obj
 0001:00062c8c       ?getTypeEncoding@UnDecorator@@CAHXZ 00463c8c f i LIBCMT:undname.obj
 0001:00063100       ?doUnderScore@UnDecorator@@SAHXZ 00464100 f i LIBCMT:undname.obj
 0001:0006310b       ?doMSKeywords@UnDecorator@@SAHXZ 0046410b f i LIBCMT:undname.obj
 0001:00063118       ?doPtr64@UnDecorator@@SAHXZ 00464118 f i LIBCMT:undname.obj
 0001:00063126       ?doFunctionReturns@UnDecorator@@SAHXZ 00464126 f i LIBCMT:undname.obj
 0001:00063134       ?doAllocationModel@UnDecorator@@SAHXZ 00464134 f i LIBCMT:undname.obj
 0001:00063142       ?doAllocationLanguage@UnDecorator@@SAHXZ 00464142 f i LIBCMT:undname.obj
 0001:00063150       ?doThisTypes@UnDecorator@@SAHXZ 00464150 f i LIBCMT:undname.obj
 0001:00063162       ?doAccessSpecifiers@UnDecorator@@SAHXZ 00464162 f i LIBCMT:undname.obj
 0001:00063170       ?doThrowTypes@UnDecorator@@SAHXZ 00464170 f i LIBCMT:undname.obj
 0001:0006317e       ?doMemberTypes@UnDecorator@@SAHXZ 0046417e f i LIBCMT:undname.obj
 0001:0006318c       ?doNameOnly@UnDecorator@@SAHXZ 0046418c f i LIBCMT:undname.obj
 0001:00063197       ?doTypeOnly@UnDecorator@@SAHXZ 00464197 f i LIBCMT:undname.obj
 0001:000631a2       ?haveTemplateParameters@UnDecorator@@SAHXZ 004641a2 f i LIBCMT:undname.obj
 0001:000631ad       ?doEcsu@UnDecorator@@SAHXZ 004641ad f i LIBCMT:undname.obj
 0001:000631bb       ?doNoIdentCharCheck@UnDecorator@@SAHXZ 004641bb f i LIBCMT:undname.obj
 0001:000631c6       ?doEllipsis@UnDecorator@@SAHXZ 004641c6 f i LIBCMT:undname.obj
 0001:000631d4       ?UScore@UnDecorator@@SAPBDW4Tokens@@@Z 004641d4 f   LIBCMT:undname.obj
 0001:000631ed       ?getMemory@HeapManager@@QAEPAXIH@Z 004641ed f   LIBCMT:undname.obj
 0001:00063271       ??0DName@@QAE@XZ           00464271 f i LIBCMT:undname.obj
 0001:0006327e       ??0DName@@QAE@PAVDNameNode@@@Z 0046427e f i LIBCMT:undname.obj
 0001:00063290       ??0DName@@QAE@ABV0@@Z      00464290 f i LIBCMT:undname.obj
 0001:0006332c       ?status@DName@@QBE?AW4DNameStatus@@XZ 0046432c f i LIBCMT:undname.obj
 0001:00063336       ?clearStatus@DName@@QAEXXZ 00464336 f i LIBCMT:undname.obj
 0001:0006333b       ?setPtrRef@DName@@QAEAAV1@XZ 0046433b f i LIBCMT:undname.obj
 0001:00063342       ?isPtrRef@DName@@QBEHXZ    00464342 f i LIBCMT:undname.obj
 0001:0006334c       ?setIsArray@DName@@QAEXXZ  0046434c f i LIBCMT:undname.obj
 0001:00063354       ?isArray@DName@@QBEHXZ     00464354 f i LIBCMT:undname.obj
 0001:0006335e       ?isNoTE@DName@@QBEHXZ      0046435e f i LIBCMT:undname.obj
 0001:00063368       ?setIsNoTE@DName@@QAEXXZ   00464368 f i LIBCMT:undname.obj
 0001:00063370       ?isPinPtr@DName@@QBEHXZ    00464370 f i LIBCMT:undname.obj
 0001:0006337a       ?setIsPinPtr@DName@@QAEXXZ 0046437a f i LIBCMT:undname.obj
 0001:00063382       ?isComArray@DName@@QBEHXZ  00464382 f i LIBCMT:undname.obj
 0001:0006338c       ?setIsComArray@DName@@QAEXXZ 0046438c f i LIBCMT:undname.obj
 0001:00063394       ?isVCallThunk@DName@@QBEHXZ 00464394 f i LIBCMT:undname.obj
 0001:0006339e       ?setIsVCallThunk@DName@@QAEXXZ 0046439e f i LIBCMT:undname.obj
 0001:000633a6       ??4DName@@QAEAAV0@ABV0@@Z  004643a6 f   LIBCMT:undname.obj
 0001:00063421       ?isFull@Replicator@@QBEHXZ 00464421 f i LIBCMT:undname.obj
 0001:0006342a       ??AReplicator@@QBEABVDName@@H@Z 0046442a f   LIBCMT:undname.obj
 0001:0006344f       ??0DNameNode@@IAE@XZ       0046444f f   LIBCMT:undname.obj
 0001:0006345c       ?nextNode@DNameNode@@QBEPAV1@XZ 0046445c f i LIBCMT:undname.obj
 0001:00063460       ??YDNameNode@@QAEAAV0@PAV0@@Z 00464460 f   LIBCMT:undname.obj
 0001:00063489       ??0charNode@@QAE@D@Z       00464489 f   LIBCMT:undname.obj
 0001:0006349f       ?length@charNode@@UBEHXZ   0046449f f i LIBCMT:undname.obj
 0001:000634a3       ?getLastChar@charNode@@UBEDXZ 004644a3 f i LIBCMT:undname.obj
 0001:000634a7       ?getString@charNode@@UBEPADPADH@Z 004644a7 f   LIBCMT:undname.obj
 0001:000634c2       ?length@pcharNode@@UBEHXZ  004644c2 f i LIBCMT:undname.obj
 0001:000634c6       ??0pDNameNode@@QAE@PAVDName@@@Z 004644c6 f   LIBCMT:undname.obj
 0001:000634f5       ??0DNameStatusNode@@QAE@W4DNameStatus@@@Z 004644f5 f   LIBCMT:undname.obj
 0001:0006351a       ?length@DNameStatusNode@@UBEHXZ 0046451a f i LIBCMT:undname.obj
 0001:0006351e       ?getLastChar@DNameStatusNode@@UBEDXZ 0046451e f i LIBCMT:undname.obj
 0001:0006357e       ?getDataIndirectType@UnDecorator@@CA?AVDName@@XZ 0046457e f i LIBCMT:undname.obj
 0001:000635b1       ?getThisType@UnDecorator@@CA?AVDName@@XZ 004645b1 f i LIBCMT:undname.obj
 0001:000635e5       ??2@YAPAXIAAVHeapManager@@H@Z 004645e5 f i LIBCMT:undname.obj
 0001:000635f8       ??0DName@@QAE@PAV0@@Z      004645f8 f   LIBCMT:undname.obj
 0001:0006364e       ??0DName@@QAE@W4DNameStatus@@@Z 0046464e f   LIBCMT:undname.obj
 0001:000636af       ?isValid@DName@@QBEHXZ     004646af f   LIBCMT:undname.obj
 0001:000636c6       ?isEmpty@DName@@QBEHXZ     004646c6 f   LIBCMT:undname.obj
 0001:000636db       ?isUDC@DName@@QBEHXZ       004646db f i LIBCMT:undname.obj
 0001:000636ef       ?setIsUDC@DName@@QAEXXZ    004646ef f i LIBCMT:undname.obj
 0001:000636fd       ?isUDTThunk@DName@@QBEHXZ  004646fd f i LIBCMT:undname.obj
 0001:00063711       ?length@DName@@QBEHXZ      00464711 f   LIBCMT:undname.obj
 0001:00063736       ?getLastChar@DName@@QBEDXZ 00464736 f   LIBCMT:undname.obj
 0001:0006376e       ?getString@DName@@QBEPADPADH@Z 0046476e f   LIBCMT:undname.obj
 0001:000637ff       ??_5DName@@QAEAAV0@ABV0@@Z 004647ff f   LIBCMT:undname.obj
 0001:00063834       ??4DName@@QAEAAV0@W4DNameStatus@@@Z 00464834 f   LIBCMT:undname.obj
 0001:000638b5       ??0Replicator@@QAE@XZ      004648b5 f i LIBCMT:undname.obj
 0001:000638d3       ??YReplicator@@QAEAAV0@ABVDName@@@Z 004648d3 f   LIBCMT:undname.obj
 0001:0006391a       ?clone@DNameNode@@QAEPAV1@XZ 0046491a f   LIBCMT:undname.obj
 0001:00063961       ??0pcharNode@@QAE@PBDH@Z   00464961 f   LIBCMT:undname.obj
 0001:000639c6       ?getLastChar@pcharNode@@UBEDXZ 004649c6 f i LIBCMT:undname.obj
 0001:000639d8       ?getString@pcharNode@@UBEPADPADH@Z 004649d8 f   LIBCMT:undname.obj
 0001:00063a09       ?length@pDNameNode@@UBEHXZ 00464a09 f i LIBCMT:undname.obj
 0001:00063a18       ?getLastChar@pDNameNode@@UBEDXZ 00464a18 f i LIBCMT:undname.obj
 0001:00063a27       ?getString@pDNameNode@@UBEPADPADH@Z 00464a27 f   LIBCMT:undname.obj
 0001:00063a44       ?getString@DNameStatusNode@@UBEPADPADH@Z 00464a44 f   LIBCMT:undname.obj
 0001:00063a77       ??0UnDecorator@@QAE@PADPBDHP6APADJ@ZK@Z 00464a77 f i LIBCMT:undname.obj
 0001:00063aea       ?getReturnType@UnDecorator@@CA?AVDName@@PAV2@@Z 00464aea f   LIBCMT:undname.obj
 0001:00063b19       ?getStorageConvention@UnDecorator@@CA?AVDName@@XZ 00464b19 f i LIBCMT:undname.obj
 0001:00063b28       ??YDName@@QAEAAV0@W4DNameStatus@@@Z 00464b28 f   LIBCMT:undname.obj
 0001:00063ba1       ??4DName@@QAEAAV0@PAV0@@Z  00464ba1 f   LIBCMT:undname.obj
 0001:00063c09       ?doPchar@DName@@AAEXPBDH@Z 00464c09 f   LIBCMT:undname.obj
 0001:00063caf       ??0DName@@QAE@D@Z          00464caf f   LIBCMT:undname.obj
 0001:00063cd5       ??0DName@@QAE@PBD@Z        00464cd5 f   LIBCMT:undname.obj
 0001:00063d06       ??0DName@@QAE@AAPBDD@Z     00464d06 f   LIBCMT:undname.obj
 0001:00063dd6       ??0DName@@QAE@_K@Z         00464dd6 f   LIBCMT:undname.obj
 0001:00063e3f       ??0DName@@QAE@_J@Z         00464e3f f   LIBCMT:undname.obj
 0001:00063ed5       ??HDName@@QBE?AV0@W4DNameStatus@@@Z 00464ed5 f   LIBCMT:undname.obj
 0001:00063f03       ??YDName@@QAEAAV0@ABV0@@Z  00464f03 f   LIBCMT:undname.obj
 0001:00063f65       ??YDName@@QAEAAV0@PAV0@@Z  00464f65 f   LIBCMT:undname.obj
 0001:00063ff0       ??4DName@@QAEAAV0@D@Z      00464ff0 f   LIBCMT:undname.obj
 0001:0006400c       ??4DName@@QAEAAV0@PBD@Z    0046500c f   LIBCMT:undname.obj
 0001:00064036       ?getCallingConvention@UnDecorator@@CA?AVDName@@XZ 00465036 f   LIBCMT:undname.obj
 0001:000640dc       ?getVCallThunkType@UnDecorator@@CA?AVDName@@XZ 004650dc f i LIBCMT:undname.obj
 0001:00064113       ??HDName@@QBE?AV0@ABV0@@Z  00465113 f   LIBCMT:undname.obj
 0001:00064164       ??HDName@@QBE?AV0@PAV0@@Z  00465164 f   LIBCMT:undname.obj
 0001:00064192       ??YDName@@QAEAAV0@D@Z      00465192 f   LIBCMT:undname.obj
 0001:000641fc       ??YDName@@QAEAAV0@PBD@Z    004651fc f   LIBCMT:undname.obj
 0001:00064268       ?getArgumentList@UnDecorator@@CA?AVDName@@XZ 00465268 f   LIBCMT:undname.obj
 0001:00064348       ?getVdispMapType@UnDecorator@@CA?AVDName@@ABV2@@Z 00465348 f i LIBCMT:undname.obj
 0001:00064397       ??H@YA?AVDName@@DABV0@@Z   00465397 f i LIBCMT:undname.obj
 0001:000643b9       ??H@YA?AVDName@@W4DNameStatus@@ABV0@@Z 004653b9 f i LIBCMT:undname.obj
 0001:000643db       ??H@YA?AVDName@@PBDABV0@@Z 004653db f i LIBCMT:undname.obj
 0001:000643fd       ??HDName@@QBE?AV0@D@Z      004653fd f   LIBCMT:undname.obj
 0001:0006442b       ??HDName@@QBE?AV0@PBD@Z    0046542b f   LIBCMT:undname.obj
 0001:00064459       ?getDimension@UnDecorator@@CA?AVDName@@_N@Z 00465459 f   LIBCMT:undname.obj
 0001:0006459a       ?getEnumType@UnDecorator@@CA?AVDName@@XZ 0046559a f i LIBCMT:undname.obj
 0001:0006466e       ?getArgumentTypes@UnDecorator@@CA?AVDName@@XZ 0046566e f   LIBCMT:undname.obj
 0001:00064732       ?getThrowTypes@UnDecorator@@CA?AVDName@@XZ 00465732 f   LIBCMT:undname.obj
 0001:000647b0       ?getExtendedDataIndirectType@UnDecorator@@CA?AVDName@@AADAA_NH@Z 004657b0 f   LIBCMT:undname.obj
 0001:000648d5       ?getArrayType@UnDecorator@@CA?AVDName@@ABV2@@Z 004658d5 f i LIBCMT:undname.obj
 0001:00064a34       ?getLexicalFrame@UnDecorator@@CA?AVDName@@XZ 00465a34 f i LIBCMT:undname.obj
 0001:00064a65       ?getDisplacement@UnDecorator@@CA?AVDName@@XZ 00465a65 f i LIBCMT:undname.obj
 0001:00064a77       ?getCallIndex@UnDecorator@@CA?AVDName@@XZ 00465a77 f i LIBCMT:undname.obj
 0001:00064a89       ?getGuardNumber@UnDecorator@@CA?AVDName@@XZ 00465a89 f i LIBCMT:undname.obj
 0001:00064a9b       ?getVfTableType@UnDecorator@@CA?AVDName@@ABV2@@Z 00465a9b f i LIBCMT:undname.obj
 0001:00064beb       ?getStringEncoding@UnDecorator@@CA?AVDName@@PADH@Z 00465beb f   LIBCMT:undname.obj
 0001:00064c8b       ?getSignedDimension@UnDecorator@@CA?AVDName@@XZ 00465c8b f   LIBCMT:undname.obj
 0001:00064cdb       ?getTemplateConstant@UnDecorator@@CA?AVDName@@XZ 00465cdb f   LIBCMT:undname.obj
 0001:00064f96       ?getPtrRefDataType@UnDecorator@@CA?AVDName@@ABV2@H@Z 00465f96 f i LIBCMT:undname.obj
 0001:0006506f       ?getVbTableType@UnDecorator@@CA?AVDName@@ABV2@@Z 0046606f f i LIBCMT:undname.obj
 0001:00065083       ?getTemplateArgumentList@UnDecorator@@CA?AVDName@@XZ 00466083 f   LIBCMT:undname.obj
 0001:0006523b       ?getOperatorName@UnDecorator@@CA?AVDName@@_NPA_N@Z 0046623b f i LIBCMT:undname.obj
 0001:000657aa       ?getTemplateName@UnDecorator@@CA?AVDName@@_N@Z 004667aa f   LIBCMT:undname.obj
 0001:000658fd       ?getZName@UnDecorator@@CA?AVDName@@_N@Z 004668fd f   LIBCMT:undname.obj
 0001:00065ae7       ?getScopedName@UnDecorator@@CA?AVDName@@XZ 00466ae7 f   LIBCMT:undname.obj
 0001:00065bcb       ?getECSUName@UnDecorator@@CA?AVDName@@XZ 00466bcb f i LIBCMT:undname.obj
 0001:00065bda       ?getECSUDataType@UnDecorator@@CA?AVDName@@XZ 00466bda f   LIBCMT:undname.obj
 0001:00065cda       ?getSymbolName@UnDecorator@@CA?AVDName@@XZ 00466cda f i LIBCMT:undname.obj
 0001:00065d20       ?getBasedType@UnDecorator@@CA?AVDName@@XZ 00466d20 f   LIBCMT:undname.obj
 0001:00065db2       ?composeDeclaration@UnDecorator@@CA?AVDName@@ABV2@@Z 00466db2 f i LIBCMT:undname.obj
 0001:000668f4       ?getDecoratedName@UnDecorator@@CA?AVDName@@XZ 004678f4 f   LIBCMT:undname.obj
 0001:00066b05       ?getScope@UnDecorator@@CA?AVDName@@XZ 00467b05 f   LIBCMT:undname.obj
 0001:00066d90       ?getFunctionIndirectType@UnDecorator@@CA?AVDName@@ABV2@@Z 00467d90 f   LIBCMT:undname.obj
 0001:000670d1       ?getDataIndirectType@UnDecorator@@CA?AVDName@@ABV2@D0H@Z 004680d1 f   LIBCMT:undname.obj
 0001:000675b5       ??BUnDecorator@@QAEPADXZ   004685b5 f i LIBCMT:undname.obj
 0001:00067701       ?getPtrRefType@UnDecorator@@CA?AVDName@@ABV2@0D@Z 00468701 f   LIBCMT:undname.obj
 0001:00067817       ?getPointerType@UnDecorator@@CA?AVDName@@ABV2@0@Z 00468817 f i LIBCMT:undname.obj
 0001:00067832       ?getPointerTypeArray@UnDecorator@@CA?AVDName@@ABV2@0@Z 00468832 f i LIBCMT:undname.obj
 0001:0006784d       ?getReferenceType@UnDecorator@@CA?AVDName@@ABV2@0@Z 0046884d f i LIBCMT:undname.obj
 0001:00067868       ___unDName                 00468868 f   LIBCMT:undname.obj
 0001:0006790b       ___unDNameEx               0046890b f   LIBCMT:undname.obj
 0001:000679ae       ?getBasicDataType@UnDecorator@@CA?AVDName@@ABV2@@Z 004689ae f   LIBCMT:undname.obj
 0001:00067d35       ?getPrimaryDataType@UnDecorator@@CA?AVDName@@ABV2@@Z 00468d35 f   LIBCMT:undname.obj
 0001:00067e73       ?getDataType@UnDecorator@@CA?AVDName@@PAV2@@Z 00468e73 f   LIBCMT:undname.obj
 0001:00067f24       ?getExternalDataType@UnDecorator@@CA?AVDName@@ABV2@@Z 00468f24 f i LIBCMT:undname.obj
 0001:00067f88       ___crtMessageBoxA          00468f88 f   LIBCMT:crtmbox.obj
 0001:00068145       _strcat_s                  00469145 f   LIBCMT:strcat_s.obj
 0001:000681b6       __set_error_mode           004691b6 f   LIBCMT:errmode.obj
 0001:000681fc       ___set_app_type            004691fc f   LIBCMT:errmode.obj
 0001:00068206       ___get_app_type            00469206 f   LIBCMT:errmode.obj
 0001:00068347       ___crtGetLocaleInfoW       00469347 f   LIBCMT:w_loc.obj
 0001:000684bf       ___crtGetLocaleInfoA       004694bf f   LIBCMT:a_loc.obj
 0001:000684fa       __validdrive               004694fa f   LIBCMT:getcwd.obj
 0001:00068531       __getdcwd_nolock           00469531 f   LIBCMT:getcwd.obj
 0001:00068666       __getcwd                   00469666 f   LIBCMT:getcwd.obj
 0001:00068666       _getcwd                    00469666 f   LIBCMT:getcwd.obj
 0001:000686af       __getdcwd                  004696af f   LIBCMT:getcwd.obj
 0001:000686f9       __mbsicmp_l                004696f9 f   LIBCMT:mbsicmp.obj
 0001:00068913       __mbsicmp                  00469913 f   LIBCMT:mbsicmp.obj
 0001:00068926       __mbsrchr_l                00469926 f   LIBCMT:mbsrchr.obj
 0001:000689e6       __mbsrchr                  004699e6 f   LIBCMT:mbsrchr.obj
 0001:000689f9       __toupper                  004699f9 f   LIBCMT:toupper.obj
 0001:00068a01       __toupper_l                00469a01 f   LIBCMT:toupper.obj
 0001:00068b19       _toupper                   00469b19 f   LIBCMT:toupper.obj
 0001:00068efc       ___crtLCMapStringA         00469efc f   LIBCMT:a_map.obj
 0001:00068f40       _strpbrk                   00469f40 f   LIBCMT:strpbrk.obj
 0001:00068fd0       __get_sse2_info            00469fd0 f   LIBCMT:cpu_disp.obj
 0001:00069030       ___sse2_available_init     0046a030 f   LIBCMT:cpu_disp.obj
 0001:0006903d       __getbuf                   0046a03d f   LIBCMT:_getbuf.obj
 0001:00069081       __isatty                   0046a081 f   LIBCMT:isatty.obj
 0001:000690df       __wctomb_s_l               0046a0df f   LIBCMT:wctomb.obj
 0001:0006923e       _wctomb_s                  0046a23e f   LIBCMT:wctomb.obj
 0001:00069259       __wctomb_l                 0046a259 f   LIBCMT:wctomb.obj
 0001:000692a8       _wctomb                    0046a2a8 f   LIBCMT:wctomb.obj
 0001:000692d8       __isleadbyte_l             0046a2d8 f i LIBCMT:_wctype.obj
 0001:0006930e       _isleadbyte                0046a30e f i LIBCMT:_wctype.obj
 0001:0006931c       __iswalpha_l               0046a31c f i LIBCMT:_wctype.obj
 0001:00069332       _iswalpha                  0046a332 f i LIBCMT:_wctype.obj
 0001:00069343       __iswupper_l               0046a343 f i LIBCMT:_wctype.obj
 0001:00069356       _iswupper                  0046a356 f i LIBCMT:_wctype.obj
 0001:00069364       __iswlower_l               0046a364 f i LIBCMT:_wctype.obj
 0001:00069377       _iswlower                  0046a377 f i LIBCMT:_wctype.obj
 0001:00069385       __iswdigit_l               0046a385 f i LIBCMT:_wctype.obj
 0001:00069398       _iswdigit                  0046a398 f i LIBCMT:_wctype.obj
 0001:000693a6       __iswxdigit_l              0046a3a6 f i LIBCMT:_wctype.obj
 0001:000693bc       _iswxdigit                 0046a3bc f i LIBCMT:_wctype.obj
 0001:000693cd       __iswspace_l               0046a3cd f i LIBCMT:_wctype.obj
 0001:000693e0       _iswspace                  0046a3e0 f i LIBCMT:_wctype.obj
 0001:000693ee       __iswpunct_l               0046a3ee f i LIBCMT:_wctype.obj
 0001:00069401       _iswpunct                  0046a401 f i LIBCMT:_wctype.obj
 0001:0006940f       __iswalnum_l               0046a40f f i LIBCMT:_wctype.obj
 0001:00069425       _iswalnum                  0046a425 f i LIBCMT:_wctype.obj
 0001:00069436       __iswprint_l               0046a436 f i LIBCMT:_wctype.obj
 0001:0006944c       _iswprint                  0046a44c f i LIBCMT:_wctype.obj
 0001:0006945d       __iswgraph_l               0046a45d f i LIBCMT:_wctype.obj
 0001:00069473       _iswgraph                  0046a473 f i LIBCMT:_wctype.obj
 0001:00069484       __iswcntrl_l               0046a484 f i LIBCMT:_wctype.obj
 0001:00069497       _iswcntrl                  0046a497 f i LIBCMT:_wctype.obj
 0001:000694a5       _iswascii                  0046a4a5 f i LIBCMT:_wctype.obj
 0001:000694b1       __iswcsym_l                0046a4b1 f i LIBCMT:_wctype.obj
 0001:000694d7       ___iswcsym                 0046a4d7 f i LIBCMT:_wctype.obj
 0001:000694f8       __iswcsymf_l               0046a4f8 f i LIBCMT:_wctype.obj
 0001:0006951e       ___iswcsymf                0046a51e f i LIBCMT:_wctype.obj
 0001:0006953f       __ungetc_nolock            0046a53f f   LIBCMT:ungetc.obj
 0001:0006965d       _ungetc                    0046a65d f   LIBCMT:ungetc.obj
 0001:000696cf       __mbtowc_l                 0046a6cf f   LIBCMT:mbtowc.obj
 0001:000697e2       _mbtowc                    0046a7e2 f   LIBCMT:mbtowc.obj
 0001:000697f9       __putwch_nolock            0046a7f9 f   LIBCMT:putwch.obj
 0001:000698bb       __cputws                   0046a8bb f   LIBCMT:putwch.obj
 0001:00069956       __putwch                   0046a956 f   LIBCMT:putwch.obj
 0001:0006999c       __matherr                  0046a99c f   LIBCMT:matherr.obj
 0001:0006999f       __frnd                     0046a99f f   LIBCMT:frnd.obj
 0001:00069d53       ___crtCompareStringA       0046ad53 f   LIBCMT:a_cmp.obj
 0001:00069d93       __strnicoll_l              0046ad93 f   LIBCMT:strnicol.obj
 0001:00069e8b       __strnicoll                0046ae8b f   LIBCMT:strnicol.obj
 0001:00069f5c       ___crtsetenv               0046af5c f   LIBCMT:setenv.obj
 0001:0006a360       ___crtGetStringTypeA       0046b360 f   LIBCMT:a_str.obj
 0001:0006a3a0       ___pwctype_func            0046b3a0 f   LIBCMT:ctype.obj
 0001:0006a3a6       ___pctype_func             0046b3a6 f   LIBCMT:ctype.obj
 0001:0006a7e8       ___free_lc_time            0046b7e8 f   LIBCMT:inittime.obj
 0001:0006a978       ___init_time               0046b978 f   LIBCMT:inittime.obj
 0001:0006aa1e       ___free_lconv_num          0046ba1e f   LIBCMT:initnum.obj
 0001:0006aa5e       ___init_numeric            0046ba5e f   LIBCMT:initnum.obj
 0001:0006ac59       ___free_lconv_mon          0046bc59 f   LIBCMT:initmon.obj
 0001:0006ace2       ___init_monetary           0046bce2 f   LIBCMT:initmon.obj
 0001:0006afa6       ___init_collate            0046bfa6 f   LIBCMT:initcoll.obj
 0001:0006afa9       __Getdays_l                0046bfa9 f   LIBCMT:strftime.obj
 0001:0006b0a7       __Getdays                  0046c0a7 f   LIBCMT:strftime.obj
 0001:0006b0b0       __Getmonths_l              0046c0b0 f   LIBCMT:strftime.obj
 0001:0006b1ae       __Getmonths                0046c1ae f   LIBCMT:strftime.obj
 0001:0006b1b7       __Gettnames_l              0046c1b7 f   LIBCMT:strftime.obj
 0001:0006b50c       __Gettnames                0046c50c f   LIBCMT:strftime.obj
 0001:0006be27       __Strftime_l               0046ce27 f   LIBCMT:strftime.obj
 0001:0006bfd6       __strftime_l               0046cfd6 f   LIBCMT:strftime.obj
 0001:0006bff4       _strftime                  0046cff4 f   LIBCMT:strftime.obj
 0001:0006c011       __Strftime                 0046d011 f   LIBCMT:strftime.obj
 0001:0006c02f       _localeconv                0046d02f f   LIBCMT:lconv.obj
 0001:0006c060       _strcspn                   0046d060 f   LIBCMT:strcspn.obj
 0001:0006c660       ___get_qualified_locale    0046d660 f   LIBCMT:getqloc.obj
 0001:0006ddb5       _memcmp                    0046edb5 f   LIBCMT:memcmp.obj
 0001:0006f486       __ismbbkalnum_l            00470486 f   LIBCMT:ismbbyte.obj
 0001:0006f49b       __ismbbkalnum              0047049b f   LIBCMT:ismbbyte.obj
 0001:0006f4ae       __ismbbkprint_l            004704ae f   LIBCMT:ismbbyte.obj
 0001:0006f4c3       __ismbbkprint              004704c3 f   LIBCMT:ismbbyte.obj
 0001:0006f4d6       __ismbbkpunct_l            004704d6 f   LIBCMT:ismbbyte.obj
 0001:0006f4eb       __ismbbkpunct              004704eb f   LIBCMT:ismbbyte.obj
 0001:0006f4fe       __ismbbalnum_l             004704fe f   LIBCMT:ismbbyte.obj
 0001:0006f516       __ismbbalnum               00470516 f   LIBCMT:ismbbyte.obj
 0001:0006f52c       __ismbbalpha_l             0047052c f   LIBCMT:ismbbyte.obj
 0001:0006f544       __ismbbalpha               00470544 f   LIBCMT:ismbbyte.obj
 0001:0006f55a       __ismbbgraph_l             0047055a f   LIBCMT:ismbbyte.obj
 0001:0006f572       __ismbbgraph               00470572 f   LIBCMT:ismbbyte.obj
 0001:0006f588       __ismbbprint_l             00470588 f   LIBCMT:ismbbyte.obj
 0001:0006f5a0       __ismbbprint               004705a0 f   LIBCMT:ismbbyte.obj
 0001:0006f5b6       __ismbbpunct_l             004705b6 f   LIBCMT:ismbbyte.obj
 0001:0006f5cb       __ismbbpunct               004705cb f   LIBCMT:ismbbyte.obj
 0001:0006f5de       __ismbblead_l              004705de f   LIBCMT:ismbbyte.obj
 0001:0006f5f3       __ismbblead                004705f3 f   LIBCMT:ismbbyte.obj
 0001:0006f606       __ismbbtrail_l             00470606 f   LIBCMT:ismbbyte.obj
 0001:0006f61b       __ismbbtrail               0047061b f   LIBCMT:ismbbyte.obj
 0001:0006f62e       __ismbbkana_l              0047062e f   LIBCMT:ismbbyte.obj
 0001:0006f681       __ismbbkana                00470681 f   LIBCMT:ismbbyte.obj
 0001:0006fde8       __open                     00470de8 f   LIBCMT:open.obj
 0001:0006fe9e       __sopen_helper             00470e9e f   LIBCMT:open.obj
 0001:0006ff6a       __sopen                    00470f6a f   LIBCMT:open.obj
 0001:0006ff9a       __sopen_s                  00470f9a f   LIBCMT:open.obj
 0001:0006ffb8       __mbsnbcmp_l               00470fb8 f   LIBCMT:mbsnbcmp.obj
 0001:00070121       __mbsnbcmp                 00471121 f   LIBCMT:mbsnbcmp.obj
 0001:00070138       __global_unwind2           00471138 f   LIBCMT:exsup.obj
 0001:0007019d       __local_unwind2            0047119d f   LIBCMT:exsup.obj
 0001:00070221       __abnormal_termination     00471221 f   LIBCMT:exsup.obj
 0001:00070244       __NLG_Notify1              00471244 f   LIBCMT:exsup.obj
 0001:0007024d       __NLG_Notify               0047124d f   LIBCMT:exsup.obj
 0001:00070264       __NLG_Dispatch             00471264     LIBCMT:exsup.obj
 0001:00070264       __NLG_Dispatch2            00471264     LIBCMT:exsup.obj
 0001:0007026c       __NLG_Call                 0047126c f   LIBCMT:exsup.obj
 0001:0007026e       __NLG_Return2              0047126e     LIBCMT:exsup.obj
 0001:0007026f       ___addl                    0047126f f i LIBCMT:intrncvt.obj
 0001:00070290       __ZeroTail                 00471290 f i LIBCMT:intrncvt.obj
 0001:000702d5       __IncMan                   004712d5 f i LIBCMT:intrncvt.obj
 0001:0007033f       __RoundMan                 0047133f f i LIBCMT:intrncvt.obj
 0001:0007042d       __CopyMan                  0047142d f i LIBCMT:intrncvt.obj
 0001:00070448       __FillZeroMan              00471448 f i LIBCMT:intrncvt.obj
 0001:00070454       __IsZeroMan                00471454 f i LIBCMT:intrncvt.obj
 0001:0007046d       __ShrMan                   0047146d f i LIBCMT:intrncvt.obj
 0001:00070505       __ld12cvt                  00471505 f i LIBCMT:intrncvt.obj
 0001:00070a2e       __ld12tod                  00471a2e f   LIBCMT:intrncvt.obj
 0001:00070f70       __ld12tof                  00471f70 f   LIBCMT:intrncvt.obj
 0001:000714b2       __ld12told                 004724b2 f   LIBCMT:intrncvt.obj
 0001:00071574       ___shl_12                  00472574 f i LIBCMT:strgtold.obj
 0001:000715a2       ___shr_12                  004725a2 f i LIBCMT:strgtold.obj
 0001:000715cf       ___ld12mul                 004725cf f i LIBCMT:strgtold.obj
 0001:00071843       ___multtenpow12            00472843 f i LIBCMT:strgtold.obj
 0001:00071b4c       ___strgtold12_l            00472b4c f   LIBCMT:strgtold.obj
 0001:0007220c       ___STRINGTOLD_L            0047320c f   LIBCMT:strgtold.obj
 0001:00072265       ___add_12                  00473265 f i LIBCMT:x10fout.obj
 0001:000722d2       _$I10_OUTPUT               004732d2 f   LIBCMT:x10fout.obj
 0001:00072b98       __set_controlfp            00473b98 f   LIBCMT:ieee87.obj
 0001:00072eee       __statusfp                 00473eee f   LIBCMT:ieee87.obj
 0001:00072f7e       __fpreset                  00473f7e f   LIBCMT:ieee87.obj
 0001:000731ae       __statusfp2                004741ae f   LIBCMT:ieee87.obj
 0001:00073206       __clearfp                  00474206 f   LIBCMT:ieee87.obj
 0001:000732dd       ___control87_2             004742dd f   LIBCMT:ieee87.obj
 0001:000735e7       __control87                004745e7 f i LIBCMT:ieee87.obj
 0001:000738ea       __controlfp                004748ea f   LIBCMT:ieee87.obj
 0001:00073bf3       ___ascii_stricmp           00474bf3 f   LIBCMT:stricmp.obj
 0001:00073c28       __stricmp_l                00474c28 f   LIBCMT:stricmp.obj
 0001:00073cfb       __stricmp                  00474cfb f   LIBCMT:stricmp.obj
 0001:00073cfb       _stricmp                   00474cfb f   LIBCMT:stricmp.obj
 0001:00073d4b       ___ansicp                  00474d4b f   LIBCMT:convrtcp.obj
 0001:00073d92       ___convertcp               00474d92 f   LIBCMT:convrtcp.obj
 0001:00073f44       __iswctype_l               00474f44 f   LIBCMT:iswctype.obj
 0001:00073fc6       _iswctype                  00474fc6 f   LIBCMT:iswctype.obj
 0001:00074034       _is_wctype                 00475034 f   LIBCMT:iswctype.obj
 0001:00074039       _wcslen                    00475039 f   LIBCMT:wcslen.obj
 0001:0007404f       __strnicmp_l               0047504f f   LIBCMT:strnicmp.obj
 0001:0007413f       __strnicmp                 0047513f f   LIBCMT:strnicmp.obj
 0001:0007419b       _strdup                    0047519b f   LIBCMT:strdup.obj
 0001:0007419b       __strdup                   0047519b f   LIBCMT:strdup.obj
 0001:000741eb       __mbschr_l                 004751eb f   LIBCMT:mbschr.obj
 0001:000742a5       __mbschr                   004752a5 f   LIBCMT:mbschr.obj
 0001:00074393       __itoa_s                   00475393 f   LIBCMT:xtoas.obj
 0001:000743bb       __ltoa_s                   004753bb f   LIBCMT:xtoas.obj
 0001:000743e0       __ultoa_s                  004753e0 f   LIBCMT:xtoas.obj
 0001:000744ee       __i64toa_s                 004754ee f   LIBCMT:xtoas.obj
 0001:00074521       __ui64toa_s                00475521 f   LIBCMT:xtoas.obj
 0001:0007453e       __chsize_nolock            0047553e f   LIBCMT:chsize.obj
 0001:000746f2       __chsize_s                 004756f2 f   LIBCMT:chsize.obj
 0001:000747df       __chsize                   004757df f   LIBCMT:chsize.obj
 0001:000747f7       __setmode_nolock           004757f7 f   LIBCMT:setmode.obj
 0001:000748b3       __set_fmode                004758b3 f   LIBCMT:setmode.obj
 0001:000748f9       __get_fmode                004758f9 f   LIBCMT:setmode.obj
 0001:0007492d       __setmode                  0047592d f   LIBCMT:setmode.obj
 0001:00074a24       ___mtold12                 00475a24 f   LIBCMT:mantold.obj
 0001:00074e14       ___crtGetStringTypeW       00475e14 f   LIBCMT:w_str.obj
 0001:00074e60       ___ascii_strnicmp          00475e60 f   LIBCMT:_strnicm.obj
 0001:00074ec2       _GetLocaleInfoA@16         00475ec2 f   kernel32:KERNEL32.dll
 0001:00074ec8       _CreateEventA@16           00475ec8 f   kernel32:KERNEL32.dll
 0001:00074ece       _SetEvent@4                00475ece f   kernel32:KERNEL32.dll
 0001:00074ed4       _ResetEvent@4              00475ed4 f   kernel32:KERNEL32.dll
 0001:00074eda       _WaitForMultipleObjects@16 00475eda f   kernel32:KERNEL32.dll
 0001:00074ee0       _GetFileAttributesExA@12   00475ee0 f   kernel32:KERNEL32.dll
 0001:00074ee6       _GetSystemDirectoryA@8     00475ee6 f   kernel32:KERNEL32.dll
 0001:00074eec       _GetWindowsDirectoryA@8    00475eec f   kernel32:KERNEL32.dll
 0001:00074ef2       _InterlockedIncrement@4    00475ef2 f   kernel32:KERNEL32.dll
 0001:00074ef8       _DeleteFileA@4             00475ef8 f   kernel32:KERNEL32.dll
 0001:00074efe       _MoveFileA@8               00475efe f   kernel32:KERNEL32.dll
 0001:00074f04       _GetTickCount@0            00475f04 f   kernel32:KERNEL32.dll
 0001:00074f0a       _QueryPerformanceCounter@4 00475f0a f   kernel32:KERNEL32.dll
 0001:00074f10       _QueryPerformanceFrequency@4 00475f10 f   kernel32:KERNEL32.dll
 0001:00074f16       _TryEnterCriticalSection@4 00475f16 f   kernel32:KERNEL32.dll
 0001:00074f1c       _InterlockedCompareExchange@12 00475f1c f   kernel32:KERNEL32.dll
 0001:00074f22       _SetThreadPriority@8       00475f22 f   kernel32:KERNEL32.dll
 0001:00074f28       _SetEndOfFile@4            00475f28 f   kernel32:KERNEL32.dll
 0001:00074f2e       _SetFilePointer@16         00475f2e f   kernel32:KERNEL32.dll
 0001:00074f34       _GetFileAttributesA@4      00475f34 f   kernel32:KERNEL32.dll
 0001:00074f3a       _GetOverlappedResult@16    00475f3a f   kernel32:KERNEL32.dll
 0001:00074f40       _CancelIo@4                00475f40 f   kernel32:KERNEL32.dll
 0001:00074f46       _WriteFile@20              00475f46 f   kernel32:KERNEL32.dll
 0001:00074f4c       _DisconnectNamedPipe@4     00475f4c f   kernel32:KERNEL32.dll
 0001:00074f52       _UnmapViewOfFile@4         00475f52 f   kernel32:KERNEL32.dll
 0001:00074f58       _FindClose@4               00475f58 f   kernel32:KERNEL32.dll
 0001:00074f5e       _FindNextFileA@8           00475f5e f   kernel32:KERNEL32.dll
 0001:00074f64       _FindFirstFileA@8          00475f64 f   kernel32:KERNEL32.dll
 0001:00074f6a       _FileTimeToSystemTime@8    00475f6a f   kernel32:KERNEL32.dll
 0001:00074f70       _FileTimeToLocalFileTime@8 00475f70 f   kernel32:KERNEL32.dll
 0001:00074f76       _GetDriveTypeA@4           00475f76 f   kernel32:KERNEL32.dll
 0001:00074f7c       _ExitProcess@4             00475f7c f   kernel32:KERNEL32.dll
 0001:00074f82       _SetConsoleCtrlHandler@8   00475f82 f   kernel32:KERNEL32.dll
 0001:00074f88       _ReadConsoleInputA@16      00475f88 f   kernel32:KERNEL32.dll
 0001:00074f8e       _SetConsoleMode@8          00475f8e f   kernel32:KERNEL32.dll
 0001:00074f94       _GetConsoleMode@8          00475f94 f   kernel32:KERNEL32.dll
 0001:00074f9a       _PeekConsoleInputA@16      00475f9a f   kernel32:KERNEL32.dll
 0001:00074fa0       _GetNumberOfConsoleInputEvents@8 00475fa0 f   kernel32:KERNEL32.dll
 0001:00074fa6       _GetCommandLineA@0         00475fa6 f   kernel32:KERNEL32.dll
 0001:00074fac       _HeapFree@12               00475fac f   kernel32:KERNEL32.dll
 0001:00074fb2       _GetVersionExA@4           00475fb2 f   kernel32:KERNEL32.dll
 0001:00074fb8       _HeapAlloc@12              00475fb8 f   kernel32:KERNEL32.dll
 0001:00074fbe       _GetProcessHeap@0          00475fbe f   kernel32:KERNEL32.dll
 0001:00074fc4       _HeapReAlloc@16            00475fc4 f   kernel32:KERNEL32.dll
 0001:00074fca       _GetFileInformationByHandle@8 00475fca f   kernel32:KERNEL32.dll
 0001:00074fd0       _PeekNamedPipe@24          00475fd0 f   kernel32:KERNEL32.dll
 0001:00074fd6       _GetFileType@4             00475fd6 f   kernel32:KERNEL32.dll
 0001:00074fdc       _SetStdHandle@8            00475fdc f   kernel32:KERNEL32.dll
 0001:00074fe2       _WideCharToMultiByte@32    00475fe2 f   kernel32:KERNEL32.dll
 0001:00074fe8       _GetTimeZoneInformation@4  00475fe8 f   kernel32:KERNEL32.dll
 0001:00074fee       _UnhandledExceptionFilter@4 00475fee f   kernel32:KERNEL32.dll
 0001:00074ff4       _SetUnhandledExceptionFilter@4 00475ff4 f   kernel32:KERNEL32.dll
 0001:00074ffa       _IsDebuggerPresent@0       00475ffa f   kernel32:KERNEL32.dll
 0001:00075000       _ExitThread@4              00476000 f   kernel32:KERNEL32.dll
 0001:00075006       _ResumeThread@4            00476006 f   kernel32:KERNEL32.dll
 0001:0007500c       _CreateThread@24           0047600c f   kernel32:KERNEL32.dll
 0001:00075012       _FlushFileBuffers@4        00476012 f   kernel32:KERNEL32.dll
 0001:00075018       _GetStdHandle@4            00476018 f   kernel32:KERNEL32.dll
 0001:0007501e       _TlsGetValue@4             0047601e f   kernel32:KERNEL32.dll
 0001:00075024       _TlsAlloc@0                00476024 f   kernel32:KERNEL32.dll
 0001:0007502a       _TlsSetValue@8             0047602a f   kernel32:KERNEL32.dll
 0001:00075030       _TlsFree@4                 00476030 f   kernel32:KERNEL32.dll
 0001:00075036       _InterlockedDecrement@4    00476036 f   kernel32:KERNEL32.dll
 0001:0007503c       _GetCurrentThread@0        0047603c f   kernel32:KERNEL32.dll
 0001:00075042       _GetCurrentDirectoryA@8    00476042 f   kernel32:KERNEL32.dll
 0001:00075048       _SetCurrentDirectoryA@4    00476048 f   kernel32:KERNEL32.dll
 0001:0007504e       _RaiseException@16         0047604e f   kernel32:KERNEL32.dll
 0001:00075054       _SetHandleCount@4          00476054 f   kernel32:KERNEL32.dll
 0001:0007505a       _GetStartupInfoA@4         0047605a f   kernel32:KERNEL32.dll
 0001:00075060       _FatalAppExitA@8           00476060 f   kernel32:KERNEL32.dll
 0001:00075066       _GetConsoleCP@0            00476066 f   kernel32:KERNEL32.dll
 0001:0007506c       _FreeLibrary@4             0047606c f   kernel32:KERNEL32.dll
 0001:00075072       _InterlockedExchange@8     00476072 f   kernel32:KERNEL32.dll
 0001:00075078       _LoadLibraryA@4            00476078 f   kernel32:KERNEL32.dll
 0001:0007507e       _GetCPInfo@8               0047607e f   kernel32:KERNEL32.dll
 0001:00075084       _GetACP@0                  00476084 f   kernel32:KERNEL32.dll
 0001:0007508a       _GetOEMCP@0                0047608a f   kernel32:KERNEL32.dll
 0001:00075090       _IsValidCodePage@4         00476090 f   kernel32:KERNEL32.dll
 0001:00075096       _FreeEnvironmentStringsA@4 00476096 f   kernel32:KERNEL32.dll
 0001:0007509c       _GetEnvironmentStrings@0   0047609c f   kernel32:KERNEL32.dll
 0001:000750a2       _FreeEnvironmentStringsW@4 004760a2 f   kernel32:KERNEL32.dll
 0001:000750a8       _GetEnvironmentStringsW@0  004760a8 f   kernel32:KERNEL32.dll
 0001:000750ae       _HeapDestroy@4             004760ae f   kernel32:KERNEL32.dll
 0001:000750b4       _HeapCreate@12             004760b4 f   kernel32:KERNEL32.dll
 0001:000750ba       _VirtualFree@12            004760ba f   kernel32:KERNEL32.dll
 0001:000750c0       _GetCurrentProcessId@0     004760c0 f   kernel32:KERNEL32.dll
 0001:000750c6       _VirtualAlloc@16           004760c6 f   kernel32:KERNEL32.dll
 0001:000750cc       _HeapSize@12               004760cc f   kernel32:KERNEL32.dll
 0001:000750d2       _RtlUnwind@16              004760d2 f   kernel32:KERNEL32.dll
 0001:000750d8       _MultiByteToWideChar@24    004760d8 f   kernel32:KERNEL32.dll
 0001:000750de       _GetLocaleInfoW@16         004760de f   kernel32:KERNEL32.dll
 0001:000750e4       _LCMapStringA@24           004760e4 f   kernel32:KERNEL32.dll
 0001:000750ea       _LCMapStringW@24           004760ea f   kernel32:KERNEL32.dll
 0001:000750f0       _WriteConsoleA@20          004760f0 f   kernel32:KERNEL32.dll
 0001:000750f6       _GetConsoleOutputCP@0      004760f6 f   kernel32:KERNEL32.dll
 0001:000750fc       _WriteConsoleW@20          004760fc f   kernel32:KERNEL32.dll
 0001:00075102       _CompareStringA@24         00476102 f   kernel32:KERNEL32.dll
 0001:00075108       _CompareStringW@24         00476108 f   kernel32:KERNEL32.dll
 0001:0007510e       _SetEnvironmentVariableA@8 0047610e f   kernel32:KERNEL32.dll
 0001:00075114       _GetStringTypeA@20         00476114 f   kernel32:KERNEL32.dll
 0001:0007511a       _GetStringTypeW@16         0047611a f   kernel32:KERNEL32.dll
 0001:00075120       _GetTimeFormatA@24         00476120 f   kernel32:KERNEL32.dll
 0001:00075126       _GetDateFormatA@24         00476126 f   kernel32:KERNEL32.dll
 0001:0007512c       _GetUserDefaultLCID@0      0047612c f   kernel32:KERNEL32.dll
 0001:00075132       _EnumSystemLocalesA@8      00476132 f   kernel32:KERNEL32.dll
 0001:00075138       _IsValidLocale@8           00476138 f   kernel32:KERNEL32.dll
 0001:0007513e       _SetTimer@16               0047613e f   user32:USER32.dll
 0001:00075144       _KillTimer@8               00476144 f   user32:USER32.dll
 0001:0007514a       _PeekMessageA@20           0047614a f   user32:USER32.dll
 0001:00075150       _RegCloseKey@4             00476150 f   advapi32:ADVAPI32.dll
 0001:00075156       _RegEnumValueA@32          00476156 f   advapi32:ADVAPI32.dll
 0001:0007515c       _RegOpenKeyExA@20          0047615c f   advapi32:ADVAPI32.dll
 0001:00075170       _my_inet_ntoa              00476170 f   mysys:my_net.obj
 0001:000751a0       ??$rotlFixed@I@TaoCrypt@@YAIII@Z 004761a0 f i taocrypt:md5.obj
 0001:000751b0       ?Init@MD5@TaoCrypt@@UAEXXZ 004761b0 f   taocrypt:md5.obj
 0001:000751e0       ??0MD5@TaoCrypt@@QAE@ABV01@@Z 004761e0 f   taocrypt:md5.obj
 0001:00075240       ?AsmTransform@MD5@TaoCrypt@@AAEXPBEI@Z 00476240 f   taocrypt:md5.obj
 0001:000758d0       ?Transform@MD5@TaoCrypt@@EAEXXZ 004768d0 f   taocrypt:md5.obj
 0001:00075ed0       ?Swap@MD5@TaoCrypt@@QAEXAAV12@@Z 00476ed0 f   taocrypt:md5.obj
 0001:00075f30       ?Update@MD5@TaoCrypt@@UAEXPBEI@Z 00476f30 f   taocrypt:md5.obj
 0001:00076000       ??4MD5@TaoCrypt@@QAEAAV01@ABV01@@Z 00477000 f   taocrypt:md5.obj
 0001:00076030       ??$rotrFixed@I@TaoCrypt@@YAIII@Z 00477030 f i taocrypt:hash.obj
 0001:00076040       ?ByteReverse@TaoCrypt@@YAII@Z 00477040 f i taocrypt:hash.obj
 0001:00076060       ?ByteReverse@TaoCrypt@@YA_K_K@Z 00477060 f i taocrypt:hash.obj
 0001:000760a0       ?GetBitCountLo@HASHwithTransform@TaoCrypt@@QBEIXZ 004770a0 f i taocrypt:hash.obj
 0001:000760b0       ?GetBitCountHi@HASHwithTransform@TaoCrypt@@QBEIXZ 004770b0 f i taocrypt:hash.obj
 0001:000760c0       ?GetBitCountLo@HASH64withTransform@TaoCrypt@@QBEIXZ 004770c0 f i taocrypt:hash.obj
 0001:000760d0       ?GetBitCountHi@HASH64withTransform@TaoCrypt@@QBEIXZ 004770d0 f i taocrypt:hash.obj
 0001:000760e0       ??0HASH@TaoCrypt@@QAE@XZ   004770e0 f i taocrypt:hash.obj
 0001:000760f0       ??0HASH64withTransform@TaoCrypt@@QAE@II@Z 004770f0 f   taocrypt:hash.obj
 0001:00076100       ??1HASH64withTransform@TaoCrypt@@UAE@XZ 00477100 f i taocrypt:hash.obj
 0001:00076110       ??_EHASH64withTransform@TaoCrypt@@UAEPAXI@Z 00477110 f i taocrypt:hash.obj
 0001:00076110       ??_GHASH64withTransform@TaoCrypt@@UAEPAXI@Z 00477110 f i taocrypt:hash.obj
 0001:00076130       ?ToEnum@?$EnumToType@W4ByteOrder@TaoCrypt@@$0A@@TaoCrypt@@SA?AW4ByteOrder@2@XZ 00477130 f i taocrypt:hash.obj
 0001:00076140       ??$ByteReverse@I@TaoCrypt@@YAXPAIPBII@Z 00477140 f i taocrypt:hash.obj
 0001:00076180       ??$RightShift@I@?$SafeShifter@$00@TaoCrypt@@SAIII@Z 00477180 f i taocrypt:hash.obj
 0001:00076190       ??$ByteReverse@_K@TaoCrypt@@YAXPA_KPB_KI@Z 00477190 f i taocrypt:hash.obj
 0001:00076200       ?GetHostByteOrder@TaoCrypt@@YA?AW4ByteOrder@1@XZ 00477200 f i taocrypt:hash.obj
 0001:00076210       ?HostByteOrderIs@TaoCrypt@@YA_NW4ByteOrder@1@@Z 00477210 f i taocrypt:hash.obj
 0001:00076220       ?ByteReverse@TaoCrypt@@YAXPAEPBEI@Z 00477220 f i taocrypt:hash.obj
 0001:00076230       ??0HASHwithTransform@TaoCrypt@@QAE@II@Z 00477230 f   taocrypt:hash.obj
 0001:00076240       ??_GHASHwithTransform@TaoCrypt@@UAEPAXI@Z 00477240 f i taocrypt:hash.obj
 0001:00076240       ??_EHASHwithTransform@TaoCrypt@@UAEPAXI@Z 00477240 f i taocrypt:hash.obj
 0001:00076260       ??$SafeRightShift@$0CA@I@TaoCrypt@@YAII@Z 00477260 f i taocrypt:hash.obj
 0001:00076270       ??$ByteReverseIf@E@TaoCrypt@@YAXPAEPBEIW4ByteOrder@0@@Z 00477270 f i taocrypt:hash.obj
 0001:000762b0       ??$ByteReverseIf@I@TaoCrypt@@YAXPAIPBIIW4ByteOrder@0@@Z 004772b0 f i taocrypt:hash.obj
 0001:000762f0       ??$ByteReverseIf@_K@TaoCrypt@@YAXPA_KPB_KIW4ByteOrder@0@@Z 004772f0 f i taocrypt:hash.obj
 0001:00076330       ?AddLength@HASHwithTransform@TaoCrypt@@IAEXI@Z 00477330 f   taocrypt:hash.obj
 0001:00076350       ?Update@HASHwithTransform@TaoCrypt@@UAEXPBEI@Z 00477350 f   taocrypt:hash.obj
 0001:00076410       ?Final@HASHwithTransform@TaoCrypt@@UAEXPAE@Z 00477410 f   taocrypt:hash.obj
 0001:00076560       ?AddLength@HASH64withTransform@TaoCrypt@@IAEXI@Z 00477560 f   taocrypt:hash.obj
 0001:00076580       ?Update@HASH64withTransform@TaoCrypt@@UAEXPBEI@Z 00477580 f   taocrypt:hash.obj
 0001:00076630       ?Final@HASH64withTransform@TaoCrypt@@UAEXPAE@Z 00477630 f   taocrypt:hash.obj
 0001:000767b0       ?Init@MD4@TaoCrypt@@UAEXXZ 004777b0 f   taocrypt:md4.obj
 0001:000767e0       ??0MD4@TaoCrypt@@QAE@ABV01@@Z 004777e0 f   taocrypt:md4.obj
 0001:00076840       ?Transform@MD4@TaoCrypt@@EAEXXZ 00477840 f   taocrypt:md4.obj
 0001:00076c70       ?Swap@MD4@TaoCrypt@@QAEXAAV12@@Z 00477c70 f   taocrypt:md4.obj
 0001:00076cd0       ??4MD4@TaoCrypt@@QAEAAV01@ABV01@@Z 00477cd0 f   taocrypt:md4.obj
 0001:00076d00       ?SetError@Error@TaoCrypt@@QAEXW4ErrorNumber@2@@Z 00477d00 f i taocrypt:coding.obj
 0001:00076d10       ?SetError@Source@TaoCrypt@@QAEXW4ErrorNumber@2@@Z 00477d10 f i taocrypt:coding.obj
 0001:00076d20       ??A?$Block@EV?$AllocatorWithCleanup@E@TaoCrypt@@@TaoCrypt@@QAEAAEI@Z 00477d20 f i taocrypt:coding.obj
 0001:00076d30       ?next@Source@TaoCrypt@@QAEEXZ 00477d30 f i taocrypt:coding.obj
 0001:00076d40       ?resize@?$Block@EV?$AllocatorWithCleanup@E@TaoCrypt@@@TaoCrypt@@QAEXI@Z 00477d40 f i taocrypt:coding.obj
 0001:00076d70       ?Encode@HexEncoder@TaoCrypt@@AAEXXZ 00477d70 f   taocrypt:coding.obj
 0001:00076df0       ?Decode@HexDecoder@TaoCrypt@@AAEXXZ 00477df0 f   taocrypt:coding.obj
 0001:00076e80       ?Encode@Base64Encoder@TaoCrypt@@AAEXXZ 00477e80 f   taocrypt:coding.obj
 0001:00077090       ?Decode@Base64Decoder@TaoCrypt@@AAEXXZ 00478090 f   taocrypt:coding.obj
 0001:000772a0       ?BytesToWords@TaoCrypt@@YAII@Z 004782a0 f i taocrypt:integer.obj
 0001:000772b0       ?BitsToWords@TaoCrypt@@YAII@Z 004782b0 f i taocrypt:integer.obj
 0001:000772c0       ?CopyWords@TaoCrypt@@YAXPAIPBII@Z 004782c0 f i taocrypt:integer.obj
 0001:000772f0       ?CountWords@TaoCrypt@@YAIPBII@Z 004782f0 f i taocrypt:integer.obj
 0001:00077310       ?SetWords@TaoCrypt@@YAXPAIII@Z 00478310 f i taocrypt:integer.obj
 0001:00077330       ?ShiftWordsLeftByBits@TaoCrypt@@YAIPAIII@Z 00478330 f i taocrypt:integer.obj
 0001:00077380       ?ShiftWordsRightByBits@TaoCrypt@@YAIPAIII@Z 00478380 f i taocrypt:integer.obj
 0001:000773d0       ?ShiftWordsLeftByWords@TaoCrypt@@YAXPAIII@Z 004783d0 f i taocrypt:integer.obj
 0001:00077410       ?ShiftWordsRightByWords@TaoCrypt@@YAXPAIII@Z 00478410 f i taocrypt:integer.obj
 0001:00077460       ?IsNegative@Integer@TaoCrypt@@QBE_NXZ 00478460 f i taocrypt:integer.obj
 0001:00077470       ?NotNegative@Integer@TaoCrypt@@QBE_NXZ 00478470 f i taocrypt:integer.obj
 0001:00077480       ??1AbstractGroup@TaoCrypt@@UAE@XZ 00478480 f i taocrypt:integer.obj
 0001:00077490       ??0AbstractGroup@TaoCrypt@@QAE@XZ 00478490 f i taocrypt:integer.obj
 0001:000774a0       ??0MultiplicativeGroupT@AbstractRing@TaoCrypt@@QAE@XZ 004784a0 f i taocrypt:integer.obj
 0001:000774b0       ?InversionIsFast@AbstractGroup@TaoCrypt@@UBE_NXZ 004784b0 f i taocrypt:integer.obj
 0001:000774c0       ?GetRing@MultiplicativeGroupT@AbstractRing@TaoCrypt@@QBEABV23@XZ 004784c0 f i taocrypt:integer.obj
 0001:000774d0       ?Equal@MultiplicativeGroupT@AbstractRing@TaoCrypt@@UBE_NABVInteger@3@0@Z 004784d0 f i taocrypt:integer.obj
 0001:000774e0       ?Identity@MultiplicativeGroupT@AbstractRing@TaoCrypt@@UBEABVInteger@3@XZ 004784e0 f i taocrypt:integer.obj
 0001:000774f0       ?Add@MultiplicativeGroupT@AbstractRing@TaoCrypt@@UBEABVInteger@3@ABV43@0@Z 004784f0 f i taocrypt:integer.obj
 0001:00077500       ?Inverse@MultiplicativeGroupT@AbstractRing@TaoCrypt@@UBEABVInteger@3@ABV43@@Z 00478500 f i taocrypt:integer.obj
 0001:00077510       ?Subtract@MultiplicativeGroupT@AbstractRing@TaoCrypt@@UBEABVInteger@3@ABV43@0@Z 00478510 f i taocrypt:integer.obj
 0001:00077520       ?Double@MultiplicativeGroupT@AbstractRing@TaoCrypt@@UBEABVInteger@3@ABV43@@Z 00478520 f i taocrypt:integer.obj
 0001:00077530       ?SimultaneousMultiply@MultiplicativeGroupT@AbstractRing@TaoCrypt@@UBEXPAVInteger@3@ABV43@PBV43@I@Z 00478530 f i taocrypt:integer.obj
 0001:00077540       ??1MultiplicativeGroupT@AbstractRing@TaoCrypt@@UAE@XZ 00478540 f i taocrypt:integer.obj
 0001:00077550       ??1AbstractRing@TaoCrypt@@UAE@XZ 00478550 f i taocrypt:integer.obj
 0001:00077560       ??_GMultiplicativeGroupT@AbstractRing@TaoCrypt@@UAEPAXI@Z 00478560 f i taocrypt:integer.obj
 0001:00077560       ??_EMultiplicativeGroupT@AbstractRing@TaoCrypt@@UAEPAXI@Z 00478560 f i taocrypt:integer.obj
 0001:00077580       ?SimultaneousExponentiate@MontgomeryRepresentation@TaoCrypt@@UBEXPAVInteger@2@ABV32@PBV32@I@Z 00478580 f i taocrypt:integer.obj
 0001:00077590       ??0DWord@TaoCrypt@@QAE@XZ  00478590 f i taocrypt:integer.obj
 0001:000775a0       ??0DWord@TaoCrypt@@QAE@I@Z 004785a0 f i taocrypt:integer.obj
 0001:000775c0       ??0DWord@TaoCrypt@@QAE@II@Z 004785c0 f i taocrypt:integer.obj
 0001:000775e0       ?Multiply@DWord@TaoCrypt@@SA?AV12@II@Z 004785e0 f i taocrypt:integer.obj
 0001:00077600       ??YDWord@TaoCrypt@@QAEAAV01@I@Z 00478600 f i taocrypt:integer.obj
 0001:00077610       ??HDWord@TaoCrypt@@QAE?AV01@I@Z 00478610 f i taocrypt:integer.obj
 0001:00077630       ??GDWord@TaoCrypt@@QAE?AV01@V01@@Z 00478630 f i taocrypt:integer.obj
 0001:00077650       ??GDWord@TaoCrypt@@QAE?AV01@I@Z 00478650 f i taocrypt:integer.obj
 0001:00077670       ??7DWord@TaoCrypt@@QBE_NXZ 00478670 f i taocrypt:integer.obj
 0001:00077680       ?GetLowHalf@DWord@TaoCrypt@@QBEIXZ 00478680 f i taocrypt:integer.obj
 0001:00077690       ?GetHighHalf@DWord@TaoCrypt@@QBEIXZ 00478690 f i taocrypt:integer.obj
 0001:000776a0       ?GetHighHalfAsBorrow@DWord@TaoCrypt@@QBEIXZ 004786a0 f i taocrypt:integer.obj
 0001:000776b0       ??KDWord@TaoCrypt@@QAEII@Z 004786b0 f i taocrypt:integer.obj
 0001:000776d0       ??LDWord@TaoCrypt@@QAEII@Z 004786d0 f i taocrypt:integer.obj
 0001:00077850       ?MultiplyRecursionLimit@Portable@TaoCrypt@@SAIXZ 00478850 f i taocrypt:integer.obj
 0001:00077860       ?MultiplyBottomRecursionLimit@Portable@TaoCrypt@@SAIXZ 00478860 f i taocrypt:integer.obj
 0001:00077870       ?Square8@Portable@TaoCrypt@@SAXPAIPBI@Z 00478870 f i taocrypt:integer.obj
 0001:00077880       ?SquareRecursionLimit@Portable@TaoCrypt@@SAIXZ 00478880 f i taocrypt:integer.obj
 0001:00077890       ?Add@Portable@TaoCrypt@@SAIPAIPBI1I@Z 00478890 f   taocrypt:integer.obj
 0001:00077920       ?Subtract@Portable@TaoCrypt@@SAIPAIPBI1I@Z 00478920 f   taocrypt:integer.obj
 0001:000779c0       ?Multiply2@Portable@TaoCrypt@@SAXPAIPBI1@Z 004789c0 f   taocrypt:integer.obj
 0001:00077aa0       ?Multiply2Bottom@Portable@TaoCrypt@@SAXPAIPBI1@Z 00478aa0 f   taocrypt:integer.obj
 0001:00077ad0       ?Multiply2Add@Portable@TaoCrypt@@SAIPAIPBI1@Z 00478ad0 f   taocrypt:integer.obj
 0001:00077cc0       ?Add@LowLevel@TaoCrypt@@SAIPAIPBI1I@Z 00478cc0 f i taocrypt:integer.obj
 0001:00077cd0       ?Subtract@LowLevel@TaoCrypt@@SAIPAIPBI1I@Z 00478cd0 f i taocrypt:integer.obj
 0001:00077ce0       ?Multiply4@LowLevel@TaoCrypt@@SAXPAIPBI1@Z 00478ce0 f i taocrypt:integer.obj
 0001:00077cf0       ?Multiply8@LowLevel@TaoCrypt@@SAXPAIPBI1@Z 00478cf0 f i taocrypt:integer.obj
 0001:00077d00       ?Multiply8Bottom@LowLevel@TaoCrypt@@SAXPAIPBI1@Z 00478d00 f i taocrypt:integer.obj
 0001:00077d10       ?Add@PentiumOptimized@TaoCrypt@@SAIPAIPBI1I@Z 00478d10 f   taocrypt:integer.obj
 0001:00077d60       ?Subtract@PentiumOptimized@TaoCrypt@@SAIPAIPBI1I@Z 00478d60 f   taocrypt:integer.obj
 0001:00077db0       ?Add@P4Optimized@TaoCrypt@@SAIPAIPBI1I@Z 00478db0 f   taocrypt:integer.obj
 0001:00077e20       ?Subtract@P4Optimized@TaoCrypt@@SAIPAIPBI1I@Z 00478e20 f   taocrypt:integer.obj
 0001:00077e90       ?Multiply4@PentiumOptimized@TaoCrypt@@SAXPAIPBI1@Z 00478e90 f   taocrypt:integer.obj
 0001:00077fc0       ?Multiply8@PentiumOptimized@TaoCrypt@@SAXPAIPBI1@Z 00478fc0 f   taocrypt:integer.obj
 0001:000783a0       ?Multiply8Bottom@PentiumOptimized@TaoCrypt@@SAXPAIPBI1@Z 004793a0 f   taocrypt:integer.obj
 0001:000786d0       ?Multiply4@P4Optimized@TaoCrypt@@SAXPAIPBI1@Z 004796d0 f   taocrypt:integer.obj
 0001:000787d0       ?Multiply8@P4Optimized@TaoCrypt@@SAXPAIPBI1@Z 004797d0 f   taocrypt:integer.obj
 0001:00078b40       ?Multiply8Bottom@P4Optimized@TaoCrypt@@SAXPAIPBI1@Z 00479b40 f   taocrypt:integer.obj
 0001:00078cf0       ?RecursiveMultiply@TaoCrypt@@YAXPAI0PBI1I@Z 00479cf0 f   taocrypt:integer.obj
 0001:00078f80       ?RecursiveMultiplyTop@TaoCrypt@@YAXPAI0PBI11I@Z 00479f80 f   taocrypt:integer.obj
 0001:00079260       ?Add@TaoCrypt@@YAIPAIPBI1I@Z 0047a260 f i taocrypt:integer.obj
 0001:00079270       ?Subtract@TaoCrypt@@YAIPAIPBI1I@Z 0047a270 f i taocrypt:integer.obj
 0001:00079280       ?Multiply@TaoCrypt@@YAXPAI0PBI1I@Z 0047a280 f i taocrypt:integer.obj
 0001:000792b0       ?DivideByPower2Mod@TaoCrypt@@YAXPAIPBII1I@Z 0047a2b0 f   taocrypt:integer.obj
 0001:00079360       ?MultiplyByPower2Mod@TaoCrypt@@YAXPAIPBII1I@Z 0047a360 f   taocrypt:integer.obj
 0001:000793f0       ?MultiplyTop@TaoCrypt@@YAXPAI0PBI11I@Z 0047a3f0 f i taocrypt:integer.obj
 0001:00079400       ??A?$Block@IV?$AlignedAllocator@I@TaoCrypt@@@TaoCrypt@@QAEAAII@Z 0047a400 f i taocrypt:integer.obj
 0001:00079410       ??A?$Block@IV?$AlignedAllocator@I@TaoCrypt@@@TaoCrypt@@QBEABII@Z 0047a410 f i taocrypt:integer.obj
 0001:00079420       ??H?$Block@IV?$AlignedAllocator@I@TaoCrypt@@@TaoCrypt@@QAEPAII@Z 0047a420 f i taocrypt:integer.obj
 0001:00079430       ??H?$Block@IV?$AlignedAllocator@I@TaoCrypt@@@TaoCrypt@@QBEPBII@Z 0047a430 f i taocrypt:integer.obj
 0001:00079440       ?size@?$Block@IV?$AlignedAllocator@I@TaoCrypt@@@TaoCrypt@@QBEIXZ 0047a440 f i taocrypt:integer.obj
 0001:00079450       ?get_buffer@?$Block@IV?$AlignedAllocator@I@TaoCrypt@@@TaoCrypt@@QBEPAIXZ 0047a450 f i taocrypt:integer.obj
 0001:00079460       ?begin@?$Block@IV?$AlignedAllocator@I@TaoCrypt@@@TaoCrypt@@QBEPAIXZ 0047a460 f i taocrypt:integer.obj
 0001:00079470       ??$swap@PBI@mySTL@@YAXAAPBI0@Z 0047a470 f i taocrypt:integer.obj
 0001:00079490       ??$swap@PAI@mySTL@@YAXAAPAI0@Z 0047a490 f i taocrypt:integer.obj
 0001:000794b0       ??$max@I@TaoCrypt@@YAABIABI0@Z 0047a4b0 f i taocrypt:integer.obj
 0001:000794d0       ??$swap@W4Sign@Integer@TaoCrypt@@@mySTL@@YAXAAW4Sign@Integer@TaoCrypt@@0@Z 0047a4d0 f i taocrypt:integer.obj
 0001:000794f0       ??$swap@V?$AlignedAllocator@I@TaoCrypt@@@mySTL@@YAXAAV?$AlignedAllocator@I@TaoCrypt@@0@Z 0047a4f0 f i taocrypt:integer.obj
 0001:00079500       ?CheckSize@?$AllocatorBase@I@TaoCrypt@@KAXI@Z 0047a500 f i taocrypt:integer.obj
 0001:00079510       ??$tcArrayDelete@I@TaoCrypt@@YAXPAI@Z 0047a510 f i taocrypt:integer.obj
 0001:00079520       ??$RightShift@K@?$SafeShifter@$00@TaoCrypt@@SAKKI@Z 0047a520 f i taocrypt:integer.obj
 0001:00079530       ??$LeftShift@K@?$SafeShifter@$00@TaoCrypt@@SAKKI@Z 0047a530 f i taocrypt:integer.obj
 0001:00079540       ??$DivideThreeWordsByTwo@IVDWord@TaoCrypt@@@TaoCrypt@@YAIPAIIIPAVDWord@0@@Z 0047a540 f i taocrypt:integer.obj
 0001:00079610       ?prev@Source@TaoCrypt@@QAEEXZ 0047a610 f i taocrypt:integer.obj
 0001:00079620       ??0AbstractRing@TaoCrypt@@QAE@XZ 0047a620 f i taocrypt:integer.obj
 0001:00079630       ?MultiplyAndAdd@DWord@TaoCrypt@@SA?AV12@III@Z 0047a630 f i taocrypt:integer.obj
 0001:000796a0       ?Multiply4@Portable@TaoCrypt@@SAXPAIPBI1@Z 0047a6a0 f   taocrypt:integer.obj
 0001:000798e0       ?Square2@Portable@TaoCrypt@@SAXPAIPBI@Z 0047a8e0 f   taocrypt:integer.obj
 0001:00079950       ?Square4@Portable@TaoCrypt@@SAXPAIPBI@Z 0047a950 f   taocrypt:integer.obj
 0001:00079970       ?Multiply8@Portable@TaoCrypt@@SAXPAIPBI1@Z 0047a970 f   taocrypt:integer.obj
 0001:0007a290       ?Multiply4Bottom@Portable@TaoCrypt@@SAXPAIPBI1@Z 0047b290 f   taocrypt:integer.obj
 0001:0007a370       ?Multiply8Bottom@Portable@TaoCrypt@@SAXPAIPBI1@Z 0047b370 f   taocrypt:integer.obj
 0001:0007a850       ?Square4@LowLevel@TaoCrypt@@SAXPAIPBI@Z 0047b850 f i taocrypt:integer.obj
 0001:0007a870       ?RecursiveSquare@TaoCrypt@@YAXPAI0PBII@Z 0047b870 f   taocrypt:integer.obj
 0001:0007a940       ?RecursiveMultiplyBottom@TaoCrypt@@YAXPAI0PBI1I@Z 0047b940 f   taocrypt:integer.obj
 0001:0007aa10       ?Square@TaoCrypt@@YAXPAI0PBII@Z 0047ba10 f i taocrypt:integer.obj
 0001:0007aa20       ?AsymmetricMultiply@TaoCrypt@@YAXPAI0PBII1I@Z 0047ba20 f   taocrypt:integer.obj
 0001:0007ac20       ?AlmostInverse@TaoCrypt@@YAIPAI0PBII1I@Z 0047bc20 f   taocrypt:integer.obj
 0001:0007af30       ?GetBit@Integer@TaoCrypt@@QBE_NI@Z 0047bf30 f   taocrypt:integer.obj
 0001:0007af60       ?GetBits@Integer@TaoCrypt@@QBEKII@Z 0047bf60 f   taocrypt:integer.obj
 0001:0007afa0       ?GetByte@Integer@TaoCrypt@@QBEEI@Z 0047bfa0 f   taocrypt:integer.obj
 0001:0007afd0       ?WordCount@Integer@TaoCrypt@@QBEIXZ 0047bfd0 f   taocrypt:integer.obj
 0001:0007b120       ?Modulo@Integer@TaoCrypt@@QBEII@Z 0047c120 f   taocrypt:integer.obj
 0001:0007b1c0       ?IsUnit@Integer@TaoCrypt@@QBE_NXZ 0047c1c0 f   taocrypt:integer.obj
 0001:0007b1e0       ?MultiplyBottom@TaoCrypt@@YAXPAI0PBI1I@Z 0047c1e0 f i taocrypt:integer.obj
 0001:0007b1f0       ?MontgomeryReduce@TaoCrypt@@YAXPAI0PBI11I@Z 0047c1f0 f   taocrypt:integer.obj
 0001:0007b270       ?RecursiveInverseModPower2@TaoCrypt@@YAXPAI0PBII@Z 0047c270 f   taocrypt:integer.obj
 0001:0007b360       ?Multiply@MontgomeryRepresentation@TaoCrypt@@UBEABVInteger@2@ABV32@0@Z 0047c360 f   taocrypt:integer.obj
 0001:0007b3f0       ?Square@MontgomeryRepresentation@TaoCrypt@@UBEABVInteger@2@ABV32@@Z 0047c3f0 f   taocrypt:integer.obj
 0001:0007b460       ?MultiplicativeInverse@MontgomeryRepresentation@TaoCrypt@@UBEABVInteger@2@ABV32@@Z 0047c460 f   taocrypt:integer.obj
 0001:0007b520       ?Swap@?$Block@IV?$AlignedAllocator@I@TaoCrypt@@@TaoCrypt@@QAEXAAV12@@Z 0047c520 f i taocrypt:integer.obj
 0001:0007b540       ?allocate@?$AlignedAllocator@I@TaoCrypt@@QAEPAIIPBX@Z 0047c540 f i taocrypt:integer.obj
 0001:0007b580       ?deallocate@?$AlignedAllocator@I@TaoCrypt@@QAEXPAXI@Z 0047c580 f i taocrypt:integer.obj
 0001:0007b5c0       ??$SafeRightShift@$0CA@K@TaoCrypt@@YAKK@Z 0047c5c0 f i taocrypt:integer.obj
 0001:0007b5d0       ??$SafeLeftShift@$0CA@K@TaoCrypt@@YAKK@Z 0047c5d0 f i taocrypt:integer.obj
 0001:0007b5e0       ??$DivideFourWordsByTwo@IVDWord@TaoCrypt@@@TaoCrypt@@YA?AVDWord@0@PAIABV10@11@Z 0047c5e0 f i taocrypt:integer.obj
 0001:0007b660       ??$StdReallocate@IV?$AlignedAllocator@I@TaoCrypt@@@TaoCrypt@@YAPAIAAV?$AlignedAllocator@I@0@PAIII_N@Z 0047c660 f i taocrypt:integer.obj
 0001:0007b6e0       ?IsEven@Integer@TaoCrypt@@QBE_NXZ 0047c6e0 f i taocrypt:integer.obj
 0001:0007b6f0       ?IsOdd@Integer@TaoCrypt@@QBE_NXZ 0047c6f0 f i taocrypt:integer.obj
 0001:0007b710       ??LTaoCrypt@@YAIABVInteger@0@I@Z 0047c710 f i taocrypt:integer.obj
 0001:0007b720       ??7Integer@TaoCrypt@@QBE_NXZ 0047c720 f   taocrypt:integer.obj
 0001:0007b740       ?PositiveSubtract@TaoCrypt@@YAXAAVInteger@1@ABV21@1@Z 0047c740 f   taocrypt:integer.obj
 0001:0007b8a0       ?PositiveCompare@Integer@TaoCrypt@@ABEHABV12@@Z 0047c8a0 f   taocrypt:integer.obj
 0001:0007b8e0       ?BitCount@Integer@TaoCrypt@@QBEIXZ 0047c8e0 f   taocrypt:integer.obj
 0001:0007b920       ?ByteCount@Integer@TaoCrypt@@QBEIXZ 0047c920 f   taocrypt:integer.obj
 0001:0007b950       ?IsConvertableToLong@Integer@TaoCrypt@@QBE_NXZ 0047c950 f   taocrypt:integer.obj
 0001:0007b990       ?ConvertToLong@Integer@TaoCrypt@@QBEJXZ 0047c990 f   taocrypt:integer.obj
 0001:0007b9a0       ?Swap@Integer@TaoCrypt@@QAEXAAV12@@Z 0047c9a0 f   taocrypt:integer.obj
 0001:0007ba30       ?Divide@TaoCrypt@@YAXPAI00PBII1I@Z 0047ca30 f   taocrypt:integer.obj
 0001:0007bce0       ?InverseMod@Integer@TaoCrypt@@QBEII@Z 0047cce0 f   taocrypt:integer.obj
 0001:0007bd50       ?Inverse@ModularArithmetic@TaoCrypt@@UBEABVInteger@2@ABV32@@Z 0047cd50 f   taocrypt:integer.obj
 0001:0007bdd0       ?reallocate@?$AlignedAllocator@I@TaoCrypt@@QAEPAIPAIII_N@Z 0047cdd0 f i taocrypt:integer.obj
 0001:0007bdf0       ?IsZero@Integer@TaoCrypt@@QBE_NXZ 0047cdf0 f i taocrypt:integer.obj
 0001:0007be00       ?NotZero@Integer@TaoCrypt@@QBE_NXZ 0047ce00 f i taocrypt:integer.obj
 0001:0007be10       ?IsPositive@Integer@TaoCrypt@@QBE_NXZ 0047ce10 f i taocrypt:integer.obj
 0001:0007be30       ?ScalarMultiply@MultiplicativeGroupT@AbstractRing@TaoCrypt@@UBE?AVInteger@3@ABV43@0@Z 0047ce30 f i taocrypt:integer.obj
 0001:0007be50       ?CascadeScalarMultiply@MultiplicativeGroupT@AbstractRing@TaoCrypt@@UBE?AVInteger@3@ABV43@000@Z 0047ce50 f i taocrypt:integer.obj
 0001:0007be80       ??1AbstractEuclideanDomain@TaoCrypt@@UAE@XZ 0047ce80 f i taocrypt:integer.obj
 0001:0007bea0       ??1EuclideanDomainOf@TaoCrypt@@UAE@XZ 0047cea0 f i taocrypt:integer.obj
 0001:0007bed0       ??1ModularArithmetic@TaoCrypt@@UAE@XZ 0047ced0 f i taocrypt:integer.obj
 0001:0007bf10       ?CascadeExponentiate@MontgomeryRepresentation@TaoCrypt@@UBE?AVInteger@2@ABV32@000@Z 0047cf10 f i taocrypt:integer.obj
 0001:0007bf40       ?Negate@Integer@TaoCrypt@@QAEXXZ 0047cf40 f   taocrypt:integer.obj
 0001:0007bf60       ?Compare@Integer@TaoCrypt@@QBEHABV12@@Z 0047cf60 f   taocrypt:integer.obj
 0001:0007bfa0       ??1MontgomeryRepresentation@TaoCrypt@@UAE@XZ 0047cfa0 f i taocrypt:integer.obj
 0001:0007c000       ?CleanGrow@?$Block@IV?$AlignedAllocator@I@TaoCrypt@@@TaoCrypt@@QAEXI@Z 0047d000 f i taocrypt:integer.obj
 0001:0007c050       ?New@?$Block@IV?$AlignedAllocator@I@TaoCrypt@@@TaoCrypt@@QAEXI@Z 0047d050 f i taocrypt:integer.obj
 0001:0007c080       ?resize@?$Block@IV?$AlignedAllocator@I@TaoCrypt@@@TaoCrypt@@QAEXI@Z 0047d080 f i taocrypt:integer.obj
 0001:0007c0b0       ??_GInteger@TaoCrypt@@QAEPAXI@Z 0047d0b0 f i taocrypt:integer.obj
 0001:0007c0e0       ??8TaoCrypt@@YA_NABVInteger@0@0@Z 0047d0e0 f i taocrypt:integer.obj
 0001:0007c100       ??OTaoCrypt@@YA_NABVInteger@0@0@Z 0047d100 f i taocrypt:integer.obj
 0001:0007c120       ??PTaoCrypt@@YA_NABVInteger@0@0@Z 0047d120 f i taocrypt:integer.obj
 0001:0007c140       ??MTaoCrypt@@YA_NABVInteger@0@0@Z 0047d140 f i taocrypt:integer.obj
 0001:0007c160       ?SetBit@Integer@TaoCrypt@@QAEXI_N@Z 0047d160 f   taocrypt:integer.obj
 0001:0007c200       ?SetByte@Integer@TaoCrypt@@QAEXIE@Z 0047d200 f   taocrypt:integer.obj
 0001:0007c2d0       ??4Integer@TaoCrypt@@QAEAAV01@ABV01@@Z 0047d2d0 f   taocrypt:integer.obj
 0001:0007c330       ??_3Integer@TaoCrypt@@QAEAAV01@I@Z 0047d330 f   taocrypt:integer.obj
 0001:0007c440       ?PositiveAdd@TaoCrypt@@YAXAAVInteger@1@ABV21@1@Z 0047d440 f   taocrypt:integer.obj
 0001:0007c580       ?CleanNew@?$Block@IV?$AlignedAllocator@I@TaoCrypt@@@TaoCrypt@@QAEXI@Z 0047d580 f i taocrypt:integer.obj
 0001:0007c5c0       ??$tcDelete@VInteger@TaoCrypt@@@TaoCrypt@@YAXPAVInteger@0@@Z 0047d5c0 f i taocrypt:integer.obj
 0001:0007c5f0       ?Accumulate@MultiplicativeGroupT@AbstractRing@TaoCrypt@@UBEAAVInteger@3@AAV43@ABV43@@Z 0047d5f0 f i taocrypt:integer.obj
 0001:0007c620       ?Reduce@MultiplicativeGroupT@AbstractRing@TaoCrypt@@UBEAAVInteger@3@AAV43@ABV43@@Z 0047d620 f i taocrypt:integer.obj
 0001:0007c650       ?Decode@Integer@TaoCrypt@@QAEXAAVSource@2@@Z 0047d650 f   taocrypt:integer.obj
 0001:0007c720       ?Decode@Integer@TaoCrypt@@QAEXPBEIW4Signedness@12@@Z 0047d720 f   taocrypt:integer.obj
 0001:0007c880       ?CleanUp@TaoCrypt@@YAXXZ   0047d880 f   taocrypt:integer.obj
 0001:0007c8b0       ?Randomize@Integer@TaoCrypt@@QAEXAAVRandomNumberGenerator@2@I@Z 0047d8b0 f   taocrypt:integer.obj
 0001:0007c940       ??YInteger@TaoCrypt@@QAEAAV01@ABV01@@Z 0047d940 f   taocrypt:integer.obj
 0001:0007c9e0       ??ZInteger@TaoCrypt@@QAEAAV01@ABV01@@Z 0047d9e0 f   taocrypt:integer.obj
 0001:0007ca80       ?Accumulate@ModularArithmetic@TaoCrypt@@UBEAAVInteger@2@AAV32@ABV32@@Z 0047da80 f   taocrypt:integer.obj
 0001:0007cb10       ?Reduce@ModularArithmetic@TaoCrypt@@UBEAAVInteger@2@AAV32@ABV32@@Z 0047db10 f   taocrypt:integer.obj
 0001:0007cb80       ??0?$Block@IV?$AlignedAllocator@I@TaoCrypt@@@TaoCrypt@@QAE@I@Z 0047db80 f i taocrypt:integer.obj
 0001:0007cbd0       ?PositiveMultiply@TaoCrypt@@YAXAAVInteger@1@ABV21@1@Z 0047dbd0 f   taocrypt:integer.obj
 0001:0007cd70       ?Multiply@TaoCrypt@@YAXAAVInteger@1@ABV21@1@Z 0047dd70 f   taocrypt:integer.obj
 0001:0007cdb0       ??0Integer@TaoCrypt@@QAE@XZ 0047ddb0 f   taocrypt:integer.obj
 0001:0007ce20       ??0Integer@TaoCrypt@@QAE@ABV01@@Z 0047de20 f   taocrypt:integer.obj
 0001:0007cee0       ??0Integer@TaoCrypt@@QAE@J@Z 0047dee0 f   taocrypt:integer.obj
 0001:0007cf60       ??0Integer@TaoCrypt@@QAE@W4Sign@01@II@Z 0047df60 f   taocrypt:integer.obj
 0001:0007cfd0       ??0Integer@TaoCrypt@@AAE@II@Z 0047dfd0 f   taocrypt:integer.obj
 0001:0007d090       ??0Integer@TaoCrypt@@QAE@PBEIW4Signedness@01@@Z 0047e090 f   taocrypt:integer.obj
 0001:0007d100       ??0Integer@TaoCrypt@@QAE@AAVSource@1@@Z 0047e100 f   taocrypt:integer.obj
 0001:0007d160       ?Zero@Integer@TaoCrypt@@SAABV12@XZ 0047e160 f   taocrypt:integer.obj
 0001:0007d190       ?One@Integer@TaoCrypt@@SAABV12@XZ 0047e190 f   taocrypt:integer.obj
 0001:0007d1c0       ?Power2@Integer@TaoCrypt@@SA?AV12@I@Z 0047e1c0 f   taocrypt:integer.obj
 0001:0007d1f0       ??GInteger@TaoCrypt@@QBE?AV01@XZ 0047e1f0 f   taocrypt:integer.obj
 0001:0007d210       ??EInteger@TaoCrypt@@QAEAAV01@XZ 0047e210 f   taocrypt:integer.obj
 0001:0007d280       ??FInteger@TaoCrypt@@QAEAAV01@XZ 0047e280 f   taocrypt:integer.obj
 0001:0007d310       ??_2Integer@TaoCrypt@@QAEAAV01@I@Z 0047e310 f   taocrypt:integer.obj
 0001:0007d380       ?MinEncodedSize@Integer@TaoCrypt@@QBEIW4Signedness@12@@Z 0047e380 f   taocrypt:integer.obj
 0001:0007d460       ?Plus@Integer@TaoCrypt@@QBE?AV12@ABV12@@Z 0047e460 f   taocrypt:integer.obj
 0001:0007d4f0       ?Minus@Integer@TaoCrypt@@QBE?AV12@ABV12@@Z 0047e4f0 f   taocrypt:integer.obj
 0001:0007d580       ?Times@Integer@TaoCrypt@@QBE?AV12@ABV12@@Z 0047e580 f   taocrypt:integer.obj
 0001:0007d5b0       ?PositiveDivide@TaoCrypt@@YAXAAVInteger@1@0ABV21@1@Z 0047e5b0 f   taocrypt:integer.obj
 0001:0007d6f0       ?AbsoluteValue@Integer@TaoCrypt@@QBE?AV12@XZ 0047e6f0 f   taocrypt:integer.obj
 0001:0007d710       ?MultiplicativeInverse@Integer@TaoCrypt@@QBE?AV12@XZ 0047e710 f   taocrypt:integer.obj
 0001:0007d750       ?ConvertOut@MontgomeryRepresentation@TaoCrypt@@UBE?AVInteger@2@ABV32@@Z 0047e750 f   taocrypt:integer.obj
 0001:0007d7d0       ??5Integer@TaoCrypt@@QBE?AV01@I@Z 0047e7d0 f i taocrypt:integer.obj
 0001:0007d820       ??6Integer@TaoCrypt@@QBE?AV01@I@Z 0047e820 f i taocrypt:integer.obj
 0001:0007d870       ?Squared@Integer@TaoCrypt@@QBE?AV12@XZ 0047e870 f i taocrypt:integer.obj
 0001:0007d890       ??HTaoCrypt@@YA?AVInteger@0@ABV10@0@Z 0047e890 f i taocrypt:integer.obj
 0001:0007d8b0       ??GTaoCrypt@@YA?AVInteger@0@ABV10@0@Z 0047e8b0 f i taocrypt:integer.obj
 0001:0007d8d0       ??DTaoCrypt@@YA?AVInteger@0@ABV10@0@Z 0047e8d0 f i taocrypt:integer.obj
 0001:0007d8f0       ??0AbstractEuclideanDomain@TaoCrypt@@QAE@XZ 0047e8f0 f i taocrypt:integer.obj
 0001:0007d910       ??0ModularArithmetic@TaoCrypt@@QAE@ABVInteger@1@@Z 0047e910 f i taocrypt:integer.obj
 0001:0007d950       ?MultiplicativeGroup@AbstractRing@TaoCrypt@@UBEABVAbstractGroup@2@XZ 0047e950 f i taocrypt:integer.obj
 0001:0007d960       ?IsMontgomeryRepresentation@ModularArithmetic@TaoCrypt@@UBE_NXZ 0047e960 f i taocrypt:integer.obj
 0001:0007d970       ?Double@ModularArithmetic@TaoCrypt@@UBEABVInteger@2@ABV32@@Z 0047e970 f i taocrypt:integer.obj
 0001:0007d980       ?Divide@ModularArithmetic@TaoCrypt@@UBEABVInteger@2@ABV32@0@Z 0047e980 f i taocrypt:integer.obj
 0001:0007d9b0       ?Equal@ModularArithmetic@TaoCrypt@@UBE_NABVInteger@2@0@Z 0047e9b0 f i taocrypt:integer.obj
 0001:0007d9d0       ??_GModularArithmetic@TaoCrypt@@UAEPAXI@Z 0047e9d0 f i taocrypt:integer.obj
 0001:0007d9d0       ??_EModularArithmetic@TaoCrypt@@UAEPAXI@Z 0047e9d0 f i taocrypt:integer.obj
 0001:0007da20       ?ConvertOut@ModularArithmetic@TaoCrypt@@UBE?AVInteger@2@ABV32@@Z 0047ea20 f i taocrypt:integer.obj
 0001:0007da40       ?Identity@ModularArithmetic@TaoCrypt@@UBEABVInteger@2@XZ 0047ea40 f i taocrypt:integer.obj
 0001:0007da50       ?MultiplicativeIdentity@ModularArithmetic@TaoCrypt@@UBEABVInteger@2@XZ 0047ea50 f i taocrypt:integer.obj
 0001:0007da60       ?Encode@Integer@TaoCrypt@@QBEIPAEIW4Signedness@12@@Z 0047ea60 f   taocrypt:integer.obj
 0001:0007db50       ?Randomize@Integer@TaoCrypt@@QAEXAAVRandomNumberGenerator@2@ABV12@1@Z 0047eb50 f   taocrypt:integer.obj
 0001:0007dbc0       ?Divide@Integer@TaoCrypt@@SAXAAV12@0ABV12@1@Z 0047ebc0 f   taocrypt:integer.obj
 0001:0007dc70       ?DivideByPowerOf2@Integer@TaoCrypt@@SAXAAV12@0ABV12@I@Z 0047ec70 f   taocrypt:integer.obj
 0001:0007dde0       ?DividedBy@Integer@TaoCrypt@@QBE?AV12@ABV12@@Z 0047ede0 f   taocrypt:integer.obj
 0001:0007de30       ?Modulo@Integer@TaoCrypt@@QBE?AV12@ABV12@@Z 0047ee30 f   taocrypt:integer.obj
 0001:0007de80       ?Divide@Integer@TaoCrypt@@SAXAAIAAV12@ABV12@I@Z 0047ee80 f   taocrypt:integer.obj
 0001:0007dfd0       ?DividedBy@Integer@TaoCrypt@@QBE?AV12@I@Z 0047efd0 f   taocrypt:integer.obj
 0001:0007e000       ?a_exp_b_mod_c@TaoCrypt@@YA?AVInteger@1@ABV21@00@Z 0047f000 f   taocrypt:integer.obj
 0001:0007e0a0       ?Half@ModularArithmetic@TaoCrypt@@QBEABVInteger@2@ABV32@@Z 0047f0a0 f   taocrypt:integer.obj
 0001:0007e1c0       ?Add@ModularArithmetic@TaoCrypt@@UBEABVInteger@2@ABV32@0@Z 0047f1c0 f   taocrypt:integer.obj
 0001:0007e280       ?Subtract@ModularArithmetic@TaoCrypt@@UBEABVInteger@2@ABV32@0@Z 0047f280 f   taocrypt:integer.obj
 0001:0007e330       ??0MontgomeryRepresentation@TaoCrypt@@QAE@ABVInteger@1@@Z 0047f330 f   taocrypt:integer.obj
 0001:0007e3e0       ?IsMontgomeryRepresentation@MontgomeryRepresentation@TaoCrypt@@UBE_NXZ 0047f3e0 f i taocrypt:integer.obj
 0001:0007e3f0       ??_GMontgomeryRepresentation@TaoCrypt@@UAEPAXI@Z 0047f3f0 f i taocrypt:integer.obj
 0001:0007e3f0       ??_EMontgomeryRepresentation@TaoCrypt@@UAEPAXI@Z 0047f3f0 f i taocrypt:integer.obj
 0001:0007e410       ??KTaoCrypt@@YA?AVInteger@0@ABV10@0@Z 0047f410 f i taocrypt:integer.obj
 0001:0007e430       ??LTaoCrypt@@YA?AVInteger@0@ABV10@0@Z 0047f430 f i taocrypt:integer.obj
 0001:0007e450       ?ModularExponentiation@TaoCrypt@@YA?AVInteger@1@ABV21@00@Z 0047f450 f i taocrypt:integer.obj
 0001:0007e480       ??0EuclideanDomainOf@TaoCrypt@@QAE@XZ 0047f480 f i taocrypt:integer.obj
 0001:0007e4b0       ?IsUnit@EuclideanDomainOf@TaoCrypt@@UBE_NABVInteger@2@@Z 0047f4b0 f i taocrypt:integer.obj
 0001:0007e4c0       ?Equal@EuclideanDomainOf@TaoCrypt@@UBE_NABVInteger@2@0@Z 0047f4c0 f i taocrypt:integer.obj
 0001:0007e4e0       ??_EEuclideanDomainOf@TaoCrypt@@UAEPAXI@Z 0047f4e0 f i taocrypt:integer.obj
 0001:0007e4e0       ??_GEuclideanDomainOf@TaoCrypt@@UAEPAXI@Z 0047f4e0 f i taocrypt:integer.obj
 0001:0007e520       ?Accumulate@EuclideanDomainOf@TaoCrypt@@UBEAAVInteger@2@AAV32@ABV32@@Z 0047f520 f i taocrypt:integer.obj
 0001:0007e540       ?Reduce@EuclideanDomainOf@TaoCrypt@@UBEAAVInteger@2@AAV32@ABV32@@Z 0047f540 f i taocrypt:integer.obj
 0001:0007e560       ?Doubled@Integer@TaoCrypt@@QBE?AV12@XZ 0047f560 f i taocrypt:integer.obj
 0001:0007e580       ?Identity@EuclideanDomainOf@TaoCrypt@@UBEABVInteger@2@XZ 0047f580 f i taocrypt:integer.obj
 0001:0007e590       ?Add@EuclideanDomainOf@TaoCrypt@@UBEABVInteger@2@ABV32@0@Z 0047f590 f i taocrypt:integer.obj
 0001:0007e5e0       ?Inverse@EuclideanDomainOf@TaoCrypt@@UBEABVInteger@2@ABV32@@Z 0047f5e0 f i taocrypt:integer.obj
 0001:0007e620       ?Subtract@EuclideanDomainOf@TaoCrypt@@UBEABVInteger@2@ABV32@0@Z 0047f620 f i taocrypt:integer.obj
 0001:0007e670       ?Double@EuclideanDomainOf@TaoCrypt@@UBEABVInteger@2@ABV32@@Z 0047f670 f i taocrypt:integer.obj
 0001:0007e6b0       ?MultiplicativeIdentity@EuclideanDomainOf@TaoCrypt@@UBEABVInteger@2@XZ 0047f6b0 f i taocrypt:integer.obj
 0001:0007e6c0       ?Multiply@EuclideanDomainOf@TaoCrypt@@UBEABVInteger@2@ABV32@0@Z 0047f6c0 f i taocrypt:integer.obj
 0001:0007e710       ?Square@EuclideanDomainOf@TaoCrypt@@UBEABVInteger@2@ABV32@@Z 0047f710 f i taocrypt:integer.obj
 0001:0007e750       ?MultiplicativeInverse@EuclideanDomainOf@TaoCrypt@@UBEABVInteger@2@ABV32@@Z 0047f750 f i taocrypt:integer.obj
 0001:0007e790       ?Divide@EuclideanDomainOf@TaoCrypt@@UBEABVInteger@2@ABV32@0@Z 0047f790 f i taocrypt:integer.obj
 0001:0007e7e0       ?Mod@EuclideanDomainOf@TaoCrypt@@UBEABVInteger@2@ABV32@0@Z 0047f7e0 f i taocrypt:integer.obj
 0001:0007e830       ?DivisionAlgorithm@EuclideanDomainOf@TaoCrypt@@UBEXAAVInteger@2@0ABV32@1@Z 0047f830 f i taocrypt:integer.obj
 0001:0007e850       ?ConvertIn@ModularArithmetic@TaoCrypt@@UBE?AVInteger@2@ABV32@@Z 0047f850 f i taocrypt:integer.obj
 0001:0007e870       ?Multiply@ModularArithmetic@TaoCrypt@@UBEABVInteger@2@ABV32@0@Z 0047f870 f i taocrypt:integer.obj
 0001:0007e8e0       ?Square@ModularArithmetic@TaoCrypt@@UBEABVInteger@2@ABV32@@Z 0047f8e0 f i taocrypt:integer.obj
 0001:0007e950       ?ConvertIn@MontgomeryRepresentation@TaoCrypt@@UBE?AVInteger@2@ABV32@@Z 0047f950 f i taocrypt:integer.obj
 0001:0007e9c0       ?MultiplicativeIdentity@MontgomeryRepresentation@TaoCrypt@@UBEABVInteger@2@XZ 0047f9c0 f i taocrypt:integer.obj
 0001:0007ea30       ??0Integer@TaoCrypt@@QAE@AAVRandomNumberGenerator@1@ABV01@1@Z 0047fa30 f   taocrypt:integer.obj
 0001:0007eaa0       ?SquareRoot@Integer@TaoCrypt@@QBE?AV12@XZ 0047faa0 f   taocrypt:integer.obj
 0001:0007ec00       ?IsSquare@Integer@TaoCrypt@@QBE_NXZ 0047fc00 f   taocrypt:integer.obj
 0001:0007ec60       ?a_times_b_mod_c@TaoCrypt@@YA?AVInteger@1@ABV21@00@Z 0047fc60 f   taocrypt:integer.obj
 0001:0007ecb0       ?Gcd@Integer@TaoCrypt@@SA?AV12@ABV12@0@Z 0047fcb0 f   taocrypt:integer.obj
 0001:0007ed30       ?InverseMod@Integer@TaoCrypt@@QBE?AV12@ABV12@@Z 0047fd30 f   taocrypt:integer.obj
 0001:0007efc0       ?CascadeExponentiate@ModularArithmetic@TaoCrypt@@UBE?AVInteger@2@ABV32@000@Z 0047ffc0 f   taocrypt:integer.obj
 0001:0007f0e0       ?SimultaneousExponentiate@ModularArithmetic@TaoCrypt@@UBEXPAVInteger@2@ABV32@PBV32@I@Z 004800e0 f   taocrypt:integer.obj
 0001:0007f210       ?CRT@TaoCrypt@@YA?AVInteger@1@ABV21@0000@Z 00480210 f   taocrypt:integer.obj
 0001:0007f2d0       ?IsUnit@ModularArithmetic@TaoCrypt@@UBE_NABVInteger@2@@Z 004802d0 f i taocrypt:integer.obj
 0001:0007f310       ?MultiplicativeInverse@ModularArithmetic@TaoCrypt@@UBEABVInteger@2@ABV32@@Z 00480310 f i taocrypt:integer.obj
 0001:0007f350       ?ModularRoot@TaoCrypt@@YA?AVInteger@1@ABV21@00000@Z 00480350 f   taocrypt:integer.obj
 0001:0007f420       ??1SHA256@TaoCrypt@@UAE@XZ 00480420 f i taocrypt:sha.obj
 0001:0007f430       ??1SHA224@TaoCrypt@@UAE@XZ 00480430 f i taocrypt:sha.obj
 0001:0007f440       ??1SHA512@TaoCrypt@@UAE@XZ 00480440 f i taocrypt:sha.obj
 0001:0007f450       ??1SHA384@TaoCrypt@@UAE@XZ 00480450 f i taocrypt:sha.obj
 0001:0007f460       ?Init@SHA@TaoCrypt@@UAEXXZ 00480460 f   taocrypt:sha.obj
 0001:0007f490       ?Init@SHA256@TaoCrypt@@UAEXXZ 00480490 f   taocrypt:sha.obj
 0001:0007f4e0       ?Init@SHA224@TaoCrypt@@UAEXXZ 004804e0 f   taocrypt:sha.obj
 0001:0007f530       ?Init@SHA512@TaoCrypt@@UAEXXZ 00480530 f   taocrypt:sha.obj
 0001:0007f5b0       ?Init@SHA384@TaoCrypt@@UAEXXZ 004805b0 f   taocrypt:sha.obj
 0001:0007f630       ??0SHA@TaoCrypt@@QAE@ABV01@@Z 00480630 f   taocrypt:sha.obj
 0001:0007f690       ??0SHA256@TaoCrypt@@QAE@ABV01@@Z 00480690 f   taocrypt:sha.obj
 0001:0007f6e0       ?getByteOrder@SHA256@TaoCrypt@@UBE?AW4ByteOrder@2@XZ 004806e0 f i taocrypt:sha.obj
 0001:0007f6f0       ?getBlockSize@SHA256@TaoCrypt@@UBEIXZ 004806f0 f i taocrypt:sha.obj
 0001:0007f700       ?getDigestSize@SHA256@TaoCrypt@@UBEIXZ 00480700 f i taocrypt:sha.obj
 0001:0007f710       ?getPadSize@SHA256@TaoCrypt@@UBEIXZ 00480710 f i taocrypt:sha.obj
 0001:0007f720       ??0SHA224@TaoCrypt@@QAE@ABV01@@Z 00480720 f   taocrypt:sha.obj
 0001:0007f770       ?getByteOrder@SHA224@TaoCrypt@@UBE?AW4ByteOrder@2@XZ 00480770 f i taocrypt:sha.obj
 0001:0007f780       ?getBlockSize@SHA224@TaoCrypt@@UBEIXZ 00480780 f i taocrypt:sha.obj
 0001:0007f790       ?getDigestSize@SHA224@TaoCrypt@@UBEIXZ 00480790 f i taocrypt:sha.obj
 0001:0007f7a0       ?getPadSize@SHA224@TaoCrypt@@UBEIXZ 004807a0 f i taocrypt:sha.obj
 0001:0007f7b0       ??0SHA512@TaoCrypt@@QAE@ABV01@@Z 004807b0 f   taocrypt:sha.obj
 0001:0007f800       ?getByteOrder@SHA512@TaoCrypt@@UBE?AW4ByteOrder@2@XZ 00480800 f i taocrypt:sha.obj
 0001:0007f810       ?getBlockSize@SHA512@TaoCrypt@@UBEIXZ 00480810 f i taocrypt:sha.obj
 0001:0007f820       ?getDigestSize@SHA512@TaoCrypt@@UBEIXZ 00480820 f i taocrypt:sha.obj
 0001:0007f830       ?getPadSize@SHA512@TaoCrypt@@UBEIXZ 00480830 f i taocrypt:sha.obj
 0001:0007f840       ??0SHA384@TaoCrypt@@QAE@ABV01@@Z 00480840 f   taocrypt:sha.obj
 0001:0007f890       ?getByteOrder@SHA384@TaoCrypt@@UBE?AW4ByteOrder@2@XZ 00480890 f i taocrypt:sha.obj
 0001:0007f8a0       ?getBlockSize@SHA384@TaoCrypt@@UBEIXZ 004808a0 f i taocrypt:sha.obj
 0001:0007f8b0       ?getDigestSize@SHA384@TaoCrypt@@UBEIXZ 004808b0 f i taocrypt:sha.obj
 0001:0007f8c0       ?getPadSize@SHA384@TaoCrypt@@UBEIXZ 004808c0 f i taocrypt:sha.obj
 0001:0007f8d0       ?Transform@SHA@TaoCrypt@@EAEXXZ 004808d0 f   taocrypt:sha.obj
 0001:000816e0       ?Transform@SHA256@TaoCrypt@@EAEXXZ 004826e0 f   taocrypt:sha.obj
 0001:00081700       ?Transform@SHA224@TaoCrypt@@EAEXXZ 00482700 f   taocrypt:sha.obj
 0001:00081720       ?AsmTransform@SHA@TaoCrypt@@AAEXPBEI@Z 00482720 f   taocrypt:sha.obj
 0001:000826c0       ??$rotrFixed@_K@TaoCrypt@@YA_K_KI@Z 004836c0 f i taocrypt:sha.obj
 0001:00082710       ??_GSHA256@TaoCrypt@@UAEPAXI@Z 00483710 f i taocrypt:sha.obj
 0001:00082710       ??_ESHA256@TaoCrypt@@UAEPAXI@Z 00483710 f i taocrypt:sha.obj
 0001:00082730       ??_GSHA224@TaoCrypt@@UAEPAXI@Z 00483730 f i taocrypt:sha.obj
 0001:00082730       ??_ESHA224@TaoCrypt@@UAEPAXI@Z 00483730 f i taocrypt:sha.obj
 0001:00082750       ??_ESHA512@TaoCrypt@@UAEPAXI@Z 00483750 f i taocrypt:sha.obj
 0001:00082750       ??_GSHA512@TaoCrypt@@UAEPAXI@Z 00483750 f i taocrypt:sha.obj
 0001:00082770       ??_ESHA384@TaoCrypt@@UAEPAXI@Z 00483770 f i taocrypt:sha.obj
 0001:00082770       ??_GSHA384@TaoCrypt@@UAEPAXI@Z 00483770 f i taocrypt:sha.obj
 0001:00082790       ?Swap@SHA@TaoCrypt@@QAEXAAV12@@Z 00483790 f   taocrypt:sha.obj
 0001:000827f0       ?Swap@SHA256@TaoCrypt@@QAEXAAV12@@Z 004837f0 f   taocrypt:sha.obj
 0001:00082840       ?Swap@SHA224@TaoCrypt@@QAEXAAV12@@Z 00483840 f   taocrypt:sha.obj
 0001:00082890       ?Swap@SHA512@TaoCrypt@@QAEXAAV12@@Z 00483890 f   taocrypt:sha.obj
 0001:000828e0       ?Swap@SHA384@TaoCrypt@@QAEXAAV12@@Z 004838e0 f   taocrypt:sha.obj
 0001:00082930       ?Update@SHA@TaoCrypt@@UAEXPBEI@Z 00483930 f   taocrypt:sha.obj
 0001:00084ce0       ?Transform@SHA512@TaoCrypt@@EAEXXZ 00485ce0 f   taocrypt:sha.obj
 0001:00084d00       ?Transform@SHA384@TaoCrypt@@EAEXXZ 00485d00 f   taocrypt:sha.obj
 0001:00084d20       ??4SHA@TaoCrypt@@QAEAAV01@ABV01@@Z 00485d20 f   taocrypt:sha.obj
 0001:00084d50       ??4SHA256@TaoCrypt@@QAEAAV01@ABV01@@Z 00485d50 f   taocrypt:sha.obj
 0001:00084d80       ??4SHA224@TaoCrypt@@QAEAAV01@ABV01@@Z 00485d80 f   taocrypt:sha.obj
 0001:00084db0       ??4SHA512@TaoCrypt@@QAEAAV01@ABV01@@Z 00485db0 f   taocrypt:sha.obj
 0001:00084de0       ??4SHA384@TaoCrypt@@QAEAAV01@ABV01@@Z 00485de0 f   taocrypt:sha.obj
 0001:00084e10       ?Init@RIPEMD160@TaoCrypt@@UAEXXZ 00485e10 f   taocrypt:ripemd.obj
 0001:00084e40       ??0RIPEMD160@TaoCrypt@@QAE@ABV01@@Z 00485e40 f   taocrypt:ripemd.obj
 0001:00084ea0       ?Transform@RIPEMD160@TaoCrypt@@EAEXXZ 00485ea0 f   taocrypt:ripemd.obj
 0001:00086980       ?AsmTransform@RIPEMD160@TaoCrypt@@AAEXPBEI@Z 00487980 f   taocrypt:ripemd.obj
 0001:000879a0       ?Swap@RIPEMD160@TaoCrypt@@QAEXAAV12@@Z 004889a0 f   taocrypt:ripemd.obj
 0001:00087a00       ?Update@RIPEMD160@TaoCrypt@@UAEXPBEI@Z 00488a00 f   taocrypt:ripemd.obj
 0001:00087ad0       ??4RIPEMD160@TaoCrypt@@QAEAAV01@ABV01@@Z 00488ad0 f   taocrypt:ripemd.obj
 0001:00087b00       ?XorWords@TaoCrypt@@YAXPAIPBII@Z 00488b00 f i taocrypt:misc.obj
 0001:00087b30       ?xorbuf@TaoCrypt@@YAXPAEPBEI@Z 00488b30 f   taocrypt:misc.obj
 0001:00087b80       ?BytePrecision@TaoCrypt@@YAII@Z 00488b80 f   taocrypt:misc.obj
 0001:00087bb0       ?BitPrecision@TaoCrypt@@YAII@Z 00488bb0 f   taocrypt:misc.obj
 0001:00087bf0       ?Crop@TaoCrypt@@YAIII@Z    00488bf0 f   taocrypt:misc.obj
 0001:00087c10       ?HaveCpuId@TaoCrypt@@YA_NXZ 00488c10 f   taocrypt:misc.obj
 0001:00087c90       ?CpuId@TaoCrypt@@YAXIPAI@Z 00488c90 f   taocrypt:misc.obj
 0001:00087cb0       ?IsPentium@TaoCrypt@@YA_NXZ 00488cb0 f   taocrypt:misc.obj
 0001:00087dd0       ?ReverseDir@TaoCrypt@@YA?AW4CipherDir@1@W421@@Z 00488dd0 f i taocrypt:des.obj
 0001:00087de0       ?UnalignedGetWordNonTemplate@TaoCrypt@@YAIW4ByteOrder@1@PBEPAI@Z 00488de0 f i taocrypt:des.obj
 0001:00087e20       ?UnalignedPutWord@TaoCrypt@@YAXW4ByteOrder@1@PAEIPBE@Z 00488e20 f i taocrypt:des.obj
 0001:00087f80       ?RawProcessBlock@BasicDES@TaoCrypt@@QBEXAAI0@Z 00488f80 f   taocrypt:des.obj
 0001:000880c0       ?AsmProcess@DES_EDE3@TaoCrypt@@ABEXPBEPAEPAX@Z 004890c0 f   taocrypt:des.obj
 0001:000896f0       ??0?$PutBlock@IU?$EnumToType@W4ByteOrder@TaoCrypt@@$00@TaoCrypt@@$00@TaoCrypt@@QAE@PBXPAX@Z 0048a6f0 f i taocrypt:des.obj
 0001:00089710       ??0?$GetBlock@IU?$EnumToType@W4ByteOrder@TaoCrypt@@$00@TaoCrypt@@$00@TaoCrypt@@QAE@PBX@Z 0048a710 f i taocrypt:des.obj
 0001:00089720       ?ToEnum@?$EnumToType@W4ByteOrder@TaoCrypt@@$00@TaoCrypt@@SA?AW4ByteOrder@2@XZ 0048a720 f i taocrypt:des.obj
 0001:00089730       ??$UnalignedGetWord@I@TaoCrypt@@YAIW4ByteOrder@0@PBEPAI@Z 0048a730 f i taocrypt:des.obj
 0001:00089770       ?SetKey@BasicDES@TaoCrypt@@QAEXPBEIW4CipherDir@2@@Z 0048a770 f   taocrypt:des.obj
 0001:00089b50       ?SetKey@DES_EDE2@TaoCrypt@@QAEXPBEIW4CipherDir@2@@Z 0048ab50 f   taocrypt:des.obj
 0001:00089b90       ?SetKey@DES_EDE3@TaoCrypt@@QAEXPBEIW4CipherDir@2@@Z 0048ab90 f   taocrypt:des.obj
 0001:00089c00       ?Process@DES_EDE3@TaoCrypt@@UAEXPAEPBEI@Z 0048ac00 f   taocrypt:des.obj
 0001:00089d40       ?Get@?$BlockGetAndPut@IU?$EnumToType@W4ByteOrder@TaoCrypt@@$00@TaoCrypt@@$00@TaoCrypt@@SA?AV?$GetBlock@IU?$EnumToType@W4ByteOrder@TaoCrypt@@$00@TaoCrypt@@$00@2@PBX@Z 0048ad40 f i taocrypt:des.obj
 0001:00089d50       ??$ByteReverseIf@I@TaoCrypt@@YAIIW4ByteOrder@0@@Z 0048ad50 f i taocrypt:des.obj
 0001:00089d80       ??$GetWord@I@TaoCrypt@@YAI_NW4ByteOrder@0@PBE@Z 0048ad80 f i taocrypt:des.obj
 0001:00089df0       ??$PutWord@I@TaoCrypt@@YAX_NW4ByteOrder@0@PAEIPBE@Z 0048adf0 f i taocrypt:des.obj
 0001:00089e90       ??$?RI@?$GetBlock@IU?$EnumToType@W4ByteOrder@TaoCrypt@@$00@TaoCrypt@@$00@TaoCrypt@@QAEAAV01@AAI@Z 0048ae90 f i taocrypt:des.obj
 0001:00089ec0       ??$?RI@?$PutBlock@IU?$EnumToType@W4ByteOrder@TaoCrypt@@$00@TaoCrypt@@$00@TaoCrypt@@QAEAAV01@I@Z 0048aec0 f i taocrypt:des.obj
 0001:00089f20       ?ProcessAndXorBlock@DES@TaoCrypt@@EBEXPBE0PAE@Z 0048af20 f   taocrypt:des.obj
 0001:00089fc0       ?ProcessAndXorBlock@DES_EDE2@TaoCrypt@@EBEXPBE0PAE@Z 0048afc0 f   taocrypt:des.obj
 0001:0008a090       ?ProcessAndXorBlock@DES_EDE3@TaoCrypt@@EBEXPBE0PAE@Z 0048b090 f   taocrypt:des.obj
 0001:0008a160       ?AsmEncrypt@AES@TaoCrypt@@ABEXPBEPAEPAX@Z 0048b160 f   taocrypt:aes.obj
 0001:0008a420       ?AsmDecrypt@AES@TaoCrypt@@ABEXPBEPAEPAX@Z 0048b420 f   taocrypt:aes.obj
 0001:0008a6e0       ??$IsPowerOf2@I@TaoCrypt@@YA_NI@Z 0048b6e0 f i taocrypt:aes.obj
 0001:0008a700       ??$ModPowerOf2@II@TaoCrypt@@YAIII@Z 0048b700 f i taocrypt:aes.obj
 0001:0008a710       ??$RoundDownToMultipleOf@I@TaoCrypt@@YAIII@Z 0048b710 f i taocrypt:aes.obj
 0001:0008a740       ?Process@AES@TaoCrypt@@UAEXPAEPBEI@Z 0048b740 f   taocrypt:aes.obj
 0001:0008a8e0       ??$RoundUpToMultipleOf@I@TaoCrypt@@YAIII@Z 0048b8e0 f i taocrypt:aes.obj
 0001:0008a910       ??$GetUserKey@I@TaoCrypt@@YAXW4ByteOrder@0@PAIIPBEI@Z 0048b910 f i taocrypt:aes.obj
 0001:0008a970       ?SetKey@AES@TaoCrypt@@QAEXPBEIW4CipherDir@2@@Z 0048b970 f   taocrypt:aes.obj
 0001:0008af60       ?encrypt@AES@TaoCrypt@@ABEXPBE0PAE@Z 0048bf60 f   taocrypt:aes.obj
 0001:0008b4b0       ?decrypt@AES@TaoCrypt@@ABEXPBE0PAE@Z 0048c4b0 f   taocrypt:aes.obj
 0001:0008ba10       ?ProcessAndXorBlock@AES@TaoCrypt@@EBEXPBE0PAE@Z 0048ca10 f   taocrypt:aes.obj
 0001:0008ba20       ?GenerateBlock@RandomNumberGenerator@TaoCrypt@@QAEXPAEI@Z 0048ca20 f   taocrypt:random.obj
 0001:0008ba50       ?GenerateByte@RandomNumberGenerator@TaoCrypt@@QAEEXZ 0048ca50 f   taocrypt:random.obj
 0001:0008ba70       ??0OS_Seed@TaoCrypt@@QAE@XZ 0048ca70 f   taocrypt:random.obj
 0001:0008baa0       ??1OS_Seed@TaoCrypt@@QAE@XZ 0048caa0 f   taocrypt:random.obj
 0001:0008bab0       ?GenerateSeed@OS_Seed@TaoCrypt@@QAEXPAEI@Z 0048cab0 f   taocrypt:random.obj
 0001:0008bae0       ??0RandomNumberGenerator@TaoCrypt@@QAE@XZ 0048cae0 f   taocrypt:random.obj
 0001:0008bb50       ?SetKey@ARC4@TaoCrypt@@QAEXPBEI@Z 0048cb50 f   taocrypt:arc4.obj
 0001:0008bbc0       ?MakeByte@?A0xdd0b7750@TaoCrypt@@YAIAAI0PAE@Z 0048cbc0 f i taocrypt:arc4.obj
 0001:0008bc10       ?AsmProcess@ARC4@TaoCrypt@@AAEXPAEPBEI@Z 0048cc10 f   taocrypt:arc4.obj
 0001:0008bca0       ?Process@ARC4@TaoCrypt@@QAEXPAEPBEI@Z 0048cca0 f   taocrypt:arc4.obj
 0001:0008bdd0       ??0BER_Decoder@TaoCrypt@@QAE@AAVSource@1@@Z 0048cdd0 f i taocrypt:dsa.obj
 0001:0008bdf0       ??1BER_Decoder@TaoCrypt@@UAE@XZ 0048cdf0 f i taocrypt:dsa.obj
 0001:0008be00       ??_GBER_Decoder@TaoCrypt@@UAEPAXI@Z 0048ce00 f i taocrypt:dsa.obj
 0001:0008be00       ??_EBER_Decoder@TaoCrypt@@UAEPAXI@Z 0048ce00 f i taocrypt:dsa.obj
 0001:0008be20       ??0DSA_Private_Decoder@TaoCrypt@@QAE@AAVSource@1@@Z 0048ce20 f i taocrypt:dsa.obj
 0001:0008be40       ??1DSA_Private_Decoder@TaoCrypt@@UAE@XZ 0048ce40 f i taocrypt:dsa.obj
 0001:0008be50       ??0DSA_Public_Decoder@TaoCrypt@@QAE@AAVSource@1@@Z 0048ce50 f i taocrypt:dsa.obj
 0001:0008be70       ??1DSA_Public_Decoder@TaoCrypt@@UAE@XZ 0048ce70 f i taocrypt:dsa.obj
 0001:0008be80       ?Swap@DSA_PublicKey@TaoCrypt@@QAEXAAV12@@Z 0048ce80 f   taocrypt:dsa.obj
 0001:0008bec0       ?Initialize@DSA_PublicKey@TaoCrypt@@QAEXAAVSource@2@@Z 0048cec0 f   taocrypt:dsa.obj
 0001:0008bef0       ?Initialize@DSA_PublicKey@TaoCrypt@@QAEXABVInteger@2@000@Z 0048cef0 f   taocrypt:dsa.obj
 0001:0008bf30       ?GetModulus@DSA_PublicKey@TaoCrypt@@QBEABVInteger@2@XZ 0048cf30 f   taocrypt:dsa.obj
 0001:0008bf40       ?GetSubGroupOrder@DSA_PublicKey@TaoCrypt@@QBEABVInteger@2@XZ 0048cf40 f   taocrypt:dsa.obj
 0001:0008bf50       ?GetSubGroupGenerator@DSA_PublicKey@TaoCrypt@@QBEABVInteger@2@XZ 0048cf50 f   taocrypt:dsa.obj
 0001:0008bf60       ?GetPublicPart@DSA_PublicKey@TaoCrypt@@QBEABVInteger@2@XZ 0048cf60 f   taocrypt:dsa.obj
 0001:0008bf70       ?SetModulus@DSA_PublicKey@TaoCrypt@@QAEXABVInteger@2@@Z 0048cf70 f   taocrypt:dsa.obj
 0001:0008bf80       ?SetSubGroupOrder@DSA_PublicKey@TaoCrypt@@QAEXABVInteger@2@@Z 0048cf80 f   taocrypt:dsa.obj
 0001:0008bf90       ?SetSubGroupGenerator@DSA_PublicKey@TaoCrypt@@QAEXABVInteger@2@@Z 0048cf90 f   taocrypt:dsa.obj
 0001:0008bfa0       ?SetPublicPart@DSA_PublicKey@TaoCrypt@@QAEXABVInteger@2@@Z 0048cfa0 f   taocrypt:dsa.obj
 0001:0008bfb0       ?SignatureLength@DSA_PublicKey@TaoCrypt@@QBEIXZ 0048cfb0 f   taocrypt:dsa.obj
 0001:0008bfc0       ?Initialize@DSA_PrivateKey@TaoCrypt@@QAEXAAVSource@2@@Z 0048cfc0 f   taocrypt:dsa.obj
 0001:0008bff0       ?Initialize@DSA_PrivateKey@TaoCrypt@@QAEXABVInteger@2@0000@Z 0048cff0 f   taocrypt:dsa.obj
 0001:0008c020       ?GetPrivatePart@DSA_PrivateKey@TaoCrypt@@QBEABVInteger@2@XZ 0048d020 f   taocrypt:dsa.obj
 0001:0008c030       ?SetPrivatePart@DSA_PrivateKey@TaoCrypt@@QAEXABVInteger@2@@Z 0048d030 f   taocrypt:dsa.obj
 0001:0008c040       ?GetR@DSA_Signer@TaoCrypt@@QBEABVInteger@2@XZ 0048d040 f   taocrypt:dsa.obj
 0001:0008c050       ?GetS@DSA_Signer@TaoCrypt@@QBEABVInteger@2@XZ 0048d050 f   taocrypt:dsa.obj
 0001:0008c060       ?GetR@DSA_Verifier@TaoCrypt@@QBEABVInteger@2@XZ 0048d060 f   taocrypt:dsa.obj
 0001:0008c070       ?GetS@DSA_Verifier@TaoCrypt@@QBEABVInteger@2@XZ 0048d070 f   taocrypt:dsa.obj
 0001:0008c080       ??_1Integer@TaoCrypt@@QAEAAV01@ABV01@@Z 0048d080 f i taocrypt:dsa.obj
 0001:0008c0c0       ??_EDSA_Private_Decoder@TaoCrypt@@UAEPAXI@Z 0048d0c0 f i taocrypt:dsa.obj
 0001:0008c0c0       ??_GDSA_Private_Decoder@TaoCrypt@@UAEPAXI@Z 0048d0c0 f i taocrypt:dsa.obj
 0001:0008c0e0       ??_EDSA_Public_Decoder@TaoCrypt@@UAEPAXI@Z 0048d0e0 f i taocrypt:dsa.obj
 0001:0008c0e0       ??_GDSA_Public_Decoder@TaoCrypt@@UAEPAXI@Z 0048d0e0 f i taocrypt:dsa.obj
 0001:0008c100       ??0DSA_PublicKey@TaoCrypt@@QAE@ABV01@@Z 0048d100 f   taocrypt:dsa.obj
 0001:0008c140       ??4DSA_PublicKey@TaoCrypt@@QAEAAV01@ABV01@@Z 0048d140 f   taocrypt:dsa.obj
 0001:0008c1c0       ??0DSA_PublicKey@TaoCrypt@@QAE@AAVSource@1@@Z 0048d1c0 f   taocrypt:dsa.obj
 0001:0008c200       ??0DSA_PrivateKey@TaoCrypt@@QAE@AAVSource@1@@Z 0048d200 f   taocrypt:dsa.obj
 0001:0008c240       ??0DSA_Signer@TaoCrypt@@QAE@ABVDSA_PrivateKey@1@@Z 0048d240 f   taocrypt:dsa.obj
 0001:0008c260       ?Sign@DSA_Signer@TaoCrypt@@QAEIPBEPAEAAVRandomNumberGenerator@2@@Z 0048d260 f   taocrypt:dsa.obj
 0001:0008c4c0       ??0DSA_Verifier@TaoCrypt@@QAE@ABVDSA_PublicKey@1@@Z 0048d4c0 f   taocrypt:dsa.obj
 0001:0008c4e0       ?Verify@DSA_Verifier@TaoCrypt@@QAE_NPBE0@Z 0048d4e0 f   taocrypt:dsa.obj
 0001:0008c820       ??0DH_Decoder@TaoCrypt@@QAE@AAVSource@1@@Z 0048d820 f i taocrypt:dh.obj
 0001:0008c840       ??1DH_Decoder@TaoCrypt@@UAE@XZ 0048d840 f i taocrypt:dh.obj
 0001:0008c850       ?DiscreteLogWorkFactor@?A0xec28e698@TaoCrypt@@YAII@Z 0048d850 f   taocrypt:dh.obj
 0001:0008c8d0       ?Initialize@DH@TaoCrypt@@QAEXAAVSource@2@@Z 0048d8d0 f   taocrypt:dh.obj
 0001:0008c900       ??$min@VInteger@TaoCrypt@@@TaoCrypt@@YAABVInteger@0@ABV10@0@Z 0048d900 f i taocrypt:dh.obj
 0001:0008c920       ??_EDH_Decoder@TaoCrypt@@UAEPAXI@Z 0048d920 f i taocrypt:dh.obj
 0001:0008c920       ??_GDH_Decoder@TaoCrypt@@UAEPAXI@Z 0048d920 f i taocrypt:dh.obj
 0001:0008c940       ?GeneratePrivate@DH@TaoCrypt@@AAEXAAVRandomNumberGenerator@2@PAE@Z 0048d940 f   taocrypt:dh.obj
 0001:0008ca20       ?GeneratePublic@DH@TaoCrypt@@AAEXPBEPAE@Z 0048da20 f   taocrypt:dh.obj
 0001:0008caa0       ?Agree@DH@TaoCrypt@@QAEXPAEPBE1I@Z 0048daa0 f   taocrypt:dh.obj
 0001:0008cb60       ??0DH@TaoCrypt@@QAE@AAVSource@1@@Z 0048db60 f   taocrypt:dh.obj
 0001:0008cb90       ?GenerateKeyPair@DH@TaoCrypt@@QAEXAAVRandomNumberGenerator@2@PAE1@Z 0048db90 f   taocrypt:dh.obj
 0001:0008cbc0       ??0RSA_Private_Decoder@TaoCrypt@@QAE@AAVSource@1@@Z 0048dbc0 f i taocrypt:rsa.obj
 0001:0008cbe0       ??1RSA_Private_Decoder@TaoCrypt@@UAE@XZ 0048dbe0 f i taocrypt:rsa.obj
 0001:0008cbf0       ??0RSA_Public_Decoder@TaoCrypt@@QAE@AAVSource@1@@Z 0048dbf0 f i taocrypt:rsa.obj
 0001:0008cc10       ??1RSA_Public_Decoder@TaoCrypt@@UAE@XZ 0048dc10 f i taocrypt:rsa.obj
 0001:0008cc20       ?Initialize@RSA_PublicKey@TaoCrypt@@QAEXAAVSource@2@@Z 0048dc20 f   taocrypt:rsa.obj
 0001:0008cc50       ?Initialize@RSA_PrivateKey@TaoCrypt@@QAEXAAVSource@2@@Z 0048dc50 f   taocrypt:rsa.obj
 0001:0008cc80       ?Pad@RSA_BlockType2@TaoCrypt@@QBEXPBEIPAEIAAVRandomNumberGenerator@2@@Z 0048dc80 f   taocrypt:rsa.obj
 0001:0008ccf0       ?Pad@RSA_BlockType1@TaoCrypt@@QBEXPBEIPAEIAAVRandomNumberGenerator@2@@Z 0048dcf0 f   taocrypt:rsa.obj
 0001:0008cd50       ??_ERSA_Private_Decoder@TaoCrypt@@UAEPAXI@Z 0048dd50 f i taocrypt:rsa.obj
 0001:0008cd50       ??_GRSA_Private_Decoder@TaoCrypt@@UAEPAXI@Z 0048dd50 f i taocrypt:rsa.obj
 0001:0008cd70       ??_GRSA_Public_Decoder@TaoCrypt@@UAEPAXI@Z 0048dd70 f i taocrypt:rsa.obj
 0001:0008cd70       ??_ERSA_Public_Decoder@TaoCrypt@@UAEPAXI@Z 0048dd70 f i taocrypt:rsa.obj
 0001:0008cd90       ?ApplyFunction@RSA_PublicKey@TaoCrypt@@QBE?AVInteger@2@ABV32@@Z 0048dd90 f   taocrypt:rsa.obj
 0001:0008cdb0       ??0RSA_PublicKey@TaoCrypt@@QAE@AAVSource@1@@Z 0048ddb0 f   taocrypt:rsa.obj
 0001:0008cde0       ?CalculateInverse@RSA_PrivateKey@TaoCrypt@@QBE?AVInteger@2@AAVRandomNumberGenerator@2@ABV32@@Z 0048dde0 f   taocrypt:rsa.obj
 0001:0008cf60       ??0RSA_PrivateKey@TaoCrypt@@QAE@AAVSource@1@@Z 0048df60 f   taocrypt:rsa.obj
 0001:0008cfc0       ?UnPad@RSA_BlockType2@TaoCrypt@@QBEIPBEIPAE@Z 0048dfc0 f   taocrypt:rsa.obj
 0001:0008d040       ?UnPad@RSA_BlockType1@TaoCrypt@@QBEIPBEIPAE@Z 0048e040 f   taocrypt:rsa.obj
 0001:0008d0c0       ?SSL_Decrypt@TaoCrypt@@YAIABVRSA_PublicKey@1@PBEPAE@Z 0048e0c0 f   taocrypt:rsa.obj
 0001:0008d1b0       ??0PKCS12_Decoder@TaoCrypt@@QAE@AAVSource@1@@Z 0048e1b0 f i taocrypt:asn.obj
 0001:0008d1d0       ??1PKCS12_Decoder@TaoCrypt@@UAE@XZ 0048e1d0 f i taocrypt:asn.obj
 0001:0008d1e0       ?GetPublicKey@Signer@TaoCrypt@@QBEABVPublicKey@2@XZ 0048e1e0 f i taocrypt:asn.obj
 0001:0008d1f0       ?GetHash@Signer@TaoCrypt@@QBEPBEXZ 0048e1f0 f i taocrypt:asn.obj
 0001:0008d200       ??0DER_Encoder@TaoCrypt@@QAE@XZ 0048e200 f i taocrypt:asn.obj
 0001:0008d210       ??1DER_Encoder@TaoCrypt@@UAE@XZ 0048e210 f i taocrypt:asn.obj
 0001:0008d220       ??_GDER_Encoder@TaoCrypt@@UAEPAXI@Z 0048e220 f i taocrypt:asn.obj
 0001:0008d220       ??_EDER_Encoder@TaoCrypt@@UAEPAXI@Z 0048e220 f i taocrypt:asn.obj
 0001:0008d240       ?get_index@Source@TaoCrypt@@QBEIXZ 0048e240 f i taocrypt:asn.obj
 0001:0008d250       ?set_index@Source@TaoCrypt@@QAEXI@Z 0048e250 f i taocrypt:asn.obj
 0001:0008d260       ?advance@Source@TaoCrypt@@QAEXI@Z 0048e260 f i taocrypt:asn.obj
 0001:0008d270       ?GetError@Source@TaoCrypt@@QAE?AUError@2@XZ 0048e270 f i taocrypt:asn.obj
 0001:0008d280       ?SetModulus@RSA_PublicKey@TaoCrypt@@QAEXABVInteger@2@@Z 0048e280 f i taocrypt:asn.obj
 0001:0008d290       ?SetPublicExponent@RSA_PublicKey@TaoCrypt@@QAEXABVInteger@2@@Z 0048e290 f i taocrypt:asn.obj
 0001:0008d2a0       ?SetPrime1@RSA_PrivateKey@TaoCrypt@@QAEXABVInteger@2@@Z 0048e2a0 f i taocrypt:asn.obj
 0001:0008d2b0       ?SetPrime2@RSA_PrivateKey@TaoCrypt@@QAEXABVInteger@2@@Z 0048e2b0 f i taocrypt:asn.obj
 0001:0008d2c0       ?SetPrivateExponent@RSA_PrivateKey@TaoCrypt@@QAEXABVInteger@2@@Z 0048e2c0 f i taocrypt:asn.obj
 0001:0008d2d0       ?SetModPrime1PrivateExponent@RSA_PrivateKey@TaoCrypt@@QAEXABVInteger@2@@Z 0048e2d0 f i taocrypt:asn.obj
 0001:0008d2e0       ?SetModPrime2PrivateExponent@RSA_PrivateKey@TaoCrypt@@QAEXABVInteger@2@@Z 0048e2e0 f i taocrypt:asn.obj
 0001:0008d2f0       ?SetMultiplicativeInverseOfPrime2ModPrime1@RSA_PrivateKey@TaoCrypt@@QAEXABVInteger@2@@Z 0048e2f0 f i taocrypt:asn.obj
 0001:0008d320       ??O?A0x11a9e2d3@TaoCrypt@@YA_NAAUtm@@0@Z 0048e320 f   taocrypt:asn.obj
 0001:0008d3a0       ??M?A0x11a9e2d3@TaoCrypt@@YA_NAAUtm@@0@Z 0048e3a0 f   taocrypt:asn.obj
 0001:0008d3c0       ?btoi@?A0x11a9e2d3@TaoCrypt@@YAIE@Z 0048e3c0 f   taocrypt:asn.obj
 0001:0008d3d0       ?GetTime@?A0x11a9e2d3@TaoCrypt@@YAXAAHPBE0@Z 0048e3d0 f   taocrypt:asn.obj
 0001:0008d410       ?ValidateDate@?A0x11a9e2d3@TaoCrypt@@YA_NPBEEW4DateType@CertDecoder@2@@Z 0048e410 f   taocrypt:asn.obj
 0001:0008d560       ?SetLength@TaoCrypt@@YAIIPAE@Z 0048e560 f   taocrypt:asn.obj
 0001:0008d5d0       ?SetSize@PublicKey@TaoCrypt@@QAEXI@Z 0048e5d0 f   taocrypt:asn.obj
 0001:0008d5f0       ?SetKey@PublicKey@TaoCrypt@@QAEXPBE@Z 0048e5f0 f   taocrypt:asn.obj
 0001:0008d610       ?GetError@BER_Decoder@TaoCrypt@@QAE?AUError@2@XZ 0048e610 f   taocrypt:asn.obj
 0001:0008d620       ?GetInteger@BER_Decoder@TaoCrypt@@QAEAAVInteger@2@AAV32@@Z 0048e620 f   taocrypt:asn.obj
 0001:0008d650       ??1Signature_Encoder@TaoCrypt@@UAE@XZ 0048e650 f i taocrypt:asn.obj
 0001:0008d660       ?SetDigest@Signature_Encoder@TaoCrypt@@AAEIPBEIPAE@Z 0048e660 f   taocrypt:asn.obj
 0001:0008d690       ?SetSequence@TaoCrypt@@YAIIPAE@Z 0048e690 f   taocrypt:asn.obj
 0001:0008d6b0       ?EncodeDSA_Signature@TaoCrypt@@YAIABVInteger@1@0PAE@Z 0048e6b0 f   taocrypt:asn.obj
 0001:0008d7c0       ??A?$Block@EV?$AllocatorWithCleanup@E@TaoCrypt@@@TaoCrypt@@QBEABEI@Z 0048e7c0 f i taocrypt:asn.obj
 0001:0008d7d0       ??0?$auto_ptr@VHASH@TaoCrypt@@@mySTL@@QAE@PAVHASH@TaoCrypt@@@Z 0048e7d0 f i taocrypt:asn.obj
 0001:0008d7e0       ??C?$auto_ptr@VHASH@TaoCrypt@@@mySTL@@QBEPAVHASH@TaoCrypt@@XZ 0048e7e0 f i taocrypt:asn.obj
 0001:0008d7f0       ??$tcDelete@VHASH@TaoCrypt@@@TaoCrypt@@YAXPAVHASH@0@@Z 0048e7f0 f i taocrypt:asn.obj
 0001:0008d810       ??_GPKCS12_Decoder@TaoCrypt@@UAEPAXI@Z 0048e810 f i taocrypt:asn.obj
 0001:0008d810       ??_EPKCS12_Decoder@TaoCrypt@@UAEPAXI@Z 0048e810 f i taocrypt:asn.obj
 0001:0008d830       ??1PublicKey@TaoCrypt@@QAE@XZ 0048e830 f i taocrypt:asn.obj
 0001:0008d840       ?get_current@Source@TaoCrypt@@QBEPBEXZ 0048e840 f i taocrypt:asn.obj
 0001:0008d850       ?add@Source@TaoCrypt@@QAEXPBEI@Z 0048e850 f i taocrypt:asn.obj
 0001:0008d880       ?GetLength@TaoCrypt@@YAIAAVSource@1@@Z 0048e880 f   taocrypt:asn.obj
 0001:0008d8d0       ??0PublicKey@TaoCrypt@@QAE@PBEI@Z 0048e8d0 f   taocrypt:asn.obj
 0001:0008d900       ??0Signer@TaoCrypt@@QAE@PBEIPBD0@Z 0048e900 f   taocrypt:asn.obj
 0001:0008d980       ??1Signer@TaoCrypt@@QAE@XZ 0048e980 f   taocrypt:asn.obj
 0001:0008d990       ?GetSequence@BER_Decoder@TaoCrypt@@QAEIXZ 0048e990 f   taocrypt:asn.obj
 0001:0008d9d0       ?GetSet@BER_Decoder@TaoCrypt@@QAEIXZ 0048e9d0 f   taocrypt:asn.obj
 0001:0008da10       ?GetVersion@BER_Decoder@TaoCrypt@@QAEIXZ 0048ea10 f   taocrypt:asn.obj
 0001:0008da80       ?GetExplicitVersion@BER_Decoder@TaoCrypt@@QAEIXZ 0048ea80 f   taocrypt:asn.obj
 0001:0008dac0       ?Decode@RSA_Private_Decoder@TaoCrypt@@QAEXAAVRSA_PrivateKey@2@@Z 0048eac0 f   taocrypt:asn.obj
 0001:0008dc50       ?ReadHeader@RSA_Private_Decoder@TaoCrypt@@EAEXXZ 0048ec50 f   taocrypt:asn.obj
 0001:0008dc60       ?Decode@DSA_Private_Decoder@TaoCrypt@@QAEXAAVDSA_PrivateKey@2@@Z 0048ec60 f   taocrypt:asn.obj
 0001:0008dd70       ?ReadHeader@DSA_Private_Decoder@TaoCrypt@@EAEXXZ 0048ed70 f   taocrypt:asn.obj
 0001:0008dd80       ?Decode@RSA_Public_Decoder@TaoCrypt@@QAEXAAVRSA_PublicKey@2@@Z 0048ed80 f   taocrypt:asn.obj
 0001:0008de00       ?ReadHeader@RSA_Public_Decoder@TaoCrypt@@EAEXXZ 0048ee00 f   taocrypt:asn.obj
 0001:0008de10       ?Decode@DSA_Public_Decoder@TaoCrypt@@QAEXAAVDSA_PublicKey@2@@Z 0048ee10 f   taocrypt:asn.obj
 0001:0008def0       ?ReadHeader@DSA_Public_Decoder@TaoCrypt@@EAEXXZ 0048eef0 f   taocrypt:asn.obj
 0001:0008df00       ?ReadHeader@DH_Decoder@TaoCrypt@@EAEXXZ 0048ef00 f   taocrypt:asn.obj
 0001:0008df10       ?Decode@DH_Decoder@TaoCrypt@@QAEXAAVDH@2@@Z 0048ef10 f   taocrypt:asn.obj
 0001:0008df90       ??1CertDecoder@TaoCrypt@@UAE@XZ 0048ef90 f   taocrypt:asn.obj
 0001:0008dfc0       ?ReadHeader@CertDecoder@TaoCrypt@@EAEXXZ 0048efc0 f   taocrypt:asn.obj
 0001:0008e030       ?StoreKey@CertDecoder@TaoCrypt@@AAEXXZ 0048f030 f   taocrypt:asn.obj
 0001:0008e0a0       ?GetAlgoId@CertDecoder@TaoCrypt@@AAEIXZ 0048f0a0 f   taocrypt:asn.obj
 0001:0008e170       ?GetSignature@CertDecoder@TaoCrypt@@AAEIXZ 0048f170 f   taocrypt:asn.obj
 0001:0008e210       ?GetDigest@CertDecoder@TaoCrypt@@AAEIXZ 0048f210 f   taocrypt:asn.obj
 0001:0008e280       ?AddTag@CertDecoder@TaoCrypt@@AAEPADPADPBD1II@Z 0048f280 f   taocrypt:asn.obj
 0001:0008e2d0       ?GetName@CertDecoder@TaoCrypt@@AAEXW4NameType@12@@Z 0048f2d0 f   taocrypt:asn.obj
 0001:0008e520       ?GetDate@CertDecoder@TaoCrypt@@AAEXW4DateType@12@@Z 0048f520 f   taocrypt:asn.obj
 0001:0008e670       ?GetValidity@CertDecoder@TaoCrypt@@AAEXXZ 0048f670 f   taocrypt:asn.obj
 0001:0008e6a0       ?SetAlgoID@DER_Encoder@TaoCrypt@@QAEIW4HashType@2@PAE@Z 0048f6a0 f   taocrypt:asn.obj
 0001:0008e780       ?EncodeDSA_Signature@TaoCrypt@@YAIPBEPAE@Z 0048f780 f   taocrypt:asn.obj
 0001:0008e7f0       ?Decode@PKCS12_Decoder@TaoCrypt@@QAEXXZ 0048f7f0 f   taocrypt:asn.obj
 0001:0008e850       ?ReadHeader@PKCS12_Decoder@TaoCrypt@@EAEXXZ 0048f850 f   taocrypt:asn.obj
 0001:0008e860       ?GetPKCS_Cert@TaoCrypt@@YAHPBDAAVSource@1@@Z 0048f860 f   taocrypt:asn.obj
 0001:0008e880       ?Swap@?$Block@EV?$AllocatorWithCleanup@E@TaoCrypt@@@TaoCrypt@@QAEXAAV12@@Z 0048f880 f i taocrypt:asn.obj
 0001:0008e8a0       ?Destroy@?$auto_ptr@VHASH@TaoCrypt@@@mySTL@@AAEXXZ 0048f8a0 f i taocrypt:asn.obj
 0001:0008e8b0       ?Swap@Source@TaoCrypt@@QAEXAAV12@@Z 0048f8b0 f i taocrypt:asn.obj
 0001:0008e8e0       ??_ECertDecoder@TaoCrypt@@UAEPAXI@Z 0048f8e0 f i taocrypt:asn.obj
 0001:0008e8e0       ??_GCertDecoder@TaoCrypt@@UAEPAXI@Z 0048f8e0 f i taocrypt:asn.obj
 0001:0008e900       ??1?$auto_ptr@VHASH@TaoCrypt@@@mySTL@@QAE@XZ 0048f900 f i taocrypt:asn.obj
 0001:0008e910       ?reset@?$auto_ptr@VHASH@TaoCrypt@@@mySTL@@QAEXPAVHASH@TaoCrypt@@@Z 0048f910 f i taocrypt:asn.obj
 0001:0008e930       ?AddToEnd@PublicKey@TaoCrypt@@QAEXPBEI@Z 0048f930 f   taocrypt:asn.obj
 0001:0008e990       ?AddDSA@CertDecoder@TaoCrypt@@AAEXXZ 0048f990 f   taocrypt:asn.obj
 0001:0008ea50       ?DecodeDSA_Signature@TaoCrypt@@YAIPAEPBEI@Z 0048fa50 f   taocrypt:asn.obj
 0001:0008ec00       ?GetCert@TaoCrypt@@YAHAAVSource@1@@Z 0048fc00 f   taocrypt:asn.obj
 0001:0008ecf0       ?CleanGrow@?$Block@EV?$AllocatorWithCleanup@E@TaoCrypt@@@TaoCrypt@@QAEXI@Z 0048fcf0 f i taocrypt:asn.obj
 0001:0008ed30       ?grow@Source@TaoCrypt@@QAEXI@Z 0048fd30 f i taocrypt:asn.obj
 0001:0008ed70       ?GetKey@CertDecoder@TaoCrypt@@AAEXXZ 0048fd70 f   taocrypt:asn.obj
 0001:0008ee20       ??0Signature_Encoder@TaoCrypt@@QAE@PBEIW4HashType@1@AAVSource@1@@Z 0048fe20 f   taocrypt:asn.obj
 0001:0008ef30       ??_GSignature_Encoder@TaoCrypt@@UAEPAXI@Z 0048ff30 f i taocrypt:asn.obj
 0001:0008ef30       ??_ESignature_Encoder@TaoCrypt@@UAEPAXI@Z 0048ff30 f i taocrypt:asn.obj
 0001:0008ef50       ??0Source@TaoCrypt@@QAE@I@Z 0048ff50 f i taocrypt:asn.obj
 0001:0008efb0       ?DecodeToKey@CertDecoder@TaoCrypt@@QAEXXZ 0048ffb0 f   taocrypt:asn.obj
 0001:0008eff0       ?ConfirmSignature@CertDecoder@TaoCrypt@@AAE_NAAVSource@2@@Z 0048fff0 f   taocrypt:asn.obj
 0001:0008f2e0       ?ValidateSelfSignature@CertDecoder@TaoCrypt@@AAE_NXZ 004902e0 f   taocrypt:asn.obj
 0001:0008f360       ?ValidateSignature@CertDecoder@TaoCrypt@@AAE_NPAV?$list@PAVSigner@TaoCrypt@@@mySTL@@@Z 00490360 f   taocrypt:asn.obj
 0001:0008f4a0       ?Decode@CertDecoder@TaoCrypt@@AAEXPAV?$list@PAVSigner@TaoCrypt@@@mySTL@@W4CertType@12@@Z 004904a0 f   taocrypt:asn.obj
 0001:0008f520       ??0CertDecoder@TaoCrypt@@QAE@AAVSource@1@_NPAV?$list@PAVSigner@TaoCrypt@@@mySTL@@1W4CertType@01@@Z 00490520 f   taocrypt:asn.obj
 0001:0008f580       ?GetCompareHash@CertDecoder@TaoCrypt@@AAEXPBEIPAEI@Z 00490580 f   taocrypt:asn.obj
 0001:0008f690       ??1FileSource@TaoCrypt@@QAE@XZ 00490690 f   taocrypt:file.obj
 0001:0008f6a0       ?size@FileSource@TaoCrypt@@QAEI_N@Z 004906a0 f   taocrypt:file.obj
 0001:0008f710       ?size_left@FileSource@TaoCrypt@@AAEIXZ 00490710 f   taocrypt:file.obj
 0001:0008f720       ??1FileSink@TaoCrypt@@QAE@XZ 00490720 f   taocrypt:file.obj
 0001:0008f730       ?put@FileSink@TaoCrypt@@AAEXAAVSource@2@@Z 00490730 f   taocrypt:file.obj
 0001:0008f750       ??0FileSink@TaoCrypt@@QAE@PBDAAVSource@1@@Z 00490750 f   taocrypt:file.obj
 0001:0008f780       ?reset@Source@TaoCrypt@@QAEXAAV?$Block@EV?$AllocatorWithCleanup@E@TaoCrypt@@@2@@Z 00490780 f   taocrypt:file.obj
 0001:0008f7b0       ?get@FileSource@TaoCrypt@@AAEIAAVSource@2@@Z 004907b0 f   taocrypt:file.obj
 0001:0008f820       ??0FileSource@TaoCrypt@@QAE@PBDAAVSource@1@@Z 00490820 f   taocrypt:file.obj
 0001:0008f850       ?Double@AbstractGroup@TaoCrypt@@UBEABVInteger@2@ABV32@@Z 00490850 f   taocrypt:algebra.obj
 0001:0008f860       ?Accumulate@AbstractGroup@TaoCrypt@@UBEAAVInteger@2@AAV32@ABV32@@Z 00490860 f   taocrypt:algebra.obj
 0001:0008f880       ?Reduce@AbstractGroup@TaoCrypt@@UBEAAVInteger@2@AAV32@ABV32@@Z 00490880 f   taocrypt:algebra.obj
 0001:0008f8a0       ?Square@AbstractRing@TaoCrypt@@UBEABVInteger@2@ABV32@@Z 004908a0 f   taocrypt:algebra.obj
 0001:0008f8b0       ?FindNextWindow@WindowSlider@TaoCrypt@@QAEXXZ 004908b0 f i taocrypt:algebra.obj
 0001:0008f960       ?size@?$vector@VInteger@TaoCrypt@@@mySTL@@QBEIXZ 00490960 f i taocrypt:algebra.obj
 0001:0008f970       ??A?$vector@VInteger@TaoCrypt@@@mySTL@@QAEAAVInteger@TaoCrypt@@I@Z 00490970 f i taocrypt:algebra.obj
 0001:0008f980       ??A?$vector@V?$vector@VInteger@TaoCrypt@@@mySTL@@@mySTL@@QAEAAV?$vector@VInteger@TaoCrypt@@@1@I@Z 00490980 f i taocrypt:algebra.obj
 0001:0008f990       ??A?$vector@UWindowSlider@TaoCrypt@@@mySTL@@QAEAAUWindowSlider@TaoCrypt@@I@Z 00490990 f i taocrypt:algebra.obj
 0001:0008f9a0       ?capacity@?$vector@UWindowSlider@TaoCrypt@@@mySTL@@QBEIXZ 004909a0 f i taocrypt:algebra.obj
 0001:0008f9c0       ?size@?$vector@UWindowSlider@TaoCrypt@@@mySTL@@QBEIXZ 004909c0 f i taocrypt:algebra.obj
 0001:0008f9e0       ??0?$vector_base@UWindowSlider@TaoCrypt@@@mySTL@@QAE@XZ 004909e0 f i taocrypt:algebra.obj
 0001:0008f9f0       ??0?$vector_base@VInteger@TaoCrypt@@@mySTL@@QAE@XZ 004909f0 f i taocrypt:algebra.obj
 0001:0008fa00       ??$GetArrayMemory@VInteger@TaoCrypt@@@mySTL@@YAPAVInteger@TaoCrypt@@I@Z 00490a00 f i taocrypt:algebra.obj
 0001:0008fa10       ??$FreeArrayMemory@VInteger@TaoCrypt@@@mySTL@@YAXPAVInteger@TaoCrypt@@@Z 00490a10 f i taocrypt:algebra.obj
 0001:0008fa20       ??$GetArrayMemory@V?$vector@VInteger@TaoCrypt@@@mySTL@@@mySTL@@YAPAV?$vector@VInteger@TaoCrypt@@@0@I@Z 00490a20 f i taocrypt:algebra.obj
 0001:0008fa40       ??$FreeArrayMemory@V?$vector@VInteger@TaoCrypt@@@mySTL@@@mySTL@@YAXPAV?$vector@VInteger@TaoCrypt@@@0@@Z 00490a40 f i taocrypt:algebra.obj
 0001:0008fa50       ??$FreeArrayMemory@UWindowSlider@TaoCrypt@@@mySTL@@YAXPAUWindowSlider@TaoCrypt@@@Z 00490a50 f i taocrypt:algebra.obj
 0001:0008fa60       ??$swap@PAVInteger@TaoCrypt@@@mySTL@@YAXAAPAVInteger@TaoCrypt@@0@Z 00490a60 f i taocrypt:algebra.obj
 0001:0008fa80       ??$GetArrayMemory@UWindowSlider@TaoCrypt@@@mySTL@@YAPAUWindowSlider@TaoCrypt@@I@Z 00490a80 f i taocrypt:algebra.obj
 0001:0008faa0       ??$swap@PAUWindowSlider@TaoCrypt@@@mySTL@@YAXAAPAUWindowSlider@TaoCrypt@@0@Z 00490aa0 f i taocrypt:algebra.obj
 0001:0008fac0       ??$construct@VInteger@TaoCrypt@@V12@@mySTL@@YAXPAVInteger@TaoCrypt@@ABV12@@Z 00490ac0 f i taocrypt:algebra.obj
 0001:0008fae0       ?Subtract@AbstractGroup@TaoCrypt@@UBEABVInteger@2@ABV32@0@Z 00490ae0 f   taocrypt:algebra.obj
 0001:0008fb30       ?Divide@AbstractRing@TaoCrypt@@UBEABVInteger@2@ABV32@0@Z 00490b30 f   taocrypt:algebra.obj
 0001:0008fb80       ?Mod@AbstractEuclideanDomain@TaoCrypt@@UBEABVInteger@2@ABV32@0@Z 00490b80 f   taocrypt:algebra.obj
 0001:0008fbd0       ?ScalarMultiply@AbstractGroup@TaoCrypt@@UBE?AVInteger@2@ABV32@0@Z 00490bd0 f   taocrypt:algebra.obj
 0001:0008fc00       ??0WindowSlider@TaoCrypt@@QAE@ABVInteger@1@_NI@Z 00490c00 f i taocrypt:algebra.obj
 0001:0008fcb0       ??1WindowSlider@TaoCrypt@@QAE@XZ 00490cb0 f i taocrypt:algebra.obj
 0001:0008fce0       ?Exponentiate@AbstractRing@TaoCrypt@@UBE?AVInteger@2@ABV32@0@Z 00490ce0 f   taocrypt:algebra.obj
 0001:0008fd10       ??0?$vector_base@VInteger@TaoCrypt@@@mySTL@@QAE@I@Z 00490d10 f i taocrypt:algebra.obj
 0001:0008fd40       ??1?$vector_base@VInteger@TaoCrypt@@@mySTL@@QAE@XZ 00490d40 f i taocrypt:algebra.obj
 0001:0008fd50       ??0?$vector_base@V?$vector@VInteger@TaoCrypt@@@mySTL@@@mySTL@@QAE@I@Z 00490d50 f i taocrypt:algebra.obj
 0001:0008fd80       ??1?$vector_base@V?$vector@VInteger@TaoCrypt@@@mySTL@@@mySTL@@QAE@XZ 00490d80 f i taocrypt:algebra.obj
 0001:0008fd90       ??1?$vector_base@UWindowSlider@TaoCrypt@@@mySTL@@QAE@XZ 00490d90 f i taocrypt:algebra.obj
 0001:0008fda0       ?Swap@?$vector_base@VInteger@TaoCrypt@@@mySTL@@QAEXAAU12@@Z 00490da0 f i taocrypt:algebra.obj
 0001:0008fdd0       ??0?$vector_base@UWindowSlider@TaoCrypt@@@mySTL@@QAE@I@Z 00490dd0 f i taocrypt:algebra.obj
 0001:0008fe00       ?Swap@?$vector_base@UWindowSlider@TaoCrypt@@@mySTL@@QAEXAAU12@@Z 00490e00 f i taocrypt:algebra.obj
 0001:0008fe30       ??$uninit_fill_n@PAVInteger@TaoCrypt@@IV12@@mySTL@@YAPAVInteger@TaoCrypt@@PAV12@IABV12@@Z 00490e30 f i taocrypt:algebra.obj
 0001:0008fe70       ??$uninit_copy@PAVInteger@TaoCrypt@@PAV12@@mySTL@@YAPAVInteger@TaoCrypt@@PAV12@00@Z 00490e70 f i taocrypt:algebra.obj
 0001:0008feb0       ??0WindowSlider@TaoCrypt@@QAE@ABU01@@Z 00490eb0 f i taocrypt:algebra.obj
 0001:0008ff00       ??_GWindowSlider@TaoCrypt@@QAEPAXI@Z 00490f00 f i taocrypt:algebra.obj
 0001:0008ff40       ??0?$vector@VInteger@TaoCrypt@@@mySTL@@QAE@ABV01@@Z 00490f40 f i taocrypt:algebra.obj
 0001:0008ff80       ??0?$vector@VInteger@TaoCrypt@@@mySTL@@QAE@I@Z 00490f80 f i taocrypt:algebra.obj
 0001:0008ffe0       ??0?$vector@UWindowSlider@TaoCrypt@@@mySTL@@QAE@XZ 00490fe0 f i taocrypt:algebra.obj
 0001:0008fff0       ??0?$vector@VInteger@TaoCrypt@@@mySTL@@QAE@XZ 00490ff0 f i taocrypt:algebra.obj
 0001:00090000       ?Swap@?$vector@VInteger@TaoCrypt@@@mySTL@@QAEXAAV12@@Z 00491000 f i taocrypt:algebra.obj
 0001:00090030       ??0?$vector@VInteger@TaoCrypt@@@mySTL@@AAE@IABV01@@Z 00491030 f i taocrypt:algebra.obj
 0001:000900a0       ?Swap@?$vector@UWindowSlider@TaoCrypt@@@mySTL@@QAEXAAV12@@Z 004910a0 f i taocrypt:algebra.obj
 0001:000900d0       ??$construct@UWindowSlider@TaoCrypt@@U12@@mySTL@@YAXPAUWindowSlider@TaoCrypt@@ABU12@@Z 004910d0 f i taocrypt:algebra.obj
 0001:000900f0       ??$uninit_copy@PAUWindowSlider@TaoCrypt@@PAU12@@mySTL@@YAPAUWindowSlider@TaoCrypt@@PAU12@00@Z 004910f0 f i taocrypt:algebra.obj
 0001:00090160       ??$destroy@VInteger@TaoCrypt@@@mySTL@@YAXPAVInteger@TaoCrypt@@@Z 00491160 f i taocrypt:algebra.obj
 0001:00090180       ??$construct@V?$vector@VInteger@TaoCrypt@@@mySTL@@V12@@mySTL@@YAXPAV?$vector@VInteger@TaoCrypt@@@0@ABV10@@Z 00491180 f i taocrypt:algebra.obj
 0001:000901d0       ??$destroy@UWindowSlider@TaoCrypt@@@mySTL@@YAXPAUWindowSlider@TaoCrypt@@@Z 004911d0 f i taocrypt:algebra.obj
 0001:00090200       ??0?$vector@UWindowSlider@TaoCrypt@@@mySTL@@AAE@IABV01@@Z 00491200 f i taocrypt:algebra.obj
 0001:00090280       ??$destroy@PAVInteger@TaoCrypt@@@mySTL@@YAXPAVInteger@TaoCrypt@@0@Z 00491280 f i taocrypt:algebra.obj
 0001:000902b0       ??$uninit_fill_n@PAV?$vector@VInteger@TaoCrypt@@@mySTL@@IV12@@mySTL@@YAPAV?$vector@VInteger@TaoCrypt@@@0@PAV10@IABV10@@Z 004912b0 f i taocrypt:algebra.obj
 0001:00090310       ??$destroy@PAUWindowSlider@TaoCrypt@@@mySTL@@YAXPAUWindowSlider@TaoCrypt@@0@Z 00491310 f i taocrypt:algebra.obj
 0001:00090350       ??1?$vector@VInteger@TaoCrypt@@@mySTL@@QAE@XZ 00491350 f i taocrypt:algebra.obj
 0001:00090370       ?resize@?$vector@VInteger@TaoCrypt@@@mySTL@@QAEXIABVInteger@TaoCrypt@@@Z 00491370 f i taocrypt:algebra.obj
 0001:00090410       ??0?$vector@V?$vector@VInteger@TaoCrypt@@@mySTL@@@mySTL@@QAE@I@Z 00491410 f i taocrypt:algebra.obj
 0001:00090480       ??1?$vector@UWindowSlider@TaoCrypt@@@mySTL@@QAE@XZ 00491480 f i taocrypt:algebra.obj
 0001:000904a0       ?push_back@?$vector@UWindowSlider@TaoCrypt@@@mySTL@@QAEXABUWindowSlider@TaoCrypt@@@Z 004914a0 f i taocrypt:algebra.obj
 0001:00090530       ?reserve@?$vector@UWindowSlider@TaoCrypt@@@mySTL@@QAEXI@Z 00491530 f i taocrypt:algebra.obj
 0001:000905a0       ??_G?$vector@VInteger@TaoCrypt@@@mySTL@@QAEPAXI@Z 004915a0 f i taocrypt:algebra.obj
 0001:000905d0       ?Gcd@AbstractEuclideanDomain@TaoCrypt@@UBEABVInteger@2@ABV32@0@Z 004915d0 f   taocrypt:algebra.obj
 0001:00090700       ?CascadeScalarMultiply@AbstractGroup@TaoCrypt@@UBE?AVInteger@2@ABV32@000@Z 00491700 f   taocrypt:algebra.obj
 0001:00090b90       ?CascadeExponentiate@AbstractRing@TaoCrypt@@UBE?AVInteger@2@ABV32@000@Z 00491b90 f   taocrypt:algebra.obj
 0001:00090bc0       ??$destroy@V?$vector@VInteger@TaoCrypt@@@mySTL@@@mySTL@@YAXPAV?$vector@VInteger@TaoCrypt@@@0@@Z 00491bc0 f i taocrypt:algebra.obj
 0001:00090be0       ??$destroy@PAV?$vector@VInteger@TaoCrypt@@@mySTL@@@mySTL@@YAXPAV?$vector@VInteger@TaoCrypt@@@0@0@Z 00491be0 f i taocrypt:algebra.obj
 0001:00090c20       ??1?$vector@V?$vector@VInteger@TaoCrypt@@@mySTL@@@mySTL@@QAE@XZ 00491c20 f i taocrypt:algebra.obj
 0001:00090c40       ?SimultaneousMultiply@AbstractGroup@TaoCrypt@@UBEXPAVInteger@2@ABV32@PBV32@I@Z 00491c40 f   taocrypt:algebra.obj
 0001:00090f40       ?SimultaneousExponentiate@AbstractRing@TaoCrypt@@UBEXPAVInteger@2@ABV32@PBV32@I@Z 00491f40 f   taocrypt:algebra.obj
 0001:00090f70       ?Init@MD2@TaoCrypt@@UAEXXZ 00491f70 f   taocrypt:md2.obj
 0001:00090fb0       ?Update@MD2@TaoCrypt@@UAEXPBEI@Z 00491fb0 f   taocrypt:md2.obj
 0001:00091150       ?Final@MD2@TaoCrypt@@UAEXPAE@Z 00492150 f   taocrypt:md2.obj
 0001:000911e0       ??0MD2@TaoCrypt@@QAE@XZ    004921e0 f   taocrypt:md2.obj
 0001:000912a0       ?getBlockSize@MD2@TaoCrypt@@UBEIXZ 004922a0 f i taocrypt:md2.obj
 0001:000912b0       ?getDigestSize@MD2@TaoCrypt@@UBEIXZ 004922b0 f i taocrypt:md2.obj
 0001:000912c0       ??1MD2@TaoCrypt@@UAE@XZ    004922c0 f i taocrypt:md2.obj
 0001:00091310       ??_EMD2@TaoCrypt@@UAEPAXI@Z 00492310 f i taocrypt:md2.obj
 0001:00091310       ??_GMD2@TaoCrypt@@UAEPAXI@Z 00492310 f i taocrypt:md2.obj
 0001:0009132e       _inet_ntoa@4               0049232e f   wsock32:WSOCK32.dll
 0001:00091334       _remove                    00492334 f   LIBCMT:unlink.obj
 0001:0009135e       _unlink                    0049235e f   LIBCMT:unlink.obj
 0001:0009135e       __unlink                   0049235e f   LIBCMT:unlink.obj
 0001:00091363       _fdopen                    00492363 f   LIBCMT:fdopen.obj
 0001:00091363       __fdopen                   00492363 f   LIBCMT:fdopen.obj
 0001:000916f8       __putenv                   004926f8 f   LIBCMT:putenv.obj
 0001:000916f8       _putenv                    004926f8 f   LIBCMT:putenv.obj
 0001:0009173d       __putenv_s                 0049273d f   LIBCMT:putenv.obj
 0001:000917b6       __chdir                    004927b6 f   LIBCMT:chdir.obj
 0001:000917b6       _chdir                     004927b6 f   LIBCMT:chdir.obj
 0001:000918e0       __aullrem                  004928e0 f   LIBCMT:ullrem.obj
 0001:00091955       __aligned_offset_malloc    00492955 f   LIBCMT:align.obj
 0001:000919ee       __aligned_msize            004929ee f   LIBCMT:align.obj
 0001:00091a40       __aligned_free             00492a40 f   LIBCMT:align.obj
 0001:00091a55       __aligned_malloc           00492a55 f   LIBCMT:align.obj
 0001:00091a68       __aligned_offset_realloc   00492a68 f   LIBCMT:align.obj
 0001:00091bd6       __aligned_offset_recalloc  00492bd6 f   LIBCMT:align.obj
 0001:00091c5f       __aligned_realloc          00492c5f f   LIBCMT:align.obj
 0001:00091c76       __aligned_recalloc         00492c76 f   LIBCMT:align.obj
 0001:00091ca0       _pow                       00492ca0 f   LIBCMT:pow.obj
 0001:00091ce0       __CIpow                    00492ce0 f   LIBCMT:pow.obj
 0001:00091d1b       __CIpow_default            00492d1b f   LIBCMT:pow.obj
 0001:00091d34       __pow_default              00492d34     LIBCMT:pow.obj
 0001:00091f30       _log                       00492f30 f   LIBCMT:log.obj
 0001:00091f70       __CIlog                    00492f70 f   LIBCMT:log.obj
 0001:00091fab       __CIlog_default            00492fab f   LIBCMT:log.obj
 0001:00091fbf       __log_default              00492fbf     LIBCMT:log.obj
 0001:00092080       __invoke_watson_if_oneof   00493080 f i LIBCMT:wassert.obj
 0001:000920cd       __wassert                  004930cd f   LIBCMT:wassert.obj
 0001:000929c0       ___crtwsetenv              004939c0 f   LIBCMT:wsetenv.obj
 0001:00092d26       __mbctoupper_l             00493d26 f   LIBCMT:mbtoupr.obj
 0001:00092dca       __mbctoupper               00493dca f   LIBCMT:mbtoupr.obj
 0001:00092dd8       __expand                   00493dd8 f   LIBCMT:expand.obj
 0001:00092ee0       __CIpow_pentium4           00493ee0 f   LIBCMT:pow_pentium4.obj
 0001:00092ef9       __pow_pentium4             00493ef9     LIBCMT:pow_pentium4.obj
 0001:00093a51       __fFEXP                    00494a51     LIBCMT:87tran.obj
 0001:00093ab8       __rtinfpopse               00494ab8     LIBCMT:87tran.obj
 0001:00093aba       __rtinfnpopse              00494aba     LIBCMT:87tran.obj
 0001:00093aca       __fFLN                     00494aca     LIBCMT:87tran.obj
 0001:00093b7f       __rtinfpop                 00494b7f     LIBCMT:87tran.obj
 0001:00093b81       __rtinfnpop                00494b81     LIBCMT:87tran.obj
 0001:00093b9e       __ffexpm1                  00494b9e     LIBCMT:87tran.obj
 0001:00093c50       __trandisp1                00494c50 f   LIBCMT:87disp.obj
 0001:00093cb7       __trandisp2                00494cb7 f   LIBCMT:87disp.obj
 0001:00093d43       __rttospopde               00494d43     LIBCMT:87disp.obj
 0001:00093d48       __rttospop                 00494d48     LIBCMT:87disp.obj
 0001:00093d4a       __rtnospop                 00494d4a     LIBCMT:87disp.obj
 0001:00093d4c       __rttosnpop                00494d4c     LIBCMT:87disp.obj
 0001:00093d4d       __rtnospopde               00494d4d     LIBCMT:87disp.obj
 0001:00093d54       __rtzeropop                00494d54     LIBCMT:87disp.obj
 0001:00093d56       __rtzeronpop               00494d56     LIBCMT:87disp.obj
 0001:00093d5b       __rtonepop                 00494d5b     LIBCMT:87disp.obj
 0001:00093d5d       __rtonenpop                00494d5d     LIBCMT:87disp.obj
 0001:00093d62       __tosnan1                  00494d62     LIBCMT:87disp.obj
 0001:00093d8d       __nosnan2                  00494d8d     LIBCMT:87disp.obj
 0001:00093d8f       __tosnan2                  00494d8f     LIBCMT:87disp.obj
 0001:00093db7       __nan2                     00494db7     LIBCMT:87disp.obj
 0001:00093df6       __rtindfpop                00494df6     LIBCMT:87disp.obj
 0001:00093df8       __rtindfnpop               00494df8     LIBCMT:87disp.obj
 0001:00093e09       __rttosnpopde              00494e09     LIBCMT:87disp.obj
 0001:00093e13       __rtchsifneg               00494e13     LIBCMT:87disp.obj
 0001:00093e20       __startTwoArgErrorHandling 00494e20 f   LIBCMT:genexcep.obj
 0001:00093e37       __startOneArgErrorHandling 00494e37 f   LIBCMT:genexcep.obj
 0001:00093e80       __twoToTOS                 00494e80 f   LIBCMT:common.obj
 0001:00093e95       __load_CW                  00494e95 f   LIBCMT:common.obj
 0001:00093eac       __convertTOStoQNaN         00494eac f   LIBCMT:common.obj
 0001:00093ec5       __fload_withFB             00494ec5 f   LIBCMT:common.obj
 0001:00093f08       __checkTOS_withFB          00494f08 f   LIBCMT:common.obj
 0001:00093f1e       __fast_exit                00494f1e f   LIBCMT:common.obj
 0001:00093f2b       __math_exit                00494f2b f   LIBCMT:common.obj
 0001:00093f55       __check_overflow_exit      00494f55 f   LIBCMT:common.obj
 0001:00093f69       __check_range_exit         00494f69 f   LIBCMT:common.obj
 0001:0009400c       __d_inttype                0049500c f   LIBCMT:powhlp.obj
 0001:00094070       __powhlp                   00495070 f   LIBCMT:powhlp.obj
 0001:000941b0       __CIlog_pentium4           004951b0 f   LIBCMT:log_pentium4.obj
 0001:000941c8       __log_pentium4             004951c8     LIBCMT:log_pentium4.obj
 0001:00094420       __vswprintf_helper         00495420 f   LIBCMT:vswprnc.obj
 0001:00094516       __vswprintf_c              00495516 f   LIBCMT:vswprnc.obj
 0001:0009453d       __vswprintf_c_l            0049553d f   LIBCMT:vswprnc.obj
 0001:00094565       __vswprintf_s_l            00495565 f   LIBCMT:vswprnc.obj
 0001:000945ec       _vswprintf_s               004955ec f   LIBCMT:vswprnc.obj
 0001:00094607       __vsnwprintf_s_l           00495607 f   LIBCMT:vswprnc.obj
 0001:0009470e       __vsnwprintf_s             0049570e f   LIBCMT:vswprnc.obj
 0001:0009472c       __vswprintf_p              0049572c f   LIBCMT:vswprnc.obj
 0001:00094753       __vswprintf_p_l            00495753 f   LIBCMT:vswprnc.obj
 0001:0009477b       _fwprintf                  0049577b f   LIBCMT:fwprintf.obj
 0001:0009480f       __fwprintf_l               0049580f f   LIBCMT:fwprintf.obj
 0001:00094829       __fwprintf_s_l             00495829 f   LIBCMT:fwprintf.obj
 0001:00094843       _fwprintf_s                00495843 f   LIBCMT:fwprintf.obj
 0001:0009485b       __fwprintf_p_l             0049585b f   LIBCMT:fwprintf.obj
 0001:00094875       __fwprintf_p               00495875 f   LIBCMT:fwprintf.obj
 0001:0009488d       ___crtMessageBoxW          0049588d f   LIBCMT:crtmboxw.obj
 0001:00094b39       __itow_s                   00495b39 f   LIBCMT:xtows.obj
 0001:00094b63       __ltow_s                   00495b63 f   LIBCMT:xtows.obj
 0001:00094b88       __ultow_s                  00495b88 f   LIBCMT:xtows.obj
 0001:00094c9e       __i64tow_s                 00495c9e f   LIBCMT:xtows.obj
 0001:00094cd1       __ui64tow_s                00495cd1 f   LIBCMT:xtows.obj
 0001:00094cee       _wcsncat_s                 00495cee f   LIBCMT:wcsncat_s.obj
 0001:00094dcf       _wcsncpy_s                 00495dcf f   LIBCMT:wcsncpy_s.obj
 0001:00094e98       _wcscat_s                  00495e98 f   LIBCMT:wcscat_s.obj
 0001:00094f12       _wcscpy_s                  00495f12 f   LIBCMT:wcscpy_s.obj
 0001:00094f7e       __assert                   00495f7e f   LIBCMT:assert.obj
 0001:00095609       __wcstombs_l_helper        00496609 f   LIBCMT:wcstombs.obj
 0001:0009584f       __wcstombs_l               0049684f f   LIBCMT:wcstombs.obj
 0001:00095854       _wcstombs                  00496854 f   LIBCMT:wcstombs.obj
 0001:0009586b       __wcstombs_s_l             0049686b f   LIBCMT:wcstombs.obj
 0001:0009591c       _wcstombs_s                0049691c f   LIBCMT:wcstombs.obj
 0001:0009593a       __wcsnicoll_l              0049693a f   LIBCMT:wcsnicol.obj
 0001:00095a7b       __wcsnicoll                00496a7b f   LIBCMT:wcsnicol.obj
 0001:00095b1d       __wcsdup                   00496b1d f   LIBCMT:wcsdup.obj
 0001:00095b70       ___mbtow_environ           00496b70 f   LIBCMT:mbtowenv.obj
 0001:00095bf5       __wsetenvp                 00496bf5 f   LIBCMT:wstdenvp.obj
 0001:00095ccf       ___crtGetEnvironmentStringsW 00496ccf f   LIBCMT:w_env.obj
 0001:00095e30       _wcschr                    00496e30 f   LIBCMT:wcschr.obj
 0001:00095e60       _fdiv_main_routine         00496e60 f   LIBCMT:adj_fdiv.obj
 0001:00095f77       __adj_fdiv_r               00496f77 f   LIBCMT:adj_fdiv.obj
 0001:00096416       __fdivp_sti_st             00497416 f   LIBCMT:adj_fdiv.obj
 0001:00096429       __fdivrp_sti_st            00497429 f   LIBCMT:adj_fdiv.obj
 0001:0009643c       __adj_fdiv_m32             0049743c f   LIBCMT:adj_fdiv.obj
 0001:00096488       __adj_fdiv_m64             00497488 f   LIBCMT:adj_fdiv.obj
 0001:000964d4       __adj_fdiv_m16i            004974d4 f   LIBCMT:adj_fdiv.obj
 0001:00096508       __adj_fdiv_m32i            00497508 f   LIBCMT:adj_fdiv.obj
 0001:0009653c       __adj_fdivr_m32            0049753c f   LIBCMT:adj_fdiv.obj
 0001:00096588       __adj_fdivr_m64            00497588 f   LIBCMT:adj_fdiv.obj
 0001:000965d4       __adj_fdivr_m16i           004975d4 f   LIBCMT:adj_fdiv.obj
 0001:00096608       __adj_fdivr_m32i           00497608 f   LIBCMT:adj_fdiv.obj
 0001:0009663c       __safe_fdiv                0049763c f   LIBCMT:adj_fdiv.obj
 0001:00096651       __safe_fdivr               00497651 f   LIBCMT:adj_fdiv.obj
 0001:00096666       __fprem_common             00497666 f   LIBCMT:adj_fdiv.obj
 0001:0009686c       __adj_fprem                0049786c f   LIBCMT:adj_fdiv.obj
 0001:0009691e       __fprem1_common            0049791e f   LIBCMT:adj_fdiv.obj
 0001:00096b24       __adj_fprem1               00497b24 f   LIBCMT:adj_fdiv.obj
 0001:00096bd9       __safe_fprem               00497bd9 f   LIBCMT:adj_fdiv.obj
 0001:00096bdf       __safe_fprem1              00497bdf f   LIBCMT:adj_fdiv.obj
 0001:00096be5       __adj_fpatan               00497be5 f   LIBCMT:adj_fdiv.obj
 0001:00096be8       __adj_fptan                00497be8 f   LIBCMT:adj_fdiv.obj
 0001:00096beb       __87except                 00497beb f   LIBCMT:87except.obj
 0001:00096d80       __woutput_l                00497d80 f   LIBCMT:woutput.obj
 0001:00097729       __woutput_s_l              00498729 f   LIBCMT:woutputs.obj
 0001:00098045       __validate_param_reuseW    00499045 f   LIBCMT:woutputp.obj
 0001:00098232       __woutput_p_l              00499232 f   LIBCMT:woutputp.obj
 0001:00099192       _vfwprintf_helper          0049a192 f   LIBCMT:vfwprint.obj
 0001:00099225       __vfwprintf_l              0049a225 f   LIBCMT:vfwprint.obj
 0001:00099243       __vfwprintf_s_l            0049a243 f   LIBCMT:vfwprint.obj
 0001:00099261       __vfwprintf_p_l            0049a261 f   LIBCMT:vfwprint.obj
 0001:0009927f       _vfwprintf                 0049a27f f   LIBCMT:vfwprint.obj
 0001:0009929b       _vfwprintf_s               0049a29b f   LIBCMT:vfwprint.obj
 0001:000992b7       __vfwprintf_p              0049a2b7 f   LIBCMT:vfwprint.obj
 0001:000992d3       __mbsnbcat_s               0049a2d3 f   LIBCMT:mbsnbcat_s.obj
 0001:000992ee       __mbsnbcpy_s               0049a2ee f   LIBCMT:mbsnbcpy_s.obj
 0001:00099575       ___crtCompareStringW       0049a575 f   LIBCMT:w_cmp.obj
 0001:000995b5       __fputwc_nolock            0049a5b5 f   LIBCMT:fputwc.obj
 0001:00099793       _fputwc                    0049a793 f   LIBCMT:fputwc.obj
 0001:0009980b       _putwc                     0049a80b f   LIBCMT:fputwc.obj
 0001:00099a07       _wcstol                    0049aa07 f   LIBCMT:wcstol.obj
 0001:00099a30       __wcstol_l                 0049aa30 f   LIBCMT:wcstol.obj
 0001:00099a4b       _wcstoul                   0049aa4b f   LIBCMT:wcstol.obj
 0001:00099a75       __wcstoul_l                0049aa75 f   LIBCMT:wcstol.obj
 0001:00099a90       __mbsnbcat_s_l             0049aa90 f   LIBCMT:mbsnbcat_s_l.obj
 0001:00099d22       __mbsnbcpy_s_l             0049ad22 f   LIBCMT:mbsnbcpy_s_l.obj
 0001:00099f2f       __flswbuf                  0049af2f f   LIBCMT:_flswbuf.obj
 0001:0009a09f       __wchartodigit             0049b09f f   LIBCMT:wchtodig.obj
 0001:0009a221       _strncat_s                 0049b221 f   LIBCMT:strncat_s.obj
 0001:0009a2e4       _GetModuleFileNameW@12     0049b2e4 f   kernel32:KERNEL32.dll
 0001:0009a2ea       _SetEnvironmentVariableW@8 0049b2ea f   kernel32:KERNEL32.dll
 0001:0009a2f0       _LoadLibraryW@4            0049b2f0 f   kernel32:KERNEL32.dll
 0001:0009a2f6       _CryptAcquireContextA@20   0049b2f6 f   advapi32:ADVAPI32.dll
 0001:0009a2fc       _CryptReleaseContext@8     0049b2fc f   advapi32:ADVAPI32.dll
 0001:0009a302       _CryptGenRandom@12         0049b302 f   advapi32:ADVAPI32.dll
 0002:00000000       ___xc_a                    004c0000     LIBCMT:crt0init.obj
 0002:00000210       ___xc_z                    004c0210     LIBCMT:crt0init.obj
 0002:00000314       ___xi_a                    004c0314     LIBCMT:crt0init.obj
 0002:00000634       ___xi_z                    004c0634     LIBCMT:crt0init.obj
 0002:00000738       ___xl_a                    004c0738     LIBCMT:tlssup.obj
 0002:0000073c       ___xl_z                    004c073c     LIBCMT:tlssup.obj
 0002:00000740       ___xp_a                    004c0740     LIBCMT:crt0init.obj
 0002:00000a4c       ___xp_z                    004c0a4c     LIBCMT:crt0init.obj
 0002:00000b50       ___xt_a                    004c0b50     LIBCMT:crt0init.obj
 0002:00000c54       ___xt_z                    004c0c54     LIBCMT:crt0init.obj
 0002:00000d7c       ??_C@_0P@GHFPNOJB@bad?5allocation?$AA@ 004c0d7c     buffer.obj
 0002:00000d90       ?BUFFER_INITIAL_SIZE@Buffer@@0IB 004c0d90     buffer.obj
 0002:00000d94       ?MAX_BUFFER_SIZE@Buffer@@0IB 004c0d94     buffer.obj
 0002:00000da0       __real@3ff8000000000000    004c0da0     buffer.obj
 0002:00000db0       __real@41f0000000000000    004c0db0     buffer.obj
 0002:00000dc0       ??_7Command@@6B@           004c0dc0     command.obj
 0002:00000ddc       ??_C@_05HDBKIDE@state?$AA@ 004c0ddc     commands.obj
 0002:00000de4       ??_C@_0O@MIFOIHFB@instance_name?$AA@ 004c0de4     commands.obj
 0002:00000df8       ??_7Instance_cmd@@6B@      004c0df8     commands.obj
 0002:00000e08       ??_7Abstract_instance_cmd@@6B@ 004c0e08     commands.obj
 0002:00000e20       ??_7Show_instance_status@@6B@ 004c0e20     commands.obj
 0002:00000e34       ??_C@_0BC@OPJMMHIK@mysqld_compatible?$AA@ 004c0e34     commands.obj
 0002:00000e4c       ??_C@_0P@LNKEPANE@version_number?$AA@ 004c0e4c     commands.obj
 0002:00000e60       ??_C@_07CPCPJPKL@version?$AA@ 004c0e60     commands.obj
 0002:00000e6c       ??_C@_02KAJCLHKP@no?$AA@   004c0e6c     commands.obj
 0002:00000e70       ??_C@_03ICICOMAL@yes?$AA@  004c0e70     commands.obj
 0002:00000e74       ??_C@_07CIFAGBMG@unknown?$AA@ 004c0e74     commands.obj
 0002:00000e84       ??_7Show_instance_options@@6B@ 004c0e84     commands.obj
 0002:00000e98       ??_C@_05MFEJDJP@value?$AA@ 004c0e98     commands.obj
 0002:00000ea0       ??_C@_0M@PNCLCLFB@option_name?$AA@ 004c0ea0     commands.obj
 0002:00000eae       ??_C@_00CNPNBAHC@?$AA@     004c0eae     commands.obj
 0002:00000eb4       ??_7Start_instance@@6B@    004c0eb4     commands.obj
 0002:00000ec8       ??_C@_0BB@EIFMIEBH@Instance?5started?$AA@ 004c0ec8     commands.obj
 0002:00000ee0       ??_7Stop_instance@@6B@     004c0ee0     commands.obj
 0002:00000ef8       ??_7Create_instance@@6B@   004c0ef8     commands.obj
 0002:00000f08       ??_7Drop_instance@@6B@     004c0f08     commands.obj
 0002:00000f14       ??_C@_0BB@JCFKCMFI@Instance?5dropped?$AA@ 004c0f14     commands.obj
 0002:00000f28       ??_C@_0EP@PLHCCCFH@Can?5not?5remove?5instance?5?8?$CFs?8?5fro@ 004c0f28     commands.obj
 0002:00000f8c       ??_7Show_instance_log@@6B@ 004c0f8c     commands.obj
 0002:00000fa0       ??_C@_03GGEOLGBL@Log?$AA@  004c0fa0     commands.obj
 0002:00000fa8       ??_7Show_instance_log_files@@6B@ 004c0fa8     commands.obj
 0002:00000fbc       ??_C@_09JPMHFEOD@File?5size?$AA@ 004c0fbc     commands.obj
 0002:00000fc8       ??_C@_04HMIIHGGM@Path?$AA@ 004c0fc8     commands.obj
 0002:00000fd0       ??_C@_07IFPLGDBI@Logfile?$AA@ 004c0fd0     commands.obj
 0002:00000fdc       ??_C@_01GBGANLPD@0?$AA@    004c0fdc     commands.obj
 0002:00000fe0       ??_C@_08FLCOKHCB@SLOW?5LOG?$AA@ 004c0fe0     commands.obj
 0002:00000fec       ??_C@_0M@CKKADIMG@GENERAL?5LOG?$AA@ 004c0fec     commands.obj
 0002:00000ffc       ??_C@_09ILJLBPE@ERROR?5LOG?$AA@ 004c0ffc     commands.obj
 0002:0000100c       ??_7Abstract_option_cmd@@6B@ 004c100c     commands.obj
 0002:00001020       ??_C@_0EL@PIIKGIKP@Can?5not?5modify?5option?5?$CI?$CFs?$CJ?5in?5de@ 004c1020     commands.obj
 0002:00001080       ??_C@_0FI@JJBPOGGF@IM?9option?5?$CI?$CFs?$CJ?5can?5not?5be?5used?5i@ 004c1080     commands.obj
 0002:000010f0       ??_7Thread@@6B@            004c10f0     guardian.obj
 0002:00001100       ??_7Guardian@@6B@          004c1100     guardian.obj
 0002:00001110       ??_C@_0EC@CLDPELEC@Guardian?3?5can?5not?5start?5?8?$CFs?8?4?5Ab@ 004c1110     guardian.obj
 0002:00001160       ??_C@_0BN@IMGFCJPE@Guardian?3?5restarting?5?8?$CFs?8?4?4?4?$AA@ 004c1160     guardian.obj
 0002:00001184       ??_C@_0BL@EJNFPJD@Guardian?3?5starting?5?8?$CFs?8?4?4?4?$AA@ 004c1184     guardian.obj
 0002:000011a4       ??_C@_0DB@OHKMODAF@Guardian?3?5?8?$CFs?8?5is?5running?0?5set?5s@ 004c11a4     guardian.obj
 0002:000011e0       ??_C@_0DD@DICFGDLN@Guardian?3?5waiting?5for?5?8?$CFs?8?5to?5st@ 004c11e0     guardian.obj
 0002:00001220       ??_C@_0CH@GBMAPFMH@Guardian?3?5pretend?5that?5?8?$CFs?8?5is?5k@ 004c1220     guardian.obj
 0002:00001250       ??_C@_0CO@NHFJHJAE@Guardian?3?5?8?$CFs?8?5hasn?8t?5stopped?5wi@ 004c1250     guardian.obj
 0002:00001288       ??_C@_0BI@LPKFLOPI@Guardian?3?5?8?$CFs?8?5stopped?4?$AA@ 004c1288     guardian.obj
 0002:000012a4       ??_C@_0BE@FBJMCIE@Guardian?3?5finished?4?$AA@ 004c12a4     guardian.obj
 0002:000012bc       ??_C@_0BD@PIJKIOJO@Guardian?3?5stopped?4?$AA@ 004c12bc     guardian.obj
 0002:000012d4       ??_C@_0CH@FBNFGIEG@Guardian?3?5all?5guarded?5mysqlds?5st@ 004c12d4     guardian.obj
 0002:00001304       ??_C@_0BD@BAONPCAI@Guardian?3?5started?4?$AA@ 004c1304     guardian.obj
 0002:0000131c       ??_C@_06IJHCJAKM@mysqld?$AA@ 004c131c     instance.obj
 0002:00001324       ?DFLT_INSTANCE_NAME@Instance@@2Ust_mysql_lex_string@@B 004c1324     instance.obj
 0002:00001330       ??_C@_02KOPDJAMB@?$CC?5?$AA@ 004c1330     instance.obj
 0002:00001334       ??_C@_01BJJEKLCA@?$CC?$AA@ 004c1334     instance.obj
 0002:00001338       ??_C@_0M@LPAKIOHO@ExitProcess?$AA@ 004c1338     instance.obj
 0002:00001348       ??_C@_08HPEMMIEC@Kernel32?$AA@ 004c1348     instance.obj
 0002:00001358       ??_7Instance_monitor@@6B@  004c1358     instance.obj
 0002:00001364       ??_C@_08FJBHPJOK@stopping?$AA@ 004c1364     instance.obj
 0002:00001370       ??_C@_09ILHOEMPA@abandoned?$AA@ 004c1370     instance.obj
 0002:0000137c       ??_C@_07HDILHIKI@crashed?$AA@ 004c137c     instance.obj
 0002:00001388       ??_C@_06ODACHPEO@failed?$AA@ 004c1388     instance.obj
 0002:00001390       ??_C@_06GNLMCJKK@online?$AA@ 004c1390     instance.obj
 0002:00001398       ??_C@_08LBGAIFHM@starting?$AA@ 004c1398     instance.obj
 0002:000013a4       ??_C@_0M@CKKENOIB@not?5started?$AA@ 004c13a4     instance.obj
 0002:000013b4       ??_C@_07OFPCFMBE@offline?$AA@ 004c13b4     instance.obj
 0002:000013c0       ??_C@_0BN@LLJOCMEH@Instance?5?8?$CFs?8?3?5destroying?4?4?4?$AA@ 004c13c0     instance.obj
 0002:000013e4       ??_C@_0CM@DPCAKKPD@Instance?5?8?$CFs?8?3?5was?5able?5to?5log?5i@ 004c13e4     instance.obj
 0002:00001418       ??_C@_09IPAEKDAI@localhost?$AA@ 004c1418     instance.obj
 0002:00001424       ??_C@_0BB@GHJAIMGF@check_connection?$AA@ 004c1424     instance.obj
 0002:00001438       ??_C@_0BH@JBEJIMON@MySQL_Instance_Manager?$AA@ 004c1438     instance.obj
 0002:00001454       ??_C@_0BH@KOCPJDOG@Access?5denied?5for?5user?$AA@ 004c1454     instance.obj
 0002:00001470       ??_C@_0BH@BODLLCCJ@Instance?5?8?$CFs?8?3?5killed?4?$AA@ 004c1470     instance.obj
 0002:0000148c       ??_C@_0BO@NFBHCDDC@Instance?5?8?$CFs?8?3?5kill?$CI?$CJ?5failed?4?$AA@ 004c148c     instance.obj
 0002:000014b0       ??_C@_0CD@JCNDMOGD@Instance?5?8?$CFs?8?3?5sending?5?$CFd?5to?5?$CFd?4@ 004c14b0     instance.obj
 0002:000014dc       ??_C@_0DC@GDKOGIBB@Instance?5?8?$CFs?8?3?5no?5pid?5file?5to?5se@ 004c14dc     instance.obj
 0002:00001518       ??_C@_0CI@JALABLCD@Instance?5?8?$CFs?8?3?5can?5not?5unlink?5pi@ 004c1518     instance.obj
 0002:00001548       ??_C@_0ED@MIOJFHEA@Instance?5?8?$CFs?8?3?5waiting?5for?5mysql@ 004c1548     instance.obj
 0002:00001598       ??_C@_0CC@GLHGGNBE@Instance?5?8?$CFs?8?3?5Monitor?3?5finished@ 004c1598     instance.obj
 0002:000015c0       ??_C@_0CI@BFKLPFHJ@Instance?5?8?$CFs?8?3?5Monitor?3?5mysqld?5s@ 004c15c0     instance.obj
 0002:000015f0       ??_C@_0DG@CDAEBOCG@Instance?5?8?$CFs?8?3?5Monitor?3?5waiting?5@ 004c15f0     instance.obj
 0002:00001630       ??_C@_0CL@GDLMAENG@Instance?5?8?$CFs?8?3?5Monitor?3?5starting@ 004c1630     instance.obj
 0002:00001664       ??_C@_0CB@BEEEIFJP@Instance?5?8?$CFs?8?3?5Monitor?3?5started?4@ 004c1664     instance.obj
 0002:0000168c       ??_C@_0DH@FCHALOJO@Instance?5?8?$CFs?8?3?5can?5not?5create?5in@ 004c168c     instance.obj
 0002:000016d0       ??_C@_0DG@MAGOENIF@Instance?5?8?$CFs?8?3?5can?5not?5kill?5mysq@ 004c16d0     instance.obj
 0002:00001710       ??_C@_0CH@BOIKBMHP@Instance?5?8?$CFs?8?3?5mysqld?5has?5been?5k@ 004c1710     instance.obj
 0002:00001740       ??_C@_0CA@KEBKADIL@Instance?8?$CFs?8?3?5killing?5mysqld?4?4?4?$AA@ 004c1740     instance.obj
 0002:00001768       ??_C@_0ED@EDMKKIGO@Instance?5?8?$CFs?8?3?5mysqld?5failed?5to?5@ 004c1768     instance.obj
 0002:000017b8       ??_C@_0CK@DAICMCAL@Instance?5?8?$CFs?8?3?5mysqld?5stopped?5gr@ 004c17b8     instance.obj
 0002:000017ec       ??_C@_0CC@LKFDENEP@Instance?5?8?$CFs?8?3?5stopping?5mysqld?4?4@ 004c17ec     instance.obj
 0002:00001814       ??_C@_0O@BAHIDACC@misconfigured?$AA@ 004c1814     instance.obj
 0002:00001824       ??_C@_0CI@LIHMLOA@Can?5not?5register?5instance?5?$CIname?3@ 004c1824     instance_map.obj
 0002:00001854       ??_C@_0DK@JKJGICIL@Can?5not?5complete?5initialization?5@ 004c1854     instance_map.obj
 0002:0000189c       ??_C@_0DC@CFEOAIDM@Warning?3?5instance?5name?5?8?$CFs?8?5is?5m@ 004c189c     instance_map.obj
 0002:000018d8       ??_C@_0FE@IILGJPJC@IM?9option?5?$CI?$CFs?$CJ?5can?5not?5be?5used?5i@ 004c18d8     instance_map.obj
 0002:0000193c       ??_C@_0CK@EBEJNCOF@Can?5not?5initialize?5instance?5?$CInam@ 004c193c     instance_map.obj
 0002:00001970       ??_C@_0CI@NKEBMEMH@Can?5not?5allocate?5instance?5?$CIname?3@ 004c1970     instance_map.obj
 0002:000019a0       ??_C@_0CO@MDKJDFNJ@Can?5not?5write?5to?5configuration?5f@ 004c19a0     instance_map.obj
 0002:000019d8       ??_C@_01NEMOKFLO@?$DN?$AA@ 004c19d8     instance_map.obj
 0002:000019dc       ??_C@_01LBDDMOBJ@?$FN?$AA@ 004c19dc     instance_map.obj
 0002:000019e0       ??_C@_01OHGJGJJP@?$FL?$AA@ 004c19e0     instance_map.obj
 0002:000019e4       ??_C@_02PCIJFNDE@?$AN?6?$AA@ 004c19e4     instance_map.obj
 0002:000019e8       ??_C@_0CK@ENFIMMHO@Can?5not?5open?5configuration?5file?5@ 004c19e8     instance_map.obj
 0002:00001a1c       ??_C@_0CI@OFOLHJNB@Configuration?5file?5?$CI?$CFs?$CJ?5does?5not@ 004c1a1c     instance_map.obj
 0002:00001a50       ??_C@_0JL@ENGJPKOG@Warning?3?5configuration?5of?5mysqld@ 004c1a50     instance_map.obj
 0002:00001b0c       ??_C@_0DC@EOJCNNLG@mysqld?5instance?5?8?$CFs?8?5has?5been?5ad@ 004c1b0c     instance_map.obj
 0002:00001b48       ??_C@_0DB@ODOAOEAB@Can?5not?5add?5default?5instance?5to?5@ 004c1b48     instance_map.obj
 0002:00001b84       ??_C@_0CB@FAMGEAGB@Can?5not?5create?5default?5instance?4@ 004c1b84     instance_map.obj
 0002:00001bac       ??_C@_0CG@MMPIFPAN@Falling?5back?5to?5compiled?9in?5defa@ 004c1bac     instance_map.obj
 0002:00001bdc       ??_C@_0BD@BMHFPFCK@?9?9defaults?9file?$DN?$CFs?$AA@ 004c1bdc     instance_map.obj
 0002:00001bf4       ??_C@_0N@MBMMAPDF@mysqlmanager?$AA@ 004c1bf4     instance_map.obj
 0002:00001c04       ??_C@_0L@PNJKAIKE@nonguarded?$AA@ 004c1c04     instance_options.obj
 0002:00001c14       ??_C@_0M@IKAFELGN@mysqld?9path?$AA@ 004c1c14     instance_options.obj
 0002:00001c24       ??_C@_0P@DLJJMICC@shutdown?9delay?$AA@ 004c1c24     instance_options.obj
 0002:00001c38       ??_C@_0CA@PNOFEODE@?5?9?9no?9defaults?5?9?9verbose?5?9?9help?$AA@ 004c1c38     instance_options.obj
 0002:00001c60       ??_C@_0DC@HCHGLGMH@Failed?5to?5get?5version?5of?5?8?$CFs?8?3?5u@ 004c1c60     instance_options.obj
 0002:00001c9c       ??_C@_03GDMIGCCC@Ver?$AA@  004c1c9c     instance_options.obj
 0002:00001ca0       ??_C@_0CO@ILMIHJFJ@Failed?5to?5get?5version?5of?5?8?$CFs?8?3?5o@ 004c1ca0     instance_options.obj
 0002:00001cd8       ??_C@_0BJ@HDFDNOPO@?5?9?9no?9defaults?5?9?9version?$AA@ 004c1cd8     instance_options.obj
 0002:00001cf8       ??_C@_09DGMGBAEA@?$FLOPTIONS?$FN?$AA@ 004c1cf8     instance_options.obj
 0002:00001d04       ??_C@_0DE@MNFMADFI@Failed?5to?5get?5real?5path?5of?5?8?$CFs?8?3@ 004c1d04     instance_options.obj
 0002:00001d44       ??_C@_07CKBCDPF@Usage?3?5?$AA@ 004c1d44     instance_options.obj
 0002:00001d50       ??_C@_0DA@BCPJGHBA@Failed?5to?5get?5real?5path?5of?5?8?$CFs?8?3@ 004c1d50     instance_options.obj
 0002:00001d8c       ??_C@_0BG@FCNLNJKD@?5?9?9no?9defaults?5?9?9help?$AA@ 004c1d8c     instance_options.obj
 0002:00001da8       ??_C@_05OLGEOJNI@mysql?$AA@ 004c1da8     instance_options.obj
 0002:00001db0       ??_C@_09HGKCAJKI@?9?9datadir?$AA@ 004c1db0     instance_options.obj
 0002:00001dbc       ??_C@_09OFFDPMNL@?9slow?4log?$AA@ 004c1dbc     instance_options.obj
 0002:00001dc8       ??_C@_0BD@OPICEAGD@?9?9log?9slow?9queries?$AA@ 004c1dc8     instance_options.obj
 0002:00001de0       ??_C@_04FPOLKAEB@?4log?$AA@ 004c1de0     instance_options.obj
 0002:00001de8       ??_C@_05NEJJJKMH@?9?9log?$AA@ 004c1de8     instance_options.obj
 0002:00001df0       ??_C@_04BKIDJPM@?4err?$AA@ 004c1df0     instance_options.obj
 0002:00001df8       ??_C@_0M@DHGGKIBL@?9?9log?9error?$AA@ 004c1df8     instance_options.obj
 0002:00001e08       ??_C@_01KMDKNFGN@?1?$AA@   004c1e08     instance_options.obj
 0002:00001e0c       ??_C@_02IKAHHCAI@?$CFi?$AA@ 004c1e0c     instance_options.obj
 0002:00001e10       ??_C@_08OLCBHKMI@pid?9file?$AA@ 004c1e10     instance_options.obj
 0002:00001e1c       ??_C@_07DJBHFDCD@datadir?$AA@ 004c1e1c     instance_options.obj
 0002:00001e28       ??_C@_04LPGMAPLE@port?$AA@ 004c1e28     instance_options.obj
 0002:00001e30       ??_C@_06HBELJPBO@socket?$AA@ 004c1e30     instance_options.obj
 0002:00001e38       ??_C@_09PGAHDFGH@argv?3?5?$CFs?6?$AA@ 004c1e38     instance_options.obj
 0002:00001e44       ??_C@_0CD@NLOANHMJ@printing?5out?5an?5instance?5?$CFs?5argv@ 004c1e44     instance_options.obj
 0002:00001e70       ??_C@_02BAABKJLB@?9?9?$AA@ 004c1e70     instance_options.obj
 0002:00001e74       ??_C@_01JOAMLHOP@?9?$AA@   004c1e74     instance_options.obj
 0002:00001e78       ??_C@_04GKIEGHBH@?4pid?$AA@ 004c1e78     instance_options.obj
 0002:00001e80       ??_C@_0O@LNAGOGFC@?9?9no?9defaults?$AA@ 004c1e80     instance_options.obj
 0002:00001e90       ?LISTEN_BACK_LOG_SIZE@Listener@@0HB 004c1e90     listener.obj
 0002:00001e98       ??_7Listener@@6B@          004c1e98     listener.obj
 0002:00001ea4       ??_C@_0DL@FELBGCJL@Listener?3?5accepting?5connections?5@ 004c1ea4     listener.obj
 0002:00001eec       ??_C@_0CI@EFCGJAL@Listener?3?5listen?$CIip?5socket?$CJ?5fail@ 004c1eec     listener.obj
 0002:00001f1c       ??_C@_0CG@DAMMONNM@Listener?3?5bind?$CIip?5socket?$CJ?5failed@ 004c1f1c     listener.obj
 0002:00001f4c       ??_C@_0CG@KCNJHJFG@Listener?3?5socket?$CIAF_INET?$CJ?5failed@ 004c1f4c     listener.obj
 0002:00001f7c       ??_C@_0CM@GIBNOMBE@Listener?3?5can?5not?5start?5connecti@ 004c1f7c     listener.obj
 0002:00001fb0       ??_C@_0BE@EKNLPMLD@Listener?3?5finished?4?$AA@ 004c1fb0     listener.obj
 0002:00001fc8       ??_C@_0CJ@GKEKOOEG@Listener?3?5shutdown?5requested?0?5ex@ 004c1fc8     listener.obj
 0002:00001ffc       ??_C@_0BP@HLLAMEBI@Listener?3?5select?$CI?$CJ?5failed?3?5?$CFs?4?$AA@ 004c1ffc     listener.obj
 0002:00002024       ??_C@_0DF@HKOKJDHM@Listener?3?5failed?5to?5initialize?4?5@ 004c2024     listener.obj
 0002:00002064       ??_C@_0BD@NCBJHKL@Listener?3?5started?4?$AA@ 004c2064     listener.obj
 0002:0000207c       ??_C@_05JMJKDBEJ@?$CFs?$CFs?6?$AA@ 004c207c     log.obj
 0002:00002084       ??_C@_0CO@EMDKHBOI@log?$CI?$CJ?3?5message?5is?5too?5big?0?5my_ma@ 004c2084     log.obj
 0002:000020bc       ??_C@_0CP@LMPLHIIL@?$FL?$CFd?1?$CFlu?$FN?5?$FL?$CF02d?1?$CF02d?1?$CF02d?5?$CF02d?3?$CF0@ 004c20bc     log.obj
 0002:000020f4       ??_C@_05MBDEGLCK@ERROR?$AA@ 004c20f4     log.obj
 0002:000020fc       ??_C@_04BEADLPGM@INFO?$AA@ 004c20fc     log.obj
 0002:00002104       ??_C@_01EEMJAFIK@?6?$AA@   004c2104     log.obj
 0002:00002108       ??_C@_04PFAOODAA@?$CFs?3?5?$AA@ 004c2108     log.obj
 0002:00002114       ??_7ThreadModelChecker@?A0x2a2a756e@@6B@ 004c2114     manager.obj
 0002:00002120       ??_C@_0N@PANILCOJ@Manager?3?5?$CFs?4?$AA@ 004c2120     manager.obj
 0002:00002130       ??_C@_0FL@OFDAGJKP@Warning?3?5password?5file?5does?5not?5@ 004c2130     manager.obj
 0002:000021a0       ??_C@_0DG@DJAIBBOJ@Manager?3?5can?5not?5initialize?5user@ 004c21a0     manager.obj
 0002:000021e0       ??_C@_0BK@PKMPDDGP@Manager?3?5sigwait?$CI?$CJ?5failed?$AA@ 004c21e0     manager.obj
 0002:00002200       ??_C@_0BD@BKGNGCAN@Manager?3?5finished?4?$AA@ 004c2200     manager.obj
 0002:00002218       ??_C@_0BO@MKKBBAKA@Manager?3?5got?5shutdown?5signal?4?$AA@ 004c2218     manager.obj
 0002:0000223c       ??_C@_0BC@LOMOBFNL@Manager?3?5started?4?$AA@ 004c223c     manager.obj
 0002:00002254       ??_C@_0CI@KODGBOEG@Manager?3?5can?5not?5start?5Listener?5@ 004c2254     manager.obj
 0002:00002284       ??_C@_0CM@OPLHEMPM@Manager?3?5can?5not?5init?5instances?5@ 004c2284     manager.obj
 0002:000022b8       ??_C@_0CI@GKNKKAIM@Manager?3?5can?5not?5start?5Guardian?5@ 004c22b8     manager.obj
 0002:000022e8       ??_C@_0CA@EMIOCEBB@Manager?3?5pid?5file?5?$CI?$CFs?$CJ?5created?4?$AA@ 004c22e8     manager.obj
 0002:00002310       ??_C@_0DK@KJHDPGIO@Manager?3?5can?5not?5initialize?5inst@ 004c2310     manager.obj
 0002:00002358       ??_C@_0BJ@DLDDEGPM@Manager?3?5initializing?4?4?4?$AA@ 004c2358     manager.obj
 0002:00002378       ??_C@_0CC@IOEEFNGH@Configuration?5file?5does?5not?5exis@ 004c2378     messages.obj
 0002:000023a0       ??_C@_0HF@JDADLGEN@Instance?5Manager?9specific?5option@ 004c23a0     messages.obj
 0002:0000242c       ??_C@_0DK@EOPGDEKG@At?5least?5one?5instance?5is?5active?4@ 004c242c     messages.obj
 0002:00002474       ??_C@_0DA@NKPLOLCO@The?5instance?5is?5active?4?5Stop?5the@ 004c2474     messages.obj
 0002:000024b0       ??_C@_0BJ@PGDOFGBC@Malformed?5instance?5name?4?$AA@ 004c24b0     messages.obj
 0002:000024d0       ??_C@_0CL@HILCLIIH@Instance?5is?5misconfigured?4?5Canno@ 004c24d0     messages.obj
 0002:00002504       ??_C@_0BI@FMHOLMKL@Instance?5already?5exists?$AA@ 004c2504     messages.obj
 0002:00002520       ??_C@_0DJ@PMBEDDFP@Cannot?5drop?5an?5active?5instance?4?5@ 004c2520     messages.obj
 0002:00002564       ??_C@_0DH@OLEIDFFJ@Cannot?5open?5the?5option?5file?5to?5e@ 004c2564     messages.obj
 0002:000025a8       ??_C@_0FE@PBJNMGMK@Cannot?5guess?5the?5log?5filename?4?5T@ 004c25a8     messages.obj
 0002:0000260c       ??_C@_0BF@CCAMAPAA@Cannot?5open?5log?5file?$AA@ 004c260c     messages.obj
 0002:00002628       ??_C@_0CF@HGFDHMPH@The?5instance?5has?5no?5such?5log?5ena@ 004c2628     messages.obj
 0002:00002654       ??_C@_0CK@BDCIGLMK@Cannot?5read?5requested?5part?5of?5th@ 004c2654     messages.obj
 0002:00002688       ??_C@_0BF@BOFNNLAC@Cannot?5stop?5instance?$AA@ 004c2688     messages.obj
 0002:000026a4       ??_C@_0CF@EPBEMJMO@Cannot?5read?5negative?5number?5of?5b@ 004c26a4     messages.obj
 0002:000026d0       ??_C@_0FJ@FAEFAGFE@Cannot?5start?5instance?4?5Possible?5@ 004c26d0     messages.obj
 0002:0000273c       ??_C@_0CA@OIEOKEDL@The?5instance?5is?5already?5started?$AA@ 004c273c     messages.obj
 0002:00002768       ??_C@_0HD@GGDAMBEA@Cannot?5stop?5instance?4?5Perhaps?5th@ 004c2768     messages.obj
 0002:000027f4       ??_C@_0BG@PFHNHGMA@Unknown?5instance?5name?$AA@ 004c27f4     messages.obj
 0002:00002810       ??_C@_0GF@CPHLBCPM@Client?5does?5not?5support?5authenti@ 004c2810     messages.obj
 0002:00002890       ??_C@_0IP@BELLFNGA@You?5have?5an?5error?5in?5your?5comman@ 004c2890     messages.obj
 0002:0000293c       ??_C@_0BA@MPOJHAMO@Unknown?5command?$AA@ 004c293c     messages.obj
 0002:00002950       ??_C@_0CK@DOCEONGH@Access?5denied?4?5Bad?5username?1pass@ 004c2950     messages.obj
 0002:00002988       ??_C@_0LH@OBGNHNPK@Out?5of?5memory?$DL?5?5Check?5if?5mysqld?5@ 004c2988     messages.obj
 0002:00002a64       ??_C@_0O@DIOIANKF@Bad?5handshake?$AA@ 004c2a64     messages.obj
 0002:00002a78       ??_7Mysql_connection@@6B@  004c2a78     mysql_connection.obj
 0002:00002a84       ??_C@_0CH@OOGLBEGM@Connection?5?$CFlu?3?5received?5QUIT?5co@ 004c2a84     mysql_connection.obj
 0002:00002ab4       ??_C@_0DH@OALJBMIN@Connection?5?$CFlu?3?5can?5not?5parse?5qu@ 004c2ab4     mysql_connection.obj
 0002:00002af8       ??_C@_0DD@KJLKCFKC@Connection?5?$CFlu?3?5can?5not?5execute?5@ 004c2af8     mysql_connection.obj
 0002:00002b38       ??_C@_0CM@PGHKHOAF@Connection?5?$CFlu?3?5query?5executed?5s@ 004c2b38     mysql_connection.obj
 0002:00002b6c       ??_C@_0CL@FBNOCNOF@Connection?5?$CFlu?3?5query?5parsed?5suc@ 004c2b6c     mysql_connection.obj
 0002:00002ba0       ??_C@_0CO@JFCMKLJ@Connection?5?$CFlu?3?5received?5QUERY?5c@ 004c2ba0     mysql_connection.obj
 0002:00002bd8       ??_C@_0CH@BOFFKBHO@Connection?5?$CFlu?3?5received?5PING?5co@ 004c2bd8     mysql_connection.obj
 0002:00002c08       ??_C@_0DD@BEOBPCHN@Connection?5?$CFlu?3?5received?5unsuppo@ 004c2c08     mysql_connection.obj
 0002:00002c48       ??_C@_0DM@LEFAKPBA@Connection?5?$CFlu?3?5received?5packet?5@ 004c2c48     mysql_connection.obj
 0002:00002c90       ??_C@_0DG@MHMJEMMF@Connection?5?$CFlu?3?5the?5user?5was?5aut@ 004c2c90     mysql_connection.obj
 0002:00002cd0       ??_C@_0CO@GLLPLBF@Connection?5?$CFlu?3?5failed?5to?5author@ 004c2cd0     mysql_connection.obj
 0002:00002d08       ??_C@_0BK@JPCGKMIE@Connection?5?$CFlu?3?5accepted?4?$AA@ 004c2d08     mysql_connection.obj
 0002:00002d28       ??_C@_0CG@IGHBHBKI@Connection?5?$CFlu?3?5can?5not?5init?5han@ 004c2d28     mysql_connection.obj
 0002:00002d58       ??_C@_0O@NICLPIJL@IM?3?5finished?4?$AA@ 004c2d58     mysqlmanager.obj
 0002:00002d68       ??_C@_0N@CPKLCEGH@IM?3?5started?4?$AA@ 004c2d68     mysqlmanager.obj
 0002:00002d78       ??_C@_0EC@PKPNDGNL@?6WARNING?3?5This?5program?5is?5deprec@ 004c2d78     mysqlmanager.obj
 0002:00002dc8       ??_C@_07JPLKDPHP@manager?$AA@ 004c2dc8     options.obj
 0002:00002dd8       ??_C@_0EP@PDDIBNOH@The?5number?5of?5seconds?5IM?5waits?5f@ 004c2dd8     options.obj
 0002:00002e38       ??_C@_0N@IKNOIIJE@wait?9timeout?$AA@ 004c2e38     options.obj
 0002:00002e48       ??_C@_0CF@PMNNCCFJ@Output?5version?5information?5and?5e@ 004c2e48     options.obj
 0002:00002e74       ??_C@_0CG@JBFFICBH@Username?5to?5update?5the?5password?5@ 004c2e74     options.obj
 0002:00002ea4       ??_C@_08ODGEKKOL@username?$AA@ 004c2ea4     options.obj
 0002:00002eb0       ??_C@_0CJ@IONBCKIB@Run?5the?5application?5in?5stand?5alo@ 004c2eb0     options.obj
 0002:00002ee4       ??_C@_0L@FLHGMILF@standalone?$AA@ 004c2ee4     options.obj
 0002:00002ef4       ??_C@_0BH@DMOGDMLA@Remove?5system?5service?4?$AA@ 004c2ef4     options.obj
 0002:00002f10       ??_C@_06LEMKAMD@remove?$AA@ 004c2f10     options.obj
 0002:00002f18       ??_C@_0CE@NDMNFMGO@Port?5number?5to?5use?5for?5connectio@ 004c2f18     options.obj
 0002:00002f44       ??_C@_0BB@DGOMPFMC@Pid?5file?5to?5use?4?$AA@ 004c2f44     options.obj
 0002:00002f58       ??_C@_0DE@HMCHLBBP@Look?5for?5Instance?5Manager?5users?5@ 004c2f58     options.obj
 0002:00002f98       ??_C@_0O@JHLAPOPF@password?9file?$AA@ 004c2f98     options.obj
 0002:00002fa8       ??_C@_0CG@HEHNPAHK@Password?5to?5update?5the?5password?5@ 004c2fa8     options.obj
 0002:00002fd8       ??_C@_08NLHBPEGP@password?$AA@ 004c2fd8     options.obj
 0002:00002fe8       ??_C@_0EB@EPMGEMEG@Print?5out?5a?5user?5entry?5as?5a?5line@ 004c2fe8     options.obj
 0002:00003038       ??_C@_0BE@JBMHOAKG@print?9password?9line?$AA@ 004c3038     options.obj
 0002:00003050       ??_C@_0DJ@HPGBHOCK@Start?5Instance?5Manager?5in?5mysqld@ 004c3050     options.obj
 0002:00003094       ??_C@_0BH@BDEONKFN@mysqld?9safe?9compatible?$AA@ 004c3094     options.obj
 0002:000030b0       ??_C@_0CK@FMEHMJFO@Interval?5to?5monitor?5instances?5in@ 004c30b0     options.obj
 0002:000030e4       ??_C@_0BE@INENLLN@monitoring?9interval?$AA@ 004c30e4     options.obj
 0002:000030fc       ??_C@_0CG@GMJENMHO@Print?5out?5a?5list?5of?5registered?5u@ 004c30fc     options.obj
 0002:0000312c       ??_C@_0L@BGBIMKCH@list?9users?$AA@ 004c312c     options.obj
 0002:0000313c       ??_C@_0BL@KHPAFIOP@Install?5as?5system?5service?4?$AA@ 004c313c     options.obj
 0002:0000315c       ??_C@_07EALBDFH@install?$AA@ 004c315c     options.obj
 0002:00003168       ??_C@_0CJ@PAHCHFBH@Edit?5existing?5user?5in?5the?5passwo@ 004c3168     options.obj
 0002:0000319c       ??_C@_09FNCIKDCH@edit?9user?$AA@ 004c319c     options.obj
 0002:000031a8       ??_C@_0CL@GCDDJALK@Drop?5existing?5user?5from?5the?5pass@ 004c31a8     options.obj
 0002:000031dc       ??_C@_09FPBANOHG@drop?9user?$AA@ 004c31dc     options.obj
 0002:000031e8       ??_C@_0CH@LIAINEMB@Where?5to?5look?5for?5MySQL?5Server?5b@ 004c31e8     options.obj
 0002:00003218       ??_C@_0BE@HCHLGHAI@default?9mysqld?9path?$AA@ 004c3218     options.obj
 0002:00003230       ??_C@_0BJ@OGOGONKD@Clean?5the?5password?5file?4?$AA@ 004c3230     options.obj
 0002:00003250       ??_C@_0BE@NIEMCJHH@clean?9password?9file?$AA@ 004c3250     options.obj
 0002:00003268       ??_C@_0CJ@LHJCNMMI@Check?5the?5password?5file?5for?5cons@ 004c3268     options.obj
 0002:0000329c       ??_C@_0BE@JPEBGJEE@check?9password?9file?$AA@ 004c329c     options.obj
 0002:000032b4       ??_C@_0CE@LKPLDHBK@Bind?5address?5to?5use?5for?5connecti@ 004c32b4     options.obj
 0002:000032e0       ??_C@_0N@KPFNDBAM@bind?9address?$AA@ 004c32e0     options.obj
 0002:000032f0       ??_C@_0CB@PCBIIIIC@Add?5a?5user?5to?5the?5password?5file?4@ 004c32f0     options.obj
 0002:00003318       ??_C@_08NJCJNMJL@add?9user?$AA@ 004c3318     options.obj
 0002:00003324       ??_C@_0BM@BKPKLHCC@Display?5this?5help?5and?5exit?4?$AA@ 004c3324     options.obj
 0002:00003348       ??_C@_04PCJFHION@help?$AA@ 004c3348     options.obj
 0002:00003350       ??_C@_0L@MFNJLFIO@?4angel?4pid?$AA@ 004c3350     options.obj
 0002:00003368       ??_7User_management_cmd@@6B@ 004c3368     options.obj
 0002:00003378       ??_7Print_password_line_cmd@@6B@ 004c3378     options.obj
 0002:00003388       ??_7Add_user_cmd@@6B@      004c3388     options.obj
 0002:00003398       ??_7Drop_user_cmd@@6B@     004c3398     options.obj
 0002:000033a8       ??_7Edit_user_cmd@@6B@     004c33a8     options.obj
 0002:000033b8       ??_7Clean_db_cmd@@6B@      004c33b8     options.obj
 0002:000033c8       ??_7Check_db_cmd@@6B@      004c33c8     options.obj
 0002:000033d8       ??_7List_users_cmd@@6B@    004c33d8     options.obj
 0002:000033e4       ??_C@_0BI@DFCIJINN@?$CFs?5Ver?5?$CFs?5for?5?$CFs?5on?5?$CFs?6?$AA@ 004c33e4     options.obj
 0002:00003400       ??_C@_05NLDAPMKH@Win32?$AA@ 004c3400     options.obj
 0002:00003408       ??_C@_04OFDIICAA@ia32?$AA@ 004c3408     options.obj
 0002:00003410       ??_C@_0BHO@MDEOLIO@?6The?5following?5options?5may?5be?5gi@ 004c3410     options.obj
 0002:000035dc       ??_C@_0BG@GNEAPHGE@Usage?3?5?$CFs?5?$FLOPTIONS?$FN?5?6?$AA@ 004c35dc     options.obj
 0002:000035f8       ??_C@_0LF@NDONKEHG@Copyright?5?$CIC?$CJ?52003?0?52004?5MySQL?5A@ 004c35f8     options.obj
 0002:000036d8       ??_C@_0EJ@JCDHKOH@Error?3?5only?5one?5password?9managem@ 004c36d8     options.obj
 0002:00003730       ??_C@_07MODGBJDN@?4passwd?$AA@ 004c3730     options.obj
 0002:0000373c       ??_C@_06GKHGEOIF@my?4ini?$AA@ 004c373c     options.obj
 0002:00003748       ??_C@_0GO@DAKIGMAO@?9?9username?5and?1or?5?9?9password?5opt@ 004c3748     options.obj
 0002:000037cc       ??_C@_0BM@PFCLOIKI@Loading?5config?5file?5?8?$CFs?8?4?4?4?$AA@ 004c37cc     options.obj
 0002:000037f0       ??_C@_0DB@FPDBENAF@Internal?5error?3?5could?5not?5setup?5@ 004c37f0     options.obj
 0002:00003830       ??_C@_0GN@NBIDIJLJ@The?5?9?9defaults?9extra?9file?5and?5?9?9@ 004c3830     options.obj
 0002:000038b4       ??_C@_0BH@HNKMCPPG@?9?9defaults?9extra?9file?$DN?$AA@ 004c38b4     options.obj
 0002:000038d0       ??_C@_0BB@LDHKPEKC@?9?9defaults?9file?$DN?$AA@ 004c38d0     options.obj
 0002:000038e4       ??_C@_05IEIDFGAH@UNSET?$AA@ 004c38e4     parse.obj
 0002:000038ec       ??_C@_04JGPCMMEF@SHOW?$AA@ 004c38ec     parse.obj
 0002:000038f4       ??_C@_04MDHMLCKF@STOP?$AA@ 004c38f4     parse.obj
 0002:000038fc       ??_C@_06DNKMJCIK@STATUS?$AA@ 004c38fc     parse.obj
 0002:00003904       ??_C@_05JLPDBANI@START?$AA@ 004c3904     parse.obj
 0002:0000390c       ??_C@_04BJJAFLBC@SLOW?$AA@ 004c390c     parse.obj
 0002:00003914       ??_C@_03KPIFFHNE@SET?$AA@  004c3914     parse.obj
 0002:00003918       ??_C@_07KDKMIPIP@OPTIONS?$AA@ 004c3918     parse.obj
 0002:00003924       ??_C@_03MLIHNEFJ@LOG?$AA@  004c3924     parse.obj
 0002:00003928       ??_C@_09CJBINDHJ@INSTANCES?$AA@ 004c3928     parse.obj
 0002:00003934       ??_C@_08DDHIOBDH@INSTANCE?$AA@ 004c3934     parse.obj
 0002:00003940       ??_C@_07EGGHCNEO@GENERAL?$AA@ 004c3940     parse.obj
 0002:0000394c       ??_C@_05KALGKIBB@FLUSH?$AA@ 004c394c     parse.obj
 0002:00003954       ??_C@_05PENKCLCM@FILES?$AA@ 004c3954     parse.obj
 0002:0000395c       ??_C@_04DENHKGOL@DROP?$AA@ 004c395c     parse.obj
 0002:00003964       ??_C@_06DDGDDNE@CREATE?$AA@ 004c3964     parse.obj
 0002:00003970       ??_7Show_instances@@6B@    004c3970     parse.obj
 0002:00003980       ??_7Flush_instances@@6B@   004c3980     parse.obj
 0002:00003990       ??_7Set_option@@6B@        004c3990     parse.obj
 0002:000039a8       ??_7Unset_option@@6B@      004c39a8     parse.obj
 0002:000039c0       ??_7Syntax_error@@6B@      004c39c0     parse.obj
 0002:000039d0       ??_7Mysqld_output_parser@?A0x60d3fd73@@6B@ 004c39d0     parse_output.obj
 0002:000039e8       ??_7Mysqld_output_parser_win@?A0x60d3fd73@@6B@ 004c39e8     parse_output.obj
 0002:000039fc       ??_C@_08BPAFEFGI@1?40?9beta?$AA@ 004c39fc     priv.obj
 0002:00003a08       ?mysqlmanager_version@@3Ust_mysql_lex_string@@B 004c3a08     priv.obj
 0002:00003a10       ?protocol_version@@3EB     004c3a10     priv.obj
 0002:00003a14       ??_C@_0CP@GKJEFFOA@Can?5not?5write?5to?5pid?5file?5?8?$CFs?8?3?5@ 004c3a14     priv.obj
 0002:00003a4c       ??_C@_03PMGGPEJJ@?$CFd?6?$AA@ 004c3a4c     priv.obj
 0002:00003a50       ??_C@_0CN@OBBKEMCL@Can?5not?5create?5pid?5file?5?8?$CFs?8?3?5?$CFs@ 004c3a50     priv.obj
 0002:00003a88       ??_C@_0CL@FCAPHNPO@Thread_registry?3?5unregistered?5th@ 004c3a88     thread_registry.obj
 0002:00003abc       ??_C@_0DE@NDBPDJDJ@Invalid?5format?5?$CIunmatched?5quote?$CJ@ 004c3abc     user_map.obj
 0002:00003afc       ??_C@_0BC@PDKJIDJA@Loaded?5user?5?8?$CFs?8?4?$AA@ 004c3afc     user_map.obj
 0002:00003b14       ??_C@_0DL@FOHBFFCN@Password?5is?5too?5long?5?$CI?$CFd?$CJ?4?5Max?5l@ 004c3b14     user_map.obj
 0002:00003b5c       ??_C@_0DN@HGKBKDMF@User?5name?5is?5too?5long?5?$CI?$CFd?$CJ?4?5Max?5@ 004c3b5c     user_map.obj
 0002:00003ba8       ??_C@_0DB@NMPOEILG@Invalid?5format?5?$CIno?5delimiter?$CJ?5of@ 004c3ba8     user_map.obj
 0002:00003be4       ??_C@_0BN@PGLFBLJB@password?5file?5?$CI?$CFs?$CJ?5corrupted?$AA@ 004c3be4     user_map.obj
 0002:00003c08       ??_C@_0CP@LBNDNLDH@out?5of?5memory?5while?5parsing?5pass@ 004c3c08     user_map.obj
 0002:00003c40       ??_C@_0CL@CBOHIHHK@The?5password?5database?5loaded?5suc@ 004c3c40     user_map.obj
 0002:00003c74       ??_C@_0CB@MHJJCEGM@Loading?5the?5password?5database?4?4?4@ 004c3c74     user_map.obj
 0002:00003c9c       ??_C@_0CE@OIJOPBDA@can?5not?5open?5password?5file?5?$CI?$CFs?$CJ?3@ 004c3c9c     user_map.obj
 0002:00003cc8       ??_C@_0CC@PHMCNMNC@password?5file?5?$CI?$CFs?$CJ?5does?5not?5exis@ 004c3cc8     user_map.obj
 0002:00003cf0       ??_C@_0CI@MBNGKPCN@can?5not?5write?5to?5password?5file?5?$CI@ 004c3cf0     user_map.obj
 0002:00003d20       ??_C@_06KCIFIIHN@?$CFs?3?$CFs?6?$AA@ 004c3d20     user_map.obj
 0002:00003d28       ??_C@_0DA@NPDFEMBE@can?5not?5open?5password?5file?5?$CI?$CFs?$CJ?5@ 004c3d28     user_map.obj
 0002:00003d68       ??_7IMService@@6B@         004c3d68     IMService.obj
 0002:00003d88       ??_C@_0N@NFIKJEB@MySqlManager?$AA@ 004c3d88     IMService.obj
 0002:00003d98       ??_C@_0O@ONNFOFNE@MySQL?5Manager?$AA@ 004c3d98     IMService.obj
 0002:00003da8       ??_C@_0IM@NOFGBDBN@The?5service?5should?5be?5started?5by@ 004c3da8     IMService.obj
 0002:00003e50       ??_C@_0BO@BDBDHFNP@Service?5failed?5to?5initialize?4?$AA@ 004c3e50     IMService.obj
 0002:00003e74       ??_C@_0CJ@CNAPJDDL@Initializing?5Instance?5Manager?5se@ 004c3e74     IMService.obj
 0002:00003ea8       ??_C@_0BK@IFOJIBEI@Service?5failed?5to?5remove?4?$AA@ 004c3ea8     IMService.obj
 0002:00003ec8       ??_C@_0BO@HJJCINL@Service?5removed?5successfully?4?$AA@ 004c3ec8     IMService.obj
 0002:00003eec       ??_C@_0BK@LBIFJAII@Service?5is?5not?5installed?4?$AA@ 004c3eec     IMService.obj
 0002:00003f0c       ??_C@_0BL@ICFMKBII@Service?5failed?5to?5install?4?$AA@ 004c3f0c     IMService.obj
 0002:00003f2c       ??_C@_0CA@BECIKCAO@Service?5installed?5successfully?4?$AA@ 004c3f2c     IMService.obj
 0002:00003f54       ??_C@_0BO@BEOPPBDB@Service?5is?5already?5installed?4?$AA@ 004c3f54     IMService.obj
 0002:00003f7c       ??_7WindowsService@@6B@    004c3f7c     WindowsService.obj
 0002:00003f9c       ??_C@_0BE@GPLHKCHK@ReportStatus?5failed?$AA@ 004c3f9c     WindowsService.obj
 0002:00003fb4       ??_C@_0BC@DEAECJAP@Enter?5user?5name?3?5?$AA@ 004c3fb4     user_management_commands.obj
 0002:00003fcc       ??_C@_0DB@KILDAHGC@Error?3?5user?5name?5must?5not?5exceed@ 004c3fcc     user_management_commands.obj
 0002:00004008       ??_C@_0CE@BEAEOAEN@Error?3?5user?5name?5can?5not?5be?5empt@ 004c4008     user_management_commands.obj
 0002:00004034       ??_C@_0CN@HDLKOHLA@Error?3?5unable?5to?5read?5user?5name?5@ 004c4034     user_management_commands.obj
 0002:0000406c       ??_C@_0CA@GOLBANMM@Error?3?5passwords?5do?5not?5match?4?6?$AA@ 004c406c     user_management_commands.obj
 0002:00004094       ??_C@_0BD@NKGLHMFK@Re?9type?5password?3?5?$AA@ 004c4094     user_management_commands.obj
 0002:000040ac       ??_C@_0BB@LAEJCAEB@Enter?5password?3?5?$AA@ 004c40ac     user_management_commands.obj
 0002:000040c0       ??_C@_0M@KGJPEMDD@Error?3?5?$CFs?4?6?$AA@ 004c40c0     user_management_commands.obj
 0002:000040d0       ??_C@_0CF@OMFDBANG@Error?3?5can?5not?5initialize?5user?5m@ 004c40d0     user_management_commands.obj
 0002:000040fc       ??_C@_0BP@NJIBNPLM@Creating?5record?5for?5new?5user?4?6?$AA@ 004c40fc     user_management_commands.obj
 0002:00004124       ??_C@_0CC@DLAOCCBA@Error?3?5user?5?8?$CFs?8?5already?5exists?4@ 004c4124     user_management_commands.obj
 0002:0000414c       ??_C@_0CC@OEEDCFII@Error?3?5user?5?8?$CFs?8?5does?5not?5exist?4@ 004c414c     user_management_commands.obj
 0002:00004174       ??_C@_03OFAPEBGM@?$CFs?6?$AA@ 004c4174     user_management_commands.obj
 0002:00004178       __real@41cfffffff800000    004c4178     password.obj
 0002:00004184       ??_C@_0L@KDJOJLDL@?$CF08lx?$CF08lx?$AA@ 004c4184     password.obj
 0002:00004198       __real@4050000000000000    004c4198     password.obj
 0002:000041a8       __real@403f000000000000    004c41a8     password.obj
 0002:000041b8       __real@4040800000000000    004c41b8     password.obj
 0002:000041c8       __real@4057800000000000    004c41c8     password.obj
 0002:000041d4       ??_C@_05EKPPILBK@XA102?$AA@ 004c41d4     sql_state.obj
 0002:000041dc       ??_C@_05COJDEOBO@XA106?$AA@ 004c41dc     sql_state.obj
 0002:000041e4       ??_C@_05HMFDNFIP@25001?$AA@ 004c41e4     sql_state.obj
 0002:000041ec       ??_C@_05BPLBLCNG@22008?$AA@ 004c41ec     sql_state.obj
 0002:000041f4       ??_C@_05FEENFEFL@XAE08?$AA@ 004c41f4     sql_state.obj
 0002:000041fc       ??_C@_05MOHDAJJP@22001?$AA@ 004c41fc     sql_state.obj
 0002:00004204       ??_C@_05HIMJOJJI@XA100?$AA@ 004c4204     sql_state.obj
 0002:0000420c       ??_C@_05LHLJINJA@XAE03?$AA@ 004c420c     sql_state.obj
 0002:00004214       ??_C@_05ENFGGFBK@XAE09?$AA@ 004c4214     sql_state.obj
 0002:0000421c       ??_C@_05NDNFEIJE@XAE07?$AA@ 004c421c     sql_state.obj
 0002:00004224       ??_C@_05OBODCKBG@XAE05?$AA@ 004c4224     sql_state.obj
 0002:0000422c       ??_C@_05PIPIBLFH@XAE04?$AA@ 004c422c     sql_state.obj
 0002:00004234       ??_C@_05OEJMDAGL@22012?$AA@ 004c4234     sql_state.obj
 0002:0000423c       ??_C@_05KNKIGLLO@20000?$AA@ 004c423c     sql_state.obj
 0002:00004244       ??_C@_05JKKAJJNF@02000?$AA@ 004c4244     sql_state.obj
 0002:0000424c       ??_C@_05FICIMNHO@24000?$AA@ 004c424c     sql_state.obj
 0002:00004254       ??_C@_05KGENIKJE@2F005?$AA@ 004c4254     sql_state.obj
 0002:0000425c       ??_C@_05EFNJJNGI@70100?$AA@ 004c425c     sql_state.obj
 0002:00004264       ??_C@_05CENCADMK@0A000?$AA@ 004c4264     sql_state.obj
 0002:0000426c       ??_C@_05PABHCNBC@2F003?$AA@ 004c426c     sql_state.obj
 0002:00004274       ??_C@_05JICJKOBJ@22007?$AA@ 004c4274     sql_state.obj
 0002:0000427c       ??_C@_05PMEFGLBN@22003?$AA@ 004c427c     sql_state.obj
 0002:00004284       ??_C@_05NNAAODAF@01000?$AA@ 004c4284     sql_state.obj
 0002:0000428c       ??_C@_05JAMIECAO@21000?$AA@ 004c428c     sql_state.obj
 0002:00004294       ??_C@_05GCOKLJOC@40001?$AA@ 004c4294     sql_state.obj
 0002:0000429c       ??_C@_05GFEIOEMO@25000?$AA@ 004c429c     sql_state.obj
 0002:000042a4       ??_C@_05LDAEPNNK@22004?$AA@ 004c42a4     sql_state.obj
 0002:000042ac       ??_C@_05BLFGILJL@42S12?$AA@ 004c42ac     sql_state.obj
 0002:000042b4       ??_C@_05IFAOCAIO@s1009?$AA@ 004c42b4     sql_state.obj
 0002:000042bc       ??_C@_05DCDNGGAB@42S21?$AA@ 004c42bc     sql_state.obj
 0002:000042c4       ??_C@_05KAEACLKC@21S01?$AA@ 004c42c4     sql_state.obj
 0002:000042cc       ??_C@_05ICKCCFLI@S1009?$AA@ 004c42cc     sql_state.obj
 0002:000042d4       ??_C@_05FPLCABKN@S0022?$AA@ 004c42d4     sql_state.obj
 0002:000042dc       ??_C@_05BJBADFMC@42S22?$AA@ 004c42dc     sql_state.obj
 0002:000042e4       ??_C@_05BKJEOBKM@42S02?$AA@ 004c42e4     sql_state.obj
 0002:000042ec       ??_C@_05DBLJLCGP@42S01?$AA@ 004c42ec     sql_state.obj
 0002:000042f4       ??_C@_05GKKGPOBE@3D000?$AA@ 004c42f4     sql_state.obj
 0002:000042fc       ??_C@_05JNNICAHP@28000?$AA@ 004c42fc     sql_state.obj
 0002:00004304       ??_C@_05BDBNLMD@42000?$AA@ 004c4304     sql_state.obj
 0002:0000430c       ??_C@_05OAJIOINI@08S01?$AA@ 004c430c     sql_state.obj
 0002:00004314       ??_C@_05LEHMEEHA@08004?$AA@ 004c4314     sql_state.obj
 0002:0000431c       ??_C@_05EKHLKPLA@S1001?$AA@ 004c431c     sql_state.obj
 0002:00004324       ??_C@_05IKCIGBGE@HY001?$AA@ 004c4324     sql_state.obj
 0002:0000432c       ??_C@_05OKAIBBGO@23000?$AA@ 004c432c     sql_state.obj
 0002:00004334       ??_C@_05JDDDFACF@HY000?$AA@ 004c4334     sql_state.obj
 0002:0000433c       ??_C@_06HPIPGHLH@MEMORY?$AA@ 004c433c     client.obj
 0002:00004344       ??_C@_04GGAEFGO@PIPE?$AA@  004c4344     client.obj
 0002:0000434c       ??_C@_06HFGAEBMM@SOCKET?$AA@ 004c434c     client.obj
 0002:00004354       ??_C@_03FCLDNGNL@TCP?$AA@  004c4354     client.obj
 0002:00004358       ??_C@_07FOPBDDAL@options?$AA@ 004c4358     client.obj
 0002:00004364       ??_C@_0BH@BONNBGIA@report?9data?9truncation?$AA@ 004c4364     client.obj
 0002:00004380       ??_C@_0M@PMDPKFDA@secure?9auth?$AA@ 004c4380     client.obj
 0002:00004390       ??_C@_0O@IGPGCENI@multi?9queries?$AA@ 004c4390     client.obj
 0002:000043a0       ??_C@_0BB@ECMBLIEH@multi?9statements?$AA@ 004c43a0     client.obj
 0002:000043b4       ??_C@_0O@CCDCLLBG@multi?9results?$AA@ 004c43b4     client.obj
 0002:000043c4       ??_C@_0BI@FOKNPLJP@shared?9memory?9base?9name?$AA@ 004c43c4     client.obj
 0002:000043e0       ??_C@_08FCFPNNHF@protocol?$AA@ 004c43e0     client.obj
 0002:000043ec       ??_C@_0BD@OFGLABCB@max?9allowed?9packet?$AA@ 004c43ec     client.obj
 0002:00004404       ??_C@_0L@PHBCGEDL@ssl?9cipher?$AA@ 004c4404     client.obj
 0002:00004414       ??_C@_0BB@HNHJLDBF@repl?9parse?9query?$AA@ 004c4414     client.obj
 0002:00004428       ??_C@_0BJ@JAEAFHJM@enable?9reads?9from?9master?$AA@ 004c4428     client.obj
 0002:00004448       ??_C@_0BC@BKIPLOIH@replication?9probe?$AA@ 004c4448     client.obj
 0002:00004460       ??_C@_0BF@DNHMICAO@disable?9local?9infile?$AA@ 004c4460     client.obj
 0002:0000447c       ??_C@_0N@DEPIEDDP@local?9infile?$AA@ 004c447c     client.obj
 0002:0000448c       ??_C@_0BA@PKFDCPCI@connect?9timeout?$AA@ 004c448c     client.obj
 0002:000044a0       ??_C@_0BE@PKKGFOHM@interactive?9timeout?$AA@ 004c44a0     client.obj
 0002:000044b8       ??_C@_0BG@BMMCDGOA@default?9character?9set?$AA@ 004c44b8     client.obj
 0002:000044d4       ??_C@_0BD@HPLEKGGN@character?9sets?9dir?$AA@ 004c44d4     client.obj
 0002:000044ec       ??_C@_0L@MLIAJKEA@ssl?9capath?$AA@ 004c44ec     client.obj
 0002:000044fc       ??_C@_06KEIFHGI@ssl?9ca?$AA@ 004c44fc     client.obj
 0002:00004504       ??_C@_08MLGPLICL@ssl?9cert?$AA@ 004c4504     client.obj
 0002:00004510       ??_C@_07HPCDODLB@ssl?9key?$AA@ 004c4510     client.obj
 0002:0000451c       ??_C@_0BC@CPNNNMD@return?9found?9rows?$AA@ 004c451c     client.obj
 0002:00004534       ??_C@_05GFCDIDHO@debug?$AA@ 004c4534     client.obj
 0002:0000453c       ??_C@_08PBOCEOLL@database?$AA@ 004c453c     client.obj
 0002:00004548       ??_C@_04OODOLJMA@host?$AA@ 004c4548     client.obj
 0002:00004550       ??_C@_0N@CJBLNCLF@init?9command?$AA@ 004c4550     client.obj
 0002:00004560       ??_C@_04CCHAHKJA@user?$AA@ 004c4560     client.obj
 0002:00004568       ??_C@_07DDHNKDGP@timeout?$AA@ 004c4568     client.obj
 0002:00004574       ??_C@_04MKFKKHBG@pipe?$AA@ 004c4574     client.obj
 0002:0000457c       ??_C@_08EJNPIMGB@compress?$AA@ 004c457c     client.obj
 0002:00004588       ??_C@_05MJALLADF@08001?$AA@ 004c4588     client.obj
 0002:00004590       ??_C@_05OAGAMKLF@00000?$AA@ 004c4590     client.obj
 0002:00004598       ??_C@_02HDBGODGB@?2?2?$AA@ 004c4598     client.obj
 0002:0000459c       ??_C@_06CKMLAALA@?2pipe?2?$AA@ 004c459c     client.obj
 0002:000045a4       ??_C@_01LFCBOECM@?4?$AA@   004c45a4     client.obj
 0002:000045a8       ??_C@_0L@MKBJOBHN@Windows_NT?$AA@ 004c45a8     client.obj
 0002:000045b8       ??_C@_02OKOOOCIH@OS?$AA@   004c45b8     client.obj
 0002:000045bc       ??_C@_0CA@ONJAFPFC@Unknown?5option?5to?5protocol?3?5?$CFs?6?$AA@ 004c45bc     client.obj
 0002:000045e4       ??_C@_06DGDLPBAN@client?$AA@ 004c45e4     client.obj
 0002:000045ec       ??_C@_04ODABKPJA@?1CN?$DN?$AA@ 004c45ec     client.obj
 0002:000045f4       ??_C@_0CP@EINHLMKL@COLLATION?5?$CFs?5is?5not?5valid?5for?5CH@ 004c45f4     client.obj
 0002:0000462c       ??_C@_0BC@BNNCKLMG@latin1_swedish_ci?$AA@ 004c462c     client.obj
 0002:00004644       ??_C@_06CDEFMFPB@latin1?$AA@ 004c4644     client.obj
 0002:0000464c       ??_C@_0N@HAKKOMP@SET?5NAMES?5?$CFs?$AA@ 004c464c     client.obj
 0002:0000465c       ??_C@_0CD@CIHNPOGB@sending?5authentication?5informati@ 004c465c     client.obj
 0002:00004688       ??_C@_0BJ@EDEHFNCE@Setting?5intital?5database?$AA@ 004c4688     client.obj
 0002:000046a8       ??_C@_0BN@NHONKCFH@sending?5password?5information?$AA@ 004c46a8     client.obj
 0002:000046cc       ??_C@_0CC@FOKDGKNL@reading?5final?5connect?5informatio@ 004c46cc     client.obj
 0002:000046f4       ??_C@_0BN@IKPBBPKC@reading?5authorization?5packet?$AA@ 004c46f4     client.obj
 0002:00004718       ??_C@_0CJ@OKBDLPBM@sending?5connection?5information?5t@ 004c4718     client.obj
 0002:0000474c       ??_C@_0CF@JIJHEKCB@reading?5initial?5communication?5pa@ 004c474c     client.obj
 0002:00004778       ??_C@_0CJ@GFOPAJCF@waiting?5for?5initial?5communicatio@ 004c4778     client.obj
 0002:000047ac       ??_C@_05OBDDCBJC@MySQL?$AA@ 004c47ac     client.obj
 0002:000047b4       ??_C@_02LOEMLMCB@my?$AA@   004c47b4     client.obj
 0002:000047b8       ??_C@_01NBENCBCI@?$CK?$AA@ 004c47b8     get_password.obj
 0002:000047bc       ??_C@_03OLJLMEOE@?$AI?5?$AI?$AA@ 004c47bc     get_password.obj
 0002:000047c0       ??_C@_0KP@MJIINCCO@The?5number?5of?5columns?5in?5the?5res@ 004c47c0     errmsg.obj
 0002:00004894       ??_C@_0DO@EFIILPCK@Statement?5closed?5indirectly?5beca@ 004c4894     errmsg.obj
 0002:000048e0       ??_C@_0DK@NDNCLJNI@Lost?5connection?5to?5MySQL?5server?5@ 004c48e0     errmsg.obj
 0002:00004928       ??_C@_0CE@HBOGEKGA@This?5feature?5is?5not?5implemented?5@ 004c4928     errmsg.obj
 0002:00004958       ??_C@_0FB@FBBFBAHN@Attempt?5to?5read?5a?5row?5while?5ther@ 004c4958     errmsg.obj
 0002:000049bc       ??_C@_0CI@HALOFLAE@Prepared?5statement?5contains?5no?5m@ 004c49bc     errmsg.obj
 0002:000049ec       ??_C@_0CP@CONJDJBD@Attempt?5to?5read?5column?5without?5p@ 004c49ec     errmsg.obj
 0002:00004a24       ??_C@_0DG@NCJJHECB@Row?5retrieval?5was?5canceled?5by?5my@ 004c4a24     errmsg.obj
 0002:00004a68       ??_C@_0GH@LCEGFGKM@Connection?5using?5old?5?$CIpre?94?41?41?$CJ@ 004c4a68     errmsg.obj
 0002:00004ae4       ??_C@_0BK@JMIMHFDF@Invalid?5connection?5handle?$AA@ 004c4ae4     errmsg.obj
 0002:00004b04       ??_C@_0BK@GLFMEDLO@Wrong?5or?5unknown?5protocol?$AA@ 004c4b04     errmsg.obj
 0002:00004b28       ??_C@_0EE@IPCCLOKB@Can?8t?5open?5shared?5memory?$DL?5cannot@ 004c4b28     errmsg.obj
 0002:00004b7c       ??_C@_0DG@KGBHPOJD@Can?8t?5open?5shared?5memory?$DL?5no?5ans@ 004c4b7c     errmsg.obj
 0002:00004bc0       ??_C@_0EB@MDFKCBGN@Can?8t?5open?5shared?5memory?$DL?5client@ 004c4bc0     errmsg.obj
 0002:00004c10       ??_C@_0EN@FCGLLCJK@Can?8t?5open?5shared?5memory?$DL?5client@ 004c4c10     errmsg.obj
 0002:00004c70       ??_C@_0EH@LNAOKCEE@Can?8t?5open?5shared?5memory?$DL?5client@ 004c4c70     errmsg.obj
 0002:00004cc8       ??_C@_0EN@PMIKFHIB@Can?8t?5open?5shared?5memory?$DL?5server@ 004c4cc8     errmsg.obj
 0002:00004d28       ??_C@_0EH@KCLOIILK@Can?8t?5open?5shared?5memory?$DL?5server@ 004c4d28     errmsg.obj
 0002:00004d80       ??_C@_0EF@KIGDFHBB@Can?8t?5open?5shared?5memory?$DL?5no?5ans@ 004c4d80     errmsg.obj
 0002:00004dd8       ??_C@_0EG@BEPMLGLN@Can?8t?5open?5shared?5memory?$DL?5client@ 004c4dd8     errmsg.obj
 0002:00004e2c       ??_C@_0BH@OHMIMHCN@Shared?5memory?3?5?$CF?9?4100s?$AA@ 004c4e2c     errmsg.obj
 0002:00004e48       ??_C@_0DD@HBOCKDGH@Using?5unsupported?5buffer?5type?3?5?$CF@ 004c4e48     errmsg.obj
 0002:00004e88       ??_C@_0EK@GGAINION@Can?8t?5send?5long?5data?5for?5non?9str@ 004c4e88     errmsg.obj
 0002:00004ee0       ??_C@_0BJ@LEKCEENG@Invalid?5parameter?5number?$AA@ 004c4ee0     errmsg.obj
 0002:00004f00       ??_C@_0CF@OAFCOHEP@No?5parameters?5exist?5in?5the?5state@ 004c4f00     errmsg.obj
 0002:00004f2c       ??_C@_0P@KJHDOAKM@Data?5truncated?$AA@ 004c4f2c     errmsg.obj
 0002:00004f40       ??_C@_0DG@PGNJOEPP@No?5data?5supplied?5for?5parameters?5@ 004c4f40     errmsg.obj
 0002:00004f80       ??_C@_0BH@OCBFPEOC@Statement?5not?5prepared?$AA@ 004c4f80     errmsg.obj
 0002:00004f9c       ??_C@_0BM@EEGCMMPG@Invalid?5use?5of?5null?5pointer?$AA@ 004c4f9c     errmsg.obj
 0002:00004fc0       ??_C@_0FE@HLHPGJMI@This?5client?5library?5is?5licensed?5@ 004c4fc0     errmsg.obj
 0002:00005024       ??_C@_0BB@DAKKIOKN@Malformed?5packet?$AA@ 004c5024     errmsg.obj
 0002:00005038       ??_C@_0BF@GNKPEKCC@SSL?5connection?5error?$AA@ 004c5038     errmsg.obj
 0002:00005054       ??_C@_0BM@DBHHCLGE@Error?5connecting?5to?5master?3?$AA@ 004c5054     errmsg.obj
 0002:00005078       ??_C@_0BL@NMFPGPDF@Error?5connecting?5to?5slave?3?$AA@ 004c5078     errmsg.obj
 0002:00005098       ??_C@_0BL@BDOEBOAG@Error?5on?5SHOW?5SLAVE?5HOSTS?3?$AA@ 004c5098     errmsg.obj
 0002:000050b8       ??_C@_0BM@KEKCHGPI@Error?5on?5SHOW?5SLAVE?5STATUS?3?$AA@ 004c50b8     errmsg.obj
 0002:000050dc       ??_C@_0BA@JILIEPGI@Embedded?5server?$AA@ 004c50dc     errmsg.obj
 0002:000050f0       ??_C@_0DC@PLGHDHHE@Got?5packet?5bigger?5than?5?8max_allo@ 004c50f0     errmsg.obj
 0002:0000512c       ??_C@_0DG@MMIKLOLE@Can?8t?5initialize?5character?5set?5?$CF@ 004c512c     errmsg.obj
 0002:00005170       ??_C@_0EC@JBHOMNCI@Can?8t?5set?5state?5of?5named?5pipe?5to@ 004c5170     errmsg.obj
 0002:000051c0       ??_C@_0DK@DGFLNGLM@Can?8t?5open?5named?5pipe?5to?5host?3?5?$CF@ 004c51c0     errmsg.obj
 0002:00005208       ??_C@_0DO@MCIKAJJD@Can?8t?5wait?5for?5named?5pipe?5to?5hos@ 004c5208     errmsg.obj
 0002:00005254       ??_C@_0BD@MONBAMLI@Named?5pipe?3?5?$CF?9?432s?$AA@ 004c5254     errmsg.obj
 0002:0000526c       ??_C@_0DF@GGAOFKDM@Commands?5out?5of?5sync?$DL?5you?5can?8t?5@ 004c526c     errmsg.obj
 0002:000052ac       ??_C@_0CN@MCPHLMHK@Lost?5connection?5to?5MySQL?5server?5@ 004c52ac     errmsg.obj
 0002:000052e4       ??_C@_0BK@OPFAEJOB@Error?5in?5server?5handshake?$AA@ 004c52e4     errmsg.obj
 0002:00005304       ??_C@_0BD@JHCOEEJ@?$CF?9?4100s?5via?5TCP?1IP?$AA@ 004c5304     errmsg.obj
 0002:0000531c       ??_C@_0BK@OAJGGGIC@Localhost?5via?5UNIX?5socket?$AA@ 004c531c     errmsg.obj
 0002:0000533c       ??_C@_0BA@OBGODAJN@Wrong?5host?5info?$AA@ 004c533c     errmsg.obj
 0002:00005350       ??_C@_0BP@LPGLBKOF@MySQL?5client?5ran?5out?5of?5memory?$AA@ 004c5350     errmsg.obj
 0002:00005378       ??_C@_0DM@BHKAADIN@Protocol?5mismatch?$DL?5server?5versio@ 004c5378     errmsg.obj
 0002:000053c0       ??_C@_0BL@GGNHAOJF@MySQL?5server?5has?5gone?5away?$AA@ 004c53c0     errmsg.obj
 0002:000053e0       ??_C@_0CJ@MGNDPAC@Unknown?5MySQL?5server?5host?5?8?$CF?9?410@ 004c53e0     errmsg.obj
 0002:00005414       ??_C@_0CA@NNJEMGCD@Can?8t?5create?5TCP?1IP?5socket?5?$CI?$CFd?$CJ?$AA@ 004c5414     errmsg.obj
 0002:0000543c       ??_C@_0DA@DGOLCCI@Can?8t?5connect?5to?5MySQL?5server?5on@ 004c543c     errmsg.obj
 0002:00005478       ??_C@_0EC@FCNCJBBO@Can?8t?5connect?5to?5local?5MySQL?5ser@ 004c5478     errmsg.obj
 0002:000054c8       ??_C@_0BO@EGFBLII@Can?8t?5create?5UNIX?5socket?5?$CI?$CFd?$CJ?$AA@ 004c54c8     errmsg.obj
 0002:000054ec       ??_C@_0BE@OOMFAHBF@Unknown?5MySQL?5error?$AA@ 004c54ec     errmsg.obj
 0002:00005504       ??_C@_04LHHHFLPP@utf8?$AA@ 004c5504     mysys:charset.obj
 0002:0000550c       ??_C@_04JKLLLNMI@ucs2?$AA@ 004c550c     mysys:charset.obj
 0002:00005514       ??_C@_09NKDKDEJM@charsets?1?$AA@ 004c5514     mysys:charset.obj
 0002:00005520       ??_C@_0CJ@GPDDGFPJ@c?3?1Program?5Files?1MySQL?1MySQL?5Ser@ 004c5520     mysys:charset.obj
 0002:0000554c       ??_C@_05KGKMKOAF@share?$AA@ 004c554c     mysys:charset.obj
 0002:00005554       ??_C@_09NJBIMGLE@Index?4xml?$AA@ 004c5554     mysys:charset.obj
 0002:00005560       ??_C@_01OGPIMHDM@?$DP?$AA@ 004c5560     mysys:charset.obj
 0002:00005564       ??_C@_04GAOAGNCM@?4xml?$AA@ 004c5564     mysys:charset.obj
 0002:0000556c       ??_C@_05HPPBHLPE@cp932?$AA@ 004c556c     mysys:charset.obj
 0002:00005574       ??_C@_02GFBACKGC@cp?$AA@   004c5574     mysys:charset.obj
 0002:00005578       ??_C@_04KOCLJNO@LPT9?$AA@  004c5578     mysys:my_access.obj
 0002:00005580       ??_C@_04BDPJIIJP@LPT8?$AA@ 004c5580     mysys:my_access.obj
 0002:00005588       ??_C@_04JEGBJEFA@LPT7?$AA@ 004c5588     mysys:my_access.obj
 0002:00005590       ??_C@_04INHKKFBB@LPT6?$AA@ 004c5590     mysys:my_access.obj
 0002:00005598       ??_C@_04KGFHPGNC@LPT5?$AA@ 004c5598     mysys:my_access.obj
 0002:000055a0       ??_C@_04LPEMMHJD@LPT4?$AA@ 004c55a0     mysys:my_access.obj
 0002:000055a8       ??_C@_04PAANFBFE@LPT3?$AA@ 004c55a8     mysys:my_access.obj
 0002:000055b0       ??_C@_04OJBGGABF@LPT2?$AA@ 004c55b0     mysys:my_access.obj
 0002:000055b8       ??_C@_04MCDLDDNG@LPT1?$AA@ 004c55b8     mysys:my_access.obj
 0002:000055c0       ??_C@_04JDDPPBDJ@COM9?$AA@ 004c55c0     mysys:my_access.obj
 0002:000055c8       ??_C@_04IKCEMAHI@COM8?$AA@ 004c55c8     mysys:my_access.obj
 0002:000055d0       ??_C@_04NLMNMLH@COM7?$AA@  004c55d0     mysys:my_access.obj
 0002:000055d8       ??_C@_04BEKHONPG@COM6?$AA@ 004c55d8     mysys:my_access.obj
 0002:000055e0       ??_C@_04DPIKLODF@COM5?$AA@ 004c55e0     mysys:my_access.obj
 0002:000055e8       ??_C@_04CGJBIPHE@COM4?$AA@ 004c55e8     mysys:my_access.obj
 0002:000055f0       ??_C@_04GJNABJLD@COM3?$AA@ 004c55f0     mysys:my_access.obj
 0002:000055f8       ??_C@_04HAMLCIPC@COM2?$AA@ 004c55f8     mysys:my_access.obj
 0002:00005600       ??_C@_04FLOGHLDB@COM1?$AA@ 004c5600     mysys:my_access.obj
 0002:00005608       ??_C@_03JDMLODLP@NUL?$AA@  004c5608     mysys:my_access.obj
 0002:0000560c       ??_C@_03OFAGCELM@AUX?$AA@  004c560c     mysys:my_access.obj
 0002:00005610       ??_C@_03BEHELHBE@PRN?$AA@  004c5610     mysys:my_access.obj
 0002:00005614       ??_C@_03ECCGHPEG@CON?$AA@  004c5614     mysys:my_access.obj
 0002:00005618       ??_C@_06LBMPDOLO@CLOCK$?$AA@ 004c5618     mysys:my_access.obj
 0002:00005620       ??_C@_04BPFBOLGB@?4cnf?$AA@ 004c5620     mysys:default.obj
 0002:00005628       ??_C@_04PHHEBHMK@?4ini?$AA@ 004c5628     mysys:default.obj
 0002:00005644       ??_C@_0BJ@KIKAGLAC@?9?9defaults?9group?9suffix?$DN?$AA@ 004c5644     mysys:default.obj
 0002:00005660       ??_C@_0DM@LOBIDFGL@error?3?5Wrong?5?8?$CB?$CFs?8?5directive?5in?5@ 004c5660     mysys:default.obj
 0002:0000569c       ??_C@_09FJGNFLHN@?2System32?$AA@ 004c569c     mysys:default.obj
 0002:000056a8       ??_C@_0N@MDJJJHMB@kernel32?4dll?$AA@ 004c56a8     mysys:default.obj
 0002:000056b8       ??_C@_0BL@CAKPALPI@GetSystemWindowsDirectoryA?$AA@ 004c56b8     mysys:default.obj
 0002:000056d4       ??_C@_0L@DODNGCIN@MYSQL_HOME?$AA@ 004c56d4     mysys:default.obj
 0002:000056e0       ??_C@_03GMPKIPBL@C?3?1?$AA@ 004c56e0     mysys:default.obj
 0002:000056e8       ??_C@_0EM@DMHOPFHM@error?3?5Found?5option?5without?5prec@ 004c56e8     mysys:default.obj
 0002:00005734       ??_C@_0DN@MBLPBICC@error?3?5Wrong?5group?5definition?5in@ 004c5734     mysys:default.obj
 0002:00005778       ??_C@_0GG@GBLJMDFL@Warning?3?5skipping?5?8?$CFs?8?5directive@ 004c5778     mysys:default.obj
 0002:000057e0       ??_C@_01CLKCMJKC@?5?$AA@   004c57e0     mysys:default.obj
 0002:000057e4       ??_C@_0DF@OKDAKIKM@Internal?5error?5initializing?5defa@ 004c57e4     mysys:default.obj
 0002:00005820       ??_C@_0EH@NKGMIPDP@?6Default?5options?5are?5read?5from?5t@ 004c5820     mysys:default.obj
 0002:00005868       ??_C@_0BFH@LPFPCOIJ@?6The?5following?5options?5may?5be?5gi@ 004c5868     mysys:default.obj
 0002:000059c0       ??_C@_0BP@MNBILDMG@The?5following?5groups?5are?5read?3?$AA@ 004c59c0     mysys:default.obj
 0002:000059e0       ??_C@_0DD@BMIFLCG@Fatal?5error?5in?5defaults?5handling@ 004c59e0     mysys:default.obj
 0002:00005a14       ??_C@_0CL@DPGKONAJ@Could?5not?5open?5required?5defaults@ 004c5a14     mysys:default.obj
 0002:00005a40       ??_C@_0BD@GMCINPDE@MYSQL_GROUP_SUFFIX?$AA@ 004c5a40     mysys:default.obj
 0002:00005a54       ??_C@_03IKGEINEE@?$CFs?5?$AA@ 004c5a54     mysys:default.obj
 0002:00005a58       ??_C@_0DK@MHCNAEBD@?$CFs?5would?5have?5been?5started?5with?5@ 004c5a58     mysys:default.obj
 0002:00005a94       ??_C@_0BB@BKNLJB@?9?9print?9defaults?$AA@ 004c5a94     mysys:default.obj
 0002:00005aa8       ??_C@_08LMJEPNLL@defaults?$AA@ 004c5aa8     mysys:default.obj
 0002:00005ab4       ??_C@_02DJGKEECL@?4?4?$AA@ 004c5ab4     mysys:mf_loadpath.obj
 0002:00005ab8       ??_C@_07CCIHIKOK@no_name?$AA@ 004c5ab8     mysys:my_thr_init.obj
 0002:00005ac0       ??_C@_0CE@CLEEBIJB@Can?8t?5initialize?5threads?3?5error?5@ 004c5ac0     mysys:my_thr_init.obj
 0002:00005ae4       ??_C@_0BL@LPICHLF@01230120022455012623010202?$AA@ 004c5ae4     mysys:my_static.obj
 0002:00005b00       ??_C@_0BA@KPMGBOMG@?$CFs?4?$CF08X?4deleted?$AA@ 004c5b00     mysys:my_delete.obj
 0002:00005b10       ??_C@_0P@NEKPODBM@SOFTWARE?2MySQL?$AA@ 004c5b10     mysys:my_init.obj
 0002:00005b20       ??_C@_0L@LKJCDLMN@HAVE_TCPIP?$AA@ 004c5b20     mysys:my_init.obj
 0002:00005b2c       ??_C@_0DF@KNCKAEOE@SYSTEM?2CurrentControlSet?2Service@ 004c5b2c     mysys:my_init.obj
 0002:00005b64       ??_C@_0DG@NPLBFMIJ@SYSTEM?2CurrentControlSet?2Service@ 004c5b64     mysys:my_init.obj
 0002:00005b9c       ??_C@_0DD@IKBMIFKO@SYSTEM?2CurrentControlSet?2Service@ 004c5b9c     mysys:my_init.obj
 0002:00005bd0       ??_C@_09KHPDOLMK@UMASK_DIR?$AA@ 004c5bd0     mysys:my_init.obj
 0002:00005bdc       ??_C@_05OMMCGCJP@UMASK?$AA@ 004c5bdc     mysys:my_init.obj
 0002:00005be4       ??_C@_04GHGFPGNC@HOME?$AA@ 004c5be4     mysys:my_init.obj
 0002:00005bec       ??_C@_05HBBNPFP@loose?$AA@ 004c5bec     mysys:my_getopt.obj
 0002:00005bf4       ??_C@_07MEIENILC@maximum?$AA@ 004c5bf4     mysys:my_getopt.obj
 0002:00005bfc       ??_C@_06OFNJOBDK@enable?$AA@ 004c5bfc     mysys:my_getopt.obj
 0002:00005c04       ??_C@_07DBNODEFN@disable?$AA@ 004c5c04     mysys:my_getopt.obj
 0002:00005c0c       ??_C@_04DLBGLKG@skip?$AA@  004c5c0c     mysys:my_getopt.obj
 0002:00005c2c       ??_C@_02DKCKIIND@?$CFs?$AA@ 004c5c2c     mysys:my_getopt.obj
 0002:00005c30       ??_C@_06EILBFPFN@Info?3?5?$AA@ 004c5c30     mysys:my_getopt.obj
 0002:00005c38       ??_C@_09CKCJCCOK@Warning?3?5?$AA@ 004c5c38     mysys:my_getopt.obj
 0002:00005c44       ??_C@_0DJ@LCKGBNKC@Unknown?5suffix?5?8?$CFc?8?5used?5for?5var@ 004c5c44     mysys:my_getopt.obj
 0002:00005c80       ??_C@_0BO@MNLPLDPE@Incorrect?5integer?5value?3?5?8?$CFs?8?$AA@ 004c5c80     mysys:my_getopt.obj
 0002:00005ca0       ??_C@_0CM@CINNIGFM@option?5?8?$CFs?8?3?5signed?5value?5?$CFs?5adj@ 004c5ca0     mysys:my_getopt.obj
 0002:00005ccc       ??_C@_0CO@JEKLPIGP@option?5?8?$CFs?8?3?5unsigned?5value?5?$CFs?5a@ 004c5ccc     mysys:my_getopt.obj
 0002:00005d00       __real@0000000000000000    004c5d00     mysys:my_getopt.obj
 0002:00005d08       ??_C@_0DC@CLHAAIAH@?$CFs?3?5ERROR?3?5Invalid?5decimal?5value@ 004c5d08     mysys:my_getopt.obj
 0002:00005d3c       ??_C@_0L@PIHEMIFO@?$CFs?$DNname?$CFs?5?$AA@ 004c5d3c     mysys:my_getopt.obj
 0002:00005d48       ??_C@_07JMJBGKBC@?$CFs?$DN?$CD?$CFs?5?$AA@ 004c5d48     mysys:my_getopt.obj
 0002:00005d50       ??_C@_04GIEADKIK@?9?9?$CFs?$AA@ 004c5d50     mysys:my_getopt.obj
 0002:00005d58       ??_C@_07NACDLBD@?5?5?9?$CFc?$CFs?$AA@ 004c5d58     mysys:my_getopt.obj
 0002:00005d60       ??_C@_02KNHHEEKP@?5?5?$AA@ 004c5d60     mysys:my_getopt.obj
 0002:00005d64       ??_C@_02KEGNLNML@?0?5?$AA@ 004c5d64     mysys:my_getopt.obj
 0002:00005d68       ??_C@_0M@EPOBBBBF@?$CIDisabled?$CJ?6?$AA@ 004c5d68     mysys:my_getopt.obj
 0002:00005d74       ??_C@_03POCAEKMA@?$CFg?6?$AA@ 004c5d74     mysys:my_getopt.obj
 0002:00005d78       ??_C@_04OJNJKCBM@?$CFlu?6?$AA@ 004c5d78     mysys:my_getopt.obj
 0002:00005d80       ??_C@_04PEDNGLFL@?$CFld?6?$AA@ 004c5d80     mysys:my_getopt.obj
 0002:00005d88       ??_C@_05MAJJAKPI@FALSE?$AA@ 004c5d88     mysys:my_getopt.obj
 0002:00005d90       ??_C@_04HCDDPBNL@TRUE?$AA@ 004c5d90     mysys:my_getopt.obj
 0002:00005d98       ??_C@_03CGNBMCEI@?$CFs?0?$AA@ 004c5d98     mysys:my_getopt.obj
 0002:00005d9c       ??_C@_0BD@IAAJELIC@?$CINo?5default?5value?$CJ?$AA@ 004c5d9c     mysys:my_getopt.obj
 0002:00005db0       ??_C@_0EB@DLNDDEIC@?9?9?9?9?9?9?9?9?9?9?9?9?9?9?9?9?9?9?9?9?9?9?9?9?9?9?9?9?9?9?9?9@ 004c5db0     mysys:my_getopt.obj
 0002:00005df8       ??_C@_0EB@MLHGNKOO@and?5boolean?5options?5?$HLFALSE?$HMTRUE?$HN@ 004c5df8     mysys:my_getopt.obj
 0002:00005e3c       ??_C@_0CE@PGFPJDHK@?6Variables?5?$CI?9?9variable?9name?$DNvalu@ 004c5e3c     mysys:my_getopt.obj
 0002:00005e60       ??_C@_0CH@FPNHAJDD@?$CFs?3?5option?5?8?9?9?$CFs?8?5requires?5an?5ar@ 004c5e60     mysys:my_getopt.obj
 0002:00005e88       ??_C@_0CK@KELFDMIH@?$CFs?3?5option?5?8?9?9?$CFs?8?5cannot?5take?5an@ 004c5e88     mysys:my_getopt.obj
 0002:00005eb4       ??_C@_0CI@IFAFNNJB@?$CFs?3?5option?5?8?$CFs?8?5cannot?5take?5an?5a@ 004c5eb4     mysys:my_getopt.obj
 0002:00005edc       ??_C@_0CF@LIKIEIBC@?$CFs?3?5ambiguous?5option?5?8?9?9?$CFs?8?5?$CI?$CFs?0@ 004c5edc     mysys:my_getopt.obj
 0002:00005f04       ??_C@_0CH@NLLNKKKI@?$CFs?3?5variable?5prefix?5?8?$CFs?8?5is?5not?5@ 004c5f04     mysys:my_getopt.obj
 0002:00005f2c       ??_C@_0CJ@FNGIKGPP@?$CFs?3?5ambiguous?5option?5?8?9?9?$CFs?9?$CFs?8?5?$CI@ 004c5f2c     mysys:my_getopt.obj
 0002:00005f58       ??_C@_0CF@MFEIKBHA@?$CFs?3?5Option?5?8?9O?8?5requires?5an?5argu@ 004c5f58     mysys:my_getopt.obj
 0002:00005f80       ??_C@_0BJ@PLKIKLOO@?$CFs?3?5unknown?5option?5?8?9?$CFc?8?$AA@ 004c5f80     mysys:my_getopt.obj
 0002:00005f9c       ??_C@_0CL@CIFFNEPP@?$CFs?3?5Error?5while?5setting?5value?5?8?$CF@ 004c5f9c     mysys:my_getopt.obj
 0002:00005fc8       ??_C@_0CG@OPCNLHEP@?$CFs?3?5option?5?8?9?$CFc?8?5requires?5an?5arg@ 004c5fc8     mysys:my_getopt.obj
 0002:00005ff0       ??_C@_0CP@OAGPFOL@?$CFs?3?5ERROR?3?5Option?5?8?9?$CFc?8?5used?0?5bu@ 004c5ff0     mysys:my_getopt.obj
 0002:00006020       ??_C@_0DF@NCABEMAI@?$CFs?3?5ignoring?5option?5?8?9?9?$CFs?8?5due?5t@ 004c6020     mysys:my_getopt.obj
 0002:00006058       ??_C@_05LAPONLG@false?$AA@ 004c6058     mysys:my_getopt.obj
 0002:00006060       ??_C@_04LOAJBDKD@true?$AA@ 004c6060     mysys:my_getopt.obj
 0002:00006068       ??_C@_0CL@BLOGDLDC@?$CFs?3?5?$CFs?3?5Option?5?8?$CFs?8?5used?0?5but?5is@ 004c6068     mysys:my_getopt.obj
 0002:00006094       ??_C@_07KCOHIFOP@WARNING?$AA@ 004c6094     mysys:my_getopt.obj
 0002:0000609c       ??_C@_0BK@HIDGBPPN@?$CFs?3?5unknown?5option?5?8?9?9?$CFs?8?$AA@ 004c609c     mysys:my_getopt.obj
 0002:000060b8       ??_C@_0BK@JFALHNEE@?$CFs?3?5unknown?5variable?5?8?$CFs?8?$AA@ 004c60b8     mysys:my_getopt.obj
 0002:000060d4       ??_C@_01HIHLOKLC@1?$AA@    004c60d4     mysys:my_getopt.obj
 0002:000060d8       ??_C@_0DB@OBCAMIPA@?$CFs?3?5Option?5?8?9?9set?9variable?8?5requ@ 004c60d8     mysys:my_getopt.obj
 0002:00006110       ??_C@_0EO@EBDGGIGH@?$CFs?3?5Option?5?8?9?9set?9variable?8?5is?5d@ 004c6110     mysys:my_getopt.obj
 0002:00006160       ??_C@_0O@LAIDGFMB@?9set?9variable?$AA@ 004c6160     mysys:my_getopt.obj
 0002:00006170       ??_C@_0EC@ICAHOJIG@?$CFs?3?5Option?5?8?9O?8?5is?5deprecated?4?5U@ 004c6170     mysys:my_getopt.obj
 0002:000061b4       ??_C@_0BB@BIKLJNJD@Unknown?5error?5?$CFd?$AA@ 004c61b4     mysys:my_error.obj
 0002:000061c8       _sha_const_key             004c61c8     mysys:sha1.obj
 0002:000061f0       ??_C@_05FGCMFDGF@?0?8?$CFs?8?$AA@ 004c61f0     mysys:typelib.obj
 0002:000061f8       ??_C@_0BH@HMCJGOJH@Alternatives?5are?3?5?8?$CFs?8?$AA@ 004c61f8     mysys:typelib.obj
 0002:00006210       ??_C@_0BK@GLIPEDIK@Unknown?5option?5to?5?$CFs?3?5?$CFs?6?$AA@ 004c6210     mysys:typelib.obj
 0002:0000622c       ??_C@_0BH@NDCEODGI@No?5option?5given?5to?5?$CFs?6?$AA@ 004c622c     mysys:typelib.obj
 0002:00006244       ??_C@_01KICIPPFI@?2?$AA@   004c6244     mysys:my_getwd.obj
 0002:00006248       ??_C@_08KKHFAPMN@UNOPENED?$AA@ 004c6248     mysys:my_div.obj
 0002:00006254       ??_C@_07NFANNNEC@UNKNOWN?$AA@ 004c6254     mysys:my_div.obj
 0002:0000625c       ??_C@_0CG@OCCIMCJO@File?5?8?$CFs?8?5?$CIfileno?3?5?$CFd?$CJ?5was?5not?5c@ 004c625c     mysys:errors.obj
 0002:00006284       ??_C@_0CC@POIIBGBO@File?5?8?$CFs?8?5not?5found?5?$CIErrcode?3?5?$CFd@ 004c6284     mysys:errors.obj
 0002:000062a8       ??_C@_0FB@HBKGDBGI@Collation?5?8?$CFs?8?5is?5not?5a?5compiled@ 004c62a8     mysys:errors.obj
 0002:000062fc       ??_C@_0CL@IPPKDKJC@Can?8t?5sync?5file?5?8?$CFs?8?5to?5disk?5?$CIEr@ 004c62fc     mysys:errors.obj
 0002:00006328       ??_C@_0CH@DMNLJIAN@Error?5on?5realpath?$CI?$CJ?5on?5?8?$CFs?8?5?$CIErr@ 004c6328     mysys:errors.obj
 0002:00006350       ??_C@_0DG@MPBGHFJG@Can?8t?5create?5symlink?5?8?$CFs?8?5pointi@ 004c6350     mysys:errors.obj
 0002:00006388       ??_C@_0CN@FDDHNKAL@Can?8t?5read?5value?5for?5symlink?5?8?$CFs@ 004c6388     mysys:errors.obj
 0002:000063b8       ??_C@_0DG@HFJCEGGP@Out?5of?5resources?5when?5opening?5fi@ 004c63b8     mysys:errors.obj
 0002:000063f0       ??_C@_0FJ@LJEFGFHC@Character?5set?5?8?$CFs?8?5is?5not?5a?5comp@ 004c63f0     mysys:errors.obj
 0002:0000644c       ??_C@_0CK@KAOBDLLK@Can?8t?5create?5directory?5?8?$CFs?8?5?$CIErr@ 004c644c     mysys:errors.obj
 0002:00006478       ??_C@_0JL@NKJOFGOC@Disk?5is?5full?5writing?5?8?$CFs?8?5?$CIErrco@ 004c6478     mysys:errors.obj
 0002:00006514       ??_C@_0CP@OFJOGNNM@Warning?3?5?$CFd?5files?5and?5?$CFd?5streams@ 004c6514     mysys:errors.obj
 0002:00006544       ??_C@_0BL@KPAFHPFA@Warning?3?5?8?$CFs?8?5had?5?$CFd?5links?$AA@ 004c6544     mysys:errors.obj
 0002:00006560       ??_C@_0CH@HKPCIIFI@Can?8t?5change?5dir?5to?5?8?$CFs?8?5?$CIErrcod@ 004c6560     mysys:errors.obj
 0002:00006588       ??_C@_0CJ@HHIGEGH@Can?8t?5get?5working?5dirctory?5?$CIErrc@ 004c6588     mysys:errors.obj
 0002:000065b4       ??_C@_0CM@IDOLEFDO@Can?8t?5open?5stream?5from?5handle?5?$CIE@ 004c65b4     mysys:errors.obj
 0002:000065e0       ??_C@_0CI@JHPDBJAP@Can?8t?5change?5size?5of?5file?5?$CIErrco@ 004c65e0     mysys:errors.obj
 0002:00006608       ??_C@_0CF@EBINEGNH@Can?8t?5get?5stat?5of?5?8?$CFs?8?5?$CIErrcode?3@ 004c6608     mysys:errors.obj
 0002:00006630       ??_C@_0CF@DKKFLCIK@Can?8t?5read?5dir?5of?5?8?$CFs?8?5?$CIErrcode?3@ 004c6630     mysys:errors.obj
 0002:00006658       ??_C@_0CA@NMCGOICJ@Can?8t?5unlock?5file?5?$CIErrcode?3?5?$CFd?$CJ?$AA@ 004c6658     mysys:errors.obj
 0002:00006678       ??_C@_0BO@FABCFMMA@Can?8t?5lock?5file?5?$CIErrcode?3?5?$CFd?$CJ?$AA@ 004c6678     mysys:errors.obj
 0002:00006698       ??_C@_0DK@OPEJLFLC@Unexpected?5eof?5found?5when?5readin@ 004c6698     mysys:errors.obj
 0002:000066d4       ??_C@_0CO@NDIKPEAP@Error?5on?5rename?5of?5?8?$CFs?8?5to?5?8?$CFs?8?5@ 004c66d4     mysys:errors.obj
 0002:00006704       ??_C@_0CG@LPKMPJNP@Error?5on?5delete?5of?5?8?$CFs?8?5?$CIErrcode@ 004c6704     mysys:errors.obj
 0002:0000672c       ??_C@_0CA@NLHLMAKD@Out?5of?5memory?5?$CINeeded?5?$CFu?5bytes?$CJ?$AA@ 004c672c     mysys:errors.obj
 0002:0000674c       ??_C@_0CF@BEDBELLH@Error?5on?5close?5of?5?8?$CFs?8?5?$CIErrcode?3@ 004c674c     mysys:errors.obj
 0002:00006774       ??_C@_0CG@CGPFOMKP@Error?5writing?5file?5?8?$CFs?8?5?$CIErrcode@ 004c6774     mysys:errors.obj
 0002:0000679c       ??_C@_0CG@NONCHHAM@Error?5reading?5file?5?8?$CFs?8?5?$CIErrcode@ 004c679c     mysys:errors.obj
 0002:000067c4       ??_C@_0CO@OHAAEPNE@Can?8t?5create?1write?5to?5file?5?8?$CFs?8?5@ 004c67c4     mysys:errors.obj
 0002:000067f4       ??_C@_0CP@BPNOAMDC@Retry?5in?5?$CFd?5secs?4?5Message?5reprin@ 004c67f4     mysys:errors.obj
 0002:00006824       ??_C@_04LFNFNAMA@?4sym?$AA@ 004c6824     mysys:mf_pack.obj
 0002:0000682c       ??_C@_02LMMGGCAJ@?3?5?$AA@ 004c682c     mysys:my_messnc.obj
 0002:00006834       ??_C@_0L@BBMDDOEP@latin1_bin?$AA@ 004c6834     strings:ctype-latin1.obj
 0002:00006840       ??_C@_0BC@JEMPBIB@latin1_german2_ci?$AA@ 004c6840     strings:ctype-latin1.obj
 0002:00006854       ??_C@_06OJHGLDPL@?$CInull?$CJ?$AA@ 004c6854     strings:my_vsnprintf.obj
 0002:0000685c       ??_C@_06FNFBAEBE@binary?$AA@ 004c685c     strings:ctype-bin.obj
 0002:00006864       ??_C@_0CD@LKLOKDOO@charsets?1charset?1collation?1rules@ 004c6864     strings:ctype.obj
 0002:00006888       ??_C@_0CD@PFPPDFCJ@charsets?1charset?1collation?1rules@ 004c6888     strings:ctype.obj
 0002:000068ac       ??_C@_0CD@NONCGGOK@charsets?1charset?1collation?1rules@ 004c68ac     strings:ctype.obj
 0002:000068d0       ??_C@_0CH@EHCCKNPN@charsets?1charset?1collation?1rules@ 004c68d0     strings:ctype.obj
 0002:000068f8       ??_C@_0BP@MDNMPBHP@charsets?1charset?1collation?1map?$AA@ 004c68f8     strings:ctype.obj
 0002:00006918       ??_C@_0CA@HCJLGNLH@charsets?1charset?1collation?1flag?$AA@ 004c6918     strings:ctype.obj
 0002:00006938       ??_C@_0CB@IEPLPKEB@charsets?1charset?1collation?1order@ 004c6938     strings:ctype.obj
 0002:0000695c       ??_C@_0BO@PKAEPDFI@charsets?1charset?1collation?1id?$AA@ 004c695c     strings:ctype.obj
 0002:0000697c       ??_C@_0CA@ILKNGFEN@charsets?1charset?1collation?1name?$AA@ 004c697c     strings:ctype.obj
 0002:0000699c       ??_C@_0BL@JFMDNPGN@charsets?1charset?1collation?$AA@ 004c699c     strings:ctype.obj
 0002:000069b8       ??_C@_0BN@PEPOLNOE@charsets?1charset?1unicode?1map?$AA@ 004c69b8     strings:ctype.obj
 0002:000069d8       ??_C@_0BJ@KHPKNFM@charsets?1charset?1unicode?$AA@ 004c69d8     strings:ctype.obj
 0002:000069f4       ??_C@_0BL@ELLNOHCD@charsets?1charset?1lower?1map?$AA@ 004c69f4     strings:ctype.obj
 0002:00006a10       ??_C@_0BH@HBDHNKIJ@charsets?1charset?1lower?$AA@ 004c6a10     strings:ctype.obj
 0002:00006a28       ??_C@_0BL@OJLKMJLI@charsets?1charset?1upper?1map?$AA@ 004c6a28     strings:ctype.obj
 0002:00006a44       ??_C@_0BH@CKIJLBDA@charsets?1charset?1upper?$AA@ 004c6a44     strings:ctype.obj
 0002:00006a5c       ??_C@_0BL@KKJMPDHK@charsets?1charset?1ctype?1map?$AA@ 004c6a5c     strings:ctype.obj
 0002:00006a78       ??_C@_0BH@GIOAFMPB@charsets?1charset?1ctype?$AA@ 004c6a78     strings:ctype.obj
 0002:00006a90       ??_C@_0BH@CENNAKLG@charsets?1charset?1alias?$AA@ 004c6a90     strings:ctype.obj
 0002:00006aa8       ??_C@_0BN@LLOCCHFI@charsets?1charset?1description?$AA@ 004c6aa8     strings:ctype.obj
 0002:00006ac8       ??_C@_0BI@ICKMEODO@charsets?1charset?1family?$AA@ 004c6ac8     strings:ctype.obj
 0002:00006ae0       ??_C@_0BG@LDPKBCKB@charsets?1charset?1name?$AA@ 004c6ae0     strings:ctype.obj
 0002:00006af8       ??_C@_0BL@LNCPEELC@charsets?1charset?1binary?9id?$AA@ 004c6af8     strings:ctype.obj
 0002:00006b14       ??_C@_0BM@NDJFGPHG@charsets?1charset?1primary?9id?$AA@ 004c6b14     strings:ctype.obj
 0002:00006b30       ??_C@_0BB@MPLJNAOI@charsets?1charset?$AA@ 004c6b30     strings:ctype.obj
 0002:00006b44       ??_C@_0BA@NFCJBDGG@charsets?1max?9id?$AA@ 004c6b44     strings:ctype.obj
 0002:00006b54       ??_C@_08PBFNHBDC@charsets?$AA@ 004c6b54     strings:ctype.obj
 0002:00006b60       ??_C@_0N@JABJMIAL@xml?1encoding?$AA@ 004c6b60     strings:ctype.obj
 0002:00006b70       ??_C@_0M@BOENADBE@xml?1version?$AA@ 004c6b70     strings:ctype.obj
 0002:00006b7c       ??_C@_03PJHHNEEI@xml?$AA@  004c6b7c     strings:ctype.obj
 0002:00006b80       ??_C@_04HHCDBDLF@?5?7?$AN?6?$AA@ 004c6b80     strings:ctype.obj
 0002:00006b88       ??_C@_06NOJLBGIH@?5?$CFs?5?$CFs?$AA@ 004c6b88     strings:ctype.obj
 0002:00006b90       ??_C@_03DKMEACPB@?$DM?$DM?$DM?$AA@ 004c6b90     strings:ctype.obj
 0002:00006b94       ??_C@_02FODMEDOG@?$DM?$DM?$AA@ 004c6b94     strings:ctype.obj
 0002:00006b98       ??_C@_01MNNFJEPP@?$DM?$AA@ 004c6b98     strings:ctype.obj
 0002:00006b9c       ??_C@_01HNPIGOCE@?$CG?$AA@ 004c6b9c     strings:ctype.obj
 0002:00006ba0       ??_C@_08DOMPDOCM@compiled?$AA@ 004c6ba0     strings:ctype.obj
 0002:00006bac       ??_C@_07CJDBHDIN@primary?$AA@ 004c6bac     strings:ctype.obj
 0002:00006bb4       ??_C@_0BC@FAACCCJD@utf8_hungarian_ci?$AA@ 004c6bb4     strings:ctype-uca.obj
 0002:00006bc8       ??_C@_0BC@MMMDBEJH@utf8_esperanto_ci?$AA@ 004c6bc8     strings:ctype-uca.obj
 0002:00006bdc       ??_C@_0BA@POPDBMKL@utf8_persian_ci?$AA@ 004c6bdc     strings:ctype-uca.obj
 0002:00006bec       ??_C@_0O@JCIJCIKH@utf8_roman_ci?$AA@ 004c6bec     strings:ctype-uca.obj
 0002:00006bfc       ??_C@_0BB@DMDMGDOP@utf8_spanish2_ci?$AA@ 004c6bfc     strings:ctype-uca.obj
 0002:00006c10       ??_C@_0P@NIJBPDBH@utf8_slovak_ci?$AA@ 004c6c10     strings:ctype-uca.obj
 0002:00006c20       ??_C@_0BD@MHPAIICH@utf8_lithuanian_ci?$AA@ 004c6c20     strings:ctype-uca.obj
 0002:00006c34       ??_C@_0P@LICOLLCI@utf8_danish_ci?$AA@ 004c6c34     strings:ctype-uca.obj
 0002:00006c44       ??_C@_0O@OMAOFLBG@utf8_czech_ci?$AA@ 004c6c44     strings:ctype-uca.obj
 0002:00006c54       ??_C@_0BA@HIEJCGP@utf8_turkish_ci?$AA@ 004c6c54     strings:ctype-uca.obj
 0002:00006c64       ??_C@_0BA@DLMLGKMF@utf8_swedish_ci?$AA@ 004c6c64     strings:ctype-uca.obj
 0002:00006c74       ??_C@_0BA@BFDLDMHI@utf8_spanish_ci?$AA@ 004c6c74     strings:ctype-uca.obj
 0002:00006c84       ??_C@_0BB@IDIAKKIG@utf8_estonian_ci?$AA@ 004c6c84     strings:ctype-uca.obj
 0002:00006c98       ??_C@_0P@BMIMEGFF@utf8_polish_ci?$AA@ 004c6c98     strings:ctype-uca.obj
 0002:00006ca8       ??_C@_0BC@ONGHKMPJ@utf8_slovenian_ci?$AA@ 004c6ca8     strings:ctype-uca.obj
 0002:00006cbc       ??_C@_0BB@EMJFIJEJ@utf8_romanian_ci?$AA@ 004c6cbc     strings:ctype-uca.obj
 0002:00006cd0       ??_C@_0BA@GIAOJNDD@utf8_latvian_ci?$AA@ 004c6cd0     strings:ctype-uca.obj
 0002:00006ce0       ??_C@_0BC@OLHAMMMB@utf8_icelandic_ci?$AA@ 004c6ce0     strings:ctype-uca.obj
 0002:00006cf4       ??_C@_0BA@GBKHDDAB@utf8_unicode_ci?$AA@ 004c6cf4     strings:ctype-uca.obj
 0002:00006d04       ??_C@_0BC@JMLAFJDL@ucs2_hungarian_ci?$AA@ 004c6d04     strings:ctype-uca.obj
 0002:00006d18       ??_C@_0BC@HBGPDP@ucs2_esperanto_ci?$AA@ 004c6d18     strings:ctype-uca.obj
 0002:00006d2c       ??_C@_0BA@PJNOLINJ@ucs2_persian_ci?$AA@ 004c6d2c     strings:ctype-uca.obj
 0002:00006d3c       ??_C@_0O@CNOJEKEN@ucs2_roman_ci?$AA@ 004c6d3c     strings:ctype-uca.obj
 0002:00006d4c       ??_C@_0BB@ICDAFOFL@ucs2_spanish2_ci?$AA@ 004c6d4c     strings:ctype-uca.obj
 0002:00006d60       ??_C@_0P@JIPBJIBD@ucs2_slovak_ci?$AA@ 004c6d60     strings:ctype-uca.obj
 0002:00006d70       ??_C@_0BD@BPDBBBIG@ucs2_lithuanian_ci?$AA@ 004c6d70     strings:ctype-uca.obj
 0002:00006d84       ??_C@_0P@PIEONACM@ucs2_danish_ci?$AA@ 004c6d84     strings:ctype-uca.obj
 0002:00006d94       ??_C@_0O@FDGODJPM@ucs2_czech_ci?$AA@ 004c6d94     strings:ctype-uca.obj
 0002:00006da4       ??_C@_0BA@KJDGBN@ucs2_turkish_ci?$AA@ 004c6da4     strings:ctype-uca.obj
 0002:00006db4       ??_C@_0BA@DMOGMOLH@ucs2_swedish_ci?$AA@ 004c6db4     strings:ctype-uca.obj
 0002:00006dc4       ??_C@_0BA@BCBGJIAK@ucs2_spanish_ci?$AA@ 004c6dc4     strings:ctype-uca.obj
 0002:00006dd4       ??_C@_0BB@DNIMJHDC@ucs2_estonian_ci?$AA@ 004c6dd4     strings:ctype-uca.obj
 0002:00006de8       ??_C@_0P@FMOMCNFB@ucs2_polish_ci?$AA@ 004c6de8     strings:ctype-uca.obj
 0002:00006df8       ??_C@_0BC@CBNFNHFB@ucs2_slovenian_ci?$AA@ 004c6df8     strings:ctype-uca.obj
 0002:00006e0c       ??_C@_0BB@PCJJLEPN@ucs2_romanian_ci?$AA@ 004c6e0c     strings:ctype-uca.obj
 0002:00006e20       ??_C@_0BA@GPCDDJEB@ucs2_latvian_ci?$AA@ 004c6e20     strings:ctype-uca.obj
 0002:00006e30       ??_C@_0BC@CHMCLHGJ@ucs2_icelandic_ci?$AA@ 004c6e30     strings:ctype-uca.obj
 0002:00006e44       ??_C@_0BA@GGIKJHHD@ucs2_unicode_ci?$AA@ 004c6e44     strings:ctype-uca.obj
 0002:00007b10       ??_C@_0L@JHIJEIOB@?$CFs?5at?5?8?$CFs?8?$AA@ 004c7b10     strings:ctype-uca.obj
 0002:00007b1c       ??_C@_0L@BNFOJFGF@?$CG?5expected?$AA@ 004c7b1c     strings:ctype-uca.obj
 0002:00007b28       ??_C@_0BA@CIAPGHM@?$CG?5or?5?$DM?5expected?$AA@ 004c7b28     strings:ctype-uca.obj
 0002:00007b38       ??_C@_0BE@OMJLCPFJ@Should?5never?5happen?$AA@ 004c7b38     strings:ctype-uca.obj
 0002:00007b4c       ??_C@_0P@MGHCGHFF@Too?5many?5rules?$AA@ 004c7b4c     strings:ctype-uca.obj
 0002:00007b5c       ??_C@_0BD@DBLGAKEN@character?5expected?$AA@ 004c7b5c     strings:ctype-uca.obj
 0002:00007b70       ??_C@_0BC@FMLIFBCF@Unknown?5character?$AA@ 004c7b70     strings:ctype-uca.obj
 0002:00007b84       ??_C@_09LKJGLAE@cp932_bin?$AA@ 004c7b84     strings:ctype-cp932.obj
 0002:00007b90       ??_C@_0BC@CHMDDICP@cp932_japanese_ci?$AA@ 004c7b90     strings:ctype-cp932.obj
 0002:00007ba8       _log_10                    004c7ba8     strings:strtod.obj
 0002:00008550       __real@7fefffffffffffff    004c8550     strings:strtod.obj
 0002:00008558       __real@3ffcc359e067a348    004c8558     strings:strtod.obj
 0002:00008560       __real@4024000000000000    004c8560     strings:strtod.obj
 0002:00008568       __real@3ff0000000000000    004c8568     strings:strtod.obj
 0002:00008570       ??_C@_0BB@LGBJIEIE@cp1250_polish_ci?$AA@ 004c8570     strings:ctype-extra.obj
 0002:00008584       ??_C@_0BC@DDCCPNHL@latin1_spanish_ci?$AA@ 004c8584     strings:ctype-extra.obj
 0002:00008598       ??_C@_0M@DIHPIFMI@geostd8_bin?$AA@ 004c8598     strings:ctype-extra.obj
 0002:000085a4       ??_C@_0BD@IFKPCMBG@geostd8_general_ci?$AA@ 004c85a4     strings:ctype-extra.obj
 0002:000085b8       ??_C@_07GCLBCFCK@geostd8?$AA@ 004c85b8     strings:ctype-extra.obj
 0002:000085c0       ??_C@_08CBKIAJIL@swe7_bin?$AA@ 004c85c0     strings:ctype-extra.obj
 0002:000085cc       ??_C@_09KENDFOKA@cp852_bin?$AA@ 004c85cc     strings:ctype-extra.obj
 0002:000085d8       ??_C@_09OJBLPPKL@cp850_bin?$AA@ 004c85d8     strings:ctype-extra.obj
 0002:000085e4       ??_C@_0L@MHJKNNFC@latin7_bin?$AA@ 004c85e4     strings:ctype-extra.obj
 0002:000085f0       ??_C@_0L@IKFCHMFJ@latin5_bin?$AA@ 004c85f0     strings:ctype-extra.obj
 0002:000085fc       ??_C@_0L@JHFHEMOB@latin2_bin?$AA@ 004c85fc     strings:ctype-extra.obj
 0002:00008608       ??_C@_09COHLDLLI@koi8u_bin?$AA@ 004c8608     strings:ctype-extra.obj
 0002:00008614       ??_C@_09DDHOALAA@koi8r_bin?$AA@ 004c8614     strings:ctype-extra.obj
 0002:00008620       ??_C@_0M@NJOCNGMA@keybcs2_bin?$AA@ 004c8620     strings:ctype-extra.obj
 0002:0000862c       ??_C@_07KIGBPGH@hp8_bin?$AA@ 004c862c     strings:ctype-extra.obj
 0002:00008634       ??_C@_0L@INPMEGLK@hebrew_bin?$AA@ 004c8634     strings:ctype-extra.obj
 0002:00008640       ??_C@_09EFLJIAMD@greek_bin?$AA@ 004c8640     strings:ctype-extra.obj
 0002:0000864c       ??_C@_08EFBBJHIK@dec8_bin?$AA@ 004c864c     strings:ctype-extra.obj
 0002:00008658       ??_C@_09OKKAGCL@cp866_bin?$AA@ 004c8658     strings:ctype-extra.obj
 0002:00008664       ??_C@_0L@OKMJAEHC@cp1256_bin?$AA@ 004c8664     strings:ctype-extra.obj
 0002:00008670       ??_C@_0L@DMJAOHGP@cp1250_bin?$AA@ 004c8670     strings:ctype-extra.obj
 0002:0000867c       ??_C@_09BDNLCGDP@ascii_bin?$AA@ 004c867c     strings:ctype-extra.obj
 0002:00008688       ??_C@_0N@KGPIBLHK@armscii8_bin?$AA@ 004c8688     strings:ctype-extra.obj
 0002:00008698       ??_C@_0BC@BKAKKOKG@cp1257_general_ci?$AA@ 004c8698     strings:ctype-extra.obj
 0002:000086ac       ??_C@_0L@CBJFNHNH@cp1257_bin?$AA@ 004c86ac     strings:ctype-extra.obj
 0002:000086b8       ??_C@_0BC@MHJMHHCD@cp1256_general_ci?$AA@ 004c86b8     strings:ctype-extra.obj
 0002:000086cc       ??_C@_06LODAGMCK@cp1256?$AA@ 004c86cc     strings:ctype-extra.obj
 0002:000086d4       ??_C@_0N@HBDGIFNG@macroman_bin?$AA@ 004c86d4     strings:ctype-extra.obj
 0002:000086e4       ??_C@_0BC@KMCILKA@cp1251_general_cs?$AA@ 004c86e4     strings:ctype-extra.obj
 0002:000086f8       ??_C@_0BC@LKOPHBHL@cp1251_general_ci?$AA@ 004c86f8     strings:ctype-extra.obj
 0002:0000870c       ??_C@_0L@PHMMDEMK@cp1251_bin?$AA@ 004c870c     strings:ctype-extra.obj
 0002:00008718       ??_C@_0BC@DDOEKG@latin1_general_cs?$AA@ 004c8718     strings:ctype-extra.obj
 0002:0000872c       ??_C@_0BC@LABOBOHN@latin1_general_ci?$AA@ 004c872c     strings:ctype-extra.obj
 0002:00008740       ??_C@_0BD@LKINKBJP@cp1250_croatian_ci?$AA@ 004c8740     strings:ctype-extra.obj
 0002:00008754       ??_C@_09FIGDDDHD@macce_bin?$AA@ 004c8754     strings:ctype-extra.obj
 0002:00008760       ??_C@_0BC@KANGDLHL@latin7_general_cs?$AA@ 004c8760     strings:ctype-extra.obj
 0002:00008774       ??_C@_0BC@BAPLMBKA@latin7_general_ci?$AA@ 004c8774     strings:ctype-extra.obj
 0002:00008788       ??_C@_0BB@HEOOOPD@cp852_general_ci?$AA@ 004c8788     strings:ctype-extra.obj
 0002:0000879c       ??_C@_05MDMAGACD@cp852?$AA@ 004c879c     strings:ctype-extra.obj
 0002:000087a4       ??_C@_0BE@BLBOGAK@macroman_general_ci?$AA@ 004c87a4     strings:ctype-extra.obj
 0002:000087b8       ??_C@_08DEGKPPEJ@macroman?$AA@ 004c87b8     strings:ctype-extra.obj
 0002:000087c4       ??_C@_0BB@PFHIEKKE@macce_general_ci?$AA@ 004c87c4     strings:ctype-extra.obj
 0002:000087d8       ??_C@_05CFINKOFD@macce?$AA@ 004c87d8     strings:ctype-extra.obj
 0002:000087e0       ??_C@_0BD@HLAPNNNE@keybcs2_general_ci?$AA@ 004c87e0     strings:ctype-extra.obj
 0002:000087f4       ??_C@_07JDFJFNII@keybcs2?$AA@ 004c87f4     strings:ctype-extra.obj
 0002:000087fc       ??_C@_0BB@LLJGKBLO@cp866_general_ci?$AA@ 004c87fc     strings:ctype-extra.obj
 0002:00008810       ??_C@_05KFOKBLHO@cp866?$AA@ 004c8810     strings:ctype-extra.obj
 0002:00008818       ??_C@_0BE@ELHAPPLJ@armscii8_general_ci?$AA@ 004c8818     strings:ctype-extra.obj
 0002:0000882c       ??_C@_08BDGJEDFB@armscii8?$AA@ 004c882c     strings:ctype-extra.obj
 0002:00008838       ??_C@_0BC@OBCEDJPK@latin5_turkish_ci?$AA@ 004c8838     strings:ctype-extra.obj
 0002:0000884c       ??_C@_06EHCJAAPF@latin5?$AA@ 004c884c     strings:ctype-extra.obj
 0002:00008854       ??_C@_0BF@MPPNICJ@cp1257_lithuanian_ci?$AA@ 004c8854     strings:ctype-extra.obj
 0002:0000886c       ??_C@_06KHCLFNGL@cp1257?$AA@ 004c886c     strings:ctype-extra.obj
 0002:00008874       ??_C@_0BD@LCIKDBGI@latin2_croatian_ci?$AA@ 004c8874     strings:ctype-extra.obj
 0002:00008888       ??_C@_0BC@GHHJKIPO@cp1250_general_ci?$AA@ 004c8888     strings:ctype-extra.obj
 0002:0000889c       ??_C@_06OIGKMLKM@cp1250?$AA@ 004c889c     strings:ctype-extra.obj
 0002:000088a4       ??_C@_0BB@CIGFIMGF@greek_general_ci?$AA@ 004c88a4     strings:ctype-extra.obj
 0002:000088b8       ??_C@_05BMDDGOIH@greek?$AA@ 004c88b8     strings:ctype-extra.obj
 0002:000088c0       ??_C@_0BE@DDCHCMKA@cp1251_ukrainian_ci?$AA@ 004c88c0     strings:ctype-extra.obj
 0002:000088d4       ??_C@_0BB@MJPFCALL@koi8u_general_ci?$AA@ 004c88d4     strings:ctype-extra.obj
 0002:000088e8       ??_C@_05JHCMAEL@koi8u?$AA@ 004c88e8     strings:ctype-extra.obj
 0002:000088f0       ??_C@_0BE@IGDBMPBG@latin2_hungarian_ci?$AA@ 004c88f0     strings:ctype-extra.obj
 0002:00008904       ??_C@_0BD@FCEAFDJA@latin7_estonian_cs?$AA@ 004c8904     strings:ctype-extra.obj
 0002:00008918       ??_C@_06HFBPGCHH@latin7?$AA@ 004c8918     strings:ctype-extra.obj
 0002:00008920       ??_C@_0BC@LFMOPFOE@hebrew_general_ci?$AA@ 004c8920     strings:ctype-extra.obj
 0002:00008934       ??_C@_06IOFFBGCK@hebrew?$AA@ 004c8934     strings:ctype-extra.obj
 0002:0000893c       ??_C@_0BB@HINPBEBI@latin1_danish_ci?$AA@ 004c893c     strings:ctype-extra.obj
 0002:00008950       ??_C@_0BE@HOCIKLDG@cp1251_bulgarian_ci?$AA@ 004c8950     strings:ctype-extra.obj
 0002:00008964       ??_C@_06PBHBPKON@cp1251?$AA@ 004c8964     strings:ctype-extra.obj
 0002:0000896c       ??_C@_0BB@EJGKFKGI@ascii_general_ci?$AA@ 004c896c     strings:ctype-extra.obj
 0002:00008980       ??_C@_05OJENGABA@ascii?$AA@ 004c8980     strings:ctype-extra.obj
 0002:00008988       ??_C@_0BA@CCDGJJLG@swe7_swedish_ci?$AA@ 004c8988     strings:ctype-extra.obj
 0002:00008998       ??_C@_04KPFMKDCH@swe7?$AA@ 004c8998     strings:ctype-extra.obj
 0002:000089a0       ??_C@_0BC@NNEHCLD@latin2_general_ci?$AA@ 004c89a0     strings:ctype-extra.obj
 0002:000089b4       ??_C@_06IGIJGDC@latin2?$AA@ 004c89b4     strings:ctype-extra.obj
 0002:000089bc       ??_C@_0BB@LEIGCGOD@koi8r_general_ci?$AA@ 004c89bc     strings:ctype-extra.obj
 0002:000089d0       ??_C@_05EGDDFGIM@koi8r?$AA@ 004c89d0     strings:ctype-extra.obj
 0002:000089d8       ??_C@_0P@FKJAJKJA@hp8_english_ci?$AA@ 004c89d8     strings:ctype-extra.obj
 0002:000089e8       ??_C@_03GDEHCLKE@hp8?$AA@  004c89e8     strings:ctype-extra.obj
 0002:000089ec       ??_C@_0BC@EOOMILFB@latin1_german1_ci?$AA@ 004c89ec     strings:ctype-extra.obj
 0002:00008a00       ??_C@_0BB@GHBCFLLI@cp850_general_ci?$AA@ 004c8a00     strings:ctype-extra.obj
 0002:00008a14       ??_C@_05PBPGACKB@cp850?$AA@ 004c8a14     strings:ctype-extra.obj
 0002:00008a1c       ??_C@_0BA@KLOOPAA@dec8_swedish_ci?$AA@ 004c8a1c     strings:ctype-extra.obj
 0002:00008a2c       ??_C@_04EJJBHNM@dec8?$AA@  004c8a2c     strings:ctype-extra.obj
 0002:00008a34       ??_C@_08BABJIOEM@filename?$AA@ 004c8a34     strings:ctype-utf8.obj
 0002:00008a40       ??_C@_08BMIDNPKK@utf8_bin?$AA@ 004c8a40     strings:ctype-utf8.obj
 0002:00008a4c       ??_C@_0BA@JGAHNPHO@utf8_general_ci?$AA@ 004c8a4c     strings:ctype-utf8.obj
 0002:00008a5c       ??_C@_0BB@JCEFLFJE@0123456789abcdef?$AA@ 004c8a5c     strings:ctype-utf8.obj
 0002:00008a70       ??_C@_08OGGFHGPF@ujis_bin?$AA@ 004c8a70     strings:ctype-ujis.obj
 0002:00008a7c       ??_C@_0BB@KEGFAMFE@ujis_japanese_ci?$AA@ 004c8a7c     strings:ctype-ujis.obj
 0002:00008a90       ??_C@_04BPGAKKKA@ujis?$AA@ 004c8a90     strings:ctype-ujis.obj
 0002:00008a98       ??_C@_08POIAHHJH@ucs2_bin?$AA@ 004c8a98     strings:ctype-ucs2.obj
 0002:00008aa4       ??_C@_0BA@JBCKHLAM@ucs2_general_ci?$AA@ 004c8aa4     strings:ctype-ucs2.obj
 0002:00008ab4       ??_C@_0L@NBGPIHPA@tis620_bin?$AA@ 004c8ab4     strings:ctype-tis620.obj
 0002:00008ac0       ??_C@_0P@GFLKKABK@tis620_thai_ci?$AA@ 004c8ac0     strings:ctype-tis620.obj
 0002:00008ad0       ??_C@_06MGNELAEE@tis620?$AA@ 004c8ad0     strings:ctype-tis620.obj
 0002:00008ad8       ??_C@_08JFHPAPHP@sjis_bin?$AA@ 004c8ad8     strings:ctype-sjis.obj
 0002:00008ae4       ??_C@_0BB@DFBLLFM@sjis_japanese_ci?$AA@ 004c8ae4     strings:ctype-sjis.obj
 0002:00008af8       ??_C@_04JACAFPAA@sjis?$AA@ 004c8af8     strings:ctype-sjis.obj
 0002:00008b00       ??_C@_07KJPNPKHF@gbk_bin?$AA@ 004c8b00     strings:ctype-gbk.obj
 0002:00008b08       ??_C@_0P@GNPIDCFN@gbk_chinese_ci?$AA@ 004c8b08     strings:ctype-gbk.obj
 0002:00008b18       ??_C@_03LFBAECHL@gbk?$AA@  004c8b18     strings:ctype-gbk.obj
 0002:00008b1c       ??_C@_0L@ODLCHMHL@gb2312_bin?$AA@ 004c8b1c     strings:ctype-gb2312.obj
 0002:00008b28       ??_C@_0BC@NLCEMJAE@gb2312_chinese_ci?$AA@ 004c8b28     strings:ctype-gb2312.obj
 0002:00008b3c       ??_C@_06JIBIJLME@gb2312?$AA@ 004c8b3c     strings:ctype-gb2312.obj
 0002:00008b44       ??_C@_09JHKEBMLO@euckr_bin?$AA@ 004c8b44     strings:ctype-euc_kr.obj
 0002:00008b50       ??_C@_0BA@EKHKJCHH@euckr_korean_ci?$AA@ 004c8b50     strings:ctype-euc_kr.obj
 0002:00008b60       ??_C@_05FHCOMIFC@euckr?$AA@ 004c8b60     strings:ctype-euc_kr.obj
 0002:00008b68       ??_C@_0M@BEKAHKLO@eucjpms_bin?$AA@ 004c8b68     strings:ctype-eucjpms.obj
 0002:00008b74       ??_C@_0BE@GEODDEKB@eucjpms_japanese_ci?$AA@ 004c8b74     strings:ctype-eucjpms.obj
 0002:00008b88       ??_C@_07MOEGLBAH@eucjpms?$AA@ 004c8b88     strings:ctype-eucjpms.obj
 0002:00008b90       ??_C@_0BA@IOACFKLD@latin2_czech_cs?$AA@ 004c8b90     strings:ctype-czech.obj
 0002:00008ba0       ??_C@_04PJNGGADL@?$AF?6?$BC?$BC?$AA@ 004c8ba0     strings:ctype-czech.obj
 0002:00008ba8       ??_C@_01GFHCPBMG@C?$AA@    004c8ba8     strings:ctype-czech.obj
 0002:00008bac       ??_C@_04NALNINKB@?$AF?6?$BB?$BB?$AA@ 004c8bac     strings:ctype-czech.obj
 0002:00008bb4       ??_C@_01PAPGNFGE@c?$AA@    004c8bb4     strings:ctype-czech.obj
 0002:00008bb8       ??_C@_04DCMIHFOD@?$AM?$BJ11?$AA@ 004c8bb8     strings:ctype-czech.obj
 0002:00008bc0       ??_C@_02EKMCNAHJ@CH?$AA@   004c8bc0     strings:ctype-czech.obj
 0002:00008bc4       ??_C@_04CKBBCOJF@?$AM?$BJ00?$AA@ 004c8bc4     strings:ctype-czech.obj
 0002:00008bcc       ??_C@_02NPEGPENL@Ch?$AA@   004c8bcc     strings:ctype-czech.obj
 0002:00008bd0       ??_C@_04PADBMEEG@?$AM?$BJ?1?1?$AA@ 004c8bd0     strings:ctype-czech.obj
 0002:00008bd8       ??_C@_02OHALLCDL@ch?$AA@   004c8bd8     strings:ctype-czech.obj
 0002:00008be0       ??_C@_0BAB@LDKHKKBE@?$LE?$LF?$LG?$LH?$LI?$LJ?$LK?$LL?$LM?$AC?$LO?$LP?$MA?A?B?C?D?E?F?G?H?I?J?K?L?M?N?O?P?Q?R?S@ 004c8be0     strings:ctype-czech.obj
 0002:00008ce8       ??_C@_0BAB@JENJBEPB@?$AA?$AA?$AA?$AA?$AA?$AA?$AA?$AA?$AA?$AC?$AA?$AA?$AA?$AA?$AA?$AA?$AA?$AA?$AA?$AA?$AA?$AA?$AA?$AA?$AA?$AA?$AA?$AA?$AA?$AA?$AA?$AA@ 004c8ce8     strings:ctype-czech.obj
 0002:00008df0       ??_C@_0BAB@GIDHDAFJ@?$AA?$AA?$AA?$AA?$AA?$AA?$AA?$AA?$AA?$AC?$AA?$AA?$AA?$AA?$AA?$AA?$AA?$AA?$AA?$AA?$AA?$AA?$AA?$AA?$AA?$AA?$AA?$AA?$AA?$AA?$AA?$AA@ 004c8df0     strings:ctype-czech.obj
 0002:00008ef8       ??_C@_0BAB@HNOGOFAJ@?$AA?$AA?$AA?$AA?$AA?$AA?$AA?$AA?$AA?$AC?$AA?$AA?$AA?$AA?$AA?$AA?$AA?$AA?$AA?$AA?$AA?$AA?$AA?$AA?$AA?$AA?$AA?$AA?$AA?$AA?$AA?$AA@ 004c8ef8     strings:ctype-czech.obj
 0002:00008ffc       ??_C@_0BA@MDKNCPKD@cp1250_czech_cs?$AA@ 004c8ffc     strings:ctype-win1250ch.obj
 0002:0000900c       ??_C@_08CJHFMMIC@big5_bin?$AA@ 004c900c     strings:ctype-big5.obj
 0002:00009018       ??_C@_0BA@HCMNJPNC@big5_chinese_ci?$AA@ 004c9018     strings:ctype-big5.obj
 0002:00009028       ??_C@_04HDKIILFF@big5?$AA@ 004c9028     strings:ctype-big5.obj
 0002:00009030       ??_C@_0O@IDJJBCJJ@unknown?5token?$AA@ 004c9030     strings:xml.obj
 0002:00009040       ??_C@_03BECJNG@?8?$CB?8?$AA@ 004c9040     strings:xml.obj
 0002:00009044       ??_C@_03BGKMKHKM@?8?$DP?8?$AA@ 004c9044     strings:xml.obj
 0002:00009048       ??_C@_04OEPMCOLO@TEXT?$AA@ 004c9048     strings:xml.obj
 0002:00009050       ??_C@_07JEDAPFNH@COMMENT?$AA@ 004c9050     strings:xml.obj
 0002:00009058       ??_C@_03KIKAENM@?8?1?8?$AA@ 004c9058     strings:xml.obj
 0002:0000905c       ??_C@_03BHGOMNJL@?8?$DO?8?$AA@ 004c905c     strings:xml.obj
 0002:00009060       ??_C@_03BEOKBJPF@?8?$DM?8?$AA@ 004c9060     strings:xml.obj
 0002:00009064       ??_C@_03BFCIHDMC@?8?$DN?8?$AA@ 004c9064     strings:xml.obj
 0002:00009068       ??_C@_05MLPNBPGH@CDATA?$AA@ 004c9068     strings:xml.obj
 0002:00009070       ??_C@_05MDAAGLOE@IDENT?$AA@ 004c9070     strings:xml.obj
 0002:00009078       ??_C@_06IGECGLFO@STRING?$AA@ 004c9078     strings:xml.obj
 0002:00009080       ??_C@_0N@KFMDIEOD@END?9OF?9INPUT?$AA@ 004c9080     strings:xml.obj
 0002:00009090       ??_C@_06NPFKMDPM@?$DP?$DN?1?$DM?$DO?$CB?$AA@ 004c9090     strings:xml.obj
 0002:00009098       ??_C@_09BLLNCBLF@?$DM?$CB?$FLCDATA?$FL?$AA@ 004c9098     strings:xml.obj
 0002:000090a4       ??_C@_04FFDNBKGC@?$DM?$CB?9?9?$AA@ 004c90a4     strings:xml.obj
 0002:000090ac       ??_C@_0M@JHPIDPOK@To?5deep?5XML?$AA@ 004c90ac     strings:xml.obj
 0002:000090b8       ??_C@_0CJ@FBAHKBHA@?8?$DM?1?$CFs?$DO?8?5unexpected?5?$CIEND?9OF?9INPUT@ 004c90b8     strings:xml.obj
 0002:000090e4       ??_C@_0CE@HIBBMALO@?8?$DM?1?$CFs?$DO?8?5unexpected?5?$CI?8?$DM?1?$CFs?$DO?8?5want@ 004c90e4     strings:xml.obj
 0002:00009108       ??_C@_0CE@KDMBOGDF@?$CFs?5unexpected?5?$CIident?5or?5?8?1?8?5want@ 004c9108     strings:xml.obj
 0002:0000912c       ??_C@_0BL@DBFJAODI@?$CFs?5unexpected?5?$CI?8?$DP?8?5wanted?$CJ?$AA@ 004c912c     strings:xml.obj
 0002:00009148       ??_C@_0CH@MBBDFLOA@?$CFs?5unexpected?5?$CIident?5or?5string?5w@ 004c9148     strings:xml.obj
 0002:00009170       ??_C@_0BN@GIJBNIHN@?$CFs?5unexpected?5?$CIident?5wanted?$CJ?$AA@ 004c9170     strings:xml.obj
 0002:00009190       ??_C@_0BI@GOAECBLB@unexpected?5END?9OF?9INPUT?$AA@ 004c9190     strings:xml.obj
 0002:000091a8       ??_C@_0BL@PANHNBPI@?$CFs?5unexpected?5?$CI?8?$DO?8?5wanted?$CJ?$AA@ 004c91a8     strings:xml.obj
 0002:000091c4       ??_C@_0M@GPMPBOKO@TCP?1IP?5?$CI?$CFd?$CJ?$AA@ 004c91c4     vio:vio.obj
 0002:000091d0       ??_C@_0M@BKHBDAGP@socket?5?$CI?$CFd?$CJ?$AA@ 004c91d0     vio:vio.obj
 0002:000091dc       ??_C@_0L@BGAKJGHL@named?5pipe?$AA@ 004c91dc     vio:vio.obj
 0002:000091e8       ??_C@_0O@CPADDGOO@shared?5memory?$AA@ 004c91e8     vio:vio.obj
 0002:000091f8       ??_C@_09PFCHIMEP@127?40?40?41?$AA@ 004c91f8     vio:viosocket.obj
 0002:00009204       ??_C@_0BD@JKAKBJG@SSL_CTX_new?5failed?$AA@ 004c9204     vio:viosslfactories.obj
 0002:00009218       ??_C@_0BN@EHNEHPHI@Failed?5to?5set?5ciphers?5to?5use?$AA@ 004c9218     vio:viosslfactories.obj
 0002:00009238       ??_C@_0FN@GPPKHFPO@Private?5key?5does?5not?5match?5the?5c@ 004c9238     vio:viosslfactories.obj
 0002:00009298       ??_C@_0BK@OJIINBMD@Unable?5to?5get?5private?5key?$AA@ 004c9298     vio:viosslfactories.obj
 0002:000092b4       ??_C@_0BK@DLGAGNNA@Unable?5to?5get?5certificate?$AA@ 004c92b4     vio:viosslfactories.obj
 0002:000092d0       ??_C@_08INEPGKHH@No?5error?$AA@ 004c92d0     vio:viosslfactories.obj
 0002:000092dc       ??_C@_0P@PDGGPCGE@SSL?5error?3?5?$CFs?6?$AA@ 004c92dc     vio:viosslfactories.obj
 0002:000092ec       ??_C@_0BJ@DBKDBMMN@SSL?5error?3?5?$CFs?5from?5?8?$CFs?8?6?$AA@ 004c92ec     vio:viosslfactories.obj
 0002:00009310       ??_7Message@yaSSL@@6B@     004c9310     yassl:ssl.obj
 0002:0000932c       ??_7HandShakeBase@yaSSL@@6B@ 004c932c     yassl:ssl.obj
 0002:00009344       ??_7HASH@TaoCrypt@@6B@     004c9344     yassl:ssl.obj
 0002:00009360       ??_7MD5@TaoCrypt@@6B@      004c9360     yassl:ssl.obj
 0002:00009388       ??_7MD4@TaoCrypt@@6B@      004c9388     yassl:ssl.obj
 0002:000093ac       ??_C@_0BM@CIPOPOID@Not?5Implemented?0?5SSLv2?5only?$AA@ 004c93ac     yassl:ssl.obj
 0002:000093c8       ??_C@_05LLIBCOJ@TLSv1?$AA@ 004c93c8     yassl:ssl.obj
 0002:000093d0       ??_C@_05MOEBAHEJ@SSLv3?$AA@ 004c93d0     yassl:ssl.obj
 0002:000093d8       ??_C@_0BL@IAMLJBHP@SSLeay?5yaSSL?5compatibility?$AA@ 004c93d8     yassl:ssl.obj
 0002:000093f4       ??_C@_0CI@BCOALAL@Please?5supply?5a?5buffer?5for?5error@ 004c93f4     yassl:ssl.obj
 0002:0000941c       ??_C@_0BA@JGKGKAME@Not?5Implemented?$AA@ 004c941c     yassl:ssl.obj
 0002:0000942c       ??_C@_03GCGHEHKJ@MD5?$AA@  004c942c     yassl:ssl.obj
 0002:00009430       ??_C@_0N@MLDFENGJ@DES?9EDE3?9CBC?$AA@ 004c9430     yassl:ssl.obj
 0002:00009440       ??_C@_0M@FOEEEMFG@AES?9256?9CBC?$AA@ 004c9440     yassl:ssl.obj
 0002:0000944c       ??_C@_0M@IMPKGDNH@AES?9192?9CBC?$AA@ 004c944c     yassl:ssl.obj
 0002:00009458       ??_C@_0M@CPGGBEEL@AES?9128?9CBC?$AA@ 004c9458     yassl:ssl.obj
 0002:00009464       ??_C@_07LDJJJFAI@DES?9CBC?$AA@ 004c9464     yassl:ssl.obj
 0002:0000946c       ??_C@_02JDPG@rb?$AA@       004c946c     yassl:ssl.obj
 0002:00009470       ??_C@_02KHDDNBB@?2?$CK?$AA@ 004c9470     yassl:ssl.obj
 0002:00009474       ??_C@_07OCFLHCIN@RC4?9MD5?$AA@ 004c9474     yassl:ssl.obj
 0002:0000947c       ??_C@_07BANEBHLH@RC4?9SHA?$AA@ 004c947c     yassl:ssl.obj
 0002:00009484       ??_C@_0M@LLIFGIFE@DES?9CBC?9SHA?$AA@ 004c9484     yassl:ssl.obj
 0002:00009490       ??_C@_0N@HCCILIJF@DES?9CBC3?9SHA?$AA@ 004c9490     yassl:ssl.obj
 0002:000094a0       ??_C@_0BE@COMFBKAK@EDH?9DSS?9DES?9CBC?9SHA?$AA@ 004c94a0     yassl:ssl.obj
 0002:000094b4       ??_C@_0BF@POGOIEBE@EDH?9DSS?9DES?9CBC3?9SHA?$AA@ 004c94b4     yassl:ssl.obj
 0002:000094cc       ??_C@_0BE@BMKPLFLB@EDH?9RSA?9DES?9CBC?9SHA?$AA@ 004c94cc     yassl:ssl.obj
 0002:000094e0       ??_C@_0BF@KCOPIELP@EDH?9RSA?9DES?9CBC3?9SHA?$AA@ 004c94e0     yassl:ssl.obj
 0002:000094f8       ??_C@_0L@FJECLCPG@AES128?9SHA?$AA@ 004c94f8     yassl:ssl.obj
 0002:00009504       ??_C@_0BD@HPNPDEHO@DHE?9DSS?9AES128?9SHA?$AA@ 004c9504     yassl:ssl.obj
 0002:00009518       ??_C@_0BD@MNBMGMFC@DHE?9RSA?9AES128?9SHA?$AA@ 004c9518     yassl:ssl.obj
 0002:0000952c       ??_C@_0L@CIGAOKOL@AES256?9SHA?$AA@ 004c952c     yassl:ssl.obj
 0002:00009538       ??_C@_0BD@OPNGMGD@DHE?9DSS?9AES256?9SHA?$AA@ 004c9538     yassl:ssl.obj
 0002:0000954c       ??_C@_0BD@LMDODEEP@DHE?9RSA?9AES256?9SHA?$AA@ 004c954c     yassl:ssl.obj
 0002:00009560       ??_C@_0BF@EGKJPLJF@DHE?9DSS?9DES?9CBC3?9RMD?$AA@ 004c9560     yassl:ssl.obj
 0002:00009578       ??_C@_0BD@LMNPGFLF@DHE?9DSS?9AES128?9RMD?$AA@ 004c9578     yassl:ssl.obj
 0002:0000958c       ??_C@_0BD@MNPNDNKI@DHE?9DSS?9AES256?9RMD?$AA@ 004c958c     yassl:ssl.obj
 0002:000095a0       ??_C@_0BF@BKCIPLDO@DHE?9RSA?9DES?9CBC3?9RMD?$AA@ 004c95a0     yassl:ssl.obj
 0002:000095b8       ??_C@_0BD@OBMDNJJ@DHE?9RSA?9AES128?9RMD?$AA@ 004c95b8     yassl:ssl.obj
 0002:000095cc       ??_C@_0BD@HPDOGFIE@DHE?9RSA?9AES256?9RMD?$AA@ 004c95cc     yassl:ssl.obj
 0002:000095e0       ??_C@_0N@LBCIOJFO@DES?9CBC3?9RMD?$AA@ 004c95e0     yassl:ssl.obj
 0002:000095f0       ??_C@_0L@JKECODDN@AES128?9RMD?$AA@ 004c95f0     yassl:ssl.obj
 0002:000095fc       ??_C@_0L@OLGALLCA@AES256?9RMD?$AA@ 004c95fc     yassl:ssl.obj
 0002:0000962c       ??_C@_07MIJDMBL@GGGGGGG?$AA@ 004c962c     yassl:yassl_int.obj
 0002:00009634       ??_C@_06CHLBDKEK@FFFFFF?$AA@ 004c9634     yassl:yassl_int.obj
 0002:0000963c       ??_C@_05NGCOEONO@EEEEE?$AA@ 004c963c     yassl:yassl_int.obj
 0002:00009644       ??_C@_03POJCPIGP@CCC?$AA@  004c9644     yassl:yassl_int.obj
 0002:00009648       ??_C@_09IKAJMJIH@yaSSL?4log?$AA@ 004c9648     yassl:yassl_int.obj
 0002:0000965c       ??_7Digest@yaSSL@@6B@      004c965c     yassl:crypto_wrapper.obj
 0002:00009678       ??_7BulkCipher@yaSSL@@6B@  004c9678     yassl:crypto_wrapper.obj
 0002:0000969c       ??_7Auth@yaSSL@@6B@        004c969c     yassl:crypto_wrapper.obj
 0002:000096b0       ??_7SHA@TaoCrypt@@6B@      004c96b0     yassl:crypto_wrapper.obj
 0002:000096d8       ??_7RIPEMD160@TaoCrypt@@6B@ 004c96d8     yassl:crypto_wrapper.obj
 0002:00009700       ??_7Mode_BASE@TaoCrypt@@6B@ 004c9700     yassl:crypto_wrapper.obj
 0002:00009710       ??_7DES@TaoCrypt@@6B@      004c9710     yassl:crypto_wrapper.obj
 0002:00009720       ??_7DES_EDE3@TaoCrypt@@6B@ 004c9720     yassl:crypto_wrapper.obj
 0002:00009730       ??_7AES@TaoCrypt@@6B@      004c9730     yassl:crypto_wrapper.obj
 0002:00009740       ??_7MD5@yaSSL@@6B@         004c9740     yassl:crypto_wrapper.obj
 0002:0000975c       ??_7SHA@yaSSL@@6B@         004c975c     yassl:crypto_wrapper.obj
 0002:00009778       ??_7RMD@yaSSL@@6B@         004c9778     yassl:crypto_wrapper.obj
 0002:00009794       ??_7RC4@yaSSL@@6B@         004c9794     yassl:crypto_wrapper.obj
 0002:000097b8       ??_7AES@yaSSL@@6B@         004c97b8     yassl:crypto_wrapper.obj
 0002:000097dc       ??_7HMAC_MD5@yaSSL@@6B@    004c97dc     yassl:crypto_wrapper.obj
 0002:000097f8       ??_7HMAC_SHA@yaSSL@@6B@    004c97f8     yassl:crypto_wrapper.obj
 0002:00009814       ??_7HMAC_RMD@yaSSL@@6B@    004c9814     yassl:crypto_wrapper.obj
 0002:00009830       ??_7DES@yaSSL@@6B@         004c9830     yassl:crypto_wrapper.obj
 0002:00009854       ??_7DES_EDE@yaSSL@@6B@     004c9854     yassl:crypto_wrapper.obj
 0002:00009878       ??_7DSS@yaSSL@@6B@         004c9878     yassl:crypto_wrapper.obj
 0002:0000988c       ??_7RSA@yaSSL@@6B@         004c988c     yassl:crypto_wrapper.obj
 0002:0000989c       ??_C@_01LIIJDEN@?$AN?$AA@  004c989c     yassl:crypto_wrapper.obj
 0002:000098a0       ??_C@_03BKNEFOAH@AES?$AA@  004c98a0     yassl:crypto_wrapper.obj
 0002:000098a4       ??_C@_01IHBHIGKO@?0?$AA@   004c98a4     yassl:crypto_wrapper.obj
 0002:000098a8       ??_C@_03CNAKKODF@DES?$AA@  004c98a8     yassl:crypto_wrapper.obj
 0002:000098ac       ??_C@_09OEEMHJLK@Proc?9Type?$AA@ 004c98ac     yassl:crypto_wrapper.obj
 0002:000098b8       ??_C@_0BO@KNLPBMJG@?9?9?9?9?9END?5RSA?5PRIVATE?5KEY?9?9?9?9?9?$AA@ 004c98b8     yassl:crypto_wrapper.obj
 0002:000098d8       ??_C@_0CA@PEOGIGIM@?9?9?9?9?9BEGIN?5RSA?5PRIVATE?5KEY?9?9?9?9?9?$AA@ 004c98d8     yassl:crypto_wrapper.obj
 0002:000098f8       ??_C@_0BK@LPPAEOGJ@?9?9?9?9?9END?5CERTIFICATE?9?9?9?9?9?$AA@ 004c98f8     yassl:crypto_wrapper.obj
 0002:00009914       ??_C@_0BM@CPJANAAJ@?9?9?9?9?9BEGIN?5CERTIFICATE?9?9?9?9?9?$AA@ 004c9914     yassl:crypto_wrapper.obj
 0002:00009940       ??_7HandShakeHeader@yaSSL@@6B@ 004c9940     yassl:yassl_imp.obj
 0002:0000995c       ??_7ServerKeyBase@yaSSL@@6B@ 004c995c     yassl:yassl_imp.obj
 0002:00009974       ??_7ClientKeyBase@yaSSL@@6B@ 004c9974     yassl:yassl_imp.obj
 0002:0000998c       ??_7ClientDiffieHellmanPublic@yaSSL@@6B@ 004c998c     yassl:yassl_imp.obj
 0002:000099a4       ??_7ChangeCipherSpec@yaSSL@@6B@ 004c99a4     yassl:yassl_imp.obj
 0002:000099c0       ??_7Alert@yaSSL@@6B@       004c99c0     yassl:yassl_imp.obj
 0002:000099dc       ??_7Data@yaSSL@@6B@        004c99dc     yassl:yassl_imp.obj
 0002:000099f8       ??_7Certificate@yaSSL@@6B@ 004c99f8     yassl:yassl_imp.obj
 0002:00009a10       ??_7ServerHello@yaSSL@@6B@ 004c9a10     yassl:yassl_imp.obj
 0002:00009a28       ??_7ServerHelloDone@yaSSL@@6B@ 004c9a28     yassl:yassl_imp.obj
 0002:00009a40       ??_7ClientHello@yaSSL@@6B@ 004c9a40     yassl:yassl_imp.obj
 0002:00009a58       ??_7ServerKeyExchange@yaSSL@@6B@ 004c9a58     yassl:yassl_imp.obj
 0002:00009a70       ??_7CertificateVerify@yaSSL@@6B@ 004c9a70     yassl:yassl_imp.obj
 0002:00009a88       ??_7ClientKeyExchange@yaSSL@@6B@ 004c9a88     yassl:yassl_imp.obj
 0002:00009aa0       ??_7Finished@yaSSL@@6B@    004c9aa0     yassl:yassl_imp.obj
 0002:00009ab8       ??_7HelloRequest@yaSSL@@6B@ 004c9ab8     yassl:yassl_imp.obj
 0002:00009ad0       ??_7RSA_Server@yaSSL@@6B@  004c9ad0     yassl:yassl_imp.obj
 0002:00009ae8       ??_7Fortezza_Server@yaSSL@@6B@ 004c9ae8     yassl:yassl_imp.obj
 0002:00009b00       ??_7FortezzaKeys@yaSSL@@6B@ 004c9b00     yassl:yassl_imp.obj
 0002:00009b18       ??_7EncryptedPreMasterSecret@yaSSL@@6B@ 004c9b18     yassl:yassl_imp.obj
 0002:00009b2c       ??_C@_0BJ@MIAIEIAP@server?5denied?5resumption?$AA@ 004c9b2c     yassl:yassl_imp.obj
 0002:00009b48       ??_C@_0BG@NFGEHEFF@session?5lookup?5failed?$AA@ 004c9b48     yassl:yassl_imp.obj
 0002:00009b64       ??_7DH_Server@yaSSL@@6B@   004c9b64     yassl:yassl_imp.obj
 0002:00009b78       ??_C@_04OKGDLNCL@NONE?$AA@ 004c9b78     yassl:yassl_imp.obj
 0002:00009b84       ??_7CertificateRequest@yaSSL@@6B@ 004c9b84     yassl:yassl_imp.obj
 0002:00009c28       ??_C@_0BF@LOHHNDDD@unknown?5error?5number?$AA@ 004c9c28     yassl:yassl_error.obj
 0002:00009c40       ??_C@_0BN@DLDIDPJM@Unable?5to?5verify?5certificate?$AA@ 004c9c40     yassl:yassl_error.obj
 0002:00009c60       ??_C@_0BK@HAFIKEEK@bad?5PEM?5format?5processing?$AA@ 004c9c60     yassl:yassl_error.obj
 0002:00009c7c       ??_C@_0BH@PIPJPDKN@bad?5content?5processing?$AA@ 004c9c7c     yassl:yassl_error.obj
 0002:00009c94       ??_C@_0CG@JIHDAALO@ASN?3?5bad?5other?5signature?5confirm@ 004c9c94     yassl:yassl_error.obj
 0002:00009cbc       ??_C@_0CF@OCOHBCCG@ASN?3?5bad?5self?5signature?5confirma@ 004c9cbc     yassl:yassl_error.obj
 0002:00009ce4       ??_C@_0BM@NEHMDLJI@ASN?3?5after?5date?5in?5the?5past?$AA@ 004c9ce4     yassl:yassl_error.obj
 0002:00009d00       ??_C@_0BP@BJJDPHIA@ASN?3?5before?5date?5in?5the?5future?$AA@ 004c9d00     yassl:yassl_error.obj
 0002:00009d20       ??_C@_0BJ@HLIMONLK@ASN?3?5bad?5DSA?5r?5or?5s?5size?$AA@ 004c9d20     yassl:yassl_error.obj
 0002:00009d3c       ??_C@_0BG@DKPAPHGN@ASN?3?5unknown?5hash?5OID?$AA@ 004c9d3c     yassl:yassl_error.obj
 0002:00009d54       ??_C@_0BL@LEANJGE@ASN?3?5unknown?5signature?5OID?$AA@ 004c9d54     yassl:yassl_error.obj
 0002:00009d70       ??_C@_0BK@DFPFLNHD@ASN?3?5bad?5Signature?5Length?$AA@ 004c9d70     yassl:yassl_error.obj
 0002:00009d8c       ??_C@_0BD@BBKHNDOD@ASN?3?5bad?5Date?5Size?$AA@ 004c9d8c     yassl:yassl_error.obj
 0002:00009da0       ??_C@_0O@NCDKAAAO@ASN?3?5bad?5TIME?$AA@ 004c9da0     yassl:yassl_error.obj
 0002:00009db0       ??_C@_0BN@GPGLBGJG@ASN?3?5bad?5Octet?5String?5Header?$AA@ 004c9db0     yassl:yassl_error.obj
 0002:00009dd0       ??_C@_0BA@CHEGMMMD@ASN?3?5expected?50?$AA@ 004c9dd0     yassl:yassl_error.obj
 0002:00009de0       ??_C@_0BH@CNGNFALI@ASN?3?5expected?5TAG?5NULL?$AA@ 004c9de0     yassl:yassl_error.obj
 0002:00009df8       ??_C@_0BK@EHIEHJHJ@ASN?3?5bad?5Ojbect?5ID?5Header?$AA@ 004c9df8     yassl:yassl_error.obj
 0002:00009e14       ??_C@_0BK@JLGAAPDA@ASN?3?5unknown?5key?5OID?5type?$AA@ 004c9e14     yassl:yassl_error.obj
 0002:00009e30       ??_C@_0BK@NEMPKOOB@ASN?3?5bad?5BitString?5Header?$AA@ 004c9e30     yassl:yassl_error.obj
 0002:00009e4c       ??_C@_0BM@EABFJODO@ASN?3?5signature?5OID?5mismatch?$AA@ 004c9e4c     yassl:yassl_error.obj
 0002:00009e68       ??_C@_0BK@PCPPAJBM@ASN?3?5version?5length?5not?51?$AA@ 004c9e68     yassl:yassl_error.obj
 0002:00009e84       ??_C@_0BE@CBIMDPIB@ASN?3?5bad?5Set?5Header?$AA@ 004c9e84     yassl:yassl_error.obj
 0002:00009e98       ??_C@_0BJ@BABNHBJL@ASN?3?5bad?5Sequence?5Header?$AA@ 004c9e98     yassl:yassl_error.obj
 0002:00009eb4       ??_C@_0BM@MLGJJFHM@ASN?3?5bad?5DER?5Integer?5Header?$AA@ 004c9eb4     yassl:yassl_error.obj
 0002:00009ed0       ??_C@_0BM@EOJLGIGG@unable?5to?5use?5random?5device?$AA@ 004c9ed0     yassl:yassl_error.obj
 0002:00009eec       ??_C@_0BF@OKLABNFB@CryptGenRandom?5error?$AA@ 004c9eec     yassl:yassl_error.obj
 0002:00009f04       ??_C@_0BF@ONICCKFL@bad?5wincrypt?5acquire?$AA@ 004c9f04     yassl:yassl_error.obj
 0002:00009f1c       ??_C@_0BD@EFIDFPA@not?5in?5error?5state?$AA@ 004c9f1c     yassl:yassl_error.obj
 0002:00009f30       ??_C@_0BP@JNLPEFPG@the?5read?5operation?5would?5block?$AA@ 004c9f30     yassl:yassl_error.obj
 0002:00009f50       ??_C@_0CC@PELKPKCF@bad?5PreMasterSecret?5version?5erro@ 004c9f50     yassl:yassl_error.obj
 0002:00009f74       ??_C@_0BE@IGBKENJK@decompression?5error?$AA@ 004c9f74     yassl:yassl_error.obj
 0002:00009f88       ??_C@_0BC@NKDLBFJI@compression?5error?$AA@ 004c9f88     yassl:yassl_error.obj
 0002:00009f9c       ??_C@_0BJ@OIPMFMB@protocl?5version?5mismatch?$AA@ 004c9f9c     yassl:yassl_error.obj
 0002:00009fb8       ??_C@_0CL@JIHDBKKF@unable?5to?5proccess?5private?5key?0?5@ 004c9fb8     yassl:yassl_error.obj
 0002:00009fe4       ??_C@_0BO@JFJFDJB@unable?5to?5proccess?5cerificate?$AA@ 004c9fe4     yassl:yassl_error.obj
 0002:0000a004       ??_C@_0BL@PNPNLENI@socket?5layer?5receive?5error?$AA@ 004ca004     yassl:yassl_error.obj
 0002:0000a020       ??_C@_0BI@IMFNBLNH@socket?5layer?5send?5error?$AA@ 004ca020     yassl:yassl_error.obj
 0002:0000a038       ??_C@_0BP@DJNJFCDO@unable?5to?5verify?5peer?5checksum?$AA@ 004ca038     yassl:yassl_error.obj
 0002:0000a058       ??_C@_0CE@JNMOHBDL@the?5server?5needs?5a?5private?5key?5f@ 004ca058     yassl:yassl_error.obj
 0002:0000a07c       ??_C@_0CJ@MGMCLLGF@unable?5to?5match?5a?5supported?5ciph@ 004ca07c     yassl:yassl_error.obj
 0002:0000a0a8       ??_C@_0BH@BJAEIFLP@bad?5cipher?5suite?5input?$AA@ 004ca0a8     yassl:yassl_error.obj
 0002:0000a0c0       ??_C@_0CK@DPEGAADO@handshake?5message?5received?5in?5wr@ 004ca0c0     yassl:yassl_error.obj
 0002:0000a0ec       ??_C@_0BO@MDNKKMLF@handshake?5layer?5not?5ready?5yet?$AA@ 004ca0ec     yassl:yassl_error.obj
 0002:0000a10c       ??_C@_0BL@JKJNJCO@record?5layer?5not?5ready?5yet?$AA@ 004ca10c     yassl:yassl_error.obj
 0002:0000a128       ??_C@_0CN@HCIHAPHI@bad?5master?5secret?5derivation?0?5pr@ 004ca128     yassl:yassl_error.obj
 0002:0000a158       ??_C@_0CA@ICDMIOMH@trying?5to?5use?5an?5unknown?5cipher?$AA@ 004ca158     yassl:yassl_error.obj
 0002:0000a178       ??_C@_0BP@HEAJNFGH@unknown?5factory?5create?5request?$AA@ 004ca178     yassl:yassl_error.obj
 0002:0000a198       ??_C@_0CB@GDMDOMBH@trying?5to?5realloc?5a?5fixed?5buffer@ 004ca198     yassl:yassl_error.obj
 0002:0000a1bc       ??_C@_0CB@GAKDHIMM@buffer?5index?5error?0?5out?5of?5range@ 004ca1bc     yassl:yassl_error.obj
 0002:0000a1e4       ??_C@_05GDHACFMB@1?42?43?$AA@ 004ca1e4     zlib:compress.obj
 0002:0000a1f0       _deflate_copyright         004ca1f0     zlib:deflate.obj
 0002:0000ab50       ??_C@_0BH@FGKKJGOC@incorrect?5length?5check?$AA@ 004cab50     zlib:inflate.obj
 0002:0000ab68       ??_C@_0BF@MEIGEHBE@incorrect?5data?5check?$AA@ 004cab68     zlib:inflate.obj
 0002:0000ab80       ??_C@_0BO@ECPMAOGG@invalid?5distance?5too?5far?5back?$AA@ 004cab80     zlib:inflate.obj
 0002:0000aba0       ??_C@_0BG@LBKINIKP@invalid?5distance?5code?$AA@ 004caba0     zlib:inflate.obj
 0002:0000abb8       ??_C@_0BM@FFFLPBBC@invalid?5literal?1length?5code?$AA@ 004cabb8     zlib:inflate.obj
 0002:0000abd4       ??_C@_0BG@GMDFCBGP@invalid?5distances?5set?$AA@ 004cabd4     zlib:inflate.obj
 0002:0000abec       ??_C@_0BK@BMMPFBBH@invalid?5bit?5length?5repeat?$AA@ 004cabec     zlib:inflate.obj
 0002:0000ac08       ??_C@_0BM@IIMGAINC@invalid?5literal?1lengths?5set?$AA@ 004cac08     zlib:inflate.obj
 0002:0000ac24       ??_C@_0CE@GMIGFPBB@too?5many?5length?5or?5distance?5symb@ 004cac24     zlib:inflate.obj
 0002:0000ac48       ??_C@_0BJ@HDEPPGOH@invalid?5code?5lengths?5set?$AA@ 004cac48     zlib:inflate.obj
 0002:0000ac64       ??_C@_0BN@LGAADGOK@invalid?5stored?5block?5lengths?$AA@ 004cac64     zlib:inflate.obj
 0002:0000ac84       ??_C@_0BD@PJCBIDD@invalid?5block?5type?$AA@ 004cac84     zlib:inflate.obj
 0002:0000ac98       ??_C@_0BE@GONKLEPM@header?5crc?5mismatch?$AA@ 004cac98     zlib:inflate.obj
 0002:0000acac       ??_C@_0BJ@BLBBCOMO@unknown?5header?5flags?5set?$AA@ 004cacac     zlib:inflate.obj
 0002:0000acc8       ??_C@_0BH@LIBMMIGA@incorrect?5header?5check?$AA@ 004cacc8     zlib:inflate.obj
 0002:0000ace0       ??_C@_0BE@EMOGCLGO@invalid?5window?5size?$AA@ 004cace0     zlib:inflate.obj
 0002:0000acf4       ??_C@_0BL@IHKGDAEE@unknown?5compression?5method?$AA@ 004cacf4     zlib:inflate.obj
 0002:0000b358       __dist_code                004cb358     zlib:trees.obj
 0002:0000b558       __length_code              004cb558     zlib:trees.obj
 0002:0000d748       ??_C@_0BF@CJFPCCEG@incompatible?5version?$AA@ 004cd748     zlib:zutil.obj
 0002:0000d760       ??_C@_0N@DFPGLBGC@buffer?5error?$AA@ 004cd760     zlib:zutil.obj
 0002:0000d770       ??_C@_0BE@OGGJBMCE@insufficient?5memory?$AA@ 004cd770     zlib:zutil.obj
 0002:0000d784       ??_C@_0L@HAHMBNLP@data?5error?$AA@ 004cd784     zlib:zutil.obj
 0002:0000d790       ??_C@_0N@MKKNPMJD@stream?5error?$AA@ 004cd790     zlib:zutil.obj
 0002:0000d7a0       ??_C@_0L@KIJFAKBJ@file?5error?$AA@ 004cd7a0     zlib:zutil.obj
 0002:0000d7ac       ??_C@_0L@FNAOCBOG@stream?5end?$AA@ 004cd7ac     zlib:zutil.obj
 0002:0000d7b8       ??_C@_0BA@MOKMMFOD@need?5dictionary?$AA@ 004cd7b8     zlib:zutil.obj
 0002:0000d7c8       _z_errmsg                  004cd7c8     zlib:zutil.obj
 0002:0000d7f0       _inflate_copyright         004cd7f0     zlib:inftrees.obj
 0002:0000d920       __FPinit                   004cd920     LIBCMT:fpinit.obj
 0002:0000d924       __FPmtinit                 004cd924     LIBCMT:fpinit.obj
 0002:0000d928       __FPmtterm                 004cd928     LIBCMT:fpinit.obj
 0002:0000d930       ??_7type_info@@6B@         004cd930     LIBCMT:typinfo.obj
 0002:0000d934       ??_C@_03LLEJOLGL@?4?1?2?$AA@ 004cd934     LIBCMT:stati32.obj
 0002:0000d938       ??_C@_02EAOCEIGI@?$DP?$CK?$AA@ 004cd938     LIBCMT:stati32.obj
 0002:0000d940       ??_7bad_alloc@std@@6B@     004cd940     LIBCMT:new.obj
 0002:0000d948       ??_C@_0EA@FCLIIPNN@Visual?5C?$CL?$CL?5CRT?3?5Not?5enough?5memor@ 004cd948     LIBCMT:strerror.obj
 0002:0000d988       ??_C@_0P@MIGLKIOC@CorExitProcess?$AA@ 004cd988     LIBCMT:crt0dat.obj
 0002:0000d998       ??_C@_0M@MBOPBNBK@mscoree?4dll?$AA@ 004cd998     LIBCMT:crt0dat.obj
 0002:0000da00       ?ProcessDetach@NativeDll@<CrtImplementationDetails>@@0IB 004cda00     LIBCMT:strtol.obj
 0002:0000da04       ?ProcessAttach@NativeDll@<CrtImplementationDetails>@@0IB 004cda04     LIBCMT:strtol.obj
 0002:0000da08       ?ThreadAttach@NativeDll@<CrtImplementationDetails>@@0IB 004cda08     LIBCMT:strtol.obj
 0002:0000da0c       ?ThreadDetach@NativeDll@<CrtImplementationDetails>@@0IB 004cda0c     LIBCMT:strtol.obj
 0002:0000da10       ?ProcessVerifier@NativeDll@<CrtImplementationDetails>@@0IB 004cda10     LIBCMT:strtol.obj
 0002:0000dd58       ??_C@_02CLFPBFFP@TZ?$AA@   004cdd58     LIBCMT:tzset.obj
 0002:0000dd5c       ??_C@_05KLBDPFGC@e?$CL000?$AA@ 004cdd5c     LIBCMT:cvt.obj
 0002:0000dd68       __real@4150017ec0000000    004cdd68     LIBCMT:testfdiv.obj
 0002:0000dd70       __real@4147ffff80000000    004cdd70     LIBCMT:testfdiv.obj
 0002:0000dd78       ??_C@_0BK@NHEOCAHP@IsProcessorFeaturePresent?$AA@ 004cdd78     LIBCMT:testfdiv.obj
 0002:0000dd94       ??_C@_08CPNIBGIE@KERNEL32?$AA@ 004cdd94     LIBCMT:testfdiv.obj
 0002:0000dda0       ??_C@_0P@GGKDKEEG@runtime?5error?5?$AA@ 004cdda0     LIBCMT:crt0msg.obj
 0002:0000ddb0       ??_C@_0O@MJNIPGOH@TLOSS?5error?$AN?6?$AA@ 004cddb0     LIBCMT:crt0msg.obj
 0002:0000ddc0       ??_C@_0N@BONNPDHF@SING?5error?$AN?6?$AA@ 004cddc0     LIBCMT:crt0msg.obj
 0002:0000ddd0       ??_C@_0P@MBDAJNE@DOMAIN?5error?$AN?6?$AA@ 004cddd0     LIBCMT:crt0msg.obj
 0002:0000dde0       ??_C@_0JL@DFDOOABL@R6034?$AN?6An?5application?5has?5made?5a@ 004cdde0     LIBCMT:crt0msg.obj
 0002:0000de80       ??_C@_0PH@EPAFIJ@R6033?$AN?6?9?5Attempt?5to?5use?5MSIL?5cod@ 004cde80     LIBCMT:crt0msg.obj
 0002:0000df78       ??_C@_0DD@BKEEABMM@R6032?$AN?6?9?5not?5enough?5space?5for?5lo@ 004cdf78     LIBCMT:crt0msg.obj
 0002:0000dfb0       ??_C@_0GD@OFKILIED@R6031?$AN?6?9?5Attempt?5to?5initialize?5t@ 004cdfb0     LIBCMT:crt0msg.obj
 0002:0000e014       ??_C@_0BP@LPMHJOKI@R6030?$AN?6?9?5CRT?5not?5initialized?$AN?6?$AA@ 004ce014     LIBCMT:crt0msg.obj
 0002:0000e034       ??_C@_0CF@KJDAIALP@R6028?$AN?6?9?5unable?5to?5initialize?5he@ 004ce034     LIBCMT:crt0msg.obj
 0002:0000e05c       ??_C@_0DF@GAKBPDFP@R6027?$AN?6?9?5not?5enough?5space?5for?5lo@ 004ce05c     LIBCMT:crt0msg.obj
 0002:0000e094       ??_C@_0DF@IBLNNAIG@R6026?$AN?6?9?5not?5enough?5space?5for?5st@ 004ce094     LIBCMT:crt0msg.obj
 0002:0000e0cc       ??_C@_0CG@IOHKGFNJ@R6025?$AN?6?9?5pure?5virtual?5function?5c@ 004ce0cc     LIBCMT:crt0msg.obj
 0002:0000e0f4       ??_C@_0DF@JIJJFJDC@R6024?$AN?6?9?5not?5enough?5space?5for?5_o@ 004ce0f4     LIBCMT:crt0msg.obj
 0002:0000e12c       ??_C@_0CJ@EGEJHFME@R6019?$AN?6?9?5unable?5to?5open?5console?5@ 004ce12c     LIBCMT:crt0msg.obj
 0002:0000e158       ??_C@_0CB@GNHNIELH@R6018?$AN?6?9?5unexpected?5heap?5error?$AN?6@ 004ce158     LIBCMT:crt0msg.obj
 0002:0000e17c       ??_C@_0CN@FOLDKNG@R6017?$AN?6?9?5unexpected?5multithread?5@ 004ce17c     LIBCMT:crt0msg.obj
 0002:0000e1ac       ??_C@_0CM@FAHFJNHO@R6016?$AN?6?9?5not?5enough?5space?5for?5th@ 004ce1ac     LIBCMT:crt0msg.obj
 0002:0000e1d8       ??_C@_0JG@LBKMGKLD@?$AN?6This?5application?5has?5requested@ 004ce1d8     LIBCMT:crt0msg.obj
 0002:0000e270       ??_C@_0CM@FLCNIPKK@R6009?$AN?6?9?5not?5enough?5space?5for?5en@ 004ce270     LIBCMT:crt0msg.obj
 0002:0000e29c       ??_C@_0CK@KMMJOAPP@R6008?$AN?6?9?5not?5enough?5space?5for?5ar@ 004ce29c     LIBCMT:crt0msg.obj
 0002:0000e2c8       ??_C@_0CN@LEKKICBM@R6002?$AN?6?9?5floating?5point?5support?5@ 004ce2c8     LIBCMT:crt0msg.obj
 0002:0000e2f8       ??_C@_0CF@GOGNBNAK@Microsoft?5Visual?5C?$CL?$CL?5Runtime?5Lib@ 004ce2f8     LIBCMT:crt0msg.obj
 0002:0000e320       ??_C@_02PHMGELLB@?6?6?$AA@ 004ce320     LIBCMT:crt0msg.obj
 0002:0000e324       ??_C@_03KHICJKCI@?4?4?4?$AA@ 004ce324     LIBCMT:crt0msg.obj
 0002:0000e328       ??_C@_0BH@DNAGHKFM@?$DMprogram?5name?5unknown?$DO?$AA@ 004ce328     LIBCMT:crt0msg.obj
 0002:0000e340       ??_C@_0BK@OFGJDLJJ@Runtime?5Error?$CB?6?6Program?3?5?$AA@ 004ce340     LIBCMT:crt0msg.obj
 0002:0000e35c       ??_C@_07EPKMNAGK@?4mixcrt?$AA@ 004ce35c     LIBCMT:tidtable.obj
 0002:0000e364       ??_C@_0O@NLDKAIKN@EncodePointer?$AA@ 004ce364     LIBCMT:tidtable.obj
 0002:0000e374       ??_C@_0N@NHGLKGEC@KERNEL32?4DLL?$AA@ 004ce374     LIBCMT:tidtable.obj
 0002:0000e384       ??_C@_0O@KBPMFGHI@DecodePointer?$AA@ 004ce384     LIBCMT:tidtable.obj
 0002:0000e394       ??_C@_07PEJMOBNF@FlsFree?$AA@ 004ce394     LIBCMT:tidtable.obj
 0002:0000e39c       ??_C@_0M@JCPCPOEF@FlsSetValue?$AA@ 004ce39c     LIBCMT:tidtable.obj
 0002:0000e3a8       ??_C@_0M@GDNOONDI@FlsGetValue?$AA@ 004ce3a8     LIBCMT:tidtable.obj
 0002:0000e3b4       ??_C@_08KNHFBNJ@FlsAlloc?$AA@ 004ce3b4     LIBCMT:tidtable.obj
 0002:0000e3c0       ??_C@_04PNGHFIJN@?4com?$AA@ 004ce3c0     LIBCMT:stat.obj
 0002:0000e3c8       ??_C@_04NEEFLLOK@?4bat?$AA@ 004ce3c8     LIBCMT:stat.obj
 0002:0000e3d0       ??_C@_04CPCBDHLK@?4cmd?$AA@ 004ce3d0     LIBCMT:stat.obj
 0002:0000e3d8       ??_C@_04JLMDILM@?4exe?$AA@ 004ce3d8     LIBCMT:stat.obj
 0002:0000e3ec       ??_7exception@std@@6B@     004ce3ec     LIBCMT:stdexcpt.obj
 0002:0000e3f4       ??_C@_0BC@EOODALEL@Unknown?5exception?$AA@ 004ce3f4     LIBCMT:stdexcpt.obj
 0002:0000e40c       ??_7bad_cast@std@@6B@      004ce40c     LIBCMT:stdexcpt.obj
 0002:0000e418       ??_7bad_typeid@std@@6B@    004ce418     LIBCMT:stdexcpt.obj
 0002:0000e424       ??_7__non_rtti_object@std@@6B@ 004ce424     LIBCMT:stdexcpt.obj
 0002:0000e44c       ??_C@_0BG@KLEAJEFJ@Illegal?5byte?5sequence?$AA@ 004ce44c     LIBCMT:syserr.obj
 0002:0000e464       ??_C@_0BE@ICMCHPHH@Directory?5not?5empty?$AA@ 004ce464     LIBCMT:syserr.obj
 0002:0000e478       ??_C@_0BJ@IHEHINLI@Function?5not?5implemented?$AA@ 004ce478     LIBCMT:syserr.obj
 0002:0000e494       ??_C@_0BD@CLHBCGPB@No?5locks?5available?$AA@ 004ce494     LIBCMT:syserr.obj
 0002:0000e4a8       ??_C@_0BC@BEDIHIDK@Filename?5too?5long?$AA@ 004ce4a8     LIBCMT:syserr.obj
 0002:0000e4bc       ??_C@_0BK@JAEBMJJM@Resource?5deadlock?5avoided?$AA@ 004ce4bc     LIBCMT:syserr.obj
 0002:0000e4d8       ??_C@_0BB@FCBJFCAJ@Result?5too?5large?$AA@ 004ce4d8     LIBCMT:syserr.obj
 0002:0000e4ec       ??_C@_0N@MMJPGLJK@Domain?5error?$AA@ 004ce4ec     LIBCMT:syserr.obj
 0002:0000e4fc       ??_C@_0M@LHEPIIOM@Broken?5pipe?$AA@ 004ce4fc     LIBCMT:syserr.obj
 0002:0000e508       ??_C@_0P@PKCJJLLM@Too?5many?5links?$AA@ 004ce508     LIBCMT:syserr.obj
 0002:0000e518       ??_C@_0BG@DDBFNKBH@Read?9only?5file?5system?$AA@ 004ce518     LIBCMT:syserr.obj
 0002:0000e530       ??_C@_0N@FEHLOILP@Invalid?5seek?$AA@ 004ce530     LIBCMT:syserr.obj
 0002:0000e540       ??_C@_0BI@FEALHKLD@No?5space?5left?5on?5device?$AA@ 004ce540     LIBCMT:syserr.obj
 0002:0000e558       ??_C@_0P@LFMMIPAE@File?5too?5large?$AA@ 004ce558     LIBCMT:syserr.obj
 0002:0000e568       ??_C@_0CE@ONOKNLPF@Inappropriate?5I?1O?5control?5operat@ 004ce568     LIBCMT:syserr.obj
 0002:0000e58c       ??_C@_0BE@INBJMKGG@Too?5many?5open?5files?$AA@ 004ce58c     LIBCMT:syserr.obj
 0002:0000e5a0       ??_C@_0BO@IIFBODJE@Too?5many?5open?5files?5in?5system?$AA@ 004ce5a0     LIBCMT:syserr.obj
 0002:0000e5c0       ??_C@_0BB@HMGGCEBG@Invalid?5argument?$AA@ 004ce5c0     LIBCMT:syserr.obj
 0002:0000e5d4       ??_C@_0P@NDHGCGKE@Is?5a?5directory?$AA@ 004ce5d4     LIBCMT:syserr.obj
 0002:0000e5e4       ??_C@_0BA@CJBACOOL@Not?5a?5directory?$AA@ 004ce5e4     LIBCMT:syserr.obj
 0002:0000e5f4       ??_C@_0P@NLEIANHE@No?5such?5device?$AA@ 004ce5f4     LIBCMT:syserr.obj
 0002:0000e604       ??_C@_0O@OAMDNOCP@Improper?5link?$AA@ 004ce604     LIBCMT:syserr.obj
 0002:0000e614       ??_C@_0M@NAAJNNGH@File?5exists?$AA@ 004ce614     LIBCMT:syserr.obj
 0002:0000e620       ??_C@_0BA@BIBLIOEK@Resource?5device?$AA@ 004ce620     LIBCMT:syserr.obj
 0002:0000e630       ??_C@_0O@NIPGCINC@Unknown?5error?$AA@ 004ce630     LIBCMT:syserr.obj
 0002:0000e640       ??_C@_0M@LOEHLCJD@Bad?5address?$AA@ 004ce640     LIBCMT:syserr.obj
 0002:0000e64c       ??_C@_0BC@HFNFNKAI@Permission?5denied?$AA@ 004ce64c     LIBCMT:syserr.obj
 0002:0000e660       ??_C@_0BB@IMDKMPFB@Not?5enough?5space?$AA@ 004ce660     LIBCMT:syserr.obj
 0002:0000e674       ??_C@_0CB@EPFKGNAK@Resource?5temporarily?5unavailable@ 004ce674     LIBCMT:syserr.obj
 0002:0000e698       ??_C@_0BD@LOHELEP@No?5child?5processes?$AA@ 004ce698     LIBCMT:syserr.obj
 0002:0000e6ac       ??_C@_0BE@NFGDDCEF@Bad?5file?5descriptor?$AA@ 004ce6ac     LIBCMT:syserr.obj
 0002:0000e6c0       ??_C@_0BC@HKPNECK@Exec?5format?5error?$AA@ 004ce6c0     LIBCMT:syserr.obj
 0002:0000e6d4       ??_C@_0BC@MFFGCDFL@Arg?5list?5too?5long?$AA@ 004ce6d4     LIBCMT:syserr.obj
 0002:0000e6e8       ??_C@_0BK@DPKMCKJ@No?5such?5device?5or?5address?$AA@ 004ce6e8     LIBCMT:syserr.obj
 0002:0000e704       ??_C@_0BD@KKNFOBBD@Input?1output?5error?$AA@ 004ce704     LIBCMT:syserr.obj
 0002:0000e718       ??_C@_0BK@FJBOAFDK@Interrupted?5function?5call?$AA@ 004ce718     LIBCMT:syserr.obj
 0002:0000e734       ??_C@_0BA@FKIAIBGA@No?5such?5process?$AA@ 004ce734     LIBCMT:syserr.obj
 0002:0000e744       ??_C@_0BK@FMDHKPNF@No?5such?5file?5or?5directory?$AA@ 004ce744     LIBCMT:syserr.obj
 0002:0000e760       ??_C@_0BI@BJFCGOHL@Operation?5not?5permitted?$AA@ 004ce760     LIBCMT:syserr.obj
 0002:0000e778       ??_C@_1O@CEDCILHN@?$AA?$CI?$AAn?$AAu?$AAl?$AAl?$AA?$CJ?$AA?$AA@ 004ce778     LIBCMT:output.obj
 0002:0000e788       ___lookuptable             004ce788     LIBCMT:output.obj
 0002:0000e7e4       ??_C@_0BC@JEAENNKH@SystemFunction036?$AA@ 004ce7e4     LIBCMT:rand_s.obj
 0002:0000e7f8       ??_C@_0N@JJPEKNFO@ADVAPI32?4DLL?$AA@ 004ce7f8     LIBCMT:rand_s.obj
 0002:0000e808       ??_C@_0CG@PKBDLMEO@InitializeCriticalSectionAndSpin@ 004ce808     LIBCMT:initcrit.obj
 0002:0000e830       ___lookuptable_s           004ce830     LIBCMT:outputs.obj
 0002:0000e8f8       ??_C@_03IIINPABG@tan?$AA@  004ce8f8     LIBCMT:libm_error.obj
 0002:0000e8fc       ??_C@_03LALBNOCG@cos?$AA@  004ce8fc     LIBCMT:libm_error.obj
 0002:0000e900       ??_C@_03BLEJJJBH@sin?$AA@  004ce900     LIBCMT:libm_error.obj
 0002:0000e904       ??_C@_04EHEDPDJG@modf?$AA@ 004ce904     LIBCMT:libm_error.obj
 0002:0000e90c       ??_C@_05PBJFFIGL@floor?$AA@ 004ce90c     LIBCMT:libm_error.obj
 0002:0000e914       ??_C@_04GFPJNGEK@ceil?$AA@ 004ce914     LIBCMT:libm_error.obj
 0002:0000e91c       ??_C@_04MLLJIGOK@atan?$AA@ 004ce91c     LIBCMT:libm_error.obj
 0002:0000e924       ??_C@_05EOHGHCHD@exp10?$AA@ 004ce924     LIBCMT:libm_error.obj
 0002:0000e92c       ??_C@_04PDIFKINK@acos?$AA@ 004ce92c     LIBCMT:libm_error.obj
 0002:0000e934       ??_C@_04FIHNOPOL@asin?$AA@ 004ce934     LIBCMT:libm_error.obj
 0002:0000e93c       ??_C@_03MGHMBJCF@log?$AA@  004ce93c     LIBCMT:libm_error.obj
 0002:0000e940       ??_C@_05HGHHAHAP@log10?$AA@ 004ce940     LIBCMT:libm_error.obj
 0002:0000e948       ??_C@_03KHJOGHMM@exp?$AA@  004ce948     LIBCMT:libm_error.obj
 0002:0000e94c       ??_C@_03JGHBODFD@pow?$AA@  004ce94c     LIBCMT:libm_error.obj
 0002:0000e950       ??_C@_07LCBHPJJN@LC_TIME?$AA@ 004ce950     LIBCMT:setlocal.obj
 0002:0000e958       ??_C@_0L@DLHIECNL@LC_NUMERIC?$AA@ 004ce958     LIBCMT:setlocal.obj
 0002:0000e964       ??_C@_0M@MIENIKLA@LC_MONETARY?$AA@ 004ce964     LIBCMT:setlocal.obj
 0002:0000e970       ??_C@_08EADHIDAD@LC_CTYPE?$AA@ 004ce970     LIBCMT:setlocal.obj
 0002:0000e97c       ??_C@_0L@KFJHEKIK@LC_COLLATE?$AA@ 004ce97c     LIBCMT:setlocal.obj
 0002:0000e988       ??_C@_06NEFDFEKB@LC_ALL?$AA@ 004ce988     LIBCMT:setlocal.obj
 0002:0000e990       ___lc_category             004ce990     LIBCMT:setlocal.obj
 0002:0000ea58       ??_C@_03EGDHDPFD@_?4?0?$AA@ 004cea58     LIBCMT:setlocal.obj
 0002:0000ea5c       ??_C@_01IDAFKMJL@_?$AA@    004cea5c     LIBCMT:setlocal.obj
 0002:0000ea60       ??_C@_01ICJEACDI@?$DL?$AA@ 004cea60     LIBCMT:setlocal.obj
 0002:0000ea64       ??_C@_02BALPLPBG@?$DN?$DL?$AA@ 004cea64     LIBCMT:setlocal.obj
 0002:0000ea68       ??_C@_06GDENEHCP@CONIN$?$AA@ 004cea68     LIBCMT:initcon.obj
 0002:0000ea70       ??_C@_07GPDNMNG@CONOUT$?$AA@ 004cea70     LIBCMT:initcon.obj
 0002:0000ea78       ___dnames                  004cea78     LIBCMT:timeset.obj
 0002:0000ea90       ___mnames                  004cea90     LIBCMT:timeset.obj
 0002:0000eadc       ??_C@_0L@KDOEJCKC@_nextafter?$AA@ 004ceadc     LIBCMT:fpexcept.obj
 0002:0000eae8       ??_C@_05JGDBENOH@_logb?$AA@ 004ceae8     LIBCMT:fpexcept.obj
 0002:0000eaf0       ??_C@_03ONILCKOB@_yn?$AA@  004ceaf0     LIBCMT:fpexcept.obj
 0002:0000eaf4       ??_C@_03NAKIGLHK@_y1?$AA@  004ceaf4     LIBCMT:fpexcept.obj
 0002:0000eaf8       ??_C@_03MJLDFKDL@_y0?$AA@  004ceaf8     LIBCMT:fpexcept.obj
 0002:0000eafc       ??_C@_05GKKHEGJL@frexp?$AA@ 004ceafc     LIBCMT:fpexcept.obj
 0002:0000eb04       ??_C@_04KEPJIHGP@fmod?$AA@ 004ceb04     LIBCMT:fpexcept.obj
 0002:0000eb0c       ??_C@_06MEIMCGCF@_hypot?$AA@ 004ceb0c     LIBCMT:fpexcept.obj
 0002:0000eb14       ??_C@_05KBKMEMPO@_cabs?$AA@ 004ceb14     LIBCMT:fpexcept.obj
 0002:0000eb1c       ??_C@_05CEJMAHNP@ldexp?$AA@ 004ceb1c     LIBCMT:fpexcept.obj
 0002:0000eb24       ??_C@_04ODHECPBC@fabs?$AA@ 004ceb24     LIBCMT:fpexcept.obj
 0002:0000eb2c       ??_C@_04EIAKFFMI@sqrt?$AA@ 004ceb2c     LIBCMT:fpexcept.obj
 0002:0000eb34       ??_C@_05KNGEOGJB@atan2?$AA@ 004ceb34     LIBCMT:fpexcept.obj
 0002:0000eb3c       ??_C@_04FJHINJAO@tanh?$AA@ 004ceb3c     LIBCMT:fpexcept.obj
 0002:0000eb44       ??_C@_04HPJJNFIM@cosh?$AA@ 004ceb44     LIBCMT:fpexcept.obj
 0002:0000eb4c       ??_C@_04COOMCNPB@sinh?$AA@ 004ceb4c     LIBCMT:fpexcept.obj
 0002:0000eb54       ??_C@_0BK@CFCOFLF@?5Complete?5Object?5Locator?8?$AA@ 004ceb54     LIBCMT:undname.obj
 0002:0000eb70       ??_C@_0BN@MECKDCOJ@?5Class?5Hierarchy?5Descriptor?8?$AA@ 004ceb70     LIBCMT:undname.obj
 0002:0000eb90       ??_C@_0BD@LGICGFMM@?5Base?5Class?5Array?8?$AA@ 004ceb90     LIBCMT:undname.obj
 0002:0000eba4       ??_C@_0BM@LDKODKLH@?5Base?5Class?5Descriptor?5at?5?$CI?$AA@ 004ceba4     LIBCMT:undname.obj
 0002:0000ebc0       ??_C@_0BC@DAFEJGAK@?5Type?5Descriptor?8?$AA@ 004cebc0     LIBCMT:undname.obj
 0002:0000ebd4       ??_C@_0BM@PMGGMLDN@?$GAlocal?5static?5thread?5guard?8?$AA@ 004cebd4     LIBCMT:undname.obj
 0002:0000ebf0       ??_C@_0CL@FGIJHLCE@?$GAmanaged?5vector?5copy?5constructor@ 004cebf0     LIBCMT:undname.obj
 0002:0000ec1c       ??_C@_0CJ@GJELGAMM@?$GAvector?5vbase?5copy?5constructor?5i@ 004cec1c     LIBCMT:undname.obj
 0002:0000ec48       ??_C@_0CD@CGAJBKEJ@?$GAvector?5copy?5constructor?5iterato@ 004cec48     LIBCMT:undname.obj
 0002:0000ec6c       ??_C@_0CB@PDBIFEP@?$GAdynamic?5atexit?5destructor?5for?5?8@ 004cec6c     LIBCMT:undname.obj
 0002:0000ec90       ??_C@_0BL@CLIPGLGB@?$GAdynamic?5initializer?5for?5?8?$AA@ 004cec90     LIBCMT:undname.obj
 0002:0000ecac       ??_C@_0CM@FCBBDIGB@?$GAeh?5vector?5vbase?5copy?5constructo@ 004cecac     LIBCMT:undname.obj
 0002:0000ecd8       ??_C@_0CG@HLDDJMAG@?$GAeh?5vector?5copy?5constructor?5iter@ 004cecd8     LIBCMT:undname.obj
 0002:0000ed00       ??_C@_0CF@IMGKMJNO@?$GAmanaged?5vector?5destructor?5itera@ 004ced00     LIBCMT:undname.obj
 0002:0000ed28       ??_C@_0CG@CFDHKGGD@?$GAmanaged?5vector?5constructor?5iter@ 004ced28     LIBCMT:undname.obj
 0002:0000ed50       ??_C@_0BN@CKNJLHMB@?$GAplacement?5delete?$FL?$FN?5closure?8?$AA@ 004ced50     LIBCMT:undname.obj
 0002:0000ed70       ??_C@_0BL@CNOONJFP@?$GAplacement?5delete?5closure?8?$AA@ 004ced70     LIBCMT:undname.obj
 0002:0000ed8c       ??_C@_0P@HJKNJFNN@?$GAomni?5callsig?8?$AA@ 004ced8c     LIBCMT:undname.obj
 0002:0000ed9c       ??_C@_09LBNFPBCA@?5delete?$FL?$FN?$AA@ 004ced9c     LIBCMT:undname.obj
 0002:0000eda8       ??_C@_06FHBGPFGH@?5new?$FL?$FN?$AA@ 004ceda8     LIBCMT:undname.obj
 0002:0000edb0       ??_C@_0CE@IIHCMGGL@?$GAlocal?5vftable?5constructor?5closu@ 004cedb0     LIBCMT:undname.obj
 0002:0000edd4       ??_C@_0BA@KKLDJDLB@?$GAlocal?5vftable?8?$AA@ 004cedd4     LIBCMT:undname.obj
 0002:0000ede4       ??_C@_05KHLCHHI@?$GARTTI?$AA@ 004cede4     LIBCMT:undname.obj
 0002:0000edec       ??_C@_03KLGMFNMG@?$GAEH?$AA@ 004cedec     LIBCMT:undname.obj
 0002:0000edf0       ??_C@_0BA@KBCDOMBN@?$GAudt?5returning?8?$AA@ 004cedf0     LIBCMT:undname.obj
 0002:0000ee00       ??_C@_0BL@LLKPOHJI@?$GAcopy?5constructor?5closure?8?$AA@ 004cee00     LIBCMT:undname.obj
 0002:0000ee1c       ??_C@_0CH@OOJPLCPH@?$GAeh?5vector?5vbase?5constructor?5ite@ 004cee1c     LIBCMT:undname.obj
 0002:0000ee44       ??_C@_0CA@GCEOPDGL@?$GAeh?5vector?5destructor?5iterator?8?$AA@ 004cee44     LIBCMT:undname.obj
 0002:0000ee64       ??_C@_0CB@JONCMFFK@?$GAeh?5vector?5constructor?5iterator?8@ 004cee64     LIBCMT:undname.obj
 0002:0000ee88       ??_C@_0BL@NILFHHPC@?$GAvirtual?5displacement?5map?8?$AA@ 004cee88     LIBCMT:undname.obj
 0002:0000eea4       ??_C@_0CE@IKBNEHA@?$GAvector?5vbase?5constructor?5iterat@ 004ceea4     LIBCMT:undname.obj
 0002:0000eec8       ??_C@_0BN@LFPFMEDL@?$GAvector?5destructor?5iterator?8?$AA@ 004ceec8     LIBCMT:undname.obj
 0002:0000eee8       ??_C@_0BO@PFGOCPJJ@?$GAvector?5constructor?5iterator?8?$AA@ 004ceee8     LIBCMT:undname.obj
 0002:0000ef08       ??_C@_0BN@IMDCHIKM@?$GAscalar?5deleting?5destructor?8?$AA@ 004cef08     LIBCMT:undname.obj
 0002:0000ef28       ??_C@_0BO@OBMKPJIG@?$GAdefault?5constructor?5closure?8?$AA@ 004cef28     LIBCMT:undname.obj
 0002:0000ef48       ??_C@_0BN@DEGPLNFK@?$GAvector?5deleting?5destructor?8?$AA@ 004cef48     LIBCMT:undname.obj
 0002:0000ef68       ??_C@_0BD@JDLKDPAB@?$GAvbase?5destructor?8?$AA@ 004cef68     LIBCMT:undname.obj
 0002:0000ef7c       ??_C@_08OBABFOLI@?$GAstring?8?$AA@ 004cef7c     LIBCMT:undname.obj
 0002:0000ef88       ??_C@_0BF@KDPPACIK@?$GAlocal?5static?5guard?8?$AA@ 004cef88     LIBCMT:undname.obj
 0002:0000efa0       ??_C@_08LLFFHHDJ@?$GAtypeof?8?$AA@ 004cefa0     LIBCMT:undname.obj
 0002:0000efac       ??_C@_07FEEIOKP@?$GAvcall?8?$AA@ 004cefac     LIBCMT:undname.obj
 0002:0000efb4       ??_C@_09BLBHBJP@?$GAvbtable?8?$AA@ 004cefb4     LIBCMT:undname.obj
 0002:0000efc0       ??_C@_09IFPLHPGF@?$GAvftable?8?$AA@ 004cefc0     LIBCMT:undname.obj
 0002:0000efcc       ??_C@_02MHEGNOJ@?$FO?$DN?$AA@ 004cefcc     LIBCMT:undname.obj
 0002:0000efd0       ??_C@_02DHLNPPGH@?$HM?$DN?$AA@ 004cefd0     LIBCMT:undname.obj
 0002:0000efd4       ??_C@_02FGJGFEAB@?$CG?$DN?$AA@ 004cefd4     LIBCMT:undname.obj
 0002:0000efd8       ??_C@_03CDNPDDLA@?$DM?$DM?$DN?$AA@ 004cefd8     LIBCMT:undname.obj
 0002:0000efdc       ??_C@_03IKFCCPFF@?$DO?$DO?$DN?$AA@ 004cefdc     LIBCMT:undname.obj
 0002:0000efe0       ??_C@_02FENAOKFI@?$CF?$DN?$AA@ 004cefe0     LIBCMT:undname.obj
 0002:0000efe4       ??_C@_02FJEHGPIO@?1?$DN?$AA@ 004cefe4     LIBCMT:undname.obj
 0002:0000efe8       ??_C@_02FKMDLLOA@?9?$DN?$AA@ 004cefe8     LIBCMT:undname.obj
 0002:0000efec       ??_C@_02FOEOMHFC@?$CL?$DN?$AA@ 004cefec     LIBCMT:undname.obj
 0002:0000eff0       ??_C@_02FPIMKNGF@?$CK?$DN?$AA@ 004ceff0     LIBCMT:undname.obj
 0002:0000eff4       ??_C@_02NONPIBCD@?$HM?$HM?$AA@ 004ceff4     LIBCMT:undname.obj
 0002:0000eff8       ??_C@_02PPKAJPJL@?$CG?$CG?$AA@ 004ceff8     LIBCMT:undname.obj
 0002:0000effc       ??_C@_01DNKMNLPK@?$HM?$AA@ 004ceffc     LIBCMT:undname.obj
 0002:0000f000       ??_C@_01JKBOJNNK@?$FO?$AA@ 004cf000     LIBCMT:undname.obj
 0002:0000f004       ??_C@_01PJKLJHI@?$HO?$AA@  004cf004     LIBCMT:undname.obj
 0002:0000f008       ??_C@_02HCKGKOFO@?$CI?$CJ?$AA@ 004cf008     LIBCMT:undname.obj
 0002:0000f00c       ??_C@_02EEKDKGMJ@?$DO?$DN?$AA@ 004cf00c     LIBCMT:undname.obj
 0002:0000f010       ??_C@_01PPODPGHN@?$DO?$AA@ 004cf010     LIBCMT:undname.obj
 0002:0000f014       ??_C@_02EHCHHCKH@?$DM?$DN?$AA@ 004cf014     LIBCMT:undname.obj
 0002:0000f018       ??_C@_01FGNFDNOH@?$CF?$AA@ 004cf018     LIBCMT:undname.obj
 0002:0000f01c       ??_C@_03MNHNFDLC@?9?$DO?$CK?$AA@ 004cf01c     LIBCMT:undname.obj
 0002:0000f020       ??_C@_01MIFGBAGJ@?$CL?$AA@ 004cf020     LIBCMT:undname.obj
 0002:0000f024       ??_C@_02ECNGHCIF@?$CL?$CL?$AA@ 004cf024     LIBCMT:undname.obj
 0002:0000f028       ??_C@_02HBOOOICD@?9?$DO?$AA@ 004cf028     LIBCMT:undname.obj
 0002:0000f02c       ??_C@_08LHJFAFGD@operator?$AA@ 004cf02c     LIBCMT:undname.obj
 0002:0000f038       ??_C@_02GPECMEKF@?$FL?$FN?$AA@ 004cf038     LIBCMT:undname.obj
 0002:0000f03c       ??_C@_02FDNJECIE@?$CB?$DN?$AA@ 004cf03c     LIBCMT:undname.obj
 0002:0000f040       ??_C@_02EGOFBIJA@?$DN?$DN?$AA@ 004cf040     LIBCMT:undname.obj
 0002:0000f044       ??_C@_01DCLJPIOD@?$CB?$AA@ 004cf044     LIBCMT:undname.obj
 0002:0000f048       ??_C@_02GPIOPFAK@?$DO?$DO?$AA@ 004cf048     LIBCMT:undname.obj
 0002:0000f04c       ??_C@_07FPCDHGMM@?5delete?$AA@ 004cf04c     LIBCMT:undname.obj
 0002:0000f054       ??_C@_04NIHEBCM@?5new?$AA@ 004cf054     LIBCMT:undname.obj
 0002:0000f05c       ??_C@_0M@GFIIJFMG@__unaligned?$AA@ 004cf05c     LIBCMT:undname.obj
 0002:0000f068       ??_C@_0L@PILCLIHE@__restrict?$AA@ 004cf068     LIBCMT:undname.obj
 0002:0000f074       ??_C@_07JOMMBBKO@__ptr64?$AA@ 004cf074     LIBCMT:undname.obj
 0002:0000f07c       ??_C@_09HIJEGCPM@__clrcall?$AA@ 004cf07c     LIBCMT:undname.obj
 0002:0000f088       ??_C@_0L@JMKHOMEK@__fastcall?$AA@ 004cf088     LIBCMT:undname.obj
 0002:0000f094       ??_C@_0L@NPHFGOKO@__thiscall?$AA@ 004cf094     LIBCMT:undname.obj
 0002:0000f0a0       ??_C@_09IFJBGAPI@__stdcall?$AA@ 004cf0a0     LIBCMT:undname.obj
 0002:0000f0ac       ??_C@_08GHMPAG@__pascal?$AA@ 004cf0ac     LIBCMT:undname.obj
 0002:0000f0b8       ??_C@_07KOLFKCDI@__cdecl?$AA@ 004cf0b8     LIBCMT:undname.obj
 0002:0000f0c0       ??_C@_08EHJDFFNH@__based?$CI?$AA@ 004cf0c0     LIBCMT:undname.obj
 0002:0000f254       ??_7DNameNode@@6B@         004cf254     LIBCMT:undname.obj
 0002:0000f264       ??_7charNode@@6B@          004cf264     LIBCMT:undname.obj
 0002:0000f274       ??_7pDNameNode@@6B@        004cf274     LIBCMT:undname.obj
 0002:0000f284       ??_7DNameStatusNode@@6B@   004cf284     LIBCMT:undname.obj
 0002:0000f294       ??_7pcharNode@@6B@         004cf294     LIBCMT:undname.obj
 0002:0000f2a0       ??_C@_04OKOHEJBO@?5?$DP?$DP?5?$AA@ 004cf2a0     LIBCMT:undname.obj
 0002:0000f2a8       ??_C@_06EEGAIFAK@?$HLflat?$HN?$AA@ 004cf2a8     LIBCMT:undname.obj
 0002:0000f2b0       ??_C@_05JIBOFOHK@?$HLfor?5?$AA@ 004cf2b0     LIBCMT:undname.obj
 0002:0000f2b8       ??_C@_0BN@IBLMMFAP@?$GAnon?9type?9template?9parameter?$AA@ 004cf2b8     LIBCMT:undname.obj
 0002:0000f2d8       ??_C@_09EBBEKKIH@unsigned?5?$AA@ 004cf2d8     LIBCMT:undname.obj
 0002:0000f2e4       ??_C@_05CJIMAING@long?5?$AA@ 004cf2e4     LIBCMT:undname.obj
 0002:0000f2ec       ??_C@_04LAHKHJMA@int?5?$AA@ 004cf2ec     LIBCMT:undname.obj
 0002:0000f2f4       ??_C@_06EHJMALKF@short?5?$AA@ 004cf2f4     LIBCMT:undname.obj
 0002:0000f2fc       ??_C@_05CIHEBHNO@char?5?$AA@ 004cf2fc     LIBCMT:undname.obj
 0002:0000f304       ??_C@_04GKJNKENE@void?$AA@ 004cf304     LIBCMT:undname.obj
 0002:0000f30c       ??_C@_0L@EGPHHEKN@?$DMellipsis?$DO?$AA@ 004cf30c     LIBCMT:undname.obj
 0002:0000f318       ??_C@_0M@ELJOJFFH@?0?$DMellipsis?$DO?$AA@ 004cf318     LIBCMT:undname.obj
 0002:0000f324       ??_C@_04EENFHACM@?0?4?4?4?$AA@ 004cf324     LIBCMT:undname.obj
 0002:0000f32c       ??_C@_07HDJPLPEK@?5throw?$CI?$AA@ 004cf32c     LIBCMT:undname.obj
 0002:0000f334       ??_C@_02GOGNNPBN@?$CJ?$FL?$AA@ 004cf334     LIBCMT:undname.obj
 0002:0000f338       ??_C@_02MDINNEEG@s?5?$AA@  004cf338     LIBCMT:undname.obj
 0002:0000f33c       ??_C@_0BE@EODMJLIF@?$GAtemplate?9parameter?$AA@ 004cf33c     LIBCMT:undname.obj
 0002:0000f350       ??_C@_01GEODFPGF@?8?$AA@   004cf350     LIBCMT:undname.obj
 0002:0000f354       ??_C@_04HIBGFPH@NULL?$AA@  004cf354     LIBCMT:undname.obj
 0002:0000f35c       ??_C@_0O@GKABPPIF@cli?3?3pin_ptr?$DM?$AA@ 004cf35c     LIBCMT:undname.obj
 0002:0000f36c       ??_C@_0M@EALIELKG@cli?3?3array?$DM?$AA@ 004cf36c     LIBCMT:undname.obj
 0002:0000f378       ??_C@_05BEFAKPML@void?5?$AA@ 004cf378     LIBCMT:undname.obj
 0002:0000f380       ??_C@_02OHHJMEON@?8?8?$AA@ 004cf380     LIBCMT:undname.obj
 0002:0000f384       ??_C@_0BG@JNJLAMPM@?$GAanonymous?5namespace?8?$AA@ 004cf384     LIBCMT:undname.obj
 0002:0000f39c       ??_C@_01NLNLIGKH@?$GA?$AA@ 004cf39c     LIBCMT:undname.obj
 0002:0000f3a0       ??_C@_0O@KHGCOMHP@generic?9type?9?$AA@ 004cf3a0     LIBCMT:undname.obj
 0002:0000f3b0       ??_C@_0BE@JAEOCHPE@template?9parameter?9?$AA@ 004cf3b0     LIBCMT:undname.obj
 0002:0000f3c4       ??_C@_02MOLJINC@?3?3?$AA@  004cf3c4     LIBCMT:undname.obj
 0002:0000f3c8       ??_C@_0P@GCIFDJCJ@?$GAunknown?5ecsu?8?$AA@ 004cf3c8     LIBCMT:undname.obj
 0002:0000f3d8       ??_C@_06MOJHIBMG@union?5?$AA@ 004cf3d8     LIBCMT:undname.obj
 0002:0000f3e0       ??_C@_07DIBCDNGL@struct?5?$AA@ 004cf3e0     LIBCMT:undname.obj
 0002:0000f3e8       ??_C@_06LJBABKPM@class?5?$AA@ 004cf3e8     LIBCMT:undname.obj
 0002:0000f3f0       ??_C@_05LJGMCFOG@enum?5?$AA@ 004cf3f0     LIBCMT:undname.obj
 0002:0000f3f8       ??_C@_08KOFANOFK@coclass?5?$AA@ 004cf3f8     LIBCMT:undname.obj
 0002:0000f404       ??_C@_0N@DLIEFKNA@cointerface?5?$AA@ 004cf404     LIBCMT:undname.obj
 0002:0000f414       ??_C@_02KCKGHPCA@?$CJ?5?$AA@ 004cf414     LIBCMT:undname.obj
 0002:0000f418       ??_C@_0M@DHNBOJMP@extern?5?$CCC?$CC?5?$AA@ 004cf418     LIBCMT:undname.obj
 0002:0000f424       ??_C@_08KJLFOPNE@?$FLthunk?$FN?3?$AA@ 004cf424     LIBCMT:undname.obj
 0002:0000f430       ??_C@_08GPDDCMKI@public?3?5?$AA@ 004cf430     LIBCMT:undname.obj
 0002:0000f43c       ??_C@_0M@GAIFPFIP@protected?3?5?$AA@ 004cf43c     LIBCMT:undname.obj
 0002:0000f448       ??_C@_09LAPHOOG@private?3?5?$AA@ 004cf448     LIBCMT:undname.obj
 0002:0000f454       ??_C@_08NIEOINHE@virtual?5?$AA@ 004cf454     LIBCMT:undname.obj
 0002:0000f460       ??_C@_07PGOEDBHP@static?5?$AA@ 004cf460     LIBCMT:undname.obj
 0002:0000f468       ??_C@_0DA@HGFJFBBE@?$GAtemplate?5static?5data?5member?5des@ 004cf468     LIBCMT:undname.obj
 0002:0000f498       ??_C@_0DB@ILEFOCIJ@?$GAtemplate?5static?5data?5member?5con@ 004cf498     LIBCMT:undname.obj
 0002:0000f4cc       ??_C@_0CB@KJDOOODE@?$GAlocal?5static?5destructor?5helper?8@ 004cf4cc     LIBCMT:undname.obj
 0002:0000f4f0       ??_C@_0L@HNGCOGAE@?$GAadjustor?$HL?$AA@ 004cf4f0     LIBCMT:undname.obj
 0002:0000f4fc       ??_C@_0L@GHPFDFH@?$GAvtordisp?$HL?$AA@ 004cf4fc     LIBCMT:undname.obj
 0002:0000f508       ??_C@_0N@CBHHHENL@?$GAvtordispex?$HL?$AA@ 004cf508     LIBCMT:undname.obj
 0002:0000f518       ??_C@_02IGFCGPIL@?$HN?8?$AA@ 004cf518     LIBCMT:undname.obj
 0002:0000f51c       ??_C@_03OPGICMGF@?$HN?8?5?$AA@ 004cf51c     LIBCMT:undname.obj
 0002:0000f520       ??_C@_06LIJLOJAG@const?5?$AA@ 004cf520     LIBCMT:undname.obj
 0002:0000f528       ??_C@_09GAIEOBLP@volatile?5?$AA@ 004cf528     LIBCMT:undname.obj
 0002:0000f534       ??_C@_04HEJADOOB@CV?3?5?$AA@ 004cf534     LIBCMT:undname.obj
 0002:0000f53c       ??_C@_08PABEKFH@volatile?$AA@ 004cf53c     LIBCMT:undname.obj
 0002:0000f548       ??_C@_09EFNPDFFP@?5volatile?$AA@ 004cf548     LIBCMT:undname.obj
 0002:0000f554       ??_C@_05BNCCCJPP@const?$AA@ 004cf554     LIBCMT:undname.obj
 0002:0000f55c       ??_C@_07EDHNAJHC@signed?5?$AA@ 004cf55c     LIBCMT:undname.obj
 0002:0000f564       ??_C@_06BNJCAIGJ@double?$AA@ 004cf564     LIBCMT:undname.obj
 0002:0000f56c       ??_C@_04DDKJGDCM@bool?$AA@ 004cf56c     LIBCMT:undname.obj
 0002:0000f574       ??_C@_07CLGGIAMF@wchar_t?$AA@ 004cf574     LIBCMT:undname.obj
 0002:0000f57c       ??_C@_08GAHOLHEO@__int128?$AA@ 004cf57c     LIBCMT:undname.obj
 0002:0000f588       ??_C@_07OFLPPHGP@__int32?$AA@ 004cf588     LIBCMT:undname.obj
 0002:0000f590       ??_C@_07LFCOJCAC@__int64?$AA@ 004cf590     LIBCMT:undname.obj
 0002:0000f598       ??_C@_07ICFHOGAF@__int16?$AA@ 004cf598     LIBCMT:undname.obj
 0002:0000f5a0       ??_C@_06GCICPBLB@__w64?5?$AA@ 004cf5a0     LIBCMT:undname.obj
 0002:0000f5a8       ??_C@_06EBGKOKIG@__int8?$AA@ 004cf5a8     LIBCMT:undname.obj
 0002:0000f5b0       ??_C@_05KNFBNCOH@float?$AA@ 004cf5b0     LIBCMT:undname.obj
 0002:0000f5b8       ??_C@_04GOKPGOLB@long?$AA@ 004cf5b8     LIBCMT:undname.obj
 0002:0000f5c0       ??_C@_03JBIPMCLC@int?$AA@  004cf5c0     LIBCMT:undname.obj
 0002:0000f5c4       ??_C@_05BFKKPKCG@short?$AA@ 004cf5c4     LIBCMT:undname.obj
 0002:0000f5cc       ??_C@_04ENMBGAPA@char?$AA@ 004cf5cc     LIBCMT:undname.obj
 0002:0000f5d4       ??_C@_0BI@DFKBFLJE@GetProcessWindowStation?$AA@ 004cf5d4     LIBCMT:crtmbox.obj
 0002:0000f5ec       ??_C@_0BK@CIDNPOGP@GetUserObjectInformationA?$AA@ 004cf5ec     LIBCMT:crtmbox.obj
 0002:0000f608       ??_C@_0BD@HHGDFDBJ@GetLastActivePopup?$AA@ 004cf608     LIBCMT:crtmbox.obj
 0002:0000f61c       ??_C@_0BA@HNOPNCHB@GetActiveWindow?$AA@ 004cf61c     LIBCMT:crtmbox.obj
 0002:0000f62c       ??_C@_0M@CHKKJDAI@MessageBoxA?$AA@ 004cf62c     LIBCMT:crtmbox.obj
 0002:0000f638       ??_C@_0L@NDEGIDAG@USER32?4DLL?$AA@ 004cf638     LIBCMT:crtmbox.obj
 0002:0000f644       ??_C@_13NOLLCAOD@?$AA?$AA?$AA?$AA@ 004cf644     LIBCMT:a_map.obj
 0002:0000f648       ___newctype                004cf648     LIBCMT:ctype.obj
 0002:0000f948       __wctype                   004cf948     LIBCMT:ctype.obj
 0002:0000fb50       ___newclmap                004cfb50     LIBCMT:ctype.obj
 0002:0000fcd0       ___newcumap                004cfcd0     LIBCMT:ctype.obj
 0002:0000fe50       ??_C@_08JCCMCCIL@HH?3mm?3ss?$AA@ 004cfe50     LIBCMT:strftime.obj
 0002:0000fe5c       ??_C@_0BE@CKGJFCPC@dddd?0?5MMMM?5dd?0?5yyyy?$AA@ 004cfe5c     LIBCMT:strftime.obj
 0002:0000fe70       ??_C@_08BPBNCDIB@MM?1dd?1yy?$AA@ 004cfe70     LIBCMT:strftime.obj
 0002:0000fe7c       ??_C@_02CJNFDJBF@PM?$AA@   004cfe7c     LIBCMT:strftime.obj
 0002:0000fe80       ??_C@_02DEDBPAFC@AM?$AA@   004cfe80     LIBCMT:strftime.obj
 0002:0000fe84       ??_C@_08EDHMEBNP@December?$AA@ 004cfe84     LIBCMT:strftime.obj
 0002:0000fe90       ??_C@_08HCHEGEOA@November?$AA@ 004cfe90     LIBCMT:strftime.obj
 0002:0000fe9c       ??_C@_07JJNFCEND@October?$AA@ 004cfe9c     LIBCMT:strftime.obj
 0002:0000fea4       ??_C@_09BHHEALKD@September?$AA@ 004cfea4     LIBCMT:strftime.obj
 0002:0000feb0       ??_C@_06LBBHFDDG@August?$AA@ 004cfeb0     LIBCMT:strftime.obj
 0002:0000feb8       ??_C@_04MIEPOIFP@July?$AA@ 004cfeb8     LIBCMT:strftime.obj
 0002:0000fec0       ??_C@_04CNLMGBGM@June?$AA@ 004cfec0     LIBCMT:strftime.obj
 0002:0000fec8       ??_C@_05DMJDNLEJ@April?$AA@ 004cfec8     LIBCMT:strftime.obj
 0002:0000fed0       ??_C@_05HPCKOFNC@March?$AA@ 004cfed0     LIBCMT:strftime.obj
 0002:0000fed8       ??_C@_08GNJGEPFN@February?$AA@ 004cfed8     LIBCMT:strftime.obj
 0002:0000fee4       ??_C@_07CGJPFGJA@January?$AA@ 004cfee4     LIBCMT:strftime.obj
 0002:0000feec       ??_C@_03MKABNOCG@Dec?$AA@  004cfeec     LIBCMT:strftime.obj
 0002:0000fef0       ??_C@_03JPJOFNIA@Nov?$AA@  004cfef0     LIBCMT:strftime.obj
 0002:0000fef4       ??_C@_03BMAOKBAD@Oct?$AA@  004cfef4     LIBCMT:strftime.obj
 0002:0000fef8       ??_C@_03GGCAPAJC@Sep?$AA@  004cfef8     LIBCMT:strftime.obj
 0002:0000fefc       ??_C@_03IFJFEIGA@Aug?$AA@  004cfefc     LIBCMT:strftime.obj
 0002:0000ff00       ??_C@_03LBGABGKK@Jul?$AA@  004cff00     LIBCMT:strftime.obj
 0002:0000ff04       ??_C@_03IDFGHECI@Jun?$AA@  004cff04     LIBCMT:strftime.obj
 0002:0000ff08       ??_C@_03CNMDKL@May?$AA@    004cff08     LIBCMT:strftime.obj
 0002:0000ff0c       ??_C@_03LEOLGMJP@Apr?$AA@  004cff0c     LIBCMT:strftime.obj
 0002:0000ff10       ??_C@_03ODNJBKGA@Mar?$AA@  004cff10     LIBCMT:strftime.obj
 0002:0000ff14       ??_C@_03HJBDCHOM@Feb?$AA@  004cff14     LIBCMT:strftime.obj
 0002:0000ff18       ??_C@_03JIHJHPIE@Jan?$AA@  004cff18     LIBCMT:strftime.obj
 0002:0000ff1c       ??_C@_08INBOOONO@Saturday?$AA@ 004cff1c     LIBCMT:strftime.obj
 0002:0000ff28       ??_C@_06JECMNKMI@Friday?$AA@ 004cff28     LIBCMT:strftime.obj
 0002:0000ff30       ??_C@_08HACCIKIA@Thursday?$AA@ 004cff30     LIBCMT:strftime.obj
 0002:0000ff3c       ??_C@_09DLIGFAKA@Wednesday?$AA@ 004cff3c     LIBCMT:strftime.obj
 0002:0000ff48       ??_C@_07BAAGCFCM@Tuesday?$AA@ 004cff48     LIBCMT:strftime.obj
 0002:0000ff50       ??_C@_06JLEDEDGH@Monday?$AA@ 004cff50     LIBCMT:strftime.obj
 0002:0000ff58       ??_C@_06OOPIFAJ@Sunday?$AA@ 004cff58     LIBCMT:strftime.obj
 0002:0000ff60       ??_C@_03FEFJNEK@Sat?$AA@   004cff60     LIBCMT:strftime.obj
 0002:0000ff64       ??_C@_03IDIOELNC@Fri?$AA@  004cff64     LIBCMT:strftime.obj
 0002:0000ff68       ??_C@_03IOFIKPDN@Thu?$AA@  004cff68     LIBCMT:strftime.obj
 0002:0000ff6c       ??_C@_03MHOMLAJA@Wed?$AA@  004cff6c     LIBCMT:strftime.obj
 0002:0000ff70       ??_C@_03NAGEINEP@Tue?$AA@  004cff70     LIBCMT:strftime.obj
 0002:0000ff74       ??_C@_03PDAGKDH@Mon?$AA@   004cff74     LIBCMT:strftime.obj
 0002:0000ff78       ??_C@_03KOEHGMDN@Sun?$AA@  004cff78     LIBCMT:strftime.obj
 0002:0000ff7c       ??_C@_03EBAPMIKO@a?1p?$AA@ 004cff7c     LIBCMT:strftime.obj
 0002:0000ff80       ??_C@_05JAMEPDIN@am?1pm?$AA@ 004cff80     LIBCMT:strftime.obj
 0002:0000ff88       ??_C@_0O@FMJNFNKE@united?9states?$AA@ 004cff88     LIBCMT:getqloc.obj
 0002:0000ff98       ??_C@_0P@NDHFFKCA@united?9kingdom?$AA@ 004cff98     LIBCMT:getqloc.obj
 0002:0000ffa8       ??_C@_0BC@HHDADLGF@trinidad?5?$CG?5tobago?$AA@ 004cffa8     LIBCMT:getqloc.obj
 0002:0000ffbc       ??_C@_0M@IOAEBDAC@south?9korea?$AA@ 004cffbc     LIBCMT:getqloc.obj
 0002:0000ffc8       ??_C@_0N@FIELFKIJ@south?9africa?$AA@ 004cffc8     LIBCMT:getqloc.obj
 0002:0000ffd8       ??_C@_0M@OPNDHCMC@south?5korea?$AA@ 004cffd8     LIBCMT:getqloc.obj
 0002:0000ffe4       ??_C@_0N@MDEOEPFI@south?5africa?$AA@ 004cffe4     LIBCMT:getqloc.obj
 0002:0000fff4       ??_C@_06FKAPCJLB@slovak?$AA@ 004cfff4     LIBCMT:getqloc.obj
 0002:0000fffc       ??_C@_0M@EFJANOAL@puerto?9rico?$AA@ 004cfffc     LIBCMT:getqloc.obj
 0002:00010008       ??_C@_08PGOJKDAI@pr?9china?$AA@ 004d0008     LIBCMT:getqloc.obj
 0002:00010014       ??_C@_08JHDOMCMI@pr?5china?$AA@ 004d0014     LIBCMT:getqloc.obj
 0002:00010020       ??_C@_02JHCHFBLL@nz?$AA@   004d0020     LIBCMT:getqloc.obj
 0002:00010024       ??_C@_0M@LINHDHKP@new?9zealand?$AA@ 004d0024     LIBCMT:getqloc.obj
 0002:00010030       ??_C@_09IIIPPBDB@hong?9kong?$AA@ 004d0030     LIBCMT:getqloc.obj
 0002:0001003c       ??_C@_07HJLCKBG@holland?$AA@ 004d003c     LIBCMT:getqloc.obj
 0002:00010044       ??_C@_0O@LEHGMHAG@great?5britain?$AA@ 004d0044     LIBCMT:getqloc.obj
 0002:00010054       ??_C@_07FACOMELA@england?$AA@ 004d0054     LIBCMT:getqloc.obj
 0002:0001005c       ??_C@_05JIHCEICB@czech?$AA@ 004d005c     LIBCMT:getqloc.obj
 0002:00010064       ??_C@_05BBJOBLGB@china?$AA@ 004d0064     LIBCMT:getqloc.obj
 0002:0001006c       ??_C@_07GPKPHICP@britain?$AA@ 004d006c     LIBCMT:getqloc.obj
 0002:00010074       ??_C@_07MHIPBHMG@america?$AA@ 004d0074     LIBCMT:getqloc.obj
 0002:0001007c       ??_C@_03KIALPMKC@usa?$AA@  004d007c     LIBCMT:getqloc.obj
 0002:00010080       ??_C@_02FGJGKGGD@us?$AA@   004d0080     LIBCMT:getqloc.obj
 0002:00010084       ??_C@_02NEINDODK@uk?$AA@   004d0084     LIBCMT:getqloc.obj
 0002:00010088       ??_C@_05JMPCFJFJ@swiss?$AA@ 004d0088     LIBCMT:getqloc.obj
 0002:00010090       ??_C@_0BA@HLOCPIOD@swedish?9finland?$AA@ 004d0090     LIBCMT:getqloc.obj
 0002:000100a0       ??_C@_0BC@PKCNIABK@spanish?9venezuela?$AA@ 004d00a0     LIBCMT:getqloc.obj
 0002:000100b4       ??_C@_0BA@GBHHMIJI@spanish?9uruguay?$AA@ 004d00b4     LIBCMT:getqloc.obj
 0002:000100c4       ??_C@_0BE@BHDOHPMC@spanish?9puerto?5rico?$AA@ 004d00c4     LIBCMT:getqloc.obj
 0002:000100d8       ??_C@_0N@KMOIDGGN@spanish?9peru?$AA@ 004d00d8     LIBCMT:getqloc.obj
 0002:000100e8       ??_C@_0BB@HMHLPGPH@spanish?9paraguay?$AA@ 004d00e8     LIBCMT:getqloc.obj
 0002:000100fc       ??_C@_0P@MCPKNGFD@spanish?9panama?$AA@ 004d00fc     LIBCMT:getqloc.obj
 0002:0001010c       ??_C@_0BC@IHOHGAIL@spanish?9nicaragua?$AA@ 004d010c     LIBCMT:getqloc.obj
 0002:00010120       ??_C@_0P@KLMJDNFJ@spanish?9modern?$AA@ 004d0120     LIBCMT:getqloc.obj
 0002:00010130       ??_C@_0BA@BPAPGBCM@spanish?9mexican?$AA@ 004d0130     LIBCMT:getqloc.obj
 0002:00010140       ??_C@_0BB@PDECHHHE@spanish?9honduras?$AA@ 004d0140     LIBCMT:getqloc.obj
 0002:00010154       ??_C@_0BC@KLHKFGDB@spanish?9guatemala?$AA@ 004d0154     LIBCMT:getqloc.obj
 0002:00010168       ??_C@_0BE@MFOOKJAI@spanish?9el?5salvador?$AA@ 004d0168     LIBCMT:getqloc.obj
 0002:0001017c       ??_C@_0BA@FCOKFPFC@spanish?9ecuador?$AA@ 004d017c     LIBCMT:getqloc.obj
 0002:0001018c       ??_C@_0BL@PLMGIMOO@spanish?9dominican?5republic?$AA@ 004d018c     LIBCMT:getqloc.obj
 0002:000101a8       ??_C@_0BD@HLGDNMHB@spanish?9costa?5rica?$AA@ 004d01a8     LIBCMT:getqloc.obj
 0002:000101bc       ??_C@_0BB@PKCBKCPE@spanish?9colombia?$AA@ 004d01bc     LIBCMT:getqloc.obj
 0002:000101d0       ??_C@_0O@MCBIJGNE@spanish?9chile?$AA@ 004d01d0     LIBCMT:getqloc.obj
 0002:000101e0       ??_C@_0BA@BEFEIGJJ@spanish?9bolivia?$AA@ 004d01e0     LIBCMT:getqloc.obj
 0002:000101f0       ??_C@_0BC@EMECMPD@spanish?9argentina?$AA@ 004d01f0     LIBCMT:getqloc.obj
 0002:00010204       ??_C@_0BF@EALFLENP@portuguese?9brazilian?$AA@ 004d0204     LIBCMT:getqloc.obj
 0002:0001021c       ??_C@_0BC@HBLEBLNN@norwegian?9nynorsk?$AA@ 004d021c     LIBCMT:getqloc.obj
 0002:00010230       ??_C@_0BB@HMACDDCK@norwegian?9bokmal?$AA@ 004d0230     LIBCMT:getqloc.obj
 0002:00010244       ??_C@_09BAFFPPHE@norwegian?$AA@ 004d0244     LIBCMT:getqloc.obj
 0002:00010250       ??_C@_0O@EAJFJDFG@italian?9swiss?$AA@ 004d0250     LIBCMT:getqloc.obj
 0002:00010260       ??_C@_0O@CNOMPGD@irish?9english?$AA@ 004d0260     LIBCMT:getqloc.obj
 0002:00010270       ??_C@_0N@EDHBGCKG@german?9swiss?$AA@ 004d0270     LIBCMT:getqloc.obj
 0002:00010280       ??_C@_0BC@JACMHNBP@german?9luxembourg?$AA@ 004d0280     LIBCMT:getqloc.obj
 0002:00010294       ??_C@_0BE@HBGMGFEG@german?9lichtenstein?$AA@ 004d0294     LIBCMT:getqloc.obj
 0002:000102a8       ??_C@_0BA@HKKBIBKL@german?9austrian?$AA@ 004d02a8     LIBCMT:getqloc.obj
 0002:000102b8       ??_C@_0N@GCAEPEBK@french?9swiss?$AA@ 004d02b8     LIBCMT:getqloc.obj
 0002:000102c8       ??_C@_0BC@DJFJJCK@french?9luxembourg?$AA@ 004d02c8     LIBCMT:getqloc.obj
 0002:000102dc       ??_C@_0BA@NNCEDFIC@french?9canadian?$AA@ 004d02dc     LIBCMT:getqloc.obj
 0002:000102ec       ??_C@_0P@CMPOCLM@french?9belgian?$AA@ 004d02ec     LIBCMT:getqloc.obj
 0002:000102fc       ??_C@_0M@GHHDJOK@english?9usa?$AA@ 004d02fc     LIBCMT:getqloc.obj
 0002:00010308       ??_C@_0L@PLDJKEIL@english?9us?$AA@ 004d0308     LIBCMT:getqloc.obj
 0002:00010314       ??_C@_0L@HJCCDMNC@english?9uk?$AA@ 004d0314     LIBCMT:getqloc.obj
 0002:00010320       ??_C@_0BK@CKLIAGJB@english?9trinidad?5y?5tobago?$AA@ 004d0320     LIBCMT:getqloc.obj
 0002:0001033c       ??_C@_0BF@JMJMGNNF@english?9south?5africa?$AA@ 004d033c     LIBCMT:getqloc.obj
 0002:00010354       ??_C@_0L@DKIIFDFD@english?9nz?$AA@ 004d0354     LIBCMT:getqloc.obj
 0002:00010360       ??_C@_0BA@ONHGJCLH@english?9jamaica?$AA@ 004d0360     LIBCMT:getqloc.obj
 0002:00010370       ??_C@_0M@HJBGHOPO@english?9ire?$AA@ 004d0370     LIBCMT:getqloc.obj
 0002:0001037c       ??_C@_0BC@LFEKMIFB@english?9caribbean?$AA@ 004d037c     LIBCMT:getqloc.obj
 0002:00010390       ??_C@_0M@OLDPFKHI@english?9can?$AA@ 004d0390     LIBCMT:getqloc.obj
 0002:0001039c       ??_C@_0P@OMDEHBMP@english?9belize?$AA@ 004d039c     LIBCMT:getqloc.obj
 0002:000103ac       ??_C@_0M@KFHFPFED@english?9aus?$AA@ 004d03ac     LIBCMT:getqloc.obj
 0002:000103b8       ??_C@_0BB@MNMBKDFE@english?9american?$AA@ 004d03b8     LIBCMT:getqloc.obj
 0002:000103cc       ??_C@_0O@KIDLNNBA@dutch?9belgian?$AA@ 004d03cc     LIBCMT:getqloc.obj
 0002:000103dc       ??_C@_0BE@JBKABBMH@chinese?9traditional?$AA@ 004d03dc     LIBCMT:getqloc.obj
 0002:000103f0       ??_C@_0BC@MJJMPKCG@chinese?9singapore?$AA@ 004d03f0     LIBCMT:getqloc.obj
 0002:00010404       ??_C@_0BD@FDKADDCP@chinese?9simplified?$AA@ 004d0404     LIBCMT:getqloc.obj
 0002:00010418       ??_C@_0BB@DBEFDDME@chinese?9hongkong?$AA@ 004d0418     LIBCMT:getqloc.obj
 0002:0001042c       ??_C@_07DHNMFMCI@chinese?$AA@ 004d042c     LIBCMT:getqloc.obj
 0002:00010434       ??_C@_03FNDDCHI@chi?$AA@   004d0434     LIBCMT:getqloc.obj
 0002:00010438       ??_C@_03BMMIADDJ@chh?$AA@  004d0438     LIBCMT:getqloc.obj
 0002:0001043c       ??_C@_08OAIPJDGI@canadian?$AA@ 004d043c     LIBCMT:getqloc.obj
 0002:00010448       ??_C@_07HBPMNPNJ@belgian?$AA@ 004d0448     LIBCMT:getqloc.obj
 0002:00010450       ??_C@_0L@OEKOPBEL@australian?$AA@ 004d0450     LIBCMT:getqloc.obj
 0002:0001045c       ??_C@_0BB@MEIMBEDG@american?9english?$AA@ 004d045c     LIBCMT:getqloc.obj
 0002:00010470       ??_C@_0BB@DFMDPDGB@american?5english?$AA@ 004d0470     LIBCMT:getqloc.obj
 0002:00010484       ??_C@_08IJLOKOLL@american?$AA@ 004d0484     LIBCMT:getqloc.obj
 0002:00010490       ___rg_language             004d0490     LIBCMT:getqloc.obj
 0002:00010698       ___rg_country              004d0698     LIBCMT:getqloc.obj
 0002:00010750       ___rglangidNotDefault      004d0750     LIBCMT:getqloc.obj
 0002:00010764       ??_C@_03NFKLAGEF@OCP?$AA@  004d0764     LIBCMT:getqloc.obj
 0002:00010768       ??_C@_03DFHEHBHG@ACP?$AA@  004d0768     LIBCMT:getqloc.obj
 0002:0001076c       ??_C@_0BC@NFIEMBLL@Norwegian?9Nynorsk?$AA@ 004d076c     LIBCMT:getqloc.obj
 0002:00010780       ??_C@_06IMKFLFPG@1?$CDQNAN?$AA@ 004d0780     LIBCMT:x10fout.obj
 0002:00010788       ??_C@_05DNEBIAHO@1?$CDINF?$AA@ 004d0788     LIBCMT:x10fout.obj
 0002:00010790       ??_C@_05PHHOCPM@1?$CDIND?$AA@ 004d0790     LIBCMT:x10fout.obj
 0002:00010798       ??_C@_06PGGFOGJG@1?$CDSNAN?$AA@ 004d0798     LIBCMT:x10fout.obj
 0002:000107a4       ??_7HASH64withTransform@TaoCrypt@@6B@ 004d07a4     taocrypt:hash.obj
 0002:000107cc       ??_7HASHwithTransform@TaoCrypt@@6B@ 004d07cc     taocrypt:hash.obj
 0002:000108d0       ??_7MultiplicativeGroupT@AbstractRing@TaoCrypt@@6B@ 004d08d0     taocrypt:integer.obj
 0002:0001090c       ??_7ModularArithmetic@TaoCrypt@@6B@ 004d090c     taocrypt:integer.obj
 0002:0001097c       ??_7MontgomeryRepresentation@TaoCrypt@@6B@ 004d097c     taocrypt:integer.obj
 0002:000109ec       ??_7EuclideanDomainOf@TaoCrypt@@6B@ 004d09ec     taocrypt:integer.obj
 0002:00010ddc       ??_7SHA256@TaoCrypt@@6B@   004d0ddc     taocrypt:sha.obj
 0002:00010e04       ??_7SHA224@TaoCrypt@@6B@   004d0e04     taocrypt:sha.obj
 0002:00010e2c       ??_7SHA512@TaoCrypt@@6B@   004d0e2c     taocrypt:sha.obj
 0002:00010e54       ??_7SHA384@TaoCrypt@@6B@   004d0e54     taocrypt:sha.obj
 0002:00010e78       ??_C@_0N@BDDFKIGD@GenuineIntel?$AA@ 004d0e78     taocrypt:misc.obj
 0002:00011720       ?Te@AES@TaoCrypt@@0QAY0BAA@$$CBIA 004d1720     taocrypt:aes.obj
 0002:00012b20       ?Td@AES@TaoCrypt@@0QAY0BAA@$$CBIA 004d2b20     taocrypt:aes.obj
 0002:00013f24       ??_7BER_Decoder@TaoCrypt@@6B@ 004d3f24     taocrypt:dsa.obj
 0002:00013f30       ??_7DSA_Private_Decoder@TaoCrypt@@6B@ 004d3f30     taocrypt:dsa.obj
 0002:00013f3c       ??_7DSA_Public_Decoder@TaoCrypt@@6B@ 004d3f3c     taocrypt:dsa.obj
 0002:00013f48       ??_7DH_Decoder@TaoCrypt@@6B@ 004d3f48     taocrypt:dh.obj
 0002:00013f50       __real@4014000000000000    004d3f50     taocrypt:dh.obj
 0002:00013f58       __real@4003333333333333    004d3f58     taocrypt:dh.obj
 0002:00013f60       __real@3fd5555555555555    004d3f60     taocrypt:dh.obj
 0002:00013f68       __real@3fe5555555555555    004d3f68     taocrypt:dh.obj
 0002:00013f74       ??_7RSA_Private_Decoder@TaoCrypt@@6B@ 004d3f74     taocrypt:rsa.obj
 0002:00013f80       ??_7RSA_Public_Decoder@TaoCrypt@@6B@ 004d3f80     taocrypt:rsa.obj
 0002:00013f8c       ??_7PKCS12_Decoder@TaoCrypt@@6B@ 004d3f8c     taocrypt:asn.obj
 0002:00013f98       ??_7DER_Encoder@TaoCrypt@@6B@ 004d3f98     taocrypt:asn.obj
 0002:00013fa0       ??_7CertDecoder@TaoCrypt@@6B@ 004d3fa0     taocrypt:asn.obj
 0002:00013fa8       ??_C@_0P@FGCJCCJK@?1emailAddress?$DN?$AA@ 004d3fa8     taocrypt:asn.obj
 0002:00013fb8       ??_C@_04LJKEFMLJ@?1OU?$DN?$AA@ 004d3fb8     taocrypt:asn.obj
 0002:00013fc0       ??_C@_03DHMEBNMI@?1O?$DN?$AA@ 004d3fc0     taocrypt:asn.obj
 0002:00013fc4       ??_C@_04KCKJNOKJ@?1ST?$DN?$AA@ 004d3fc4     taocrypt:asn.obj
 0002:00013fcc       ??_C@_03DFICKDJB@?1L?$DN?$AA@ 004d3fcc     taocrypt:asn.obj
 0002:00013fd0       ??_C@_03DONOOEKM@?1C?$DN?$AA@ 004d3fd0     taocrypt:asn.obj
 0002:00013fd4       ??_C@_04LDBIPIAP@?1SN?$DN?$AA@ 004d3fd4     taocrypt:asn.obj
 0002:00014000       ??_7Signature_Encoder@TaoCrypt@@6B@ 004d4000     taocrypt:asn.obj
 0002:00014004       ??_C@_02GMLFBBN@wb?$AA@    004d4004     taocrypt:file.obj
 0002:00014008       ??_C@_1CC@LJGHMMH@?$AAn?$AA?5?$AA?$DO?$AA?5?$AAo?$AAt?$AAh?$AAe?$AAr?$AA?4?$AAs?$AAi?$AAz?$AAe?$AA?$CI?$AA?$CJ?$AA?$AA@ 004d4008     taocrypt:algebra.obj
 0002:00014030       ??_C@_1LO@MLJPEKBP@?$AAG?$AA?3?$AA?2?$AAm?$AAy?$AAs?$AAq?$AAl?$AA?9?$AA5?$AA?4?$AA1?$AA?4?$AA4?$AA6?$AA?9?$AAw?$AAi?$AAn?$AAb?$AAu?$AAi?$AAl?$AAd?$AA?2?$AAm?$AAy?$AAs?$AAq?$AAl?$AA?9?$AAc@ 004d4030     taocrypt:algebra.obj
 0002:000140f0       ??_C@_1DA@DMJEOLMN@?$AAe?$AAx?$AAp?$AAB?$AAe?$AAg?$AAi?$AAn?$AA?9?$AA?$DO?$AAN?$AAo?$AAt?$AAN?$AAe?$AAg?$AAa?$AAt?$AAi?$AAv?$AAe?$AA?$CI?$AA?$CJ?$AA?$AA@ 004d40f0     taocrypt:algebra.obj
 0002:00014120       ??_C@_1CE@JDMHDBFO@?$AA?4?$AA?2?$AAs?$AAr?$AAc?$AA?2?$AAa?$AAl?$AAg?$AAe?$AAb?$AAr?$AAa?$AA?4?$AAc?$AAp?$AAp?$AA?$AA@ 004d4120     taocrypt:algebra.obj
 0002:00014144       ?rcon_@AES@TaoCrypt@@0QBIB 004d4144     taocrypt:aestables.obj
 0002:00014274       ??_7MD2@TaoCrypt@@6B@      004d4274     taocrypt:md2.obj
 0002:0001428c       ??_C@_15IABLJNFO@?$AA?6?$AA?6?$AA?$AA@ 004d428c     LIBCMT:wassert.obj
 0002:00014294       ??_C@_13LBAGMAIH@?$AA?6?$AA?$AA@ 004d4294     LIBCMT:wassert.obj
 0002:00014298       ??_C@_17LGKOMLJ@?$AA?4?$AA?4?$AA?4?$AA?$AA@ 004d4298     LIBCMT:wassert.obj
 0002:000142a0       ??_C@_1EK@MBDPDCGA@?$AAM?$AAi?$AAc?$AAr?$AAo?$AAs?$AAo?$AAf?$AAt?$AA?5?$AAV?$AAi?$AAs?$AAu?$AAa?$AAl?$AA?5?$AAC?$AA?$CL?$AA?$CL?$AA?5?$AAR?$AAu?$AAn?$AAt?$AAi?$AAm?$AAe?$AA?5?$AAL?$AAi?$AAb@ 004d42a0     LIBCMT:wassert.obj
 0002:000142f0       ??_C@_1HK@POCJMFGK@?$AA?$CI?$AAP?$AAr?$AAe?$AAs?$AAs?$AA?5?$AAR?$AAe?$AAt?$AAr?$AAy?$AA?5?$AAt?$AAo?$AA?5?$AAd?$AAe?$AAb?$AAu?$AAg?$AA?5?$AAt?$AAh?$AAe?$AA?5?$AAa?$AAp?$AAp?$AAl?$AAi?$AAc@ 004d42f0     LIBCMT:wassert.obj
 0002:00014370       ??_C@_1OA@EGMLFBHJ@?$AAF?$AAo?$AAr?$AA?5?$AAi?$AAn?$AAf?$AAo?$AAr?$AAm?$AAa?$AAt?$AAi?$AAo?$AAn?$AA?5?$AAo?$AAn?$AA?5?$AAh?$AAo?$AAw?$AA?5?$AAy?$AAo?$AAu?$AAr?$AA?5?$AAp?$AAr?$AAo?$AAg@ 004d4370     LIBCMT:wassert.obj
 0002:00014450       ??_C@_1BK@PEDCIPMA@?$AAE?$AAx?$AAp?$AAr?$AAe?$AAs?$AAs?$AAi?$AAo?$AAn?$AA?3?$AA?5?$AA?$AA@ 004d4450     LIBCMT:wassert.obj
 0002:0001446c       ??_C@_1O@KCAFKHJE@?$AAL?$AAi?$AAn?$AAe?$AA?3?$AA?5?$AA?$AA@ 004d446c     LIBCMT:wassert.obj
 0002:0001447c       ??_C@_1O@HEMHKNDC@?$AAF?$AAi?$AAl?$AAe?$AA?3?$AA?5?$AA?$AA@ 004d447c     LIBCMT:wassert.obj
 0002:0001448c       ??_C@_1CO@EAEJAADC@?$AA?$DM?$AAp?$AAr?$AAo?$AAg?$AAr?$AAa?$AAm?$AA?5?$AAn?$AAa?$AAm?$AAe?$AA?5?$AAu?$AAn?$AAk?$AAn?$AAo?$AAw?$AAn?$AA?$DO?$AA?$AA@ 004d448c     LIBCMT:wassert.obj
 0002:000144bc       ??_C@_1BE@PHKBBGE@?$AAP?$AAr?$AAo?$AAg?$AAr?$AAa?$AAm?$AA?3?$AA?5?$AA?$AA@ 004d44bc     LIBCMT:wassert.obj
 0002:000144d0       ??_C@_1CE@OJBNHDMO@?$AAA?$AAs?$AAs?$AAe?$AAr?$AAt?$AAi?$AAo?$AAn?$AA?5?$AAf?$AAa?$AAi?$AAl?$AAe?$AAd?$AA?$CB?$AA?$AA@ 004d44d0     LIBCMT:wassert.obj
 0002:000144f4       ??_C@_0CG@KNFFOMBO@Filename?5cannot?5be?5displayed?5on?5@ 004d44f4     LIBCMT:wassert.obj
 0002:0001451c       ??_C@_0CI@FDIHEIE@Expression?5cannot?5be?5displayed?5o@ 004d451c     LIBCMT:wassert.obj
 0002:00017e98       __DEFAULT_CW_in_mem        004d7e98     LIBCMT:common.obj
 0002:00017e9a       __pi_by_2_to_61            004d7e9a     LIBCMT:common.obj
 0002:00017ed8       __real@3fe0000000000000    004d7ed8     LIBCMT:powhlp.obj
 0002:000187e0       ??_C@_0BK@DEKFELLI@GetUserObjectInformationW?$AA@ 004d87e0     LIBCMT:crtmboxw.obj
 0002:000187fc       ??_C@_0M@DLDCCGNP@MessageBoxW?$AA@ 004d87fc     LIBCMT:crtmboxw.obj
 0002:00018808       ??_C@_1BG@GOEBHBDC@?$AAU?$AAS?$AAE?$AAR?$AA3?$AA2?$AA?4?$AAD?$AAL?$AAL?$AA?$AA@ 004d8808     LIBCMT:crtmboxw.obj
 0002:00018820       ??_C@_0DN@EBBNMLME@?$CIPress?5Retry?5to?5debug?5the?5applic@ 004d8820     LIBCMT:assert.obj
 0002:00018860       ??_C@_0HA@OJHAGA@For?5information?5on?5how?5your?5prog@ 004d8860     LIBCMT:assert.obj
 0002:000188d0       ??_C@_0N@MEECIJGN@Expression?3?5?$AA@ 004d88d0     LIBCMT:assert.obj
 0002:000188e0       ??_C@_06FIEBOLOH@Line?3?5?$AA@ 004d88e0     LIBCMT:assert.obj
 0002:000188e8       ??_C@_06IGPBOHMJ@File?3?5?$AA@ 004d88e8     LIBCMT:assert.obj
 0002:000188f0       ??_C@_09KLGCKDOD@Program?3?5?$AA@ 004d88f0     LIBCMT:assert.obj
 0002:000188fc       ??_C@_0BC@LAIDCHCH@Assertion?5failed?$CB?$AA@ 004d88fc     LIBCMT:assert.obj
 0002:00018910       __load_config_used         004d8910     LIBCMT:loadcfg.obj
 0002:0001c978       __tls_used                 004dc978     LIBCMT:tlssup.obj
 0002:0001cc40       ??_R4Command@@6B@          004dcc40     command.obj
 0002:0001cc58       ??_R3Command@@8            004dcc58     command.obj
 0002:0001cc6c       ??_R2Command@@8            004dcc6c     command.obj
 0002:0001cc74       ??_R1A@?0A@EA@Command@@8   004dcc74     command.obj
 0002:0001cc98       ??_R4Instance_cmd@@6B@     004dcc98     commands.obj
 0002:0001ccb0       ??_R3Instance_cmd@@8       004dccb0     commands.obj
 0002:0001ccc4       ??_R2Instance_cmd@@8       004dccc4     commands.obj
 0002:0001ccd0       ??_R1A@?0A@EA@Instance_cmd@@8 004dccd0     commands.obj
 0002:0001ccf4       ??_R4Abstract_instance_cmd@@6B@ 004dccf4     commands.obj
 0002:0001cd0c       ??_R3Abstract_instance_cmd@@8 004dcd0c     commands.obj
 0002:0001cd20       ??_R2Abstract_instance_cmd@@8 004dcd20     commands.obj
 0002:0001cd30       ??_R1A@?0A@EA@Abstract_instance_cmd@@8 004dcd30     commands.obj
 0002:0001cd54       ??_R4Show_instance_status@@6B@ 004dcd54     commands.obj
 0002:0001cd6c       ??_R3Show_instance_status@@8 004dcd6c     commands.obj
 0002:0001cd80       ??_R2Show_instance_status@@8 004dcd80     commands.obj
 0002:0001cd94       ??_R1A@?0A@EA@Show_instance_status@@8 004dcd94     commands.obj
 0002:0001cdb8       ??_R4Show_instance_options@@6B@ 004dcdb8     commands.obj
 0002:0001cdd0       ??_R3Show_instance_options@@8 004dcdd0     commands.obj
 0002:0001cde4       ??_R2Show_instance_options@@8 004dcde4     commands.obj
 0002:0001cdf8       ??_R1A@?0A@EA@Show_instance_options@@8 004dcdf8     commands.obj
 0002:0001ce1c       ??_R4Start_instance@@6B@   004dce1c     commands.obj
 0002:0001ce34       ??_R3Start_instance@@8     004dce34     commands.obj
 0002:0001ce48       ??_R2Start_instance@@8     004dce48     commands.obj
 0002:0001ce5c       ??_R1A@?0A@EA@Start_instance@@8 004dce5c     commands.obj
 0002:0001ce80       ??_R4Stop_instance@@6B@    004dce80     commands.obj
 0002:0001ce98       ??_R3Stop_instance@@8      004dce98     commands.obj
 0002:0001ceac       ??_R2Stop_instance@@8      004dceac     commands.obj
 0002:0001cec0       ??_R1A@?0A@EA@Stop_instance@@8 004dcec0     commands.obj
 0002:0001cee4       ??_R4Create_instance@@6B@  004dcee4     commands.obj
 0002:0001cefc       ??_R3Create_instance@@8    004dcefc     commands.obj
 0002:0001cf10       ??_R2Create_instance@@8    004dcf10     commands.obj
 0002:0001cf20       ??_R1A@?0A@EA@Create_instance@@8 004dcf20     commands.obj
 0002:0001cf44       ??_R4Drop_instance@@6B@    004dcf44     commands.obj
 0002:0001cf5c       ??_R3Drop_instance@@8      004dcf5c     commands.obj
 0002:0001cf70       ??_R2Drop_instance@@8      004dcf70     commands.obj
 0002:0001cf80       ??_R1A@?0A@EA@Drop_instance@@8 004dcf80     commands.obj
 0002:0001cfa4       ??_R4Show_instance_log@@6B@ 004dcfa4     commands.obj
 0002:0001cfbc       ??_R3Show_instance_log@@8  004dcfbc     commands.obj
 0002:0001cfd0       ??_R2Show_instance_log@@8  004dcfd0     commands.obj
 0002:0001cfe4       ??_R1A@?0A@EA@Show_instance_log@@8 004dcfe4     commands.obj
 0002:0001d008       ??_R4Show_instance_log_files@@6B@ 004dd008     commands.obj
 0002:0001d020       ??_R3Show_instance_log_files@@8 004dd020     commands.obj
 0002:0001d034       ??_R2Show_instance_log_files@@8 004dd034     commands.obj
 0002:0001d048       ??_R1A@?0A@EA@Show_instance_log_files@@8 004dd048     commands.obj
 0002:0001d06c       ??_R4Abstract_option_cmd@@6B@ 004dd06c     commands.obj
 0002:0001d084       ??_R3Abstract_option_cmd@@8 004dd084     commands.obj
 0002:0001d098       ??_R2Abstract_option_cmd@@8 004dd098     commands.obj
 0002:0001d0a4       ??_R1A@?0A@EA@Abstract_option_cmd@@8 004dd0a4     commands.obj
 0002:0001d0c8       ??_R4Thread@@6B@           004dd0c8     guardian.obj
 0002:0001d0e0       ??_R3Thread@@8             004dd0e0     guardian.obj
 0002:0001d0f4       ??_R2Thread@@8             004dd0f4     guardian.obj
 0002:0001d0fc       ??_R1A@?0A@EA@Thread@@8    004dd0fc     guardian.obj
 0002:0001d120       ??_R4Guardian@@6B@         004dd120     guardian.obj
 0002:0001d138       ??_R3Guardian@@8           004dd138     guardian.obj
 0002:0001d14c       ??_R2Guardian@@8           004dd14c     guardian.obj
 0002:0001d158       ??_R1A@?0A@EA@Guardian@@8  004dd158     guardian.obj
 0002:0001d17c       ??_R4Instance_monitor@@6B@ 004dd17c     instance.obj
 0002:0001d194       ??_R3Instance_monitor@@8   004dd194     instance.obj
 0002:0001d1a8       ??_R2Instance_monitor@@8   004dd1a8     instance.obj
 0002:0001d1b4       ??_R1A@?0A@EA@Instance_monitor@@8 004dd1b4     instance.obj
 0002:0001d1d8       ??_R4Listener@@6B@         004dd1d8     listener.obj
 0002:0001d1f0       ??_R3Listener@@8           004dd1f0     listener.obj
 0002:0001d204       ??_R2Listener@@8           004dd204     listener.obj
 0002:0001d210       ??_R1A@?0A@EA@Listener@@8  004dd210     listener.obj
 0002:0001d234       ??_R4ThreadModelChecker@?A0x2a2a756e@@6B@ 004dd234     manager.obj
 0002:0001d24c       ??_R3ThreadModelChecker@?A0x2a2a756e@@8 004dd24c     manager.obj
 0002:0001d260       ??_R2ThreadModelChecker@?A0x2a2a756e@@8 004dd260     manager.obj
 0002:0001d26c       ??_R1A@?0A@EA@ThreadModelChecker@?A0x2a2a756e@@8 004dd26c     manager.obj
 0002:0001d290       ??_R4Mysql_connection@@6B@ 004dd290     mysql_connection.obj
 0002:0001d2a8       ??_R3Mysql_connection@@8   004dd2a8     mysql_connection.obj
 0002:0001d2bc       ??_R2Mysql_connection@@8   004dd2bc     mysql_connection.obj
 0002:0001d2c8       ??_R1A@?0A@EA@Mysql_connection@@8 004dd2c8     mysql_connection.obj
 0002:0001d2ec       ??_R4User_management_cmd@@6B@ 004dd2ec     options.obj
 0002:0001d304       ??_R3User_management_cmd@@8 004dd304     options.obj
 0002:0001d318       ??_R2User_management_cmd@@8 004dd318     options.obj
 0002:0001d320       ??_R1A@?0A@EA@User_management_cmd@@8 004dd320     options.obj
 0002:0001d344       ??_R4Print_password_line_cmd@@6B@ 004dd344     options.obj
 0002:0001d35c       ??_R3Print_password_line_cmd@@8 004dd35c     options.obj
 0002:0001d370       ??_R2Print_password_line_cmd@@8 004dd370     options.obj
 0002:0001d37c       ??_R1A@?0A@EA@Print_password_line_cmd@@8 004dd37c     options.obj
 0002:0001d3a0       ??_R4Add_user_cmd@@6B@     004dd3a0     options.obj
 0002:0001d3b8       ??_R3Add_user_cmd@@8       004dd3b8     options.obj
 0002:0001d3cc       ??_R2Add_user_cmd@@8       004dd3cc     options.obj
 0002:0001d3d8       ??_R1A@?0A@EA@Add_user_cmd@@8 004dd3d8     options.obj
 0002:0001d3fc       ??_R4Drop_user_cmd@@6B@    004dd3fc     options.obj
 0002:0001d414       ??_R3Drop_user_cmd@@8      004dd414     options.obj
 0002:0001d428       ??_R2Drop_user_cmd@@8      004dd428     options.obj
 0002:0001d434       ??_R1A@?0A@EA@Drop_user_cmd@@8 004dd434     options.obj
 0002:0001d458       ??_R4Edit_user_cmd@@6B@    004dd458     options.obj
 0002:0001d470       ??_R3Edit_user_cmd@@8      004dd470     options.obj
 0002:0001d484       ??_R2Edit_user_cmd@@8      004dd484     options.obj
 0002:0001d490       ??_R1A@?0A@EA@Edit_user_cmd@@8 004dd490     options.obj
 0002:0001d4b4       ??_R4Clean_db_cmd@@6B@     004dd4b4     options.obj
 0002:0001d4cc       ??_R3Clean_db_cmd@@8       004dd4cc     options.obj
 0002:0001d4e0       ??_R2Clean_db_cmd@@8       004dd4e0     options.obj
 0002:0001d4ec       ??_R1A@?0A@EA@Clean_db_cmd@@8 004dd4ec     options.obj
 0002:0001d510       ??_R4Check_db_cmd@@6B@     004dd510     options.obj
 0002:0001d528       ??_R3Check_db_cmd@@8       004dd528     options.obj
 0002:0001d53c       ??_R2Check_db_cmd@@8       004dd53c     options.obj
 0002:0001d548       ??_R1A@?0A@EA@Check_db_cmd@@8 004dd548     options.obj
 0002:0001d56c       ??_R4List_users_cmd@@6B@   004dd56c     options.obj
 0002:0001d584       ??_R3List_users_cmd@@8     004dd584     options.obj
 0002:0001d598       ??_R2List_users_cmd@@8     004dd598     options.obj
 0002:0001d5a4       ??_R1A@?0A@EA@List_users_cmd@@8 004dd5a4     options.obj
 0002:0001d5c8       ??_R4Show_instances@@6B@   004dd5c8     parse.obj
 0002:0001d5e0       ??_R3Show_instances@@8     004dd5e0     parse.obj
 0002:0001d5f4       ??_R2Show_instances@@8     004dd5f4     parse.obj
 0002:0001d600       ??_R1A@?0A@EA@Show_instances@@8 004dd600     parse.obj
 0002:0001d624       ??_R4Flush_instances@@6B@  004dd624     parse.obj
 0002:0001d63c       ??_R3Flush_instances@@8    004dd63c     parse.obj
 0002:0001d650       ??_R2Flush_instances@@8    004dd650     parse.obj
 0002:0001d65c       ??_R1A@?0A@EA@Flush_instances@@8 004dd65c     parse.obj
 0002:0001d680       ??_R4Set_option@@6B@       004dd680     parse.obj
 0002:0001d698       ??_R3Set_option@@8         004dd698     parse.obj
 0002:0001d6ac       ??_R2Set_option@@8         004dd6ac     parse.obj
 0002:0001d6bc       ??_R1A@?0A@EA@Set_option@@8 004dd6bc     parse.obj
 0002:0001d6e0       ??_R4Unset_option@@6B@     004dd6e0     parse.obj
 0002:0001d6f8       ??_R3Unset_option@@8       004dd6f8     parse.obj
 0002:0001d70c       ??_R2Unset_option@@8       004dd70c     parse.obj
 0002:0001d71c       ??_R1A@?0A@EA@Unset_option@@8 004dd71c     parse.obj
 0002:0001d740       ??_R4Syntax_error@@6B@     004dd740     parse.obj
 0002:0001d758       ??_R3Syntax_error@@8       004dd758     parse.obj
 0002:0001d76c       ??_R2Syntax_error@@8       004dd76c     parse.obj
 0002:0001d778       ??_R1A@?0A@EA@Syntax_error@@8 004dd778     parse.obj
 0002:0001d79c       ??_R4Mysqld_output_parser@?A0x60d3fd73@@6B@ 004dd79c     parse_output.obj
 0002:0001d7b4       ??_R3Mysqld_output_parser@?A0x60d3fd73@@8 004dd7b4     parse_output.obj
 0002:0001d7c8       ??_R2Mysqld_output_parser@?A0x60d3fd73@@8 004dd7c8     parse_output.obj
 0002:0001d7d0       ??_R1A@?0A@EA@Mysqld_output_parser@?A0x60d3fd73@@8 004dd7d0     parse_output.obj
 0002:0001d7f4       ??_R4Mysqld_output_parser_win@?A0x60d3fd73@@6B@ 004dd7f4     parse_output.obj
 0002:0001d80c       ??_R3Mysqld_output_parser_win@?A0x60d3fd73@@8 004dd80c     parse_output.obj
 0002:0001d820       ??_R2Mysqld_output_parser_win@?A0x60d3fd73@@8 004dd820     parse_output.obj
 0002:0001d82c       ??_R1A@?0A@EA@Mysqld_output_parser_win@?A0x60d3fd73@@8 004dd82c     parse_output.obj
 0002:0001d850       ??_R4IMService@@6B@        004dd850     IMService.obj
 0002:0001d868       ??_R3IMService@@8          004dd868     IMService.obj
 0002:0001d87c       ??_R2IMService@@8          004dd87c     IMService.obj
 0002:0001d888       ??_R1A@?0A@EA@IMService@@8 004dd888     IMService.obj
 0002:0001d8ac       ??_R1A@?0A@EA@WindowsService@@8 004dd8ac     IMService.obj
 0002:0001d8d0       ??_R3WindowsService@@8     004dd8d0     IMService.obj
 0002:0001d8e4       ??_R2WindowsService@@8     004dd8e4     IMService.obj
 0002:0001d8ec       ??_R4WindowsService@@6B@   004dd8ec     WindowsService.obj
 0002:0001d904       ??_R4Message@yaSSL@@6B@    004dd904     yassl:ssl.obj
 0002:0001d918       ??_R3Message@yaSSL@@8      004dd918     yassl:ssl.obj
 0002:0001d928       ??_R2Message@yaSSL@@8      004dd928     yassl:ssl.obj
 0002:0001d934       ??_R1A@?0A@EA@Message@yaSSL@@8 004dd934     yassl:ssl.obj
 0002:0001d950       ??_R13?0A@EA@virtual_base@yaSSL@@8 004dd950     yassl:ssl.obj
 0002:0001d96c       ??_R3virtual_base@yaSSL@@8 004dd96c     yassl:ssl.obj
 0002:0001d97c       ??_R2virtual_base@yaSSL@@8 004dd97c     yassl:ssl.obj
 0002:0001d984       ??_R1A@?0A@EA@virtual_base@yaSSL@@8 004dd984     yassl:ssl.obj
 0002:0001d9a0       ??_R4HandShakeBase@yaSSL@@6B@ 004dd9a0     yassl:ssl.obj
 0002:0001d9b4       ??_R3HandShakeBase@yaSSL@@8 004dd9b4     yassl:ssl.obj
 0002:0001d9c4       ??_R2HandShakeBase@yaSSL@@8 004dd9c4     yassl:ssl.obj
 0002:0001d9d0       ??_R1A@?0A@EA@HandShakeBase@yaSSL@@8 004dd9d0     yassl:ssl.obj
 0002:0001d9ec       ??_R4HASH@TaoCrypt@@6B@    004dd9ec     yassl:ssl.obj
 0002:0001da00       ??_R3HASH@TaoCrypt@@8      004dda00     yassl:ssl.obj
 0002:0001da10       ??_R2HASH@TaoCrypt@@8      004dda10     yassl:ssl.obj
 0002:0001da1c       ??_R1A@?0A@EA@HASH@TaoCrypt@@8 004dda1c     yassl:ssl.obj
 0002:0001da38       ??_R13?0A@EA@virtual_base@TaoCrypt@@8 004dda38     yassl:ssl.obj
 0002:0001da54       ??_R3virtual_base@TaoCrypt@@8 004dda54     yassl:ssl.obj
 0002:0001da64       ??_R2virtual_base@TaoCrypt@@8 004dda64     yassl:ssl.obj
 0002:0001da6c       ??_R1A@?0A@EA@virtual_base@TaoCrypt@@8 004dda6c     yassl:ssl.obj
 0002:0001da88       ??_R4MD5@TaoCrypt@@6B@     004dda88     yassl:ssl.obj
 0002:0001da9c       ??_R3MD5@TaoCrypt@@8       004dda9c     yassl:ssl.obj
 0002:0001daac       ??_R2MD5@TaoCrypt@@8       004ddaac     yassl:ssl.obj
 0002:0001dac0       ??_R1A@?0A@EA@MD5@TaoCrypt@@8 004ddac0     yassl:ssl.obj
 0002:0001dadc       ??_R1A@?0A@EA@HASHwithTransform@TaoCrypt@@8 004ddadc     yassl:ssl.obj
 0002:0001daf8       ??_R3HASHwithTransform@TaoCrypt@@8 004ddaf8     yassl:ssl.obj
 0002:0001db08       ??_R2HASHwithTransform@TaoCrypt@@8 004ddb08     yassl:ssl.obj
 0002:0001db18       ??_R4MD4@TaoCrypt@@6B@     004ddb18     yassl:ssl.obj
 0002:0001db2c       ??_R3MD4@TaoCrypt@@8       004ddb2c     yassl:ssl.obj
 0002:0001db3c       ??_R2MD4@TaoCrypt@@8       004ddb3c     yassl:ssl.obj
 0002:0001db50       ??_R1A@?0A@EA@MD4@TaoCrypt@@8 004ddb50     yassl:ssl.obj
 0002:0001db6c       ??_R4Digest@yaSSL@@6B@     004ddb6c     yassl:crypto_wrapper.obj
 0002:0001db80       ??_R3Digest@yaSSL@@8       004ddb80     yassl:crypto_wrapper.obj
 0002:0001db90       ??_R2Digest@yaSSL@@8       004ddb90     yassl:crypto_wrapper.obj
 0002:0001db9c       ??_R1A@?0A@EA@Digest@yaSSL@@8 004ddb9c     yassl:crypto_wrapper.obj
 0002:0001dbb8       ??_R4BulkCipher@yaSSL@@6B@ 004ddbb8     yassl:crypto_wrapper.obj
 0002:0001dbcc       ??_R3BulkCipher@yaSSL@@8   004ddbcc     yassl:crypto_wrapper.obj
 0002:0001dbdc       ??_R2BulkCipher@yaSSL@@8   004ddbdc     yassl:crypto_wrapper.obj
 0002:0001dbe8       ??_R1A@?0A@EA@BulkCipher@yaSSL@@8 004ddbe8     yassl:crypto_wrapper.obj
 0002:0001dc04       ??_R4Auth@yaSSL@@6B@       004ddc04     yassl:crypto_wrapper.obj
 0002:0001dc18       ??_R3Auth@yaSSL@@8         004ddc18     yassl:crypto_wrapper.obj
 0002:0001dc28       ??_R2Auth@yaSSL@@8         004ddc28     yassl:crypto_wrapper.obj
 0002:0001dc34       ??_R1A@?0A@EA@Auth@yaSSL@@8 004ddc34     yassl:crypto_wrapper.obj
 0002:0001dc50       ??_R4SHA@TaoCrypt@@6B@     004ddc50     yassl:crypto_wrapper.obj
 0002:0001dc64       ??_R3SHA@TaoCrypt@@8       004ddc64     yassl:crypto_wrapper.obj
 0002:0001dc74       ??_R2SHA@TaoCrypt@@8       004ddc74     yassl:crypto_wrapper.obj
 0002:0001dc88       ??_R1A@?0A@EA@SHA@TaoCrypt@@8 004ddc88     yassl:crypto_wrapper.obj
 0002:0001dca4       ??_R4RIPEMD160@TaoCrypt@@6B@ 004ddca4     yassl:crypto_wrapper.obj
 0002:0001dcb8       ??_R3RIPEMD160@TaoCrypt@@8 004ddcb8     yassl:crypto_wrapper.obj
 0002:0001dcc8       ??_R2RIPEMD160@TaoCrypt@@8 004ddcc8     yassl:crypto_wrapper.obj
 0002:0001dcdc       ??_R1A@?0A@EA@RIPEMD160@TaoCrypt@@8 004ddcdc     yassl:crypto_wrapper.obj
 0002:0001dcf8       ??_R4Mode_BASE@TaoCrypt@@6B@ 004ddcf8     yassl:crypto_wrapper.obj
 0002:0001dd0c       ??_R3Mode_BASE@TaoCrypt@@8 004ddd0c     yassl:crypto_wrapper.obj
 0002:0001dd1c       ??_R2Mode_BASE@TaoCrypt@@8 004ddd1c     yassl:crypto_wrapper.obj
 0002:0001dd28       ??_R1A@?0A@EA@Mode_BASE@TaoCrypt@@8 004ddd28     yassl:crypto_wrapper.obj
 0002:0001dd44       ??_R4DES@TaoCrypt@@6B@     004ddd44     yassl:crypto_wrapper.obj
 0002:0001dd58       ??_R3DES@TaoCrypt@@8       004ddd58     yassl:crypto_wrapper.obj
 0002:0001dd68       ??_R2DES@TaoCrypt@@8       004ddd68     yassl:crypto_wrapper.obj
 0002:0001dd7c       ??_R1A@?0A@EA@DES@TaoCrypt@@8 004ddd7c     yassl:crypto_wrapper.obj
 0002:0001dd98       ??_R1DI@?0A@EA@BasicDES@TaoCrypt@@8 004ddd98     yassl:crypto_wrapper.obj
 0002:0001ddb4       ??_R3BasicDES@TaoCrypt@@8  004dddb4     yassl:crypto_wrapper.obj
 0002:0001ddc4       ??_R2BasicDES@TaoCrypt@@8  004dddc4     yassl:crypto_wrapper.obj
 0002:0001ddcc       ??_R1A@?0A@EA@BasicDES@TaoCrypt@@8 004dddcc     yassl:crypto_wrapper.obj
 0002:0001dde8       ??_R4DES_EDE3@TaoCrypt@@6B@ 004ddde8     yassl:crypto_wrapper.obj
 0002:0001ddfc       ??_R3DES_EDE3@TaoCrypt@@8  004dddfc     yassl:crypto_wrapper.obj
 0002:0001de0c       ??_R2DES_EDE3@TaoCrypt@@8  004dde0c     yassl:crypto_wrapper.obj
 0002:0001de1c       ??_R1A@?0A@EA@DES_EDE3@TaoCrypt@@8 004dde1c     yassl:crypto_wrapper.obj
 0002:0001de38       ??_R4AES@TaoCrypt@@6B@     004dde38     yassl:crypto_wrapper.obj
 0002:0001de4c       ??_R3AES@TaoCrypt@@8       004dde4c     yassl:crypto_wrapper.obj
 0002:0001de5c       ??_R2AES@TaoCrypt@@8       004dde5c     yassl:crypto_wrapper.obj
 0002:0001de6c       ??_R1A@?0A@EA@AES@TaoCrypt@@8 004dde6c     yassl:crypto_wrapper.obj
 0002:0001de88       ??_R4MD5@yaSSL@@6B@        004dde88     yassl:crypto_wrapper.obj
 0002:0001de9c       ??_R3MD5@yaSSL@@8          004dde9c     yassl:crypto_wrapper.obj
 0002:0001deac       ??_R2MD5@yaSSL@@8          004ddeac     yassl:crypto_wrapper.obj
 0002:0001debc       ??_R1A@?0A@EA@MD5@yaSSL@@8 004ddebc     yassl:crypto_wrapper.obj
 0002:0001ded8       ??_R4SHA@yaSSL@@6B@        004dded8     yassl:crypto_wrapper.obj
 0002:0001deec       ??_R3SHA@yaSSL@@8          004ddeec     yassl:crypto_wrapper.obj
 0002:0001defc       ??_R2SHA@yaSSL@@8          004ddefc     yassl:crypto_wrapper.obj
 0002:0001df0c       ??_R1A@?0A@EA@SHA@yaSSL@@8 004ddf0c     yassl:crypto_wrapper.obj
 0002:0001df28       ??_R4RMD@yaSSL@@6B@        004ddf28     yassl:crypto_wrapper.obj
 0002:0001df3c       ??_R3RMD@yaSSL@@8          004ddf3c     yassl:crypto_wrapper.obj
 0002:0001df4c       ??_R2RMD@yaSSL@@8          004ddf4c     yassl:crypto_wrapper.obj
 0002:0001df5c       ??_R1A@?0A@EA@RMD@yaSSL@@8 004ddf5c     yassl:crypto_wrapper.obj
 0002:0001df78       ??_R4RC4@yaSSL@@6B@        004ddf78     yassl:crypto_wrapper.obj
 0002:0001df8c       ??_R3RC4@yaSSL@@8          004ddf8c     yassl:crypto_wrapper.obj
 0002:0001df9c       ??_R2RC4@yaSSL@@8          004ddf9c     yassl:crypto_wrapper.obj
 0002:0001dfac       ??_R1A@?0A@EA@RC4@yaSSL@@8 004ddfac     yassl:crypto_wrapper.obj
 0002:0001dfc8       ??_R4AES@yaSSL@@6B@        004ddfc8     yassl:crypto_wrapper.obj
 0002:0001dfdc       ??_R3AES@yaSSL@@8          004ddfdc     yassl:crypto_wrapper.obj
 0002:0001dfec       ??_R2AES@yaSSL@@8          004ddfec     yassl:crypto_wrapper.obj
 0002:0001dffc       ??_R1A@?0A@EA@AES@yaSSL@@8 004ddffc     yassl:crypto_wrapper.obj
 0002:0001e018       ??_R4HMAC_MD5@yaSSL@@6B@   004de018     yassl:crypto_wrapper.obj
 0002:0001e02c       ??_R3HMAC_MD5@yaSSL@@8     004de02c     yassl:crypto_wrapper.obj
 0002:0001e03c       ??_R2HMAC_MD5@yaSSL@@8     004de03c     yassl:crypto_wrapper.obj
 0002:0001e04c       ??_R1A@?0A@EA@HMAC_MD5@yaSSL@@8 004de04c     yassl:crypto_wrapper.obj
 0002:0001e068       ??_R4HMAC_SHA@yaSSL@@6B@   004de068     yassl:crypto_wrapper.obj
 0002:0001e07c       ??_R3HMAC_SHA@yaSSL@@8     004de07c     yassl:crypto_wrapper.obj
 0002:0001e08c       ??_R2HMAC_SHA@yaSSL@@8     004de08c     yassl:crypto_wrapper.obj
 0002:0001e09c       ??_R1A@?0A@EA@HMAC_SHA@yaSSL@@8 004de09c     yassl:crypto_wrapper.obj
 0002:0001e0b8       ??_R4HMAC_RMD@yaSSL@@6B@   004de0b8     yassl:crypto_wrapper.obj
 0002:0001e0cc       ??_R3HMAC_RMD@yaSSL@@8     004de0cc     yassl:crypto_wrapper.obj
 0002:0001e0dc       ??_R2HMAC_RMD@yaSSL@@8     004de0dc     yassl:crypto_wrapper.obj
 0002:0001e0ec       ??_R1A@?0A@EA@HMAC_RMD@yaSSL@@8 004de0ec     yassl:crypto_wrapper.obj
 0002:0001e108       ??_R4DES@yaSSL@@6B@        004de108     yassl:crypto_wrapper.obj
 0002:0001e11c       ??_R3DES@yaSSL@@8          004de11c     yassl:crypto_wrapper.obj
 0002:0001e12c       ??_R2DES@yaSSL@@8          004de12c     yassl:crypto_wrapper.obj
 0002:0001e13c       ??_R1A@?0A@EA@DES@yaSSL@@8 004de13c     yassl:crypto_wrapper.obj
 0002:0001e158       ??_R4DES_EDE@yaSSL@@6B@    004de158     yassl:crypto_wrapper.obj
 0002:0001e16c       ??_R3DES_EDE@yaSSL@@8      004de16c     yassl:crypto_wrapper.obj
 0002:0001e17c       ??_R2DES_EDE@yaSSL@@8      004de17c     yassl:crypto_wrapper.obj
 0002:0001e18c       ??_R1A@?0A@EA@DES_EDE@yaSSL@@8 004de18c     yassl:crypto_wrapper.obj
 0002:0001e1a8       ??_R4DSS@yaSSL@@6B@        004de1a8     yassl:crypto_wrapper.obj
 0002:0001e1bc       ??_R3DSS@yaSSL@@8          004de1bc     yassl:crypto_wrapper.obj
 0002:0001e1cc       ??_R2DSS@yaSSL@@8          004de1cc     yassl:crypto_wrapper.obj
 0002:0001e1dc       ??_R1A@?0A@EA@DSS@yaSSL@@8 004de1dc     yassl:crypto_wrapper.obj
 0002:0001e1f8       ??_R4RSA@yaSSL@@6B@        004de1f8     yassl:crypto_wrapper.obj
 0002:0001e20c       ??_R3RSA@yaSSL@@8          004de20c     yassl:crypto_wrapper.obj
 0002:0001e21c       ??_R2RSA@yaSSL@@8          004de21c     yassl:crypto_wrapper.obj
 0002:0001e22c       ??_R1A@?0A@EA@RSA@yaSSL@@8 004de22c     yassl:crypto_wrapper.obj
 0002:0001e248       ??_R4HandShakeHeader@yaSSL@@6B@ 004de248     yassl:yassl_imp.obj
 0002:0001e25c       ??_R3HandShakeHeader@yaSSL@@8 004de25c     yassl:yassl_imp.obj
 0002:0001e26c       ??_R2HandShakeHeader@yaSSL@@8 004de26c     yassl:yassl_imp.obj
 0002:0001e27c       ??_R1A@?0A@EA@HandShakeHeader@yaSSL@@8 004de27c     yassl:yassl_imp.obj
 0002:0001e298       ??_R4ServerKeyBase@yaSSL@@6B@ 004de298     yassl:yassl_imp.obj
 0002:0001e2ac       ??_R3ServerKeyBase@yaSSL@@8 004de2ac     yassl:yassl_imp.obj
 0002:0001e2bc       ??_R2ServerKeyBase@yaSSL@@8 004de2bc     yassl:yassl_imp.obj
 0002:0001e2c8       ??_R1A@?0A@EA@ServerKeyBase@yaSSL@@8 004de2c8     yassl:yassl_imp.obj
 0002:0001e2e4       ??_R4ClientKeyBase@yaSSL@@6B@ 004de2e4     yassl:yassl_imp.obj
 0002:0001e2f8       ??_R3ClientKeyBase@yaSSL@@8 004de2f8     yassl:yassl_imp.obj
 0002:0001e308       ??_R2ClientKeyBase@yaSSL@@8 004de308     yassl:yassl_imp.obj
 0002:0001e314       ??_R1A@?0A@EA@ClientKeyBase@yaSSL@@8 004de314     yassl:yassl_imp.obj
 0002:0001e330       ??_R4ClientDiffieHellmanPublic@yaSSL@@6B@ 004de330     yassl:yassl_imp.obj
 0002:0001e344       ??_R3ClientDiffieHellmanPublic@yaSSL@@8 004de344     yassl:yassl_imp.obj
 0002:0001e354       ??_R2ClientDiffieHellmanPublic@yaSSL@@8 004de354     yassl:yassl_imp.obj
 0002:0001e364       ??_R1A@?0A@EA@ClientDiffieHellmanPublic@yaSSL@@8 004de364     yassl:yassl_imp.obj
 0002:0001e380       ??_R4ChangeCipherSpec@yaSSL@@6B@ 004de380     yassl:yassl_imp.obj
 0002:0001e394       ??_R3ChangeCipherSpec@yaSSL@@8 004de394     yassl:yassl_imp.obj
 0002:0001e3a4       ??_R2ChangeCipherSpec@yaSSL@@8 004de3a4     yassl:yassl_imp.obj
 0002:0001e3b4       ??_R1A@?0A@EA@ChangeCipherSpec@yaSSL@@8 004de3b4     yassl:yassl_imp.obj
 0002:0001e3d0       ??_R4Alert@yaSSL@@6B@      004de3d0     yassl:yassl_imp.obj
 0002:0001e3e4       ??_R3Alert@yaSSL@@8        004de3e4     yassl:yassl_imp.obj
 0002:0001e3f4       ??_R2Alert@yaSSL@@8        004de3f4     yassl:yassl_imp.obj
 0002:0001e404       ??_R1A@?0A@EA@Alert@yaSSL@@8 004de404     yassl:yassl_imp.obj
 0002:0001e420       ??_R4Data@yaSSL@@6B@       004de420     yassl:yassl_imp.obj
 0002:0001e434       ??_R3Data@yaSSL@@8         004de434     yassl:yassl_imp.obj
 0002:0001e444       ??_R2Data@yaSSL@@8         004de444     yassl:yassl_imp.obj
 0002:0001e454       ??_R1A@?0A@EA@Data@yaSSL@@8 004de454     yassl:yassl_imp.obj
 0002:0001e470       ??_R4Certificate@yaSSL@@6B@ 004de470     yassl:yassl_imp.obj
 0002:0001e484       ??_R3Certificate@yaSSL@@8  004de484     yassl:yassl_imp.obj
 0002:0001e494       ??_R2Certificate@yaSSL@@8  004de494     yassl:yassl_imp.obj
 0002:0001e4a4       ??_R1A@?0A@EA@Certificate@yaSSL@@8 004de4a4     yassl:yassl_imp.obj
 0002:0001e4c0       ??_R4ServerHello@yaSSL@@6B@ 004de4c0     yassl:yassl_imp.obj
 0002:0001e4d4       ??_R3ServerHello@yaSSL@@8  004de4d4     yassl:yassl_imp.obj
 0002:0001e4e4       ??_R2ServerHello@yaSSL@@8  004de4e4     yassl:yassl_imp.obj
 0002:0001e4f4       ??_R1A@?0A@EA@ServerHello@yaSSL@@8 004de4f4     yassl:yassl_imp.obj
 0002:0001e510       ??_R4ServerHelloDone@yaSSL@@6B@ 004de510     yassl:yassl_imp.obj
 0002:0001e524       ??_R3ServerHelloDone@yaSSL@@8 004de524     yassl:yassl_imp.obj
 0002:0001e534       ??_R2ServerHelloDone@yaSSL@@8 004de534     yassl:yassl_imp.obj
 0002:0001e544       ??_R1A@?0A@EA@ServerHelloDone@yaSSL@@8 004de544     yassl:yassl_imp.obj
 0002:0001e560       ??_R4ClientHello@yaSSL@@6B@ 004de560     yassl:yassl_imp.obj
 0002:0001e574       ??_R3ClientHello@yaSSL@@8  004de574     yassl:yassl_imp.obj
 0002:0001e584       ??_R2ClientHello@yaSSL@@8  004de584     yassl:yassl_imp.obj
 0002:0001e594       ??_R1A@?0A@EA@ClientHello@yaSSL@@8 004de594     yassl:yassl_imp.obj
 0002:0001e5b0       ??_R4ServerKeyExchange@yaSSL@@6B@ 004de5b0     yassl:yassl_imp.obj
 0002:0001e5c4       ??_R3ServerKeyExchange@yaSSL@@8 004de5c4     yassl:yassl_imp.obj
 0002:0001e5d4       ??_R2ServerKeyExchange@yaSSL@@8 004de5d4     yassl:yassl_imp.obj
 0002:0001e5e4       ??_R1A@?0A@EA@ServerKeyExchange@yaSSL@@8 004de5e4     yassl:yassl_imp.obj
 0002:0001e600       ??_R4CertificateVerify@yaSSL@@6B@ 004de600     yassl:yassl_imp.obj
 0002:0001e614       ??_R3CertificateVerify@yaSSL@@8 004de614     yassl:yassl_imp.obj
 0002:0001e624       ??_R2CertificateVerify@yaSSL@@8 004de624     yassl:yassl_imp.obj
 0002:0001e634       ??_R1A@?0A@EA@CertificateVerify@yaSSL@@8 004de634     yassl:yassl_imp.obj
 0002:0001e650       ??_R4ClientKeyExchange@yaSSL@@6B@ 004de650     yassl:yassl_imp.obj
 0002:0001e664       ??_R3ClientKeyExchange@yaSSL@@8 004de664     yassl:yassl_imp.obj
 0002:0001e674       ??_R2ClientKeyExchange@yaSSL@@8 004de674     yassl:yassl_imp.obj
 0002:0001e684       ??_R1A@?0A@EA@ClientKeyExchange@yaSSL@@8 004de684     yassl:yassl_imp.obj
 0002:0001e6a0       ??_R4Finished@yaSSL@@6B@   004de6a0     yassl:yassl_imp.obj
 0002:0001e6b4       ??_R3Finished@yaSSL@@8     004de6b4     yassl:yassl_imp.obj
 0002:0001e6c4       ??_R2Finished@yaSSL@@8     004de6c4     yassl:yassl_imp.obj
 0002:0001e6d4       ??_R1A@?0A@EA@Finished@yaSSL@@8 004de6d4     yassl:yassl_imp.obj
 0002:0001e6f0       ??_R4HelloRequest@yaSSL@@6B@ 004de6f0     yassl:yassl_imp.obj
 0002:0001e704       ??_R3HelloRequest@yaSSL@@8 004de704     yassl:yassl_imp.obj
 0002:0001e714       ??_R2HelloRequest@yaSSL@@8 004de714     yassl:yassl_imp.obj
 0002:0001e724       ??_R1A@?0A@EA@HelloRequest@yaSSL@@8 004de724     yassl:yassl_imp.obj
 0002:0001e740       ??_R4RSA_Server@yaSSL@@6B@ 004de740     yassl:yassl_imp.obj
 0002:0001e754       ??_R3RSA_Server@yaSSL@@8   004de754     yassl:yassl_imp.obj
 0002:0001e764       ??_R2RSA_Server@yaSSL@@8   004de764     yassl:yassl_imp.obj
 0002:0001e774       ??_R1A@?0A@EA@RSA_Server@yaSSL@@8 004de774     yassl:yassl_imp.obj
 0002:0001e790       ??_R4Fortezza_Server@yaSSL@@6B@ 004de790     yassl:yassl_imp.obj
 0002:0001e7a4       ??_R3Fortezza_Server@yaSSL@@8 004de7a4     yassl:yassl_imp.obj
 0002:0001e7b4       ??_R2Fortezza_Server@yaSSL@@8 004de7b4     yassl:yassl_imp.obj
 0002:0001e7c4       ??_R1A@?0A@EA@Fortezza_Server@yaSSL@@8 004de7c4     yassl:yassl_imp.obj
 0002:0001e7e0       ??_R4FortezzaKeys@yaSSL@@6B@ 004de7e0     yassl:yassl_imp.obj
 0002:0001e7f4       ??_R3FortezzaKeys@yaSSL@@8 004de7f4     yassl:yassl_imp.obj
 0002:0001e804       ??_R2FortezzaKeys@yaSSL@@8 004de804     yassl:yassl_imp.obj
 0002:0001e814       ??_R1A@?0A@EA@FortezzaKeys@yaSSL@@8 004de814     yassl:yassl_imp.obj
 0002:0001e830       ??_R4EncryptedPreMasterSecret@yaSSL@@6B@ 004de830     yassl:yassl_imp.obj
 0002:0001e844       ??_R3EncryptedPreMasterSecret@yaSSL@@8 004de844     yassl:yassl_imp.obj
 0002:0001e854       ??_R2EncryptedPreMasterSecret@yaSSL@@8 004de854     yassl:yassl_imp.obj
 0002:0001e864       ??_R1A@?0A@EA@EncryptedPreMasterSecret@yaSSL@@8 004de864     yassl:yassl_imp.obj
 0002:0001e880       ??_R4DH_Server@yaSSL@@6B@  004de880     yassl:yassl_imp.obj
 0002:0001e894       ??_R3DH_Server@yaSSL@@8    004de894     yassl:yassl_imp.obj
 0002:0001e8a4       ??_R2DH_Server@yaSSL@@8    004de8a4     yassl:yassl_imp.obj
 0002:0001e8b4       ??_R1A@?0A@EA@DH_Server@yaSSL@@8 004de8b4     yassl:yassl_imp.obj
 0002:0001e8d0       ??_R4CertificateRequest@yaSSL@@6B@ 004de8d0     yassl:yassl_imp.obj
 0002:0001e8e4       ??_R3CertificateRequest@yaSSL@@8 004de8e4     yassl:yassl_imp.obj
 0002:0001e8f4       ??_R2CertificateRequest@yaSSL@@8 004de8f4     yassl:yassl_imp.obj
 0002:0001e904       ??_R1A@?0A@EA@CertificateRequest@yaSSL@@8 004de904     yassl:yassl_imp.obj
 0002:0001e920       ??_R4type_info@@6B@        004de920     LIBCMT:typinfo.obj
 0002:0001e934       ??_R3type_info@@8          004de934     LIBCMT:typinfo.obj
 0002:0001e944       ??_R2type_info@@8          004de944     LIBCMT:typinfo.obj
 0002:0001e94c       ??_R1A@?0A@EA@type_info@@8 004de94c     LIBCMT:typinfo.obj
 0002:0001e968       ??_R4bad_alloc@std@@6B@    004de968     LIBCMT:new.obj
 0002:0001e97c       ??_R3bad_alloc@std@@8      004de97c     LIBCMT:new.obj
 0002:0001e98c       ??_R2bad_alloc@std@@8      004de98c     LIBCMT:new.obj
 0002:0001e998       ??_R1A@?0A@EA@bad_alloc@std@@8 004de998     LIBCMT:new.obj
 0002:0001e9b4       ??_R1A@?0A@EA@exception@std@@8 004de9b4     LIBCMT:new.obj
 0002:0001e9d0       ??_R3exception@std@@8      004de9d0     LIBCMT:new.obj
 0002:0001e9e0       ??_R2exception@std@@8      004de9e0     LIBCMT:new.obj
 0002:0001e9e8       ??_R4exception@std@@6B@    004de9e8     LIBCMT:stdexcpt.obj
 0002:0001e9fc       ??_R4bad_cast@std@@6B@     004de9fc     LIBCMT:stdexcpt.obj
 0002:0001ea10       ??_R3bad_cast@std@@8       004dea10     LIBCMT:stdexcpt.obj
 0002:0001ea20       ??_R2bad_cast@std@@8       004dea20     LIBCMT:stdexcpt.obj
 0002:0001ea2c       ??_R1A@?0A@EA@bad_cast@std@@8 004dea2c     LIBCMT:stdexcpt.obj
 0002:0001ea48       ??_R4bad_typeid@std@@6B@   004dea48     LIBCMT:stdexcpt.obj
 0002:0001ea5c       ??_R3bad_typeid@std@@8     004dea5c     LIBCMT:stdexcpt.obj
 0002:0001ea6c       ??_R2bad_typeid@std@@8     004dea6c     LIBCMT:stdexcpt.obj
 0002:0001ea78       ??_R1A@?0A@EA@bad_typeid@std@@8 004dea78     LIBCMT:stdexcpt.obj
 0002:0001ea94       ??_R4__non_rtti_object@std@@6B@ 004dea94     LIBCMT:stdexcpt.obj
 0002:0001eaa8       ??_R3__non_rtti_object@std@@8 004deaa8     LIBCMT:stdexcpt.obj
 0002:0001eab8       ??_R2__non_rtti_object@std@@8 004deab8     LIBCMT:stdexcpt.obj
 0002:0001eac8       ??_R1A@?0A@EA@__non_rtti_object@std@@8 004deac8     LIBCMT:stdexcpt.obj
 0002:0001eae4       ??_R4DNameNode@@6B@        004deae4     LIBCMT:undname.obj
 0002:0001eaf8       ??_R3DNameNode@@8          004deaf8     LIBCMT:undname.obj
 0002:0001eb08       ??_R2DNameNode@@8          004deb08     LIBCMT:undname.obj
 0002:0001eb10       ??_R1A@?0A@EA@DNameNode@@8 004deb10     LIBCMT:undname.obj
 0002:0001eb2c       ??_R4charNode@@6B@         004deb2c     LIBCMT:undname.obj
 0002:0001eb40       ??_R3charNode@@8           004deb40     LIBCMT:undname.obj
 0002:0001eb50       ??_R2charNode@@8           004deb50     LIBCMT:undname.obj
 0002:0001eb5c       ??_R1A@?0A@EA@charNode@@8  004deb5c     LIBCMT:undname.obj
 0002:0001eb78       ??_R4pDNameNode@@6B@       004deb78     LIBCMT:undname.obj
 0002:0001eb8c       ??_R3pDNameNode@@8         004deb8c     LIBCMT:undname.obj
 0002:0001eb9c       ??_R2pDNameNode@@8         004deb9c     LIBCMT:undname.obj
 0002:0001eba8       ??_R1A@?0A@EA@pDNameNode@@8 004deba8     LIBCMT:undname.obj
 0002:0001ebc4       ??_R4DNameStatusNode@@6B@  004debc4     LIBCMT:undname.obj
 0002:0001ebd8       ??_R3DNameStatusNode@@8    004debd8     LIBCMT:undname.obj
 0002:0001ebe8       ??_R2DNameStatusNode@@8    004debe8     LIBCMT:undname.obj
 0002:0001ebf4       ??_R1A@?0A@EA@DNameStatusNode@@8 004debf4     LIBCMT:undname.obj
 0002:0001ec10       ??_R4pcharNode@@6B@        004dec10     LIBCMT:undname.obj
 0002:0001ec24       ??_R3pcharNode@@8          004dec24     LIBCMT:undname.obj
 0002:0001ec34       ??_R2pcharNode@@8          004dec34     LIBCMT:undname.obj
 0002:0001ec40       ??_R1A@?0A@EA@pcharNode@@8 004dec40     LIBCMT:undname.obj
 0002:0001ec5c       ??_R4HASH64withTransform@TaoCrypt@@6B@ 004dec5c     taocrypt:hash.obj
 0002:0001ec70       ??_R3HASH64withTransform@TaoCrypt@@8 004dec70     taocrypt:hash.obj
 0002:0001ec80       ??_R2HASH64withTransform@TaoCrypt@@8 004dec80     taocrypt:hash.obj
 0002:0001ec90       ??_R1A@?0A@EA@HASH64withTransform@TaoCrypt@@8 004dec90     taocrypt:hash.obj
 0002:0001ecac       ??_R4HASHwithTransform@TaoCrypt@@6B@ 004decac     taocrypt:hash.obj
 0002:0001ecc0       ??_R4MultiplicativeGroupT@AbstractRing@TaoCrypt@@6B@ 004decc0     taocrypt:integer.obj
 0002:0001ecd4       ??_R3MultiplicativeGroupT@AbstractRing@TaoCrypt@@8 004decd4     taocrypt:integer.obj
 0002:0001ece4       ??_R2MultiplicativeGroupT@AbstractRing@TaoCrypt@@8 004dece4     taocrypt:integer.obj
 0002:0001ecf4       ??_R1A@?0A@EA@MultiplicativeGroupT@AbstractRing@TaoCrypt@@8 004decf4     taocrypt:integer.obj
 0002:0001ed10       ??_R1A@?0A@EA@AbstractGroup@TaoCrypt@@8 004ded10     taocrypt:integer.obj
 0002:0001ed2c       ??_R3AbstractGroup@TaoCrypt@@8 004ded2c     taocrypt:integer.obj
 0002:0001ed3c       ??_R2AbstractGroup@TaoCrypt@@8 004ded3c     taocrypt:integer.obj
 0002:0001ed48       ??_R4ModularArithmetic@TaoCrypt@@6B@ 004ded48     taocrypt:integer.obj
 0002:0001ed5c       ??_R3ModularArithmetic@TaoCrypt@@8 004ded5c     taocrypt:integer.obj
 0002:0001ed6c       ??_R2ModularArithmetic@TaoCrypt@@8 004ded6c     taocrypt:integer.obj
 0002:0001ed80       ??_R1A@?0A@EA@ModularArithmetic@TaoCrypt@@8 004ded80     taocrypt:integer.obj
 0002:0001ed9c       ??_R1A@?0A@EA@AbstractRing@TaoCrypt@@8 004ded9c     taocrypt:integer.obj
 0002:0001edb8       ??_R3AbstractRing@TaoCrypt@@8 004dedb8     taocrypt:integer.obj
 0002:0001edc8       ??_R2AbstractRing@TaoCrypt@@8 004dedc8     taocrypt:integer.obj
 0002:0001edd8       ??_R4MontgomeryRepresentation@TaoCrypt@@6B@ 004dedd8     taocrypt:integer.obj
 0002:0001edec       ??_R3MontgomeryRepresentation@TaoCrypt@@8 004dedec     taocrypt:integer.obj
 0002:0001edfc       ??_R2MontgomeryRepresentation@TaoCrypt@@8 004dedfc     taocrypt:integer.obj
 0002:0001ee14       ??_R1A@?0A@EA@MontgomeryRepresentation@TaoCrypt@@8 004dee14     taocrypt:integer.obj
 0002:0001ee30       ??_R4EuclideanDomainOf@TaoCrypt@@6B@ 004dee30     taocrypt:integer.obj
 0002:0001ee44       ??_R3EuclideanDomainOf@TaoCrypt@@8 004dee44     taocrypt:integer.obj
 0002:0001ee54       ??_R2EuclideanDomainOf@TaoCrypt@@8 004dee54     taocrypt:integer.obj
 0002:0001ee6c       ??_R1A@?0A@EA@EuclideanDomainOf@TaoCrypt@@8 004dee6c     taocrypt:integer.obj
 0002:0001ee88       ??_R1A@?0A@EA@AbstractEuclideanDomain@TaoCrypt@@8 004dee88     taocrypt:integer.obj
 0002:0001eea4       ??_R3AbstractEuclideanDomain@TaoCrypt@@8 004deea4     taocrypt:integer.obj
 0002:0001eeb4       ??_R2AbstractEuclideanDomain@TaoCrypt@@8 004deeb4     taocrypt:integer.obj
 0002:0001eec8       ??_R4SHA256@TaoCrypt@@6B@  004deec8     taocrypt:sha.obj
 0002:0001eedc       ??_R3SHA256@TaoCrypt@@8    004deedc     taocrypt:sha.obj
 0002:0001eeec       ??_R2SHA256@TaoCrypt@@8    004deeec     taocrypt:sha.obj
 0002:0001ef00       ??_R1A@?0A@EA@SHA256@TaoCrypt@@8 004def00     taocrypt:sha.obj
 0002:0001ef1c       ??_R4SHA224@TaoCrypt@@6B@  004def1c     taocrypt:sha.obj
 0002:0001ef30       ??_R3SHA224@TaoCrypt@@8    004def30     taocrypt:sha.obj
 0002:0001ef40       ??_R2SHA224@TaoCrypt@@8    004def40     taocrypt:sha.obj
 0002:0001ef54       ??_R1A@?0A@EA@SHA224@TaoCrypt@@8 004def54     taocrypt:sha.obj
 0002:0001ef70       ??_R4SHA512@TaoCrypt@@6B@  004def70     taocrypt:sha.obj
 0002:0001ef84       ??_R3SHA512@TaoCrypt@@8    004def84     taocrypt:sha.obj
 0002:0001ef94       ??_R2SHA512@TaoCrypt@@8    004def94     taocrypt:sha.obj
 0002:0001efa8       ??_R1A@?0A@EA@SHA512@TaoCrypt@@8 004defa8     taocrypt:sha.obj
 0002:0001efc4       ??_R4SHA384@TaoCrypt@@6B@  004defc4     taocrypt:sha.obj
 0002:0001efd8       ??_R3SHA384@TaoCrypt@@8    004defd8     taocrypt:sha.obj
 0002:0001efe8       ??_R2SHA384@TaoCrypt@@8    004defe8     taocrypt:sha.obj
 0002:0001effc       ??_R1A@?0A@EA@SHA384@TaoCrypt@@8 004deffc     taocrypt:sha.obj
 0002:0001f018       ??_R4BER_Decoder@TaoCrypt@@6B@ 004df018     taocrypt:dsa.obj
 0002:0001f02c       ??_R3BER_Decoder@TaoCrypt@@8 004df02c     taocrypt:dsa.obj
 0002:0001f03c       ??_R2BER_Decoder@TaoCrypt@@8 004df03c     taocrypt:dsa.obj
 0002:0001f048       ??_R1A@?0A@EA@BER_Decoder@TaoCrypt@@8 004df048     taocrypt:dsa.obj
 0002:0001f064       ??_R4DSA_Private_Decoder@TaoCrypt@@6B@ 004df064     taocrypt:dsa.obj
 0002:0001f078       ??_R3DSA_Private_Decoder@TaoCrypt@@8 004df078     taocrypt:dsa.obj
 0002:0001f088       ??_R2DSA_Private_Decoder@TaoCrypt@@8 004df088     taocrypt:dsa.obj
 0002:0001f098       ??_R1A@?0A@EA@DSA_Private_Decoder@TaoCrypt@@8 004df098     taocrypt:dsa.obj
 0002:0001f0b4       ??_R4DSA_Public_Decoder@TaoCrypt@@6B@ 004df0b4     taocrypt:dsa.obj
 0002:0001f0c8       ??_R3DSA_Public_Decoder@TaoCrypt@@8 004df0c8     taocrypt:dsa.obj
 0002:0001f0d8       ??_R2DSA_Public_Decoder@TaoCrypt@@8 004df0d8     taocrypt:dsa.obj
 0002:0001f0e8       ??_R1A@?0A@EA@DSA_Public_Decoder@TaoCrypt@@8 004df0e8     taocrypt:dsa.obj
 0002:0001f104       ??_R4DH_Decoder@TaoCrypt@@6B@ 004df104     taocrypt:dh.obj
 0002:0001f118       ??_R3DH_Decoder@TaoCrypt@@8 004df118     taocrypt:dh.obj
 0002:0001f128       ??_R2DH_Decoder@TaoCrypt@@8 004df128     taocrypt:dh.obj
 0002:0001f138       ??_R1A@?0A@EA@DH_Decoder@TaoCrypt@@8 004df138     taocrypt:dh.obj
 0002:0001f154       ??_R4RSA_Private_Decoder@TaoCrypt@@6B@ 004df154     taocrypt:rsa.obj
 0002:0001f168       ??_R3RSA_Private_Decoder@TaoCrypt@@8 004df168     taocrypt:rsa.obj
 0002:0001f178       ??_R2RSA_Private_Decoder@TaoCrypt@@8 004df178     taocrypt:rsa.obj
 0002:0001f188       ??_R1A@?0A@EA@RSA_Private_Decoder@TaoCrypt@@8 004df188     taocrypt:rsa.obj
 0002:0001f1a4       ??_R4RSA_Public_Decoder@TaoCrypt@@6B@ 004df1a4     taocrypt:rsa.obj
 0002:0001f1b8       ??_R3RSA_Public_Decoder@TaoCrypt@@8 004df1b8     taocrypt:rsa.obj
 0002:0001f1c8       ??_R2RSA_Public_Decoder@TaoCrypt@@8 004df1c8     taocrypt:rsa.obj
 0002:0001f1d8       ??_R1A@?0A@EA@RSA_Public_Decoder@TaoCrypt@@8 004df1d8     taocrypt:rsa.obj
 0002:0001f1f4       ??_R4PKCS12_Decoder@TaoCrypt@@6B@ 004df1f4     taocrypt:asn.obj
 0002:0001f208       ??_R3PKCS12_Decoder@TaoCrypt@@8 004df208     taocrypt:asn.obj
 0002:0001f218       ??_R2PKCS12_Decoder@TaoCrypt@@8 004df218     taocrypt:asn.obj
 0002:0001f228       ??_R1A@?0A@EA@PKCS12_Decoder@TaoCrypt@@8 004df228     taocrypt:asn.obj
 0002:0001f244       ??_R4DER_Encoder@TaoCrypt@@6B@ 004df244     taocrypt:asn.obj
 0002:0001f258       ??_R3DER_Encoder@TaoCrypt@@8 004df258     taocrypt:asn.obj
 0002:0001f268       ??_R2DER_Encoder@TaoCrypt@@8 004df268     taocrypt:asn.obj
 0002:0001f274       ??_R1A@?0A@EA@DER_Encoder@TaoCrypt@@8 004df274     taocrypt:asn.obj
 0002:0001f290       ??_R4CertDecoder@TaoCrypt@@6B@ 004df290     taocrypt:asn.obj
 0002:0001f2a4       ??_R3CertDecoder@TaoCrypt@@8 004df2a4     taocrypt:asn.obj
 0002:0001f2b4       ??_R2CertDecoder@TaoCrypt@@8 004df2b4     taocrypt:asn.obj
 0002:0001f2c4       ??_R1A@?0A@EA@CertDecoder@TaoCrypt@@8 004df2c4     taocrypt:asn.obj
 0002:0001f2e0       ??_R4Signature_Encoder@TaoCrypt@@6B@ 004df2e0     taocrypt:asn.obj
 0002:0001f2f4       ??_R3Signature_Encoder@TaoCrypt@@8 004df2f4     taocrypt:asn.obj
 0002:0001f304       ??_R2Signature_Encoder@TaoCrypt@@8 004df304     taocrypt:asn.obj
 0002:0001f314       ??_R1A@?0A@EA@Signature_Encoder@TaoCrypt@@8 004df314     taocrypt:asn.obj
 0002:0001f330       ??_R4MD2@TaoCrypt@@6B@     004df330     taocrypt:md2.obj
 0002:0001f344       ??_R3MD2@TaoCrypt@@8       004df344     taocrypt:md2.obj
 0002:0001f354       ??_R2MD2@TaoCrypt@@8       004df354     taocrypt:md2.obj
 0002:0001f364       ??_R1A@?0A@EA@MD2@TaoCrypt@@8 004df364     taocrypt:md2.obj
 0002:0001fa30       ___safe_se_handler_table   004dfa30     <linker-defined>
 0002:0001fb40       ___rtc_iaa                 004dfb40     LIBCMT:initsect.obj
 0002:0001fc44       ___rtc_izz                 004dfc44     LIBCMT:initsect.obj
 0002:0001fd48       ___rtc_taa                 004dfd48     LIBCMT:initsect.obj
 0002:0001fe4c       ___rtc_tzz                 004dfe4c     LIBCMT:initsect.obj
 0002:0001ff50       __TI2?AVbad_alloc@std@@    004dff50     LIBCMT:new.obj
 0002:0001ff60       __CTA2?AVbad_alloc@std@@   004dff60     LIBCMT:new.obj
 0002:0001ff6c       __CT??_R0?AVbad_alloc@std@@@8??0bad_alloc@std@@QAE@ABV01@@Z12 004dff6c     LIBCMT:new.obj
 0002:0001ff88       __CT??_R0?AVexception@std@@@8??0exception@std@@QAE@ABV01@@Z12 004dff88     LIBCMT:new.obj
 0003:00000008       ??_R0?AVCommand@@@8        004e1008     command.obj
 0003:00000028       ??_R0?AVInstance_cmd@@@8   004e1028     commands.obj
 0003:00000048       ??_R0?AVAbstract_instance_cmd@@@8 004e1048     commands.obj
 0003:00000074       ??_R0?AVShow_instance_status@@@8 004e1074     commands.obj
 0003:000000a0       ??_R0?AVShow_instance_options@@@8 004e10a0     commands.obj
 0003:000000cc       ??_R0?AVStart_instance@@@8 004e10cc     commands.obj
 0003:000000f0       ??_R0?AVStop_instance@@@8  004e10f0     commands.obj
 0003:00000114       ??_R0?AVCreate_instance@@@8 004e1114     commands.obj
 0003:00000138       ??_R0?AVDrop_instance@@@8  004e1138     commands.obj
 0003:0000015c       ??_R0?AVShow_instance_log@@@8 004e115c     commands.obj
 0003:00000184       ??_R0?AVShow_instance_log_files@@@8 004e1184     commands.obj
 0003:000001b4       ??_R0?AVAbstract_option_cmd@@@8 004e11b4     commands.obj
 0003:000001e0       ??_R0?AVThread@@@8         004e11e0     guardian.obj
 0003:000001fc       ??_R0?AVGuardian@@@8       004e11fc     guardian.obj
 0003:0000021c       ??_R0?AVInstance_monitor@@@8 004e121c     instance.obj
 0003:00000270       ??_R0?AVListener@@@8       004e1270     listener.obj
 0003:00000294       ??_R0?AVThreadModelChecker@?A0x2a2a756e@@@8 004e1294     manager.obj
 0003:000002d4       ??_R0?AVMysql_connection@@@8 004e12d4     mysql_connection.obj
 0003:00000304       ?config_file@Main@Options@@2PBDB 004e1304     options.obj
 0003:00000308       ?password_file_name@Main@Options@@2PBDB 004e1308     options.obj
 0003:0000030c       ?pid_file_name@Main@Options@@2PBDB 004e130c     options.obj
 0003:00000310       ?default_mysqld_path@Main@Options@@2PBDB 004e1310     options.obj
 0003:00000314       ?monitoring_interval@Main@Options@@2IA 004e1314     options.obj
 0003:00000318       ?port_number@Main@Options@@2IA 004e1318     options.obj
 0003:00000af8       ??_R0?AVUser_management_cmd@@@8 004e1af8     options.obj
 0003:00000b20       ??_R0?AVPrint_password_line_cmd@@@8 004e1b20     options.obj
 0003:00000b50       ??_R0?AVAdd_user_cmd@@@8   004e1b50     options.obj
 0003:00000b70       ??_R0?AVDrop_user_cmd@@@8  004e1b70     options.obj
 0003:00000b94       ??_R0?AVEdit_user_cmd@@@8  004e1b94     options.obj
 0003:00000bb8       ??_R0?AVClean_db_cmd@@@8   004e1bb8     options.obj
 0003:00000bd8       ??_R0?AVCheck_db_cmd@@@8   004e1bd8     options.obj
 0003:00000bf8       ??_R0?AVList_users_cmd@@@8 004e1bf8     options.obj
 0003:00000ccc       ??_R0?AVShow_instances@@@8 004e1ccc     parse.obj
 0003:00000cf0       ??_R0?AVFlush_instances@@@8 004e1cf0     parse.obj
 0003:00000d14       ??_R0?AVSet_option@@@8     004e1d14     parse.obj
 0003:00000d34       ??_R0?AVUnset_option@@@8   004e1d34     parse.obj
 0003:00000d54       ??_R0?AVSyntax_error@@@8   004e1d54     parse.obj
 0003:00000d78       ??_R0?AVMysqld_output_parser@?A0x60d3fd73@@@8 004e1d78     parse_output.obj
 0003:00000db4       ??_R0?AVMysqld_output_parser_win@?A0x60d3fd73@@@8 004e1db4     parse_output.obj
 0003:00000df8       ?net_buffer_length@@3KA    004e1df8     priv.obj
 0003:00000dfc       ?max_allowed_packet@@3KA   004e1dfc     priv.obj
 0003:00000e00       ?net_read_timeout@@3KA     004e1e00     priv.obj
 0003:00000e04       ?net_write_timeout@@3KA    004e1e04     priv.obj
 0003:00000e08       ?net_retry_count@@3KA      004e1e08     priv.obj
 0003:00000e0c       ?mysqld_net_retry_count@@3KA 004e1e0c     priv.obj
 0003:00000e2c       ??_R0?AVIMService@@@8      004e1e2c     IMService.obj
 0003:00000e48       ??_R0?AVWindowsService@@@8 004e1e48     IMService.obj
 0003:00000e78       _sqlstate_map              004e1e78     sql_state.obj
 0003:00001a40       _unknown_sqlstate          004e2a40     client.obj
 0003:00001a44       _not_error_sqlstate        004e2a44     client.obj
 0003:00001a48       _cant_connect_sqlstate     004e2a48     client.obj
 0003:00001a4c       _default_client_charset_info 004e2a4c     client.obj
 0003:00001aec       _sql_protocol_names_lib    004e2aec     client.obj
 0003:00001b00       _sql_protocol_typelib      004e2b00     client.obj
 0003:00001b58       _client_errors             004e2b58     errmsg.obj
 0003:00001c74       _default_charset_info      004e2c74     mysys:charset.obj
 0003:00001de4       _my_thread_end_wait_time   004e2de4     mysys:my_thr_init.obj
 0003:00001de8       _my_umask                  004e2de8     mysys:my_static.obj
 0003:00001dec       _my_umask_dir              004e2dec     mysys:my_static.obj
 0003:00001df0       _my_file_limit             004e2df0     mysys:my_static.obj
 0003:00001df4       _my_file_info              004e2df4     mysys:my_static.obj
 0003:00001df8       _my_default_record_cache_size 004e2df8     mysys:my_static.obj
 0003:00001dfc       _soundex_map               004e2dfc     mysys:my_static.obj
 0003:00001e00       _my_once_extra             004e2e00     mysys:my_static.obj
 0003:00001e04       _sf_min_adress             004e2e04     mysys:my_static.obj
 0003:00001e08       _my_time_to_wait_for_lock  004e2e08     mysys:my_static.obj
 0003:00001e0c       _my_abort_hook             004e2e0c     mysys:my_static.obj
 0003:00001e10       _error_handler_hook        004e2e10     mysys:my_static.obj
 0003:00001e14       _fatal_error_handler_hook  004e2e14     mysys:my_static.obj
 0003:00001e18       _my_thread_stack_size      004e2e18     mysys:my_init.obj
 0003:00001e1c       _my_getopt_error_reporter  004e2e1c     mysys:my_getopt.obj
 0003:00001e38       _disabled_my_option        004e2e38     mysys:my_getopt.obj
 0003:00001e3c       _my_getopt_print_errors    004e2e3c     mysys:my_getopt.obj
 0003:00001e40       _my_pthread_create_detached 004e2e40     mysys:my_pthread.obj
 0003:00001e60       _next_alarm_expire_time    004e2e60     mysys:thr_alarm.obj
 0003:00001e68       _globerrs                  004e2e68     mysys:errors.obj
 0003:00001ee0       __dig_vec_upper            004e2ee0     strings:int2str.obj
 0003:00001f08       __dig_vec_lower            004e2f08     strings:int2str.obj
 0003:00002360       _cs_to_uni                 004e3360     strings:ctype-latin1.obj
 0003:00002560       _pl00                      004e3560     strings:ctype-latin1.obj
 0003:00002660       _pl01                      004e3660     strings:ctype-latin1.obj
 0003:00002760       _pl02                      004e3760     strings:ctype-latin1.obj
 0003:00002860       _pl20                      004e3860     strings:ctype-latin1.obj
 0003:00002960       _pl21                      004e3960     strings:ctype-latin1.obj
 0003:00002a60       _uni_to_cs                 004e3a60     strings:ctype-latin1.obj
 0003:00002ed0       _my_charset_latin1         004e3ed0     strings:ctype-latin1.obj
 0003:00003040       _combo1map                 004e4040     strings:ctype-latin1.obj
 0003:00003140       _combo2map                 004e4140     strings:ctype-latin1.obj
 0003:00003270       _my_charset_latin1_german2_ci 004e4270     strings:ctype-latin1.obj
 0003:000032e0       _my_charset_latin1_bin     004e42e0     strings:ctype-latin1.obj
 0003:000033f0       _my_charset_8bit_handler   004e43f0     strings:ctype-simple.obj
 0003:0000345c       _my_collation_8bit_simple_ci_handler 004e445c     strings:ctype-simple.obj
 0003:00003690       _my_collation_8bit_bin_handler 004e4690     strings:ctype-bin.obj
 0003:00003758       _my_charset_bin            004e4758     strings:ctype-bin.obj
 0003:000038c0       _page000data               004e48c0     strings:ctype-uca.obj
 0003:000040c0       _page001data               004e50c0     strings:ctype-uca.obj
 0003:000046c0       _page002data               004e56c0     strings:ctype-uca.obj
 0003:00004cc0       _page003data               004e5cc0     strings:ctype-uca.obj
 0003:000054c0       _page004data               004e64c0     strings:ctype-uca.obj
 0003:00005ac0       _page005data               004e6ac0     strings:ctype-uca.obj
 0003:000060c0       _page006data               004e70c0     strings:ctype-uca.obj
 0003:000066c0       _page007data               004e76c0     strings:ctype-uca.obj
 0003:00006cc0       _page009data               004e7cc0     strings:ctype-uca.obj
 0003:000072c0       _page00Adata               004e82c0     strings:ctype-uca.obj
 0003:000078c0       _page00Bdata               004e88c0     strings:ctype-uca.obj
 0003:00007ec0       _page00Cdata               004e8ec0     strings:ctype-uca.obj
 0003:000084c0       _page00Ddata               004e94c0     strings:ctype-uca.obj
 0003:00008ac0       _page00Edata               004e9ac0     strings:ctype-uca.obj
 0003:000090c0       _page00Fdata               004ea0c0     strings:ctype-uca.obj
 0003:000096c0       _page010data               004ea6c0     strings:ctype-uca.obj
 0003:00009cc0       _page011data               004eacc0     strings:ctype-uca.obj
 0003:0000a2c0       _page012data               004eb2c0     strings:ctype-uca.obj
 0003:0000a8c0       _page013data               004eb8c0     strings:ctype-uca.obj
 0003:0000aec0       _page014data               004ebec0     strings:ctype-uca.obj
 0003:0000b4c0       _page015data               004ec4c0     strings:ctype-uca.obj
 0003:0000b8c0       _page016data               004ec8c0     strings:ctype-uca.obj
 0003:0000bec0       _page017data               004ecec0     strings:ctype-uca.obj
 0003:0000c4c0       _page018data               004ed4c0     strings:ctype-uca.obj
 0003:0000cac0       _page019data               004edac0     strings:ctype-uca.obj
 0003:0000d0c0       _page01Ddata               004ee0c0     strings:ctype-uca.obj
 0003:0000d6c0       _page01Edata               004ee6c0     strings:ctype-uca.obj
 0003:0000dcc0       _page01Fdata               004eecc0     strings:ctype-uca.obj
 0003:0000e2c0       _page020data               004ef2c0     strings:ctype-uca.obj
 0003:0000ecc0       _page021data               004efcc0     strings:ctype-uca.obj
 0003:0000f6c0       _page022data               004f06c0     strings:ctype-uca.obj
 0003:0000fec0       _page023data               004f0ec0     strings:ctype-uca.obj
 0003:000104c0       _page024data               004f14c0     strings:ctype-uca.obj
 0003:00010ec0       _page025data               004f1ec0     strings:ctype-uca.obj
 0003:000112c0       _page026data               004f22c0     strings:ctype-uca.obj
 0003:000118c0       _page027data               004f28c0     strings:ctype-uca.obj
 0003:00011ec0       _page028data               004f2ec0     strings:ctype-uca.obj
 0003:000122c0       _page029data               004f32c0     strings:ctype-uca.obj
 0003:000126c0       _page02Adata               004f36c0     strings:ctype-uca.obj
 0003:000130c0       _page02Bdata               004f40c0     strings:ctype-uca.obj
 0003:000136c0       _page02Edata               004f46c0     strings:ctype-uca.obj
 0003:00013cc0       _page02Fdata               004f4cc0     strings:ctype-uca.obj
 0003:000142c0       _page030data               004f52c0     strings:ctype-uca.obj
 0003:000148c0       _page031data               004f58c0     strings:ctype-uca.obj
 0003:00014ec0       _page032data               004f5ec0     strings:ctype-uca.obj
 0003:00015ec0       _page033data               004f6ec0     strings:ctype-uca.obj
 0003:000170c0       _page04Ddata               004f80c0     strings:ctype-uca.obj
 0003:000176c0       _page0A0data               004f86c0     strings:ctype-uca.obj
 0003:00017ac0       _page0A1data               004f8ac0     strings:ctype-uca.obj
 0003:00017ec0       _page0A2data               004f8ec0     strings:ctype-uca.obj
 0003:000182c0       _page0A3data               004f92c0     strings:ctype-uca.obj
 0003:000186c0       _page0A4data               004f96c0     strings:ctype-uca.obj
 0003:00018cc0       _page0F9data               004f9cc0     strings:ctype-uca.obj
 0003:000192c0       _page0FAdata               004fa2c0     strings:ctype-uca.obj
 0003:000198c0       _page0FBdata               004fa8c0     strings:ctype-uca.obj
 0003:0001a0c0       _page0FCdata               004fb0c0     strings:ctype-uca.obj
 0003:0001a6c0       _page0FDdata               004fb6c0     strings:ctype-uca.obj
 0003:0001b8c0       _page0FEdata               004fc8c0     strings:ctype-uca.obj
 0003:0001bec0       _page0FFdata               004fcec0     strings:ctype-uca.obj
 0003:0001c4c0       _uca_length                004fd4c0     strings:ctype-uca.obj
 0003:0001c5c0       _uca_weight                004fd5c0     strings:ctype-uca.obj
 0003:0001c9d0       _my_collation_ucs2_uca_handler 004fd9d0     strings:ctype-uca.obj
 0003:0001c9fc       _my_collation_any_uca_handler 004fd9fc     strings:ctype-uca.obj
 0003:0001ca28       _my_charset_ucs2_unicode_ci 004fda28     strings:ctype-uca.obj
 0003:0001ca98       _my_charset_ucs2_icelandic_uca_ci 004fda98     strings:ctype-uca.obj
 0003:0001cb08       _my_charset_ucs2_latvian_uca_ci 004fdb08     strings:ctype-uca.obj
 0003:0001cb78       _my_charset_ucs2_romanian_uca_ci 004fdb78     strings:ctype-uca.obj
 0003:0001cbe8       _my_charset_ucs2_slovenian_uca_ci 004fdbe8     strings:ctype-uca.obj
 0003:0001cc58       _my_charset_ucs2_polish_uca_ci 004fdc58     strings:ctype-uca.obj
 0003:0001ccc8       _my_charset_ucs2_estonian_uca_ci 004fdcc8     strings:ctype-uca.obj
 0003:0001cd38       _my_charset_ucs2_spanish_uca_ci 004fdd38     strings:ctype-uca.obj
 0003:0001cda8       _my_charset_ucs2_swedish_uca_ci 004fdda8     strings:ctype-uca.obj
 0003:0001ce18       _my_charset_ucs2_turkish_uca_ci 004fde18     strings:ctype-uca.obj
 0003:0001ce88       _my_charset_ucs2_czech_uca_ci 004fde88     strings:ctype-uca.obj
 0003:0001cef8       _my_charset_ucs2_danish_uca_ci 004fdef8     strings:ctype-uca.obj
 0003:0001cf68       _my_charset_ucs2_lithuanian_uca_ci 004fdf68     strings:ctype-uca.obj
 0003:0001cfd8       _my_charset_ucs2_slovak_uca_ci 004fdfd8     strings:ctype-uca.obj
 0003:0001d048       _my_charset_ucs2_spanish2_uca_ci 004fe048     strings:ctype-uca.obj
 0003:0001d0b8       _my_charset_ucs2_roman_uca_ci 004fe0b8     strings:ctype-uca.obj
 0003:0001d128       _my_charset_ucs2_persian_uca_ci 004fe128     strings:ctype-uca.obj
 0003:0001d198       _my_charset_ucs2_esperanto_uca_ci 004fe198     strings:ctype-uca.obj
 0003:0001d208       _my_charset_ucs2_hungarian_uca_ci 004fe208     strings:ctype-uca.obj
 0003:0001d380       _my_charset_utf8_unicode_ci 004fe380     strings:ctype-uca.obj
 0003:0001d3f0       _my_charset_utf8_icelandic_uca_ci 004fe3f0     strings:ctype-uca.obj
 0003:0001d460       _my_charset_utf8_latvian_uca_ci 004fe460     strings:ctype-uca.obj
 0003:0001d4d0       _my_charset_utf8_romanian_uca_ci 004fe4d0     strings:ctype-uca.obj
 0003:0001d540       _my_charset_utf8_slovenian_uca_ci 004fe540     strings:ctype-uca.obj
 0003:0001d5b0       _my_charset_utf8_polish_uca_ci 004fe5b0     strings:ctype-uca.obj
 0003:0001d620       _my_charset_utf8_estonian_uca_ci 004fe620     strings:ctype-uca.obj
 0003:0001d690       _my_charset_utf8_spanish_uca_ci 004fe690     strings:ctype-uca.obj
 0003:0001d700       _my_charset_utf8_swedish_uca_ci 004fe700     strings:ctype-uca.obj
 0003:0001d770       _my_charset_utf8_turkish_uca_ci 004fe770     strings:ctype-uca.obj
 0003:0001d7e0       _my_charset_utf8_czech_uca_ci 004fe7e0     strings:ctype-uca.obj
 0003:0001d850       _my_charset_utf8_danish_uca_ci 004fe850     strings:ctype-uca.obj
 0003:0001d8c0       _my_charset_utf8_lithuanian_uca_ci 004fe8c0     strings:ctype-uca.obj
 0003:0001d930       _my_charset_utf8_slovak_uca_ci 004fe930     strings:ctype-uca.obj
 0003:0001d9a0       _my_charset_utf8_spanish2_uca_ci 004fe9a0     strings:ctype-uca.obj
 0003:0001da10       _my_charset_utf8_roman_uca_ci 004fea10     strings:ctype-uca.obj
 0003:0001da80       _my_charset_utf8_persian_uca_ci 004fea80     strings:ctype-uca.obj
 0003:0001daf0       _my_charset_utf8_esperanto_uca_ci 004feaf0     strings:ctype-uca.obj
 0003:0001db60       _my_charset_utf8_hungarian_uca_ci 004feb60     strings:ctype-uca.obj
 0003:00030f00       _my_charset_cp932_japanese_ci 00511f00     strings:ctype-cp932.obj
 0003:00030f70       _my_charset_cp932_bin      00511f70     strings:ctype-cp932.obj
 0003:00030fe0       _ctype_dec8_swedish_ci     00511fe0     strings:ctype-extra.obj
 0003:000310e8       _to_lower_dec8_swedish_ci  005120e8     strings:ctype-extra.obj
 0003:000311e8       _to_upper_dec8_swedish_ci  005121e8     strings:ctype-extra.obj
 0003:000312e8       _sort_order_dec8_swedish_ci 005122e8     strings:ctype-extra.obj
 0003:000313e8       _to_uni_dec8_swedish_ci    005123e8     strings:ctype-extra.obj
 0003:000315e8       _ctype_cp850_general_ci    005125e8     strings:ctype-extra.obj
 0003:000316f0       _to_lower_cp850_general_ci 005126f0     strings:ctype-extra.obj
 0003:000317f0       _to_upper_cp850_general_ci 005127f0     strings:ctype-extra.obj
 0003:000318f0       _sort_order_cp850_general_ci 005128f0     strings:ctype-extra.obj
 0003:000319f0       _to_uni_cp850_general_ci   005129f0     strings:ctype-extra.obj
 0003:00031bf0       _ctype_latin1_german1_ci   00512bf0     strings:ctype-extra.obj
 0003:00031cf8       _to_lower_latin1_german1_ci 00512cf8     strings:ctype-extra.obj
 0003:00031df8       _to_upper_latin1_german1_ci 00512df8     strings:ctype-extra.obj
 0003:00031ef8       _sort_order_latin1_german1_ci 00512ef8     strings:ctype-extra.obj
 0003:00031ff8       _to_uni_latin1_german1_ci  00512ff8     strings:ctype-extra.obj
 0003:000321f8       _ctype_hp8_english_ci      005131f8     strings:ctype-extra.obj
 0003:00032300       _to_lower_hp8_english_ci   00513300     strings:ctype-extra.obj
 0003:00032400       _to_upper_hp8_english_ci   00513400     strings:ctype-extra.obj
 0003:00032500       _sort_order_hp8_english_ci 00513500     strings:ctype-extra.obj
 0003:00032600       _to_uni_hp8_english_ci     00513600     strings:ctype-extra.obj
 0003:00032800       _ctype_koi8r_general_ci    00513800     strings:ctype-extra.obj
 0003:00032908       _to_lower_koi8r_general_ci 00513908     strings:ctype-extra.obj
 0003:00032a08       _to_upper_koi8r_general_ci 00513a08     strings:ctype-extra.obj
 0003:00032b08       _sort_order_koi8r_general_ci 00513b08     strings:ctype-extra.obj
 0003:00032c08       _to_uni_koi8r_general_ci   00513c08     strings:ctype-extra.obj
 0003:00032e08       _ctype_latin2_general_ci   00513e08     strings:ctype-extra.obj
 0003:00032f10       _to_lower_latin2_general_ci 00513f10     strings:ctype-extra.obj
 0003:00033010       _to_upper_latin2_general_ci 00514010     strings:ctype-extra.obj
 0003:00033110       _sort_order_latin2_general_ci 00514110     strings:ctype-extra.obj
 0003:00033210       _to_uni_latin2_general_ci  00514210     strings:ctype-extra.obj
 0003:00033410       _ctype_swe7_swedish_ci     00514410     strings:ctype-extra.obj
 0003:00033518       _to_lower_swe7_swedish_ci  00514518     strings:ctype-extra.obj
 0003:00033618       _to_upper_swe7_swedish_ci  00514618     strings:ctype-extra.obj
 0003:00033718       _sort_order_swe7_swedish_ci 00514718     strings:ctype-extra.obj
 0003:00033818       _to_uni_swe7_swedish_ci    00514818     strings:ctype-extra.obj
 0003:00033a18       _ctype_ascii_general_ci    00514a18     strings:ctype-extra.obj
 0003:00033b20       _to_lower_ascii_general_ci 00514b20     strings:ctype-extra.obj
 0003:00033c20       _to_upper_ascii_general_ci 00514c20     strings:ctype-extra.obj
 0003:00033d20       _sort_order_ascii_general_ci 00514d20     strings:ctype-extra.obj
 0003:00033e20       _to_uni_ascii_general_ci   00514e20     strings:ctype-extra.obj
 0003:00034020       _ctype_cp1251_bulgarian_ci 00515020     strings:ctype-extra.obj
 0003:00034128       _to_lower_cp1251_bulgarian_ci 00515128     strings:ctype-extra.obj
 0003:00034228       _to_upper_cp1251_bulgarian_ci 00515228     strings:ctype-extra.obj
 0003:00034328       _sort_order_cp1251_bulgarian_ci 00515328     strings:ctype-extra.obj
 0003:00034428       _to_uni_cp1251_bulgarian_ci 00515428     strings:ctype-extra.obj
 0003:00034628       _ctype_latin1_danish_ci    00515628     strings:ctype-extra.obj
 0003:00034730       _to_lower_latin1_danish_ci 00515730     strings:ctype-extra.obj
 0003:00034830       _to_upper_latin1_danish_ci 00515830     strings:ctype-extra.obj
 0003:00034930       _sort_order_latin1_danish_ci 00515930     strings:ctype-extra.obj
 0003:00034a30       _to_uni_latin1_danish_ci   00515a30     strings:ctype-extra.obj
 0003:00034c30       _ctype_hebrew_general_ci   00515c30     strings:ctype-extra.obj
 0003:00034d38       _to_lower_hebrew_general_ci 00515d38     strings:ctype-extra.obj
 0003:00034e38       _to_upper_hebrew_general_ci 00515e38     strings:ctype-extra.obj
 0003:00034f38       _sort_order_hebrew_general_ci 00515f38     strings:ctype-extra.obj
 0003:00035038       _to_uni_hebrew_general_ci  00516038     strings:ctype-extra.obj
 0003:00035238       _ctype_latin7_estonian_cs  00516238     strings:ctype-extra.obj
 0003:00035340       _to_lower_latin7_estonian_cs 00516340     strings:ctype-extra.obj
 0003:00035440       _to_upper_latin7_estonian_cs 00516440     strings:ctype-extra.obj
 0003:00035540       _sort_order_latin7_estonian_cs 00516540     strings:ctype-extra.obj
 0003:00035640       _to_uni_latin7_estonian_cs 00516640     strings:ctype-extra.obj
 0003:00035840       _ctype_latin2_hungarian_ci 00516840     strings:ctype-extra.obj
 0003:00035948       _to_lower_latin2_hungarian_ci 00516948     strings:ctype-extra.obj
 0003:00035a48       _to_upper_latin2_hungarian_ci 00516a48     strings:ctype-extra.obj
 0003:00035b48       _sort_order_latin2_hungarian_ci 00516b48     strings:ctype-extra.obj
 0003:00035c48       _to_uni_latin2_hungarian_ci 00516c48     strings:ctype-extra.obj
 0003:00035e48       _ctype_koi8u_general_ci    00516e48     strings:ctype-extra.obj
 0003:00035f50       _to_lower_koi8u_general_ci 00516f50     strings:ctype-extra.obj
 0003:00036050       _to_upper_koi8u_general_ci 00517050     strings:ctype-extra.obj
 0003:00036150       _sort_order_koi8u_general_ci 00517150     strings:ctype-extra.obj
 0003:00036250       _to_uni_koi8u_general_ci   00517250     strings:ctype-extra.obj
 0003:00036450       _ctype_cp1251_ukrainian_ci 00517450     strings:ctype-extra.obj
 0003:00036558       _to_lower_cp1251_ukrainian_ci 00517558     strings:ctype-extra.obj
 0003:00036658       _to_upper_cp1251_ukrainian_ci 00517658     strings:ctype-extra.obj
 0003:00036758       _sort_order_cp1251_ukrainian_ci 00517758     strings:ctype-extra.obj
 0003:00036858       _to_uni_cp1251_ukrainian_ci 00517858     strings:ctype-extra.obj
 0003:00036a58       _ctype_greek_general_ci    00517a58     strings:ctype-extra.obj
 0003:00036b60       _to_lower_greek_general_ci 00517b60     strings:ctype-extra.obj
 0003:00036c60       _to_upper_greek_general_ci 00517c60     strings:ctype-extra.obj
 0003:00036d60       _sort_order_greek_general_ci 00517d60     strings:ctype-extra.obj
 0003:00036e60       _to_uni_greek_general_ci   00517e60     strings:ctype-extra.obj
 0003:00037060       _ctype_cp1250_general_ci   00518060     strings:ctype-extra.obj
 0003:00037168       _to_lower_cp1250_general_ci 00518168     strings:ctype-extra.obj
 0003:00037268       _to_upper_cp1250_general_ci 00518268     strings:ctype-extra.obj
 0003:00037368       _sort_order_cp1250_general_ci 00518368     strings:ctype-extra.obj
 0003:00037468       _to_uni_cp1250_general_ci  00518468     strings:ctype-extra.obj
 0003:00037668       _ctype_latin2_croatian_ci  00518668     strings:ctype-extra.obj
 0003:00037770       _to_lower_latin2_croatian_ci 00518770     strings:ctype-extra.obj
 0003:00037870       _to_upper_latin2_croatian_ci 00518870     strings:ctype-extra.obj
 0003:00037970       _sort_order_latin2_croatian_ci 00518970     strings:ctype-extra.obj
 0003:00037a70       _to_uni_latin2_croatian_ci 00518a70     strings:ctype-extra.obj
 0003:00037c70       _ctype_cp1257_lithuanian_ci 00518c70     strings:ctype-extra.obj
 0003:00037d78       _to_lower_cp1257_lithuanian_ci 00518d78     strings:ctype-extra.obj
 0003:00037e78       _to_upper_cp1257_lithuanian_ci 00518e78     strings:ctype-extra.obj
 0003:00037f78       _sort_order_cp1257_lithuanian_ci 00518f78     strings:ctype-extra.obj
 0003:00038078       _to_uni_cp1257_lithuanian_ci 00519078     strings:ctype-extra.obj
 0003:00038278       _ctype_latin5_turkish_ci   00519278     strings:ctype-extra.obj
 0003:00038380       _to_lower_latin5_turkish_ci 00519380     strings:ctype-extra.obj
 0003:00038480       _to_upper_latin5_turkish_ci 00519480     strings:ctype-extra.obj
 0003:00038580       _sort_order_latin5_turkish_ci 00519580     strings:ctype-extra.obj
 0003:00038680       _to_uni_latin5_turkish_ci  00519680     strings:ctype-extra.obj
 0003:00038880       _ctype_armscii8_general_ci 00519880     strings:ctype-extra.obj
 0003:00038988       _to_lower_armscii8_general_ci 00519988     strings:ctype-extra.obj
 0003:00038a88       _to_upper_armscii8_general_ci 00519a88     strings:ctype-extra.obj
 0003:00038b88       _sort_order_armscii8_general_ci 00519b88     strings:ctype-extra.obj
 0003:00038c88       _to_uni_armscii8_general_ci 00519c88     strings:ctype-extra.obj
 0003:00038e88       _ctype_cp866_general_ci    00519e88     strings:ctype-extra.obj
 0003:00038f90       _to_lower_cp866_general_ci 00519f90     strings:ctype-extra.obj
 0003:00039090       _to_upper_cp866_general_ci 0051a090     strings:ctype-extra.obj
 0003:00039190       _sort_order_cp866_general_ci 0051a190     strings:ctype-extra.obj
 0003:00039290       _to_uni_cp866_general_ci   0051a290     strings:ctype-extra.obj
 0003:00039490       _ctype_keybcs2_general_ci  0051a490     strings:ctype-extra.obj
 0003:00039598       _to_lower_keybcs2_general_ci 0051a598     strings:ctype-extra.obj
 0003:00039698       _to_upper_keybcs2_general_ci 0051a698     strings:ctype-extra.obj
 0003:00039798       _sort_order_keybcs2_general_ci 0051a798     strings:ctype-extra.obj
 0003:00039898       _to_uni_keybcs2_general_ci 0051a898     strings:ctype-extra.obj
 0003:00039a98       _ctype_macce_general_ci    0051aa98     strings:ctype-extra.obj
 0003:00039ba0       _to_lower_macce_general_ci 0051aba0     strings:ctype-extra.obj
 0003:00039ca0       _to_upper_macce_general_ci 0051aca0     strings:ctype-extra.obj
 0003:00039da0       _sort_order_macce_general_ci 0051ada0     strings:ctype-extra.obj
 0003:00039ea0       _to_uni_macce_general_ci   0051aea0     strings:ctype-extra.obj
 0003:0003a0a0       _ctype_macroman_general_ci 0051b0a0     strings:ctype-extra.obj
 0003:0003a1a8       _to_lower_macroman_general_ci 0051b1a8     strings:ctype-extra.obj
 0003:0003a2a8       _to_upper_macroman_general_ci 0051b2a8     strings:ctype-extra.obj
 0003:0003a3a8       _sort_order_macroman_general_ci 0051b3a8     strings:ctype-extra.obj
 0003:0003a4a8       _to_uni_macroman_general_ci 0051b4a8     strings:ctype-extra.obj
 0003:0003a6a8       _ctype_cp852_general_ci    0051b6a8     strings:ctype-extra.obj
 0003:0003a7b0       _to_lower_cp852_general_ci 0051b7b0     strings:ctype-extra.obj
 0003:0003a8b0       _to_upper_cp852_general_ci 0051b8b0     strings:ctype-extra.obj
 0003:0003a9b0       _sort_order_cp852_general_ci 0051b9b0     strings:ctype-extra.obj
 0003:0003aab0       _to_uni_cp852_general_ci   0051bab0     strings:ctype-extra.obj
 0003:0003acb0       _ctype_latin7_general_ci   0051bcb0     strings:ctype-extra.obj
 0003:0003adb8       _to_lower_latin7_general_ci 0051bdb8     strings:ctype-extra.obj
 0003:0003aeb8       _to_upper_latin7_general_ci 0051beb8     strings:ctype-extra.obj
 0003:0003afb8       _sort_order_latin7_general_ci 0051bfb8     strings:ctype-extra.obj
 0003:0003b0b8       _to_uni_latin7_general_ci  0051c0b8     strings:ctype-extra.obj
 0003:0003b2b8       _ctype_latin7_general_cs   0051c2b8     strings:ctype-extra.obj
 0003:0003b3c0       _to_lower_latin7_general_cs 0051c3c0     strings:ctype-extra.obj
 0003:0003b4c0       _to_upper_latin7_general_cs 0051c4c0     strings:ctype-extra.obj
 0003:0003b5c0       _sort_order_latin7_general_cs 0051c5c0     strings:ctype-extra.obj
 0003:0003b6c0       _to_uni_latin7_general_cs  0051c6c0     strings:ctype-extra.obj
 0003:0003b8c0       _ctype_macce_bin           0051c8c0     strings:ctype-extra.obj
 0003:0003b9c8       _to_lower_macce_bin        0051c9c8     strings:ctype-extra.obj
 0003:0003bac8       _to_upper_macce_bin        0051cac8     strings:ctype-extra.obj
 0003:0003bbc8       _to_uni_macce_bin          0051cbc8     strings:ctype-extra.obj
 0003:0003bdc8       _ctype_cp1250_croatian_ci  0051cdc8     strings:ctype-extra.obj
 0003:0003bed0       _to_lower_cp1250_croatian_ci 0051ced0     strings:ctype-extra.obj
 0003:0003bfd0       _to_upper_cp1250_croatian_ci 0051cfd0     strings:ctype-extra.obj
 0003:0003c0d0       _sort_order_cp1250_croatian_ci 0051d0d0     strings:ctype-extra.obj
 0003:0003c1d0       _to_uni_cp1250_croatian_ci 0051d1d0     strings:ctype-extra.obj
 0003:0003c3d0       _ctype_latin1_general_ci   0051d3d0     strings:ctype-extra.obj
 0003:0003c4d8       _to_lower_latin1_general_ci 0051d4d8     strings:ctype-extra.obj
 0003:0003c5d8       _to_upper_latin1_general_ci 0051d5d8     strings:ctype-extra.obj
 0003:0003c6d8       _sort_order_latin1_general_ci 0051d6d8     strings:ctype-extra.obj
 0003:0003c7d8       _to_uni_latin1_general_ci  0051d7d8     strings:ctype-extra.obj
 0003:0003c9d8       _ctype_latin1_general_cs   0051d9d8     strings:ctype-extra.obj
 0003:0003cae0       _to_lower_latin1_general_cs 0051dae0     strings:ctype-extra.obj
 0003:0003cbe0       _to_upper_latin1_general_cs 0051dbe0     strings:ctype-extra.obj
 0003:0003cce0       _sort_order_latin1_general_cs 0051dce0     strings:ctype-extra.obj
 0003:0003cde0       _to_uni_latin1_general_cs  0051dde0     strings:ctype-extra.obj
 0003:0003cfe0       _ctype_cp1251_bin          0051dfe0     strings:ctype-extra.obj
 0003:0003d0e8       _to_lower_cp1251_bin       0051e0e8     strings:ctype-extra.obj
 0003:0003d1e8       _to_upper_cp1251_bin       0051e1e8     strings:ctype-extra.obj
 0003:0003d2e8       _to_uni_cp1251_bin         0051e2e8     strings:ctype-extra.obj
 0003:0003d4e8       _ctype_cp1251_general_ci   0051e4e8     strings:ctype-extra.obj
 0003:0003d5f0       _to_lower_cp1251_general_ci 0051e5f0     strings:ctype-extra.obj
 0003:0003d6f0       _to_upper_cp1251_general_ci 0051e6f0     strings:ctype-extra.obj
 0003:0003d7f0       _sort_order_cp1251_general_ci 0051e7f0     strings:ctype-extra.obj
 0003:0003d8f0       _to_uni_cp1251_general_ci  0051e8f0     strings:ctype-extra.obj
 0003:0003daf0       _ctype_cp1251_general_cs   0051eaf0     strings:ctype-extra.obj
 0003:0003dbf8       _to_lower_cp1251_general_cs 0051ebf8     strings:ctype-extra.obj
 0003:0003dcf8       _to_upper_cp1251_general_cs 0051ecf8     strings:ctype-extra.obj
 0003:0003ddf8       _sort_order_cp1251_general_cs 0051edf8     strings:ctype-extra.obj
 0003:0003def8       _to_uni_cp1251_general_cs  0051eef8     strings:ctype-extra.obj
 0003:0003e0f8       _ctype_macroman_bin        0051f0f8     strings:ctype-extra.obj
 0003:0003e200       _to_lower_macroman_bin     0051f200     strings:ctype-extra.obj
 0003:0003e300       _to_upper_macroman_bin     0051f300     strings:ctype-extra.obj
 0003:0003e400       _to_uni_macroman_bin       0051f400     strings:ctype-extra.obj
 0003:0003e600       _ctype_cp1256_general_ci   0051f600     strings:ctype-extra.obj
 0003:0003e708       _to_lower_cp1256_general_ci 0051f708     strings:ctype-extra.obj
 0003:0003e808       _to_upper_cp1256_general_ci 0051f808     strings:ctype-extra.obj
 0003:0003e908       _sort_order_cp1256_general_ci 0051f908     strings:ctype-extra.obj
 0003:0003ea08       _to_uni_cp1256_general_ci  0051fa08     strings:ctype-extra.obj
 0003:0003ec08       _ctype_cp1257_bin          0051fc08     strings:ctype-extra.obj
 0003:0003ed10       _to_lower_cp1257_bin       0051fd10     strings:ctype-extra.obj
 0003:0003ee10       _to_upper_cp1257_bin       0051fe10     strings:ctype-extra.obj
 0003:0003ef10       _to_uni_cp1257_bin         0051ff10     strings:ctype-extra.obj
 0003:0003f110       _ctype_cp1257_general_ci   00520110     strings:ctype-extra.obj
 0003:0003f218       _to_lower_cp1257_general_ci 00520218     strings:ctype-extra.obj
 0003:0003f318       _to_upper_cp1257_general_ci 00520318     strings:ctype-extra.obj
 0003:0003f418       _sort_order_cp1257_general_ci 00520418     strings:ctype-extra.obj
 0003:0003f518       _to_uni_cp1257_general_ci  00520518     strings:ctype-extra.obj
 0003:0003f718       _ctype_armscii8_bin        00520718     strings:ctype-extra.obj
 0003:0003f820       _to_lower_armscii8_bin     00520820     strings:ctype-extra.obj
 0003:0003f920       _to_upper_armscii8_bin     00520920     strings:ctype-extra.obj
 0003:0003fa20       _to_uni_armscii8_bin       00520a20     strings:ctype-extra.obj
 0003:0003fc20       _ctype_ascii_bin           00520c20     strings:ctype-extra.obj
 0003:0003fd28       _to_lower_ascii_bin        00520d28     strings:ctype-extra.obj
 0003:0003fe28       _to_upper_ascii_bin        00520e28     strings:ctype-extra.obj
 0003:0003ff28       _to_uni_ascii_bin          00520f28     strings:ctype-extra.obj
 0003:00040128       _ctype_cp1250_bin          00521128     strings:ctype-extra.obj
 0003:00040230       _to_lower_cp1250_bin       00521230     strings:ctype-extra.obj
 0003:00040330       _to_upper_cp1250_bin       00521330     strings:ctype-extra.obj
 0003:00040430       _to_uni_cp1250_bin         00521430     strings:ctype-extra.obj
 0003:00040630       _ctype_cp1256_bin          00521630     strings:ctype-extra.obj
 0003:00040738       _to_lower_cp1256_bin       00521738     strings:ctype-extra.obj
 0003:00040838       _to_upper_cp1256_bin       00521838     strings:ctype-extra.obj
 0003:00040938       _to_uni_cp1256_bin         00521938     strings:ctype-extra.obj
 0003:00040b38       _ctype_cp866_bin           00521b38     strings:ctype-extra.obj
 0003:00040c40       _to_lower_cp866_bin        00521c40     strings:ctype-extra.obj
 0003:00040d40       _to_upper_cp866_bin        00521d40     strings:ctype-extra.obj
 0003:00040e40       _to_uni_cp866_bin          00521e40     strings:ctype-extra.obj
 0003:00041040       _ctype_dec8_bin            00522040     strings:ctype-extra.obj
 0003:00041148       _to_lower_dec8_bin         00522148     strings:ctype-extra.obj
 0003:00041248       _to_upper_dec8_bin         00522248     strings:ctype-extra.obj
 0003:00041348       _to_uni_dec8_bin           00522348     strings:ctype-extra.obj
 0003:00041548       _ctype_greek_bin           00522548     strings:ctype-extra.obj
 0003:00041650       _to_lower_greek_bin        00522650     strings:ctype-extra.obj
 0003:00041750       _to_upper_greek_bin        00522750     strings:ctype-extra.obj
 0003:00041850       _to_uni_greek_bin          00522850     strings:ctype-extra.obj
 0003:00041a50       _ctype_hebrew_bin          00522a50     strings:ctype-extra.obj
 0003:00041b58       _to_lower_hebrew_bin       00522b58     strings:ctype-extra.obj
 0003:00041c58       _to_upper_hebrew_bin       00522c58     strings:ctype-extra.obj
 0003:00041d58       _to_uni_hebrew_bin         00522d58     strings:ctype-extra.obj
 0003:00041f58       _ctype_hp8_bin             00522f58     strings:ctype-extra.obj
 0003:00042060       _to_lower_hp8_bin          00523060     strings:ctype-extra.obj
 0003:00042160       _to_upper_hp8_bin          00523160     strings:ctype-extra.obj
 0003:00042260       _to_uni_hp8_bin            00523260     strings:ctype-extra.obj
 0003:00042460       _ctype_keybcs2_bin         00523460     strings:ctype-extra.obj
 0003:00042568       _to_lower_keybcs2_bin      00523568     strings:ctype-extra.obj
 0003:00042668       _to_upper_keybcs2_bin      00523668     strings:ctype-extra.obj
 0003:00042768       _to_uni_keybcs2_bin        00523768     strings:ctype-extra.obj
 0003:00042968       _ctype_koi8r_bin           00523968     strings:ctype-extra.obj
 0003:00042a70       _to_lower_koi8r_bin        00523a70     strings:ctype-extra.obj
 0003:00042b70       _to_upper_koi8r_bin        00523b70     strings:ctype-extra.obj
 0003:00042c70       _to_uni_koi8r_bin          00523c70     strings:ctype-extra.obj
 0003:00042e70       _ctype_koi8u_bin           00523e70     strings:ctype-extra.obj
 0003:00042f78       _to_lower_koi8u_bin        00523f78     strings:ctype-extra.obj
 0003:00043078       _to_upper_koi8u_bin        00524078     strings:ctype-extra.obj
 0003:00043178       _to_uni_koi8u_bin          00524178     strings:ctype-extra.obj
 0003:00043378       _ctype_latin2_bin          00524378     strings:ctype-extra.obj
 0003:00043480       _to_lower_latin2_bin       00524480     strings:ctype-extra.obj
 0003:00043580       _to_upper_latin2_bin       00524580     strings:ctype-extra.obj
 0003:00043680       _to_uni_latin2_bin         00524680     strings:ctype-extra.obj
 0003:00043880       _ctype_latin5_bin          00524880     strings:ctype-extra.obj
 0003:00043988       _to_lower_latin5_bin       00524988     strings:ctype-extra.obj
 0003:00043a88       _to_upper_latin5_bin       00524a88     strings:ctype-extra.obj
 0003:00043b88       _to_uni_latin5_bin         00524b88     strings:ctype-extra.obj
 0003:00043d88       _ctype_latin7_bin          00524d88     strings:ctype-extra.obj
 0003:00043e90       _to_lower_latin7_bin       00524e90     strings:ctype-extra.obj
 0003:00043f90       _to_upper_latin7_bin       00524f90     strings:ctype-extra.obj
 0003:00044090       _to_uni_latin7_bin         00525090     strings:ctype-extra.obj
 0003:00044290       _ctype_cp850_bin           00525290     strings:ctype-extra.obj
 0003:00044398       _to_lower_cp850_bin        00525398     strings:ctype-extra.obj
 0003:00044498       _to_upper_cp850_bin        00525498     strings:ctype-extra.obj
 0003:00044598       _to_uni_cp850_bin          00525598     strings:ctype-extra.obj
 0003:00044798       _ctype_cp852_bin           00525798     strings:ctype-extra.obj
 0003:000448a0       _to_lower_cp852_bin        005258a0     strings:ctype-extra.obj
 0003:000449a0       _to_upper_cp852_bin        005259a0     strings:ctype-extra.obj
 0003:00044aa0       _to_uni_cp852_bin          00525aa0     strings:ctype-extra.obj
 0003:00044ca0       _ctype_swe7_bin            00525ca0     strings:ctype-extra.obj
 0003:00044da8       _to_lower_swe7_bin         00525da8     strings:ctype-extra.obj
 0003:00044ea8       _to_upper_swe7_bin         00525ea8     strings:ctype-extra.obj
 0003:00044fa8       _to_uni_swe7_bin           00525fa8     strings:ctype-extra.obj
 0003:000451a8       _ctype_geostd8_general_ci  005261a8     strings:ctype-extra.obj
 0003:000452b0       _to_lower_geostd8_general_ci 005262b0     strings:ctype-extra.obj
 0003:000453b0       _to_upper_geostd8_general_ci 005263b0     strings:ctype-extra.obj
 0003:000454b0       _sort_order_geostd8_general_ci 005264b0     strings:ctype-extra.obj
 0003:000455b0       _to_uni_geostd8_general_ci 005265b0     strings:ctype-extra.obj
 0003:000457b0       _ctype_geostd8_bin         005267b0     strings:ctype-extra.obj
 0003:000458b8       _to_lower_geostd8_bin      005268b8     strings:ctype-extra.obj
 0003:000459b8       _to_upper_geostd8_bin      005269b8     strings:ctype-extra.obj
 0003:00045ab8       _to_uni_geostd8_bin        00526ab8     strings:ctype-extra.obj
 0003:00045cb8       _ctype_latin1_spanish_ci   00526cb8     strings:ctype-extra.obj
 0003:00045dc0       _to_lower_latin1_spanish_ci 00526dc0     strings:ctype-extra.obj
 0003:00045ec0       _to_upper_latin1_spanish_ci 00526ec0     strings:ctype-extra.obj
 0003:00045fc0       _sort_order_latin1_spanish_ci 00526fc0     strings:ctype-extra.obj
 0003:000460c0       _to_uni_latin1_spanish_ci  005270c0     strings:ctype-extra.obj
 0003:000462c0       _ctype_cp1250_polish_ci    005272c0     strings:ctype-extra.obj
 0003:000463c8       _to_lower_cp1250_polish_ci 005273c8     strings:ctype-extra.obj
 0003:000464c8       _to_upper_cp1250_polish_ci 005274c8     strings:ctype-extra.obj
 0003:000465c8       _sort_order_cp1250_polish_ci 005275c8     strings:ctype-extra.obj
 0003:000466c8       _to_uni_cp1250_polish_ci   005276c8     strings:ctype-extra.obj
 0003:000468c8       _compiled_charsets         005278c8     strings:ctype-extra.obj
 0003:0004bfc8       _my_uni_ctype              0052cfc8     strings:ctype-utf8.obj
 0003:000509c8       _my_unicase_default        005319c8     strings:ctype-utf8.obj
 0003:000513c8       _my_unicase_turkish        005323c8     strings:ctype-utf8.obj
 0003:00051b00       _my_charset_utf8_handler   00532b00     strings:ctype-utf8.obj
 0003:00051b70       _my_charset_utf8_general_ci 00532b70     strings:ctype-utf8.obj
 0003:00051be0       _my_charset_utf8_bin       00532be0     strings:ctype-utf8.obj
 0003:00055d08       _my_charset_filename       00536d08     strings:ctype-utf8.obj
 0003:00070348       _my_charset_ujis_japanese_ci 00551348     strings:ctype-ujis.obj
 0003:000703b8       _my_charset_ujis_bin       005513b8     strings:ctype-ujis.obj
 0003:000707b0       _my_charset_ucs2_handler   005517b0     strings:ctype-ucs2.obj
 0003:00070820       _my_charset_ucs2_general_ci 00551820     strings:ctype-ucs2.obj
 0003:00070890       _my_charset_ucs2_bin       00551890     strings:ctype-ucs2.obj
 0003:00072aa8       _my_charset_tis620_thai_ci 00553aa8     strings:ctype-tis620.obj
 0003:00072b18       _my_charset_tis620_bin     00553b18     strings:ctype-tis620.obj
 0003:00082c10       _my_charset_sjis_japanese_ci 00563c10     strings:ctype-sjis.obj
 0003:00082c80       _my_charset_sjis_bin       00563c80     strings:ctype-sjis.obj
 0003:000aa498       _my_charset_gbk_chinese_ci 0058b498     strings:ctype-gbk.obj
 0003:000aa508       _my_charset_gbk_bin        0058b508     strings:ctype-gbk.obj
 0003:000bfa00       _my_charset_gb2312_chinese_ci 005a0a00     strings:ctype-gb2312.obj
 0003:000bfa70       _my_charset_gb2312_bin     005a0a70     strings:ctype-gb2312.obj
 0003:000e06c8       _my_charset_euckr_korean_ci 005c16c8     strings:ctype-euc_kr.obj
 0003:000e0738       _my_charset_euckr_bin      005c1738     strings:ctype-euc_kr.obj
 0003:000fb220       _my_charset_eucjpms_japanese_ci 005dc220     strings:ctype-eucjpms.obj
 0003:000fb290       _my_charset_eucjpms_bin    005dc290     strings:ctype-eucjpms.obj
 0003:000fbb28       _my_charset_latin2_czech_ci 005dcb28     strings:ctype-czech.obj
 0003:000fc860       _my_charset_cp1250_czech_ci 005dd860     strings:ctype-win1250ch.obj
 0003:00113110       _my_charset_big5_chinese_ci 005f4110     strings:ctype-big5.obj
 0003:00113180       _my_charset_big5_bin       005f4180     strings:ctype-big5.obj
 0003:001148f0       _my_collation_mb_bin_handler 005f58f0     strings:ctype-mb.obj
 0003:0011491c       _my_str_malloc             005f591c     strings:str_alloc.obj
 0003:00114920       _my_str_free               005f5920     strings:str_alloc.obj
 0003:00114b90       ??_R0?AUMessage@yaSSL@@@8  005f5b90     yassl:ssl.obj
 0003:00114bac       ??_R0?AVvirtual_base@yaSSL@@@8 005f5bac     yassl:ssl.obj
 0003:00114bd0       ??_R0?AVHandShakeBase@yaSSL@@@8 005f5bd0     yassl:ssl.obj
 0003:00114bf4       ??_R0?AVHASH@TaoCrypt@@@8  005f5bf4     yassl:ssl.obj
 0003:00114c10       ??_R0?AVvirtual_base@TaoCrypt@@@8 005f5c10     yassl:ssl.obj
 0003:00114c34       ??_R0?AVMD5@TaoCrypt@@@8   005f5c34     yassl:ssl.obj
 0003:00114c50       ??_R0?AVHASHwithTransform@TaoCrypt@@@8 005f5c50     yassl:ssl.obj
 0003:00114c7c       ??_R0?AVMD4@TaoCrypt@@@8   005f5c7c     yassl:ssl.obj
 0003:001150c8       ??_R0?AUDigest@yaSSL@@@8   005f60c8     yassl:crypto_wrapper.obj
 0003:001150e4       ??_R0?AUBulkCipher@yaSSL@@@8 005f60e4     yassl:crypto_wrapper.obj
 0003:00115104       ??_R0?AUAuth@yaSSL@@@8     005f6104     yassl:crypto_wrapper.obj
 0003:00115120       ??_R0?AVSHA@TaoCrypt@@@8   005f6120     yassl:crypto_wrapper.obj
 0003:0011513c       ??_R0?AVRIPEMD160@TaoCrypt@@@8 005f613c     yassl:crypto_wrapper.obj
 0003:00115160       ??_R0?AVMode_BASE@TaoCrypt@@@8 005f6160     yassl:crypto_wrapper.obj
 0003:00115184       ??_R0?AVDES@TaoCrypt@@@8   005f6184     yassl:crypto_wrapper.obj
 0003:001151a0       ??_R0?AVBasicDES@TaoCrypt@@@8 005f61a0     yassl:crypto_wrapper.obj
 0003:001151c0       ??_R0?AVDES_EDE3@TaoCrypt@@@8 005f61c0     yassl:crypto_wrapper.obj
 0003:001151e0       ??_R0?AVAES@TaoCrypt@@@8   005f61e0     yassl:crypto_wrapper.obj
 0003:001151fc       ??_R0?AVMD5@yaSSL@@@8      005f61fc     yassl:crypto_wrapper.obj
 0003:00115214       ??_R0?AVSHA@yaSSL@@@8      005f6214     yassl:crypto_wrapper.obj
 0003:0011522c       ??_R0?AVRMD@yaSSL@@@8      005f622c     yassl:crypto_wrapper.obj
 0003:00115244       ??_R0?AVRC4@yaSSL@@@8      005f6244     yassl:crypto_wrapper.obj
 0003:0011525c       ??_R0?AVAES@yaSSL@@@8      005f625c     yassl:crypto_wrapper.obj
 0003:00115274       ??_R0?AVHMAC_MD5@yaSSL@@@8 005f6274     yassl:crypto_wrapper.obj
 0003:00115294       ??_R0?AVHMAC_SHA@yaSSL@@@8 005f6294     yassl:crypto_wrapper.obj
 0003:001152b4       ??_R0?AVHMAC_RMD@yaSSL@@@8 005f62b4     yassl:crypto_wrapper.obj
 0003:001152d4       ??_R0?AVDES@yaSSL@@@8      005f62d4     yassl:crypto_wrapper.obj
 0003:001152ec       ??_R0?AVDES_EDE@yaSSL@@@8  005f62ec     yassl:crypto_wrapper.obj
 0003:00115308       ??_R0?AVDSS@yaSSL@@@8      005f6308     yassl:crypto_wrapper.obj
 0003:00115320       ??_R0?AVRSA@yaSSL@@@8      005f6320     yassl:crypto_wrapper.obj
 0003:00115540       ??_R0?AVHandShakeHeader@yaSSL@@@8 005f6540     yassl:yassl_imp.obj
 0003:00115564       ??_R0?AUServerKeyBase@yaSSL@@@8 005f6564     yassl:yassl_imp.obj
 0003:00115588       ??_R0?AUClientKeyBase@yaSSL@@@8 005f6588     yassl:yassl_imp.obj
 0003:001155ac       ??_R0?AVClientDiffieHellmanPublic@yaSSL@@@8 005f65ac     yassl:yassl_imp.obj
 0003:001155dc       ??_R0?AVChangeCipherSpec@yaSSL@@@8 005f65dc     yassl:yassl_imp.obj
 0003:00115604       ??_R0?AVAlert@yaSSL@@@8    005f6604     yassl:yassl_imp.obj
 0003:00115620       ??_R0?AVData@yaSSL@@@8     005f6620     yassl:yassl_imp.obj
 0003:0011563c       ??_R0?AVCertificate@yaSSL@@@8 005f663c     yassl:yassl_imp.obj
 0003:0011565c       ??_R0?AVServerHello@yaSSL@@@8 005f665c     yassl:yassl_imp.obj
 0003:0011567c       ??_R0?AUServerHelloDone@yaSSL@@@8 005f667c     yassl:yassl_imp.obj
 0003:001156a0       ??_R0?AVClientHello@yaSSL@@@8 005f66a0     yassl:yassl_imp.obj
 0003:001156c0       ??_R0?AVServerKeyExchange@yaSSL@@@8 005f66c0     yassl:yassl_imp.obj
 0003:001156e8       ??_R0?AVCertificateVerify@yaSSL@@@8 005f66e8     yassl:yassl_imp.obj
 0003:00115710       ??_R0?AVClientKeyExchange@yaSSL@@@8 005f6710     yassl:yassl_imp.obj
 0003:00115738       ??_R0?AVFinished@yaSSL@@@8 005f6738     yassl:yassl_imp.obj
 0003:00115758       ??_R0?AUHelloRequest@yaSSL@@@8 005f6758     yassl:yassl_imp.obj
 0003:0011577c       ??_R0?AURSA_Server@yaSSL@@@8 005f677c     yassl:yassl_imp.obj
 0003:0011579c       ??_R0?AUFortezza_Server@yaSSL@@@8 005f679c     yassl:yassl_imp.obj
 0003:001157c0       ??_R0?AUFortezzaKeys@yaSSL@@@8 005f67c0     yassl:yassl_imp.obj
 0003:001157e4       ??_R0?AVEncryptedPreMasterSecret@yaSSL@@@8 005f67e4     yassl:yassl_imp.obj
 0003:00115814       ??_R0?AVDH_Server@yaSSL@@@8 005f6814     yassl:yassl_imp.obj
 0003:00115834       ??_R0?AVCertificateRequest@yaSSL@@@8 005f6834     yassl:yassl_imp.obj
 0003:00115eb0       __fltused                  005f6eb0     LIBCMT:fpinit.obj
 0003:00115eb4       __ldused                   005f6eb4     LIBCMT:fpinit.obj
 0003:00115ebc       ??_R0?AVtype_info@@@8      005f6ebc     LIBCMT:typinfo.obj
 0003:00115ee0       ___security_cookie         005f6ee0     LIBCMT:gs_cookie.obj
 0003:00115ee4       ___security_cookie_complement 005f6ee4     LIBCMT:gs_cookie.obj
 0003:00115eec       ??_R0?AVbad_alloc@std@@@8  005f6eec     LIBCMT:new.obj
 0003:00115f08       ??_R0?AVexception@std@@@8  005f6f08     LIBCMT:new.obj
 0003:001160a0       __iob                      005f70a0     LIBCMT:_file.obj
 0003:00116320       __aexit_rtn                005f7320     LIBCMT:crt0dat.obj
 0003:00116334       ___app_type                005f7334     LIBCMT:crt0.obj
 0003:00116360       __cfltcvt_tab              005f7360     LIBCMT:cmiscdat.obj
 0003:00116390       ___abort_behavior          005f7390     LIBCMT:abort.obj
 0003:00116450       ___flsindex                005f7450     LIBCMT:tidtable.obj
 0003:00116454       ___getvalueindex           005f7454     LIBCMT:tidtable.obj
 0003:00116464       ??_R0?AVbad_cast@std@@@8   005f7464     LIBCMT:stdexcpt.obj
 0003:00116480       ??_R0?AVbad_typeid@std@@@8 005f7480     LIBCMT:stdexcpt.obj
 0003:001164a0       ??_R0?AV__non_rtti_object@std@@@8 005f74a0     LIBCMT:stdexcpt.obj
 0003:001164c8       __sys_errlist              005f74c8     LIBCMT:syserr.obj
 0003:00116578       __sys_nerr                 005f7578     LIBCMT:syserr.obj
 0003:0011657c       ___nullstring              005f757c     LIBCMT:output.obj
 0003:00116580       ___wnullstring             005f7580     LIBCMT:output.obj
 0003:00116588       ___badioinfo               005f7588     LIBCMT:ioinit.obj
 0003:001166e8       __XcptActTab               005f76e8     LIBCMT:winxfltr.obj
 0003:00116760       __First_FPE_Indx           005f7760     LIBCMT:winxfltr.obj
 0003:00116764       __Num_FPE                  005f7764     LIBCMT:winxfltr.obj
 0003:00116768       __XcptActTabSize           005f7768     LIBCMT:winxfltr.obj
 0003:0011676c       __XcptActTabCount          005f776c     LIBCMT:winxfltr.obj
 0003:00116778       ___initialmbcinfo          005f7778     LIBCMT:mbctype.obj
 0003:00116998       __mbctype                  005f7998     LIBCMT:mbctype.obj
 0003:00116aa0       __mbcasemap                005f7aa0     LIBCMT:mbctype.obj
 0003:00116ba0       ___ptmbcinfo               005f7ba0     LIBCMT:mbctype.obj
 0003:00116c9c       ___globallocalestatus      005f7c9c     LIBCMT:glstatus.obj
 0003:00116ca0       ___clocalestr              005f7ca0     LIBCMT:nlsdata2.obj
 0003:00116ca8       ___initiallocinfo          005f7ca8     LIBCMT:nlsdata2.obj
 0003:00116d80       ___ptlocinfo               005f7d80     LIBCMT:nlsdata2.obj
 0003:00116d84       ___lc_clike                005f7d84     LIBCMT:nlsdata2.obj
 0003:00116d88       ___initiallocalestructinfo 005f7d88     LIBCMT:nlsdata2.obj
 0003:00116d90       __coninpfh                 005f7d90     LIBCMT:initcon.obj
 0003:00116d94       __confh                    005f7d94     LIBCMT:initcon.obj
 0003:00116d98       __amblksiz                 005f7d98     LIBCMT:heapinit.obj
 0003:00116da0       __timezone                 005f7da0     LIBCMT:timeset.obj
 0003:00116da4       __daylight                 005f7da4     LIBCMT:timeset.obj
 0003:00116da8       __dstbias                  005f7da8     LIBCMT:timeset.obj
 0003:00116e30       __tzname                   005f7e30     LIBCMT:timeset.obj
 0003:00116e40       __lpdays                   005f7e40     LIBCMT:days.obj
 0003:00116e74       __days                     005f7e74     LIBCMT:days.obj
 0003:00116ea8       __lookuptrailbytes         005f7ea8     LIBCMT:read.obj
 0003:00116fa8       __d_inf                    005f7fa8     LIBCMT:util.obj
 0003:00116fb0       __d_ind                    005f7fb0     LIBCMT:util.obj
 0003:00116fb8       __d_max                    005f7fb8     LIBCMT:util.obj
 0003:00116fc0       __d_min                    005f7fc0     LIBCMT:util.obj
 0003:00116fc8       __d_mzero                  005f7fc8     LIBCMT:util.obj
 0003:001170e0       ??_R0?AVDNameNode@@@8      005f80e0     LIBCMT:undname.obj
 0003:001170f8       ??_R0?AVcharNode@@@8       005f80f8     LIBCMT:undname.obj
 0003:00117110       ??_R0?AVpDNameNode@@@8     005f8110     LIBCMT:undname.obj
 0003:0011712c       ??_R0?AVDNameStatusNode@@@8 005f812c     LIBCMT:undname.obj
 0003:0011714c       ??_R0?AVpcharNode@@@8      005f814c     LIBCMT:undname.obj
 0003:00117174       __matherr_flag             005f8174     LIBCMT:matherr.obj
 0003:00117178       __pctype                   005f8178     LIBCMT:ctype.obj
 0003:0011717c       __pwctype                  005f817c     LIBCMT:ctype.obj
 0003:00117180       ___lc_time_c               005f8180     LIBCMT:strftime.obj
 0003:00117238       ___lc_time_curr            005f8238     LIBCMT:strftime.obj
 0003:0011723c       ___lconv_static_decimal    005f823c     LIBCMT:lconv.obj
 0003:00117240       ___lconv_c                 005f8240     LIBCMT:lconv.obj
 0003:00117270       ___lconv                   005f8270     LIBCMT:lconv.obj
 0003:00117274       ___mb_cur_max              005f8274     LIBCMT:nlsdata1.obj
 0003:00117278       ___decimal_point           005f8278     LIBCMT:nlsdata1.obj
 0003:0011727c       ___decimal_point_length    005f827c     LIBCMT:nlsdata1.obj
 0003:00117280       __NLG_Destination          005f8280     LIBCMT:exsup.obj
 0003:001172c0       __pow10pos                 005f82c0     LIBCMT:constpow.obj
 0003:00117420       __pow10neg                 005f8420     LIBCMT:constpow.obj
 0003:00117580       ??_R0?AVHASH64withTransform@TaoCrypt@@@8 005f8580     taocrypt:hash.obj
 0003:001175b0       ??_R0?AVMultiplicativeGroupT@AbstractRing@TaoCrypt@@@8 005f85b0     taocrypt:integer.obj
 0003:001175ec       ??_R0?AVAbstractGroup@TaoCrypt@@@8 005f85ec     taocrypt:integer.obj
 0003:00117614       ??_R0?AVModularArithmetic@TaoCrypt@@@8 005f8614     taocrypt:integer.obj
 0003:00117640       ??_R0?AVAbstractRing@TaoCrypt@@@8 005f8640     taocrypt:integer.obj
 0003:00117664       ??_R0?AVMontgomeryRepresentation@TaoCrypt@@@8 005f8664     taocrypt:integer.obj
 0003:00117694       ??_R0?AVEuclideanDomainOf@TaoCrypt@@@8 005f8694     taocrypt:integer.obj
 0003:001176c0       ??_R0?AVAbstractEuclideanDomain@TaoCrypt@@@8 005f86c0     taocrypt:integer.obj
 0003:001176f0       ??_R0?AVSHA256@TaoCrypt@@@8 005f86f0     taocrypt:sha.obj
 0003:00117710       ??_R0?AVSHA224@TaoCrypt@@@8 005f8710     taocrypt:sha.obj
 0003:00117730       ??_R0?AVSHA512@TaoCrypt@@@8 005f8730     taocrypt:sha.obj
 0003:00117750       ??_R0?AVSHA384@TaoCrypt@@@8 005f8750     taocrypt:sha.obj
 0003:00117770       ?Te0@AES@TaoCrypt@@0PBIB   005f8770     taocrypt:aes.obj
 0003:00117774       ?Te1@AES@TaoCrypt@@0PBIB   005f8774     taocrypt:aes.obj
 0003:00117778       ?Te2@AES@TaoCrypt@@0PBIB   005f8778     taocrypt:aes.obj
 0003:0011777c       ?Te3@AES@TaoCrypt@@0PBIB   005f877c     taocrypt:aes.obj
 0003:00117780       ?Te4@AES@TaoCrypt@@0PBIB   005f8780     taocrypt:aes.obj
 0003:00117784       ?Td0@AES@TaoCrypt@@0PBIB   005f8784     taocrypt:aes.obj
 0003:00117788       ?Td1@AES@TaoCrypt@@0PBIB   005f8788     taocrypt:aes.obj
 0003:0011778c       ?Td2@AES@TaoCrypt@@0PBIB   005f878c     taocrypt:aes.obj
 0003:00117790       ?Td3@AES@TaoCrypt@@0PBIB   005f8790     taocrypt:aes.obj
 0003:00117794       ?Td4@AES@TaoCrypt@@0PBIB   005f8794     taocrypt:aes.obj
 0003:0011779c       ??_R0?AVBER_Decoder@TaoCrypt@@@8 005f879c     taocrypt:dsa.obj
 0003:001177c0       ??_R0?AVDSA_Private_Decoder@TaoCrypt@@@8 005f87c0     taocrypt:dsa.obj
 0003:001177ec       ??_R0?AVDSA_Public_Decoder@TaoCrypt@@@8 005f87ec     taocrypt:dsa.obj
 0003:0011781c       ??_R0?AVDH_Decoder@TaoCrypt@@@8 005f881c     taocrypt:dh.obj
 0003:00117844       ??_R0?AVRSA_Private_Decoder@TaoCrypt@@@8 005f8844     taocrypt:rsa.obj
 0003:00117870       ??_R0?AVRSA_Public_Decoder@TaoCrypt@@@8 005f8870     taocrypt:rsa.obj
 0003:001178a0       ??_R0?AVPKCS12_Decoder@TaoCrypt@@@8 005f88a0     taocrypt:asn.obj
 0003:001178c8       ??_R0?AVDER_Encoder@TaoCrypt@@@8 005f88c8     taocrypt:asn.obj
 0003:001178ec       ??_R0?AVCertDecoder@TaoCrypt@@@8 005f88ec     taocrypt:asn.obj
 0003:00117910       ??_R0?AVSignature_Encoder@TaoCrypt@@@8 005f8910     taocrypt:asn.obj
 0003:00117940       ??_R0?AVMD2@TaoCrypt@@@8   005f8940     taocrypt:md2.obj
 0003:00117960       __half                     005f8960     LIBCMT:pow.obj
 0003:001179e0       __infinity                 005f89e0     LIBCMT:87tran.obj
 0003:001179ea       __minfinity                005f89ea     LIBCMT:87tran.obj
 0003:001179f4       __logemax                  005f89f4     LIBCMT:87tran.obj
 0003:00117a1a       __OP_EXPjmptab             005f8a1a     LIBCMT:87tran.obj
 0003:00117a40       __indefinite               005f8a40     LIBCMT:87disp.obj
 0003:00117a4a       __piby2                    005f8a4a     LIBCMT:87disp.obj
 0003:0014f6e0       ?p_user_map@Manager@@0PAVUser_map@@A 006306e0     manager.obj
 0003:0014f6e4       ?p_guardian@Manager@@0PAVGuardian@@A 006306e4     manager.obj
 0003:0014f6e8       ?have_signal@@3_NA         006306e8     manager.obj
 0003:0014f6ec       ?p_instance_map@Manager@@0PAVInstance_map@@A 006306ec     manager.obj
 0003:0014f6f0       ?p_thread_registry@Manager@@0PAVThread_registry@@A 006306f0     manager.obj
 0003:0014f6f8       ?remove_service@Service@Options@@2DA 006306f8     options.obj
 0003:0014f6f9       ?install_as_service@Service@Options@@2DA 006306f9     options.obj
 0003:0014f6fa       ?stand_alone@Service@Options@@2DA 006306fa     options.obj
 0003:0014ff00       ?is_forced_default_file@Main@Options@@2_NA 00630f00     options.obj
 0003:0014ff01       ?mysqld_safe_compatible@Main@Options@@2DA 00630f01     options.obj
 0003:0014ff04       ?bind_address@Main@Options@@2PBDB 00630f04     options.obj
 0003:0014ff08       ?default_directories@Options@@2PAPBDA 00630f08     options.obj
 0003:0014ff0c       ?user_name@User_management@Options@@2PADA 00630f0c     options.obj
 0003:0014ff10       ?password@User_management@Options@@2PADA 00630f10     options.obj
 0003:0014ff14       ?cmd@User_management@Options@@2PAVUser_management_cmd@@A 00630f14     options.obj
 0003:0014ff18       ?saved_argv@Options@@0PAPADA 00630f18     options.obj
 0003:001500bc       ?open_files_limit@@3KA     006310bc     priv.obj
 0003:001500c0       ?test_flags@@3IA           006310c0     priv.obj
 0003:001500c4       ?bytes_sent@@3KA           006310c4     priv.obj
 0003:001500c8       ?bytes_received@@3KA       006310c8     priv.obj
 0003:0015080c       _mysql_port                0063180c     client.obj
 0003:00150810       _mysql_unix_port           00631810     client.obj
 0003:00150818       _charsets_dir              00631818     mysys:charset.obj
 0003:00150820       _all_charsets              00631820     mysys:charset.obj
 0003:00150c28       _my_defaults_file          00631c28     mysys:default.obj
 0003:00150c2c       _my_defaults_group_suffix  00631c2c     mysys:default.obj
 0003:00150c30       _my_defaults_extra_file    00631c30     mysys:default.obj
 0003:00150c38       _THR_thread_count          00631c38     mysys:my_thr_init.obj
 0003:00150c40       _timed_mutexes             00631c40     mysys:my_static.obj
 0003:00150c41       _my_disable_locking        00631c41     mysys:my_static.obj
 0003:00150c42       _my_disable_async_io       00631c42     mysys:my_static.obj
 0003:00150c43       _my_disable_flush_key_blocks 00631c43     mysys:my_static.obj
 0003:00150c44       _home_dir                  00631c44     mysys:my_static.obj
 0003:00150c48       _my_progname               00631c48     mysys:my_static.obj
 0003:00150c4c       _my_stream_opened          00631c4c     mysys:my_static.obj
 0003:00150c50       _curr_dir                  00631c50     mysys:my_static.obj
 0003:00150e50       _home_dir_buff             00631e50     mysys:my_static.obj
 0003:00151050       _my_file_opened            00632050     mysys:my_static.obj
 0003:00151054       _my_tmp_file_created       00632054     mysys:my_static.obj
 0003:00151058       _my_file_total_opened      00632058     mysys:my_static.obj
 0003:0015105c       _my_dont_interrupt         0063205c     mysys:my_static.obj
 0003:00151060       _my_file_info_default      00632060     mysys:my_static.obj
 0003:00151860       __my_signals               00632860     mysys:my_static.obj
 0003:00151864       _my_once_root_block        00632864     mysys:my_static.obj
 0003:00151868       __my_sig_remember          00632868     mysys:my_static.obj
 0003:001518b8       _sf_malloc_prehunc         006328b8     mysys:my_static.obj
 0003:001518bc       _sf_malloc_endhunc         006328bc     mysys:my_static.obj
 0003:001518c0       _sf_malloc_quick           006328c0     mysys:my_static.obj
 0003:001518c4       _sf_malloc_cur_memory      006328c4     mysys:my_static.obj
 0003:001518c8       _sf_malloc_max_memory      006328c8     mysys:my_static.obj
 0003:001518cc       _sf_malloc_count           006328cc     mysys:my_static.obj
 0003:001518d0       _sf_max_adress             006328d0     mysys:my_static.obj
 0003:001518d4       _sf_malloc_root            006328d4     mysys:my_static.obj
 0003:001518d8       _my_have_got_alarm         006328d8     mysys:my_static.obj
 0003:001518dc       _my_disable_symlinks       006328dc     mysys:my_static.obj
 0003:001518dd       _mysys_uses_curses         006328dd     mysys:my_static.obj
 0003:001518e0       _have_tcpip                006328e0     mysys:my_init.obj
 0003:001518e1       _my_init_done              006328e1     mysys:my_init.obj
 0003:001518e4       _mysys_usage_id            006328e4     mysys:my_init.obj
 0003:001518ec       _my_getopt_skip_unknown    006328ec     mysys:my_getopt.obj
 0003:001518f0       _thd_lib_detected          006328f0     mysys:my_pthread.obj
 0003:0015190c       _thr_alarm_inited          0063290c     mysys:thr_alarm.obj
 0003:0015190d       _alarm_thread_running      0063290d     mysys:thr_alarm.obj
 0003:0015190e       _my_use_symdir             0063290e     mysys:mf_pack.obj
 0003:00151934       ___fastflag                00632934     LIBCMT:fpinit.obj
 0003:00151938       __adjust_fdiv              00632938     LIBCMT:fpinit.obj
 0003:00151950       __cflush                   00632950     LIBCMT:_file.obj
 0003:00151954       __umaskval                 00632954     LIBCMT:crt0dat.obj
 0003:00151958       __osplatform               00632958     LIBCMT:crt0dat.obj
 0003:0015195c       __osver                    0063295c     LIBCMT:crt0dat.obj
 0003:00151960       __winver                   00632960     LIBCMT:crt0dat.obj
 0003:00151964       __winmajor                 00632964     LIBCMT:crt0dat.obj
 0003:00151968       __winminor                 00632968     LIBCMT:crt0dat.obj
 0003:0015196c       ___argc                    0063296c     LIBCMT:crt0dat.obj
 0003:00151970       ___argv                    00632970     LIBCMT:crt0dat.obj
 0003:00151974       ___wargv                   00632974     LIBCMT:crt0dat.obj
 0003:00151978       __environ                  00632978     LIBCMT:crt0dat.obj
 0003:0015197c       ___initenv                 0063297c     LIBCMT:crt0dat.obj
 0003:00151980       __wenviron                 00632980     LIBCMT:crt0dat.obj
 0003:00151984       ___winitenv                00632984     LIBCMT:crt0dat.obj
 0003:00151988       __pgmptr                   00632988     LIBCMT:crt0dat.obj
 0003:0015198c       __wpgmptr                  0063298c     LIBCMT:crt0dat.obj
 0003:00151990       __exitflag                 00632990     LIBCMT:crt0dat.obj
 0003:00151994       __C_Termination_Done       00632994     LIBCMT:crt0dat.obj
 0003:00151998       __C_Exit_Done              00632998     LIBCMT:crt0dat.obj
 0003:001519b0       __aenvptr                  006329b0     LIBCMT:crt0.obj
 0003:001519b4       __wenvptr                  006329b4     LIBCMT:crt0.obj
 0003:001519b8       ___error_mode              006329b8     LIBCMT:crt0.obj
 0003:001519bc       __tls_index                006329bc     LIBCMT:tlssup.obj
 0003:00151a78       ___pInvalidArgHandler      00632a78     LIBCMT:invarg.obj
 0003:00151d9c       _gpFlsAlloc                00632d9c     LIBCMT:tidtable.obj
 0003:00151da0       _gpFlsGetValue             00632da0     LIBCMT:tidtable.obj
 0003:00151da4       _gpFlsSetValue             00632da4     LIBCMT:tidtable.obj
 0003:00151da8       _gpFlsFree                 00632da8     LIBCMT:tidtable.obj
 0003:00151db4       ___pPurecall               00632db4     LIBCMT:inithelp.obj
 0003:001520dc       ?_pnhHeap@@3P6AHI@ZA       006330dc     LIBCMT:handler.obj
 0003:001520e0       __maxwait                  006330e0     LIBCMT:crtheap.obj
 0003:001520e4       __stdbuf                   006330e4     LIBCMT:_sftbuf.obj
 0003:00152240       ?__pInconsistency@@3P6AXXZA 00633240     LIBCMT:hooks.obj
 0003:00152254       ___mbulinfo                00633254     LIBCMT:mbctype.obj
 0003:00152260       ___mbcodepage              00633260     LIBCMT:mbctype.obj
 0003:00152264       ___ismbcodepage            00633264     LIBCMT:mbctype.obj
 0003:00152268       ___mblcid                  00633268     LIBCMT:mbctype.obj
 0003:0015226c       ___locale_changed          0063326c     LIBCMT:setlocal.obj
 0003:00152270       ___lc_handle               00633270     LIBCMT:nlsdata2.obj
 0003:00152288       ___lc_codepage             00633288     LIBCMT:nlsdata2.obj
 0003:0015228c       ___lc_collate_cp           0063328c     LIBCMT:nlsdata2.obj
 0003:0015239c       __crtheap                  0063339c     LIBCMT:heapinit.obj
 0003:001523a0       __newmode                  006333a0     LIBCMT:_newmode.obj
 0003:001523a4       ___sbh_pHeaderDefer        006333a4     LIBCMT:sbheap.obj
 0003:001523a8       __outputformat             006333a8     LIBCMT:outputformat.obj
 0003:001523c0       ?pArgList@UnDecorator@@0PAVReplicator@@A 006333c0     LIBCMT:undname.obj
 0003:001523c4       ?pZNameList@UnDecorator@@0PAVReplicator@@A 006333c4     LIBCMT:undname.obj
 0003:001523c8       ?pTemplateArgList@UnDecorator@@0PAVReplicator@@A 006333c8     LIBCMT:undname.obj
 0003:001523cc       ?gName@UnDecorator@@0PBDB  006333cc     LIBCMT:undname.obj
 0003:001523d0       ?name@UnDecorator@@0PBDB   006333d0     LIBCMT:undname.obj
 0003:001523d4       ?outputString@UnDecorator@@0PADA 006333d4     LIBCMT:undname.obj
 0003:001523d8       ?maxStringLength@UnDecorator@@0HA 006333d8     LIBCMT:undname.obj
 0003:001523dc       ?disableFlags@UnDecorator@@0KA 006333dc     LIBCMT:undname.obj
 0003:001523e0       ?m_pGetParameter@UnDecorator@@0P6APADJ@ZA 006333e0     LIBCMT:undname.obj
 0003:001523e4       ?fExplicitTemplateParams@UnDecorator@@0_NA 006333e4     LIBCMT:undname.obj
 0003:001523e5       ?fGetTemplateArgumentList@UnDecorator@@0_NA 006333e5     LIBCMT:undname.obj
 0003:00152410       ___lconv_static_null       00633410     LIBCMT:lconv.obj
 0003:00152414       __commode                  00633414     LIBCMT:ncommode.obj
 0003:0015241c       __fmode                    0063341c     LIBCMT:txtmode.obj
 0003:0015243d       ?isMMX@TaoCrypt@@3_NA      0063343d     taocrypt:misc.obj
 0003:00152460       _mysql_server_last_error   00633460     <common>
 0003:001526d0       _mysql_server_last_errno   006336d0     <common>
 0003:001526d4       _thr_client_alarm          006336d4     <common>
 0003:001526e0       _query_performance_frequency 006336e0     <common>
 0003:001526f4       _my_signals                006336f4     <common>
 0003:001526f8       _query_performance_offset  006336f8     <common>
 0003:00152700       _THR_LOCK_threads          00633700     <common>
 0003:00152780       _LOCK_gethostbyname_r      00633780     <common>
 0003:001527a0       _THR_LOCK_myisam_mmap      006337a0     <common>
 0003:001527c0       _THR_LOCK_time             006337c0     <common>
 0003:001527e0       _THR_COND_threads          006337e0     <common>
 0003:00152820       _THR_LOCK_malloc           00633820     <common>
 0003:00152840       _THR_LOCK_isam             00633840     <common>
 0003:00152860       _THR_LOCK_myisam           00633860     <common>
 0003:00152880       _THR_LOCK_heap             00633880     <common>
 0003:001528a0       _THR_LOCK_open             006338a0     <common>
 0003:001528c0       _THR_LOCK_charset          006338c0     <common>
 0003:001528e0       _THR_LOCK_lock             006338e0     <common>
 0003:00152900       _LOCK_localtime_r          00633900     <common>
 0003:00152920       _THR_LOCK_net              00633920     <common>
 0003:00152938       __debugger_hook_dummy      00633938     <common>
 0003:00152944       ___sbh_initialized         00633944     <common>
 0003:00152958       ___sbh_cntHeaderList       00633958     <common>
 0003:0015295c       ___sbh_pHeaderList         0063395c     <common>
 0003:00152960       ___sbh_threshold           00633960     <common>
 0003:00152964       ___sbh_pHeaderScan         00633964     <common>
 0003:00152968       ___sbh_sizeHeaderList      00633968     <common>
 0003:0015296c       ___sbh_indGroupDefer       0063396c     <common>
 0003:00152970       ___active_heap             00633970     <common>
 0003:0015297c       ___setlc_active            0063397c     <common>
 0003:0015298c       ___unguarded_readlc_active 0063398c     <common>
 0003:00152990       __pmatherr                 00633990     <common>
 0003:0015299c       __pDestructExceptionObject 0063399c     <common>
 0003:001529a8       __nhandle                  006339a8     <common>
 0003:00152a00       ___pioinfo                 00633a00     <common>
 0003:00152b00       ___use_sse2_mathfcns       00633b00     <common>
 0003:00152b10       ___sse2_available          00633b10     <common>
 0003:00152b14       __acmdln                   00633b14     <common>
 0003:00152b20       ___env_initialized         00633b20     <common>
 0003:00152b30       ___onexitend               00633b30     <common>
 0003:00152b34       ___onexitbegin             00633b34     <common>
 0003:00152b38       ___mbctype_initialized     00633b38     <common>
 0003:00152b3c       ___dyn_tls_init_callback   00633b3c     <common>
 0003:00152b40       ___piob                    00633b40     <common>
 0003:00152e80       __bufin                    00633e80     <common>
 0003:00153e80       __nstream                  00634e80     <common>
 0004:00000000       __IMPORT_DESCRIPTOR_KERNEL32 00635000     kernel32:KERNEL32.dll
 0004:00000014       __IMPORT_DESCRIPTOR_ADVAPI32 00635014     advapi32:ADVAPI32.dll
 0004:00000028       __IMPORT_DESCRIPTOR_WSOCK32 00635028     wsock32:WSOCK32.dll
 0004:0000003c       __IMPORT_DESCRIPTOR_USER32 0063503c     user32:USER32.dll
 0004:00000050       __NULL_IMPORT_DESCRIPTOR   00635050     kernel32:KERNEL32.dll
 0004:00000468       __imp__CryptGenRandom@12   00635468     advapi32:ADVAPI32.dll
 0004:0000046c       __imp__RegEnumValueA@32    0063546c     advapi32:ADVAPI32.dll
 0004:00000470       __imp__RegOpenKeyExA@20    00635470     advapi32:ADVAPI32.dll
 0004:00000474       __imp__CryptAcquireContextA@20 00635474     advapi32:ADVAPI32.dll
 0004:00000478       __imp__CryptReleaseContext@8 00635478     advapi32:ADVAPI32.dll
 0004:0000047c       __imp__StartServiceCtrlDispatcherA@4 0063547c     advapi32:ADVAPI32.dll
 0004:00000480       __imp__RegisterServiceCtrlHandlerA@8 00635480     advapi32:ADVAPI32.dll
 0004:00000484       __imp__DeleteService@4     00635484     advapi32:ADVAPI32.dll
 0004:00000488       __imp__CreateServiceA@52   00635488     advapi32:ADVAPI32.dll
 0004:0000048c       __imp__SetServiceStatus@8  0063548c     advapi32:ADVAPI32.dll
 0004:00000490       __imp__OpenSCManagerA@12   00635490     advapi32:ADVAPI32.dll
 0004:00000494       __imp__OpenServiceA@12     00635494     advapi32:ADVAPI32.dll
 0004:00000498       __imp__CloseServiceHandle@4 00635498     advapi32:ADVAPI32.dll
 0004:0000049c       __imp__RegCloseKey@4       0063549c     advapi32:ADVAPI32.dll
 0004:000004a0       \177ADVAPI32_NULL_THUNK_DATA 006354a0     advapi32:ADVAPI32.dll
 0004:000004d4       __imp__GetModuleHandleA@4  006354d4     kernel32:KERNEL32.dll
 0004:000004d8       __imp__TerminateProcess@8  006354d8     kernel32:KERNEL32.dll
 0004:000004dc       __imp__OpenProcess@12      006354dc     kernel32:KERNEL32.dll
 0004:000004e0       __imp__GetCurrentThreadId@0 006354e0     kernel32:KERNEL32.dll
 0004:000004e4       __imp__Sleep@4             006354e4     kernel32:KERNEL32.dll
 0004:000004e8       __imp__GetFullPathNameA@16 006354e8     kernel32:KERNEL32.dll
 0004:000004ec       __imp__GetModuleFileNameA@12 006354ec     kernel32:KERNEL32.dll
 0004:000004f0       __imp__SetHandleInformation@12 006354f0     kernel32:KERNEL32.dll
 0004:000004f4       __imp__GetCurrentProcess@0 006354f4     kernel32:KERNEL32.dll
 0004:000004f8       __imp__ReadFile@20         006354f8     kernel32:KERNEL32.dll
 0004:000004fc       __imp__SetNamedPipeHandleState@16 006354fc     kernel32:KERNEL32.dll
 0004:00000500       __imp__WaitNamedPipeA@8    00635500     kernel32:KERNEL32.dll
 0004:00000504       __imp__CreateFileA@28      00635504     kernel32:KERNEL32.dll
 0004:00000508       __imp__DuplicateHandle@28  00635508     kernel32:KERNEL32.dll
 0004:0000050c       __imp__GetProcAddress@8    0063550c     kernel32:KERNEL32.dll
 0004:00000510       __imp__CreateRemoteThread@28 00635510     kernel32:KERNEL32.dll
 0004:00000514       __imp__GetLastError@0      00635514     kernel32:KERNEL32.dll
 0004:00000518       __imp__SetLastError@4      00635518     kernel32:KERNEL32.dll
 0004:0000051c       __imp__CreateProcessA@40   0063551c     kernel32:KERNEL32.dll
 0004:00000520       __imp__WaitForSingleObject@8 00635520     kernel32:KERNEL32.dll
 0004:00000524       __imp__GetExitCodeProcess@8 00635524     kernel32:KERNEL32.dll
 0004:00000528       __imp__CloseHandle@4       00635528     kernel32:KERNEL32.dll
 0004:0000052c       __imp__GetSystemTimeAsFileTime@4 0063552c     kernel32:KERNEL32.dll
 0004:00000530       __imp__DeleteCriticalSection@4 00635530     kernel32:KERNEL32.dll
 0004:00000534       __imp__LoadLibraryW@4      00635534     kernel32:KERNEL32.dll
 0004:00000538       __imp__SetEnvironmentVariableW@8 00635538     kernel32:KERNEL32.dll
 0004:0000053c       __imp__GetModuleFileNameW@12 0063553c     kernel32:KERNEL32.dll
 0004:00000540       __imp__LeaveCriticalSection@4 00635540     kernel32:KERNEL32.dll
 0004:00000544       __imp__EnterCriticalSection@4 00635544     kernel32:KERNEL32.dll
 0004:00000548       __imp__CreatePipe@16       00635548     kernel32:KERNEL32.dll
 0004:0000054c       __imp__IsValidLocale@8     0063554c     kernel32:KERNEL32.dll
 0004:00000550       __imp__EnumSystemLocalesA@8 00635550     kernel32:KERNEL32.dll
 0004:00000554       __imp__GetUserDefaultLCID@0 00635554     kernel32:KERNEL32.dll
 0004:00000558       __imp__GetDateFormatA@24   00635558     kernel32:KERNEL32.dll
 0004:0000055c       __imp__GetTimeFormatA@24   0063555c     kernel32:KERNEL32.dll
 0004:00000560       __imp__GetStringTypeW@16   00635560     kernel32:KERNEL32.dll
 0004:00000564       __imp__GetStringTypeA@20   00635564     kernel32:KERNEL32.dll
 0004:00000568       __imp__SetEnvironmentVariableA@8 00635568     kernel32:KERNEL32.dll
 0004:0000056c       __imp__CompareStringW@24   0063556c     kernel32:KERNEL32.dll
 0004:00000570       __imp__CompareStringA@24   00635570     kernel32:KERNEL32.dll
 0004:00000574       __imp__WriteConsoleW@20    00635574     kernel32:KERNEL32.dll
 0004:00000578       __imp__GetConsoleOutputCP@0 00635578     kernel32:KERNEL32.dll
 0004:0000057c       __imp__WriteConsoleA@20    0063557c     kernel32:KERNEL32.dll
 0004:00000580       __imp__LCMapStringW@24     00635580     kernel32:KERNEL32.dll
 0004:00000584       __imp__LCMapStringA@24     00635584     kernel32:KERNEL32.dll
 0004:00000588       __imp__GetLocaleInfoW@16   00635588     kernel32:KERNEL32.dll
 0004:0000058c       __imp__MultiByteToWideChar@24 0063558c     kernel32:KERNEL32.dll
 0004:00000590       __imp__GetLocaleInfoA@16   00635590     kernel32:KERNEL32.dll
 0004:00000594       __imp__CreateEventA@16     00635594     kernel32:KERNEL32.dll
 0004:00000598       __imp__SetEvent@4          00635598     kernel32:KERNEL32.dll
 0004:0000059c       __imp__ResetEvent@4        0063559c     kernel32:KERNEL32.dll
 0004:000005a0       __imp__WaitForMultipleObjects@16 006355a0     kernel32:KERNEL32.dll
 0004:000005a4       __imp__GetFileAttributesExA@12 006355a4     kernel32:KERNEL32.dll
 0004:000005a8       __imp__GetSystemDirectoryA@8 006355a8     kernel32:KERNEL32.dll
 0004:000005ac       __imp__GetWindowsDirectoryA@8 006355ac     kernel32:KERNEL32.dll
 0004:000005b0       __imp__InterlockedIncrement@4 006355b0     kernel32:KERNEL32.dll
 0004:000005b4       __imp__DeleteFileA@4       006355b4     kernel32:KERNEL32.dll
 0004:000005b8       __imp__MoveFileA@8         006355b8     kernel32:KERNEL32.dll
 0004:000005bc       __imp__GetTickCount@0      006355bc     kernel32:KERNEL32.dll
 0004:000005c0       __imp__QueryPerformanceCounter@4 006355c0     kernel32:KERNEL32.dll
 0004:000005c4       __imp__QueryPerformanceFrequency@4 006355c4     kernel32:KERNEL32.dll
 0004:000005c8       __imp__TryEnterCriticalSection@4 006355c8     kernel32:KERNEL32.dll
 0004:000005cc       __imp__InterlockedCompareExchange@12 006355cc     kernel32:KERNEL32.dll
 0004:000005d0       __imp__SetThreadPriority@8 006355d0     kernel32:KERNEL32.dll
 0004:000005d4       __imp__SetEndOfFile@4      006355d4     kernel32:KERNEL32.dll
 0004:000005d8       __imp__SetFilePointer@16   006355d8     kernel32:KERNEL32.dll
 0004:000005dc       __imp__GetFileAttributesA@4 006355dc     kernel32:KERNEL32.dll
 0004:000005e0       __imp__GetOverlappedResult@16 006355e0     kernel32:KERNEL32.dll
 0004:000005e4       __imp__CancelIo@4          006355e4     kernel32:KERNEL32.dll
 0004:000005e8       __imp__WriteFile@20        006355e8     kernel32:KERNEL32.dll
 0004:000005ec       __imp__DisconnectNamedPipe@4 006355ec     kernel32:KERNEL32.dll
 0004:000005f0       __imp__UnmapViewOfFile@4   006355f0     kernel32:KERNEL32.dll
 0004:000005f4       __imp__FindClose@4         006355f4     kernel32:KERNEL32.dll
 0004:000005f8       __imp__FindNextFileA@8     006355f8     kernel32:KERNEL32.dll
 0004:000005fc       __imp__FindFirstFileA@8    006355fc     kernel32:KERNEL32.dll
 0004:00000600       __imp__FileTimeToSystemTime@8 00635600     kernel32:KERNEL32.dll
 0004:00000604       __imp__FileTimeToLocalFileTime@8 00635604     kernel32:KERNEL32.dll
 0004:00000608       __imp__GetDriveTypeA@4     00635608     kernel32:KERNEL32.dll
 0004:0000060c       __imp__ExitProcess@4       0063560c     kernel32:KERNEL32.dll
 0004:00000610       __imp__SetConsoleCtrlHandler@8 00635610     kernel32:KERNEL32.dll
 0004:00000614       __imp__ReadConsoleInputA@16 00635614     kernel32:KERNEL32.dll
 0004:00000618       __imp__SetConsoleMode@8    00635618     kernel32:KERNEL32.dll
 0004:0000061c       __imp__GetConsoleMode@8    0063561c     kernel32:KERNEL32.dll
 0004:00000620       __imp__PeekConsoleInputA@16 00635620     kernel32:KERNEL32.dll
 0004:00000624       __imp__GetNumberOfConsoleInputEvents@8 00635624     kernel32:KERNEL32.dll
 0004:00000628       __imp__GetCommandLineA@0   00635628     kernel32:KERNEL32.dll
 0004:0000062c       __imp__HeapFree@12         0063562c     kernel32:KERNEL32.dll
 0004:00000630       __imp__GetVersionExA@4     00635630     kernel32:KERNEL32.dll
 0004:00000634       __imp__HeapAlloc@12        00635634     kernel32:KERNEL32.dll
 0004:00000638       __imp__GetProcessHeap@0    00635638     kernel32:KERNEL32.dll
 0004:0000063c       __imp__HeapReAlloc@16      0063563c     kernel32:KERNEL32.dll
 0004:00000640       __imp__GetFileInformationByHandle@8 00635640     kernel32:KERNEL32.dll
 0004:00000644       __imp__PeekNamedPipe@24    00635644     kernel32:KERNEL32.dll
 0004:00000648       __imp__GetFileType@4       00635648     kernel32:KERNEL32.dll
 0004:0000064c       __imp__SetStdHandle@8      0063564c     kernel32:KERNEL32.dll
 0004:00000650       __imp__WideCharToMultiByte@32 00635650     kernel32:KERNEL32.dll
 0004:00000654       __imp__GetTimeZoneInformation@4 00635654     kernel32:KERNEL32.dll
 0004:00000658       __imp__UnhandledExceptionFilter@4 00635658     kernel32:KERNEL32.dll
 0004:0000065c       __imp__SetUnhandledExceptionFilter@4 0063565c     kernel32:KERNEL32.dll
 0004:00000660       __imp__IsDebuggerPresent@0 00635660     kernel32:KERNEL32.dll
 0004:00000664       __imp__ExitThread@4        00635664     kernel32:KERNEL32.dll
 0004:00000668       __imp__ResumeThread@4      00635668     kernel32:KERNEL32.dll
 0004:0000066c       __imp__CreateThread@24     0063566c     kernel32:KERNEL32.dll
 0004:00000670       __imp__FlushFileBuffers@4  00635670     kernel32:KERNEL32.dll
 0004:00000674       __imp__GetStdHandle@4      00635674     kernel32:KERNEL32.dll
 0004:00000678       __imp__TlsGetValue@4       00635678     kernel32:KERNEL32.dll
 0004:0000067c       __imp__TlsAlloc@0          0063567c     kernel32:KERNEL32.dll
 0004:00000680       __imp__TlsSetValue@8       00635680     kernel32:KERNEL32.dll
 0004:00000684       __imp__TlsFree@4           00635684     kernel32:KERNEL32.dll
 0004:00000688       __imp__InterlockedDecrement@4 00635688     kernel32:KERNEL32.dll
 0004:0000068c       __imp__GetCurrentThread@0  0063568c     kernel32:KERNEL32.dll
 0004:00000690       __imp__GetCurrentDirectoryA@8 00635690     kernel32:KERNEL32.dll
 0004:00000694       __imp__SetCurrentDirectoryA@4 00635694     kernel32:KERNEL32.dll
 0004:00000698       __imp__RaiseException@16   00635698     kernel32:KERNEL32.dll
 0004:0000069c       __imp__SetHandleCount@4    0063569c     kernel32:KERNEL32.dll
 0004:000006a0       __imp__GetStartupInfoA@4   006356a0     kernel32:KERNEL32.dll
 0004:000006a4       __imp__FatalAppExitA@8     006356a4     kernel32:KERNEL32.dll
 0004:000006a8       __imp__GetConsoleCP@0      006356a8     kernel32:KERNEL32.dll
 0004:000006ac       __imp__FreeLibrary@4       006356ac     kernel32:KERNEL32.dll
 0004:000006b0       __imp__InterlockedExchange@8 006356b0     kernel32:KERNEL32.dll
 0004:000006b4       __imp__LoadLibraryA@4      006356b4     kernel32:KERNEL32.dll
 0004:000006b8       __imp__GetCPInfo@8         006356b8     kernel32:KERNEL32.dll
 0004:000006bc       __imp__GetACP@0            006356bc     kernel32:KERNEL32.dll
 0004:000006c0       __imp__GetOEMCP@0          006356c0     kernel32:KERNEL32.dll
 0004:000006c4       __imp__IsValidCodePage@4   006356c4     kernel32:KERNEL32.dll
 0004:000006c8       __imp__FreeEnvironmentStringsA@4 006356c8     kernel32:KERNEL32.dll
 0004:000006cc       __imp__GetEnvironmentStrings@0 006356cc     kernel32:KERNEL32.dll
 0004:000006d0       __imp__FreeEnvironmentStringsW@4 006356d0     kernel32:KERNEL32.dll
 0004:000006d4       __imp__GetEnvironmentStringsW@0 006356d4     kernel32:KERNEL32.dll
 0004:000006d8       __imp__HeapDestroy@4       006356d8     kernel32:KERNEL32.dll
 0004:000006dc       __imp__HeapCreate@12       006356dc     kernel32:KERNEL32.dll
 0004:000006e0       __imp__VirtualFree@12      006356e0     kernel32:KERNEL32.dll
 0004:000006e4       __imp__GetCurrentProcessId@0 006356e4     kernel32:KERNEL32.dll
 0004:000006e8       __imp__VirtualAlloc@16     006356e8     kernel32:KERNEL32.dll
 0004:000006ec       __imp__HeapSize@12         006356ec     kernel32:KERNEL32.dll
 0004:000006f0       __imp__RtlUnwind@16        006356f0     kernel32:KERNEL32.dll
 0004:000006f4       __imp__InitializeCriticalSection@4 006356f4     kernel32:KERNEL32.dll
 0004:000006f8       \177KERNEL32_NULL_THUNK_DATA 006356f8     kernel32:KERNEL32.dll
 0004:00000790       __imp__PeekMessageA@20     00635790     user32:USER32.dll
 0004:00000794       __imp__KillTimer@8         00635794     user32:USER32.dll
 0004:00000798       __imp__SetTimer@16         00635798     user32:USER32.dll
 0004:0000079c       \177USER32_NULL_THUNK_DATA 0063579c     user32:USER32.dll
 0004:000007c8       __imp__recv@16             006357c8     wsock32:WSOCK32.dll
 0004:000007cc       __imp__gethostbyname@4     006357cc     wsock32:WSOCK32.dll
 0004:000007d0       __imp__WSAStartup@8        006357d0     wsock32:WSOCK32.dll
 0004:000007d4       __imp__WSACleanup@0        006357d4     wsock32:WSOCK32.dll
 0004:000007d8       __imp__WSAGetLastError@0   006357d8     wsock32:WSOCK32.dll
 0004:000007dc       __imp__send@16             006357dc     wsock32:WSOCK32.dll
 0004:000007e0       __imp__select@20           006357e0     wsock32:WSOCK32.dll
 0004:000007e4       __imp____WSAFDIsSet@8      006357e4     wsock32:WSOCK32.dll
 0004:000007e8       __imp__accept@12           006357e8     wsock32:WSOCK32.dll
 0004:000007ec       __imp__shutdown@8          006357ec     wsock32:WSOCK32.dll
 0004:000007f0       __imp__socket@12           006357f0     wsock32:WSOCK32.dll
 0004:000007f4       __imp__inet_addr@4         006357f4     wsock32:WSOCK32.dll
 0004:000007f8       __imp__ntohs@4             006357f8     wsock32:WSOCK32.dll
 0004:000007fc       __imp__getpeername@12      006357fc     wsock32:WSOCK32.dll
 0004:00000800       __imp__WSASetLastError@4   00635800     wsock32:WSOCK32.dll
 0004:00000804       __imp__connect@12          00635804     wsock32:WSOCK32.dll
 0004:00000808       __imp__htonl@4             00635808     wsock32:WSOCK32.dll
 0004:0000080c       __imp__htons@4             0063580c     wsock32:WSOCK32.dll
 0004:00000810       __imp__setsockopt@20       00635810     wsock32:WSOCK32.dll
 0004:00000814       __imp__inet_ntoa@4         00635814     wsock32:WSOCK32.dll
 0004:00000818       __imp__bind@12             00635818     wsock32:WSOCK32.dll
 0004:0000081c       __imp__listen@8            0063581c     wsock32:WSOCK32.dll
 0004:00000820       __imp__closesocket@4       00635820     wsock32:WSOCK32.dll
 0004:00000824       __imp__ioctlsocket@12      00635824     wsock32:WSOCK32.dll
 0004:00000828       __imp__gethostname@8       00635828     wsock32:WSOCK32.dll
 0004:0000082c       \177WSOCK32_NULL_THUNK_DATA 0063582c     wsock32:WSOCK32.dll
 0005:00000000       __tls_start                00637000     LIBCMT:tlssup.obj
 0005:00000108       _THR_KEY_mysys             00637108     mysys:my_thr_init.obj
 0005:0000028e       __tls_end                  0063728e     LIBCMT:tlssup.obj

 entry point at        0001:0004f2bf

